 GameServerManager_x64

 Timestamp is 6101915a (Thu Jul 29 02:18:18 2021)

 Preferred load address is 0000000140000000

 Start         Length     Name                   Class
 0001:00000000 000005a0H .text$di                CODE
 0001:000005a0 00046e30H .text$mn                CODE
 0001:000473d0 00000020H .text$mn$00             CODE
 0001:000473f0 000015a0H .text$x                 CODE
 0001:00048990 000007f0H .text$yd                CODE
 0002:00000000 00000ef0H .idata$5                DATA
 0002:00000ef0 00000010H .00cfg                  DATA
 0002:00000f00 00000008H .CRT$XCA                DATA
 0002:00000f08 00000008H .CRT$XCAA               DATA
 0002:00000f10 00000018H .CRT$XCL                DATA
 0002:00000f28 00000110H .CRT$XCU                DATA
 0002:00001038 00000008H .CRT$XCZ                DATA
 0002:00001040 00000008H .CRT$XIA                DATA
 0002:00001048 00000008H .CRT$XIAA               DATA
 0002:00001050 00000008H .CRT$XIAC               DATA
 0002:00001058 00000008H .CRT$XIC                DATA
 0002:00001060 00000008H .CRT$XIZ                DATA
 0002:00001068 00000008H .CRT$XLA                DATA
 0002:00001070 00000008H .CRT$XLZ                DATA
 0002:00001078 00000008H .CRT$XPA                DATA
 0002:00001080 00000008H .CRT$XPZ                DATA
 0002:00001088 00000008H .CRT$XTA                DATA
 0002:00001090 00000010H .CRT$XTZ                DATA
 0002:00001098 00000000H .gfids$y                DATA
 0002:000010a0 0000b7d0H .rdata                  DATA
 0002:0000c870 00000030H .rdata$T                DATA
 0002:0000c8a0 0000157cH .rdata$r                DATA
 0002:0000de1c 000003e4H .rdata$zzzdbg           DATA
 0002:0000e200 00000008H .rtc$IAA                DATA
 0002:0000e208 00000008H .rtc$IZZ                DATA
 0002:0000e210 00000008H .rtc$TAA                DATA
 0002:0000e218 00000008H .rtc$TZZ                DATA
 0002:0000e220 00000010H .tls                    DATA
 0002:0000e230 00000004H .tls$                   DATA
 0002:0000e234 0000000cH .tls$ZZZ                DATA
 0002:0000e240 00004ed0H .xdata                  DATA
 0002:00013110 00000058H .xdata$x                DATA
 0002:00013168 00000000H ATL$__a                 DATA
 0002:00013168 00000000H ATL$__z                 DATA
 0002:00013168 00000000H .edata                  DATA
 0002:00013168 000001e0H .idata$2                DATA
 0002:00013348 00000018H .idata$3                DATA
 0002:00013360 00000ef0H .idata$4                DATA
 0002:00014250 0000188eH .idata$6                DATA
 0003:00000000 000016d0H .data                   DATA
 0003:000016d0 00000880H .data$r                 DATA
 0003:00001f50 0000f4d0H .bss                    DATA
 0004:00000000 00002268H .pdata                  DATA
 0005:00000000 000001e0H .rsrc$01                DATA
 0005:000001e0 00000c80H .rsrc$02                DATA

  Address         Publics by Value              Rva+Base               Lib:Object

 0000:00000000       __guard_iat_count          0000000000000000     <absolute>
 0000:00000000       __hybrid_code_map_count    0000000000000000     <absolute>
 0000:00000000       __guard_fids_count         0000000000000000     <absolute>
 0000:00000000       __volatile_metadata        0000000000000000     <absolute>
 0000:00000000       __guard_longjmp_count      0000000000000000     <absolute>
 0000:00000000       __guard_longjmp_table      0000000000000000     <absolute>
 0000:00000000       __hybrid_code_map          0000000000000000     <absolute>
 0000:00000000       __guard_iat_table          0000000000000000     <absolute>
 0000:00000000       ___safe_se_handler_count   0000000000000000     <absolute>
 0000:00000000       __enclave_config           0000000000000000     <absolute>
 0000:00000000       ___safe_se_handler_table   0000000000000000     <absolute>
 0000:00000000       __guard_fids_table         0000000000000000     <absolute>
 0000:00000000       __hybrid_auxiliary_iat     0000000000000000     <absolute>
 0000:00000000       __dynamic_value_reloc_table 0000000000000000     <absolute>
 0000:00000100       __guard_flags              0000000000000100     <absolute>
 0000:00000000       __ImageBase                0000000140000000     <linker-defined>
 0001:000005a0       ??1DivisionPacket@@QEAA@XZ 00000001400015a0 f   DivisionPacket.obj
 0001:000005b0       ?AppendPacket@DivisionPacket@@AEAA?BW4DIVISION_PACKET_RESULT@@PEADG@Z 00000001400015b0 f   DivisionPacket.obj
 0001:000006a0       _guard_check_icall_nop     00000001400016a0 f i msvcrt:guard_support.obj
 0001:000006a0       ?OnReceivePacket@CClientLib@@MEAAXPEAVCPacket@@@Z 00000001400016a0 f i ClientLib.obj
 0001:000006a0       ?__empty_global_delete@@YAXPEAX_K@Z 00000001400016a0 f i DivisionPacket.obj
 0001:000006a0       _initialize_invalid_parameter_handler 00000001400016a0 f i msvcrt:invalid_parameter_handler.obj
 0001:000006a0       ?__global_delete@@YAXPEAX_K@Z 00000001400016a0 f i * CIL library *:* CIL module *
 0001:000006a0       ?onError@CReceiver@@UEAAXW4ErrorCode@sggm@@@Z 00000001400016a0 f i SGGMCallBackObj.obj
 0001:000006a0       ?OnBnClickedOk@CGameServerManagerDlg@@QEAAXXZ 00000001400016a0 f i GameServerManagerDlg.obj
 0001:000006a0       ?AssertValid@CObject@@UEBAXXZ 00000001400016a0 f i AppInfoDlg.obj
 0001:000006a0       ?Dump@CObject@@UEBAXAEAVCDumpContext@@@Z 00000001400016a0 f i AppInfoDlg.obj
 0001:000006a0       _initialize_denormal_control 00000001400016a0 f i msvcrt:denormal_control.obj
 0001:000006a0       ?Serialize@CObject@@UEAAXAEAVCArchive@@@Z 00000001400016a0 f i AppInfoDlg.obj
 0001:000006a0       ?DoDataExchange@CWnd@@MEAAXPEAVCDataExchange@@@Z 00000001400016a0 f i AppInfoDlg.obj
 0001:000006b0       ?_Tidy@?$vector@UPART_PACKET@@V?$allocator@UPART_PACKET@@@std@@@std@@AEAAXXZ 00000001400016b0 f i DivisionPacket.obj
 0001:00000730       ??$_Emplace_reallocate@AEBUPART_PACKET@@@?$vector@UPART_PACKET@@V?$allocator@UPART_PACKET@@@std@@@std@@QEAAPEAUPART_PACKET@@QEAU2@AEBU2@@Z 0000000140001730 f i DivisionPacket.obj
 0001:00000950       ?_Xlength@?$vector@DV?$allocator@D@std@@@std@@CAXXZ 0000000140001950 f i mailer.obj
 0001:00000950       ?_Xlength@?$vector@UPART_PACKET@@V?$allocator@UPART_PACKET@@@std@@@std@@CAXXZ 0000000140001950 f i DivisionPacket.obj
 0001:00000950       ?_Xlength@?$vector@USOCKADDR_IN@jwsmtp@@V?$allocator@USOCKADDR_IN@jwsmtp@@@std@@@std@@CAXXZ 0000000140001950 f i mailer.obj
 0001:00000950       ?_Xlength@?$vector@PEAXV?$allocator@PEAX@std@@@std@@CAXXZ 0000000140001950 f i LogMsgManager.obj
 0001:00000950       ?_Xlength@?$vector@U?$pair@UAddress@mailer@jwsmtp@@F@std@@V?$allocator@U?$pair@UAddress@mailer@jwsmtp@@F@std@@@2@@std@@CAXXZ 0000000140001950 f i mailer.obj
 0001:00000950       ?_Xlength@?$vector@V?$basic_string@DU?$char_traits@D@std@@V?$allocator@D@2@@std@@V?$allocator@V?$basic_string@DU?$char_traits@D@std@@V?$allocator@D@2@@std@@@2@@std@@CAXXZ 0000000140001950 f i CSmtp.obj
 0001:00000a20       ?Instance@DivisionPacketReceiver@@SAPEAV1@XZ 0000000140001a20 f   DivisionPacketReceiver.obj
 0001:00000ac0       ?GetPacketBuffer@DivisionPacketReceiver@@QEAA?BW4DIVISION_PACKET_RESULT@@EEEEEPEADG0H@Z 0000000140001ac0 f   DivisionPacketReceiver.obj
 0001:00000cf0       ??1?$pair@_JVDivisionPacket@@@std@@QEAA@XZ 0000000140001cf0 f i DivisionPacketReceiver.obj
 0001:00000d00       ?_Buyheadnode@?$_Tree_comp_alloc@V?$_Tmap_traits@_JVDivisionPacket@@U?$less@_J@std@@V?$allocator@U?$pair@$$CB_JVDivisionPacket@@@std@@@3@$0A@@std@@@std@@QEAAPEAU?$_Tree_node@U?$pair@$$CB_JVDivisionPacket@@@std@@PEAX@2@XZ 0000000140001d00 f i DivisionPacketReceiver.obj
 0001:00000d30       ?_Erase@?$_Tree@V?$_Tmap_traits@_JVDivisionPacket@@U?$less@_J@std@@V?$allocator@U?$pair@$$CB_JVDivisionPacket@@@std@@@3@$0A@@std@@@std@@IEAAXPEAU?$_Tree_node@U?$pair@$$CB_JVDivisionPacket@@@std@@PEAX@2@@Z 0000000140001d30 f i DivisionPacketReceiver.obj
 0001:00000d90       ??0?$vector@UPART_PACKET@@V?$allocator@UPART_PACKET@@@std@@@std@@QEAA@AEBV01@@Z 0000000140001d90 f i DivisionPacketReceiver.obj
 0001:00000ea0       ??$_Buynode@U?$pair@_JVDivisionPacket@@@std@@@?$_Tree_comp_alloc@V?$_Tmap_traits@_JVDivisionPacket@@U?$less@_J@std@@V?$allocator@U?$pair@$$CB_JVDivisionPacket@@@std@@@3@$0A@@std@@@std@@QEAAPEAU?$_Tree_node@U?$pair@$$CB_JVDivisionPacket@@@std@@PEAX@1@$$QEAU?$pair@_JVDivisionPacket@@@1@@Z 0000000140001ea0 f i DivisionPacketReceiver.obj
 0001:00000f00       ??$_Insert_nohint@AEAU?$pair@$$CB_JVDivisionPacket@@@std@@PEAU?$_Tree_node@U?$pair@$$CB_JVDivisionPacket@@@std@@PEAX@2@@?$_Tree@V?$_Tmap_traits@_JVDivisionPacket@@U?$less@_J@std@@V?$allocator@U?$pair@$$CB_JVDivisionPacket@@@std@@@3@$0A@@std@@@std@@IEAA?AU?$pair@V?$_Tree_iterator@V?$_Tree_val@U?$_Tree_simple_types@U?$pair@$$CB_JVDivisionPacket@@@std@@@std@@@std@@@std@@_N@1@_NAEAU?$pair@$$CB_JVDivisionPacket@@@1@PEAU?$_Tree_node@U?$pair@$$CB_JVDivisionPacket@@@std@@PEAX@1@@Z 0000000140001f00 f i DivisionPacketReceiver.obj
 0001:00001070       ?_Freenode0@?$_Tree_comp_alloc@V?$_Tmap_traits@_JVDivisionPacket@@U?$less@_J@std@@V?$allocator@U?$pair@$$CB_JVDivisionPacket@@@std@@@3@$0A@@std@@@std@@QEAAXPEAU?$_Tree_node@U?$pair@$$CB_JVDivisionPacket@@@std@@PEAX@2@@Z 0000000140002070 f i DivisionPacketReceiver.obj
 0001:00001080       ?_Buynode0@?$_Tree_comp_alloc@V?$_Tmap_traits@_JVDivisionPacket@@U?$less@_J@std@@V?$allocator@U?$pair@$$CB_JVDivisionPacket@@@std@@@3@$0A@@std@@@std@@QEAAPEAU?$_Tree_node@U?$pair@$$CB_JVDivisionPacket@@@std@@PEAX@2@XZ 0000000140002080 f i DivisionPacketReceiver.obj
 0001:000010b0       ?_Destroy_if_node@?$_Tree@V?$_Tmap_traits@_JVDivisionPacket@@U?$less@_J@std@@V?$allocator@U?$pair@$$CB_JVDivisionPacket@@@std@@@3@$0A@@std@@@std@@IEAAXPEAU?$_Tree_node@U?$pair@$$CB_JVDivisionPacket@@@std@@PEAX@2@@Z 00000001400020b0 f i DivisionPacketReceiver.obj
 0001:000010e0       ??$_Insert_at@AEAU?$pair@$$CB_JVDivisionPacket@@@std@@PEAU?$_Tree_node@U?$pair@$$CB_JVDivisionPacket@@@std@@PEAX@2@@?$_Tree@V?$_Tmap_traits@_JVDivisionPacket@@U?$less@_J@std@@V?$allocator@U?$pair@$$CB_JVDivisionPacket@@@std@@@3@$0A@@std@@@std@@IEAA?AV?$_Tree_iterator@V?$_Tree_val@U?$_Tree_simple_types@U?$pair@$$CB_JVDivisionPacket@@@std@@@std@@@std@@@1@_NPEAU?$_Tree_node@U?$pair@$$CB_JVDivisionPacket@@@std@@PEAX@1@AEAU?$pair@$$CB_JVDivisionPacket@@@1@1@Z 00000001400020e0 f i DivisionPacketReceiver.obj
 0001:00001500       ?threadCreateDumpFile@@YAKPEAX@Z 0000000140002500 f   BugReporter.obj
 0001:000018e0       ?CrashExceptionDump@@YAJPEAU_EXCEPTION_POINTERS@@@Z 00000001400028e0 f   BugReporter.obj
 0001:00001950       ?InvalidParameterHandler@@YAXPEB_W00I_K@Z 0000000140002950 f   BugReporter.obj
 0001:00001970       ?InitBugReporter@@YAXPEAD0000@Z 0000000140002970 f   BugReporter.obj
 0001:00001cc0       ??$sprintf_s@$0BAA@@cf@@YAHAEAY0BAA@DPEBDZZ 0000000140002cc0 f i BugReporter.obj
 0001:00001d00       ??$sprintf_s@$0BJB@@cf@@YAHAEAY0BJB@DPEBDZZ 0000000140002d00 f i BugReporter.obj
 0001:00001d40       ??$sprintf_s@$0BE@@cf@@YAHAEAY0BE@DPEBDZZ 0000000140002d40 f i BugReporter.obj
 0001:00001d80       ??$sprintf_s@$0DOJ@@cf@@YAHAEAY0DOJ@DPEBDZZ 0000000140002d80 f i BugReporter.obj
 0001:00001dc0       ??$sprintf_s@$0BAE@@cf@@YAHAEAY0BAE@DPEBDZZ 0000000140002dc0 f i BugReporter.obj
 0001:00001e00       ??1?$basic_string@DU?$char_traits@D@std@@V?$allocator@D@2@@std@@QEAA@XZ 0000000140002e00 f i BugReporter.obj
 0001:00001e00       ?_Tidy_deallocate@?$basic_string@DU?$char_traits@D@std@@V?$allocator@D@2@@std@@QEAAXXZ 0000000140002e00 f i BugReporter.obj
 0001:00001e60       ?_Xlen@?$basic_string@DU?$char_traits@D@std@@V?$allocator@D@2@@std@@SAXXZ 0000000140002e60 f i BugReporter.obj
 0001:00001e60       ?_Xlen@?$basic_string@_WU?$char_traits@_W@std@@V?$allocator@_W@2@@std@@SAXXZ 0000000140002e60 f i crs_uploader.obj
 0001:00001e80       ?assign@?$basic_string@DU?$char_traits@D@std@@V?$allocator@D@2@@std@@QEAAAEAV12@QEBD_K@Z 0000000140002e80 f i BugReporter.obj
 0001:00001fe0       ?assign@?$basic_string@DU?$char_traits@D@std@@V?$allocator@D@2@@std@@QEAAAEAV12@QEBD@Z 0000000140002fe0 f i BugReporter.obj
 0001:00002000       ??0?$basic_string@DU?$char_traits@D@std@@V?$allocator@D@2@@std@@QEAA@QEBD@Z 0000000140003000 f i BugReporter.obj
 0001:00002040       _snprintf_s                0000000140003040 f i BugReporter.obj
 0001:000020b0       __local_stdio_printf_options 00000001400030b0 f i BugReporter.obj
 0001:000020c0       ?recordExceptionLog@Uploader@crs@@QEAAXAEAVLogBuffer@2@PEBDZZ 00000001400030c0 f i crs_uploader.obj
 0001:000021d0       ?readURL@Uploader@crs@@AEAAXAEAV?$basic_string@_WU?$char_traits@_W@std@@V?$allocator@_W@2@@std@@@Z 00000001400031d0 f i crs_uploader.obj
 0001:000023e0       ?iniPath@Uploader@crs@@AEAA?AV?$basic_string@_WU?$char_traits@_W@std@@V?$allocator@_W@2@@std@@AEBV34@@Z 00000001400033e0 f i crs_uploader.obj
 0001:00002600       ?makeBaseInfo@Uploader@crs@@AEAAXPEAD0@Z 0000000140003600 f i crs_uploader.obj
 0001:00002850       ?error@Uploader@crs@@AEAA_NPEBDZZ 0000000140003850 f i crs_uploader.obj
 0001:000028b0       ??1Uploader@crs@@QEAA@XZ   00000001400038b0 f   crs_uploader.obj
 0001:00002aa0       ?init@Uploader@crs@@QEAA_N_NPEAD1@Z 0000000140003aa0 f   crs_uploader.obj
 0001:00002ef0       ?upload@Uploader@crs@@QEAA_N_NAEBV?$basic_string@DU?$char_traits@D@std@@V?$allocator@D@2@@std@@AEAVLogBuffer@2@@Z 0000000140003ef0 f   crs_uploader.obj
 0001:00003180       ?makeExceptionLog@Uploader@crs@@QEAAXPEAU_EXCEPTION_POINTERS@@AEAVLogBuffer@2@@Z 0000000140004180 f   crs_uploader.obj
 0001:00003540       ?prepare@Uploader@crs@@AEAA_NAEAVHttpHandles@2@@Z 0000000140004540 f   crs_uploader.obj
 0001:00003640       ?uploadHTTP@Uploader@crs@@AEAA_NAEAVHttpHandle@2@PEBDPEB_W2@Z 0000000140004640 f   crs_uploader.obj
 0001:000039a0       ?uploadLOG@Uploader@crs@@AEAA_NAEAVHttpHandle@2@AEAU_SYSTEMTIME@@AEAVLogBuffer@2@@Z 00000001400049a0 f   crs_uploader.obj
 0001:00003c90       ?success@Uploader@crs@@AEAA_NPEBDAEAVHttpHandle@2@@Z 0000000140004c90 f   crs_uploader.obj
 0001:00003dd0       ??1?$auto_ptr@VUrl@crs@@@std@@QEAA@XZ 0000000140004dd0 f i crs_uploader.obj
 0001:00003ef0       ??$_snprintf_s@$0IA@@@YAHAEAY0IA@D_KPEBDZZ 0000000140004ef0 f i crs_uploader.obj
 0001:00003f60       ??$_Reallocate_grow_by@V<lambda_1dfe18491bcca09701d8ccb01d0b0af4>@@PEB_W_K@?$basic_string@_WU?$char_traits@_W@std@@V?$allocator@_W@2@@std@@QEAAAEAV01@_KV<lambda_1dfe18491bcca09701d8ccb01d0b0af4>@@PEB_W_K@Z 0000000140004f60 f i crs_uploader.obj
 0001:00004110       ?append@?$basic_string@_WU?$char_traits@_W@std@@V?$allocator@_W@2@@std@@QEAAAEAV12@QEB_W_K@Z 0000000140005110 f i crs_uploader.obj
 0001:00004190       ??0?$basic_string@DU?$char_traits@D@std@@V?$allocator@D@2@@std@@QEAA@XZ 0000000140005190 f i crs_uploader.obj
 0001:000041b0       _snwprintf_s               00000001400051b0 f i crs_uploader.obj
 0001:00004220       ?_Tidy_deallocate@?$basic_string@_WU?$char_traits@_W@std@@V?$allocator@_W@2@@std@@QEAAXXZ 0000000140005220 f i crs_uploader.obj
 0001:00004220       ??1?$basic_string@_WU?$char_traits@_W@std@@V?$allocator@_W@2@@std@@QEAA@XZ 0000000140005220 f i crs_uploader.obj
 0001:00004290       ?assign@?$basic_string@_WU?$char_traits@_W@std@@V?$allocator@_W@2@@std@@QEAAAEAV12@QEB_W_K@Z 0000000140005290 f i crs_uploader.obj
 0001:00004420       ??_ECServerLog@@UEAAPEAXI@Z 0000000140005420 f i * CIL library *:* CIL module *
 0001:00004420       ??_GCServerLog@@UEAAPEAXI@Z 0000000140005420 f i LogMgmt.obj
 0001:00004460       ??1CServerLog@@UEAA@XZ     0000000140005460 f   LogMgmt.obj
 0001:00004590       ?LOG_MAILER@CServerLog@@QEAAXHPEBD@Z 0000000140005590 f   LogMgmt.obj
 0001:00004680       fprintf                    0000000140005680 f i LogMgmt.obj
 0001:000046d0       sprintf                    00000001400056d0 f i LogMgmt.obj
 0001:00004730       ?Log@rwpmlog@@YAXPEBDFPEBUGAMEPROTO_SC_REMOVECLIENT@@@Z 0000000140005730 f   RWPMLog.obj
 0001:00004ad0       ?Log@rwpmlog@@YAXPEBDFPEBUGAMEPROTO_SS_GAMEEND@@@Z 0000000140005ad0 f   RWPMLog.obj
 0001:00005650       ?Log@rwpmlog@@YAXPEBDFPEBUGAMEPROTO_SC_HOST_USER_STAT@@@Z 0000000140006650 f   RWPMLog.obj
 0001:00006230       ?Log@rwpmlog@@YAXPEBDFPEBUCLANSTATREPORTDATA@@@Z 0000000140007230 f   RWPMLog.obj
 0001:000065c0       ?Log@rwpmlog@@YAXPEBDFPEBUGAMEPROTO_SC_HOST_STAT@@@Z 00000001400075c0 f   RWPMLog.obj
 0001:000068e0       ?Log@rwpmlog@@YAXPEBDFPEBUPROTO_GAMEGT_INGAME_AIGACHA_ITEM_INSERT@@@Z 00000001400078e0 f   RWPMLog.obj
 0001:00006bc0       ?Log@rwpmlog@@YAXPEBDFPEBUPROTO_SPEC_RECOMMENDROOM_INGAME_DATA@@@Z 0000000140007bc0 f   RWPMLog.obj
 0001:000070d0       ?Log@rwpmlog@@YAXPEBDFPEBUPROTO_GAMEGT_AUTO_SIDE_CHANGE_TEAM_INFO_NTY@@@Z 00000001400080d0 f   RWPMLog.obj
 0001:000077b0       ??$sprintf_s@$0EA@@cf@@YAHAEAY0EA@DPEBDZZ 00000001400087b0 f i RWPMLog.obj
 0001:000077f0       ?onHeartBeat@CReceiver@@UEAA_NXZ 00000001400087f0 f i SGGMCallBackObj.obj
 0001:000077f0       __acrt_uninitialize        00000001400087f0 f i msvcrt:ucrt_stubs.obj
 0001:000077f0       __scrt_stub_for_acrt_uninitialize 00000001400087f0 f i msvcrt:ucrt_stubs.obj
 0001:000077f0       ?PreWriteData@GAMEPROTO_SC_COMMON@@UEAA_NPEAVILTMessage_Write@@@Z 00000001400087f0 f i AppInfoDlg.obj
 0001:000077f0       ?onAnnouncement@CReceiver@@UEAA_NPEBD@Z 00000001400087f0 f i SGGMCallBackObj.obj
 0001:000077f0       __vcrt_uninitialize        00000001400087f0 f i msvcrt:ucrt_stubs.obj
 0001:000077f0       __acrt_initialize          00000001400087f0 f i msvcrt:ucrt_stubs.obj
 0001:000077f0       ?PreReadData@GAMEPROTO_SC_COMMON@@UEAA_NPEAVILTMessage_Read@@@Z 00000001400087f0 f i AppInfoDlg.obj
 0001:000077f0       _should_initialize_environment 00000001400087f0 f i msvcrt:env_mode.obj
 0001:000077f0       __scrt_stub_for_acrt_initialize 00000001400087f0 f i msvcrt:ucrt_stubs.obj
 0001:000077f0       __vcrt_initialize          00000001400087f0 f i msvcrt:ucrt_stubs.obj
 0001:00007800       ?onGameData@CReceiver@@UEAA_NAEAVGameData@sggm@@@Z 0000000140008800 f i SGGMCallBackObj.obj
 0001:00007850       ??_ECReceiver@@UEAAPEAXI@Z 0000000140008850 f i * CIL library *:* CIL module *
 0001:00007850       ??_GCReceiver@@UEAAPEAXI@Z 0000000140008850 f i SGGMCallBackObj.obj
 0001:00007880       ??_GCSGGMCallBackObj@@UEAAPEAXI@Z 0000000140008880 f i SGGMCallBackObj.obj
 0001:00007880       ??_ECSGGMCallBackObj@@UEAAPEAXI@Z 0000000140008880 f i * CIL library *:* CIL module *
 0001:000078d0       ??1MultiReceiver@sggm_proxy@@UEAA@XZ 00000001400088d0 f i SGGMCallBackObj.obj
 0001:000078f0       ??_GMultiReceiver@sggm_proxy@@UEAAPEAXI@Z 00000001400088f0 f i SGGMCallBackObj.obj
 0001:000078f0       ??_EMultiReceiver@sggm_proxy@@UEAAPEAXI@Z 00000001400088f0 f i * CIL library *:* CIL module *
 0001:00007940       ?GetSendParam@SendBuffer@@QEAAHPEAPEAEAEAH@Z 0000000140008940 f i ClientLib.obj
 0001:00007a60       ?Write@SendBuffer@@QEAAHPEAEG@Z 0000000140008a60 f i ClientLib.obj
 0001:00007b40       ??_ESendBuffer@@UEAAPEAXI@Z 0000000140008b40 f i * CIL library *:* CIL module *
 0001:00007b40       ??_GSendBuffer@@UEAAPEAXI@Z 0000000140008b40 f i ClientLib.obj
 0001:00007b90       ??_ECClientLib@@UEAAPEAXI@Z 0000000140008b90 f i * CIL library *:* CIL module *
 0001:00007b90       ??_GCClientLib@@UEAAPEAXI@Z 0000000140008b90 f i ClientLib.obj
 0001:00007c10       ?CloseSocket@CClientLib@@MEAAHXZ 0000000140008c10 f   ClientLib.obj
 0001:00007c90       ?RecvBufferHasCompletePacket@CClientLib@@IEAAHXZ 0000000140008c90 f   ClientLib.obj
 0001:00007cc0       ?ProcessSend@CClientLib@@QEAAHXZ 0000000140008cc0 f   ClientLib.obj
 0001:00007ed0       ?CopySendBuffer@CClientLib@@QEAAHPEAVSendBuffer@@@Z 0000000140008ed0 f   ClientLib.obj
 0001:00007fa0       ?ProcessSocketEvent@CClientLib@@QEAAXXZ 0000000140008fa0 f   ClientLib.obj
 0001:000081b0       ??_E?$CircuitQueue@E@@UEAAPEAXI@Z 00000001400091b0 f i * CIL library *:* CIL module *
 0001:000081b0       ??_G?$CircuitQueue@E@@UEAAPEAXI@Z 00000001400091b0 f i ClientLib.obj
 0001:00008210       ??_GCPacket@@UEAAPEAXI@Z   0000000140009210 f i Packet.obj
 0001:00008210       ??_ECPacket@@UEAAPEAXI@Z   0000000140009210 f i * CIL library *:* CIL module *
 0001:00008240       ??1CPacket@@UEAA@XZ        0000000140009240 f   Packet.obj
 0001:00008250       ?CopyFromUserDataArea@CPacket@@QEAAHPEAXK@Z 0000000140009250 f   Packet.obj
 0001:00008370       ??0CSFGameServerClientLib@@QEAA@XZ 0000000140009370 f   SFGameServerClientLib.obj
 0001:00008530       ??1CSFGameServerClientLib@@UEAA@XZ 0000000140009530 f   SFGameServerClientLib.obj
 0001:000085a0       ?Connect@CSFGameServerClientLib@@QEAAHH@Z 00000001400095a0 f   SFGameServerClientLib.obj
 0001:00008950       ?CloseSocket@CSFGameServerClientLib@@UEAAHXZ 0000000140009950 f   SFGameServerClientLib.obj
 0001:000089f0       ?OnReceivePacket@CSFGameServerClientLib@@MEAAXPEAVCPacket@@@Z 00000001400099f0 f   SFGameServerClientLib.obj
 0001:00008a10       ?Create@CDialog@@UEAAHIPEAVCWnd@@@Z 0000000140009a10 f i AppInfoDlg.obj
 0001:00008a20       ?ReadData@GAMEPROTO_SC_HOST_STAT@@UEAA_NPEAVILTMessage_Read@@@Z 0000000140009a20 f i AppInfoDlg.obj
 0001:00008cc0       ?WriteData@GAMEPROTO_SC_HOST_STAT@@UEAA_NPEAVILTMessage_Write@@@Z 0000000140009cc0 f i AppInfoDlg.obj
 0001:00008e30       ?ReadData@GAMEPROTO_SC_HOST_USER_STAT@@UEAA_NPEAVILTMessage_Read@@@Z 0000000140009e30 f i AppInfoDlg.obj
 0001:00009b00       ?WriteData@GAMEPROTO_SC_HOST_USER_STAT@@UEAA_NPEAVILTMessage_Write@@@Z 000000014000ab00 f i AppInfoDlg.obj
 0001:0000a3e0       ?ReadData@GAMEPROTO_SC_REMOVECLIENT@@UEAA_NPEAVILTMessage_Read@@@Z 000000014000b3e0 f i AppInfoDlg.obj
 0001:0000a4d0       ?WriteData@GAMEPROTO_SC_REMOVECLIENT@@UEAA_NPEAVILTMessage_Write@@@Z 000000014000b4d0 f i AppInfoDlg.obj
 0001:0000a5e0       ?PreReadData@GAMEPROTO_CS_COMMON@@UEAA_NPEAVILTMessage_Read@@@Z 000000014000b5e0 f i AppInfoDlg.obj
 0001:0000a630       ?PostReadData@GAMEPROTO_SC_COMMON@@UEAA_NPEAVILTMessage_Read@@@Z 000000014000b630 f i AppInfoDlg.obj
 0001:0000a630       ?PostReadData@GAMEPROTO_CS_COMMON@@UEAA_NPEAVILTMessage_Read@@@Z 000000014000b630 f i AppInfoDlg.obj
 0001:0000a640       ?PreWriteData@GAMEPROTO_CS_COMMON@@UEAA_NPEAVILTMessage_Write@@@Z 000000014000b640 f i AppInfoDlg.obj
 0001:0000a6a0       ?PostWriteData@GAMEPROTO_CS_COMMON@@UEAA_NPEAVILTMessage_Write@@@Z 000000014000b6a0 f i AppInfoDlg.obj
 0001:0000a6a0       ?PostWriteData@GAMEPROTO_SC_COMMON@@UEAA_NPEAVILTMessage_Write@@@Z 000000014000b6a0 f i AppInfoDlg.obj
 0001:0000a700       ??0exception@std@@QEAA@QEBD@Z 000000014000b700 f i AppInfoDlg.obj
 0001:0000a750       ??1exception@std@@UEAA@XZ  000000014000b750 f i AppInfoDlg.obj
 0001:0000a770       ??_Gexception@std@@UEAAPEAXI@Z 000000014000b770 f i AppInfoDlg.obj
 0001:0000a770       ??_Eexception@std@@UEAAPEAXI@Z 000000014000b770 f i * CIL library *:* CIL module *
 0001:0000a7c0       ?what@exception@std@@UEBAPEBDXZ 000000014000b7c0 f i AppInfoDlg.obj
 0001:0000a7e0       ??0exception@std@@QEAA@AEBV01@@Z 000000014000b7e0 f i AppInfoDlg.obj
 0001:0000a820       ?ReadData@GAMEPROTO_SS_GAMEEND@@UEAA_NPEAVILTMessage_Read@@@Z 000000014000b820 f i AppInfoDlg.obj
 0001:0000c470       ?WriteData@GAMEPROTO_SS_GAMEEND@@UEAA_NPEAVILTMessage_Write@@@Z 000000014000d470 f i AppInfoDlg.obj
 0001:0000d950       ?PostReadData@GAMEPROTO_COMMON@@UEAA_NPEAVILTMessage_Read@@@Z 000000014000e950 f i AppInfoDlg.obj
 0001:0000d9e0       ??_ECEdit@@UEAAPEAXI@Z     000000014000e9e0 f i * CIL library *:* CIL module *
 0001:0000d9e0       ??_GCEdit@@UEAAPEAXI@Z     000000014000e9e0 f i AppInfoDlg.obj
 0001:0000da30       ?BeginModalState@CWnd@@UEAAXXZ 000000014000ea30 f i AppInfoDlg.obj
 0001:0000da40       ?EndModalState@CWnd@@UEAAXXZ 000000014000ea40 f i AppInfoDlg.obj
 0001:0000da50       ?IsProcessInTrouble@CHECK_MEM_USAGE@@YA_NPEAXHH@Z 000000014000ea50 f   CheckMemUsage.obj
 0001:0000db00       ?EmptyWorkingset@CHECK_MEM_USAGE@@YA_NPEAXH@Z 000000014000eb00 f   CheckMemUsage.obj
 0001:0000dd00       ?GetProcessMemoryUsage@@YAKPEAXH@Z 000000014000ed00 f   CheckMemUsage.obj
 0001:0000df20       ??1?$map@GUExtraStatsFPSVerify@CHostStat@@U?$less@G@std@@V?$allocator@U?$pair@$$CBGUExtraStatsFPSVerify@CHostStat@@@std@@@4@@std@@QEAA@XZ 000000014000ef20 f i HostStat.obj
 0001:0000df20       ??1?$map@GPEAUtagIP4Address@@U?$less@G@std@@V?$allocator@U?$pair@$$CBGPEAUtagIP4Address@@@std@@@3@@std@@QEAA@XZ 000000014000ef20 f i cSnmpEX.obj
 0001:0000df40       ??1cSnmpEX@@QEAA@XZ        000000014000ef40 f   cSnmpEX.obj
 0001:0000dfa0       ?ReleaseUDPPortAddressMap@cSnmpEX@@QEAAXXZ 000000014000efa0 f   cSnmpEX.obj
 0001:0000e040       ?ReleaseTCPPortAddressMap@cSnmpEX@@QEAAXXZ 000000014000f040 f   cSnmpEX.obj
 0001:0000e0e0       ?clear@?$_Tree@V?$_Tmap_traits@GUExtraStatsMemVerify@CHostStat@@U?$less@G@std@@V?$allocator@U?$pair@$$CBGUExtraStatsMemVerify@CHostStat@@@std@@@4@$0A@@std@@@std@@QEAAXXZ 000000014000f0e0 f i HostStat.obj
 0001:0000e0e0       ?clear@?$_Tree@V?$_Tmap_traits@GPEAUtagIP4Address@@U?$less@G@std@@V?$allocator@U?$pair@$$CBGPEAUtagIP4Address@@@std@@@3@$0A@@std@@@std@@QEAAXXZ 000000014000f0e0 f i cSnmpEX.obj
 0001:0000e0e0       ?clear@?$_Tree@V?$_Tmap_traits@GUExtraStatsFPSVerify@CHostStat@@U?$less@G@std@@V?$allocator@U?$pair@$$CBGUExtraStatsFPSVerify@CHostStat@@@std@@@4@$0A@@std@@@std@@QEAAXXZ 000000014000f0e0 f i HostStat.obj
 0001:0000e170       ?_Erase@?$_Tree@V?$_Tmap_traits@GUExtraStatsFPSVerify@CHostStat@@U?$less@G@std@@V?$allocator@U?$pair@$$CBGUExtraStatsFPSVerify@CHostStat@@@std@@@4@$0A@@std@@@std@@IEAAXPEAU?$_Tree_node@U?$pair@$$CBGUExtraStatsFPSVerify@CHostStat@@@std@@PEAX@2@@Z 000000014000f170 f i HostStat.obj
 0001:0000e170       ?_Erase@?$_Tree@V?$_Tmap_traits@GUExtraStatsMemVerify@CHostStat@@U?$less@G@std@@V?$allocator@U?$pair@$$CBGUExtraStatsMemVerify@CHostStat@@@std@@@4@$0A@@std@@@std@@IEAAXPEAU?$_Tree_node@U?$pair@$$CBGUExtraStatsMemVerify@CHostStat@@@std@@PEAX@2@@Z 000000014000f170 f i HostStat.obj
 0001:0000e170       ?_Erase@?$_Tree@V?$_Tmap_traits@GPEAUtagIP4Address@@U?$less@G@std@@V?$allocator@U?$pair@$$CBGPEAUtagIP4Address@@@std@@@3@$0A@@std@@@std@@IEAAXPEAU?$_Tree_node@U?$pair@$$CBGPEAUtagIP4Address@@@std@@PEAX@2@@Z 000000014000f170 f i cSnmpEX.obj
 0001:0000e1d0       ?_Buyheadnode@?$_Tree_comp_alloc@V?$_Tmap_traits@GUExtraStatsMemVerify@CHostStat@@U?$less@G@std@@V?$allocator@U?$pair@$$CBGUExtraStatsMemVerify@CHostStat@@@std@@@4@$0A@@std@@@std@@QEAAPEAU?$_Tree_node@U?$pair@$$CBGUExtraStatsMemVerify@CHostStat@@@std@@PEAX@2@XZ 000000014000f1d0 f i HostStat.obj
 0001:0000e1d0       ?_Buyheadnode@?$_Tree_comp_alloc@V?$_Tmap_traits@GUExtraStatsFPSVerify@CHostStat@@U?$less@G@std@@V?$allocator@U?$pair@$$CBGUExtraStatsFPSVerify@CHostStat@@@std@@@4@$0A@@std@@@std@@QEAAPEAU?$_Tree_node@U?$pair@$$CBGUExtraStatsFPSVerify@CHostStat@@@std@@PEAX@2@XZ 000000014000f1d0 f i HostStat.obj
 0001:0000e1d0       ?_Buyheadnode@?$_Tree_comp_alloc@V?$_Tmap_traits@GPEAUtagIP4Address@@U?$less@G@std@@V?$allocator@U?$pair@$$CBGPEAUtagIP4Address@@@std@@@3@$0A@@std@@@std@@QEAAPEAU?$_Tree_node@U?$pair@$$CBGPEAUtagIP4Address@@@std@@PEAX@2@XZ 000000014000f1d0 f i cSnmpEX.obj
 0001:0000e200       ??0PROTO_GAME_USER_INFO_tag@@QEAA@XZ 000000014000f200 f i DividePacket.obj
 0001:0000e7b0       ??0PROTO_START_HOST_tag@@QEAA@XZ 000000014000f7b0 f i DividePacket.obj
 0001:0000e830       ?GetMessageMap@CGameServerManagerApp@@MEBAPEBUAFX_MSGMAP@@XZ 000000014000f830 f   GameServerManager.obj
 0001:0000e840       ?KillServiceWithErrorcode@@YAXPEAUSERVICE_STATUS_HANDLE__@@K@Z 000000014000f840 f   GameServerManager.obj
 0001:0000e8a0       ??_GCGameServerManagerApp@@UEAAPEAXI@Z 000000014000f8a0 f i GameServerManager.obj
 0001:0000e8a0       ??_ECGameServerManagerApp@@UEAAPEAXI@Z 000000014000f8a0 f i * CIL library *:* CIL module *
 0001:0000e8f0       ?InitInstance@CGameServerManagerApp@@UEAAHXZ 000000014000f8f0 f   GameServerManager.obj
 0001:0000e940       ?SetMyServiceStatus@@YAXKK@Z 000000014000f940 f   GameServerManager.obj
 0001:0000e9a0       ?MyServiceMain@@YAXKPEAPEAD@Z 000000014000f9a0 f   GameServerManager.obj
 0001:0000ed00       ?MyServiceHandler@@YAXK@Z  000000014000fd00 f   GameServerManager.obj
 0001:0000edc0       ?GetApplicationRecoveryPingInterval@CWinApp@@UEAAKXZ 000000014000fdc0 f i GameServerManager.obj
 0001:0000edd0       ?_Get_deleter@_Ref_count_base@std@@UEBAPEAXAEBVtype_info@@@Z 000000014000fdd0 f i GameServerManagerDlg.obj
 0001:0000edd0       __scrt_initialize_winrt    000000014000fdd0 f i msvcrt:utility_desktop.obj
 0001:0000edd0       _get_startup_thread_locale_mode 000000014000fdd0 f i msvcrt:thread_locale.obj
 0001:0000edd0       ?GetClientLib@IClientHandler@@UEAAPEAVCClientLib@@XZ 000000014000fdd0 f i GameServerManagerDlg.obj
 0001:0000edd0       _get_startup_new_mode      000000014000fdd0 f i msvcrt:new_mode.obj
 0001:0000edd0       __scrt_stub_for_initialize_mta 000000014000fdd0 f i msvcrt:utility_desktop.obj
 0001:0000edd0       ?GetApplicationRecoveryParameter@CWinApp@@UEAAPEAXXZ 000000014000fdd0 f i GameServerManager.obj
 0001:0000edd0       _get_startup_commit_mode   000000014000fdd0 f i msvcrt:commit_mode.obj
 0001:0000edd0       __scrt_exe_initialize_mta  000000014000fdd0 f i msvcrt:utility_desktop.obj
 0001:0000edd0       _matherr                   000000014000fdd0 f i msvcrt:matherr.obj
 0001:0000edd0       ?thdPing@CHostStat@@KAIPEAX@Z 000000014000fdd0 f i HostStat.obj
 0001:0000edd0       ?GetApplicationRestartFlags@CWinApp@@UEAAKXZ 000000014000fdd0 f i GameServerManager.obj
 0001:0000ede0       ?RestoreAutosavedFilesAtRestart@CWinApp@@UEBAHXZ 000000014000fde0 f i GameServerManager.obj
 0001:0000edf0       ?ReopenPreviousFilesAtRestart@CWinApp@@UEBAHXZ 000000014000fdf0 f i GameServerManager.obj
 0001:0000ee00       ?SupportsAutosaveAtInterval@CWinApp@@UEBAHXZ 000000014000fe00 f i GameServerManager.obj
 0001:0000ee10       ?SupportsAutosaveAtRestart@CWinApp@@UEBAHXZ 000000014000fe10 f i GameServerManager.obj
 0001:0000ee20       ?SupportsApplicationRecovery@CWinApp@@UEBAHXZ 000000014000fe20 f i GameServerManager.obj
 0001:0000ee30       ?SupportsRestartManager@CWinApp@@UEBAHXZ 000000014000fe30 f i GameServerManager.obj
 0001:0000ee40       ??1IClientHandler@@UEAA@XZ 000000014000fe40 f i GameServerManagerDlg.obj
 0001:0000ee50       ??_EIClientHandler@@UEAAPEAXI@Z 000000014000fe50 f i * CIL library *:* CIL module *
 0001:0000ee50       ??_GIClientHandler@@UEAAPEAXI@Z 000000014000fe50 f i GameServerManagerDlg.obj
 0001:0000ee80       ?Init@GameServerIPCMemory@@QEAAXXZ 000000014000fe80 f i GameServerManagerDlg.obj
 0001:0000f360       ?Init@GAMESERVERINFO@@QEAAXXZ 0000000140010360 f i GameServerManagerDlg.obj
 0001:0000f440       ?GetGAME_MGMT_SETTING_FILE_PATH@@YAPEBDXZ 0000000140010440 f   GameServerManagerDlg.obj
 0001:0000f4e0       ?GetStringFormat@@YA?AV?$basic_string@DU?$char_traits@D@std@@V?$allocator@D@2@@std@@PEADZZ 00000001400104e0 f   GameServerManagerDlg.obj
 0001:0000f5c0       ?KillRemoteProcess@@YA_NK@Z 00000001400105c0 f   GameServerManagerDlg.obj
 0001:0000fa30       ??0CGameServerManagerDlg@@QEAA@PEAVCWnd@@@Z 0000000140010a30 f   GameServerManagerDlg.obj
 0001:0000fd20       ??_GCGameServerManagerDlg@@UEAAPEAXI@Z 0000000140010d20 f i GameServerManagerDlg.obj
 0001:0000fd20       ??_ECGameServerManagerDlg@@UEAAPEAXI@Z 0000000140010d20 f i * CIL library *:* CIL module *
 0001:0000fd70       ??1?$map@IUPORTINFO@@U?$less@I@std@@V?$allocator@U?$pair@$$CBIUPORTINFO@@@std@@@3@@std@@QEAA@XZ 0000000140010d70 f i GameServerManagerDlg.obj
 0001:0000fd90       ??0GAMESERVERINFO@@QEAA@XZ 0000000140010d90 f i GameServerManagerDlg.obj
 0001:0000fe20       ??0GameServerIPCMemory@@QEAA@XZ 0000000140010e20 f i GameServerManagerDlg.obj
 0001:00010be0       ??0PROTO_SPEC_RECOMMENDROOM_INGAME_DATA@@QEAA@XZ 0000000140011be0 f i GameServerManagerDlg.obj
 0001:00010f00       ??1CGameServerManagerDlg@@UEAA@XZ 0000000140011f00 f   GameServerManagerDlg.obj
 0001:00011320       ?DoDataExchange@CGameServerManagerDlg@@MEAAXPEAVCDataExchange@@@Z 0000000140012320 f   GameServerManagerDlg.obj
 0001:00011370       ?WindowProc@CGameServerManagerDlg@@MEAA_JI_K_J@Z 0000000140012370 f   GameServerManagerDlg.obj
 0001:00011380       ?GetMessageMap@CGameServerManagerDlg@@MEBAPEBUAFX_MSGMAP@@XZ 0000000140012380 f   GameServerManagerDlg.obj
 0001:00011390       ?OnInitDialog@CGameServerManagerDlg@@MEAAHXZ 0000000140012390 f   GameServerManagerDlg.obj
 0001:00011470       ?OnPaint@CGameServerManagerDlg@@IEAAXXZ 0000000140012470 f   GameServerManagerDlg.obj
 0001:00011580       ?OnQueryDragIcon@CGameServerManagerDlg@@IEAAPEAUHICON__@@XZ 0000000140012580 f   GameServerManagerDlg.obj
 0001:00011590       ?InitializeManager@CGameServerManagerDlg@@QEAAHPEADKPEAPEAD@Z 0000000140012590 f   GameServerManagerDlg.obj
 0001:00012110       ?DestroyManager@CGameServerManagerDlg@@QEAAXXZ 0000000140013110 f   GameServerManagerDlg.obj
 0001:000121e0       ?ReadSettings@CGameServerManagerDlg@@QEAAHXZ 00000001400131e0 f   GameServerManagerDlg.obj
 0001:00012740       ?ConnectToMatchMakingServer@CGameServerManagerDlg@@QEAAHXZ 0000000140013740 f   GameServerManagerDlg.obj
 0001:000129d0       ?StartGameServer@CGameServerManagerDlg@@QEAAHF@Z 00000001400139d0 f   GameServerManagerDlg.obj
 0001:00012cf0       ?OnGameServerMsg@CGameServerManagerDlg@@IEAA_J_K_J@Z 0000000140013cf0 f   GameServerManagerDlg.obj
 0001:00015240       ?KillServerApp@CGameServerManagerDlg@@IEAAXI_N@Z 0000000140016240 f   GameServerManagerDlg.obj
 0001:00015a30       ??0PROTO_GAME_ENDED_tag@@QEAA@XZ 0000000140016a30 f i GameServerManagerDlg.obj
 0001:00015a80       ??0PROTO_USER_STAT_tag@@QEAA@XZ 0000000140016a80 f i GameServerManagerDlg.obj
 0001:00015b90       ?OnTimer@CGameServerManagerDlg@@IEAAX_K@Z 0000000140016b90 f   GameServerManagerDlg.obj
 0001:000164a0       ?OnButtonGo@CGameServerManagerDlg@@IEAAXXZ 00000001400174a0 f   GameServerManagerDlg.obj
 0001:00016560       ?OnDisconnect@CGameServerManagerDlg@@UEAAXXZ 0000000140017560 f   GameServerManagerDlg.obj
 0001:000165a0       ?TerminateGameServer@CGameServerManagerDlg@@QEAAXF@Z 00000001400175a0 f   GameServerManagerDlg.obj
 0001:00016aa0       ?TerminateGSThread@CGameServerManagerDlg@@SAIPEAX@Z 0000000140017aa0 f   GameServerManagerDlg.obj
 0001:00016ae0       ?SendMessageToWriteLogFile@CGameServerManagerDlg@@QEAAXFPEAUHWND__@@0AEAUtagCOPYDATASTRUCT@@@Z 0000000140017ae0 f   GameServerManagerDlg.obj
 0001:00016ba0       ?VerifyServerAppTermination@CGameServerManagerDlg@@AEAAXXZ 0000000140017ba0 f   GameServerManagerDlg.obj
 0001:00016f60       ?StringSplitToNumArray@CGameServerManagerDlg@@AEAAXV?$basic_string@DU?$char_traits@D@std@@V?$allocator@D@2@@std@@0PEAHAEAH@Z 0000000140017f60 f   GameServerManagerDlg.obj
 0001:00017300       ?FindFreePorts@CGameServerManagerDlg@@AEAA_NXZ 0000000140018300 f   GameServerManagerDlg.obj
 0001:000175a0       ?_GetFreePort@CGameServerManagerDlg@@AEBA_NFPEAI@Z 00000001400185a0 f   GameServerManagerDlg.obj
 0001:000176a0       ?RestoreFreePort@CGameServerManagerDlg@@AEAAXXZ 00000001400186a0 f   GameServerManagerDlg.obj
 0001:000178d0       ?ReservePort@CGameServerManagerDlg@@AEAAXIF@Z 00000001400188d0 f   GameServerManagerDlg.obj
 0001:000179c0       ?ChangeNumRoomsReserved@CGameServerManagerDlg@@QEAAXHH_N@Z 00000001400189c0 f   GameServerManagerDlg.obj
 0001:00017be0       ?ChangeNumActiveServers@CGameServerManagerDlg@@QEAAXH@Z 0000000140018be0 f   GameServerManagerDlg.obj
 0001:00017cc0       ?ServerAppUseCountLog@CGameServerManagerDlg@@AEAAXXZ 0000000140018cc0 f   GameServerManagerDlg.obj
 0001:00017d70       ??0CSharedMemoryLoader@@QEAA@XZ 0000000140018d70 f   GameServerManagerDlg.obj
 0001:00017fd0       ??1CSharedMemoryLoader@@QEAA@XZ 0000000140018fd0 f   GameServerManagerDlg.obj
 0001:000180d0       ?_PreLoad@CSharedMemoryLoader@@AEAA_NXZ 00000001400190d0 f   GameServerManagerDlg.obj
 0001:00018290       ?_Load@CSharedMemoryLoader@@AEAA_NXZ 0000000140019290 f   GameServerManagerDlg.obj
 0001:000186e0       ?Load@CSharedMemoryLoader@@QEAA_NXZ 00000001400196e0 f   GameServerManagerDlg.obj
 0001:00018870       ?Release@CSharedMemoryLoader@@QEAA_NXZ 0000000140019870 f   GameServerManagerDlg.obj
 0001:000188f0       ?ProcessThread@CGameServerManagerDlg@@CAIPEAX@Z 00000001400198f0 f   GameServerManagerDlg.obj
 0001:000189b0       ?ProcessSocketEventThread@CGameServerManagerDlg@@CAIPEAX@Z 00000001400199b0 f   GameServerManagerDlg.obj
 0001:00018a00       ?PostMessageToWriteLogFile@CGameServerManagerDlg@@AEAA_NFPEAUHWND__@@_K_J@Z 0000000140019a00 f   GameServerManagerDlg.obj
 0001:00018ac0       ?OnCopyData@CGameServerManagerDlg@@IEAAHPEAVCWnd@@PEAUtagCOPYDATASTRUCT@@@Z 0000000140019ac0 f   GameServerManagerDlg.obj
 0001:00019300       ?RECV_MSG_REMOVE_CLIENT@CGameServerManagerDlg@@AEAAXFPEBUGAMEPROTO_SC_REMOVECLIENT@@@Z 000000014001a300 f   GameServerManagerDlg.obj
 0001:00019430       ?RECV_MSG_GAMEEND@CGameServerManagerDlg@@AEAAXFPEBUGAMEPROTO_SS_GAMEEND@@@Z 000000014001a430 f   GameServerManagerDlg.obj
 0001:0001de30       ?RECV_MSG_HOST_USER_STAT@CGameServerManagerDlg@@AEAAXFPEBUGAMEPROTO_SC_HOST_USER_STAT@@@Z 000000014001ee30 f   GameServerManagerDlg.obj
 0001:0001f560       ?RECV_MSG_BAN_USER@CGameServerManagerDlg@@AEAAXFPEAUPROTO_BAN_USER_tag@@@Z 0000000140020560 f   GameServerManagerDlg.obj
 0001:0001f600       ?RECV_MSG_HOST_STAT@CGameServerManagerDlg@@AEAAXFPEBUGAMEPROTO_SC_HOST_STAT@@@Z 0000000140020600 f   GameServerManagerDlg.obj
 0001:0001f8c0       ?RECV_MSG_INGAME_AIGACHA_ITEM_INSERT@CGameServerManagerDlg@@AEAAXFPEAUPROTO_GAMEGT_INGAME_AIGACHA_ITEM_INSERT@@@Z 00000001400208c0 f   GameServerManagerDlg.obj
 0001:0001f990       ?RECV_MSG_MAPLOADING_COMPLETE_NTY@CGameServerManagerDlg@@AEAAXFPEAUPROTO_GAMEGT_MAPLOADING_COMPLETE_NTY_tag@@@Z 0000000140020990 f   GameServerManagerDlg.obj
 0001:0001fa20       ?RECV_MSG_SPY_CHANGE@CGameServerManagerDlg@@AEAAXFPEAUGAMEPROTO_SC_SPY_CHANGE@@@Z 0000000140020a20 f   GameServerManagerDlg.obj
 0001:0001fb00       ?RECV_MSG_INGAME_FARMING_ITEM_REQ@CGameServerManagerDlg@@AEAAXFPEAUPROTO_GAMEGT_INGAME_FARMING_ITEM_REQ@@@Z 0000000140020b00 f   GameServerManagerDlg.obj
 0001:0001fbb0       ?RECV_MSG_AI2_BONUSROUND_REWARD@CGameServerManagerDlg@@AEAAXFPEAUPROTOCOL_AI2_BONUSROUND_REWARD_REQ_tag@@@Z 0000000140020bb0 f   GameServerManagerDlg.obj
 0001:0001fc60       ?RECV_MSG_AI3_BONUS_REWARD_ITEM@CGameServerManagerDlg@@AEAAXFPEAUPROTO_GAMEGT_INGAME_AI3_BONUS_REWARD_ITEM_REQ@@@Z 0000000140020c60 f   GameServerManagerDlg.obj
 0001:0001fd10       ?RECV_MSG_AI_EXTRA_REWARD@CGameServerManagerDlg@@AEAAXFPEAUPROTO_AI_EXTRA_REWARD_REQ@@@Z 0000000140020d10 f   GameServerManagerDlg.obj
 0001:0001ff30       ?RECV_MSG_FINISHED_GAME_PREV@CGameServerManagerDlg@@AEAAXFPEAUPROTO_FINISHED_GAME_PREV_tag@@@Z 0000000140020f30 f   GameServerManagerDlg.obj
 0001:0001fff0       ?RECV_MSG_SPEC_RECOMMENDROOM_INGAME_DATA@CGameServerManagerDlg@@AEAAXFPEBUPROTO_SPEC_RECOMMENDROOM_INGAME_DATA@@@Z 0000000140020ff0 f   GameServerManagerDlg.obj
 0001:00020150       ?RECV_MSG_AUTO_SIDE_CHANGE_TEAM_INFO_NTY@CGameServerManagerDlg@@AEAAXFPEAUPROTO_GAMEGT_AUTO_SIDE_CHANGE_TEAM_INFO_NTY@@@Z 0000000140021150 f   GameServerManagerDlg.obj
 0001:000202d0       ?RECV_MSG_INSERTCHARACTER_ACK@CGameServerManagerDlg@@AEAAXFPEBUPROTO_INSERT_CHARACTER_RESULT_tag@@@Z 00000001400212d0 f   GameServerManagerDlg.obj
 0001:00020440       ?OnReceive@CGameServerManagerDlg@@UEAAXPEAVCPacket@@@Z 0000000140021440 f   GameServerManagerDlg.obj
 0001:00020570       ?OnReceiveFromGms@CGameServerManagerDlg@@AEAAXPEAVCPacket@@@Z 0000000140021570 f   GameServerManagerDlg.obj
 0001:00020ab0       ?OnReceiveFromGms@CGameServerManagerDlg@@AEAAXAEBUPROTO_STARTING_GAME_tag@@@Z 0000000140021ab0 f   GameServerManagerDlg.obj
 0001:00020de0       ?OnReceiveFromGms@CGameServerManagerDlg@@AEAAXAEBUPROTO_INSERT_CHARACTER_tag@@@Z 0000000140021de0 f   GameServerManagerDlg.obj
 0001:00021220       ?OnReceiveFromGms@CGameServerManagerDlg@@AEAAXAEBUPROTO_MMSERVER_TERMINATED_tag@@@Z 0000000140022220 f   GameServerManagerDlg.obj
 0001:00021590       ?OnReceiveFromGms@CGameServerManagerDlg@@AEAAXAEBUPROTO_USER_DISCONNECTED_tag@@@Z 0000000140022590 f   GameServerManagerDlg.obj
 0001:000217d0       ?OnReceiveFromGms@CGameServerManagerDlg@@AEAAXAEBUPROTO_GAMEGT_INGAME_AIGACHA_ITEM_INSERT_RESULT@@@Z 00000001400227d0 f   GameServerManagerDlg.obj
 0001:00021a40       ?OnReceiveFromGms@CGameServerManagerDlg@@AEAAXAEBUPROTO_AUTOMATCH_GAME_START_REQ@@@Z 0000000140022a40 f   GameServerManagerDlg.obj
 0001:00021d60       ?OnReceiveFromGms@CGameServerManagerDlg@@AEAAXAEBUPROTO_AUTOMATCH_GAME_ENTER_REQ@@@Z 0000000140022d60 f   GameServerManagerDlg.obj
 0001:00022210       ?FindServerApp@CGameServerManagerDlg@@AEAA?B_NFKAEAF@Z 0000000140023210 f   GameServerManagerDlg.obj
 0001:000222e0       ?AssignServerApp@CGameServerManagerDlg@@AEAAXAEBUPROTO_STARTING_GAME_tag@@F@Z 00000001400232e0 f   GameServerManagerDlg.obj
 0001:000233b0       ?AssignServerApp@CGameServerManagerDlg@@AEAAXAEBUPROTO_AUTOMATCH_GAME_START_REQ@@F@Z 00000001400243b0 f   GameServerManagerDlg.obj
 0001:00024420       ?SendToGmsStartingGameRes@CGameServerManagerDlg@@AEAAXAEBUGAMESERVERINFO@@FW4START_HOST_RESULT@@@Z 0000000140025420 f   GameServerManagerDlg.obj
 0001:00024530       ?SendToGmsAutoMatchGameStartRes@CGameServerManagerDlg@@AEAAXAEBUGAMESERVERINFO@@FW4START_HOST_RESULT@@@Z 0000000140025530 f   GameServerManagerDlg.obj
 0001:00024960       ?SendToGmsAutoMatchGameEnterNty@CGameServerManagerDlg@@AEAAXF@Z 0000000140025960 f   GameServerManagerDlg.obj
 0001:00024e60       ?SendToServerAppAutoMatchGameEnterNty@CGameServerManagerDlg@@AEAAXF@Z 0000000140025e60 f   GameServerManagerDlg.obj
 0001:00024f20       ??1?$shared_ptr@UGAMESERVERINFO@@@std@@QEAA@XZ 0000000140025f20 f i GameServerManagerDlg.obj
 0001:00024f80       ??1?$list@UverifyTerminationStatus_t@@V?$allocator@UverifyTerminationStatus_t@@@std@@@std@@QEAA@XZ 0000000140025f80 f i GameServerManagerDlg.obj
 0001:00024fe0       ?clear@?$_Tree@V?$_Tmap_traits@IUPORTINFO@@U?$less@I@std@@V?$allocator@U?$pair@$$CBIUPORTINFO@@@std@@@3@$0A@@std@@@std@@QEAAXXZ 0000000140025fe0 f i GameServerManagerDlg.obj
 0001:00025070       ?find_first_of@?$basic_string@DU?$char_traits@D@std@@V?$allocator@D@2@@std@@QEBA_KAEBV12@_K@Z 0000000140026070 f i GameServerManagerDlg.obj
 0001:00025160       ?_Erase@?$_Tree@V?$_Tmap_traits@IUPORTINFO@@U?$less@I@std@@V?$allocator@U?$pair@$$CBIUPORTINFO@@@std@@@3@$0A@@std@@@std@@IEAAXPEAU?$_Tree_node@U?$pair@$$CBIUPORTINFO@@@std@@PEAX@2@@Z 0000000140026160 f i GameServerManagerDlg.obj
 0001:000251c0       ?_Buynode0@?$_List_alloc@U?$_List_base_types@UverifyTerminationStatus_t@@V?$allocator@UverifyTerminationStatus_t@@@std@@@std@@@std@@QEAAPEAU?$_List_node@UverifyTerminationStatus_t@@PEAX@2@PEAU32@0@Z 00000001400261c0 f i GameServerManagerDlg.obj
 0001:00025200       ?_Extract@?$_Tree_val@U?$_Tree_simple_types@U?$pair@$$CBIUPORTINFO@@@std@@@std@@@std@@QEAAPEAU?$_Tree_node@U?$pair@$$CBIUPORTINFO@@@std@@PEAX@2@V?$_Tree_const_iterator@V?$_Tree_val@U?$_Tree_simple_types@U?$pair@$$CBIUPORTINFO@@@std@@@std@@@std@@@2@@Z 0000000140026200 f i GameServerManagerDlg.obj
 0001:00025580       ?_Buyheadnode@?$_Tree_comp_alloc@V?$_Tmap_traits@IUPORTINFO@@U?$less@I@std@@V?$allocator@U?$pair@$$CBIUPORTINFO@@@std@@@3@$0A@@std@@@std@@QEAAPEAU?$_Tree_node@U?$pair@$$CBIUPORTINFO@@@std@@PEAX@2@XZ 0000000140026580 f i GameServerManagerDlg.obj
 0001:000255b0       ?_Rrotate@?$_Tree_val@U?$_Tree_simple_types@U?$pair@$$CBIUPORTINFO@@@std@@@std@@@std@@QEAAXPEAU?$_Tree_node@U?$pair@$$CBIUPORTINFO@@@std@@PEAX@2@@Z 00000001400265b0 f i GameServerManagerDlg.obj
 0001:00025610       ?_Lrotate@?$_Tree_val@U?$_Tree_simple_types@U?$pair@$$CBIUPORTINFO@@@std@@@std@@@std@@QEAAXPEAU?$_Tree_node@U?$pair@$$CBIUPORTINFO@@@std@@PEAX@2@@Z 0000000140026610 f i GameServerManagerDlg.obj
 0001:00025670       ??$sprintf_s@$0GE@@cf@@YAHAEAY0GE@DPEBDZZ 0000000140026670 f i GameServerManagerDlg.obj
 0001:000256b0       ??$sprintf_s@$0PP@@cf@@YAHAEAY0PP@DPEBDZZ 00000001400266b0 f i GameServerManagerDlg.obj
 0001:000256f0       ?reserve@?$basic_string@DU?$char_traits@D@std@@V?$allocator@D@2@@std@@QEAAX_K@Z 00000001400266f0 f i GameServerManagerDlg.obj
 0001:000258b0       ??$_Setp@UGAMESERVERINFO@@@?$shared_ptr@UGAMESERVERINFO@@@std@@AEAAXPEAUGAMESERVERINFO@@U?$integral_constant@_N$0A@@1@@Z 00000001400268b0 f i GameServerManagerDlg.obj
 0001:00025910       ??$_Buynode@AEBUverifyTerminationStatus_t@@@?$_List_buy@UverifyTerminationStatus_t@@V?$allocator@UverifyTerminationStatus_t@@@std@@@std@@QEAAPEAU?$_List_node@UverifyTerminationStatus_t@@PEAX@1@PEAU21@0AEBUverifyTerminationStatus_t@@@Z 0000000140026910 f i GameServerManagerDlg.obj
 0001:00025940       ?_Delete_this@?$_Ref_count@UGAMESERVERINFO@@@std@@EEAAXXZ 0000000140026940 f i GameServerManagerDlg.obj
 0001:00025960       ?_Destroy@?$_Ref_count@UGAMESERVERINFO@@@std@@EEAAXXZ 0000000140026960 f i GameServerManagerDlg.obj
 0001:00025970       ??_E?$_Ref_count@UGAMESERVERINFO@@@std@@UEAAPEAXI@Z 0000000140026970 f i * CIL library *:* CIL module *
 0001:00025970       ??_G?$_Ref_count@UGAMESERVERINFO@@@std@@UEAAPEAXI@Z 0000000140026970 f i GameServerManagerDlg.obj
 0001:000259a0       ??$_Buynode@U?$pair@IUPORTINFO@@@std@@@?$_Tree_comp_alloc@V?$_Tmap_traits@IUPORTINFO@@U?$less@I@std@@V?$allocator@U?$pair@$$CBIUPORTINFO@@@std@@@3@$0A@@std@@@std@@QEAAPEAU?$_Tree_node@U?$pair@$$CBIUPORTINFO@@@std@@PEAX@1@$$QEAU?$pair@IUPORTINFO@@@1@@Z 00000001400269a0 f i GameServerManagerDlg.obj
 0001:000259d0       ??$_Insert_nohint@AEAU?$pair@$$CBIUPORTINFO@@@std@@PEAU?$_Tree_node@U?$pair@$$CBIUPORTINFO@@@std@@PEAX@2@@?$_Tree@V?$_Tmap_traits@IUPORTINFO@@U?$less@I@std@@V?$allocator@U?$pair@$$CBIUPORTINFO@@@std@@@3@$0A@@std@@@std@@IEAA?AU?$pair@V?$_Tree_iterator@V?$_Tree_val@U?$_Tree_simple_types@U?$pair@$$CBIUPORTINFO@@@std@@@std@@@std@@@std@@_N@1@_NAEAU?$pair@$$CBIUPORTINFO@@@1@PEAU?$_Tree_node@U?$pair@$$CBIUPORTINFO@@@std@@PEAX@1@@Z 00000001400269d0 f i GameServerManagerDlg.obj
 0001:00025b30       ?_Buynode0@?$_Tree_comp_alloc@V?$_Tmap_traits@IUPORTINFO@@U?$less@I@std@@V?$allocator@U?$pair@$$CBIUPORTINFO@@@std@@@3@$0A@@std@@@std@@QEAAPEAU?$_Tree_node@U?$pair@$$CBIUPORTINFO@@@std@@PEAX@2@XZ 0000000140026b30 f i GameServerManagerDlg.obj
 0001:00025b60       ?_Destroy_if_node@?$_Tree@V?$_Tmap_traits@IUPORTINFO@@U?$less@I@std@@V?$allocator@U?$pair@$$CBIUPORTINFO@@@std@@@3@$0A@@std@@@std@@IEAAXPEAU?$_Tree_node@U?$pair@$$CBIUPORTINFO@@@std@@PEAX@2@@Z 0000000140026b60 f i GameServerManagerDlg.obj
 0001:00025b70       ??$_Insert_at@AEAU?$pair@$$CBIUPORTINFO@@@std@@PEAU?$_Tree_node@U?$pair@$$CBIUPORTINFO@@@std@@PEAX@2@@?$_Tree@V?$_Tmap_traits@IUPORTINFO@@U?$less@I@std@@V?$allocator@U?$pair@$$CBIUPORTINFO@@@std@@@3@$0A@@std@@@std@@IEAA?AV?$_Tree_iterator@V?$_Tree_val@U?$_Tree_simple_types@U?$pair@$$CBIUPORTINFO@@@std@@@std@@@std@@@1@_NPEAU?$_Tree_node@U?$pair@$$CBIUPORTINFO@@@std@@PEAX@1@AEAU?$pair@$$CBIUPORTINFO@@@1@1@Z 0000000140026b70 f i GameServerManagerDlg.obj
 0001:00025e20       ??$_Buynode@AEBUpiecewise_construct_t@std@@V?$tuple@AEBI@2@V?$tuple@$$V@2@@?$_Tree_comp_alloc@V?$_Tmap_traits@IUPORTINFO@@U?$less@I@std@@V?$allocator@U?$pair@$$CBIUPORTINFO@@@std@@@3@$0A@@std@@@std@@QEAAPEAU?$_Tree_node@U?$pair@$$CBIUPORTINFO@@@std@@PEAX@1@AEBUpiecewise_construct_t@1@$$QEAV?$tuple@AEBI@1@$$QEAV?$tuple@$$V@1@@Z 0000000140026e20 f i GameServerManagerDlg.obj
 0001:00025e50       ??$_Insert_hint@AEAU?$pair@$$CBIUPORTINFO@@@std@@PEAU?$_Tree_node@U?$pair@$$CBIUPORTINFO@@@std@@PEAX@2@@?$_Tree@V?$_Tmap_traits@IUPORTINFO@@U?$less@I@std@@V?$allocator@U?$pair@$$CBIUPORTINFO@@@std@@@3@$0A@@std@@@std@@IEAA?AV?$_Tree_iterator@V?$_Tree_val@U?$_Tree_simple_types@U?$pair@$$CBIUPORTINFO@@@std@@@std@@@std@@@1@V?$_Tree_const_iterator@V?$_Tree_val@U?$_Tree_simple_types@U?$pair@$$CBIUPORTINFO@@@std@@@std@@@std@@@1@AEAU?$pair@$$CBIUPORTINFO@@@1@PEAU?$_Tree_node@U?$pair@$$CBIUPORTINFO@@@std@@PEAX@1@@Z 0000000140026e50 f i GameServerManagerDlg.obj
 0001:00026098       ??_ECGameServerManagerDlg@@WBDA@EAAPEAXI@Z 0000000140027098 f i GameServerManagerDlg.obj
 0001:000260b0       ?append@?$basic_string@DU?$char_traits@D@std@@V?$allocator@D@2@@std@@QEAAAEAV12@AEBV12@@Z 00000001400270b0 f i GameServerManagerDlg.obj
 0001:00026270       ??4WEAPON_INFO@@QEAAAEAU0@AEBU0@@Z 0000000140027270 f i GameServerManagerDlg.obj
 0001:000263b0       ?find_last_of@?$basic_string@DU?$char_traits@D@std@@V?$allocator@D@2@@std@@QEBA_KQEBD_K@Z 00000001400273b0 f i GameServerManagerDlg.obj
 0001:00026470       ??4?$basic_string@DU?$char_traits@D@std@@V?$allocator@D@2@@std@@QEAAAEAV01@$$QEAV01@@Z 0000000140027470 f i GameServerManagerDlg.obj
 0001:000264c0       ?_Xran@?$_String_val@U?$_Simple_types@D@std@@@std@@SAXXZ 00000001400274c0 f i GameServerManagerDlg.obj
 0001:000264e0       ?substr@?$basic_string@DU?$char_traits@D@std@@V?$allocator@D@2@@std@@QEBA?AV12@_K0@Z 00000001400274e0 f i GameServerManagerDlg.obj
 0001:00026540       ??$_Reallocate_grow_by@V<lambda_65e615be2a453ca0576c979606f46740>@@PEBD_K@?$basic_string@DU?$char_traits@D@std@@V?$allocator@D@2@@std@@QEAAAEAV01@_KV<lambda_65e615be2a453ca0576c979606f46740>@@PEBD_K@Z 0000000140027540 f i GameServerManagerDlg.obj
 0001:000266c0       ?append@?$basic_string@DU?$char_traits@D@std@@V?$allocator@D@2@@std@@QEAAAEAV12@QEBD_K@Z 00000001400276c0 f i GameServerManagerDlg.obj
 0001:00026740       ?append@?$basic_string@DU?$char_traits@D@std@@V?$allocator@D@2@@std@@QEAAAEAV12@QEBD@Z 0000000140027740 f i GameServerManagerDlg.obj
 0001:00026760       ?init@SGGMProxyLoader@sggm_proxy@@QEAA_NPEAVMultiReceiver@2@@Z 0000000140027760 f i GameServerManagerDlg.obj
 0001:00026990       __local_stdio_scanf_options 0000000140027990 f i GameServerManagerDlg.obj
 0001:000269a0       sscanf                     00000001400279a0 f i GameServerManagerDlg.obj
 0001:00026a00       ??0BATTLE_ROYAL_RESULT@@QEAA@XZ 0000000140027a00 f i GameServerManagerDlg.obj
 0001:00026da0       ??0GAMEPROTO_SC_HOST_USER_STAT@@QEAA@XZ 0000000140027da0 f i GameServerManagerDlg.obj
 0001:00026ff0       ??0GAMEPROTO_SS_GAMEEND@@QEAA@XZ 0000000140027ff0 f i GameServerManagerDlg.obj
 0001:00028950       ??1SGGMProxyLoader@sggm_proxy@@QEAA@XZ 0000000140029950 f i GameServerManagerDlg.obj
 0001:00028a10       ?StringCchCopyA@@YAJPEAD_KPEBD@Z 0000000140029a10 f i GameServerManagerDlg.obj
 0001:00028a90       ?Send@CGMSConnManager@@AEAAHPEAVCPacket@@@Z 0000000140029a90 f   GMSConnManager.obj
 0001:00028bf0       ?SendDiv@CGMSConnManager@@AEAAHEEEPEADK@Z 0000000140029bf0 f   GMSConnManager.obj
 0001:00028e00       ?SortFinishedGameUserInfo@CGMSConnManager@@AEAAXAEAUPROTO_FINISHED_GAME_tag@@@Z 0000000140029e00 f   GMSConnManager.obj
 0001:00028f20       ??4PROTO_USER_STAT_tag@@QEAAAEAU0@AEBU0@@Z 0000000140029f20 f i GMSConnManager.obj
 0001:0002a100       ??1CGMSConnManager@@QEAA@XZ 000000014002b100 f   GMSConnManager.obj
 0001:0002a130       ??_ECSFGameServerClientLib@@UEAAPEAXI@Z 000000014002b130 f i GMSConnManager.obj
 0001:0002a1d0       ?IsConnected@CGMSConnManager@@QEAAHXZ 000000014002b1d0 f   GMSConnManager.obj
 0001:0002a210       ?StartingReport@CGMSConnManager@@QEAAHFHHHHHHHQEAHHH@Z 000000014002b210 f   GMSConnManager.obj
 0001:0002a5e0       ?StartingGameResult@CGMSConnManager@@QEAAHUPROTO_STARTING_GAME_RESULT_tag@@W4START_HOST_RESULT@@@Z 000000014002b5e0 f   GMSConnManager.obj
 0001:0002a750       ?FinishedGame@CGMSConnManager@@QEAAHUPROTO_FINISHED_GAME_tag@@@Z 000000014002b750 f   GMSConnManager.obj
 0001:0002a7b0       ?UpdateCharacterStat@CGMSConnManager@@QEAAHUPROTO_UPDATE_CHARACTER_STAT_tag@@@Z 000000014002b7b0 f   GMSConnManager.obj
 0001:0002a8c0       ?InsertCharacterResult@CGMSConnManager@@QEAAHUPROTO_INSERT_CHARACTER_RESULT_tag@@@Z 000000014002b8c0 f   GMSConnManager.obj
 0001:0002a9c0       ?SendHeartBeat@CGMSConnManager@@QEAAHH@Z 000000014002b9c0 f   GMSConnManager.obj
 0001:0002aad0       ?SendForceLeavePollResult@CGMSConnManager@@QEAAHPEBUPROTO_BAN_USER_tag@@@Z 000000014002bad0 f   GMSConnManager.obj
 0001:0002abd0       ?NotifyAllocableRoomCountChanged@CGMSConnManager@@QEAAHJHHHHHQEAHHH@Z 000000014002bbd0 f   GMSConnManager.obj
 0001:0002afe0       ?SendRoundChange@CGMSConnManager@@QEAAHPEBUPROTO_GAMEGT_ROUND_CHANGE_NTY_tag@@@Z 000000014002bfe0 f   GMSConnManager.obj
 0001:0002b0e0       ?SendGameStart@CGMSConnManager@@QEAAHPEBUPROTO_GAMEGT_GAME_START_NTY@@@Z 000000014002c0e0 f   GMSConnManager.obj
 0001:0002b1e0       ?SendTeamDeathMatchKillCnt@CGMSConnManager@@QEAAHPEBUPROTO_GAMEGT_TEAM_DEATH_KILL_CNT_NTY@@@Z 000000014002c1e0 f   GMSConnManager.obj
 0001:0002b2e0       ?SendAIItemInsert@CGMSConnManager@@QEAAHPEAUPROTO_GAMEGT_INGAME_AIGACHA_ITEM_INSERT@@@Z 000000014002c2e0 f   GMSConnManager.obj
 0001:0002b440       ?SendIntrusionCoinDec@CGMSConnManager@@QEAAHPEAUPROTO_GAMEGT_MAPLOADING_COMPLETE_NTY_tag@@@Z 000000014002c440 f   GMSConnManager.obj
 0001:0002b540       ?SendSpyChange@CGMSConnManager@@QEAAHPEAUPROTO_GAMEGT_SPY_CHANGE_NTY_tag@@@Z 000000014002c540 f   GMSConnManager.obj
 0001:0002b640       ?SendFarmingItemReq@CGMSConnManager@@QEAAHPEAUPROTO_GAMEGT_INGAME_FARMING_ITEM_REQ@@@Z 000000014002c640 f   GMSConnManager.obj
 0001:0002b790       ?SendBattleShipBonusCoinReq@CGMSConnManager@@QEAAHPEAUPROTOCOL_AI2_BONUSROUND_REWARD_REQ_tag@@@Z 000000014002c790 f   GMSConnManager.obj
 0001:0002b8d0       ?SendAI3BonusClearItemReq@CGMSConnManager@@QEAAHPEAUPROTO_GAMEGT_INGAME_AI3_BONUS_REWARD_ITEM_REQ@@@Z 000000014002c8d0 f   GMSConnManager.obj
 0001:0002b9f0       ?SendAIExtraRewardReq@CGMSConnManager@@QEAAHPEAUPROTO_AI_EXTRA_REWARD_REQ@@@Z 000000014002c9f0 f   GMSConnManager.obj
 0001:0002bb20       ?SendBossTowerRewardReq@CGMSConnManager@@QEAAHPEAUPROTO_AI_BOSS_TOWER_REWARD_REQ@@@Z 000000014002cb20 f   GMSConnManager.obj
 0001:0002bcb0       ?SendIngameRewardReq@CGMSConnManager@@QEAAHPEAUPROTO_INGAME_RESULT_REQ@@@Z 000000014002ccb0 f   GMSConnManager.obj
 0001:0002be40       ?SendKickUserInfo@CGMSConnManager@@QEAAHPEAUPROTO_GAMEMGT_KICK_USER@@@Z 000000014002ce40 f   GMSConnManager.obj
 0001:0002bf50       ?SendSpectatorRecommendRoomData@CGMSConnManager@@QEAAHPEAUPROTO_SPECTATOR_RECOMMEND_ROOM_INGAME_DATA_NTY@@@Z 000000014002cf50 f   GMSConnManager.obj
 0001:0002c0f0       ?SendPrevGameFinishNotify@CGMSConnManager@@QEAAHPEAUPROTO_FINISHED_GAME_PREV_tag@@@Z 000000014002d0f0 f   GMSConnManager.obj
 0001:0002c1f0       ?SendAutoSideChangeTeamInfoNotify@CGMSConnManager@@QEAAHPEAUPROTO_GAMEGT_AUTO_SIDE_CHANGE_TEAM_INFO_NTY@@@Z 000000014002d1f0 f   GMSConnManager.obj
 0001:0002c300       ?SendAIExtraMiddleRewardReq@CGMSConnManager@@QEAAHPEAUPROTO_AI_EXTRA_MIDDLE_REWARD_REQ@@@Z 000000014002d300 f   GMSConnManager.obj
 0001:0002c430       ?SendAutoMatchGameStartRes@CGMSConnManager@@QEAAHAEBUPROTO_AUTOMATCH_GAME_START_RES@@W4START_HOST_RESULT@@@Z 000000014002d430 f   GMSConnManager.obj
 0001:0002c620       ?SendAutoMatchGameEnterRes@CGMSConnManager@@QEAAHAEBUPROTO_AUTOMATCH_GAME_ENTER_RES@@@Z 000000014002d620 f   GMSConnManager.obj
 0001:0002c720       ?SendAutoMatchIngameEnterNty@CGMSConnManager@@QEAAHAEBUPROTO_AUTOMATCH_INGAME_ENTER_NTY@@@Z 000000014002d720 f   GMSConnManager.obj
 0001:0002c8a0       ??$sprintf_s@$0EBA@@cf@@YAHAEAY0EBA@DPEBDZZ 000000014002d8a0 f i GMSConnManager.obj
 0001:0002c8e0       ??$_Reallocate_grow_by@V<lambda_319d5e083f45f90dcdce5dce53cbb275>@@D@?$basic_string@DU?$char_traits@D@std@@V?$allocator@D@2@@std@@QEAAAEAV01@_KV<lambda_319d5e083f45f90dcdce5dce53cbb275>@@D@Z 000000014002d8e0 f i base64.obj
 0001:0002ca40       ?_Tidy@?$vector@V?$basic_string@DU?$char_traits@D@std@@V?$allocator@D@2@@std@@V?$allocator@V?$basic_string@DU?$char_traits@D@std@@V?$allocator@D@2@@std@@@2@@std@@AEAAXXZ 000000014002da40 f i CSmtp.obj
 0001:0002ca40       ??1?$vector@V?$basic_string@DU?$char_traits@D@std@@V?$allocator@D@2@@std@@V?$allocator@V?$basic_string@DU?$char_traits@D@std@@V?$allocator@D@2@@std@@@2@@std@@QEAA@XZ 000000014002da40 f i CSmtp.obj
 0001:0002cab0       ?_Destroy@?$vector@V?$basic_string@DU?$char_traits@D@std@@V?$allocator@D@2@@std@@V?$allocator@V?$basic_string@DU?$char_traits@D@std@@V?$allocator@D@2@@std@@@2@@std@@AEAAXPEAV?$basic_string@DU?$char_traits@D@std@@V?$allocator@D@2@@2@0@Z 000000014002dab0 f i CSmtp.obj
 0001:0002cac0       ?deallocate@?$allocator@V?$basic_string@DU?$char_traits@D@std@@V?$allocator@D@2@@std@@@std@@QEAAXQEAV?$basic_string@DU?$char_traits@D@std@@V?$allocator@D@2@@2@_K@Z 000000014002dac0 f i CSmtp.obj
 0001:0002cb10       ??$?HDU?$char_traits@D@std@@V?$allocator@D@1@@std@@YA?AV?$basic_string@DU?$char_traits@D@std@@V?$allocator@D@2@@0@QEBDAEBV10@@Z 000000014002db10 f i CSmtp.obj
 0001:0002cbc0       ??$_Traits_find@U?$char_traits@D@std@@@std@@YA_KQEBD_K101@Z 000000014002dbc0 f i CSmtp.obj
 0001:0002cc90       ??$_Destroy_range@V?$allocator@V?$basic_string@DU?$char_traits@D@std@@V?$allocator@D@2@@std@@@std@@@std@@YAXPEAV?$basic_string@DU?$char_traits@D@std@@V?$allocator@D@2@@0@0AEAV?$allocator@V?$basic_string@DU?$char_traits@D@std@@V?$allocator@D@2@@std@@@0@@Z 000000014002dc90 f i CSmtp.obj
 0001:0002cd20       ??0?$basic_string@DU?$char_traits@D@std@@V?$allocator@D@2@@std@@QEAA@AEBV01@@Z 000000014002dd20 f i CSmtp.obj
 0001:0002ce00       ??1sentry@?$basic_ostream@DU?$char_traits@D@std@@@std@@QEAA@XZ 000000014002de00 f i md5_csmtp.obj
 0001:0002ce50       ??1_Sentry_base@?$basic_ostream@DU?$char_traits@D@std@@@std@@QEAA@XZ 000000014002de50 f i md5_csmtp.obj
 0001:0002ce80       ??$?6U?$char_traits@D@std@@@std@@YAAEAV?$basic_ostream@DU?$char_traits@D@std@@@0@AEAV10@PEBD@Z 000000014002de80 f i md5_csmtp.obj
 0001:0002d050       ??$endl@DU?$char_traits@D@std@@@std@@YAAEAV?$basic_ostream@DU?$char_traits@D@std@@@0@AEAV10@@Z 000000014002e050 f i md5_csmtp.obj
 0001:0002d090       ?a2toi@@YAHPEADHH@Z        000000014002e090 f i DateTime.obj
 0001:0002d140       ?Add@datetime@@QEAAXV1@@Z  000000014002e140 f   DateTime.obj
 0001:0002d370       ?GetCurrentLocalTime@datetime@@QEAAXXZ 000000014002e370 f   DateTime.obj
 0001:0002d3e0       ?regulate@datetime@@QEAAXXZ 000000014002e3e0 f   DateTime.obj
 0001:0002d4d0       ?addcarry@datetime@@IEAAHAEAHHHH@Z 000000014002e4d0 f   DateTime.obj
 0001:0002d5b0       ?getDay@datetime@@IEAAHHH@Z 000000014002e5b0 f   DateTime.obj
 0001:0002d6e0       ??_ECHostStat@@UEAAPEAXI@Z 000000014002e6e0 f i * CIL library *:* CIL module *
 0001:0002d6e0       ??_GCHostStat@@UEAAPEAXI@Z 000000014002e6e0 f i HostStat.obj
 0001:0002d720       ??1CHostStat@@UEAA@XZ      000000014002e720 f   HostStat.obj
 0001:0002d810       ?setup@CHostStat@@QEAAXHH@Z 000000014002e810 f   HostStat.obj
 0001:0002dcb0       ?thdMail@CHostStat@@KAIPEAX@Z 000000014002ecb0 f   HostStat.obj
 0001:0002e900       ?timer@CHostStat@@QEAAXXZ  000000014002f900 f   HostStat.obj
 0001:0002ede0       ?getData64@CHostStat@@QEAA_JGEEG@Z 000000014002fde0 f   HostStat.obj
 0001:0002f0a0       ?setData64@CHostStat@@QEAAXGEEG_J@Z 00000001400300a0 f   HostStat.obj
 0001:0002f3a0       ?addData@CHostStat@@QEAAXGEEG@Z 00000001400303a0 f   HostStat.obj
 0001:0002f6c0       ?addExtraData@CHostStat@@QEAAXGE@Z 00000001400306c0 f   HostStat.obj
 0001:0002fc20       ?addExtraData@CHostStat@@QEAAXGEEGIII@Z 0000000140030c20 f   HostStat.obj
 0001:0002ffa0       ?send@CHostStat@@IEAA_NPEAD0@Z 0000000140030fa0 f   HostStat.obj
 0001:00030970       ?timerPerfMem@CHostStat@@QEAAXXZ 0000000140031970 f   HostStat.obj
 0001:00030ee0       ?timerLogUser@CHostStat@@QEAAXHHHHH@Z 0000000140031ee0 f   HostStat.obj
 0001:00031190       ?AddLog@CHostStat@@QEAAXPEBDZZ 0000000140032190 f   HostStat.obj
 0001:00031480       ?GatherFiles@CHostStat@@QEAAXPEAD@Z 0000000140032480 f   HostStat.obj
 0001:00031b30       ?GetDataFolder@CHostStat@@QEAAXPEAD_K@Z 0000000140032b30 f   HostStat.obj
 0001:00031bd0       ?AddUserPCSpec@CHostStat@@QEAAXGPEBD00I@Z 0000000140032bd0 f   HostStat.obj
 0001:00031f80       ??$sprintf_s@$0CAA@@cf@@YAHAEAY0CAA@DPEBDZZ 0000000140032f80 f i HostStat.obj
 0001:00031fc0       ??$_Buynode@U?$pair@GUExtraStatsMemVerify@CHostStat@@@std@@@?$_Tree_comp_alloc@V?$_Tmap_traits@GUExtraStatsMemVerify@CHostStat@@U?$less@G@std@@V?$allocator@U?$pair@$$CBGUExtraStatsMemVerify@CHostStat@@@std@@@4@$0A@@std@@@std@@QEAAPEAU?$_Tree_node@U?$pair@$$CBGUExtraStatsMemVerify@CHostStat@@@std@@PEAX@1@$$QEAU?$pair@GUExtraStatsMemVerify@CHostStat@@@1@@Z 0000000140032fc0 f i HostStat.obj
 0001:00031fc0       ??$_Buynode@U?$pair@GUExtraStatsFPSVerify@CHostStat@@@std@@@?$_Tree_comp_alloc@V?$_Tmap_traits@GUExtraStatsFPSVerify@CHostStat@@U?$less@G@std@@V?$allocator@U?$pair@$$CBGUExtraStatsFPSVerify@CHostStat@@@std@@@4@$0A@@std@@@std@@QEAAPEAU?$_Tree_node@U?$pair@$$CBGUExtraStatsFPSVerify@CHostStat@@@std@@PEAX@1@$$QEAU?$pair@GUExtraStatsFPSVerify@CHostStat@@@1@@Z 0000000140032fc0 f i HostStat.obj
 0001:00031ff0       ??$_Insert_nohint@AEAU?$pair@$$CBGUExtraStatsFPSVerify@CHostStat@@@std@@PEAU?$_Tree_node@U?$pair@$$CBGUExtraStatsFPSVerify@CHostStat@@@std@@PEAX@2@@?$_Tree@V?$_Tmap_traits@GUExtraStatsFPSVerify@CHostStat@@U?$less@G@std@@V?$allocator@U?$pair@$$CBGUExtraStatsFPSVerify@CHostStat@@@std@@@4@$0A@@std@@@std@@IEAA?AU?$pair@V?$_Tree_iterator@V?$_Tree_val@U?$_Tree_simple_types@U?$pair@$$CBGUExtraStatsFPSVerify@CHostStat@@@std@@@std@@@std@@@std@@_N@1@_NAEAU?$pair@$$CBGUExtraStatsFPSVerify@CHostStat@@@1@PEAU?$_Tree_node@U?$pair@$$CBGUExtraStatsFPSVerify@CHostStat@@@std@@PEAX@1@@Z 0000000140032ff0 f i HostStat.obj
 0001:00031ff0       ??$_Insert_nohint@AEAU?$pair@$$CBGUExtraStatsMemVerify@CHostStat@@@std@@PEAU?$_Tree_node@U?$pair@$$CBGUExtraStatsMemVerify@CHostStat@@@std@@PEAX@2@@?$_Tree@V?$_Tmap_traits@GUExtraStatsMemVerify@CHostStat@@U?$less@G@std@@V?$allocator@U?$pair@$$CBGUExtraStatsMemVerify@CHostStat@@@std@@@4@$0A@@std@@@std@@IEAA?AU?$pair@V?$_Tree_iterator@V?$_Tree_val@U?$_Tree_simple_types@U?$pair@$$CBGUExtraStatsMemVerify@CHostStat@@@std@@@std@@@std@@@std@@_N@1@_NAEAU?$pair@$$CBGUExtraStatsMemVerify@CHostStat@@@1@PEAU?$_Tree_node@U?$pair@$$CBGUExtraStatsMemVerify@CHostStat@@@std@@PEAX@1@@Z 0000000140032ff0 f i HostStat.obj
 0001:00032160       ?_Buynode0@?$_Tree_comp_alloc@V?$_Tmap_traits@GUExtraStatsMemVerify@CHostStat@@U?$less@G@std@@V?$allocator@U?$pair@$$CBGUExtraStatsMemVerify@CHostStat@@@std@@@4@$0A@@std@@@std@@QEAAPEAU?$_Tree_node@U?$pair@$$CBGUExtraStatsMemVerify@CHostStat@@@std@@PEAX@2@XZ 0000000140033160 f i HostStat.obj
 0001:00032160       ?_Buynode0@?$_Tree_comp_alloc@V?$_Tmap_traits@GUExtraStatsFPSVerify@CHostStat@@U?$less@G@std@@V?$allocator@U?$pair@$$CBGUExtraStatsFPSVerify@CHostStat@@@std@@@4@$0A@@std@@@std@@QEAAPEAU?$_Tree_node@U?$pair@$$CBGUExtraStatsFPSVerify@CHostStat@@@std@@PEAX@2@XZ 0000000140033160 f i HostStat.obj
 0001:00032190       ?_Destroy_if_node@?$_Tree@V?$_Tmap_traits@GUExtraStatsFPSVerify@CHostStat@@U?$less@G@std@@V?$allocator@U?$pair@$$CBGUExtraStatsFPSVerify@CHostStat@@@std@@@4@$0A@@std@@@std@@IEAAXPEAU?$_Tree_node@U?$pair@$$CBGUExtraStatsFPSVerify@CHostStat@@@std@@PEAX@2@@Z 0000000140033190 f i HostStat.obj
 0001:00032190       ?_Destroy_if_node@?$_Tree@V?$_Tmap_traits@GUExtraStatsMemVerify@CHostStat@@U?$less@G@std@@V?$allocator@U?$pair@$$CBGUExtraStatsMemVerify@CHostStat@@@std@@@4@$0A@@std@@@std@@IEAAXPEAU?$_Tree_node@U?$pair@$$CBGUExtraStatsMemVerify@CHostStat@@@std@@PEAX@2@@Z 0000000140033190 f i HostStat.obj
 0001:000321a0       ??$_Insert_at@AEAU?$pair@$$CBGUExtraStatsMemVerify@CHostStat@@@std@@PEAU?$_Tree_node@U?$pair@$$CBGUExtraStatsMemVerify@CHostStat@@@std@@PEAX@2@@?$_Tree@V?$_Tmap_traits@GUExtraStatsMemVerify@CHostStat@@U?$less@G@std@@V?$allocator@U?$pair@$$CBGUExtraStatsMemVerify@CHostStat@@@std@@@4@$0A@@std@@@std@@IEAA?AV?$_Tree_iterator@V?$_Tree_val@U?$_Tree_simple_types@U?$pair@$$CBGUExtraStatsMemVerify@CHostStat@@@std@@@std@@@std@@@1@_NPEAU?$_Tree_node@U?$pair@$$CBGUExtraStatsMemVerify@CHostStat@@@std@@PEAX@1@AEAU?$pair@$$CBGUExtraStatsMemVerify@CHostStat@@@1@1@Z 00000001400331a0 f i HostStat.obj
 0001:000321a0       ??$_Insert_at@AEAU?$pair@$$CBGUExtraStatsFPSVerify@CHostStat@@@std@@PEAU?$_Tree_node@U?$pair@$$CBGUExtraStatsFPSVerify@CHostStat@@@std@@PEAX@2@@?$_Tree@V?$_Tmap_traits@GUExtraStatsFPSVerify@CHostStat@@U?$less@G@std@@V?$allocator@U?$pair@$$CBGUExtraStatsFPSVerify@CHostStat@@@std@@@4@$0A@@std@@@std@@IEAA?AV?$_Tree_iterator@V?$_Tree_val@U?$_Tree_simple_types@U?$pair@$$CBGUExtraStatsFPSVerify@CHostStat@@@std@@@std@@@std@@@1@_NPEAU?$_Tree_node@U?$pair@$$CBGUExtraStatsFPSVerify@CHostStat@@@std@@PEAX@1@AEAU?$pair@$$CBGUExtraStatsFPSVerify@CHostStat@@@1@1@Z 00000001400331a0 f i HostStat.obj
 0001:00032450       ?write@CIniSection@CIniReader@@QEAAKPEAX@Z 0000000140033450 f   iniReader.obj
 0001:00032730       ?setString@CIniSection@CIniReader@@QEAAXPEBD0@Z 0000000140033730 f   iniReader.obj
 0001:000329e0       ?getString@CIniSection@CIniReader@@QEAA_KPEBDPEAD_K@Z 00000001400339e0 f   iniReader.obj
 0001:00032c00       ??1CIniReader@@QEAA@XZ     0000000140033c00 f   iniReader.obj
 0001:00032c40       ?clear@CIniReader@@QEAAXXZ 0000000140033c40 f   iniReader.obj
 0001:00032d50       ?read@CIniReader@@QEAAKPEBD@Z 0000000140033d50 f   iniReader.obj
 0001:00032eb0       ?write@CIniReader@@QEAAKPEBD@Z 0000000140033eb0 f   iniReader.obj
 0001:00033210       ?parse@CIniReader@@QEAAKPEBD@Z 0000000140034210 f   iniReader.obj
 0001:000336e0       ?getInt@CIniReader@@QEAAHPEBD0H@Z 00000001400346e0 f   iniReader.obj
 0001:000338c0       ?getString@CIniReader@@QEAA_KPEBD0PEAD_K@Z 00000001400348c0 f   iniReader.obj
 0001:00033a20       ?getIntArray@CIniReader@@QEAA_KPEBD0PEAH_K@Z 0000000140034a20 f   iniReader.obj
 0001:00033b90       ?setString@CIniReader@@QEAAXPEBD00@Z 0000000140034b90 f   iniReader.obj
 0001:00033d80       ?find@?$_Tree@V?$_Tmap_traits@V?$basic_string@DU?$char_traits@D@std@@V?$allocator@D@2@@std@@PEAVCIniSection@CIniReader@@U?$less@V?$basic_string@DU?$char_traits@D@std@@V?$allocator@D@2@@std@@@2@V?$allocator@U?$pair@$$CBV?$basic_string@DU?$char_traits@D@std@@V?$allocator@D@2@@std@@PEAVCIniSection@CIniReader@@@std@@@2@$0A@@std@@@std@@QEAA?AV?$_Tree_iterator@V?$_Tree_val@U?$_Tree_simple_types@U?$pair@$$CBV?$basic_string@DU?$char_traits@D@std@@V?$allocator@D@2@@std@@PEAVCIniSection@CIniReader@@@std@@@std@@@std@@@2@AEBV?$basic_string@DU?$char_traits@D@std@@V?$allocator@D@2@@2@@Z 0000000140034d80 f i iniReader.obj
 0001:00033e80       ?_Erase@?$_Tree@V?$_Tmap_traits@V?$basic_string@DU?$char_traits@D@std@@V?$allocator@D@2@@std@@PEAVCIniSection@CIniReader@@U?$less@V?$basic_string@DU?$char_traits@D@std@@V?$allocator@D@2@@std@@@2@V?$allocator@U?$pair@$$CBV?$basic_string@DU?$char_traits@D@std@@V?$allocator@D@2@@std@@PEAVCIniSection@CIniReader@@@std@@@2@$0A@@std@@@std@@IEAAXPEAU?$_Tree_node@U?$pair@$$CBV?$basic_string@DU?$char_traits@D@std@@V?$allocator@D@2@@std@@PEAVCIniSection@CIniReader@@@std@@PEAX@2@@Z 0000000140034e80 f i iniReader.obj
 0001:00033f40       ?lower_bound@?$_Tree@V?$_Tmap_traits@V?$basic_string@DU?$char_traits@D@std@@V?$allocator@D@2@@std@@V12@U?$less@V?$basic_string@DU?$char_traits@D@std@@V?$allocator@D@2@@std@@@2@V?$allocator@U?$pair@$$CBV?$basic_string@DU?$char_traits@D@std@@V?$allocator@D@2@@std@@V12@@std@@@2@$0A@@std@@@std@@QEAA?AV?$_Tree_iterator@V?$_Tree_val@U?$_Tree_simple_types@U?$pair@$$CBV?$basic_string@DU?$char_traits@D@std@@V?$allocator@D@2@@std@@V12@@std@@@std@@@std@@@2@AEBV?$basic_string@DU?$char_traits@D@std@@V?$allocator@D@2@@2@@Z 0000000140034f40 f i iniReader.obj
 0001:00034010       ?erase@?$_Tree@V?$_Tmap_traits@V?$basic_string@DU?$char_traits@D@std@@V?$allocator@D@2@@std@@PEAVCIniSection@CIniReader@@U?$less@V?$basic_string@DU?$char_traits@D@std@@V?$allocator@D@2@@std@@@2@V?$allocator@U?$pair@$$CBV?$basic_string@DU?$char_traits@D@std@@V?$allocator@D@2@@std@@PEAVCIniSection@CIniReader@@@std@@@2@$0A@@std@@@std@@QEAA?AV?$_Tree_iterator@V?$_Tree_val@U?$_Tree_simple_types@U?$pair@$$CBV?$basic_string@DU?$char_traits@D@std@@V?$allocator@D@2@@std@@PEAVCIniSection@CIniReader@@@std@@@std@@@std@@@2@V?$_Tree_const_iterator@V?$_Tree_val@U?$_Tree_simple_types@U?$pair@$$CBV?$basic_string@DU?$char_traits@D@std@@V?$allocator@D@2@@std@@PEAVCIniSection@CIniReader@@@std@@@std@@@std@@@2@0@Z 0000000140035010 f i iniReader.obj
 0001:000341c0       ?erase@?$_Tree@V?$_Tmap_traits@V?$basic_string@DU?$char_traits@D@std@@V?$allocator@D@2@@std@@V12@U?$less@V?$basic_string@DU?$char_traits@D@std@@V?$allocator@D@2@@std@@@2@V?$allocator@U?$pair@$$CBV?$basic_string@DU?$char_traits@D@std@@V?$allocator@D@2@@std@@V12@@std@@@2@$0A@@std@@@std@@QEAA?AV?$_Tree_iterator@V?$_Tree_val@U?$_Tree_simple_types@U?$pair@$$CBV?$basic_string@DU?$char_traits@D@std@@V?$allocator@D@2@@std@@V12@@std@@@std@@@std@@@2@V?$_Tree_const_iterator@V?$_Tree_val@U?$_Tree_simple_types@U?$pair@$$CBV?$basic_string@DU?$char_traits@D@std@@V?$allocator@D@2@@std@@V12@@std@@@std@@@std@@@2@0@Z 00000001400351c0 f i iniReader.obj
 0001:00034360       ?_Extract@?$_Tree_val@U?$_Tree_simple_types@U?$pair@$$CB_JV?$basic_string@DU?$char_traits@D@std@@V?$allocator@D@2@@std@@@std@@@std@@@std@@QEAAPEAU?$_Tree_node@U?$pair@$$CB_JV?$basic_string@DU?$char_traits@D@std@@V?$allocator@D@2@@std@@@std@@PEAX@2@V?$_Tree_const_iterator@V?$_Tree_val@U?$_Tree_simple_types@U?$pair@$$CB_JV?$basic_string@DU?$char_traits@D@std@@V?$allocator@D@2@@std@@@std@@@std@@@std@@@2@@Z 0000000140035360 f i LoadXlsMsg.obj
 0001:00034360       ?_Extract@?$_Tree_val@U?$_Tree_simple_types@U?$pair@$$CBV?$basic_string@DU?$char_traits@D@std@@V?$allocator@D@2@@std@@V12@@std@@@std@@@std@@QEAAPEAU?$_Tree_node@U?$pair@$$CBV?$basic_string@DU?$char_traits@D@std@@V?$allocator@D@2@@std@@V12@@std@@PEAX@2@V?$_Tree_const_iterator@V?$_Tree_val@U?$_Tree_simple_types@U?$pair@$$CBV?$basic_string@DU?$char_traits@D@std@@V?$allocator@D@2@@std@@V12@@std@@@std@@@std@@@2@@Z 0000000140035360 f i iniReader.obj
 0001:00034360       ?_Extract@?$_Tree_val@U?$_Tree_simple_types@U?$pair@$$CBV?$basic_string@DU?$char_traits@D@std@@V?$allocator@D@2@@std@@PEAVCIniSection@CIniReader@@@std@@@std@@@std@@QEAAPEAU?$_Tree_node@U?$pair@$$CBV?$basic_string@DU?$char_traits@D@std@@V?$allocator@D@2@@std@@PEAVCIniSection@CIniReader@@@std@@PEAX@2@V?$_Tree_const_iterator@V?$_Tree_val@U?$_Tree_simple_types@U?$pair@$$CBV?$basic_string@DU?$char_traits@D@std@@V?$allocator@D@2@@std@@PEAVCIniSection@CIniReader@@@std@@@std@@@std@@@2@@Z 0000000140035360 f i iniReader.obj
 0001:000347f0       ?_Buyheadnode@?$_Tree_comp_alloc@V?$_Tmap_traits@V?$basic_string@DU?$char_traits@D@std@@V?$allocator@D@2@@std@@PEAVCIniSection@CIniReader@@U?$less@V?$basic_string@DU?$char_traits@D@std@@V?$allocator@D@2@@std@@@2@V?$allocator@U?$pair@$$CBV?$basic_string@DU?$char_traits@D@std@@V?$allocator@D@2@@std@@PEAVCIniSection@CIniReader@@@std@@@2@$0A@@std@@@std@@QEAAPEAU?$_Tree_node@U?$pair@$$CBV?$basic_string@DU?$char_traits@D@std@@V?$allocator@D@2@@std@@PEAVCIniSection@CIniReader@@@std@@PEAX@2@XZ 00000001400357f0 f i iniReader.obj
 0001:000347f0       ?_Buyheadnode@?$_Tree_comp_alloc@V?$_Tmap_traits@_JV?$basic_string@DU?$char_traits@D@std@@V?$allocator@D@2@@std@@U?$less@_J@2@V?$allocator@U?$pair@$$CB_JV?$basic_string@DU?$char_traits@D@std@@V?$allocator@D@2@@std@@@std@@@2@$0A@@std@@@std@@QEAAPEAU?$_Tree_node@U?$pair@$$CB_JV?$basic_string@DU?$char_traits@D@std@@V?$allocator@D@2@@std@@@std@@PEAX@2@XZ 00000001400357f0 f i LoadXlsMsg.obj
 0001:00034820       ?_Buyheadnode@?$_Tree_comp_alloc@V?$_Tmap_traits@V?$basic_string@DU?$char_traits@D@std@@V?$allocator@D@2@@std@@V12@U?$less@V?$basic_string@DU?$char_traits@D@std@@V?$allocator@D@2@@std@@@2@V?$allocator@U?$pair@$$CBV?$basic_string@DU?$char_traits@D@std@@V?$allocator@D@2@@std@@V12@@std@@@2@$0A@@std@@@std@@QEAAPEAU?$_Tree_node@U?$pair@$$CBV?$basic_string@DU?$char_traits@D@std@@V?$allocator@D@2@@std@@V12@@std@@PEAX@2@XZ 0000000140035820 f i iniReader.obj
 0001:00034850       ?_Erase@?$_Tree@V?$_Tmap_traits@V?$basic_string@DU?$char_traits@D@std@@V?$allocator@D@2@@std@@V12@U?$less@V?$basic_string@DU?$char_traits@D@std@@V?$allocator@D@2@@std@@@2@V?$allocator@U?$pair@$$CBV?$basic_string@DU?$char_traits@D@std@@V?$allocator@D@2@@std@@V12@@std@@@2@$0A@@std@@@std@@IEAAXPEAU?$_Tree_node@U?$pair@$$CBV?$basic_string@DU?$char_traits@D@std@@V?$allocator@D@2@@std@@V12@@std@@PEAX@2@@Z 0000000140035850 f i iniReader.obj
 0001:000348b0       ??$?HDU?$char_traits@D@std@@V?$allocator@D@1@@std@@YA?AV?$basic_string@DU?$char_traits@D@std@@V?$allocator@D@2@@0@$$QEAV10@QEBD@Z 00000001400358b0 f i iniReader.obj
 0001:00034910       ??1?$pair@$$CBV?$basic_string@DU?$char_traits@D@std@@V?$allocator@D@2@@std@@V12@@std@@QEAA@XZ 0000000140035910 f i iniReader.obj
 0001:00034910       ??1Address@mailer@jwsmtp@@QEAA@XZ 0000000140035910 f i mailer.obj
 0001:000349c0       ??$_Buynode@U?$pair@PEADPEAVCIniSection@CIniReader@@@std@@@?$_Tree_comp_alloc@V?$_Tmap_traits@V?$basic_string@DU?$char_traits@D@std@@V?$allocator@D@2@@std@@PEAVCIniSection@CIniReader@@U?$less@V?$basic_string@DU?$char_traits@D@std@@V?$allocator@D@2@@std@@@2@V?$allocator@U?$pair@$$CBV?$basic_string@DU?$char_traits@D@std@@V?$allocator@D@2@@std@@PEAVCIniSection@CIniReader@@@std@@@2@$0A@@std@@@std@@QEAAPEAU?$_Tree_node@U?$pair@$$CBV?$basic_string@DU?$char_traits@D@std@@V?$allocator@D@2@@std@@PEAVCIniSection@CIniReader@@@std@@PEAX@1@$$QEAU?$pair@PEADPEAVCIniSection@CIniReader@@@1@@Z 00000001400359c0 f i iniReader.obj
 0001:00034a40       ??$_Insert_nohint@AEAU?$pair@$$CBV?$basic_string@DU?$char_traits@D@std@@V?$allocator@D@2@@std@@PEAVCIniSection@CIniReader@@@std@@PEAU?$_Tree_node@U?$pair@$$CBV?$basic_string@DU?$char_traits@D@std@@V?$allocator@D@2@@std@@PEAVCIniSection@CIniReader@@@std@@PEAX@2@@?$_Tree@V?$_Tmap_traits@V?$basic_string@DU?$char_traits@D@std@@V?$allocator@D@2@@std@@PEAVCIniSection@CIniReader@@U?$less@V?$basic_string@DU?$char_traits@D@std@@V?$allocator@D@2@@std@@@2@V?$allocator@U?$pair@$$CBV?$basic_string@DU?$char_traits@D@std@@V?$allocator@D@2@@std@@PEAVCIniSection@CIniReader@@@std@@@2@$0A@@std@@@std@@IEAA?AU?$pair@V?$_Tree_iterator@V?$_Tree_val@U?$_Tree_simple_types@U?$pair@$$CBV?$basic_string@DU?$char_traits@D@std@@V?$allocator@D@2@@std@@PEAVCIniSection@CIniReader@@@std@@@std@@@std@@@std@@_N@1@_NAEAU?$pair@$$CBV?$basic_string@DU?$char_traits@D@std@@V?$allocator@D@2@@std@@PEAVCIniSection@CIniReader@@@1@PEAU?$_Tree_node@U?$pair@$$CBV?$basic_string@DU?$char_traits@D@std@@V?$allocator@D@2@@std@@PEAVCIniSection@CIniReader@@@std@@PEAX@1@@Z 0000000140035a40 f i iniReader.obj
 0001:00034c70       ?_Freenode0@?$_Tree_comp_alloc@V?$_Tmap_traits@V?$basic_string@DU?$char_traits@D@std@@V?$allocator@D@2@@std@@PEAVCIniSection@CIniReader@@U?$less@V?$basic_string@DU?$char_traits@D@std@@V?$allocator@D@2@@std@@@2@V?$allocator@U?$pair@$$CBV?$basic_string@DU?$char_traits@D@std@@V?$allocator@D@2@@std@@PEAVCIniSection@CIniReader@@@std@@@2@$0A@@std@@@std@@QEAAXPEAU?$_Tree_node@U?$pair@$$CBV?$basic_string@DU?$char_traits@D@std@@V?$allocator@D@2@@std@@PEAVCIniSection@CIniReader@@@std@@PEAX@2@@Z 0000000140035c70 f i iniReader.obj
 0001:00034c80       ?_Buynode0@?$_Tree_comp_alloc@V?$_Tmap_traits@_JV?$basic_string@DU?$char_traits@D@std@@V?$allocator@D@2@@std@@U?$less@_J@2@V?$allocator@U?$pair@$$CB_JV?$basic_string@DU?$char_traits@D@std@@V?$allocator@D@2@@std@@@std@@@2@$0A@@std@@@std@@QEAAPEAU?$_Tree_node@U?$pair@$$CB_JV?$basic_string@DU?$char_traits@D@std@@V?$allocator@D@2@@std@@@std@@PEAX@2@XZ 0000000140035c80 f i LoadXlsMsg.obj
 0001:00034c80       ?_Buynode0@?$_Tree_comp_alloc@V?$_Tmap_traits@V?$basic_string@DU?$char_traits@D@std@@V?$allocator@D@2@@std@@PEAVCIniSection@CIniReader@@U?$less@V?$basic_string@DU?$char_traits@D@std@@V?$allocator@D@2@@std@@@2@V?$allocator@U?$pair@$$CBV?$basic_string@DU?$char_traits@D@std@@V?$allocator@D@2@@std@@PEAVCIniSection@CIniReader@@@std@@@2@$0A@@std@@@std@@QEAAPEAU?$_Tree_node@U?$pair@$$CBV?$basic_string@DU?$char_traits@D@std@@V?$allocator@D@2@@std@@PEAVCIniSection@CIniReader@@@std@@PEAX@2@XZ 0000000140035c80 f i iniReader.obj
 0001:00034cb0       ?_Destroy_if_node@?$_Tree@V?$_Tmap_traits@V?$basic_string@DU?$char_traits@D@std@@V?$allocator@D@2@@std@@PEAVCIniSection@CIniReader@@U?$less@V?$basic_string@DU?$char_traits@D@std@@V?$allocator@D@2@@std@@@2@V?$allocator@U?$pair@$$CBV?$basic_string@DU?$char_traits@D@std@@V?$allocator@D@2@@std@@PEAVCIniSection@CIniReader@@@std@@@2@$0A@@std@@@std@@IEAAXPEAU?$_Tree_node@U?$pair@$$CBV?$basic_string@DU?$char_traits@D@std@@V?$allocator@D@2@@std@@PEAVCIniSection@CIniReader@@@std@@PEAX@2@@Z 0000000140035cb0 f i iniReader.obj
 0001:00034d20       ??$_Insert_at@AEAU?$pair@$$CBV?$basic_string@DU?$char_traits@D@std@@V?$allocator@D@2@@std@@PEAVCIniSection@CIniReader@@@std@@PEAU?$_Tree_node@U?$pair@$$CBV?$basic_string@DU?$char_traits@D@std@@V?$allocator@D@2@@std@@PEAVCIniSection@CIniReader@@@std@@PEAX@2@@?$_Tree@V?$_Tmap_traits@V?$basic_string@DU?$char_traits@D@std@@V?$allocator@D@2@@std@@PEAVCIniSection@CIniReader@@U?$less@V?$basic_string@DU?$char_traits@D@std@@V?$allocator@D@2@@std@@@2@V?$allocator@U?$pair@$$CBV?$basic_string@DU?$char_traits@D@std@@V?$allocator@D@2@@std@@PEAVCIniSection@CIniReader@@@std@@@2@$0A@@std@@@std@@IEAA?AV?$_Tree_iterator@V?$_Tree_val@U?$_Tree_simple_types@U?$pair@$$CBV?$basic_string@DU?$char_traits@D@std@@V?$allocator@D@2@@std@@PEAVCIniSection@CIniReader@@@std@@@std@@@std@@@1@_NPEAU?$_Tree_node@U?$pair@$$CBV?$basic_string@DU?$char_traits@D@std@@V?$allocator@D@2@@std@@PEAVCIniSection@CIniReader@@@std@@PEAX@1@AEAU?$pair@$$CBV?$basic_string@DU?$char_traits@D@std@@V?$allocator@D@2@@std@@PEAVCIniSection@CIniReader@@@1@1@Z 0000000140035d20 f i iniReader.obj
 0001:00034fd0       ??$_Buynode@AEBUpiecewise_construct_t@std@@V?$tuple@$$QEAV?$basic_string@DU?$char_traits@D@std@@V?$allocator@D@2@@std@@@2@V?$tuple@$$V@2@@?$_Tree_comp_alloc@V?$_Tmap_traits@V?$basic_string@DU?$char_traits@D@std@@V?$allocator@D@2@@std@@V12@U?$less@V?$basic_string@DU?$char_traits@D@std@@V?$allocator@D@2@@std@@@2@V?$allocator@U?$pair@$$CBV?$basic_string@DU?$char_traits@D@std@@V?$allocator@D@2@@std@@V12@@std@@@2@$0A@@std@@@std@@QEAAPEAU?$_Tree_node@U?$pair@$$CBV?$basic_string@DU?$char_traits@D@std@@V?$allocator@D@2@@std@@V12@@std@@PEAX@1@AEBUpiecewise_construct_t@1@$$QEAV?$tuple@$$QEAV?$basic_string@DU?$char_traits@D@std@@V?$allocator@D@2@@std@@@1@$$QEAV?$tuple@$$V@1@@Z 0000000140035fd0 f i iniReader.obj
 0001:00035030       ??$_Insert_hint@AEAU?$pair@$$CBV?$basic_string@DU?$char_traits@D@std@@V?$allocator@D@2@@std@@V12@@std@@PEAU?$_Tree_node@U?$pair@$$CBV?$basic_string@DU?$char_traits@D@std@@V?$allocator@D@2@@std@@V12@@std@@PEAX@2@@?$_Tree@V?$_Tmap_traits@V?$basic_string@DU?$char_traits@D@std@@V?$allocator@D@2@@std@@V12@U?$less@V?$basic_string@DU?$char_traits@D@std@@V?$allocator@D@2@@std@@@2@V?$allocator@U?$pair@$$CBV?$basic_string@DU?$char_traits@D@std@@V?$allocator@D@2@@std@@V12@@std@@@2@$0A@@std@@@std@@IEAA?AV?$_Tree_iterator@V?$_Tree_val@U?$_Tree_simple_types@U?$pair@$$CBV?$basic_string@DU?$char_traits@D@std@@V?$allocator@D@2@@std@@V12@@std@@@std@@@std@@@1@V?$_Tree_const_iterator@V?$_Tree_val@U?$_Tree_simple_types@U?$pair@$$CBV?$basic_string@DU?$char_traits@D@std@@V?$allocator@D@2@@std@@V12@@std@@@std@@@std@@@1@AEAU?$pair@$$CBV?$basic_string@DU?$char_traits@D@std@@V?$allocator@D@2@@std@@V12@@1@PEAU?$_Tree_node@U?$pair@$$CBV?$basic_string@DU?$char_traits@D@std@@V?$allocator@D@2@@std@@V12@@std@@PEAX@1@@Z 0000000140036030 f i iniReader.obj
 0001:000354a0       ?_Buynode0@?$_Tree_comp_alloc@V?$_Tmap_traits@V?$basic_string@DU?$char_traits@D@std@@V?$allocator@D@2@@std@@V12@U?$less@V?$basic_string@DU?$char_traits@D@std@@V?$allocator@D@2@@std@@@2@V?$allocator@U?$pair@$$CBV?$basic_string@DU?$char_traits@D@std@@V?$allocator@D@2@@std@@V12@@std@@@2@$0A@@std@@@std@@QEAAPEAU?$_Tree_node@U?$pair@$$CBV?$basic_string@DU?$char_traits@D@std@@V?$allocator@D@2@@std@@V12@@std@@PEAX@2@XZ 00000001400364a0 f i iniReader.obj
 0001:000354d0       ?_Destroy_if_node@?$_Tree@V?$_Tmap_traits@V?$basic_string@DU?$char_traits@D@std@@V?$allocator@D@2@@std@@V12@U?$less@V?$basic_string@DU?$char_traits@D@std@@V?$allocator@D@2@@std@@@2@V?$allocator@U?$pair@$$CBV?$basic_string@DU?$char_traits@D@std@@V?$allocator@D@2@@std@@V12@@std@@@2@$0A@@std@@@std@@IEAAXPEAU?$_Tree_node@U?$pair@$$CBV?$basic_string@DU?$char_traits@D@std@@V?$allocator@D@2@@std@@V12@@std@@PEAX@2@@Z 00000001400364d0 f i iniReader.obj
 0001:00035500       ??$_Insert_at@AEAU?$pair@$$CBV?$basic_string@DU?$char_traits@D@std@@V?$allocator@D@2@@std@@V12@@std@@PEAU?$_Tree_node@U?$pair@$$CBV?$basic_string@DU?$char_traits@D@std@@V?$allocator@D@2@@std@@V12@@std@@PEAX@2@@?$_Tree@V?$_Tmap_traits@V?$basic_string@DU?$char_traits@D@std@@V?$allocator@D@2@@std@@V12@U?$less@V?$basic_string@DU?$char_traits@D@std@@V?$allocator@D@2@@std@@@2@V?$allocator@U?$pair@$$CBV?$basic_string@DU?$char_traits@D@std@@V?$allocator@D@2@@std@@V12@@std@@@2@$0A@@std@@@std@@IEAA?AV?$_Tree_iterator@V?$_Tree_val@U?$_Tree_simple_types@U?$pair@$$CBV?$basic_string@DU?$char_traits@D@std@@V?$allocator@D@2@@std@@V12@@std@@@std@@@std@@@1@_NPEAU?$_Tree_node@U?$pair@$$CBV?$basic_string@DU?$char_traits@D@std@@V?$allocator@D@2@@std@@V12@@std@@PEAX@1@AEAU?$pair@$$CBV?$basic_string@DU?$char_traits@D@std@@V?$allocator@D@2@@std@@V12@@1@1@Z 0000000140036500 f i iniReader.obj
 0001:000357b0       ??$_Insert_nohint@AEAU?$pair@$$CBV?$basic_string@DU?$char_traits@D@std@@V?$allocator@D@2@@std@@V12@@std@@PEAU?$_Tree_node@U?$pair@$$CBV?$basic_string@DU?$char_traits@D@std@@V?$allocator@D@2@@std@@V12@@std@@PEAX@2@@?$_Tree@V?$_Tmap_traits@V?$basic_string@DU?$char_traits@D@std@@V?$allocator@D@2@@std@@V12@U?$less@V?$basic_string@DU?$char_traits@D@std@@V?$allocator@D@2@@std@@@2@V?$allocator@U?$pair@$$CBV?$basic_string@DU?$char_traits@D@std@@V?$allocator@D@2@@std@@V12@@std@@@2@$0A@@std@@@std@@IEAA?AU?$pair@V?$_Tree_iterator@V?$_Tree_val@U?$_Tree_simple_types@U?$pair@$$CBV?$basic_string@DU?$char_traits@D@std@@V?$allocator@D@2@@std@@V12@@std@@@std@@@std@@@std@@_N@1@_NAEAU?$pair@$$CBV?$basic_string@DU?$char_traits@D@std@@V?$allocator@D@2@@std@@V12@@1@PEAU?$_Tree_node@U?$pair@$$CBV?$basic_string@DU?$char_traits@D@std@@V?$allocator@D@2@@std@@V12@@std@@PEAX@1@@Z 00000001400367b0 f i iniReader.obj
 0001:000359f0       ?auth_NTLM@mailer@jwsmtp@@AEAA_NAEBV?$basic_string@DU?$char_traits@D@std@@V?$allocator@D@2@@std@@AEB_K@Z 00000001400369f0 f   auth.obj
 0001:00036290       ?Send@jwsmtp@@YA_NAEAH_KPEBD1H@Z 0000000140037290 f   compat.obj
 0001:000362e0       ?Recv@jwsmtp@@YA_NAEAH_KPEAD1H@Z 00000001400372e0 f   compat.obj
 0001:00036350       ?initNetworking@jwsmtp@@YAXXZ 0000000140037350 f   compat.obj
 0001:00036400       ??0mailer@jwsmtp@@QEAA@PEBD0000G_N@Z 0000000140037400 f   mailer.obj
 0001:000368b0       ??1mailer@jwsmtp@@QEAA@XZ  00000001400378b0 f   mailer.obj
 0001:00036d90       ?checkRFCcompat@mailer@jwsmtp@@AEAAXXZ 0000000140037d90 f   mailer.obj
 0001:00037260       ?setsender@mailer@jwsmtp@@QEAA_NAEBV?$basic_string@DU?$char_traits@D@std@@V?$allocator@D@2@@std@@@Z 0000000140038260 f   mailer.obj
 0001:00037390       ?addrecipient@mailer@jwsmtp@@QEAA_NAEBV?$basic_string@DU?$char_traits@D@std@@V?$allocator@D@2@@std@@F@Z 0000000140038390 f   mailer.obj
 0001:00037630       ??1?$pair@UAddress@mailer@jwsmtp@@F@std@@QEAA@XZ 0000000140038630 f i mailer.obj
 0001:00037640       ??Rmailer@jwsmtp@@QEAAXXZ  0000000140038640 f   mailer.obj
 0001:00039390       ?makesmtpmessage@mailer@jwsmtp@@AEBA?AV?$vector@DV?$allocator@D@std@@@std@@XZ 000000014003a390 f   mailer.obj
 0001:0003aa30       ??1?$pair@V?$vector@DV?$allocator@D@std@@@std@@V?$basic_string@DU?$char_traits@D@std@@V?$allocator@D@2@@2@@std@@QEAA@XZ 000000014003ba30 f i mailer.obj
 0001:0003aae0       ?gethostaddresses@mailer@jwsmtp@@AEAA_NAEAV?$vector@USOCKADDR_IN@jwsmtp@@V?$allocator@USOCKADDR_IN@jwsmtp@@@std@@@std@@@Z 000000014003bae0 f   mailer.obj
 0001:0003b810       ?parsename@mailer@jwsmtp@@AEAAXAEAHQEBEAEAV?$basic_string@DU?$char_traits@D@std@@V?$allocator@D@2@@std@@@Z 000000014003c810 f   mailer.obj
 0001:0003b930       ?parseaddress@mailer@jwsmtp@@AEAA?AUAddress@12@AEBV?$basic_string@DU?$char_traits@D@std@@V?$allocator@D@2@@std@@@Z 000000014003c930 f   mailer.obj
 0001:0003bdf0       ?authenticate@mailer@jwsmtp@@AEAA_NAEBV?$basic_string@DU?$char_traits@D@std@@V?$allocator@D@2@@std@@AEB_K@Z 000000014003cdf0 f   mailer.obj
 0001:0003cd30       ??1?$vector@U?$pair@UAddress@mailer@jwsmtp@@F@std@@V?$allocator@U?$pair@UAddress@mailer@jwsmtp@@F@std@@@2@@std@@QEAA@XZ 000000014003dd30 f i mailer.obj
 0001:0003cdf0       ?size@?$vector@U?$pair@V?$vector@DV?$allocator@D@std@@@std@@V?$basic_string@DU?$char_traits@D@std@@V?$allocator@D@2@@2@@std@@V?$allocator@U?$pair@V?$vector@DV?$allocator@D@std@@@std@@V?$basic_string@DU?$char_traits@D@std@@V?$allocator@D@2@@2@@std@@@2@@std@@QEBA_KXZ 000000014003ddf0 f i mailer.obj
 0001:0003ce20       ??1?$vector@U?$pair@V?$vector@DV?$allocator@D@std@@@std@@V?$basic_string@DU?$char_traits@D@std@@V?$allocator@D@2@@2@@std@@V?$allocator@U?$pair@V?$vector@DV?$allocator@D@std@@@std@@V?$basic_string@DU?$char_traits@D@std@@V?$allocator@D@2@@2@@std@@@2@@std@@QEAA@XZ 000000014003de20 f i mailer.obj
 0001:0003ced0       ??1?$vector@USOCKADDR_IN@jwsmtp@@V?$allocator@USOCKADDR_IN@jwsmtp@@@std@@@std@@QEAA@XZ 000000014003ded0 f i mailer.obj
 0001:0003ced0       ?_Tidy@?$vector@USOCKADDR_IN@jwsmtp@@V?$allocator@USOCKADDR_IN@jwsmtp@@@std@@@std@@AEAAXXZ 000000014003ded0 f i mailer.obj
 0001:0003cf50       ?_Tidy@?$vector@DV?$allocator@D@std@@@std@@AEAAXXZ 000000014003df50 f i mailer.obj
 0001:0003cf50       ??1?$vector@DV?$allocator@D@std@@@std@@QEAA@XZ 000000014003df50 f i mailer.obj
 0001:0003cfb0       ?end@?$basic_string@DU?$char_traits@D@std@@V?$allocator@D@2@@std@@QEAA?AV?$_String_iterator@V?$_String_val@U?$_Simple_types@D@std@@@std@@@2@XZ 000000014003dfb0 f i mailer.obj
 0001:0003cfd0       ?begin@?$basic_string@DU?$char_traits@D@std@@V?$allocator@D@2@@std@@QEAA?AV?$_String_iterator@V?$_String_val@U?$_Simple_types@D@std@@@std@@@2@XZ 000000014003dfd0 f i mailer.obj
 0001:0003cff0       ??$?HDU?$char_traits@D@std@@V?$allocator@D@1@@std@@YA?AV?$basic_string@DU?$char_traits@D@std@@V?$allocator@D@2@@0@$$QEAV10@0@Z 000000014003dff0 f i mailer.obj
 0001:0003d170       ??$?9DU?$char_traits@D@std@@V?$allocator@D@1@@std@@YA_NAEBV?$basic_string@DU?$char_traits@D@std@@V?$allocator@D@2@@0@0@Z 000000014003e170 f i mailer.obj
 0001:0003d1c0       ??$?9DU?$char_traits@D@std@@V?$allocator@D@1@@std@@YA_NAEBV?$basic_string@DU?$char_traits@D@std@@V?$allocator@D@2@@0@QEBD@Z 000000014003e1c0 f i mailer.obj
 0001:0003d210       ??$insert@V?$_String_iterator@V?$_String_val@U?$_Simple_types@D@std@@@std@@@std@@X@?$vector@DV?$allocator@D@std@@@std@@QEAA?AV?$_Vector_iterator@V?$_Vector_val@U?$_Simple_types@D@std@@@std@@@1@V?$_Vector_const_iterator@V?$_Vector_val@U?$_Simple_types@D@std@@@std@@@1@V?$_String_iterator@V?$_String_val@U?$_Simple_types@D@std@@@std@@@1@1@Z 000000014003e210 f i mailer.obj
 0001:0003d210       ??$insert@V?$_Vector_const_iterator@V?$_Vector_val@U?$_Simple_types@D@std@@@std@@@std@@X@?$vector@DV?$allocator@D@std@@@std@@QEAA?AV?$_Vector_iterator@V?$_Vector_val@U?$_Simple_types@D@std@@@std@@@1@V?$_Vector_const_iterator@V?$_Vector_val@U?$_Simple_types@D@std@@@std@@@1@00@Z 000000014003e210 f i mailer.obj
 0001:0003d260       ??$_Emplace_reallocate@AEBV?$basic_string@DU?$char_traits@D@std@@V?$allocator@D@2@@std@@@?$vector@V?$basic_string@DU?$char_traits@D@std@@V?$allocator@D@2@@std@@V?$allocator@V?$basic_string@DU?$char_traits@D@std@@V?$allocator@D@2@@std@@@2@@std@@QEAAPEAV?$basic_string@DU?$char_traits@D@std@@V?$allocator@D@2@@1@QEAV21@AEBV21@@Z 000000014003e260 f i mailer.obj
 0001:0003d570       ??$_Emplace_reallocate@U?$pair@UAddress@mailer@jwsmtp@@F@std@@@?$vector@U?$pair@UAddress@mailer@jwsmtp@@F@std@@V?$allocator@U?$pair@UAddress@mailer@jwsmtp@@F@std@@@2@@std@@QEAAPEAU?$pair@UAddress@mailer@jwsmtp@@F@1@QEAU21@$$QEAU21@@Z 000000014003e570 f i mailer.obj
 0001:0003d800       ??$_Emplace_reallocate@AEBUSOCKADDR_IN@jwsmtp@@@?$vector@USOCKADDR_IN@jwsmtp@@V?$allocator@USOCKADDR_IN@jwsmtp@@@std@@@std@@QEAAPEAUSOCKADDR_IN@jwsmtp@@QEAU23@AEBU23@@Z 000000014003e800 f i mailer.obj
 0001:0003da80       ??$_Emplace_reallocate@AEBD@?$vector@DV?$allocator@D@std@@@std@@QEAAPEADQEADAEBD@Z 000000014003ea80 f i mailer.obj
 0001:0003da80       ??$_Emplace_reallocate@D@?$vector@DV?$allocator@D@std@@@std@@QEAAPEADQEAD$$QEAD@Z 000000014003ea80 f i mailer.obj
 0001:0003dbc0       ?_Change_array@?$vector@DV?$allocator@D@std@@@std@@AEAAXQEAD_K1@Z 000000014003ebc0 f i mailer.obj
 0001:0003dc50       ?_Equal@?$basic_string@DU?$char_traits@D@std@@V?$allocator@D@2@@std@@QEBA_NQEBD@Z 000000014003ec50 f i mailer.obj
 0001:0003dca0       ??$_Insert_range@PEBD@?$vector@DV?$allocator@D@std@@@std@@AEAAXV?$_Vector_const_iterator@V?$_Vector_val@U?$_Simple_types@D@std@@@std@@@1@PEBD1Uforward_iterator_tag@1@@Z 000000014003eca0 f i mailer.obj
 0001:0003dca0       ??$_Insert_range@PEAD@?$vector@DV?$allocator@D@std@@@std@@AEAAXV?$_Vector_const_iterator@V?$_Vector_val@U?$_Simple_types@D@std@@@std@@@1@PEAD1Uforward_iterator_tag@1@@Z 000000014003eca0 f i mailer.obj
 0001:0003de90       ??$_Uninitialized_move@PEAU?$pair@UAddress@mailer@jwsmtp@@F@std@@PEAU12@V?$allocator@U?$pair@UAddress@mailer@jwsmtp@@F@std@@@2@@std@@YAPEAU?$pair@UAddress@mailer@jwsmtp@@F@0@QEAU10@0PEAU10@AEAV?$allocator@U?$pair@UAddress@mailer@jwsmtp@@F@std@@@0@@Z 000000014003ee90 f i mailer.obj
 0001:0003df30       ??$_Reallocate_grow_by@V<lambda_f3a66ab6a0570788f31503db83886f49>@@_KPEBD_K@?$basic_string@DU?$char_traits@D@std@@V?$allocator@D@2@@std@@QEAAAEAV01@_KV<lambda_f3a66ab6a0570788f31503db83886f49>@@_KPEBD2@Z 000000014003ef30 f i mailer.obj
 0001:0003e090       ?_Eos@?$basic_string@DU?$char_traits@D@std@@V?$allocator@D@2@@std@@QEAAX_K@Z 000000014003f090 f i mailer.obj
 0001:0003e7b0       gl_des_ecb_crypt           000000014003f7b0 f   des.obj
 0001:0003f2a0       md4_finish_ctx             00000001400402a0 f   md4.obj
 0001:0003f370       md4_process_bytes          0000000140040370 f   md4.obj
 0001:0003f500       md4_process_block          0000000140040500 f   md4.obj
 0001:0003fda0       buildSmbNtlmAuthResponse   0000000140040da0 f   smbutil.obj
 0001:00040300       ??1md5wrapper@@QEAA@XZ     0000000140041300 f   md5wrapper.obj
 0001:00040310       ?getHashFromFile@md5wrapper@@QEAA?AV?$basic_string@DU?$char_traits@D@std@@V?$allocator@D@2@@std@@V23@@Z 0000000140041310 f   md5wrapper.obj
 0001:00040640       ?_InitPathNameInfo@CHLogger@@CAXPEBD000@Z 0000000140041640 f   HostLogger.obj
 0001:00040b20       ?Log@CHLogger@@SAXW4ELOG_LEVEL@1@PEBDZZ 0000000140041b20 f   HostLogger.obj
 0001:00040b70       ?LogTimeOut@CHLogger@@SAXPEBDZZ 0000000140041b70 f   HostLogger.obj
 0001:00040d80       ?LogPacket@CHLogger@@SAXPEBDZZ 0000000140041d80 f   HostLogger.obj
 0001:00040fa0       ?LogModeUserCount@CHLogger@@SAXPEBDZZ 0000000140041fa0 f   HostLogger.obj
 0001:00041150       ?LogServerAppUseCount@CHLogger@@SAXPEBDZZ 0000000140042150 f   HostLogger.obj
 0001:000412d0       ?LogRWProcessMemory@CHLogger@@SAXPEBDZZ 00000001400422d0 f   HostLogger.obj
 0001:000414a0       ?LogIPCMessage@CHLogger@@SAXPEBDZZ 00000001400424a0 f   HostLogger.obj
 0001:00041670       ?_BuildDirectory@CHLogger@@CAXAEBU_SYSTEMTIME@@@Z 0000000140042670 f   HostLogger.obj
 0001:00041ab0       ?_DoLogWithLevel@CHLogger@@CAXPEBDW4ELOG_LEVEL@1@0PEAD@Z 0000000140042ab0 f   HostLogger.obj
 0001:00041cb0       ??1CSynchronizedLog@@QEAA@XZ 0000000140042cb0 f i HostLogger.obj
 0001:00041cd0       ??_GCMustSyncObjectLog@@UEAAPEAXI@Z 0000000140042cd0 f i HostLogger.obj
 0001:00041cd0       ??_ECMustSyncObjectLog@@UEAAPEAXI@Z 0000000140042cd0 f i * CIL library *:* CIL module *
 0001:00041d20       ?Init@CLogMsgManager@@SA_NW4ESHARED_MEM_USAGE_TYPE@1@@Z 0000000140042d20 f   LogMsgManager.obj
 0001:00042030       ?GetString@CLogMsgManager@@SA?BV?$basic_string@DU?$char_traits@D@std@@V?$allocator@D@2@@std@@I@Z 0000000140043030 f   LogMsgManager.obj
 0001:000421d0       ?_WriteXlsDataToSharedMemory@CLogMsgManager@@CA_NXZ 00000001400431d0 f   LogMsgManager.obj
 0001:000424c0       ??$sprintf_s@$0CA@@cf@@YAHAEAY0CA@DPEBDZZ 00000001400434c0 f i LogMsgManager.obj
 0001:00042500       ??$_Emplace_reallocate@AEBQEAX@?$vector@PEAXV?$allocator@PEAX@std@@@std@@QEAAPEAPEAXQEAPEAXAEBQEAX@Z 0000000140043500 f i LogMsgManager.obj
 0001:000426b0       ??0FindXlsMsg@@QEAA@XZ     00000001400436b0 f   LoadXlsMsg.obj
 0001:00042710       ??_GFindXlsMsg@@UEAAPEAXI@Z 0000000140043710 f i LoadXlsMsg.obj
 0001:00042710       ??_EFindXlsMsg@@UEAAPEAXI@Z 0000000140043710 f i * CIL library *:* CIL module *
 0001:00042810       ?LoadWMszFile@FindXlsMsg@@QEAA_NPEAD@Z 0000000140043810 f   LoadXlsMsg.obj
 0001:00042b00       ??A?$map@_JV?$basic_string@DU?$char_traits@D@std@@V?$allocator@D@2@@std@@U?$less@_J@2@V?$allocator@U?$pair@$$CB_JV?$basic_string@DU?$char_traits@D@std@@V?$allocator@D@2@@std@@@std@@@2@@std@@QEAAAEAV?$basic_string@DU?$char_traits@D@std@@V?$allocator@D@2@@1@AEB_J@Z 0000000140043b00 f i LoadXlsMsg.obj
 0001:00042b90       ?_Erase@?$_Tree@V?$_Tmap_traits@_JV?$basic_string@DU?$char_traits@D@std@@V?$allocator@D@2@@std@@U?$less@_J@2@V?$allocator@U?$pair@$$CB_JV?$basic_string@DU?$char_traits@D@std@@V?$allocator@D@2@@std@@@std@@@2@$0A@@std@@@std@@IEAAXPEAU?$_Tree_node@U?$pair@$$CB_JV?$basic_string@DU?$char_traits@D@std@@V?$allocator@D@2@@std@@@std@@PEAX@2@@Z 0000000140043b90 f i LoadXlsMsg.obj
 0001:00042c50       ?erase@?$_Tree@V?$_Tmap_traits@_JV?$basic_string@DU?$char_traits@D@std@@V?$allocator@D@2@@std@@U?$less@_J@2@V?$allocator@U?$pair@$$CB_JV?$basic_string@DU?$char_traits@D@std@@V?$allocator@D@2@@std@@@std@@@2@$0A@@std@@@std@@QEAA?AV?$_Tree_iterator@V?$_Tree_val@U?$_Tree_simple_types@U?$pair@$$CB_JV?$basic_string@DU?$char_traits@D@std@@V?$allocator@D@2@@std@@@std@@@std@@@std@@@2@V?$_Tree_const_iterator@V?$_Tree_val@U?$_Tree_simple_types@U?$pair@$$CB_JV?$basic_string@DU?$char_traits@D@std@@V?$allocator@D@2@@std@@@std@@@std@@@std@@@2@0@Z 0000000140043c50 f i LoadXlsMsg.obj
 0001:00042e00       ??$_Buynode@AEBUpiecewise_construct_t@std@@V?$tuple@AEB_J@2@V?$tuple@$$V@2@@?$_Tree_comp_alloc@V?$_Tmap_traits@_JV?$basic_string@DU?$char_traits@D@std@@V?$allocator@D@2@@std@@U?$less@_J@2@V?$allocator@U?$pair@$$CB_JV?$basic_string@DU?$char_traits@D@std@@V?$allocator@D@2@@std@@@std@@@2@$0A@@std@@@std@@QEAAPEAU?$_Tree_node@U?$pair@$$CB_JV?$basic_string@DU?$char_traits@D@std@@V?$allocator@D@2@@std@@@std@@PEAX@1@AEBUpiecewise_construct_t@1@$$QEAV?$tuple@AEB_J@1@$$QEAV?$tuple@$$V@1@@Z 0000000140043e00 f i LoadXlsMsg.obj
 0001:00042e40       ??$_Insert_hint@AEAU?$pair@$$CB_JV?$basic_string@DU?$char_traits@D@std@@V?$allocator@D@2@@std@@@std@@PEAU?$_Tree_node@U?$pair@$$CB_JV?$basic_string@DU?$char_traits@D@std@@V?$allocator@D@2@@std@@@std@@PEAX@2@@?$_Tree@V?$_Tmap_traits@_JV?$basic_string@DU?$char_traits@D@std@@V?$allocator@D@2@@std@@U?$less@_J@2@V?$allocator@U?$pair@$$CB_JV?$basic_string@DU?$char_traits@D@std@@V?$allocator@D@2@@std@@@std@@@2@$0A@@std@@@std@@IEAA?AV?$_Tree_iterator@V?$_Tree_val@U?$_Tree_simple_types@U?$pair@$$CB_JV?$basic_string@DU?$char_traits@D@std@@V?$allocator@D@2@@std@@@std@@@std@@@std@@@1@V?$_Tree_const_iterator@V?$_Tree_val@U?$_Tree_simple_types@U?$pair@$$CB_JV?$basic_string@DU?$char_traits@D@std@@V?$allocator@D@2@@std@@@std@@@std@@@std@@@1@AEAU?$pair@$$CB_JV?$basic_string@DU?$char_traits@D@std@@V?$allocator@D@2@@std@@@1@PEAU?$_Tree_node@U?$pair@$$CB_JV?$basic_string@DU?$char_traits@D@std@@V?$allocator@D@2@@std@@@std@@PEAX@1@@Z 0000000140043e40 f i LoadXlsMsg.obj
 0001:00043090       ?_Destroy_if_node@?$_Tree@V?$_Tmap_traits@_JV?$basic_string@DU?$char_traits@D@std@@V?$allocator@D@2@@std@@U?$less@_J@2@V?$allocator@U?$pair@$$CB_JV?$basic_string@DU?$char_traits@D@std@@V?$allocator@D@2@@std@@@std@@@2@$0A@@std@@@std@@IEAAXPEAU?$_Tree_node@U?$pair@$$CB_JV?$basic_string@DU?$char_traits@D@std@@V?$allocator@D@2@@std@@@std@@PEAX@2@@Z 0000000140044090 f i LoadXlsMsg.obj
 0001:00043100       ??$_Insert_at@AEAU?$pair@$$CB_JV?$basic_string@DU?$char_traits@D@std@@V?$allocator@D@2@@std@@@std@@PEAU?$_Tree_node@U?$pair@$$CB_JV?$basic_string@DU?$char_traits@D@std@@V?$allocator@D@2@@std@@@std@@PEAX@2@@?$_Tree@V?$_Tmap_traits@_JV?$basic_string@DU?$char_traits@D@std@@V?$allocator@D@2@@std@@U?$less@_J@2@V?$allocator@U?$pair@$$CB_JV?$basic_string@DU?$char_traits@D@std@@V?$allocator@D@2@@std@@@std@@@2@$0A@@std@@@std@@IEAA?AV?$_Tree_iterator@V?$_Tree_val@U?$_Tree_simple_types@U?$pair@$$CB_JV?$basic_string@DU?$char_traits@D@std@@V?$allocator@D@2@@std@@@std@@@std@@@std@@@1@_NPEAU?$_Tree_node@U?$pair@$$CB_JV?$basic_string@DU?$char_traits@D@std@@V?$allocator@D@2@@std@@@std@@PEAX@1@AEAU?$pair@$$CB_JV?$basic_string@DU?$char_traits@D@std@@V?$allocator@D@2@@std@@@1@1@Z 0000000140044100 f i LoadXlsMsg.obj
 0001:000433b0       ??$_Insert_nohint@AEAU?$pair@$$CB_JV?$basic_string@DU?$char_traits@D@std@@V?$allocator@D@2@@std@@@std@@PEAU?$_Tree_node@U?$pair@$$CB_JV?$basic_string@DU?$char_traits@D@std@@V?$allocator@D@2@@std@@@std@@PEAX@2@@?$_Tree@V?$_Tmap_traits@_JV?$basic_string@DU?$char_traits@D@std@@V?$allocator@D@2@@std@@U?$less@_J@2@V?$allocator@U?$pair@$$CB_JV?$basic_string@DU?$char_traits@D@std@@V?$allocator@D@2@@std@@@std@@@2@$0A@@std@@@std@@IEAA?AU?$pair@V?$_Tree_iterator@V?$_Tree_val@U?$_Tree_simple_types@U?$pair@$$CB_JV?$basic_string@DU?$char_traits@D@std@@V?$allocator@D@2@@std@@@std@@@std@@@std@@@std@@_N@1@_NAEAU?$pair@$$CB_JV?$basic_string@DU?$char_traits@D@std@@V?$allocator@D@2@@std@@@1@PEAU?$_Tree_node@U?$pair@$$CB_JV?$basic_string@DU?$char_traits@D@std@@V?$allocator@D@2@@std@@@std@@PEAX@1@@Z 00000001400443b0 f i LoadXlsMsg.obj
 0001:00043510       ?_AtlInitializeCriticalSectionEx@ATL@@YAHPEAU_RTL_CRITICAL_SECTION@@KK@Z 0000000140044510 f i StdAfx.obj
 0001:00043520       ?getbase64character@jwsmtp@@YADAEBD@Z 0000000140044520 f   base6409cee8549d9fd00dfa06fdadc87a8424.obj
 0001:00043710       ?base64encode@jwsmtp@@YA?AV?$vector@DV?$allocator@D@std@@@std@@AEBV23@_N@Z 0000000140044710 f   base6409cee8549d9fd00dfa06fdadc87a8424.obj
 0001:00043990       ?base64encode@jwsmtp@@YA?AV?$basic_string@DU?$char_traits@D@std@@V?$allocator@D@2@@std@@AEBV23@_N@Z 0000000140044990 f   base6409cee8549d9fd00dfa06fdadc87a8424.obj
 0001:00043bc0       ?base64encode@jwsmtp@@YAXPEBDHPEAD_N@Z 0000000140044bc0 f   base6409cee8549d9fd00dfa06fdadc87a8424.obj
 0001:00043d90       ?base64decode@jwsmtp@@YAXAEBV?$vector@DV?$allocator@D@std@@@std@@AEAV23@@Z 0000000140044d90 f   base6409cee8549d9fd00dfa06fdadc87a8424.obj
 0001:00043f20       ?MD5Update@MD5@@QEAAXPEAUMD5_CTX@@PEAEI@Z 0000000140044f20 f   md55d7732e46e8b0b019ace15d3c50ded71.obj
 0001:00044030       ?MD5Final@MD5@@QEAAXQEAEPEAUMD5_CTX@@@Z 0000000140045030 f   md55d7732e46e8b0b019ace15d3c50ded71.obj
 0001:00044140       ?MD5Transform@MD5@@AEAAXQEAKQEAE@Z 0000000140045140 f   md55d7732e46e8b0b019ace15d3c50ded71.obj
 0001:00044a10       ?sprintf_s@internal@cf@@YAHPEAD_KPEBDAEAPEAD@Z 0000000140045a10 f   safe_string_x64:safe_string.obj
 0001:00044cf0       ??_D?$basic_stringstream@DU?$char_traits@D@std@@V?$allocator@D@2@@std@@QEAAXXZ 0000000140045cf0 f i safe_string_x64:safe_string.obj
 0001:00044d50       ?strcpy_s@cf@@YAHPEAD_KPEBD@Z 0000000140045d50 f   safe_string_x64:safe_string.obj
 0001:00045000       ?strncpy_s@cf@@YAHPEAD_KPEBD1@Z 0000000140046000 f   safe_string_x64:safe_string.obj
 0001:000452d0       ?sprintf_s@cf@@YAHPEAD_KPEBDZZ 00000001400462d0 f   safe_string_x64:safe_string.obj
 0001:00045300       ??0?$basic_stringstream@DU?$char_traits@D@std@@V?$allocator@D@2@@std@@QEAA@H@Z 0000000140046300 f i safe_string_x64:safe_string.obj
 0001:000453c0       ?seekpos@?$basic_stringbuf@DU?$char_traits@D@std@@V?$allocator@D@2@@std@@MEAA?AV?$fpos@U_Mbstatet@@@2@V32@H@Z 00000001400463c0 f i safe_string_x64:safe_string.obj
 0001:000454b0       ?seekoff@?$basic_stringbuf@DU?$char_traits@D@std@@V?$allocator@D@2@@std@@MEAA?AV?$fpos@U_Mbstatet@@@2@_JHH@Z 00000001400464b0 f i safe_string_x64:safe_string.obj
 0001:00045600       ?underflow@?$basic_stringbuf@DU?$char_traits@D@std@@V?$allocator@D@2@@std@@MEAAHXZ 0000000140046600 f i safe_string_x64:safe_string.obj
 0001:00045670       ?pbackfail@?$basic_stringbuf@DU?$char_traits@D@std@@V?$allocator@D@2@@std@@MEAAHH@Z 0000000140046670 f i safe_string_x64:safe_string.obj
 0001:000456d0       ?overflow@?$basic_stringbuf@DU?$char_traits@D@std@@V?$allocator@D@2@@std@@MEAAHH@Z 00000001400466d0 f i safe_string_x64:safe_string.obj
 0001:000458d0       ??1?$basic_stringbuf@DU?$char_traits@D@std@@V?$allocator@D@2@@std@@UEAA@XZ 00000001400468d0 f i safe_string_x64:safe_string.obj
 0001:00045990       ??_G?$basic_stringstream@DU?$char_traits@D@std@@V?$allocator@D@2@@std@@UEAAPEAXI@Z 0000000140046990 f i safe_string_x64:safe_string.obj
 0001:00045990       ??_E?$basic_stringstream@DU?$char_traits@D@std@@V?$allocator@D@2@@std@@UEAAPEAXI@Z 0000000140046990 f i * CIL library *:* CIL module *
 0001:00045a30       ??_E?$basic_stringbuf@DU?$char_traits@D@std@@V?$allocator@D@2@@std@@UEAAPEAXI@Z 0000000140046a30 f i * CIL library *:* CIL module *
 0001:00045a30       ??_G?$basic_stringbuf@DU?$char_traits@D@std@@V?$allocator@D@2@@std@@UEAAPEAXI@Z 0000000140046a30 f i safe_string_x64:safe_string.obj
 0001:00045a64       ??_E?$basic_stringstream@DU?$char_traits@D@std@@V?$allocator@D@2@@std@@$4PPPPPPPM@A@EAAPEAXI@Z 0000000140046a64 f i safe_string_x64:safe_string.obj
 0001:00045a70       ??3@YAXPEAX@Z              0000000140046a70 f   mfc140:mfc140.dll
 0001:00045a76       ??_V@YAXPEAX@Z             0000000140046a76 f   mfc140:mfc140.dll
 0001:00045a7c       ?GetOccDialogInfo@CWnd@@MEAAPEAU_AFX_OCC_DIALOG_INFO@@XZ 0000000140046a7c f   mfc140:mfc140.dll
 0001:00045a82       ?SetOccDialogInfo@CWnd@@MEAAHPEAU_AFX_OCC_DIALOG_INFO@@@Z 0000000140046a82 f   mfc140:mfc140.dll
 0001:00045a88       ?CreateControlSite@CWnd@@MEAAHPEAVCOleControlContainer@@PEAPEAVCOleControlSite@@IAEBU_GUID@@@Z 0000000140046a88 f   mfc140:mfc140.dll
 0001:00045a8e       ?CreateControlContainer@CWnd@@MEAAHPEAPEAVCOleControlContainer@@@Z 0000000140046a8e f   mfc140:mfc140.dll
 0001:00045a94       ?IsFrameWnd@CWnd@@UEBAHXZ  0000000140046a94 f   mfc140:mfc140.dll
 0001:00045a9a       ?CheckAutoCenter@CWnd@@UEAAHXZ 0000000140046a9a f   mfc140:mfc140.dll
 0001:00045aa0       ?ResizeDynamicLayout@CWnd@@MEAAXXZ 0000000140046aa0 f   mfc140:mfc140.dll
 0001:00045aa6       ?OnGesturePressAndTap@CWnd@@MEAAHVCPoint@@J@Z 0000000140046aa6 f   mfc140:mfc140.dll
 0001:00045aac       ?OnGestureTwoFingerTap@CWnd@@MEAAHVCPoint@@@Z 0000000140046aac f   mfc140:mfc140.dll
 0001:00045ab2       ?OnGestureRotate@CWnd@@MEAAHVCPoint@@N@Z 0000000140046ab2 f   mfc140:mfc140.dll
 0001:00045ab8       ?OnGesturePan@CWnd@@MEAAHVCPoint@@0@Z 0000000140046ab8 f   mfc140:mfc140.dll
 0001:00045abe       ?OnGestureZoom@CWnd@@MEAAHVCPoint@@J@Z 0000000140046abe f   mfc140:mfc140.dll
 0001:00045ac4       ?GetGestureStatus@CWnd@@MEAAKVCPoint@@@Z 0000000140046ac4 f   mfc140:mfc140.dll
 0001:00045aca       ?OnTouchInput@CWnd@@MEAAHVCPoint@@HHPEAUtagTOUCHINPUT@@@Z 0000000140046aca f   mfc140:mfc140.dll
 0001:00045ad0       ?OnTouchInputs@CWnd@@MEAAHIPEAUtagTOUCHINPUT@@@Z 0000000140046ad0 f   mfc140:mfc140.dll
 0001:00045ad6       ?OnChildNotify@CWnd@@MEAAHI_K_JPEA_J@Z 0000000140046ad6 f   mfc140:mfc140.dll
 0001:00045adc       ?PostNcDestroy@CWnd@@MEAAXXZ 0000000140046adc f   mfc140:mfc140.dll
 0001:00045ae2       ?DefWindowProcA@CWnd@@MEAA_JI_K_J@Z 0000000140046ae2 f   mfc140:mfc140.dll
 0001:00045ae8       ?OnWndMsg@CWnd@@MEAAHI_K_JPEA_J@Z 0000000140046ae8 f   mfc140:mfc140.dll
 0001:00045aee       ?WindowProc@CWnd@@MEAA_JI_K_J@Z 0000000140046aee f   mfc140:mfc140.dll
 0001:00045af4       ?OnAmbientProperty@CWnd@@UEAAHPEAVCOleControlSite@@JPEAUtagVARIANT@@@Z 0000000140046af4 f   mfc140:mfc140.dll
 0001:00045afa       ?PreTranslateMessage@CWnd@@UEAAHPEAUtagMSG@@@Z 0000000140046afa f   mfc140:mfc140.dll
 0001:00045b00       ?GetSuperWndProcAddr@CWnd@@MEAAPEAP6A_JPEAUHWND__@@I_K_J@ZXZ 0000000140046b00 f   mfc140:mfc140.dll
 0001:00045b06       ?OnNotify@CWnd@@MEAAH_K_JPEA_J@Z 0000000140046b06 f   mfc140:mfc140.dll
 0001:00045b0c       ?OnCommand@CWnd@@MEAAH_K_J@Z 0000000140046b0c f   mfc140:mfc140.dll
 0001:00045b12       ?CreateAccessibleProxy@CWnd@@UEAAJ_K_JPEA_J@Z 0000000140046b12 f   mfc140:mfc140.dll
 0001:00045b18       ?SetProxy@CWnd@@UEAAJPEAUIAccessibleProxy@@@Z 0000000140046b18 f   mfc140:mfc140.dll
 0001:00045b1e       ?put_accValue@CWnd@@UEAAJUtagVARIANT@@PEA_W@Z 0000000140046b1e f   mfc140:mfc140.dll
 0001:00045b24       ?put_accName@CWnd@@UEAAJUtagVARIANT@@PEA_W@Z 0000000140046b24 f   mfc140:mfc140.dll
 0001:00045b2a       ?accDoDefaultAction@CWnd@@UEAAJUtagVARIANT@@@Z 0000000140046b2a f   mfc140:mfc140.dll
 0001:00045b30       ?accHitTest@CWnd@@UEAAJJJPEAUtagVARIANT@@@Z 0000000140046b30 f   mfc140:mfc140.dll
 0001:00045b36       ?accNavigate@CWnd@@UEAAJJUtagVARIANT@@PEAU2@@Z 0000000140046b36 f   mfc140:mfc140.dll
 0001:00045b3c       ?accLocation@CWnd@@UEAAJPEAJ000UtagVARIANT@@@Z 0000000140046b3c f   mfc140:mfc140.dll
 0001:00045b42       ?accSelect@CWnd@@UEAAJJUtagVARIANT@@@Z 0000000140046b42 f   mfc140:mfc140.dll
 0001:00045b48       ?get_accDefaultAction@CWnd@@UEAAJUtagVARIANT@@PEAPEA_W@Z 0000000140046b48 f   mfc140:mfc140.dll
 0001:00045b4e       ?get_accSelection@CWnd@@UEAAJPEAUtagVARIANT@@@Z 0000000140046b4e f   mfc140:mfc140.dll
 0001:00045b54       ?get_accFocus@CWnd@@UEAAJPEAUtagVARIANT@@@Z 0000000140046b54 f   mfc140:mfc140.dll
 0001:00045b5a       ?get_accKeyboardShortcut@CWnd@@UEAAJUtagVARIANT@@PEAPEA_W@Z 0000000140046b5a f   mfc140:mfc140.dll
 0001:00045b60       ?get_accHelpTopic@CWnd@@UEAAJPEAPEA_WUtagVARIANT@@PEAJ@Z 0000000140046b60 f   mfc140:mfc140.dll
 0001:00045b66       ?get_accHelp@CWnd@@UEAAJUtagVARIANT@@PEAPEA_W@Z 0000000140046b66 f   mfc140:mfc140.dll
 0001:00045b6c       ?get_accState@CWnd@@UEAAJUtagVARIANT@@PEAU2@@Z 0000000140046b6c f   mfc140:mfc140.dll
 0001:00045b72       ?get_accRole@CWnd@@UEAAJUtagVARIANT@@PEAU2@@Z 0000000140046b72 f   mfc140:mfc140.dll
 0001:00045b78       ?get_accDescription@CWnd@@UEAAJUtagVARIANT@@PEAPEA_W@Z 0000000140046b78 f   mfc140:mfc140.dll
 0001:00045b7e       ?get_accValue@CWnd@@UEAAJUtagVARIANT@@PEAPEA_W@Z 0000000140046b7e f   mfc140:mfc140.dll
 0001:00045b84       ?get_accName@CWnd@@UEAAJUtagVARIANT@@PEAPEA_W@Z 0000000140046b84 f   mfc140:mfc140.dll
 0001:00045b8a       ?get_accChild@CWnd@@UEAAJUtagVARIANT@@PEAPEAUIDispatch@@@Z 0000000140046b8a f   mfc140:mfc140.dll
 0001:00045b90       ?get_accChildCount@CWnd@@UEAAJPEAJ@Z 0000000140046b90 f   mfc140:mfc140.dll
 0001:00045b96       ?get_accParent@CWnd@@UEAAJPEAPEAUIDispatch@@@Z 0000000140046b96 f   mfc140:mfc140.dll
 0001:00045b9c       ?EnsureStdObj@CWnd@@UEAAJXZ 0000000140046b9c f   mfc140:mfc140.dll
 0001:00045ba2       ?OnDrawIconicThumbnailOrLivePreview@CWnd@@UEAAXAEAVCDC@@VCRect@@VCSize@@HAEAH@Z 0000000140046ba2 f   mfc140:mfc140.dll
 0001:00045ba8       ?EndModalLoop@CWnd@@UEAAXH@Z 0000000140046ba8 f   mfc140:mfc140.dll
 0001:00045bae       ?ContinueModal@CWnd@@UEAAHXZ 0000000140046bae f   mfc140:mfc140.dll
 0001:00045bb4       ?WinHelpInternal@CWnd@@UEAAX_KI@Z 0000000140046bb4 f   mfc140:mfc140.dll
 0001:00045bba       ?HtmlHelpA@CWnd@@UEAAX_KI@Z 0000000140046bba f   mfc140:mfc140.dll
 0001:00045bc0       ?WinHelpA@CWnd@@UEAAX_KI@Z 0000000140046bc0 f   mfc140:mfc140.dll
 0001:00045bc6       ?GetScrollBarCtrl@CWnd@@UEBAPEAVCScrollBar@@H@Z 0000000140046bc6 f   mfc140:mfc140.dll
 0001:00045bcc       ?OnToolHitTest@CWnd@@UEBA_JVCPoint@@PEAUtagTOOLINFOA@@@Z 0000000140046bcc f   mfc140:mfc140.dll
 0001:00045bd2       ?SetMenu@CWnd@@UEAAHPEAVCMenu@@@Z 0000000140046bd2 f   mfc140:mfc140.dll
 0001:00045bd8       ?GetMenu@CWnd@@UEBAPEAVCMenu@@XZ 0000000140046bd8 f   mfc140:mfc140.dll
 0001:00045bde       ?CalcWindowRect@CWnd@@UEAAXPEAUtagRECT@@I@Z 0000000140046bde f   mfc140:mfc140.dll
 0001:00045be4       ?PreCreateWindow@CWnd@@UEAAHAEAUtagCREATESTRUCTA@@@Z 0000000140046be4 f   mfc140:mfc140.dll
 0001:00045bea       ?DestroyWindow@CWnd@@UEAAHXZ 0000000140046bea f   mfc140:mfc140.dll
 0001:00045bf0       ?CreateEx@CWnd@@UEAAHKPEBD0KHHHHPEAUHWND__@@PEAUHMENU__@@PEAX@Z 0000000140046bf0 f   mfc140:mfc140.dll
 0001:00045bf6       ?CreateEx@CWnd@@UEAAHKPEBD0KAEBUtagRECT@@PEAV1@IPEAX@Z 0000000140046bf6 f   mfc140:mfc140.dll
 0001:00045bfc       ?Create@CWnd@@UEAAHPEBD0KAEBUtagRECT@@PEAV1@IPEAUCCreateContext@@@Z 0000000140046bfc f   mfc140:mfc140.dll
 0001:00045c02       ?PreSubclassWindow@CWnd@@UEAAXXZ 0000000140046c02 f   mfc140:mfc140.dll
 0001:00045c08       ?GetConnectionHook@CCmdTarget@@MEAAPEAUIConnectionPoint@@AEBU_GUID@@@Z 0000000140046c08 f   mfc140:mfc140.dll
 0001:00045c0e       ?GetExtraConnectionPoints@CCmdTarget@@MEAAHPEAVCPtrArray@@@Z 0000000140046c0e f   mfc140:mfc140.dll
 0001:00045c14       ?GetInterfaceHook@CCmdTarget@@UEAAPEAUIUnknown@@PEBX@Z 0000000140046c14 f   mfc140:mfc140.dll
 0001:00045c1a       ?OnCreateAggregates@CCmdTarget@@UEAAHXZ 0000000140046c1a f   mfc140:mfc140.dll
 0001:00045c20       ?GetEventSinkMap@CCmdTarget@@MEBAPEBUAFX_EVENTSINKMAP@@XZ 0000000140046c20 f   mfc140:mfc140.dll
 0001:00045c26       ?GetInterfaceMap@CWnd@@MEBAPEBUAFX_INTERFACEMAP@@XZ 0000000140046c26 f   mfc140:mfc140.dll
 0001:00045c2c       ?GetConnectionMap@CCmdTarget@@MEBAPEBUAFX_CONNECTIONMAP@@XZ 0000000140046c2c f   mfc140:mfc140.dll
 0001:00045c32       ?GetDispatchMap@CCmdTarget@@MEBAPEBUAFX_DISPMAP@@XZ 0000000140046c32 f   mfc140:mfc140.dll
 0001:00045c38       ?GetCommandMap@CCmdTarget@@MEBAPEBUAFX_OLECMDMAP@@XZ 0000000140046c38 f   mfc140:mfc140.dll
 0001:00045c3e       ?GetMessageMap@CWnd@@MEBAPEBUAFX_MSGMAP@@XZ 0000000140046c3e f   mfc140:mfc140.dll
 0001:00045c44       ?GetTypeLib@CCmdTarget@@UEAAJKPEAPEAUITypeLib@@@Z 0000000140046c44 f   mfc140:mfc140.dll
 0001:00045c4a       ?GetTypeLibCache@CCmdTarget@@UEAAPEAVCTypeLibCache@@XZ 0000000140046c4a f   mfc140:mfc140.dll
 0001:00045c50       ?GetTypeInfoCount@CCmdTarget@@UEAAIXZ 0000000140046c50 f   mfc140:mfc140.dll
 0001:00045c56       ?GetDispatchIID@CCmdTarget@@UEAAHPEAU_GUID@@@Z 0000000140046c56 f   mfc140:mfc140.dll
 0001:00045c5c       ?IsInvokeAllowed@CCmdTarget@@UEAAHJ@Z 0000000140046c5c f   mfc140:mfc140.dll
 0001:00045c62       ?OnFinalRelease@CWnd@@UEAAXXZ 0000000140046c62 f   mfc140:mfc140.dll
 0001:00045c68       ?OnCmdMsg@CCmdTarget@@UEAAHIHPEAXPEAUAFX_CMDHANDLERINFO@@@Z 0000000140046c68 f   mfc140:mfc140.dll
 0001:00045c6e       ?GetRuntimeClass@CEdit@@UEBAPEAUCRuntimeClass@@XZ 0000000140046c6e f   mfc140:mfc140.dll
 0001:00045c74       ?GetThisMessageMap@CDialog@@KAPEBUAFX_MSGMAP@@XZ 0000000140046c74 f   mfc140:mfc140.dll
 0001:00045c7a       ?OnCmdMsg@CDialog@@UEAAHIHPEAXPEAUAFX_CMDHANDLERINFO@@@Z 0000000140046c7a f   mfc140:mfc140.dll
 0001:00045c80       ?PreTranslateMessage@CDialog@@UEAAHPEAUtagMSG@@@Z 0000000140046c80 f   mfc140:mfc140.dll
 0001:00045c86       ?CheckAutoCenter@CDialog@@UEAAHXZ 0000000140046c86 f   mfc140:mfc140.dll
 0001:00045c8c       ?SetOccDialogInfo@CDialog@@MEAAHPEAU_AFX_OCC_DIALOG_INFO@@@Z 0000000140046c8c f   mfc140:mfc140.dll
 0001:00045c92       ?GetOccDialogInfo@CDialog@@MEAAPEAU_AFX_OCC_DIALOG_INFO@@XZ 0000000140046c92 f   mfc140:mfc140.dll
 0001:00045c98       ?Create@CDialog@@UEAAHPEBDPEAVCWnd@@@Z 0000000140046c98 f   mfc140:mfc140.dll
 0001:00045c9e       ?CreateIndirect@CDialog@@UEAAHPEAXPEAVCWnd@@@Z 0000000140046c9e f   mfc140:mfc140.dll
 0001:00045ca4       ?CreateIndirect@CDialog@@UEAAHPEBUDLGTEMPLATE@@PEAVCWnd@@PEAX@Z 0000000140046ca4 f   mfc140:mfc140.dll
 0001:00045caa       ?DoModal@CDialog@@UEAA_JXZ 0000000140046caa f   mfc140:mfc140.dll
 0001:00045cb0       ?OnSetFont@CDialog@@UEAAXPEAVCFont@@@Z 0000000140046cb0 f   mfc140:mfc140.dll
 0001:00045cb6       ?OnOK@CDialog@@MEAAXXZ     0000000140046cb6 f   mfc140:mfc140.dll
 0001:00045cbc       ?OnCancel@CDialog@@MEAAXXZ 0000000140046cbc f   mfc140:mfc140.dll
 0001:00045cc2       ?PreInitDialog@CDialog@@MEAAXXZ 0000000140046cc2 f   mfc140:mfc140.dll
 0001:00045cc8       ?OnHelp@CWinApp@@IEAAXXZ   0000000140046cc8 f   mfc140:mfc140.dll
 0001:00045cce       ?GetThisMessageMap@CWinApp@@KAPEBUAFX_MSGMAP@@XZ 0000000140046cce f   mfc140:mfc140.dll
 0001:00045cd4       ?GetRuntimeClass@CWinApp@@UEBAPEAUCRuntimeClass@@XZ 0000000140046cd4 f   mfc140:mfc140.dll
 0001:00045cda       ?OnFinalRelease@CCmdTarget@@UEAAXXZ 0000000140046cda f   mfc140:mfc140.dll
 0001:00045ce0       ?GetInterfaceMap@CCmdTarget@@MEBAPEBUAFX_INTERFACEMAP@@XZ 0000000140046ce0 f   mfc140:mfc140.dll
 0001:00045ce6       ?Run@CWinApp@@UEAAHXZ      0000000140046ce6 f   mfc140:mfc140.dll
 0001:00045cec       ?PreTranslateMessage@CWinThread@@UEAAHPEAUtagMSG@@@Z 0000000140046cec f   mfc140:mfc140.dll
 0001:00045cf2       ?PumpMessage@CWinThread@@UEAAHXZ 0000000140046cf2 f   mfc140:mfc140.dll
 0001:00045cf8       ?OnIdle@CWinApp@@UEAAHJ@Z  0000000140046cf8 f   mfc140:mfc140.dll
 0001:00045cfe       ?IsIdleMessage@CWinThread@@UEAAHPEAUtagMSG@@@Z 0000000140046cfe f   mfc140:mfc140.dll
 0001:00045d04       ?ExitInstance@CWinApp@@UEAAHXZ 0000000140046d04 f   mfc140:mfc140.dll
 0001:00045d0a       ?ProcessWndProcException@CWinApp@@UEAA_JPEAVCException@@PEBUtagMSG@@@Z 0000000140046d0a f   mfc140:mfc140.dll
 0001:00045d10       ?ProcessMessageFilter@CWinThread@@UEAAHHPEAUtagMSG@@@Z 0000000140046d10 f   mfc140:mfc140.dll
 0001:00045d16       ?GetMainWnd@CWinThread@@UEAAPEAVCWnd@@XZ 0000000140046d16 f   mfc140:mfc140.dll
 0001:00045d1c       ?Delete@CWinThread@@UEAAXXZ 0000000140046d1c f   mfc140:mfc140.dll
 0001:00045d22       ?GetProfileIntA@CWinApp@@UEAAIPEBD0H@Z 0000000140046d22 f   mfc140:mfc140.dll
 0001:00045d28       ?WriteProfileInt@CWinApp@@UEAAHPEBD0H@Z 0000000140046d28 f   mfc140:mfc140.dll
 0001:00045d2e       ?GetProfileStringA@CWinApp@@UEAA?AV?$CStringT@DV?$StrTraitMFC_DLL@DV?$ChTraitsCRT@D@ATL@@@@@ATL@@PEBD00@Z 0000000140046d2e f   mfc140:mfc140.dll
 0001:00045d34       ?WriteProfileStringA@CWinApp@@UEAAHPEBD00@Z 0000000140046d34 f   mfc140:mfc140.dll
 0001:00045d3a       ?GetProfileBinary@CWinApp@@UEAAHPEBD0PEAPEAEPEAI@Z 0000000140046d3a f   mfc140:mfc140.dll
 0001:00045d40       ?WriteProfileBinary@CWinApp@@UEAAHPEBD0PEAEI@Z 0000000140046d40 f   mfc140:mfc140.dll
 0001:00045d46       ?InitLibId@CWinApp@@UEAAXXZ 0000000140046d46 f   mfc140:mfc140.dll
 0001:00045d4c       ?Register@CWinApp@@UEAAHXZ 0000000140046d4c f   mfc140:mfc140.dll
 0001:00045d52       ?Unregister@CWinApp@@UEAAHXZ 0000000140046d52 f   mfc140:mfc140.dll
 0001:00045d58       ?OpenDocumentFile@CWinApp@@UEAAPEAVCDocument@@PEBDH@Z 0000000140046d58 f   mfc140:mfc140.dll
 0001:00045d5e       ?OpenDocumentFile@CWinApp@@UEAAPEAVCDocument@@PEBD@Z 0000000140046d5e f   mfc140:mfc140.dll
 0001:00045d64       ?AddToRecentFileList@CWinApp@@UEAAXPEBD@Z 0000000140046d64 f   mfc140:mfc140.dll
 0001:00045d6a       ?InitApplication@CWinApp@@UEAAHXZ 0000000140046d6a f   mfc140:mfc140.dll
 0001:00045d70       ?SaveAllModified@CWinApp@@UEAAHXZ 0000000140046d70 f   mfc140:mfc140.dll
 0001:00045d76       ?DoMessageBox@CWinApp@@UEAAHPEBDII@Z 0000000140046d76 f   mfc140:mfc140.dll
 0001:00045d7c       ?DoWaitCursor@CWinApp@@UEAAXH@Z 0000000140046d7c f   mfc140:mfc140.dll
 0001:00045d82       ?OnDDECommand@CWinApp@@UEAAHPEAD@Z 0000000140046d82 f   mfc140:mfc140.dll
 0001:00045d88       ?WinHelpA@CWinApp@@UEAAX_KI@Z 0000000140046d88 f   mfc140:mfc140.dll
 0001:00045d8e       ?HtmlHelpA@CWinApp@@UEAAX_KI@Z 0000000140046d8e f   mfc140:mfc140.dll
 0001:00045d94       ?WinHelpInternal@CWinApp@@UEAAX_KI@Z 0000000140046d94 f   mfc140:mfc140.dll
 0001:00045d9a       ?RegisterWithRestartManager@CWinApp@@UEAAJPEB_WKP6AKPEAX@Z1KK@Z 0000000140046d9a f   mfc140:mfc140.dll
 0001:00045da0       ?RegisterWithRestartManager@CWinApp@@UEAAJHAEBV?$CStringT@DV?$StrTraitMFC_DLL@DV?$ChTraitsCRT@D@ATL@@@@@ATL@@@Z 0000000140046da0 f   mfc140:mfc140.dll
 0001:00045da6       ?ApplicationRecoveryCallback@CWinApp@@UEAAKPEAX@Z 0000000140046da6 f   mfc140:mfc140.dll
 0001:00045dac       ?GetDataRecoveryHandler@CWinApp@@UEAAPEAVCDataRecoveryHandler@@XZ 0000000140046dac f   mfc140:mfc140.dll
 0001:00045db2       ?IsTaskbarInteractionEnabled@CWinApp@@UEAAHXZ 0000000140046db2 f   mfc140:mfc140.dll
 0001:00045db8       ?RestartInstance@CWinApp@@UEAAHXZ 0000000140046db8 f   mfc140:mfc140.dll
 0001:00045dbe       ?LoadAppLangResourceDLL@CWinApp@@UEAAPEAUHINSTANCE__@@XZ 0000000140046dbe f   mfc140:mfc140.dll
 0001:00045dc4       ?LoadSysPolicies@CWinApp@@UEAAHXZ 0000000140046dc4 f   mfc140:mfc140.dll
 0001:00045dca       ?AfxGetModuleState@@YAPEAVAFX_MODULE_STATE@@XZ 0000000140046dca f   mfc140:mfc140.dll
 0001:00045dd0       ?GetRuntimeClass@CDialog@@UEBAPEAUCRuntimeClass@@XZ 0000000140046dd0 f   mfc140:mfc140.dll
 0001:00045df0       __security_check_cookie    0000000140046df0 f   msvcrt:amdsecgs.obj
 0001:00045e14       ??3@YAXPEAX_K@Z            0000000140046e14 f   msvcrt:delete_scalar_size.obj
 0001:00045fa4       _Init_thread_abort         0000000140046fa4 f   msvcrt:thread_safe_statics.obj
 0001:00045fd4       _Init_thread_footer        0000000140046fd4 f   msvcrt:thread_safe_statics.obj
 0001:00046034       _Init_thread_header        0000000140047034 f   msvcrt:thread_safe_statics.obj
 0001:0004609c       _Init_thread_notify        000000014004709c f   msvcrt:thread_safe_statics.obj
 0001:000460ec       _Init_thread_wait          00000001400470ec f   msvcrt:thread_safe_statics.obj
 0001:00046164       __scrt_acquire_startup_lock 0000000140047164 f   msvcrt:utility.obj
 0001:000461a0       __scrt_initialize_crt      00000001400471a0 f   msvcrt:utility.obj
 0001:000461ec       __scrt_initialize_onexit_tables 00000001400471ec f   msvcrt:utility.obj
 0001:000462c4       __scrt_is_nonwritable_in_current_image 00000001400472c4 f   msvcrt:utility.obj
 0001:00046360       __scrt_release_startup_lock 0000000140047360 f   msvcrt:utility.obj
 0001:00046384       __scrt_uninitialize_crt    0000000140047384 f   msvcrt:utility.obj
 0001:000463b0       _onexit                    00000001400473b0 f   msvcrt:utility.obj
 0001:00046400       atexit                     0000000140047400 f   msvcrt:utility.obj
 0001:00046418       ??_Etype_info@@UEAAPEAXI@Z 0000000140047418 f i msvcrt:std_type_info_static.obj
 0001:00046418       ??_Gtype_info@@UEAAPEAXI@Z 0000000140047418 f i msvcrt:std_type_info_static.obj
 0001:00046444       ??_L@YAXPEAX_K1P6AX0@Z2@Z  0000000140047444 f   msvcrt:ehvecctr.obj
 0001:000464b4       ??_M@YAXPEAX_K1P6AX0@Z@Z   00000001400474b4 f   msvcrt:ehvecdtr.obj
 0001:00046520       ?__ArrayUnwind@@YAXPEAX_K1P6AX0@Z@Z 0000000140047520 f   msvcrt:ehvecdtr.obj
 0001:00046584       ??_V@YAXPEAX_K@Z           0000000140047584 f   msvcrt:delete_array_size.obj
 0001:0004658c       __raise_securityfailure    000000014004758c f   msvcrt:gs_report.obj
 0001:000465c0       __report_gsfailure         00000001400475c0 f   msvcrt:gs_report.obj
 0001:00046694       __report_rangecheckfailure 0000000140047694 f   msvcrt:gs_report.obj
 0001:000466a8       __report_securityfailure   00000001400476a8 f   msvcrt:gs_report.obj
 0001:00046a80       WinMainCRTStartup          0000000140047a80 f   msvcrt:exe_winmain.obj
 0001:00046a94       __crt_debugger_hook        0000000140047a94 f   msvcrt:utility_desktop.obj
 0001:00046a9c       __scrt_fastfail            0000000140047a9c f   msvcrt:utility_desktop.obj
 0001:00046be8       __scrt_get_show_window_mode 0000000140047be8 f   msvcrt:utility_desktop.obj
 0001:00046c24       __scrt_initialize_mta      0000000140047c24 f   msvcrt:utility_desktop.obj
 0001:00046c2c       __scrt_is_managed_app      0000000140047c2c f   msvcrt:utility_desktop.obj
 0001:00046c80       __scrt_set_unhandled_exception_filter 0000000140047c80 f   msvcrt:utility_desktop.obj
 0001:00046c90       __scrt_unhandled_exception_filter 0000000140047c90 f   msvcrt:utility_desktop.obj
 0001:00046cc8       __isa_available_init       0000000140047cc8 f   msvcrt:cpu_disp.obj
 0001:00046e44       _get_startup_argv_mode     0000000140047e44 f   msvcrt:argv_mode.obj
 0001:00046e4c       __scrt_is_ucrt_dll_in_use  0000000140047e4c f   msvcrt:ucrt_detection.obj
 0001:00046e58       __security_init_cookie     0000000140047e58 f   msvcrt:gs_support.obj
 0001:00046f04       _get_startup_file_mode     0000000140047f04 f   msvcrt:file_mode.obj
 0001:00046f0c       ?__scrt_initialize_type_info@@YAXXZ 0000000140047f0c f   msvcrt:tncleanup.obj
 0001:00046f1c       __scrt_initialize_default_local_stdio_options 0000000140047f1c f   msvcrt:default_local_stdio_options.obj
 0001:00046f38       __scrt_is_user_matherr_present 0000000140047f38 f   msvcrt:matherr_detection.obj
 0001:00046f44       __scrt_get_dyn_tls_init_callback 0000000140047f44 f   msvcrt:dyn_tls_init.obj
 0001:00046f4c       __scrt_get_dyn_tls_dtor_callback 0000000140047f4c f   msvcrt:dyn_tls_dtor.obj
 0001:00046f54       _RTC_Initialize            0000000140047f54 f   msvcrt:initsect.obj
 0001:00046f90       _RTC_Terminate             0000000140047f90 f   msvcrt:initsect.obj
 0001:00046fcc       __GSHandlerCheck           0000000140047fcc f   msvcrt:gshandler.obj
 0001:00046fec       __GSHandlerCheckCommon     0000000140047fec f   msvcrt:gshandler.obj
 0001:00047050       IsProcessorFeaturePresent  0000000140048050 f   kernel32:KERNEL32.dll
 0001:00047058       ??0CAtlBaseModule@ATL@@QEAA@XZ 0000000140048058 f   atls:atlbase.obj
 0001:00047100       ??1CAtlBaseModule@ATL@@QEAA@XZ 0000000140048100 f   atls:atlbase.obj
 0001:00047134       ?xsputn@?$basic_streambuf@DU?$char_traits@D@std@@@std@@MEAA_JPEBD_J@Z 0000000140048134 f   msvcprt:MSVCP140.dll
 0001:0004713a       ?xsgetn@?$basic_streambuf@DU?$char_traits@D@std@@@std@@MEAA_JPEAD_J@Z 000000014004813a f   msvcprt:MSVCP140.dll
 0001:00047140       ??1_Fac_tidy_reg_t@std@@QEAA@XZ 0000000140048140 f i msvcprt:locale0_implib.obj
 0001:000471a7       ?showmanyc@?$basic_streambuf@DU?$char_traits@D@std@@@std@@MEAA_JXZ 00000001400481a7 f   msvcprt:MSVCP140.dll
 0001:000471ad       __CxxFrameHandler3         00000001400481ad f   vcruntime:VCRUNTIME140.dll
 0001:000471b3       __std_terminate            00000001400481b3 f   vcruntime:VCRUNTIME140.dll
 0001:000471b9       _purecall                  00000001400481b9 f   vcruntime:VCRUNTIME140.dll
 0001:000471bf       memset                     00000001400481bf f   vcruntime:VCRUNTIME140.dll
 0001:000471c5       __C_specific_handler       00000001400481c5 f   vcruntime:VCRUNTIME140.dll
 0001:000471cb       memmove                    00000001400481cb f   vcruntime:VCRUNTIME140.dll
 0001:000471d1       free                       00000001400481d1 f   ucrt:api-ms-win-crt-heap-l1-1-0.dll
 0001:000471d7       _configure_narrow_argv     00000001400481d7 f   ucrt:api-ms-win-crt-runtime-l1-1-0.dll
 0001:000471dd       _initialize_narrow_environment 00000001400481dd f   ucrt:api-ms-win-crt-runtime-l1-1-0.dll
 0001:000471e3       _initialize_onexit_table   00000001400481e3 f   ucrt:api-ms-win-crt-runtime-l1-1-0.dll
 0001:000471e9       _register_onexit_function  00000001400481e9 f   ucrt:api-ms-win-crt-runtime-l1-1-0.dll
 0001:000471ef       _crt_atexit                00000001400481ef f   ucrt:api-ms-win-crt-runtime-l1-1-0.dll
 0001:000471f5       _cexit                     00000001400481f5 f   ucrt:api-ms-win-crt-runtime-l1-1-0.dll
 0001:000471fb       terminate                  00000001400481fb f   ucrt:api-ms-win-crt-runtime-l1-1-0.dll
 0001:00047201       _seh_filter_exe            0000000140048201 f   ucrt:api-ms-win-crt-runtime-l1-1-0.dll
 0001:00047207       _set_app_type              0000000140048207 f   ucrt:api-ms-win-crt-runtime-l1-1-0.dll
 0001:0004720d       __setusermatherr           000000014004820d f   ucrt:api-ms-win-crt-math-l1-1-0.dll
 0001:00047213       _get_narrow_winmain_command_line 0000000140048213 f   ucrt:api-ms-win-crt-runtime-l1-1-0.dll
 0001:00047219       _initterm                  0000000140048219 f   ucrt:api-ms-win-crt-runtime-l1-1-0.dll
 0001:0004721f       _initterm_e                000000014004821f f   ucrt:api-ms-win-crt-runtime-l1-1-0.dll
 0001:00047225       exit                       0000000140048225 f   ucrt:api-ms-win-crt-runtime-l1-1-0.dll
 0001:0004722b       _exit                      000000014004822b f   ucrt:api-ms-win-crt-runtime-l1-1-0.dll
 0001:00047231       _set_fmode                 0000000140048231 f   ucrt:api-ms-win-crt-stdio-l1-1-0.dll
 0001:00047237       _c_exit                    0000000140048237 f   ucrt:api-ms-win-crt-runtime-l1-1-0.dll
 0001:0004723d       _register_thread_local_exe_atexit_callback 000000014004823d f   ucrt:api-ms-win-crt-runtime-l1-1-0.dll
 0001:00047243       _configthreadlocale        0000000140048243 f   ucrt:api-ms-win-crt-locale-l1-1-0.dll
 0001:00047249       _set_new_mode              0000000140048249 f   ucrt:api-ms-win-crt-heap-l1-1-0.dll
 0001:0004724f       __p__commode               000000014004824f f   ucrt:api-ms-win-crt-stdio-l1-1-0.dll
 0001:00047258       ?AfxInitialize@@YAHHK@Z    0000000140048258 f   mfcs140:appmodul.obj
 0001:00047290       WinMain                    0000000140048290 f   mfcs140:appmodul.obj
 0001:00047295       ?_Lock@?$basic_streambuf@DU?$char_traits@D@std@@@std@@UEAAXXZ 0000000140048295 f   msvcprt:MSVCP140.dll
 0001:0004729b       ?_Unlock@?$basic_streambuf@DU?$char_traits@D@std@@@std@@UEAAXXZ 000000014004829b f   msvcprt:MSVCP140.dll
 0001:000472a1       ?uflow@?$basic_streambuf@DU?$char_traits@D@std@@@std@@MEAAHXZ 00000001400482a1 f   msvcprt:MSVCP140.dll
 0001:000472a7       ?setbuf@?$basic_streambuf@DU?$char_traits@D@std@@@std@@MEAAPEAV12@PEAD_J@Z 00000001400482a7 f   msvcprt:MSVCP140.dll
 0001:000472ad       ?sync@?$basic_streambuf@DU?$char_traits@D@std@@@std@@MEAAHXZ 00000001400482ad f   msvcprt:MSVCP140.dll
 0001:000472b3       ?imbue@?$basic_streambuf@DU?$char_traits@D@std@@@std@@MEAAXAEBVlocale@2@@Z 00000001400482b3 f   msvcprt:MSVCP140.dll
 0001:000472b9       ?AfxWinMain@@YAHPEAUHINSTANCE__@@0PEADH@Z 00000001400482b9 f   mfc140:mfc140.dll
 0001:000472c0       __GSHandlerCheck_EH        00000001400482c0 f   msvcrt:gshandlereh.obj
 0001:00047350       _alloca_probe              0000000140048350 f   msvcrt:chkstk.obj
 0001:00047350       __chkstk                   0000000140048350 f   msvcrt:chkstk.obj
 0001:000473a1       _CxxThrowException         00000001400483a1 f   vcruntime:VCRUNTIME140.dll
 0001:000473a7       memchr                     00000001400483a7 f   vcruntime:VCRUNTIME140.dll
 0001:000473ad       memcmp                     00000001400483ad f   vcruntime:VCRUNTIME140.dll
 0001:000473b3       memcpy                     00000001400483b3 f   vcruntime:VCRUNTIME140.dll
 0001:000473b9       atan                       00000001400483b9 f   ucrt:api-ms-win-crt-math-l1-1-0.dll
 0001:000473bf       sqrtf                      00000001400483bf f   ucrt:api-ms-win-crt-math-l1-1-0.dll
 0001:000473c5       strcmp                     00000001400483c5 f   ucrt:api-ms-win-crt-string-l1-1-0.dll
 0001:000473e0       _guard_dispatch_icall_nop  00000001400483e0 f   msvcrt:guard_dispatch.obj
 0002:00000000       __imp_SetServiceStatus     000000014004b000     advapi32:ADVAPI32.dll
 0002:00000008       __imp_RegisterServiceCtrlHandlerA 000000014004b008     advapi32:ADVAPI32.dll
 0002:00000010       __imp_OpenSCManagerA       000000014004b010     advapi32:ADVAPI32.dll
 0002:00000018       __imp_OpenServiceA         000000014004b018     advapi32:ADVAPI32.dll
 0002:00000020       __imp_ChangeServiceConfigA 000000014004b020     advapi32:ADVAPI32.dll
 0002:00000028       __imp_CloseServiceHandle   000000014004b028     advapi32:ADVAPI32.dll
 0002:00000030       __imp_StartServiceCtrlDispatcherA 000000014004b030     advapi32:ADVAPI32.dll
 0002:00000038       \177ADVAPI32_NULL_THUNK_DATA 000000014004b038     advapi32:ADVAPI32.dll
 0002:00000040       __imp_GetAdaptersInfo      000000014004b040     ipHlpapi:IPHLPAPI.DLL
 0002:00000048       \177IPHLPAPI_NULL_THUNK_DATA 000000014004b048     ipHlpapi:IPHLPAPI.DLL
 0002:00000050       __imp_CreateThread         000000014004b050     kernel32:KERNEL32.dll
 0002:00000058       __imp_WaitForSingleObject  000000014004b058     kernel32:KERNEL32.dll
 0002:00000060       __imp_GetCurrentProcessId  000000014004b060     kernel32:KERNEL32.dll
 0002:00000068       __imp_SetUnhandledExceptionFilter 000000014004b068     kernel32:KERNEL32.dll
 0002:00000070       __imp_GetPrivateProfileStringW 000000014004b070     kernel32:KERNEL32.dll
 0002:00000078       __imp_GetModuleFileNameW   000000014004b078     kernel32:KERNEL32.dll
 0002:00000080       __imp_OutputDebugStringW   000000014004b080     kernel32:KERNEL32.dll
 0002:00000088       __imp_GetCurrentProcess    000000014004b088     kernel32:KERNEL32.dll
 0002:00000090       __imp_RaiseException       000000014004b090     kernel32:KERNEL32.dll
 0002:00000098       __imp_MultiByteToWideChar  000000014004b098     kernel32:KERNEL32.dll
 0002:000000a0       __imp_GetComputerNameW     000000014004b0a0     kernel32:KERNEL32.dll
 0002:000000a8       __imp_WideCharToMultiByte  000000014004b0a8     kernel32:KERNEL32.dll
 0002:000000b0       __imp_GetLastError         000000014004b0b0     kernel32:KERNEL32.dll
 0002:000000b8       __imp_GetCurrentThread     000000014004b0b8     kernel32:KERNEL32.dll
 0002:000000c0       __imp_CreateFileW          000000014004b0c0     kernel32:KERNEL32.dll
 0002:000000c8       __imp_GetFileSize          000000014004b0c8     kernel32:KERNEL32.dll
 0002:000000d0       __imp_InitializeCriticalSection 000000014004b0d0     kernel32:KERNEL32.dll
 0002:000000d8       __imp_DeleteCriticalSection 000000014004b0d8     kernel32:KERNEL32.dll
 0002:000000e0       __imp_EnterCriticalSection 000000014004b0e0     kernel32:KERNEL32.dll
 0002:000000e8       __imp_LeaveCriticalSection 000000014004b0e8     kernel32:KERNEL32.dll
 0002:000000f0       __imp_ResetEvent           000000014004b0f0     kernel32:KERNEL32.dll
 0002:000000f8       __imp_GetProcessId         000000014004b0f8     kernel32:KERNEL32.dll
 0002:00000100       __imp_OpenProcess          000000014004b100     kernel32:KERNEL32.dll
 0002:00000108       __imp_LoadLibraryA         000000014004b108     kernel32:KERNEL32.dll
 0002:00000110       __imp_GetProcAddress       000000014004b110     kernel32:KERNEL32.dll
 0002:00000118       __imp_GetTickCount         000000014004b118     kernel32:KERNEL32.dll
 0002:00000120       __imp_FreeLibrary          000000014004b120     kernel32:KERNEL32.dll
 0002:00000128       __imp_CreateEventA         000000014004b128     kernel32:KERNEL32.dll
 0002:00000130       __imp_GetModuleFileNameA   000000014004b130     kernel32:KERNEL32.dll
 0002:00000138       __imp_GetModuleHandleA     000000014004b138     kernel32:KERNEL32.dll
 0002:00000140       __imp_CreateRemoteThread   000000014004b140     kernel32:KERNEL32.dll
 0002:00000148       __imp_GetCurrentThreadId   000000014004b148     kernel32:KERNEL32.dll
 0002:00000150       __imp_TerminateThread      000000014004b150     kernel32:KERNEL32.dll
 0002:00000158       __imp_GetPrivateProfileStringA 000000014004b158     kernel32:KERNEL32.dll
 0002:00000160       __imp_ResumeThread         000000014004b160     kernel32:KERNEL32.dll
 0002:00000168       __imp_GetExitCodeProcess   000000014004b168     kernel32:KERNEL32.dll
 0002:00000170       __imp_CreateMutexA         000000014004b170     kernel32:KERNEL32.dll
 0002:00000178       __imp_CreateFileMappingA   000000014004b178     kernel32:KERNEL32.dll
 0002:00000180       __imp_MapViewOfFile        000000014004b180     kernel32:KERNEL32.dll
 0002:00000188       __imp_ReleaseMutex         000000014004b188     kernel32:KERNEL32.dll
 0002:00000190       __imp_UnmapViewOfFile      000000014004b190     kernel32:KERNEL32.dll
 0002:00000198       __imp_Sleep                000000014004b198     kernel32:KERNEL32.dll
 0002:000001a0       __imp_OutputDebugStringA   000000014004b1a0     kernel32:KERNEL32.dll
 0002:000001a8       __imp_GetSystemTimes       000000014004b1a8     kernel32:KERNEL32.dll
 0002:000001b0       __imp_TryEnterCriticalSection 000000014004b1b0     kernel32:KERNEL32.dll
 0002:000001b8       __imp_FindFirstFileA       000000014004b1b8     kernel32:KERNEL32.dll
 0002:000001c0       __imp_CopyFileA            000000014004b1c0     kernel32:KERNEL32.dll
 0002:000001c8       __imp_DeleteFileA          000000014004b1c8     kernel32:KERNEL32.dll
 0002:000001d0       __imp_FindNextFileA        000000014004b1d0     kernel32:KERNEL32.dll
 0002:000001d8       __imp_FindClose            000000014004b1d8     kernel32:KERNEL32.dll
 0002:000001e0       __imp_WriteFile            000000014004b1e0     kernel32:KERNEL32.dll
 0002:000001e8       __imp_FormatMessageA       000000014004b1e8     kernel32:KERNEL32.dll
 0002:000001f0       __imp_GetVersionExA        000000014004b1f0     kernel32:KERNEL32.dll
 0002:000001f8       __imp_GetSystemInfo        000000014004b1f8     kernel32:KERNEL32.dll
 0002:00000200       __imp_OpenFileMappingA     000000014004b200     kernel32:KERNEL32.dll
 0002:00000208       __imp_InitializeCriticalSectionAndSpinCount 000000014004b208     kernel32:KERNEL32.dll
 0002:00000210       __imp_GetPrivateProfileIntA 000000014004b210     kernel32:KERNEL32.dll
 0002:00000218       __imp_GetLocalTime         000000014004b218     kernel32:KERNEL32.dll
 0002:00000220       __imp_SetCurrentDirectoryA 000000014004b220     kernel32:KERNEL32.dll
 0002:00000228       __imp_GetCurrentDirectoryA 000000014004b228     kernel32:KERNEL32.dll
 0002:00000230       __imp_CloseHandle          000000014004b230     kernel32:KERNEL32.dll
 0002:00000238       __imp_ReadFile             000000014004b238     kernel32:KERNEL32.dll
 0002:00000240       __imp_TerminateProcess     000000014004b240     kernel32:KERNEL32.dll
 0002:00000248       __imp_GetModuleHandleW     000000014004b248     kernel32:KERNEL32.dll
 0002:00000250       __imp_SetEvent             000000014004b250     kernel32:KERNEL32.dll
 0002:00000258       __imp_InitializeSListHead  000000014004b258     kernel32:KERNEL32.dll
 0002:00000260       __imp_GetSystemTimeAsFileTime 000000014004b260     kernel32:KERNEL32.dll
 0002:00000268       __imp_QueryPerformanceCounter 000000014004b268     kernel32:KERNEL32.dll
 0002:00000270       __imp_GetStartupInfoW      000000014004b270     kernel32:KERNEL32.dll
 0002:00000278       __imp_IsDebuggerPresent    000000014004b278     kernel32:KERNEL32.dll
 0002:00000280       __imp_IsProcessorFeaturePresent 000000014004b280     kernel32:KERNEL32.dll
 0002:00000288       __imp_UnhandledExceptionFilter 000000014004b288     kernel32:KERNEL32.dll
 0002:00000290       __imp_RtlVirtualUnwind     000000014004b290     kernel32:KERNEL32.dll
 0002:00000298       __imp_RtlLookupFunctionEntry 000000014004b298     kernel32:KERNEL32.dll
 0002:000002a0       __imp_RtlCaptureContext    000000014004b2a0     kernel32:KERNEL32.dll
 0002:000002a8       __imp_WaitForSingleObjectEx 000000014004b2a8     kernel32:KERNEL32.dll
 0002:000002b0       __imp_CreateEventW         000000014004b2b0     kernel32:KERNEL32.dll
 0002:000002b8       __imp_CreateFileA          000000014004b2b8     kernel32:KERNEL32.dll
 0002:000002c0       \177KERNEL32_NULL_THUNK_DATA 000000014004b2c0     kernel32:KERNEL32.dll
 0002:000002c8       __imp_??1?$basic_iostream@DU?$char_traits@D@std@@@std@@UEAA@XZ 000000014004b2c8     msvcprt:MSVCP140.dll
 0002:000002d0       __imp_??6?$basic_ostream@DU?$char_traits@D@std@@@std@@QEAAAEAV01@_K@Z 000000014004b2d0     msvcprt:MSVCP140.dll
 0002:000002d8       __imp_?_Xlength_error@std@@YAXPEBD@Z 000000014004b2d8     msvcprt:MSVCP140.dll
 0002:000002e0       __imp_?_Xout_of_range@std@@YAXPEBD@Z 000000014004b2e0     msvcprt:MSVCP140.dll
 0002:000002e8       __imp_?uncaught_exception@std@@YA_NXZ 000000014004b2e8     msvcprt:MSVCP140.dll
 0002:000002f0       __imp_?sputc@?$basic_streambuf@DU?$char_traits@D@std@@@std@@QEAAHD@Z 000000014004b2f0     msvcprt:MSVCP140.dll
 0002:000002f8       __imp_?widen@?$basic_ios@DU?$char_traits@D@std@@@std@@QEBADD@Z 000000014004b2f8     msvcprt:MSVCP140.dll
 0002:00000300       __imp_?sputn@?$basic_streambuf@DU?$char_traits@D@std@@@std@@QEAA_JPEBD_J@Z 000000014004b300     msvcprt:MSVCP140.dll
 0002:00000308       __imp_?put@?$basic_ostream@DU?$char_traits@D@std@@@std@@QEAAAEAV12@D@Z 000000014004b308     msvcprt:MSVCP140.dll
 0002:00000310       __imp_?_Osfx@?$basic_ostream@DU?$char_traits@D@std@@@std@@QEAAXXZ 000000014004b310     msvcprt:MSVCP140.dll
 0002:00000318       __imp_?flush@?$basic_ostream@DU?$char_traits@D@std@@@std@@QEAAAEAV12@XZ 000000014004b318     msvcprt:MSVCP140.dll
 0002:00000320       __imp_?setstate@?$basic_ios@DU?$char_traits@D@std@@@std@@QEAAXH_N@Z 000000014004b320     msvcprt:MSVCP140.dll
 0002:00000328       __imp_??6?$basic_ostream@DU?$char_traits@D@std@@@std@@QEAAAEAV01@P6AAEAV01@AEAV01@@Z@Z 000000014004b328     msvcprt:MSVCP140.dll
 0002:00000330       __imp_??1?$basic_ios@DU?$char_traits@D@std@@@std@@UEAA@XZ 000000014004b330     msvcprt:MSVCP140.dll
 0002:00000338       __imp_?xsputn@?$basic_streambuf@DU?$char_traits@D@std@@@std@@MEAA_JPEBD_J@Z 000000014004b338     msvcprt:MSVCP140.dll
 0002:00000340       __imp_?xsgetn@?$basic_streambuf@DU?$char_traits@D@std@@@std@@MEAA_JPEAD_J@Z 000000014004b340     msvcprt:MSVCP140.dll
 0002:00000348       __imp_?_Pninc@?$basic_streambuf@DU?$char_traits@D@std@@@std@@IEAAPEADXZ 000000014004b348     msvcprt:MSVCP140.dll
 0002:00000350       __imp_??1?$basic_streambuf@DU?$char_traits@D@std@@@std@@UEAA@XZ 000000014004b350     msvcprt:MSVCP140.dll
 0002:00000358       __imp_?showmanyc@?$basic_streambuf@DU?$char_traits@D@std@@@std@@MEAA_JXZ 000000014004b358     msvcprt:MSVCP140.dll
 0002:00000360       __imp_??0?$basic_streambuf@DU?$char_traits@D@std@@@std@@IEAA@XZ 000000014004b360     msvcprt:MSVCP140.dll
 0002:00000368       __imp_??0?$basic_ios@DU?$char_traits@D@std@@@std@@IEAA@XZ 000000014004b368     msvcprt:MSVCP140.dll
 0002:00000370       __imp_?imbue@?$basic_streambuf@DU?$char_traits@D@std@@@std@@MEAAXAEBVlocale@2@@Z 000000014004b370     msvcprt:MSVCP140.dll
 0002:00000378       __imp_??0?$basic_iostream@DU?$char_traits@D@std@@@std@@QEAA@PEAV?$basic_streambuf@DU?$char_traits@D@std@@@1@@Z 000000014004b378     msvcprt:MSVCP140.dll
 0002:00000380       __imp_?_Lock@?$basic_streambuf@DU?$char_traits@D@std@@@std@@UEAAXXZ 000000014004b380     msvcprt:MSVCP140.dll
 0002:00000388       __imp_?_Unlock@?$basic_streambuf@DU?$char_traits@D@std@@@std@@UEAAXXZ 000000014004b388     msvcprt:MSVCP140.dll
 0002:00000390       __imp_?uflow@?$basic_streambuf@DU?$char_traits@D@std@@@std@@MEAAHXZ 000000014004b390     msvcprt:MSVCP140.dll
 0002:00000398       __imp_?setbuf@?$basic_streambuf@DU?$char_traits@D@std@@@std@@MEAAPEAV12@PEAD_J@Z 000000014004b398     msvcprt:MSVCP140.dll
 0002:000003a0       __imp_?sync@?$basic_streambuf@DU?$char_traits@D@std@@@std@@MEAAHXZ 000000014004b3a0     msvcprt:MSVCP140.dll
 0002:000003a8       \177MSVCP140_NULL_THUNK_DATA 000000014004b3a8     msvcprt:MSVCP140.dll
 0002:000003b0       __imp_GetProcessImageFileNameA 000000014004b3b0     Psapi:PSAPI.DLL
 0002:000003b8       __imp_GetModuleBaseNameA   000000014004b3b8     Psapi:PSAPI.DLL
 0002:000003c0       __imp_EnumProcessModules   000000014004b3c0     Psapi:PSAPI.DLL
 0002:000003c8       __imp_EnumProcesses        000000014004b3c8     Psapi:PSAPI.DLL
 0002:000003d0       __imp_GetProcessMemoryInfo 000000014004b3d0     Psapi:PSAPI.DLL
 0002:000003d8       __imp_EmptyWorkingSet      000000014004b3d8     Psapi:PSAPI.DLL
 0002:000003e0       \177PSAPI_NULL_THUNK_DATA  000000014004b3e0     Psapi:PSAPI.DLL
 0002:000003e8       __imp_ShellExecuteExA      000000014004b3e8     shell32:SHELL32.dll
 0002:000003f0       __imp_SHCreateDirectoryExA 000000014004b3f0     shell32:SHELL32.dll
 0002:000003f8       \177SHELL32_NULL_THUNK_DATA 000000014004b3f8     shell32:SHELL32.dll
 0002:00000400       __imp_PathFileExistsW      000000014004b400     shlwapi:SHLWAPI.dll
 0002:00000408       \177SHLWAPI_NULL_THUNK_DATA 000000014004b408     shlwapi:SHLWAPI.dll
 0002:00000410       __imp_SendMessageTimeoutA  000000014004b410     user32:USER32.dll
 0002:00000418       __imp_PostMessageA         000000014004b418     user32:USER32.dll
 0002:00000420       __imp_IsWindow             000000014004b420     user32:USER32.dll
 0002:00000428       __imp_DrawIcon             000000014004b428     user32:USER32.dll
 0002:00000430       __imp_GetClientRect        000000014004b430     user32:USER32.dll
 0002:00000438       __imp_GetSystemMetrics     000000014004b438     user32:USER32.dll
 0002:00000440       __imp_IsIconic             000000014004b440     user32:USER32.dll
 0002:00000448       __imp_LoadIconW            000000014004b448     user32:USER32.dll
 0002:00000450       __imp_SetTimer             000000014004b450     user32:USER32.dll
 0002:00000458       __imp_SendMessageA         000000014004b458     user32:USER32.dll
 0002:00000460       __imp_wsprintfA            000000014004b460     user32:USER32.dll
 0002:00000468       __imp_EnableWindow         000000014004b468     user32:USER32.dll
 0002:00000470       \177USER32_NULL_THUNK_DATA 000000014004b470     user32:USER32.dll
 0002:00000478       __imp_memcmp               000000014004b478     vcruntime:VCRUNTIME140.dll
 0002:00000480       __imp_memchr               000000014004b480     vcruntime:VCRUNTIME140.dll
 0002:00000488       __imp__CxxThrowException   000000014004b488     vcruntime:VCRUNTIME140.dll
 0002:00000490       __imp___CxxFrameHandler3   000000014004b490     vcruntime:VCRUNTIME140.dll
 0002:00000498       __imp___std_terminate      000000014004b498     vcruntime:VCRUNTIME140.dll
 0002:000004a0       __imp_wcsrchr              000000014004b4a0     vcruntime:VCRUNTIME140.dll
 0002:000004a8       __imp__purecall            000000014004b4a8     vcruntime:VCRUNTIME140.dll
 0002:000004b0       __imp___std_exception_copy 000000014004b4b0     vcruntime:VCRUNTIME140.dll
 0002:000004b8       __imp___std_exception_destroy 000000014004b4b8     vcruntime:VCRUNTIME140.dll
 0002:000004c0       __imp_strrchr              000000014004b4c0     vcruntime:VCRUNTIME140.dll
 0002:000004c8       __imp_strstr               000000014004b4c8     vcruntime:VCRUNTIME140.dll
 0002:000004d0       __imp_memmove              000000014004b4d0     vcruntime:VCRUNTIME140.dll
 0002:000004d8       __imp_memset               000000014004b4d8     vcruntime:VCRUNTIME140.dll
 0002:000004e0       __imp___C_specific_handler 000000014004b4e0     vcruntime:VCRUNTIME140.dll
 0002:000004e8       __imp_memcpy               000000014004b4e8     vcruntime:VCRUNTIME140.dll
 0002:000004f0       \177VCRUNTIME140_NULL_THUNK_DATA 000000014004b4f0     vcruntime:VCRUNTIME140.dll
 0002:000004f8       __imp_WinHttpCloseHandle   000000014004b4f8     winhttp:WINHTTP.dll
 0002:00000500       __imp_WinHttpCrackUrl      000000014004b500     winhttp:WINHTTP.dll
 0002:00000508       __imp_WinHttpOpenRequest   000000014004b508     winhttp:WINHTTP.dll
 0002:00000510       __imp_WinHttpSendRequest   000000014004b510     winhttp:WINHTTP.dll
 0002:00000518       __imp_WinHttpOpen          000000014004b518     winhttp:WINHTTP.dll
 0002:00000520       __imp_WinHttpQueryHeaders  000000014004b520     winhttp:WINHTTP.dll
 0002:00000528       __imp_WinHttpWriteData     000000014004b528     winhttp:WINHTTP.dll
 0002:00000530       __imp_WinHttpConnect       000000014004b530     winhttp:WINHTTP.dll
 0002:00000538       __imp_WinHttpReceiveResponse 000000014004b538     winhttp:WINHTTP.dll
 0002:00000540       \177WINHTTP_NULL_THUNK_DATA 000000014004b540     winhttp:WINHTTP.dll
 0002:00000548       __imp_timeGetTime          000000014004b548     winmm:WINMM.dll
 0002:00000550       \177WINMM_NULL_THUNK_DATA  000000014004b550     winmm:WINMM.dll
 0002:00000558       __imp_WSAGetLastError      000000014004b558     ws2_32:WS2_32.dll
 0002:00000560       __imp_inet_addr            000000014004b560     ws2_32:WS2_32.dll
 0002:00000568       __imp_WSAWaitForMultipleEvents 000000014004b568     ws2_32:WS2_32.dll
 0002:00000570       __imp_connect              000000014004b570     ws2_32:WS2_32.dll
 0002:00000578       __imp_WSAStartup           000000014004b578     ws2_32:WS2_32.dll
 0002:00000580       __imp_WSACloseEvent        000000014004b580     ws2_32:WS2_32.dll
 0002:00000588       __imp_WSAEnumNetworkEvents 000000014004b588     ws2_32:WS2_32.dll
 0002:00000590       __imp_ioctlsocket          000000014004b590     ws2_32:WS2_32.dll
 0002:00000598       __imp_WSAAsyncSelect       000000014004b598     ws2_32:WS2_32.dll
 0002:000005a0       __imp_ntohs                000000014004b5a0     ws2_32:WS2_32.dll
 0002:000005a8       __imp_gethostname          000000014004b5a8     ws2_32:WS2_32.dll
 0002:000005b0       __imp_gethostbyaddr        000000014004b5b0     ws2_32:WS2_32.dll
 0002:000005b8       __imp_socket               000000014004b5b8     ws2_32:WS2_32.dll
 0002:000005c0       __imp_gethostbyname        000000014004b5c0     ws2_32:WS2_32.dll
 0002:000005c8       __imp_WSAEventSelect       000000014004b5c8     ws2_32:WS2_32.dll
 0002:000005d0       __imp_inet_ntoa            000000014004b5d0     ws2_32:WS2_32.dll
 0002:000005d8       __imp_send                 000000014004b5d8     ws2_32:WS2_32.dll
 0002:000005e0       __imp_htons                000000014004b5e0     ws2_32:WS2_32.dll
 0002:000005e8       __imp_recv                 000000014004b5e8     ws2_32:WS2_32.dll
 0002:000005f0       __imp_WSAGetOverlappedResult 000000014004b5f0     ws2_32:WS2_32.dll
 0002:000005f8       __imp_WSASend              000000014004b5f8     ws2_32:WS2_32.dll
 0002:00000600       __imp_closesocket          000000014004b600     ws2_32:WS2_32.dll
 0002:00000608       __imp_WSASocketA           000000014004b608     ws2_32:WS2_32.dll
 0002:00000610       __imp_WSACleanup           000000014004b610     ws2_32:WS2_32.dll
 0002:00000618       __imp_WSACreateEvent       000000014004b618     ws2_32:WS2_32.dll
 0002:00000620       __imp_WSAIoctl             000000014004b620     ws2_32:WS2_32.dll
 0002:00000628       \177WS2_32_NULL_THUNK_DATA 000000014004b628     ws2_32:WS2_32.dll
 0002:00000630       __imp_atoi                 000000014004b630     ucrt:api-ms-win-crt-convert-l1-1-0.dll
 0002:00000638       __imp__itoa_s              000000014004b638     ucrt:api-ms-win-crt-convert-l1-1-0.dll
 0002:00000640       __imp_mbstowcs             000000014004b640     ucrt:api-ms-win-crt-convert-l1-1-0.dll
 0002:00000648       __imp__itoa                000000014004b648     ucrt:api-ms-win-crt-convert-l1-1-0.dll
 0002:00000648       __imp_itoa                 000000014004b648     ucrt:api-ms-win-crt-convert-l1-1-0.dll
 0002:00000650       \177api-ms-win-crt-convert-l1-1-0_NULL_THUNK_DATA 000000014004b650     ucrt:api-ms-win-crt-convert-l1-1-0.dll
 0002:00000658       __imp__splitpath_s         000000014004b658     ucrt:api-ms-win-crt-filesystem-l1-1-0.dll
 0002:00000660       __imp__mkdir               000000014004b660     ucrt:api-ms-win-crt-filesystem-l1-1-0.dll
 0002:00000668       \177api-ms-win-crt-filesystem-l1-1-0_NULL_THUNK_DATA 000000014004b668     ucrt:api-ms-win-crt-filesystem-l1-1-0.dll
 0002:00000670       __imp_realloc              000000014004b670     ucrt:api-ms-win-crt-heap-l1-1-0.dll
 0002:00000678       __imp_free                 000000014004b678     ucrt:api-ms-win-crt-heap-l1-1-0.dll
 0002:00000680       __imp__set_new_mode        000000014004b680     ucrt:api-ms-win-crt-heap-l1-1-0.dll
 0002:00000688       __imp_malloc               000000014004b688     ucrt:api-ms-win-crt-heap-l1-1-0.dll
 0002:00000690       \177api-ms-win-crt-heap-l1-1-0_NULL_THUNK_DATA 000000014004b690     ucrt:api-ms-win-crt-heap-l1-1-0.dll
 0002:00000698       __imp__setmbcp             000000014004b698     ucrt:api-ms-win-crt-locale-l1-1-0.dll
 0002:000006a0       __imp__configthreadlocale  000000014004b6a0     ucrt:api-ms-win-crt-locale-l1-1-0.dll
 0002:000006a8       \177api-ms-win-crt-locale-l1-1-0_NULL_THUNK_DATA 000000014004b6a8     ucrt:api-ms-win-crt-locale-l1-1-0.dll
 0002:000006b0       __imp___setusermatherr     000000014004b6b0     ucrt:api-ms-win-crt-math-l1-1-0.dll
 0002:000006b8       __imp_sqrtf                000000014004b6b8     ucrt:api-ms-win-crt-math-l1-1-0.dll
 0002:000006c0       __imp_atan                 000000014004b6c0     ucrt:api-ms-win-crt-math-l1-1-0.dll
 0002:000006c8       \177api-ms-win-crt-math-l1-1-0_NULL_THUNK_DATA 000000014004b6c8     ucrt:api-ms-win-crt-math-l1-1-0.dll
 0002:000006d0       __imp__mbsicmp             000000014004b6d0     ucrt:api-ms-win-crt-multibyte-l1-1-0.dll
 0002:000006d8       __imp__mbschr              000000014004b6d8     ucrt:api-ms-win-crt-multibyte-l1-1-0.dll
 0002:000006e0       __imp__mbscmp              000000014004b6e0     ucrt:api-ms-win-crt-multibyte-l1-1-0.dll
 0002:000006e8       __imp__mbslwr_s            000000014004b6e8     ucrt:api-ms-win-crt-multibyte-l1-1-0.dll
 0002:000006f0       __imp__mbctolower          000000014004b6f0     ucrt:api-ms-win-crt-multibyte-l1-1-0.dll
 0002:000006f8       \177api-ms-win-crt-multibyte-l1-1-0_NULL_THUNK_DATA 000000014004b6f8     ucrt:api-ms-win-crt-multibyte-l1-1-0.dll
 0002:00000700       __imp__register_thread_local_exe_atexit_callback 000000014004b700     ucrt:api-ms-win-crt-runtime-l1-1-0.dll
 0002:00000708       __imp__set_app_type        000000014004b708     ucrt:api-ms-win-crt-runtime-l1-1-0.dll
 0002:00000710       __imp__seh_filter_exe      000000014004b710     ucrt:api-ms-win-crt-runtime-l1-1-0.dll
 0002:00000718       __imp_terminate            000000014004b718     ucrt:api-ms-win-crt-runtime-l1-1-0.dll
 0002:00000720       __imp__beginthreadex       000000014004b720     ucrt:api-ms-win-crt-runtime-l1-1-0.dll
 0002:00000728       __imp__cexit               000000014004b728     ucrt:api-ms-win-crt-runtime-l1-1-0.dll
 0002:00000730       __imp__get_narrow_winmain_command_line 000000014004b730     ucrt:api-ms-win-crt-runtime-l1-1-0.dll
 0002:00000738       __imp__set_invalid_parameter_handler 000000014004b738     ucrt:api-ms-win-crt-runtime-l1-1-0.dll
 0002:00000740       __imp__crt_atexit          000000014004b740     ucrt:api-ms-win-crt-runtime-l1-1-0.dll
 0002:00000748       __imp__initterm            000000014004b748     ucrt:api-ms-win-crt-runtime-l1-1-0.dll
 0002:00000750       __imp__invalid_parameter_noinfo_noreturn 000000014004b750     ucrt:api-ms-win-crt-runtime-l1-1-0.dll
 0002:00000758       __imp__register_onexit_function 000000014004b758     ucrt:api-ms-win-crt-runtime-l1-1-0.dll
 0002:00000760       __imp__initterm_e          000000014004b760     ucrt:api-ms-win-crt-runtime-l1-1-0.dll
 0002:00000768       __imp__invalid_parameter_noinfo 000000014004b768     ucrt:api-ms-win-crt-runtime-l1-1-0.dll
 0002:00000770       __imp_exit                 000000014004b770     ucrt:api-ms-win-crt-runtime-l1-1-0.dll
 0002:00000778       __imp__exit                000000014004b778     ucrt:api-ms-win-crt-runtime-l1-1-0.dll
 0002:00000780       __imp__initialize_onexit_table 000000014004b780     ucrt:api-ms-win-crt-runtime-l1-1-0.dll
 0002:00000788       __imp__initialize_narrow_environment 000000014004b788     ucrt:api-ms-win-crt-runtime-l1-1-0.dll
 0002:00000790       __imp__c_exit              000000014004b790     ucrt:api-ms-win-crt-runtime-l1-1-0.dll
 0002:00000798       __imp__configure_narrow_argv 000000014004b798     ucrt:api-ms-win-crt-runtime-l1-1-0.dll
 0002:000007a0       __imp__errno               000000014004b7a0     ucrt:api-ms-win-crt-runtime-l1-1-0.dll
 0002:000007a8       \177api-ms-win-crt-runtime-l1-1-0_NULL_THUNK_DATA 000000014004b7a8     ucrt:api-ms-win-crt-runtime-l1-1-0.dll
 0002:000007b0       __imp___acrt_iob_func      000000014004b7b0     ucrt:api-ms-win-crt-stdio-l1-1-0.dll
 0002:000007b8       __imp___stdio_common_vsnwprintf_s 000000014004b7b8     ucrt:api-ms-win-crt-stdio-l1-1-0.dll
 0002:000007c0       __imp_fwrite               000000014004b7c0     ucrt:api-ms-win-crt-stdio-l1-1-0.dll
 0002:000007c8       __imp___stdio_common_vsprintf 000000014004b7c8     ucrt:api-ms-win-crt-stdio-l1-1-0.dll
 0002:000007d0       __imp___p__commode         000000014004b7d0     ucrt:api-ms-win-crt-stdio-l1-1-0.dll
 0002:000007d8       __imp_fopen                000000014004b7d8     ucrt:api-ms-win-crt-stdio-l1-1-0.dll
 0002:000007e0       __imp___stdio_common_vsscanf 000000014004b7e0     ucrt:api-ms-win-crt-stdio-l1-1-0.dll
 0002:000007e8       __imp__setmaxstdio         000000014004b7e8     ucrt:api-ms-win-crt-stdio-l1-1-0.dll
 0002:000007f0       __imp___stdio_common_vsnprintf_s 000000014004b7f0     ucrt:api-ms-win-crt-stdio-l1-1-0.dll
 0002:000007f8       __imp___stdio_common_vfprintf 000000014004b7f8     ucrt:api-ms-win-crt-stdio-l1-1-0.dll
 0002:00000800       __imp_fread                000000014004b800     ucrt:api-ms-win-crt-stdio-l1-1-0.dll
 0002:00000808       __imp_fopen_s              000000014004b808     ucrt:api-ms-win-crt-stdio-l1-1-0.dll
 0002:00000810       __imp___stdio_common_vsprintf_s 000000014004b810     ucrt:api-ms-win-crt-stdio-l1-1-0.dll
 0002:00000818       __imp_fclose               000000014004b818     ucrt:api-ms-win-crt-stdio-l1-1-0.dll
 0002:00000820       __imp_fputs                000000014004b820     ucrt:api-ms-win-crt-stdio-l1-1-0.dll
 0002:00000828       __imp__set_fmode           000000014004b828     ucrt:api-ms-win-crt-stdio-l1-1-0.dll
 0002:00000830       \177api-ms-win-crt-stdio-l1-1-0_NULL_THUNK_DATA 000000014004b830     ucrt:api-ms-win-crt-stdio-l1-1-0.dll
 0002:00000838       __imp_strncmp              000000014004b838     ucrt:api-ms-win-crt-string-l1-1-0.dll
 0002:00000840       __imp_strncpy_s            000000014004b840     ucrt:api-ms-win-crt-string-l1-1-0.dll
 0002:00000848       __imp_strcpy_s             000000014004b848     ucrt:api-ms-win-crt-string-l1-1-0.dll
 0002:00000850       __imp__stricmp             000000014004b850     ucrt:api-ms-win-crt-string-l1-1-0.dll
 0002:00000858       __imp_wcscpy_s             000000014004b858     ucrt:api-ms-win-crt-string-l1-1-0.dll
 0002:00000860       __imp_isspace              000000014004b860     ucrt:api-ms-win-crt-string-l1-1-0.dll
 0002:00000868       __imp__wcsicmp             000000014004b868     ucrt:api-ms-win-crt-string-l1-1-0.dll
 0002:00000870       __imp_strcat_s             000000014004b870     ucrt:api-ms-win-crt-string-l1-1-0.dll
 0002:00000878       __imp_strncpy              000000014004b878     ucrt:api-ms-win-crt-string-l1-1-0.dll
 0002:00000880       __imp_toupper              000000014004b880     ucrt:api-ms-win-crt-string-l1-1-0.dll
 0002:00000888       __imp_strcmp               000000014004b888     ucrt:api-ms-win-crt-string-l1-1-0.dll
 0002:00000890       \177api-ms-win-crt-string-l1-1-0_NULL_THUNK_DATA 000000014004b890     ucrt:api-ms-win-crt-string-l1-1-0.dll
 0002:00000898       __imp_strftime             000000014004b898     ucrt:api-ms-win-crt-time-l1-1-0.dll
 0002:000008a0       __imp__time32              000000014004b8a0     ucrt:api-ms-win-crt-time-l1-1-0.dll
 0002:000008a8       __imp__time64              000000014004b8a8     ucrt:api-ms-win-crt-time-l1-1-0.dll
 0002:000008b0       __imp__localtime64         000000014004b8b0     ucrt:api-ms-win-crt-time-l1-1-0.dll
 0002:000008b8       \177api-ms-win-crt-time-l1-1-0_NULL_THUNK_DATA 000000014004b8b8     ucrt:api-ms-win-crt-time-l1-1-0.dll
 0002:000008c0       __imp_SymGetModuleBase64   000000014004b8c0     DbgHelp:dbghelp.dll
 0002:000008c8       __imp_StackWalk64          000000014004b8c8     DbgHelp:dbghelp.dll
 0002:000008d0       __imp_MiniDumpWriteDump    000000014004b8d0     DbgHelp:dbghelp.dll
 0002:000008d8       __imp_EnumerateLoadedModules64 000000014004b8d8     DbgHelp:dbghelp.dll
 0002:000008e0       __imp_SymFunctionTableAccess64 000000014004b8e0     DbgHelp:dbghelp.dll
 0002:000008e8       __imp_SymInitialize        000000014004b8e8     DbgHelp:dbghelp.dll
 0002:000008f0       __imp_SymSetOptions        000000014004b8f0     DbgHelp:dbghelp.dll
 0002:000008f8       __imp_SymCleanup           000000014004b8f8     DbgHelp:dbghelp.dll
 0002:00000900       \177dbghelp_NULL_THUNK_DATA 000000014004b900     DbgHelp:dbghelp.dll
 0002:00000908       __imp_??3@YAXPEAX@Z        000000014004b908     mfc140:mfc140.dll
 0002:00000910       __imp_??2@YAPEAX_K@Z       000000014004b910     mfc140:mfc140.dll
 0002:00000918       __imp_??_V@YAXPEAX@Z       000000014004b918     mfc140:mfc140.dll
 0002:00000920       __imp_??_U@YAPEAX_K@Z      000000014004b920     mfc140:mfc140.dll
 0002:00000928       __imp_?SetProxy@CWnd@@UEAAJPEAUIAccessibleProxy@@@Z 000000014004b928     mfc140:mfc140.dll
 0002:00000930       __imp_?put_accValue@CWnd@@UEAAJUtagVARIANT@@PEA_W@Z 000000014004b930     mfc140:mfc140.dll
 0002:00000938       __imp_?put_accName@CWnd@@UEAAJUtagVARIANT@@PEA_W@Z 000000014004b938     mfc140:mfc140.dll
 0002:00000940       __imp_?accDoDefaultAction@CWnd@@UEAAJUtagVARIANT@@@Z 000000014004b940     mfc140:mfc140.dll
 0002:00000948       __imp_?accHitTest@CWnd@@UEAAJJJPEAUtagVARIANT@@@Z 000000014004b948     mfc140:mfc140.dll
 0002:00000950       __imp_?accNavigate@CWnd@@UEAAJJUtagVARIANT@@PEAU2@@Z 000000014004b950     mfc140:mfc140.dll
 0002:00000958       __imp_??0CDialog@@QEAA@IPEAVCWnd@@@Z 000000014004b958     mfc140:mfc140.dll
 0002:00000960       __imp_??1CDialog@@UEAA@XZ  000000014004b960     mfc140:mfc140.dll
 0002:00000968       __imp_?GetOccDialogInfo@CWnd@@MEAAPEAU_AFX_OCC_DIALOG_INFO@@XZ 000000014004b968     mfc140:mfc140.dll
 0002:00000970       __imp_?SetOccDialogInfo@CWnd@@MEAAHPEAU_AFX_OCC_DIALOG_INFO@@@Z 000000014004b970     mfc140:mfc140.dll
 0002:00000978       __imp_?CreateControlSite@CWnd@@MEAAHPEAVCOleControlContainer@@PEAPEAVCOleControlSite@@IAEBU_GUID@@@Z 000000014004b978     mfc140:mfc140.dll
 0002:00000980       __imp_?CreateControlContainer@CWnd@@MEAAHPEAPEAVCOleControlContainer@@@Z 000000014004b980     mfc140:mfc140.dll
 0002:00000988       __imp_?CreateAccessibleProxy@CWnd@@UEAAJ_K_JPEA_J@Z 000000014004b988     mfc140:mfc140.dll
 0002:00000990       __imp_?CheckAutoCenter@CWnd@@UEAAHXZ 000000014004b990     mfc140:mfc140.dll
 0002:00000998       __imp_?accLocation@CWnd@@UEAAJPEAJ000UtagVARIANT@@@Z 000000014004b998     mfc140:mfc140.dll
 0002:000009a0       __imp_?accSelect@CWnd@@UEAAJJUtagVARIANT@@@Z 000000014004b9a0     mfc140:mfc140.dll
 0002:000009a8       __imp_?get_accDefaultAction@CWnd@@UEAAJUtagVARIANT@@PEAPEA_W@Z 000000014004b9a8     mfc140:mfc140.dll
 0002:000009b0       __imp_?get_accSelection@CWnd@@UEAAJPEAUtagVARIANT@@@Z 000000014004b9b0     mfc140:mfc140.dll
 0002:000009b8       __imp_?get_accFocus@CWnd@@UEAAJPEAUtagVARIANT@@@Z 000000014004b9b8     mfc140:mfc140.dll
 0002:000009c0       __imp_?get_accKeyboardShortcut@CWnd@@UEAAJUtagVARIANT@@PEAPEA_W@Z 000000014004b9c0     mfc140:mfc140.dll
 0002:000009c8       __imp_?get_accHelpTopic@CWnd@@UEAAJPEAPEA_WUtagVARIANT@@PEAJ@Z 000000014004b9c8     mfc140:mfc140.dll
 0002:000009d0       __imp_?get_accHelp@CWnd@@UEAAJUtagVARIANT@@PEAPEA_W@Z 000000014004b9d0     mfc140:mfc140.dll
 0002:000009d8       __imp_?get_accState@CWnd@@UEAAJUtagVARIANT@@PEAU2@@Z 000000014004b9d8     mfc140:mfc140.dll
 0002:000009e0       __imp_?get_accRole@CWnd@@UEAAJUtagVARIANT@@PEAU2@@Z 000000014004b9e0     mfc140:mfc140.dll
 0002:000009e8       __imp_?get_accDescription@CWnd@@UEAAJUtagVARIANT@@PEAPEA_W@Z 000000014004b9e8     mfc140:mfc140.dll
 0002:000009f0       __imp_?get_accValue@CWnd@@UEAAJUtagVARIANT@@PEAPEA_W@Z 000000014004b9f0     mfc140:mfc140.dll
 0002:000009f8       __imp_?get_accName@CWnd@@UEAAJUtagVARIANT@@PEAPEA_W@Z 000000014004b9f8     mfc140:mfc140.dll
 0002:00000a00       __imp_?get_accChild@CWnd@@UEAAJUtagVARIANT@@PEAPEAUIDispatch@@@Z 000000014004ba00     mfc140:mfc140.dll
 0002:00000a08       __imp_?get_accChildCount@CWnd@@UEAAJPEAJ@Z 000000014004ba08     mfc140:mfc140.dll
 0002:00000a10       __imp_?get_accParent@CWnd@@UEAAJPEAPEAUIDispatch@@@Z 000000014004ba10     mfc140:mfc140.dll
 0002:00000a18       __imp_?EnsureStdObj@CWnd@@UEAAJXZ 000000014004ba18     mfc140:mfc140.dll
 0002:00000a20       __imp_?OnDrawIconicThumbnailOrLivePreview@CWnd@@UEAAXAEAVCDC@@VCRect@@VCSize@@HAEAH@Z 000000014004ba20     mfc140:mfc140.dll
 0002:00000a28       __imp_?EndModalLoop@CWnd@@UEAAXH@Z 000000014004ba28     mfc140:mfc140.dll
 0002:00000a30       __imp_?ContinueModal@CWnd@@UEAAHXZ 000000014004ba30     mfc140:mfc140.dll
 0002:00000a38       __imp_?WinHelpInternal@CWnd@@UEAAX_KI@Z 000000014004ba38     mfc140:mfc140.dll
 0002:00000a40       __imp_?HtmlHelpA@CWnd@@UEAAX_KI@Z 000000014004ba40     mfc140:mfc140.dll
 0002:00000a48       __imp_?WinHelpA@CWnd@@UEAAX_KI@Z 000000014004ba48     mfc140:mfc140.dll
 0002:00000a50       __imp_?GetScrollBarCtrl@CWnd@@UEBAPEAVCScrollBar@@H@Z 000000014004ba50     mfc140:mfc140.dll
 0002:00000a58       __imp_?OnToolHitTest@CWnd@@UEBA_JVCPoint@@PEAUtagTOOLINFOA@@@Z 000000014004ba58     mfc140:mfc140.dll
 0002:00000a60       __imp_?SetMenu@CWnd@@UEAAHPEAVCMenu@@@Z 000000014004ba60     mfc140:mfc140.dll
 0002:00000a68       __imp_?GetMenu@CWnd@@UEBAPEAVCMenu@@XZ 000000014004ba68     mfc140:mfc140.dll
 0002:00000a70       __imp_?CalcWindowRect@CWnd@@UEAAXPEAUtagRECT@@I@Z 000000014004ba70     mfc140:mfc140.dll
 0002:00000a78       __imp_?PreCreateWindow@CWnd@@UEAAHAEAUtagCREATESTRUCTA@@@Z 000000014004ba78     mfc140:mfc140.dll
 0002:00000a80       __imp_?DestroyWindow@CWnd@@UEAAHXZ 000000014004ba80     mfc140:mfc140.dll
 0002:00000a88       __imp_?CreateEx@CWnd@@UEAAHKPEBD0KHHHHPEAUHWND__@@PEAUHMENU__@@PEAX@Z 000000014004ba88     mfc140:mfc140.dll
 0002:00000a90       __imp_?CreateEx@CWnd@@UEAAHKPEBD0KAEBUtagRECT@@PEAV1@IPEAX@Z 000000014004ba90     mfc140:mfc140.dll
 0002:00000a98       __imp_?Create@CWnd@@UEAAHPEBD0KAEBUtagRECT@@PEAV1@IPEAUCCreateContext@@@Z 000000014004ba98     mfc140:mfc140.dll
 0002:00000aa0       __imp_?PreSubclassWindow@CWnd@@UEAAXXZ 000000014004baa0     mfc140:mfc140.dll
 0002:00000aa8       __imp_?GetConnectionHook@CCmdTarget@@MEAAPEAUIConnectionPoint@@AEBU_GUID@@@Z 000000014004baa8     mfc140:mfc140.dll
 0002:00000ab0       __imp_?GetExtraConnectionPoints@CCmdTarget@@MEAAHPEAVCPtrArray@@@Z 000000014004bab0     mfc140:mfc140.dll
 0002:00000ab8       __imp_?GetInterfaceHook@CCmdTarget@@UEAAPEAUIUnknown@@PEBX@Z 000000014004bab8     mfc140:mfc140.dll
 0002:00000ac0       __imp_?OnCreateAggregates@CCmdTarget@@UEAAHXZ 000000014004bac0     mfc140:mfc140.dll
 0002:00000ac8       __imp_?GetEventSinkMap@CCmdTarget@@MEBAPEBUAFX_EVENTSINKMAP@@XZ 000000014004bac8     mfc140:mfc140.dll
 0002:00000ad0       __imp_?GetInterfaceMap@CWnd@@MEBAPEBUAFX_INTERFACEMAP@@XZ 000000014004bad0     mfc140:mfc140.dll
 0002:00000ad8       __imp_?GetConnectionMap@CCmdTarget@@MEBAPEBUAFX_CONNECTIONMAP@@XZ 000000014004bad8     mfc140:mfc140.dll
 0002:00000ae0       __imp_?GetDispatchMap@CCmdTarget@@MEBAPEBUAFX_DISPMAP@@XZ 000000014004bae0     mfc140:mfc140.dll
 0002:00000ae8       __imp_?GetCommandMap@CCmdTarget@@MEBAPEBUAFX_OLECMDMAP@@XZ 000000014004bae8     mfc140:mfc140.dll
 0002:00000af0       __imp_?GetMessageMap@CWnd@@MEBAPEBUAFX_MSGMAP@@XZ 000000014004baf0     mfc140:mfc140.dll
 0002:00000af8       __imp_?GetTypeLib@CCmdTarget@@UEAAJKPEAPEAUITypeLib@@@Z 000000014004baf8     mfc140:mfc140.dll
 0002:00000b00       __imp_?GetTypeLibCache@CCmdTarget@@UEAAPEAVCTypeLibCache@@XZ 000000014004bb00     mfc140:mfc140.dll
 0002:00000b08       __imp_?GetTypeInfoCount@CCmdTarget@@UEAAIXZ 000000014004bb08     mfc140:mfc140.dll
 0002:00000b10       __imp_?GetDispatchIID@CCmdTarget@@UEAAHPEAU_GUID@@@Z 000000014004bb10     mfc140:mfc140.dll
 0002:00000b18       __imp_?IsInvokeAllowed@CCmdTarget@@UEAAHJ@Z 000000014004bb18     mfc140:mfc140.dll
 0002:00000b20       __imp_?ResizeDynamicLayout@CWnd@@MEAAXXZ 000000014004bb20     mfc140:mfc140.dll
 0002:00000b28       __imp_?OnGesturePressAndTap@CWnd@@MEAAHVCPoint@@J@Z 000000014004bb28     mfc140:mfc140.dll
 0002:00000b30       __imp_?OnFinalRelease@CWnd@@UEAAXXZ 000000014004bb30     mfc140:mfc140.dll
 0002:00000b38       __imp_?OnCmdMsg@CCmdTarget@@UEAAHIHPEAXPEAUAFX_CMDHANDLERINFO@@@Z 000000014004bb38     mfc140:mfc140.dll
 0002:00000b40       __imp_?GetRuntimeClass@CEdit@@UEBAPEAUCRuntimeClass@@XZ 000000014004bb40     mfc140:mfc140.dll
 0002:00000b48       __imp_??0CWnd@@QEAA@XZ     000000014004bb48     mfc140:mfc140.dll
 0002:00000b50       __imp_??1CEdit@@UEAA@XZ    000000014004bb50     mfc140:mfc140.dll
 0002:00000b58       __imp_?OnGestureTwoFingerTap@CWnd@@MEAAHVCPoint@@@Z 000000014004bb58     mfc140:mfc140.dll
 0002:00000b60       __imp_?DDX_Control@@YAXPEAVCDataExchange@@HAEAVCWnd@@@Z 000000014004bb60     mfc140:mfc140.dll
 0002:00000b68       __imp_?GetThisMessageMap@CDialog@@KAPEBUAFX_MSGMAP@@XZ 000000014004bb68     mfc140:mfc140.dll
 0002:00000b70       __imp_??0?$CStringT@DV?$StrTraitMFC_DLL@DV?$ChTraitsCRT@D@ATL@@@@@ATL@@QEAA@XZ 000000014004bb70     mfc140:mfc140.dll
 0002:00000b78       __imp_??1?$CStringT@DV?$StrTraitMFC_DLL@DV?$ChTraitsCRT@D@ATL@@@@@ATL@@QEAA@XZ 000000014004bb78     mfc140:mfc140.dll
 0002:00000b80       __imp_?OnInitDialog@CDialog@@UEAAHXZ 000000014004bb80     mfc140:mfc140.dll
 0002:00000b88       __imp_?Default@CWnd@@IEAA_JXZ 000000014004bb88     mfc140:mfc140.dll
 0002:00000b90       __imp_?OnCmdMsg@CDialog@@UEAAHIHPEAXPEAUAFX_CMDHANDLERINFO@@@Z 000000014004bb90     mfc140:mfc140.dll
 0002:00000b98       __imp_?PreTranslateMessage@CDialog@@UEAAHPEAUtagMSG@@@Z 000000014004bb98     mfc140:mfc140.dll
 0002:00000ba0       __imp_?CheckAutoCenter@CDialog@@UEAAHXZ 000000014004bba0     mfc140:mfc140.dll
 0002:00000ba8       __imp_?SetOccDialogInfo@CDialog@@MEAAHPEAU_AFX_OCC_DIALOG_INFO@@@Z 000000014004bba8     mfc140:mfc140.dll
 0002:00000bb0       __imp_?GetOccDialogInfo@CDialog@@MEAAPEAU_AFX_OCC_DIALOG_INFO@@XZ 000000014004bbb0     mfc140:mfc140.dll
 0002:00000bb8       __imp_?Create@CDialog@@UEAAHPEBDPEAVCWnd@@@Z 000000014004bbb8     mfc140:mfc140.dll
 0002:00000bc0       __imp_?CreateIndirect@CDialog@@UEAAHPEAXPEAVCWnd@@@Z 000000014004bbc0     mfc140:mfc140.dll
 0002:00000bc8       __imp_?CreateIndirect@CDialog@@UEAAHPEBUDLGTEMPLATE@@PEAVCWnd@@PEAX@Z 000000014004bbc8     mfc140:mfc140.dll
 0002:00000bd0       __imp_?DoModal@CDialog@@UEAA_JXZ 000000014004bbd0     mfc140:mfc140.dll
 0002:00000bd8       __imp_?OnSetFont@CDialog@@UEAAXPEAVCFont@@@Z 000000014004bbd8     mfc140:mfc140.dll
 0002:00000be0       __imp_?OnOK@CDialog@@MEAAXXZ 000000014004bbe0     mfc140:mfc140.dll
 0002:00000be8       __imp_?OnGestureRotate@CWnd@@MEAAHVCPoint@@N@Z 000000014004bbe8     mfc140:mfc140.dll
 0002:00000bf0       __imp_?OnCancel@CDialog@@MEAAXXZ 000000014004bbf0     mfc140:mfc140.dll
 0002:00000bf8       __imp_?PreInitDialog@CDialog@@MEAAXXZ 000000014004bbf8     mfc140:mfc140.dll
 0002:00000c00       __imp_??Y?$CStringT@DV?$StrTraitMFC_DLL@DV?$ChTraitsCRT@D@ATL@@@@@ATL@@QEAAAEAV01@PEBD@Z 000000014004bc00     mfc140:mfc140.dll
 0002:00000c08       __imp_?OnHelp@CWinApp@@IEAAXXZ 000000014004bc08     mfc140:mfc140.dll
 0002:00000c10       __imp_?GetThisMessageMap@CWinApp@@KAPEBUAFX_MSGMAP@@XZ 000000014004bc10     mfc140:mfc140.dll
 0002:00000c18       __imp_??0CWinApp@@QEAA@PEBD@Z 000000014004bc18     mfc140:mfc140.dll
 0002:00000c20       __imp_?OnGesturePan@CWnd@@MEAAHVCPoint@@0@Z 000000014004bc20     mfc140:mfc140.dll
 0002:00000c28       __imp_??1CWinApp@@UEAA@XZ  000000014004bc28     mfc140:mfc140.dll
 0002:00000c30       __imp_?GetRuntimeClass@CWinApp@@UEBAPEAUCRuntimeClass@@XZ 000000014004bc30     mfc140:mfc140.dll
 0002:00000c38       __imp_?OnFinalRelease@CCmdTarget@@UEAAXXZ 000000014004bc38     mfc140:mfc140.dll
 0002:00000c40       __imp_?GetInterfaceMap@CCmdTarget@@MEBAPEBUAFX_INTERFACEMAP@@XZ 000000014004bc40     mfc140:mfc140.dll
 0002:00000c48       __imp_?Run@CWinApp@@UEAAHXZ 000000014004bc48     mfc140:mfc140.dll
 0002:00000c50       __imp_?OnGestureZoom@CWnd@@MEAAHVCPoint@@J@Z 000000014004bc50     mfc140:mfc140.dll
 0002:00000c58       __imp_?PreTranslateMessage@CWinThread@@UEAAHPEAUtagMSG@@@Z 000000014004bc58     mfc140:mfc140.dll
 0002:00000c60       __imp_?PumpMessage@CWinThread@@UEAAHXZ 000000014004bc60     mfc140:mfc140.dll
 0002:00000c68       __imp_?OnIdle@CWinApp@@UEAAHJ@Z 000000014004bc68     mfc140:mfc140.dll
 0002:00000c70       __imp_?IsIdleMessage@CWinThread@@UEAAHPEAUtagMSG@@@Z 000000014004bc70     mfc140:mfc140.dll
 0002:00000c78       __imp_?ExitInstance@CWinApp@@UEAAHXZ 000000014004bc78     mfc140:mfc140.dll
 0002:00000c80       __imp_?ProcessWndProcException@CWinApp@@UEAA_JPEAVCException@@PEBUtagMSG@@@Z 000000014004bc80     mfc140:mfc140.dll
 0002:00000c88       __imp_?ProcessMessageFilter@CWinThread@@UEAAHHPEAUtagMSG@@@Z 000000014004bc88     mfc140:mfc140.dll
 0002:00000c90       __imp_?GetMainWnd@CWinThread@@UEAAPEAVCWnd@@XZ 000000014004bc90     mfc140:mfc140.dll
 0002:00000c98       __imp_?Delete@CWinThread@@UEAAXXZ 000000014004bc98     mfc140:mfc140.dll
 0002:00000ca0       __imp_?GetProfileIntA@CWinApp@@UEAAIPEBD0H@Z 000000014004bca0     mfc140:mfc140.dll
 0002:00000ca8       __imp_?WriteProfileInt@CWinApp@@UEAAHPEBD0H@Z 000000014004bca8     mfc140:mfc140.dll
 0002:00000cb0       __imp_?GetProfileStringA@CWinApp@@UEAA?AV?$CStringT@DV?$StrTraitMFC_DLL@DV?$ChTraitsCRT@D@ATL@@@@@ATL@@PEBD00@Z 000000014004bcb0     mfc140:mfc140.dll
 0002:00000cb8       __imp_?WriteProfileStringA@CWinApp@@UEAAHPEBD00@Z 000000014004bcb8     mfc140:mfc140.dll
 0002:00000cc0       __imp_?GetProfileBinary@CWinApp@@UEAAHPEBD0PEAPEAEPEAI@Z 000000014004bcc0     mfc140:mfc140.dll
 0002:00000cc8       __imp_?WriteProfileBinary@CWinApp@@UEAAHPEBD0PEAEI@Z 000000014004bcc8     mfc140:mfc140.dll
 0002:00000cd0       __imp_?InitLibId@CWinApp@@UEAAXXZ 000000014004bcd0     mfc140:mfc140.dll
 0002:00000cd8       __imp_?Register@CWinApp@@UEAAHXZ 000000014004bcd8     mfc140:mfc140.dll
 0002:00000ce0       __imp_?GetGestureStatus@CWnd@@MEAAKVCPoint@@@Z 000000014004bce0     mfc140:mfc140.dll
 0002:00000ce8       __imp_?Unregister@CWinApp@@UEAAHXZ 000000014004bce8     mfc140:mfc140.dll
 0002:00000cf0       __imp_?OpenDocumentFile@CWinApp@@UEAAPEAVCDocument@@PEBDH@Z 000000014004bcf0     mfc140:mfc140.dll
 0002:00000cf8       __imp_?OpenDocumentFile@CWinApp@@UEAAPEAVCDocument@@PEBD@Z 000000014004bcf8     mfc140:mfc140.dll
 0002:00000d00       __imp_?AddToRecentFileList@CWinApp@@UEAAXPEBD@Z 000000014004bd00     mfc140:mfc140.dll
 0002:00000d08       __imp_?InitApplication@CWinApp@@UEAAHXZ 000000014004bd08     mfc140:mfc140.dll
 0002:00000d10       __imp_?SaveAllModified@CWinApp@@UEAAHXZ 000000014004bd10     mfc140:mfc140.dll
 0002:00000d18       __imp_?DoMessageBox@CWinApp@@UEAAHPEBDII@Z 000000014004bd18     mfc140:mfc140.dll
 0002:00000d20       __imp_?DoWaitCursor@CWinApp@@UEAAXH@Z 000000014004bd20     mfc140:mfc140.dll
 0002:00000d28       __imp_?OnDDECommand@CWinApp@@UEAAHPEAD@Z 000000014004bd28     mfc140:mfc140.dll
 0002:00000d30       __imp_?WinHelpA@CWinApp@@UEAAX_KI@Z 000000014004bd30     mfc140:mfc140.dll
 0002:00000d38       __imp_?HtmlHelpA@CWinApp@@UEAAX_KI@Z 000000014004bd38     mfc140:mfc140.dll
 0002:00000d40       __imp_?WinHelpInternal@CWinApp@@UEAAX_KI@Z 000000014004bd40     mfc140:mfc140.dll
 0002:00000d48       __imp_?RegisterWithRestartManager@CWinApp@@UEAAJPEB_WKP6AKPEAX@Z1KK@Z 000000014004bd48     mfc140:mfc140.dll
 0002:00000d50       __imp_?RegisterWithRestartManager@CWinApp@@UEAAJHAEBV?$CStringT@DV?$StrTraitMFC_DLL@DV?$ChTraitsCRT@D@ATL@@@@@ATL@@@Z 000000014004bd50     mfc140:mfc140.dll
 0002:00000d58       __imp_?ApplicationRecoveryCallback@CWinApp@@UEAAKPEAX@Z 000000014004bd58     mfc140:mfc140.dll
 0002:00000d60       __imp_?GetDataRecoveryHandler@CWinApp@@UEAAPEAVCDataRecoveryHandler@@XZ 000000014004bd60     mfc140:mfc140.dll
 0002:00000d68       __imp_?IsTaskbarInteractionEnabled@CWinApp@@UEAAHXZ 000000014004bd68     mfc140:mfc140.dll
 0002:00000d70       __imp_?RestartInstance@CWinApp@@UEAAHXZ 000000014004bd70     mfc140:mfc140.dll
 0002:00000d78       __imp_?LoadAppLangResourceDLL@CWinApp@@UEAAPEAUHINSTANCE__@@XZ 000000014004bd78     mfc140:mfc140.dll
 0002:00000d80       __imp_?Left@?$CStringT@DV?$StrTraitMFC_DLL@DV?$ChTraitsCRT@D@ATL@@@@@ATL@@QEBA?AV12@H@Z 000000014004bd80     mfc140:mfc140.dll
 0002:00000d88       __imp_?Mid@?$CStringT@DV?$StrTraitMFC_DLL@DV?$ChTraitsCRT@D@ATL@@@@@ATL@@QEBA?AV12@H@Z 000000014004bd88     mfc140:mfc140.dll
 0002:00000d90       __imp_?FindOneOf@?$CStringT@DV?$StrTraitMFC_DLL@DV?$ChTraitsCRT@D@ATL@@@@@ATL@@QEBAHPEBD@Z 000000014004bd90     mfc140:mfc140.dll
 0002:00000d98       __imp_?Compare@?$CStringT@DV?$StrTraitMFC_DLL@DV?$ChTraitsCRT@D@ATL@@@@@ATL@@QEBAHPEBD@Z 000000014004bd98     mfc140:mfc140.dll
 0002:00000da0       __imp_??Y?$CStringT@DV?$StrTraitMFC_DLL@DV?$ChTraitsCRT@D@ATL@@@@@ATL@@QEAAAEAV01@AEBV?$CSimpleStringT@D$00@1@@Z 000000014004bda0     mfc140:mfc140.dll
 0002:00000da8       __imp_?GetBuffer@?$CSimpleStringT@D$00@ATL@@QEAAPEADXZ 000000014004bda8     mfc140:mfc140.dll
 0002:00000db0       __imp_?GetRuntimeClass@CDialog@@UEBAPEAUCRuntimeClass@@XZ 000000014004bdb0     mfc140:mfc140.dll
 0002:00000db8       __imp_?AfxFreeLibrary@@YAHPEAUHINSTANCE__@@@Z 000000014004bdb8     mfc140:mfc140.dll
 0002:00000dc0       __imp_?AfxThrowInvalidArgException@@YAXXZ 000000014004bdc0     mfc140:mfc140.dll
 0002:00000dc8       __imp_?Close@CFileFind@@QEAAXXZ 000000014004bdc8     mfc140:mfc140.dll
 0002:00000dd0       __imp_?AddTail@CStringList@@QEAAPEAU__POSITION@@AEBV?$CStringT@DV?$StrTraitMFC_DLL@DV?$ChTraitsCRT@D@ATL@@@@@ATL@@@Z 000000014004bdd0     mfc140:mfc140.dll
 0002:00000dd8       __imp_?GetFileName@CFileFind@@UEBA?AV?$CStringT@DV?$StrTraitMFC_DLL@DV?$ChTraitsCRT@D@ATL@@@@@ATL@@XZ 000000014004bdd8     mfc140:mfc140.dll
 0002:00000de0       __imp_?IsDots@CFileFind@@UEBAHXZ 000000014004bde0     mfc140:mfc140.dll
 0002:00000de8       __imp_?FindNextFileA@CFileFind@@UEAAHXZ 000000014004bde8     mfc140:mfc140.dll
 0002:00000df0       __imp_?FindFile@CFileFind@@UEAAHPEBDK@Z 000000014004bdf0     mfc140:mfc140.dll
 0002:00000df8       __imp_??1CFileFind@@UEAA@XZ 000000014004bdf8     mfc140:mfc140.dll
 0002:00000e00       __imp_??0CFileFind@@QEAA@XZ 000000014004be00     mfc140:mfc140.dll
 0002:00000e08       __imp_??1CStringList@@UEAA@XZ 000000014004be08     mfc140:mfc140.dll
 0002:00000e10       __imp_??0CStringList@@QEAA@_J@Z 000000014004be10     mfc140:mfc140.dll
 0002:00000e18       __imp_?AfxLoadLibrary@@YAPEAUHINSTANCE__@@PEBD@Z 000000014004be18     mfc140:mfc140.dll
 0002:00000e20       __imp_?AfxBeginThread@@YAPEAVCWinThread@@P6AIPEAX@Z0HIKPEAU_SECURITY_ATTRIBUTES@@@Z 000000014004be20     mfc140:mfc140.dll
 0002:00000e28       __imp_?UpdateData@CWnd@@QEAAHH@Z 000000014004be28     mfc140:mfc140.dll
 0002:00000e30       __imp_?OnPaint@CDialog@@IEAAXXZ 000000014004be30     mfc140:mfc140.dll
 0002:00000e38       __imp_??1CPaintDC@@UEAA@XZ 000000014004be38     mfc140:mfc140.dll
 0002:00000e40       __imp_?OnTouchInput@CWnd@@MEAAHVCPoint@@HHPEAUtagTOUCHINPUT@@@Z 000000014004be40     mfc140:mfc140.dll
 0002:00000e48       __imp_??0CPaintDC@@QEAA@PEAVCWnd@@@Z 000000014004be48     mfc140:mfc140.dll
 0002:00000e50       __imp_?OnTouchInputs@CWnd@@MEAAHIPEAUtagTOUCHINPUT@@@Z 000000014004be50     mfc140:mfc140.dll
 0002:00000e58       __imp_?DDX_Text@@YAXPEAVCDataExchange@@HAEAV?$CStringT@DV?$StrTraitMFC_DLL@DV?$ChTraitsCRT@D@ATL@@@@@ATL@@@Z 000000014004be58     mfc140:mfc140.dll
 0002:00000e60       __imp_?AfxGetModuleState@@YAPEAVAFX_MODULE_STATE@@XZ 000000014004be60     mfc140:mfc140.dll
 0002:00000e68       __imp_?AfxFindResourceHandle@@YAPEAUHINSTANCE__@@PEBD0@Z 000000014004be68     mfc140:mfc140.dll
 0002:00000e70       __imp_?Empty@?$CSimpleStringT@D$00@ATL@@QEAAXXZ 000000014004be70     mfc140:mfc140.dll
 0002:00000e78       __imp_?OnChildNotify@CWnd@@MEAAHI_K_JPEA_J@Z 000000014004be78     mfc140:mfc140.dll
 0002:00000e80       __imp_?PostNcDestroy@CWnd@@MEAAXXZ 000000014004be80     mfc140:mfc140.dll
 0002:00000e88       __imp_?DefWindowProcA@CWnd@@MEAA_JI_K_J@Z 000000014004be88     mfc140:mfc140.dll
 0002:00000e90       __imp_?OnWndMsg@CWnd@@MEAAHI_K_JPEA_J@Z 000000014004be90     mfc140:mfc140.dll
 0002:00000e98       __imp_?WindowProc@CWnd@@MEAA_JI_K_J@Z 000000014004be98     mfc140:mfc140.dll
 0002:00000ea0       __imp_?OnAmbientProperty@CWnd@@UEAAHPEAVCOleControlSite@@JPEAUtagVARIANT@@@Z 000000014004bea0     mfc140:mfc140.dll
 0002:00000ea8       __imp_?PreTranslateMessage@CWnd@@UEAAHPEAUtagMSG@@@Z 000000014004bea8     mfc140:mfc140.dll
 0002:00000eb0       __imp_?GetSuperWndProcAddr@CWnd@@MEAAPEAP6A_JPEAUHWND__@@I_K_J@ZXZ 000000014004beb0     mfc140:mfc140.dll
 0002:00000eb8       __imp_?OnNotify@CWnd@@MEAAH_K_JPEA_J@Z 000000014004beb8     mfc140:mfc140.dll
 0002:00000ec0       __imp_?OnCommand@CWnd@@MEAAH_K_J@Z 000000014004bec0     mfc140:mfc140.dll
 0002:00000ec8       __imp_??4?$CStringT@DV?$StrTraitMFC_DLL@DV?$ChTraitsCRT@D@ATL@@@@@ATL@@QEAAAEAV01@PEBD@Z 000000014004bec8     mfc140:mfc140.dll
 0002:00000ed0       __imp_?IsFrameWnd@CWnd@@UEBAHXZ 000000014004bed0     mfc140:mfc140.dll
 0002:00000ed8       __imp_?AfxWinMain@@YAHPEAUHINSTANCE__@@0PEADH@Z 000000014004bed8     mfc140:mfc140.dll
 0002:00000ee0       __imp_?LoadSysPolicies@CWinApp@@UEAAHXZ 000000014004bee0     mfc140:mfc140.dll
 0002:00000ee8       \177mfc140_NULL_THUNK_DATA 000000014004bee8     mfc140:mfc140.dll
 0002:00000ef0       __guard_check_icall_fptr   000000014004bef0     msvcrt:guard_support.obj
 0002:00000ef8       __guard_dispatch_icall_fptr 000000014004bef8     msvcrt:guard_support.obj
 0002:00000f00       __xc_a                     000000014004bf00     msvcrt:initializers.obj
 0002:00001038       __xc_z                     000000014004c038     msvcrt:initializers.obj
 0002:00001040       __xi_a                     000000014004c040     msvcrt:initializers.obj
 0002:00001060       __xi_z                     000000014004c060     msvcrt:initializers.obj
 0002:00001068       __xl_a                     000000014004c068     msvcrt:tlssup.obj
 0002:00001070       __xl_z                     000000014004c070     msvcrt:tlssup.obj
 0002:00001078       __xp_a                     000000014004c078     msvcrt:initializers.obj
 0002:00001080       __xp_z                     000000014004c080     msvcrt:initializers.obj
 0002:00001088       __xt_a                     000000014004c088     msvcrt:initializers.obj
 0002:00001090       __xt_z                     000000014004c090     msvcrt:initializers.obj
 0002:000010d0       ??_C@_1EC@JIJBPKFM@?$AAa?$AAp?$AAi?$AA?9?$AAm?$AAs?$AA?9?$AAw?$AAi?$AAn?$AA?9?$AAc?$AAo?$AAr?$AAe@ 000000014004c0d0     msvcrt:thread_safe_statics.obj
 0002:00001118       ??_C@_1BK@MGMFAEKH@?$AAk?$AAe?$AAr?$AAn?$AAe?$AAl?$AA3?$AA2?$AA?4?$AAd?$AAl?$AAl@ 000000014004c118     msvcrt:thread_safe_statics.obj
 0002:00001138       ??_C@_0BM@HLJJNPAH@InitializeConditionVariable@ 000000014004c138     msvcrt:thread_safe_statics.obj
 0002:00001158       ??_C@_0BJ@JEBJOJFJ@SleepConditionVariableCS@ 000000014004c158     msvcrt:thread_safe_statics.obj
 0002:00001178       ??_C@_0BJ@PGPPEPCC@WakeAllConditionVariable@ 000000014004c178     msvcrt:thread_safe_statics.obj
 0002:000011a0       ??_7type_info@@6B@         000000014004c1a0     msvcrt:std_type_info_static.obj
 0002:000011b8       GUID_ATLVer110             000000014004c1b8     atls:atlbase.obj
 0002:000011d0       ??_C@_1IC@ONKHOIDK@?$AAE?$AAR?$AAR?$AAO?$AAR?$AA?5?$AA?3?$AA?5?$AAU?$AAn?$AAa?$AAb?$AAl?$AAe?$AA?5@ 000000014004c1d0     atls:atlbase.obj
 0002:00001280       ??_C@_0BD@OLBABOEK@vector?$DMT?$DO?5too?5long@ 000000014004c280     DivisionPacket.obj
 0002:00001298       ??_C@_0BE@JONHPENG@map?1set?$DMT?$DO?5too?5long@ 000000014004c298     DivisionPacketReceiver.obj
 0002:000012b0       ??_C@_0BE@OHABKPEK@C?3?2log?2crossfire?2?$CFs@ 000000014004c2b0     BugReporter.obj
 0002:000012c8       ??_C@_0BC@OFAGFEDM@?$CFs?2?$CFsdmp_?$CFs_?$CFs_?$CFs@ 000000014004c2c8     BugReporter.obj
 0002:000012e0       ??_C@_0CC@FCEOPKOK@?$CF04d?$CF02d?$CF02d?9?$CF02d?$CF02d?$CF02d?$CF03d?4d@ 000000014004c2e0     BugReporter.obj
 0002:00001304       ??_C@_02DKCKIIND@?$CFs@    000000014004c304     BugReporter.obj
 0002:00001308       ??_C@_0BF@IAOALLHJ@C?3?2log?2crossfire?2?$CFs?2@ 000000014004c308     BugReporter.obj
 0002:00001320       ??_C@_04KBDJOJNB@?$FL?$CFd?$FN@ 000000014004c320     BugReporter.obj
 0002:00001328       ??_C@_0L@IFPJGDKC@?$CFd?$CF02d?$CF02d@ 000000014004c328     BugReporter.obj
 0002:00001338       ??_C@_0O@EMHFIMLF@?4?2Setting?4ini@ 000000014004c338     BugReporter.obj
 0002:00001348       ??_C@_08PNEMGIDK@FullDump@ 000000014004c348     BugReporter.obj
 0002:00001358       ??_C@_08NCCBLF@GameMgmt@   000000014004c358     BugReporter.obj
 0002:00001368       ??_C@_0BJ@DAFBOCMI@CRS?5Upload?5Succeeded?3?5?$CFs@ 000000014004c368     BugReporter.obj
 0002:00001388       ??_C@_0BG@LEKOEBGH@CRS?5Upload?5Failed?3?5?$CFs@ 000000014004c388     BugReporter.obj
 0002:000013a0       ??_C@_03GIOIKFCO@C?3?2@    000000014004c3a0     BugReporter.obj
 0002:000013a4       ??_C@_03MGHMBJCF@log@      000000014004c3a4     BugReporter.obj
 0002:000013a8       ??_C@_04FNMMLKAG@log?2@    000000014004c3a8     BugReporter.obj
 0002:000013b0       ??_C@_09LOKONNNP@crossfire@ 000000014004c3b0     BugReporter.obj
 0002:000013bc       ??_C@_05BMGBEOOC@?$CFs?2?$CFs@ 000000014004c3bc     BugReporter.obj
 0002:000013c4       ??_C@_01KICIPPFI@?2@       000000014004c3c4     BugReporter.obj
 0002:000013c8       ??_C@_0BA@JFNIOLAK@string?5too?5long@ 000000014004c3c8     BugReporter.obj
 0002:000013fc       ?g_dwCheckGSMOnTimerTime@@3KA 000000014004c3fc     GameServerManagerDlg.obj
 0002:00005f30       ??_C@_1BA@HDJCCPDO@?$AAC?$AAR?$AAS?$AA?4?$AAi?$AAn?$AAi@ 0000000140050f30     crs_uploader.obj
 0002:00005f40       ??_C@_17BHJPJDEN@?$AAU?$AAR?$AAL@ 0000000140050f40     crs_uploader.obj
 0002:00005f48       ??_C@_17KFDBOMCI@?$AAC?$AAR?$AAS@ 0000000140050f48     crs_uploader.obj
 0002:00005f50       ??_C@_1CG@KLCLFNNP@?$AAD?$AAe?$AAl?$AAe?$AAt?$AAe?$AAM?$AAi?$AAn?$AAi?$AAd?$AAu?$AAm?$AAp?$AAF@ 0000000140050f50     crs_uploader.obj
 0002:00005f78       ??_C@_19FKLFLPMF@?$AAt?$AAr?$AAu?$AAe@ 0000000140050f78     crs_uploader.obj
 0002:00005f88       ??_C@_1BG@BMKKPDAI@?$AA?$CF?$AAs?$AA?2?$AAC?$AAR?$AAS?$AA?4?$AAi?$AAn?$AAi@ 0000000140050f88     crs_uploader.obj
 0002:00005fa0       ??_C@_1BA@ODBNFJPP@?$AAu?$AAn?$AAk?$AAn?$AAw?$AAo?$AAn@ 0000000140050fa0     crs_uploader.obj
 0002:00005fb0       ??_C@_1M@LLCLNBHO@?$AA?$CF?$AAs?$AA_?$AA?$CF?$AAs@ 0000000140050fb0     crs_uploader.obj
 0002:00005fc0       ??_C@_0L@CIKECLEP@version?3?$CFd@ 0000000140050fc0     crs_uploader.obj
 0002:00005fd0       ??_C@_09BNNAOANA@empty?5url@ 0000000140050fd0     crs_uploader.obj
 0002:00005fe0       ??_C@_1O@NBDODAKG@?$AAu?$AAp?$AAl?$AAo?$AAa?$AAd@ 0000000140050fe0     crs_uploader.obj
 0002:00005ff0       ??_C@_0BL@ININHFIP@output_dir?5is?5empty?5URL?$DN?$CFs@ 0000000140050ff0     crs_uploader.obj
 0002:00006010       ??_C@_0BI@LFPNAEAK@invalid?5url?$FL?$CFlu?$FN?5URL?$DN?$CFs@ 0000000140051010     crs_uploader.obj
 0002:00006028       ??_C@_0BA@ELPOGNCH@disabled?5URL?$DN?$CFs@ 0000000140051028     crs_uploader.obj
 0002:00006038       ??_C@_0BA@GOHDMMKI@unknown?5path?$DN?$CFs@ 0000000140051038     crs_uploader.obj
 0002:00006048       ??_C@_0BD@BMMMPMLP@exists?5not?5path?$DN?$CFs@ 0000000140051048     crs_uploader.obj
 0002:00006060       ??_C@_0CC@NKABMACB@?$CFs?5WinHttpOpenRequest?$FL?$CFlu?$FN?5URL?$DN@ 0000000140051060     crs_uploader.obj
 0002:00006088       ??_C@_0CC@MFDBFDLN@?$CFs?5WinHttpSendRequest?$FL?$CFlu?$FN?5URL?$DN@ 0000000140051088     crs_uploader.obj
 0002:000060b0       ??_C@_07CIFAGBMG@unknown@  00000001400510b0     crs_uploader.obj
 0002:000060b8       ??_C@_0L@KCOBBBIC@?$CFs?$CL0x?$CFI64X@ 00000001400510b8     crs_uploader.obj
 0002:000060c8       ??_C@_0DE@FBPBPEDJ@?$CD?5Exception?5Infomation?5?3?5EXCEPT@ 00000001400510c8     crs_uploader.obj
 0002:00006100       ??_C@_0BH@GDOLEHPB@?$CD?5Exception?5Infomation@ 0000000140051100     crs_uploader.obj
 0002:00006118       ??_C@_08ONNNDKLF@02?318?303@ 0000000140051118     crs_uploader.obj
 0002:00006128       ??_C@_0M@KPOGGKFB@Jul?529?52021@ 0000000140051128     crs_uploader.obj
 0002:00006138       ??_C@_0BC@CEMNINJG@?$CD?5DATESTAMP?$DN?$CFs?5?$CFs@ 0000000140051138     crs_uploader.obj
 0002:00006150       ??_C@_0BC@KFCCOPHA@?$CD?5Address?$DN0x?$CF016X@ 0000000140051150     crs_uploader.obj
 0002:00006168       ??_C@_0BF@CCECPKIO@?$CD?5ExceptionCode?$DN0x?$CFX@ 0000000140051168     crs_uploader.obj
 0002:00006180       ??_C@_0BO@HFLEEEGJ@?$CF2d?50x?$CF08X?50x?$CF08X?50x?$CF08X?5?$CI?$CFs?$CJ@ 0000000140051180     crs_uploader.obj
 0002:000061a0       ??_C@_0BK@ENPPOBB@?$CD?5SymInitialize?5FAIL?$FL?$CFlu?$FN@ 00000001400511a0     crs_uploader.obj
 0002:000061c0       ??_C@_1BM@PEICEKM@?$AAS?$AAm?$AAi?$AAl?$AAe?$AAG?$AAa?$AAt?$AAe?$AA?5?$AAC?$AAR?$AAS@ 00000001400511c0     crs_uploader.obj
 0002:000061e0       ??_C@_0BI@JANBAAPF@WinHttpOpen?$FL?$CFlu?$FN?5URL?$DN?$CFs@ 00000001400511e0     crs_uploader.obj
 0002:000061f8       ??_C@_0BL@EFGBFCEJ@WinHttpConnect?$FL?$CFlu?$FN?5URL?$DN?$CFs@ 00000001400511f8     crs_uploader.obj
 0002:00006218       ??_C@_17NHNHNCOB@?$AAP?$AAU?$AAT@ 0000000140051218     crs_uploader.obj
 0002:00006220       ??_C@_0BP@IIOECOIJ@?$CFs?5CreateFile?5READ?$FL?$CFlu?$FN?5URL?$DN?$CFs@ 0000000140051220     crs_uploader.obj
 0002:00006240       ??_C@_0BL@MLCFLFFE@?$CFs?5GetFileSize?$FL?$CFlu?$FN?5URL?$DN?$CFs@ 0000000140051240     crs_uploader.obj
 0002:00006260       ??_C@_0BI@GHDKNBPJ@?$CFs?5ReadFile?$FL?$CFlu?$FN?5URL?$DN?$CFs@ 0000000140051260     crs_uploader.obj
 0002:00006278       ??_C@_0CA@OMIDHMOL@?$CFs?5WinHttpWriteData?$FL?$CFlu?$FN?5URL?$DN?$CFs@ 0000000140051278     crs_uploader.obj
 0002:00006298       ??_C@_1BA@NCJLFNJB@?$AAc?$AAr?$AAs?$AA?4?$AAl?$AAo?$AAg@ 0000000140051298     crs_uploader.obj
 0002:000062a8       ??_C@_0CG@LLGLPKJE@?$CFs?5WinHttpReceiveResponse?$FL?$CFlu?$FN?5@ 00000001400512a8     crs_uploader.obj
 0002:000062d0       ??_C@_0CD@ODMPMKPE@?$CFs?5WinHttpQueryHeaders?$FL?$CFlu?$FN?5URL@ 00000001400512d0     crs_uploader.obj
 0002:000062f8       ??_C@_0BE@IDLGBAE@?$CFs?5HTTP?$FL?$CFlu?$FN?5URL?$DN?$CFs@ 00000001400512f8     crs_uploader.obj
 0002:00006310       ??_C@_1FA@CNNLBJGF@?$AA?$CF?$AAs?$AA_?$AA?$CF?$AA0?$AA4?$AAd?$AA?$CF?$AA0?$AA2?$AAd?$AA?$CF?$AA0?$AA2?$AAd@ 0000000140051310     crs_uploader.obj
 0002:00006360       ??_C@_1M@BHHLEAOO@?$AA?$CF?$AAs?$AA?1?$AA?$CF?$AAs@ 0000000140051360     crs_uploader.obj
 0002:00006370       ??_C@_19LJDFFCJJ@?$AA?$CF?$AAs?$AA?$CF?$AAs@ 0000000140051370     crs_uploader.obj
 0002:00006380       ??_C@_0BI@CFPLBAOH@invalid?5string?5position@ 0000000140051380     crs_uploader.obj
 0002:00006398       ??_C@_11LOCGONAA@@         0000000140051398     crs_uploader.obj
 0002:000063a0       ??_C@_0BE@DLJIFIGP@?$CFs?2timeout_?$CFs_?$CFs_?$CFs@ 00000001400513a0     LogMgmt.obj
 0002:000063b8       ??_C@_0BC@BCEHJAGO@?$CFs?2error_?$CFs_?$CFs_?$CFs@ 00000001400513b8     LogMgmt.obj
 0002:000063d0       ??_C@_0BE@KIEDFKMI@?$CFs?2etcinfo_?$CFs_?$CFs_?$CFs@ 00000001400513d0     LogMgmt.obj
 0002:000063e8       ??_C@_0BG@NJNBAHKK@?$CF04d?$CF02d?$CF02d_?$CF02d?4log@ 00000001400513e8     LogMgmt.obj
 0002:00006400       ??_C@_0BB@FLNJAMGH@?$CF04d?$CF02d?$CF02d?4log@ 0000000140051400     LogMgmt.obj
 0002:00006414       ??_C@_02DPNLHKJD@a?$CL@    0000000140051414     LogMgmt.obj
 0002:00006418       ??_C@_0BE@MNIJIMLO@?$CF02d?3?$CF02d?3?$CF02d?4?$CF03d@ 0000000140051418     LogMgmt.obj
 0002:0000642c       ??_C@_02CPIDLAI@at@        000000014005142c     LogMgmt.obj
 0002:00006438       ??_7CServerLog@@6B@        0000000140051438     LogMgmt.obj
 0002:00006440       ??_C@_00CNPNBAHC@@         0000000140051440     LogMgmt.obj
 0002:00006444       ??_C@_04LIFAFMCE@?$FL?$CFs?$FN@ 0000000140051444     RWPMLog.obj
 0002:0000644c       ??_C@_06HJNJJLFL@?$FL?$CFlld?$FN@ 000000014005144c     RWPMLog.obj
 0002:00006458       ??_C@_0BP@BMCLPMN@?$CFs?0?5?$CFd?0?5MEMORY_ADDRESS?$FL?$CFd?$FN?0?5?$CFs@ 0000000140051458     RWPMLog.obj
 0002:00006478       ??_C@_0CG@MCFHKALN@?$CFs?0?5?$CFd?0?5GAMEPROTO_SC_REMOVECLIE@ 0000000140051478     RWPMLog.obj
 0002:000064a0       ??_C@_0CB@GMLIEFM@?$CFs?0?5?$CFd?0?5GAMEPROTO_SS_GAMEEND?0?5?$CF@ 00000001400514a0     RWPMLog.obj
 0002:000064c8       ??_C@_0CI@FMLCGOEC@?$CFs?0?5?$CFd?0?5GAMEPROTO_SC_HOST_USER_@ 00000001400514c8     RWPMLog.obj
 0002:000064f0       ??_C@_0BP@FHPFEAAB@?$CFs?0?5?$CFd?0?5CLANSTATREPORTDATA?0?5?$CFs@ 00000001400514f0     RWPMLog.obj
 0002:00006510       ??_C@_0BL@NGCIOLCH@?$CFs?0?5?$CFd?0?5PROTO_BAN_USER?0?5?$CFs@ 0000000140051510     RWPMLog.obj
 0002:00006530       ??_C@_0CD@LJIJHLEG@?$CFs?0?5?$CFd?0?5GAMEPROTO_SC_HOST_STAT?0@ 0000000140051530     RWPMLog.obj
 0002:00006558       ??_C@_0DE@DCEKNMHJ@?$CFs?0?5?$CFd?0?5PROTO_GAMEGT_INGAME_AIG@ 0000000140051558     RWPMLog.obj
 0002:00006590       ??_C@_0DB@KKCKHLAM@?$CFs?0?5?$CFd?0?5PROTO_GAMEGT_MAPLOADING@ 0000000140051590     RWPMLog.obj
 0002:000065c8       ??_C@_0CE@NNGOJKJJ@?$CFs?0?5?$CFd?0?5GAMEPROTO_SC_SPY_CHANGE@ 00000001400515c8     RWPMLog.obj
 0002:000065f0       ??_C@_0DB@CHJEFLPF@?$CFs?0?5?$CFd?0?5PROTO_GAMEGT_INGAME_FAR@ 00000001400515f0     RWPMLog.obj
 0002:00006628       ??_C@_0CM@HCGEFML@?$CFs?0?5?$CFd?0?5PROTO_AI2_BONUSROUND_RE@ 0000000140051628     RWPMLog.obj
 0002:00006658       ??_C@_0DK@CBOHEJM@?$CFs?0?5?$CFd?0?5PROTO_GAMEGT_INGAME_AI3@ 0000000140051658     RWPMLog.obj
 0002:00006698       ??_C@_0CK@BAHPFFKB@?$CFs?0?5?$CFd?0?5PROTO_INSERT_CHARACTER_@ 0000000140051698     RWPMLog.obj
 0002:000066c8       ??_C@_0CG@MMMIDGFA@?$CFs?0?5?$CFd?0?5PROTO_AI_EXTRA_REWARD_R@ 00000001400516c8     RWPMLog.obj
 0002:000066f0       ??_C@_0CF@MEMHOFAF@?$CFs?0?5?$CFd?0?5PROTO_FINISHED_GAME_PRE@ 00000001400516f0     RWPMLog.obj
 0002:00006718       ??_C@_0DB@LMMMOHOA@?$CFs?0?5?$CFd?0?5PROTO_SPEC_RECOMMENDROO@ 0000000140051718     RWPMLog.obj
 0002:00006750       ??_C@_0DI@NJDEIFAK@?$CFs?0?5?$CFd?0?5PROTO_GAMEGT_AUTO_SIDE_@ 0000000140051750     RWPMLog.obj
 0002:00006790       ??_7CSGGMCallBackObj@@6B@  0000000140051790     SGGMCallBackObj.obj
 0002:000067a0       ??_7MultiReceiver@sggm_proxy@@6B@ 00000001400517a0     SGGMCallBackObj.obj
 0002:000067b0       ??_7CReceiver@@6B@         00000001400517b0     SGGMCallBackObj.obj
 0002:000067d8       ??_C@_0BO@CCNGFBBL@SendQueued?$CI?$CJ?5WSASend?5Error?5?$CFd@ 00000001400517d8     ClientLib.obj
 0002:000067f8       ??_C@_0DL@FAAPJGPH@CheckSendCompleteEvent?$CI?$CJ?5WSAGet@ 00000001400517f8     ClientLib.obj
 0002:00006838       ??_C@_0CD@DCDLLIKH@CClientLib?3?3CheckSendCompleteEv@ 0000000140051838     ClientLib.obj
 0002:00006860       ??_C@_0CI@NKCMALEF@?$FL?$CFs?$FN?5WSASendTime?3?$CFu?0?5ResultTime@ 0000000140051860     ClientLib.obj
 0002:00006888       ??_C@_0BP@IKLINECJ@CClientLib?3?3ProcessSocketEvent@ 0000000140051888     ClientLib.obj
 0002:000068a8       ??_C@_0CM@HFOCLINH@?$CFs?5NetworkEvents?4iErrorCode?$FLFD_@ 00000001400518a8     ClientLib.obj
 0002:000068d8       ??_C@_0CN@GHCPDFJF@?$CFs?5NetworkEvents?4iErrorCode?$FLFD_@ 00000001400518d8     ClientLib.obj
 0002:00006910       ??_7?$CircuitQueue@E@@6B@  0000000140051910     ClientLib.obj
 0002:00006920       ??_7CClientLib@@6B@        0000000140051920     ClientLib.obj
 0002:00006940       ??_7SendBuffer@@6B@        0000000140051940     ClientLib.obj
 0002:00006950       ??_7CPacket@@6B@           0000000140051950     Packet.obj
 0002:00006958       ??_C@_0DO@EEMEKEMN@CSFGameServerClientLib?3?3Connect@ 0000000140051958     SFGameServerClientLib.obj
 0002:000069a0       ??_C@_0EC@LALPNAOK@CSFGameServerClientLib?3?3Connect@ 00000001400519a0     SFGameServerClientLib.obj
 0002:000069e8       ??_C@_0O@NAPDBOAI@CloseSocket?$CI?$CJ@ 00000001400519e8     SFGameServerClientLib.obj
 0002:00006a00       ??_7CSFGameServerClientLib@@6B@ 0000000140051a00     SFGameServerClientLib.obj
 0002:00006a18       ??_C@_04NOJCDH@?$CF02x@    0000000140051a18     md5.obj
 0002:00006a20       ??_C@_02JDPG@rb@           0000000140051a20     md5.obj
 0002:00006a24       ??_C@_02PCIJFNDE@?$AN?6@   0000000140051a24     AppInfoDlg.obj
 0002:00006a30       ??_7GAMEPROTO_SC_HOST_STAT@@6B@ 0000000140051a30     AppInfoDlg.obj
 0002:00006a68       ??_7GAMEPROTO_SC_HOST_USER_STAT@@6B@ 0000000140051a68     AppInfoDlg.obj
 0002:00006aa0       ??_7GAMEPROTO_SC_REMOVECLIENT@@6B@ 0000000140051aa0     AppInfoDlg.obj
 0002:00006ad0       ??_C@_0L@JBGDLKBH@read?5error@ 0000000140051ad0     AppInfoDlg.obj
 0002:00006ae0       ??_C@_0BC@EOODALEL@Unknown?5exception@ 0000000140051ae0     AppInfoDlg.obj
 0002:00006b00       ??_7exception@std@@6B@     0000000140051b00     AppInfoDlg.obj
 0002:00006b18       ??_7GAMEPROTO_SS_GAMEEND@@6B@ 0000000140051b18     AppInfoDlg.obj
 0002:00006b50       ??_7GAMEPROTO_SC_SPY_CHANGE@@6B@ 0000000140051b50     AppInfoDlg.obj
 0002:00006b70       ??_C@_04BFAHMMK@?$CFlld@   0000000140051b70     AppInfoDlg.obj
 0002:00006b80       ??_7CEdit@@6B@             0000000140051b80     AppInfoDlg.obj
 0002:00006e58       ??_C@_06EFAGIKOH@Normal@   0000000140051e58     CheckMemUsage.obj
 0002:00006e60       ??_C@_08HAPIFNIB@MemUsage@ 0000000140051e60     CheckMemUsage.obj
 0002:00006e70       ??_C@_0CN@INENPBKG@CHECK_MEM_USAGE?5?3?5ServerAppIdx?5@ 0000000140051e70     CheckMemUsage.obj
 0002:00006ea0       ??_C@_0DD@NNCKBAHE@CHECK_MEM_USAGE?5error?5?3?5ServerA@ 0000000140051ea0     CheckMemUsage.obj
 0002:00006ed8       ??_C@_0N@EOFHHCCD@INETMIB1?4DLL@ 0000000140051ed8     cSnmpEX.obj
 0002:00006ee8       ??_C@_0BD@BMAIGDOA@SnmpExtensionQuery@ 0000000140051ee8     cSnmpEX.obj
 0002:00006f00       ??_C@_0BC@MFBDBJPG@SnmpExtensionInit@ 0000000140051f00     cSnmpEX.obj
 0002:00006f18       ??_C@_0BC@NKHLAHHO@ServerApp_x64?4exe@ 0000000140051f18     GameServerManager.obj
 0002:00006f30       ??_C@_0M@GCJIADCJ@IsDebugMode@ 0000000140051f30     GameServerManager.obj
 0002:00006f40       ??_C@_0P@CFNGHFNG@object_x64?4dll@ 0000000140051f40     GameServerManager.obj
 0002:00006f50       ??_C@_0P@DBKFBJAC@server_x64?4dll@ 0000000140051f50     GameServerManager.obj
 0002:00006f60       ??_C@_0BC@PFGMLLEF@GameServerManager@ 0000000140051f60     GameServerManager.obj
 0002:00006f74       ??_C@_04GOLNGIJ@EXIT@      0000000140051f74     GameServerManager.obj
 0002:00006f80       ??_C@_0BF@EFPNECCJ@SERVICE_STOP_PENDING@ 0000000140051f80     GameServerManager.obj
 0002:00006fa0       ??_7CGameServerManagerApp@@6B@ 0000000140051fa0     GameServerManager.obj
 0002:00007220       ??_C@_0N@JEEFJOKI@?2Setting?4ini@ 0000000140052220     GameServerManagerDlg.obj
 0002:00007230       ??_C@_0M@LPAKIOHO@ExitProcess@ 0000000140052230     GameServerManagerDlg.obj
 0002:00007240       ??_C@_0CC@OIOGGMFK@CGameServerManagerDlg?5Clear?5Sta@ 0000000140052240     GameServerManagerDlg.obj
 0002:00007268       ??_C@_0CE@BHENJAK@CGameServerManagerDlg?5Clear?5Pha@ 0000000140052268     GameServerManagerDlg.obj
 0002:00007290       ??_C@_0CE@CKFJIKMJ@CGameServerManagerDlg?5Clear?5Pha@ 0000000140052290     GameServerManagerDlg.obj
 0002:000072b8       ??_C@_0CE@DDECLLII@CGameServerManagerDlg?5Clear?5Pha@ 00000001400522b8     GameServerManagerDlg.obj
 0002:000072e0       ??_C@_0CE@HMADCNEP@CGameServerManagerDlg?5Clear?5Pha@ 00000001400522e0     GameServerManagerDlg.obj
 0002:00007308       ??_C@_0CE@GFBIBMAO@CGameServerManagerDlg?5Clear?5Pha@ 0000000140052308     GameServerManagerDlg.obj
 0002:00007330       ??_C@_0CE@EODFEPMN@CGameServerManagerDlg?5Clear?5Pha@ 0000000140052330     GameServerManagerDlg.obj
 0002:00007358       ??_C@_0CE@FHCOHOIM@CGameServerManagerDlg?5Clear?5Pha@ 0000000140052358     GameServerManagerDlg.obj
 0002:00007380       ??_C@_0CE@NALGGCED@CGameServerManagerDlg?5Clear?5Pha@ 0000000140052380     GameServerManagerDlg.obj
 0002:000073a8       ??_C@_0CE@MJKNFDAC@CGameServerManagerDlg?5Clear?5Pha@ 00000001400523a8     GameServerManagerDlg.obj
 0002:000073d0       ??_C@_0CF@DPJCKLDE@CGameServerManagerDlg?5Clear?5Pha@ 00000001400523d0     GameServerManagerDlg.obj
 0002:000073f8       ??_C@_0CF@CGIJJKHF@CGameServerManagerDlg?5Clear?5Pha@ 00000001400523f8     GameServerManagerDlg.obj
 0002:00007420       ??_C@_0CG@PKMJOIO@CGameServerManagerDlg?5Clear?5Pha@ 0000000140052420     GameServerManagerDlg.obj
 0002:00007448       ??_C@_02HAOIJKIC@?$CFc@    0000000140052448     GameServerManagerDlg.obj
 0002:00007450       ??_C@_0N@PNPLDJGI@?1CNFGFILE?3?$CFs@ 0000000140052450     GameServerManagerDlg.obj
 0002:00007460       ??_C@_0BE@OOKKAOIA@GameServerManager?$CFd@ 0000000140052460     GameServerManagerDlg.obj
 0002:00007478       ??_C@_0BO@NIKEONNF@C?3?2pmang?2crossfire?2cf_hostsrv@ 0000000140052478     GameServerManagerDlg.obj
 0002:00007498       ??_C@_0CA@OJAMDDLG@Failed?5to?5initialize?5SGGM_PROXY@ 0000000140052498     GameServerManagerDlg.obj
 0002:000074b8       ??_C@_0BG@FBDPKLJI@GameServerManager?4exe@ 00000001400524b8     GameServerManagerDlg.obj
 0002:000074d0       ??_C@_0O@GDJDINEI@ServerApp?4exe@ 00000001400524d0     GameServerManagerDlg.obj
 0002:000074e0       ??_C@_0N@JNKMCOLL@SharedMemory@ 00000001400524e0     GameServerManagerDlg.obj
 0002:000074f0       ??_C@_0BC@LFNIPHGA@ReadProcessMemory@ 00000001400524f0     GameServerManagerDlg.obj
 0002:00007508       ??_C@_0BD@PBGEEFCK@WriteProcessMemory@ 0000000140052508     GameServerManagerDlg.obj
 0002:00007520       ??_C@_0CM@GMMNNKDE@ReadProcessMemory?$DN?$CFd?0?5WriteProc@ 0000000140052520     GameServerManagerDlg.obj
 0002:00007550       ??_C@_0EF@OAINCLCA@GSM?5InitializeManager?$CI?$CJ?9Before?5@ 0000000140052550     GameServerManagerDlg.obj
 0002:00007598       ??_C@_0CA@ICDPDEEN@m_sManagerSetting?4uiNumber?5?3?5?$CFd@ 0000000140052598     GameServerManagerDlg.obj
 0002:000075b8       ??_C@_0CN@FLHCCAIP@CGameServerManagerDlg?5DestroySe@ 00000001400525b8     GameServerManagerDlg.obj
 0002:000075e8       ??_C@_0CL@JFNEDFOP@CGameServerManagerDlg?5DestroySe@ 00000001400525e8     GameServerManagerDlg.obj
 0002:00007618       ??_C@_0BC@EOFFKHON@GameServerAppPath@ 0000000140052618     GameServerManagerDlg.obj
 0002:00007630       ??_C@_0BB@JFHPGGHO@GameServerAppDir@ 0000000140052630     GameServerManagerDlg.obj
 0002:00007648       ??_C@_0O@EJLILIAL@GameServerNum@ 0000000140052648     GameServerManagerDlg.obj
 0002:00007658       ??_C@_07OHKHACFK@0?40?40?40@ 0000000140052658     GameServerManagerDlg.obj
 0002:00007660       ??_C@_0P@OPLGOGOA@GameServerAddr@ 0000000140052660     GameServerManagerDlg.obj
 0002:00007670       ??_C@_0O@OBICEAPF@PrivateIPRule@ 0000000140052670     GameServerManagerDlg.obj
 0002:00007680       ??_C@_0BD@CCCIMJNE@GameServerPortBase@ 0000000140052680     GameServerManagerDlg.obj
 0002:00007698       ??_C@_0BH@HPPBCKGI@MatchMakingServerCount@ 0000000140052698     GameServerManagerDlg.obj
 0002:000076b0       ??_C@_0BI@JFOOEFJL@MatchMakingServerAddr?$CFd@ 00000001400526b0     GameServerManagerDlg.obj
 0002:000076c8       ??_C@_0BI@PEELBPNM@MatchMakingServerPort?$CFd@ 00000001400526c8     GameServerManagerDlg.obj
 0002:000076e0       ??_C@_0BG@JKBNCGBC@MatchMakingServerAddr@ 00000001400526e0     GameServerManagerDlg.obj
 0002:000076f8       ??_C@_0BG@FOGNGHGF@MatchMakingServerPort@ 00000001400526f8     GameServerManagerDlg.obj
 0002:00007710       ??_C@_01GBGANLPD@0@        0000000140052710     GameServerManagerDlg.obj
 0002:00007718       ??_C@_08IGDKGKJM@SGGMConn@ 0000000140052718     GameServerManagerDlg.obj
 0002:00007728       ??_C@_0BC@HEODEKJK@BridgeServerExist@ 0000000140052728     GameServerManagerDlg.obj
 0002:0000773c       ??_C@_03IPHJCBHH@YES@      000000014005273c     GameServerManagerDlg.obj
 0002:00007740       ??_C@_0P@KGAOCENG@MessageTimeout@ 0000000140052740     GameServerManagerDlg.obj
 0002:00007750       ??_C@_0BH@MBIKFMOK@StartGameServers?$CI?$CJ?5end@ 0000000140052750     GameServerManagerDlg.obj
 0002:00007768       ??_C@_0BB@LAPCEPOI@?$CFd?5?$CFld?5?$CFd?5?$CFd?5?$CFld@ 0000000140052768     GameServerManagerDlg.obj
 0002:00007780       ??_C@_0CD@GOBAOJAO@ShellExecuteEx?$CI?$CJ?5Error?$CB?$CB?$CB?$CB?$CB?$CB?$CB?$CB?$CB@ 0000000140052780     GameServerManagerDlg.obj
 0002:000077a8       ??_C@_0CN@BHNPGPMA@info?4hInstApp?5?$DN?$DN?5?$CIHINSTANCE?$CJ32?5@ 00000001400527a8     GameServerManagerDlg.obj
 0002:000077d8       ??_C@_0BP@DGLGJOHC@info?4hInstApp?5?$DN?$DN?5?$CIHINSTANCE?$CJ32@ 00000001400527d8     GameServerManagerDlg.obj
 0002:000077f8       ??_C@_0DI@PAOFCAL@StartGameServer?5Hwnd?3?5?$CFp?5index?3@ 00000001400527f8     GameServerManagerDlg.obj
 0002:00007830       ??_C@_0EH@BNNIDBFK@GAMESERVERMSG_REPORT_HWND?5?$CFd?0?5C@ 0000000140052830     GameServerManagerDlg.obj
 0002:00007878       ??_C@_06FKAFBJKH@?$FLSEND?$FN@ 0000000140052878     GameServerManagerDlg.obj
 0002:00007880       ??_C@_0DN@BPOIKBBM@GAMESERVERMSG_REPORT_HWND?5INVAL@ 0000000140052880     GameServerManagerDlg.obj
 0002:000078c0       ??_C@_0DC@EOEBPNDD@GAMESERVERMSG_FAILED_BINDTOPORT@ 00000001400528c0     GameServerManagerDlg.obj
 0002:00007900       ??_C@_0HO@HABMKHBO@GAMESERVERMSG_LOADING?5FAILED?5?9?5@ 0000000140052900     GameServerManagerDlg.obj
 0002:00007980       ??_C@_0CE@OPEAPJJJ@?$FLError?$FN?5?$DL?5Map?5Info?5Ptr?5Error?4?4?4@ 0000000140052980     GameServerManagerDlg.obj
 0002:000079a8       ??_C@_0CE@NGJODGNH@?$FLError?$FN?5?$DL?5Map?5Index?5Boundary?4?4?4@ 00000001400529a8     GameServerManagerDlg.obj
 0002:000079d0       ??_C@_0CE@FOMJAHCF@?$FLError?$FN?5?$DL?5Map?5FileLoad?5Failed?4?4@ 00000001400529d0     GameServerManagerDlg.obj
 0002:000079f8       ??_C@_0CE@HAAEJKLP@?$FLError?$FN?5?$DL?5Run?5World?5Failed?4?4?4?4?4@ 00000001400529f8     GameServerManagerDlg.obj
 0002:00007a20       ??_C@_0CO@LDBFNNEA@?$FLError?$FN?5?$DL?5UCC?5Map?5Download?5Fail@ 0000000140052a20     GameServerManagerDlg.obj
 0002:00007a50       ??_C@_0DB@LJPNLBJI@?$FLError?$FN?5?$DL?5UCC?5Map?5Download?5Fail@ 0000000140052a50     GameServerManagerDlg.obj
 0002:00007a90       ??_C@_0EF@PFLPCJJD@?$FLHOST?5KILLED?$FN?5Map?5Load?5Failed?5?3@ 0000000140052a90     GameServerManagerDlg.obj
 0002:00007ad8       ??_C@_0BN@CIMCCFIJ@?$FLError?$FN?5?$DL?5Map?5Load?5Failed?4?4?4@ 0000000140052ad8     GameServerManagerDlg.obj
 0002:00007af8       ??_C@_0DB@OEKFNOII@GAMESERVERMSG_LOADING_COMPLETE?5@ 0000000140052af8     GameServerManagerDlg.obj
 0002:00007b30       ??_C@_0CJ@LBGIHIFK@GAMESERVERMSG_ROOMINFO?5?3?5Server@ 0000000140052b30     GameServerManagerDlg.obj
 0002:00007b60       ??_C@_0DN@EBPCFPMJ@Unqueued?5server?5sent?5loading?5co@ 0000000140052b60     GameServerManagerDlg.obj
 0002:00007ba0       ??_C@_0CN@GKFECKMH@GAMESERVERMSG_ROOMINFO_ACK?5?3?5Se@ 0000000140052ba0     GameServerManagerDlg.obj
 0002:00007bd0       ??_C@_0FF@GFFFGPHB@?$FLHOST?5KILLED?5?9?5GAMESERVERMSG_RO@ 0000000140052bd0     GameServerManagerDlg.obj
 0002:00007c30       ??_C@_0EA@PCJKOGDJ@?$FLRECV?$FN?5tIndex?$FL?$CF02d?$FN?0?5msgID?$FL?$CF02d@ 0000000140052c30     GameServerManagerDlg.obj
 0002:00007c70       ??_C@_06HMJBGFMB@?$FLRECV?$FN@ 0000000140052c70     GameServerManagerDlg.obj
 0002:00007c78       ??_C@_0DI@HCDCEGBE@?$FLRWPM?$FNNot?5Supported?5Message?$CB?$CB?$CB?$CB@ 0000000140052c78     GameServerManagerDlg.obj
 0002:00007cb0       ??_C@_0GF@COBJLBOB@?$CI?$CF2d?5?$CF2d?5?$CF2d?5?3?5?$CFs?$CJ?5OnTimer?5?9?5Ga@ 0000000140052cb0     GameServerManagerDlg.obj
 0002:00007d18       ??_C@_0CM@FKFENBNH@CGameServerManagerDlg?3?3OnTimer?5@ 0000000140052d18     GameServerManagerDlg.obj
 0002:00007d48       ??_C@_0BK@NOIFNJNA@S_P_F?3?5GSM_HEARTBEAT?5?3?5?$CFd@ 0000000140052d48     GameServerManagerDlg.obj
 0002:00007d70       ??_C@_0EB@DPHBPILO@KillServerApp?5?3?5m_sGameServerIn@ 0000000140052d70     GameServerManagerDlg.obj
 0002:00007db8       ??_C@_0DG@KLMIGDKN@OnTimer?5call?5StartGameServer?$CI?$CFd@ 0000000140052db8     GameServerManagerDlg.obj
 0002:00007df0       ??_C@_0DM@GJCHKLOD@CGameServerManagerDlg?3?3OnTimer?5@ 0000000140052df0     GameServerManagerDlg.obj
 0002:00007e2c       ??_C@_04LHJJONAO@?1add@    0000000140052e2c     GameServerManagerDlg.obj
 0002:00007e38       ??_C@_0BG@JJJIONME@GMS?5Disconnect?$CB?$CB?$CB?$CB?5?$AN?6@ 0000000140052e38     GameServerManagerDlg.obj
 0002:00007e50       ??_C@_0BD@BIDAHFAD@MaxRemovePortCount@ 0000000140052e50     GameServerManagerDlg.obj
 0002:00007e70       ??_C@_0EE@DBALGLBK@WM?5COPYDATA?5?9?5FINISH?5FAILED?5?3?5?$CF@ 0000000140052e70     GameServerManagerDlg.obj
 0002:00007eb8       ??_C@_0BG@EKBPLJLF@GameServerPortBaseEnd@ 0000000140052eb8     GameServerManagerDlg.obj
 0002:00007ed0       ??_C@_0L@BALHJKMC@ExceptPort@ 0000000140052ed0     GameServerManagerDlg.obj
 0002:00007edc       ??_C@_01CLKCMJKC@?5@       0000000140052edc     GameServerManagerDlg.obj
 0002:00007ee0       ??_C@_0DF@DFFIGGK@PortRemoved?5?$CFdPort?5eternal?5UnUs@ 0000000140052ee0     GameServerManagerDlg.obj
 0002:00007f18       ??_C@_0BF@CMFCHDBN@RestoreFreePort?5?3?5?$CFs@ 0000000140052f18     GameServerManagerDlg.obj
 0002:00007f30       ??_C@_0BB@EMNMHPBF@Invalid?5Port?3?5?$CFd@ 0000000140052f30     GameServerManagerDlg.obj
 0002:00007f50       ??_C@_0GD@JOOJKABP@?$FLROOM_COUNT?$FN?5NewRoomCount?$CI?$CFd?$CJ?5N@ 0000000140052f50     GameServerManagerDlg.obj
 0002:00007fb8       ??_C@_0CB@EMGJKHPD@Logger?5Init?5Failed?5?3?5ErrCode?$FL?$CFd@ 0000000140052fb8     GameServerManagerDlg.obj
 0002:00007fe0       ??_C@_0CC@ILNGBDNH@Log?5Msz?5File?5Load?5Failed?4?5Level@ 0000000140052fe0     GameServerManagerDlg.obj
 0002:00008008       ??_C@_0CC@KAPLEABE@Log?5Msz?5File?5Load?5Failed?4?5Level@ 0000000140053008     GameServerManagerDlg.obj
 0002:00008030       ??_C@_0BL@BMLEPNEM@Logger?5USAGE_NOUSE?5Setted?4@ 0000000140053030     GameServerManagerDlg.obj
 0002:00008050       ??_C@_0EE@JIJKMCEJ@?$FLHOST?5KILLED?$FN?5No?5UDP?5Connection@ 0000000140053050     GameServerManagerDlg.obj
 0002:00008094       ??_C@_03IOOJPBPG@?$CFu?5@  0000000140053094     GameServerManagerDlg.obj
 0002:00008098       ??_C@_05IBGOOFKP@Mutex@    0000000140053098     GameServerManagerDlg.obj
 0002:000080a0       ??_C@_07NJKPPODG@Mapping@  00000001400530a0     GameServerManagerDlg.obj
 0002:000080a8       ??_C@_0N@MGAIABNC@CreateServer@ 00000001400530a8     GameServerManagerDlg.obj
 0002:000080b8       ??_C@_03IEEBNAED@rez@      00000001400530b8     GameServerManagerDlg.obj
 0002:000080c0       ??_C@_08JFAGHOJI@?$CFs?2?$CK?4rez@ 00000001400530c0     GameServerManagerDlg.obj
 0002:000080d0       ??_C@_0N@LBFNJNAG@DeleteServer@ 00000001400530d0     GameServerManagerDlg.obj
 0002:000080e0       ??_C@_0FL@EFNFKJMP@?$FLRWPM?$FNSEND?5PostMessage?5Failed?5M@ 00000001400530e0     GameServerManagerDlg.obj
 0002:00008140       ??_C@_0EC@GHMLIALF@?$FLRWPM?$FNSEND?5PostMessage?5Failed?5t@ 0000000140053140     GameServerManagerDlg.obj
 0002:00008188       ??_C@_0CP@LALOJJGA@?$FLSEND?$FN?5tIndex?$FL?$CF02d?$FN?0?5msgID?$FL?$CF02d@ 0000000140053188     GameServerManagerDlg.obj
 0002:000081c0       ??_C@_0EC@BJGNEKLM@GAMESERVERMSG_AUTO_MATCH_STARTI@ 00000001400531c0     GameServerManagerDlg.obj
 0002:00008208       ??_C@_0BM@OGFIALEA@InValid?5Message?5Type?$DN?$CFd?5?$CB?$CB?$CB@ 0000000140053208     GameServerManagerDlg.obj
 0002:00008228       ??_C@_0CA@BBKIPFND@GAMEPROTO_SS_GAMEEND?5?3?5USN?5?$CFlld@ 0000000140053228     GameServerManagerDlg.obj
 0002:00008250       ??_C@_0FE@NEDCEMHF@tProtoFinishedGame?5Name?5?$CFs?5ID?5?$CF@ 0000000140053250     GameServerManagerDlg.obj
 0002:000082b0       ??_C@_0EN@JEHKCMBM@GAMESERVERMSG_GAMEEND?5?3?5?$FL?$CFd?5?$CFd?5@ 00000001400532b0     GameServerManagerDlg.obj
 0002:00008300       ??_C@_0FM@DHLNNDGB@PROTO_FINISHED_GAME?5?9?5GameLogSr@ 0000000140053300     GameServerManagerDlg.obj
 0002:00008360       ??_C@_0CI@DIBMMCOB@PostMessage?5?9?5GAMESERVERMSG_KIC@ 0000000140053360     GameServerManagerDlg.obj
 0002:00008388       ??_C@_0DK@PFKIMCDC@GAMESERVERMSG_CHARACTERSTAT?5?3?5i@ 0000000140053388     GameServerManagerDlg.obj
 0002:000083d0       ??_C@_0HE@DPHLENBL@?6?9?9?9?9?9?9?9?9?9?9?9?9?9?9?9?9?9?9?9?9?9?9?9?9?9?9?9?9?9?9@ 00000001400533d0     GameServerManagerDlg.obj
 0002:00008448       ??_C@_0BE@HCNDODKC@iKill?5?5?5?5?5?5?5?5?5?3?5?$CFd?6@ 0000000140053448     GameServerManagerDlg.obj
 0002:00008460       ??_C@_0BE@KPENLJFP@iDeath?5?5?5?5?5?5?5?5?3?5?$CFd?6@ 0000000140053460     GameServerManagerDlg.obj
 0002:00008478       ??_C@_0BE@HHMIEENL@nAIPlayRound?5?5?3?5?$CFd?6@ 0000000140053478     GameServerManagerDlg.obj
 0002:00008490       ??_C@_0BE@CMHHFMOB@iWinRounds?5?5?5?5?3?5?$CFd?6@ 0000000140053490     GameServerManagerDlg.obj
 0002:000084a8       ??_C@_0BE@MMIHDLL@iDrawRounds?5?5?5?3?5?$CFd?6@ 00000001400534a8     GameServerManagerDlg.obj
 0002:000084c0       ??_C@_0BE@JJOOMCBD@iAliveRounds?5?5?3?5?$CFd?6@ 00000001400534c0     GameServerManagerDlg.obj
 0002:000084d8       ??_C@_0BE@PMDBBCHD@iNumC4Plant?5?5?5?3?5?$CFd?6@ 00000001400534d8     GameServerManagerDlg.obj
 0002:000084f0       ??_C@_0BE@JIACHAPB@iNumC4Explode?5?3?5?$CFd?6@ 00000001400534f0     GameServerManagerDlg.obj
 0002:00008508       ??_C@_0BE@DKOKIMHF@nAIScore?5?5?5?5?5?5?3?5?$CFd?6@ 0000000140053508     GameServerManagerDlg.obj
 0002:00008520       ??_C@_0BE@PPHENGHM@iTotalDamage?5?5?3?5?$CFd?6@ 0000000140053520     GameServerManagerDlg.obj
 0002:00008538       ??_C@_0BN@LNFAIOK@iWeaponTypeKillCount?$FL0?$FN?3?5?$CFd?6@ 0000000140053538     GameServerManagerDlg.obj
 0002:00008558       ??_C@_0BN@MHHPAIHE@iWeaponTypeKillCount?$FL1?$FN?3?5?$CFd?6@ 0000000140053558     GameServerManagerDlg.obj
 0002:00008578       ??_C@_0BN@EJPAAPJH@iWeaponTypeKillCount?$FL2?$FN?3?5?$CFd?6@ 0000000140053578     GameServerManagerDlg.obj
 0002:00008598       ??_C@_0BF@MKOENOMA@iNumC4Defuse?5?5?5?3?5?$CFd?6@ 0000000140053598     GameServerManagerDlg.obj
 0002:000085b0       ??_C@_0HC@POIOEJMA@?6?9?9?9?9?9?9?9?9?9?9?9?9?9?9?9?9?9?9?9?9?9?9?9?9?9?9?9?9?9?9@ 00000001400535b0     GameServerManagerDlg.obj
 0002:00008628       ??_C@_0BL@FDFMLHI@nAim_Hit_Avg?5?5?5?5?5?5?5?5?5?3?5?$CFd?6@ 0000000140053628     GameServerManagerDlg.obj
 0002:00008648       ??_C@_0BL@NKLPBGLH@nAim_Shot_Avg?5?5?5?5?5?5?5?5?3?5?$CFd?6@ 0000000140053648     GameServerManagerDlg.obj
 0002:00008668       ??_C@_0BI@BOFDJPCM@nAim_Headshot_Avg?7?3?5?$CFd?6@ 0000000140053668     GameServerManagerDlg.obj
 0002:00008680       ??_C@_0BF@FHGGGDHM@nAim_Kill_Avg?7?7?3?5?$CFd?6@ 0000000140053680     GameServerManagerDlg.obj
 0002:00008698       ??_C@_0BH@PNOCPAOF@nAim_Assist_Avg?7?7?3?5?$CFd?6@ 0000000140053698     GameServerManagerDlg.obj
 0002:000086b0       ??_C@_0BJ@PICLMOLF@nAim_Play_Time_Avg?7?3?5?$CFd?6@ 00000001400536b0     GameServerManagerDlg.obj
 0002:000086d0       ??_C@_0CD@LKFICJNG@?$FLRWPM?$FNNot?5Processing?5tIndex?$FL?$CFd?$FN@ 00000001400536d0     GameServerManagerDlg.obj
 0002:000086f8       ??_C@_0DP@GOABOJEI@PROTO_GAMEGT_INGAME_AIGACHA_ITE@ 00000001400536f8     GameServerManagerDlg.obj
 0002:00008738       ??_C@_0DP@JLNCNAAJ@CGameServerManagerDlg?3?3RECV_MSG@ 0000000140053738     GameServerManagerDlg.obj
 0002:00008778       ??_C@_0DJ@EALHJMML@?7usn?5?$DN?5?$CFs?0?5Loop?5?$DN?5?$CFd?0?5IsReward?5@ 0000000140053778     GameServerManagerDlg.obj
 0002:000087c0       ??_C@_0EI@OAGFOPLM@GAMESERVERMSG_AUTO_SIDE_CHANGE_@ 00000001400537c0     GameServerManagerDlg.obj
 0002:00008808       ??_C@_0CN@LGNPEFKO@GAMESERVERMSG_INSERTCHARACTER_A@ 0000000140053808     GameServerManagerDlg.obj
 0002:00008840       ??_C@_0EO@KPIBEEEN@PROTOCOL_STARTING_GAME?5?9?5Check?5@ 0000000140053840     GameServerManagerDlg.obj
 0002:00008890       ??_C@_0CJ@LACMIMDI@PROTOCOL_STARTING_GAME?5?9?5Invali@ 0000000140053890     GameServerManagerDlg.obj
 0002:000088c0       ??_C@_0CI@ICNJDFAC@PROTOCOL_DESTROY_ROOM?5?9?5Invalid@ 00000001400538c0     GameServerManagerDlg.obj
 0002:000088e8       ??_C@_0CM@IIGBNHNC@PROTOCOL_INSERT_CHARACTER?5?9?5Inv@ 00000001400538e8     GameServerManagerDlg.obj
 0002:00008918       ??_C@_0CP@OAMCCHLG@PROTOCOL_MMSERVER_TERMINATED?5?9?5@ 0000000140053918     GameServerManagerDlg.obj
 0002:00008948       ??_C@_0CN@OCAJLFFO@PROTOCOL_USER_DISCONNECTED?5?9?5In@ 0000000140053948     GameServerManagerDlg.obj
 0002:00008980       ??_C@_0EE@FAJNOCKH@PROTOCOL_GAMEGT_INGAME_AIGACHA_@ 0000000140053980     GameServerManagerDlg.obj
 0002:000089c8       ??_C@_0CO@FDFLEIIH@PROTOCOL_GAMEGT_CODE_HUNTER?5?9?5I@ 00000001400539c8     GameServerManagerDlg.obj
 0002:000089f8       ??_C@_0DP@JBJDCCFM@PROTOCOL_SPECTATOR_RECOMMEND_RO@ 00000001400539f8     GameServerManagerDlg.obj
 0002:00008a38       ??_C@_0DE@OAOLACKN@PROTOCOL_AUTOMATCH_GAME_START_R@ 0000000140053a38     GameServerManagerDlg.obj
 0002:00008a70       ??_C@_0DE@POEHHEMJ@PROTOCOL_AUTOMATCH_GAME_ENTER_R@ 0000000140053a70     GameServerManagerDlg.obj
 0002:00008aa8       ??_C@_0CK@DHILECPN@PROTOCOL_STARTING_GAME?5?9?5Wrong?5@ 0000000140053aa8     GameServerManagerDlg.obj
 0002:00008ae0       ??_C@_0FA@CJLKCNIA@PROTOCOL_STARTING_GAME?5?9?5Assign@ 0000000140053ae0     GameServerManagerDlg.obj
 0002:00008b30       ??_C@_0EF@HHAOBBEM@PROTOCOL_STARTING_GAME?5?9?5Kill?5S@ 0000000140053b30     GameServerManagerDlg.obj
 0002:00008b80       ??_C@_0EE@ICMBCKPK@PROTOCOL_DESTROY_ROOM?5?9?5Kill?5Se@ 0000000140053b80     GameServerManagerDlg.obj
 0002:00008bc8       ??_C@_0CN@HHGMAEMA@PROTOCOL_INSERT_CHARACTER?5?9?5Wro@ 0000000140053bc8     GameServerManagerDlg.obj
 0002:00008c00       ??_C@_0HI@PNNNHNNB@PROTOCOL_INSERT_CHARACTER?5?3?5?$FL?$CFd@ 0000000140053c00     GameServerManagerDlg.obj
 0002:00008c78       ??_C@_0DI@FFJEJCIM@GAMESERVERMSG_INSERTCHARACTER?5?3@ 0000000140053c78     GameServerManagerDlg.obj
 0002:00008cb0       ??_C@_0DA@DNNLACHB@PROTOCOL_MMSERVER_TERMINATED?5?9?5@ 0000000140053cb0     GameServerManagerDlg.obj
 0002:00008ce0       ??_C@_0BK@IFHHIKHF@GAMESERVERMSG_KICKCLIENTS@ 0000000140053ce0     GameServerManagerDlg.obj
 0002:00008d00       ??_C@_0CO@JDAIKDKJ@PROTOCOL_USER_DISCONNECTED?5?9?5Wr@ 0000000140053d00     GameServerManagerDlg.obj
 0002:00008d30       ??_C@_0DJ@KDDALFMI@GAMESERVERMSG_USER_DISCONNECTED@ 0000000140053d30     GameServerManagerDlg.obj
 0002:00008d70       ??_C@_0DM@DKLDAHLA@PROTO_GAMEGT_INGAME_AIGACHA_ITE@ 0000000140053d70     GameServerManagerDlg.obj
 0002:00008db0       ??_C@_0CD@HHKHKHGE@USN?5?$CFlld?0?5ItemCount?5?$CFd?0?5Success@ 0000000140053db0     GameServerManagerDlg.obj
 0002:00008dd8       ??_C@_0DC@BKIEFOHD@PROTO_AUTOMATCH_GAME_START_REQ?5@ 0000000140053dd8     GameServerManagerDlg.obj
 0002:00008e10       ??_C@_0FI@EGKHAHLF@PROTO_AUTOMATCH_GAME_START_REQ?5@ 0000000140053e10     GameServerManagerDlg.obj
 0002:00008e70       ??_C@_0EN@GEKPHMND@PROTO_AUTOMATCH_GAME_START_REQ?5@ 0000000140053e70     GameServerManagerDlg.obj
 0002:00008ec0       ??_C@_0DC@FAEFFHEE@PROTO_AUTOMATCH_GAME_ENTER_REQ?5@ 0000000140053ec0     GameServerManagerDlg.obj
 0002:00008f00       ??_C@_0EF@OFIFDLII@PROTO_AUTOMATCH_GAME_ENTER_REQ?5@ 0000000140053f00     GameServerManagerDlg.obj
 0002:00008f50       ??_C@_0FE@LHECHLMH@PROTO_AUTOMATCH_GAME_ENTER_REQ?5@ 0000000140053f50     GameServerManagerDlg.obj
 0002:00008fb0       ??_C@_0FC@FANCBCIJ@PROTO_AUTOMATCH_GAME_ENTER_REQ?5@ 0000000140053fb0     GameServerManagerDlg.obj
 0002:00009010       ??_C@_0JB@KKMGKEOH@PROTO_AUTOMATCH_GAME_ENTER_REQ?5@ 0000000140054010     GameServerManagerDlg.obj
 0002:000090b0       ??_C@_0FA@NOMFLEIP@PROTOCOL_STARTING_GAME?5?9?5Server@ 00000001400540b0     GameServerManagerDlg.obj
 0002:00009100       ??_C@_0HA@GIGIOAGE@PROTOCOL_STARTING_GAME?5?9?5Wrong?5@ 0000000140054100     GameServerManagerDlg.obj
 0002:00009170       ??_C@_0FN@JKNIAPKP@PROTOCOL_STARTING_GAME?5?3?5USN?5?$CFs@ 0000000140054170     GameServerManagerDlg.obj
 0002:000091d0       ??_C@_0EG@JADNHOLE@GAMESERVERMSG_LOAD_MAP?5?3?5GameLo@ 00000001400541d0     GameServerManagerDlg.obj
 0002:00009220       ??_C@_0FI@LBNIJOLK@PROTO_AUTOMATCH_GAME_START_REQ?5@ 0000000140054220     GameServerManagerDlg.obj
 0002:00009280       ??_C@_0HI@NLDNGEDM@PROTO_AUTOMATCH_GAME_START_REQ?5@ 0000000140054280     GameServerManagerDlg.obj
 0002:00009300       ??_C@_0GP@LGBALBFF@PROTO_AUTOMATCH_GAME_START_REQ?5@ 0000000140054300     GameServerManagerDlg.obj
 0002:00009370       ??_C@_0FO@OCFMLFFO@PROTO_STARTING_GAME_RESULT?5?9?5ST@ 0000000140054370     GameServerManagerDlg.obj
 0002:000093d0       ??_C@_0FN@JOBJLDME@PROTO_STARTING_GAME_RESULT?5?9?5ST@ 00000001400543d0     GameServerManagerDlg.obj
 0002:00009430       ??_C@_0GC@OEEMHMKB@PROTO_AUTOMATCH_GAME_START_RES?5@ 0000000140054430     GameServerManagerDlg.obj
 0002:000094a0       ??_C@_0GB@DIGFFDIB@PROTO_AUTOMATCH_GAME_START_RES?5@ 00000001400544a0     GameServerManagerDlg.obj
 0002:00009508       ??_C@_0DN@CMJNEIBB@PROTO_AUTOMATCH_GAME_ENTER_RES?5@ 0000000140054508     GameServerManagerDlg.obj
 0002:00009548       ??_C@_0DL@BCMCPOIM@PROTO_AUTOMATCH_GAME_ENTER_RES?5@ 0000000140054548     GameServerManagerDlg.obj
 0002:00009588       ??_C@_0DO@OHPBKMIB@PROTO_AUTOMATCH_INGAME_ENTER_NT@ 0000000140054588     GameServerManagerDlg.obj
 0002:000095c8       ??_C@_0DO@DEOMHJEE@GAMESERVERMSG_AUTO_MATCH_STARTI@ 00000001400545c8     GameServerManagerDlg.obj
 0002:00009608       ??_C@_0CK@OBJHBBJK@InValid?5CopyData?5copy_data?9?$DOdwD@ 0000000140054608     GameServerManagerDlg.obj
 0002:00009638       ??_C@_0CM@ELGDMFLB@InValid?5GAMESERVERINDEX?5server_@ 0000000140054638     GameServerManagerDlg.obj
 0002:00009668       ??_C@_0BB@MOGOBHAF@list?$DMT?$DO?5too?5long@ 0000000140054668     GameServerManagerDlg.obj
 0002:00009688       ??_7?$_Ref_count@UGAMESERVERINFO@@@std@@6B@ 0000000140054688     GameServerManagerDlg.obj
 0002:000096a8       ??_C@_0L@JODCLDGE@RTID?3?$CFs?3?$CFd@ 00000001400546a8     GameServerManagerDlg.obj
 0002:000096b4       ??_C@_01IDAFKMJL@_@        00000001400546b4     GameServerManagerDlg.obj
 0002:000096b8       ??_C@_0BC@HBDDANDP@sggm_proxy_64?4dll@ 00000001400546b8     GameServerManagerDlg.obj
 0002:000096d0       ??_C@_0BE@PBACKDJE@getManagerSingleton@ 00000001400546d0     GameServerManagerDlg.obj
 0002:000096e4       ??_C@_02DPKJAMEF@?$CFd@    00000001400546e4     GameServerManagerDlg.obj
 0002:00009808       ??_7CGameServerManagerDlg@@6BIClientHandler@@@ 0000000140054808     GameServerManagerDlg.obj
 0002:00009830       ??_7CGameServerManagerDlg@@6BCDialog@@@ 0000000140054830     GameServerManagerDlg.obj
 0002:00009b58       ??_C@_0N@MDJJJHMB@kernel32?4dll@ 0000000140054b58     GameServerManagerDlg.obj
 0002:00009b70       ??_7IClientHandler@@6B@    0000000140054b70     GameServerManagerDlg.obj
 0002:00009b90       ??_C@_0BG@DDHFAIIG@CGMSConnManager?3?3Send@ 0000000140054b90     GMSConnManager.obj
 0002:00009ba8       ??_C@_0CJ@FPDEPCKA@?$FL?$CFs?$FN?5m_pSendBuffer?9?$DOWrite?5buffe@ 0000000140054ba8     GMSConnManager.obj
 0002:00009be0       ??_C@_0EP@PJPDMIGO@PROTOCOL_FINISHED_GAME?5?9?5Check?5@ 0000000140054be0     GMSConnManager.obj
 0002:00009c30       ??_C@_0DO@DKCACIIN@CGMSConnManager?3?3UpdateConnecti@ 0000000140054c30     GMSConnManager.obj
 0002:00009c70       ??_C@_0DJ@JBIEMPEN@CGMSConnManager?3?3UpdateConnecti@ 0000000140054c70     GMSConnManager.obj
 0002:00009cb0       ??_C@_0DK@FBGGFFEM@CGMSConnManager?3?3UpdateConnecti@ 0000000140054cb0     GMSConnManager.obj
 0002:00009cf0       ??_C@_0CM@NLEOHKJM@No?5Heartbeat?5Response?5Over?5Limi@ 0000000140054cf0     GMSConnManager.obj
 0002:00009d20       ??_C@_0CF@KGFDLMG@PROTOCOL_ALLOCABLEROOMCOUNT_CHA@ 0000000140054d20     GMSConnManager.obj
 0002:00009d48       ??_C@_08PJDNIBPN@?$HM?$CI?$CFd?$CJ?$HM?$CFd@ 0000000140054d48     GMSConnManager.obj
 0002:00009d58       ??_C@_0BF@DEODNPPB@GMS?5Spare?5send?5?$CFd?9?$CFd@ 0000000140054d58     GMSConnManager.obj
 0002:00009d70       ??_C@_0EB@NFPJKBDG@ABCDEFGHIJKLMNOPQRSTUVWXYZabcde@ 0000000140054d70     base64.obj
 0002:00009db4       ??_C@_06KNPIFKI@DATA?$AN?6@ 0000000140054db4     CSmtp.obj
 0002:00009dbc       ??_C@_03CGLHDMIP@?$CC?$AN?6@ 0000000140054dbc     CSmtp.obj
 0002:00009dc0       ??_C@_0CE@HELJGHDP@Content?9Transfer?9Encoding?3?5base@ 0000000140054dc0     CSmtp.obj
 0002:00009de8       ??_C@_0CM@KHGNHNHL@Content?9Disposition?3?5attachment@ 0000000140054de8     CSmtp.obj
 0002:00009e14       ??_C@_05KMJPGPH@?$AN?6?4?$AN?6@ 0000000140054e14     CSmtp.obj
 0002:00009e1c       ??_C@_05PLHGOPJD@LOGIN@    0000000140054e1c     CSmtp.obj
 0002:00009e24       ??_C@_05ONKJAIHP@PLAIN@    0000000140054e24     CSmtp.obj
 0002:00009e2c       ??_C@_01BJJEKLCA@?$CC@     0000000140054e2c     CSmtp.obj
 0002:00009e30       ??_C@_01JLIPDDHJ@?3@       0000000140054e30     CSmtp.obj
 0002:00009e34       ??_C@_06GNPEEHKO@From?3?5@ 0000000140054e34     CSmtp.obj
 0002:00009e3c       ??_C@_03DMHINEKI@?$DO?$AN?6@ 0000000140054e3c     CSmtp.obj
 0002:00009e40       ??_C@_04CLHDMCFI@To?3?5@   0000000140054e40     CSmtp.obj
 0002:00009e48       ??_C@_04LDGFDGHC@Cc?3?5@   0000000140054e48     CSmtp.obj
 0002:00009e50       ??_C@_09JHOEHIGO@Subject?3?5@ 0000000140054e50     CSmtp.obj
 0002:00009e5c       ??_C@_02BAABKJLB@?9?9@     0000000140054e5c     CSmtp.obj
 0002:00009e60       ??_C@_06FIMJICNC@QUIT?$AN?6@ 0000000140054e60     CSmtp.obj
 0002:00009e68       ??_C@_0BC@MNENJGIJ@HostStat?5Stopped?4@ 0000000140054e68     HostStat.obj
 0002:00009e80       ??_C@_0N@PEDACFPD@hoststat?4ini@ 0000000140054e80     HostStat.obj
 0002:00009e90       ??_C@_07PIJOPIMD@FileExt@  0000000140054e90     HostStat.obj
 0002:00009e98       ??_C@_07CKMABNOK@Setting@  0000000140054e98     HostStat.obj
 0002:00009ea0       ??_C@_07JAJNKICC@HackExt@  0000000140054ea0     HostStat.obj
 0002:00009ea8       ??_C@_06IOPDAEEL@LogExt@   0000000140054ea8     HostStat.obj
 0002:00009eb0       ??_C@_0O@CMFGOJCG@UserSystemExt@ 0000000140054eb0     HostStat.obj
 0002:00009ec0       ??_C@_0P@MBJBELOO@GameOption?4ini@ 0000000140054ec0     HostStat.obj
 0002:00009ed0       ??_C@_0BJ@HCNFFNOD@MD5?$CIGameOption?4ini?$CJ?$DN?$FL?$CFs?$FN@ 0000000140054ed0     HostStat.obj
 0002:00009ef0       ??_C@_0CF@CJLIKOPF@HostStat?5Started?5?$CG?5Exec?5ServerA@ 0000000140054ef0     HostStat.obj
 0002:00009f18       ??_C@_04FGAJMCLA@?2?$CK?4?$CK@ 0000000140054f18     HostStat.obj
 0002:00009f20       ??_C@_02DJGKEECL@?4?4@     0000000140054f20     HostStat.obj
 0002:00009f24       ??_C@_06GEKNBBDK@000000@   0000000140054f24     HostStat.obj
 0002:00009f2c       ??_C@_05BDHMEGNH@Retry@    0000000140054f2c     HostStat.obj
 0002:00009f38       ??_C@_07PBILKAFL@Success@  0000000140054f38     HostStat.obj
 0002:00009f40       ??_C@_06MAFFGDO@Active@    0000000140054f40     HostStat.obj
 0002:00009f48       ??_C@_06IANKLPDP@SendAt@   0000000140054f48     HostStat.obj
 0002:00009f50       ??_C@_07HAAJMFIA@Country@  0000000140054f50     HostStat.obj
 0002:00009f58       ??_C@_04FABLJDN@Name@      0000000140054f58     HostStat.obj
 0002:00009f60       ??_C@_0BI@NCBJMABA@?$CFs?2?$CF04d?$CF02d?$CF02d_?$CFs_?$CFs?$CFs@ 0000000140054f60     HostStat.obj
 0002:00009f78       ??_C@_08MLPOGMMH@?$CFd_?$CFd?3?$CFd@ 0000000140054f78     HostStat.obj
 0002:00009f84       ??_C@_04DICKPMGH@Data@     0000000140054f84     HostStat.obj
 0002:00009f90       ??_C@_0P@GANPGBFO@?$CFd?0?$CFd?0?$CFd?0?$CFd?0?$CFd@ 0000000140054f90     HostStat.obj
 0002:00009fa0       ??_C@_04CPPPJGME@Host@     0000000140054fa0     HostStat.obj
 0002:00009fa8       ??_C@_04JEGKNAHI@Mail@     0000000140054fa8     HostStat.obj
 0002:00009fb0       ??_C@_04HOKNCALA@Port@     0000000140054fb0     HostStat.obj
 0002:00009fb8       ??_C@_02IJGONHOJ@To@       0000000140054fb8     HostStat.obj
 0002:00009fbc       ??_C@_04LMIAFEOL@From@     0000000140054fbc     HostStat.obj
 0002:00009fc4       ??_C@_04ODLBFFJE@User@     0000000140054fc4     HostStat.obj
 0002:00009fd0       ??_C@_08FJIAHGMM@Password@ 0000000140054fd0     HostStat.obj
 0002:00009fdc       ??_C@_06OINDDGEP@Prefix@   0000000140054fdc     HostStat.obj
 0002:00009fe4       ??_C@_04KOACHJEN@Type@     0000000140054fe4     HostStat.obj
 0002:00009fec       ??_C@_06HFDFFJHI@Domain@   0000000140054fec     HostStat.obj
 0002:00009ff4       ??_C@_04KGCGDDND@NTLM@     0000000140054ff4     HostStat.obj
 0002:00009ffc       ??_C@_03HJHPABEB@250@      0000000140054ffc     HostStat.obj
 0002:0000a000       ??_C@_06CMLPEGNC@Failed@   0000000140055000     HostStat.obj
 0002:0000a008       ??_C@_0BG@FOGKECKD@?$FLHSS?$FN?5Sending?5?$CFs?5?$FL?$CFs?$FN@ 0000000140055008     HostStat.obj
 0002:0000a020       ??_C@_09GIPKOBEB@CPUActive@ 0000000140055020     HostStat.obj
 0002:0000a02c       ??_C@_04GJOELAAH@Perf@     000000014005502c     HostStat.obj
 0002:0000a038       ??_C@_08EDEGIDPJ@CPUTimer@ 0000000140055038     HostStat.obj
 0002:0000a048       ??_C@_0N@CKLMACF@MemoryActive@ 0000000140055048     HostStat.obj
 0002:0000a058       ??_C@_0M@KCEHBFOI@MemoryTimer@ 0000000140055058     HostStat.obj
 0002:0000a068       ??_C@_09LJFKOFBJ@MemoryBig@ 0000000140055068     HostStat.obj
 0002:0000a078       ??_C@_0N@BNIJLLIL@ServerAppBig@ 0000000140055078     HostStat.obj
 0002:0000a088       ??_C@_0CB@EIBAJGEI@Max?9Process?5?$FL?5name?$DN?$CFs?0?5size?$DN?$CFd?5@ 0000000140055088     HostStat.obj
 0002:0000a0b0       ??_C@_0L@BGPICFFH@UserActive@ 00000001400550b0     HostStat.obj
 0002:0000a0c0       ??_C@_09PAPOCIPE@UserTimer@ 00000001400550c0     HostStat.obj
 0002:0000a0d0       ??_C@_0CO@FCJBCHHE@?$CF04d?$CF02d?$CF02d?$CF02d?$CF02d?$CF02d?$DNuser?3?$CF@ 00000001400550d0     HostStat.obj
 0002:0000a100       ??_C@_09KPJBOBMP@LogActive@ 0000000140055100     HostStat.obj
 0002:0000a110       ??_C@_0BN@EAJBDIBA@?$CF04d?$CF02d?$CF02d?$CF02d?$CF02d?$CF02d?$DN?$CFs?6@ 0000000140055110     HostStat.obj
 0002:0000a130       ??_C@_0P@MCDGMPHH@?$CF04d?9?$CF02d?9?$CF02d@ 0000000140055130     HostStat.obj
 0002:0000a140       ??_C@_04BJPIHCBA@Info@     0000000140055140     HostStat.obj
 0002:0000a148       ??_C@_04FMEGDJGD@Date@     0000000140055148     HostStat.obj
 0002:0000a150       ??_C@_02MFEOMNPG@IP@       0000000140055150     HostStat.obj
 0002:0000a158       ??_C@_08EJIMMOH@HostName@  0000000140055158     HostStat.obj
 0002:0000a164       ??_C@_06BIMDCNJE@?$FLLog?$FN?6@ 0000000140055164     HostStat.obj
 0002:0000a170       ??_C@_0BH@PNAPDCDJ@UserPCSpecReportActive@ 0000000140055170     HostStat.obj
 0002:0000a188       ??_C@_09KKFGPCKE@?$FLDevice?$FN?6@ 0000000140055188     HostStat.obj
 0002:0000a198       ??_C@_0L@BICIGMKH@DataFolder@ 0000000140055198     HostStat.obj
 0002:0000a1a8       ??_C@_0N@NBCLACF@BackupFolder@ 00000001400551a8     HostStat.obj
 0002:0000a1b8       ??_C@_02BMJICGCB@rt@       00000001400551b8     HostStat.obj
 0002:0000a1c0       ??_C@_0O@FKEBMOAD@NetworkActive@ 00000001400551c0     HostStat.obj
 0002:0000a1d0       ??_C@_0BE@HAFMLGBJ@HostKillCountActive@ 00000001400551d0     HostStat.obj
 0002:0000a1e8       ??_C@_0BO@PAGBBCJF@SendMessageTimeOutCountActive@ 00000001400551e8     HostStat.obj
 0002:0000a208       ??_C@_05GKICOFAF@OS?3?$CFs@ 0000000140055208     HostStat.obj
 0002:0000a210       ??_C@_06EOAPLBNC@CPU?3?$CFs@ 0000000140055210     HostStat.obj
 0002:0000a218       ??_C@_06LKEAJFMB@GPU?3?$CFs@ 0000000140055218     HostStat.obj
 0002:0000a220       ??_C@_08CHDAIDJE@RAM?3?$CFdMB@ 0000000140055220     HostStat.obj
 0002:0000a22c       ??_C@_01LFCBOECM@?4@       000000014005522c     HostStat.obj
 0002:0000a238       ??_7CHostStat@@6B@         0000000140055238     HostStat.obj
 0002:0000a240       ??_C@_01NEMOKFLO@?$DN@     0000000140055240     iniReader.obj
 0002:0000a244       ??_C@_01LBDDMOBJ@?$FN@     0000000140055244     iniReader.obj
 0002:0000a248       ??_C@_01OHGJGJJP@?$FL@     0000000140055248     iniReader.obj
 0002:0000a250       ??_C@_0L@CDNOKCN@AUTH?5NTLM?5@ 0000000140055250     auth.obj
 0002:0000a25c       ??_C@_03KBCCNPJC@334@      000000014005525c     auth.obj
 0002:0000a260       ??_C@_03IFIJLG@235@        0000000140055260     auth.obj
 0002:0000a268       ??_C@_0DL@FAKPCBIM@451?5Requested?5action?5aborted?3?5l@ 0000000140055268     mailer.obj
 0002:0000a2a8       ??_C@_0DD@HEMFHKCO@451?5Requested?5action?5aborted?3?5l@ 00000001400552a8     mailer.obj
 0002:0000a2e0       ??_C@_0EK@NHOKGADJ@451?5Requested?5action?5aborted?3?5l@ 00000001400552e0     mailer.obj
 0002:0000a330       ??_C@_0DI@LAHDHEEJ@451?5Requested?5action?5aborted?3?5N@ 0000000140055330     mailer.obj
 0002:0000a368       ??_C@_0DI@MBLOLIGI@451?5Requested?5action?5aborted?3?5l@ 0000000140055368     mailer.obj
 0002:0000a3a0       ??_C@_0DE@MADOJHJN@451?5Requested?5action?5aborted?3?5s@ 00000001400553a0     mailer.obj
 0002:0000a3d8       ??_C@_0CO@BGNPEFON@554?5Transaction?5failed?3?5server?5@ 00000001400553d8     mailer.obj
 0002:0000a408       ??_C@_0DH@HNIHLPID@554?5Transaction?5failed?3?5server?5@ 0000000140055408     mailer.obj
 0002:0000a440       ??_C@_0M@KHMCPMBE@flibbletoot@ 0000000140055440     mailer.obj
 0002:0000a44c       ??_C@_05EGKLNPNB@EHLO?5@   000000014005544c     mailer.obj
 0002:0000a458       ??_C@_0CC@KHHGHGBH@554?5Transaction?5failed?3?5EHLO?5se@ 0000000140055458     mailer.obj
 0002:0000a480       ??_C@_0CF@MNLCOJPA@554?5Transaction?5failed?3?5EHLO?5re@ 0000000140055480     mailer.obj
 0002:0000a4a8       ??_C@_0DN@PJGGNHBC@554?5possibly?5trying?5to?5use?5AUTH@ 00000001400554a8     mailer.obj
 0002:0000a4e8       ??_C@_0CC@KDMHBKPA@554?5Transaction?5failed?3?5HELO?5se@ 00000001400554e8     mailer.obj
 0002:0000a510       ??_C@_0CF@BEDBIIGA@554?5Transaction?5failed?3?5HELO?5re@ 0000000140055510     mailer.obj
 0002:0000a538       ??_C@_0CB@GHKBDBNB@535?5Authentificaton?5unsuccessfu@ 0000000140055538     mailer.obj
 0002:0000a560       ??_C@_0M@BBBAEIPA@MAIL?5FROM?3?$DM@ 0000000140055560     mailer.obj
 0002:0000a570       ??_C@_0BM@BOABMLB@554?5MAIL?5FROM?5sending?5error@ 0000000140055570     mailer.obj
 0002:0000a590       ??_C@_0BM@FFPIIMMC@554?5MAIL?5FROM?5receipt?5error@ 0000000140055590     mailer.obj
 0002:0000a5b0       ??_C@_0L@DEDALBCA@RCPT?5TO?3?5?$DM@ 00000001400555b0     mailer.obj
 0002:0000a5c0       ??_C@_0BH@EIIENGPK@554?5Transaction?5failed@ 00000001400555c0     mailer.obj
 0002:0000a5d8       ??_C@_0BE@KINGKHJO@554?5DATA?5send?5error@ 00000001400555d8     mailer.obj
 0002:0000a5f0       ??_C@_0CA@LKIPLPAG@554?5DATA?0?5server?5response?5error@ 00000001400555f0     mailer.obj
 0002:0000a610       ??_C@_03KFKPKDCA@354@      0000000140055610     mailer.obj
 0002:0000a618       ??_C@_0CO@HMPIOICJ@554?5DATA?0?5server?5response?5error@ 0000000140055618     mailer.obj
 0002:0000a648       ??_C@_01EOFPKCAF@?$EA@     0000000140055648     mailer.obj
 0002:0000a650       ??_C@_0P@GHDLBHE@?$CJ?5?$AN?6Reply?9To?3?5@ 0000000140055650     mailer.obj
 0002:0000a660       ??_C@_02GFKOMOKH@?5?$CI@   0000000140055660     mailer.obj
 0002:0000a668       ??_C@_0N@ONAHKFDI@?$AN?6Reply?9To?3?5@ 0000000140055668     mailer.obj
 0002:0000a678       ??_C@_04FHJFLDEO@?0?$AN?6?5@ 0000000140055678     mailer.obj
 0002:0000a680       ??_C@_0CF@FECDGLOI@bounds?$DN_NextP_0056wi_0_8_ty7894@ 0000000140055680     mailer.obj
 0002:0000a6a8       ??_C@_0DP@CMMJOPIB@MIME?9Version?3?51?40?$AN?6Content?9Type@ 00000001400556a8     mailer.obj
 0002:0000a6e8       ??_C@_0BL@HPBMONOH@Date?3?5?$CFd?5?$CFb?5?$CFy?5?$CFH?3?$CFM?3?$CFS?5?$CFZ@ 00000001400556e8     mailer.obj
 0002:0000a704       ??_C@_04FMMHFHOO@?$AN?6?$AN?6@ 0000000140055704     mailer.obj
 0002:0000a710       ??_C@_0CI@PDOFMDNF@This?5is?5a?5MIME?5encapsulated?5mes@ 0000000140055710     mailer.obj
 0002:0000a740       ??_C@_0FC@IPCNFJKD@Content?9type?3?5text?1plain?$DL?5chars@ 0000000140055740     mailer.obj
 0002:0000a794       ??_C@_06CFENMJKO@?$AN?6?$AN?6?9?9@ 0000000140055794     mailer.obj
 0002:0000a7a0       ??_C@_0BN@HKKLOHFL@inner_jfd_0078hj_0_8_part_tp@ 00000001400557a0     mailer.obj
 0002:0000a7c0       ??_C@_0DC@GLDGJDED@Content?9Type?3?5multipart?1alterna@ 00000001400557c0     mailer.obj
 0002:0000a800       ??_C@_0FD@DEJLGDCA@Content?9type?3?5text?1html?$DL?5charse@ 0000000140055800     mailer.obj
 0002:0000a854       ??_C@_04KAODOPGN@?9?9?$AN?6@ 0000000140055854     mailer.obj
 0002:0000a85c       ??_C@_04LOEPKDGL@?$AN?6?9?9@ 000000014005585c     mailer.obj
 0002:0000a864       ??_C@_04JFHMGKLD@?4gif@    0000000140055864     mailer.obj
 0002:0000a870       ??_C@_0BL@PNONEHPN@Content?9Type?3?5image?1gif?$DL?$AN?6@ 0000000140055870     mailer.obj
 0002:0000a88c       ??_C@_04GNPKBLNA@?4jpg@    000000014005588c     mailer.obj
 0002:0000a894       ??_C@_04OFMADDDJ@jpeg@     0000000140055894     mailer.obj
 0002:0000a8a0       ??_C@_0BL@IFIDFMNO@Content?9Type?3?5image?1jpg?$DL?$AN?6@ 00000001400558a0     mailer.obj
 0002:0000a8bc       ??_C@_04LCMACLFG@?4txt@    00000001400558bc     mailer.obj
 0002:0000a8c8       ??_C@_0BL@ENNKJKEB@Content?9Type?3?5plain?1txt?$DL?$AN?6@ 00000001400558c8     mailer.obj
 0002:0000a8e4       ??_C@_04LJDDIHIK@?4bmp@    00000001400558e4     mailer.obj
 0002:0000a8f0       ??_C@_0BL@NLOEEIGO@Content?9Type?3?5image?1bmp?$DL?$AN?6@ 00000001400558f0     mailer.obj
 0002:0000a90c       ??_C@_04DKBFJDAN@?4htm@    000000014005590c     mailer.obj
 0002:0000a914       ??_C@_04PNIFHPHN@html@     0000000140055914     mailer.obj
 0002:0000a920       ??_C@_0BL@PHJGFJHD@Content?9Type?3?5plain?1htm?$DL?$AN?6@ 0000000140055920     mailer.obj
 0002:0000a93c       ??_C@_04EEOGCCFB@?4png@    000000014005593c     mailer.obj
 0002:0000a948       ??_C@_0BL@HPPBPMLF@Content?9Type?3?5image?1png?$DL?$AN?6@ 0000000140055948     mailer.obj
 0002:0000a964       ??_C@_04JLMDILM@?4exe@     0000000140055964     mailer.obj
 0002:0000a970       ??_C@_0CK@CAMLCJAN@Content?9Type?3?5application?1X?9exe@ 0000000140055970     mailer.obj
 0002:0000a9a0       ??_C@_0CH@LNEPLNBH@Content?9Type?3?5application?1X?9oth@ 00000001400559a0     mailer.obj
 0002:0000a9c8       ??_C@_07HLOIFENE@?7name?$DN?$CC@ 00000001400559c8     mailer.obj
 0002:0000a9d0       ??_C@_05GBEDKFGN@?$CC?$AN?6?$AN?6@ 00000001400559d0     mailer.obj
 0002:0000a9d8       ??_C@_0DE@HMAMCJKP@550?5Requested?5action?5not?5taken?3@ 00000001400559d8     mailer.obj
 0002:0000aa10       ??_C@_0DF@OGOOKDFI@451?5Requested?5action?5aborted?3?5d@ 0000000140055a10     mailer.obj
 0002:0000aa50       ??_C@_0EB@OKKDPGHP@451?5Requested?5action?5aborted?3?5s@ 0000000140055a50     mailer.obj
 0002:0000aaa0       ??_C@_0EI@BJOBFJMH@554?5jwSMTP?5only?5handles?5LOGIN?5o@ 0000000140055aa0     mailer.obj
 0002:0000aae8       ??_C@_05ILLKGEON@auth?5@   0000000140055ae8     mailer.obj
 0002:0000aaf0       ??_C@_0BJ@PNOLHJPG@554?5send?5failure?3?5?$CCauth?5@ 0000000140055af0     mailer.obj
 0002:0000ab10       ??_C@_0DD@EONLELJG@554?5receive?5failure?3?5waiting?5on@ 0000000140055b10     mailer.obj
 0002:0000ab48       ??_C@_0BB@LFFFMAKC@334?5VXNlcm5hbWU6@ 0000000140055b48     mailer.obj
 0002:0000ab60       ??_C@_0CD@LHABOJFE@554?5send?5failure?3?5sending?5usern@ 0000000140055b60     mailer.obj
 0002:0000ab88       ??_C@_0DD@LEHCKMHD@554?5receive?5failure?3?5waiting?5on@ 0000000140055b88     mailer.obj
 0002:0000abc0       ??_C@_0BB@LPENDHLO@334?5UGFzc3dvcmQ6@ 0000000140055bc0     mailer.obj
 0002:0000abd8       ??_C@_0CD@IPBELHNA@554?5send?5failure?3?5sending?5passw@ 0000000140055bd8     mailer.obj
 0002:0000ac00       ??_C@_0DF@LDLMMKNI@554?5receive?5failure?3?5waiting?5on@ 0000000140055c00     mailer.obj
 0002:0000ac38       ??_C@_0M@PPCILILI@auth?5plain?5@ 0000000140055c38     mailer.obj
 0002:0000ac48       ??_C@_0DJ@EEMHIHKA@554?5send?5failure?3?5sending?5login@ 0000000140055c48     mailer.obj
 0002:0000ac90       ??_C@_0EC@IMOCLIGP@554?5receive?5failure?3?5waiting?5on@ 0000000140055c90     mailer.obj
 0002:0000ace0       ??_C@_0EB@OBNNBDCF@554?5receive?5failure?3?5timeout?5er@ 0000000140055ce0     mailer.obj
 0002:0000ad28       ??_C@_0BE@HLKFLAJF@GetNativeSystemInfo@ 0000000140055d28     smbutil.obj
 0002:0000ad3c       ??_C@_02PGHGPEOM@?91@      0000000140055d3c     md5wrapper.obj
 0002:0000ad40       ??_C@_08IGMCDLDE@LogLevel@ 0000000140055d40     HostLogger.obj
 0002:0000ad50       ??_C@_07KMMFIOCI@LogInfo@  0000000140055d50     HostLogger.obj
 0002:0000ad58       ??_C@_06LFKIJBMM@IPCMsg@   0000000140055d58     HostLogger.obj
 0002:0000ad60       ??_C@_09HNBAJPOD@IPCMemory@ 0000000140055d60     HostLogger.obj
 0002:0000ad70       ??_C@_0N@MJMCCHJI@?2?$CFd?$CF02d?$CF02d?2@ 0000000140055d70     HostLogger.obj
 0002:0000ad80       ??_C@_0BI@PDBNHNN@?$CFs?2BattleRoyal_?$CFs_?$CFs_?$CFs@ 0000000140055d80     HostLogger.obj
 0002:0000ad98       ??_C@_0BD@PBMCFJCL@?$CFs?2kernel_?$CFs_?$CFs_?$CFs@ 0000000140055d98     HostLogger.obj
 0002:0000adb0       ??_C@_0BD@DFOFGCOM@?$CFs?2packet_?$CFs_?$CFs_?$CFs@ 0000000140055db0     HostLogger.obj
 0002:0000adc8       ??_C@_0BM@EPJGHEGG@?$CFs?2mode_user_count_?$CFs_?$CFs_?$CFs@ 0000000140055dc8     HostLogger.obj
 0002:0000ade8       ??_C@_0CA@HLCLJLLN@?$CFs?2serverapp_use_count_?$CFs_?$CFs_?$CFs@ 0000000140055de8     HostLogger.obj
 0002:0000ae08       ??_C@_0BB@HFDGAAKA@?$CFs?2RWPM_?$CFs_?$CFs_?$CFs@ 0000000140055e08     HostLogger.obj
 0002:0000ae20       ??_C@_0BD@PILJABOB@?$CFs?2IPCMSG_?$CFs_?$CFs_?$CFs@ 0000000140055e20     HostLogger.obj
 0002:0000ae38       ??_C@_0DE@LGCHENKA@?$CFs?0?$CFs?0?$CF04d?4?$CF02d?4?$CF02d?5?$CF02d?3?$CF02d?3@ 0000000140055e38     HostLogger.obj
 0002:0000ae70       ??_C@_0CN@CAJJCFEC@?$CF04d?4?$CF02d?4?$CF02d?5?$CF02d?3?$CF02d?3?$CF02d?4?$CF@ 0000000140055e70     HostLogger.obj
 0002:0000aea0       ??_C@_0BP@NPJOKJI@?$CF02d?3?$CF02d?3?$CF02d?4?$CF03d?0Count?0?$CFs?5?6@ 0000000140055ea0     HostLogger.obj
 0002:0000aec0       ??_C@_0CJ@NOHHCMFI@?$CF04d?9?$CF02d?9?$CF02d?9?$CF02d?3?$CF02d?3?$CF02d?4?$CF@ 0000000140055ec0     HostLogger.obj
 0002:0000aef0       ??_C@_0L@PIHNNPCB@?$CFs?5?$FLLOW__?$FN@ 0000000140055ef0     HostLogger.obj
 0002:0000af00       ??_C@_0L@GMIAMKIO@?$CFs?5?$FLINFO_?$FN@ 0000000140055f00     HostLogger.obj
 0002:0000af10       ??_C@_0L@IHOLMJOP@?$CFs?5?$FLWARN_?$FN@ 0000000140055f10     HostLogger.obj
 0002:0000af20       ??_C@_0L@ECIMMAAL@?$CFs?5?$FLERROR?$FN@ 0000000140055f20     HostLogger.obj
 0002:0000af30       ??_C@_0L@IPABKGEK@?$CFs?5?$FLFATAL?$FN@ 0000000140055f30     HostLogger.obj
 0002:0000af40       ??_C@_08IHOEFJCP@?$CFs?5?$CFs?5?$AN?6@ 0000000140055f40     HostLogger.obj
 0002:0000af58       ??_7CMustSyncObjectLog@@6B@ 0000000140055f58     HostLogger.obj
 0002:0000af60       ??_C@_0CH@PGEFEDF@?4?1rez?1NationMsz?1MSG_DEFINE_GSM_@ 0000000140055f60     LogMsgManager.obj
 0002:0000af88       ??_C@_0BA@HOCBHDBJ@GSM_LogDataSize@ 0000000140055f88     LogMsgManager.obj
 0002:0000af98       ??_C@_0P@ILPGKNAO@GSM_LogData?9?$CFd@ 0000000140055f98     LogMsgManager.obj
 0002:0000afb0       ??_7FindXlsMsg@@6B@        0000000140055fb0     LoadXlsMsg.obj
 0002:0000afb8       ??_C@_03JMHOMAJH@?$CJ?5?$CC@ 0000000140055fb8     safe_string_x64:safe_string.obj
 0002:0000afbc       ??_C@_03MFPIGDOF@?5?$DO?5@ 0000000140055fbc     safe_string_x64:safe_string.obj
 0002:0000afc0       ??_C@_0BE@EGPJCBFC@?5warning?5sprintf?3?5?$CI@ 0000000140055fc0     safe_string_x64:safe_string.obj
 0002:0000afd8       ??_C@_07DNAEFDKF@sprintf@  0000000140055fd8     safe_string_x64:safe_string.obj
 0002:0000afe0       ??_C@_0BD@MFEJDGPJ@?5warning?5strcpy?3?5?$CI@ 0000000140055fe0     safe_string_x64:safe_string.obj
 0002:0000aff8       ??_C@_08IBECHLLM@strcpy_s@ 0000000140055ff8     safe_string_x64:safe_string.obj
 0002:0000b008       ??_C@_0BD@JCAAKJFN@warning?5strncpy?3?5?$CI@ 0000000140056008     safe_string_x64:safe_string.obj
 0002:0000b020       ??_C@_07EDFCNFDJ@strncpy@  0000000140056020     safe_string_x64:safe_string.obj
 0002:0000b028       ??_8?$basic_stringstream@DU?$char_traits@D@std@@V?$allocator@D@2@@std@@7B?$basic_ostream@DU?$char_traits@D@std@@@1@@ 0000000140056028     safe_string_x64:safe_string.obj
 0002:0000b038       ??_7?$basic_stringbuf@DU?$char_traits@D@std@@V?$allocator@D@2@@std@@6B@ 0000000140056038     safe_string_x64:safe_string.obj
 0002:0000b0b8       ??_7?$basic_stringstream@DU?$char_traits@D@std@@V?$allocator@D@2@@std@@6B@ 00000001400560b8     safe_string_x64:safe_string.obj
 0002:0000b0c0       ??_8?$basic_stringstream@DU?$char_traits@D@std@@V?$allocator@D@2@@std@@7B?$basic_istream@DU?$char_traits@D@std@@@1@@ 00000001400560c0     safe_string_x64:safe_string.obj
 0002:0000b0c8       __real@3b800000            00000001400560c8     HostStat.obj
 0002:0000b0cc       __real@3e666666            00000001400560cc     StdAfx.obj
 0002:0000b0d0       __real@3f466666            00000001400560d0     StdAfx.obj
 0002:0000b0d8       __real@3ff0000000000000    00000001400560d8     StdAfx.obj
 0002:0000b0e0       __real@4010000000000000    00000001400560e0     StdAfx.obj
 0002:0000b0e8       __real@41800000            00000001400560e8     StdAfx.obj
 0002:0000b0ec       __real@42c80000            00000001400560ec     HostStat.obj
 0002:0000b0f0       __xmm@00000000000000010000000100000001 00000001400560f0     HostStat.obj
 0002:0000b100       __xmm@00000000000000070000000000000000 0000000140056100     crs_uploader.obj
 0002:0000b110       __xmm@000000000000000f0000000000000000 0000000140056110     safe_string_x64:safe_string.obj
 0002:0000b120       __xmm@00000000ffffffffffffffffffffffff 0000000140056120     StdAfx.obj
 0002:0000b130       __xmm@0000001e0000001f0000001e0000001f 0000000140056130     DateTime.obj
 0002:0000b140       __xmm@0000001f0000001c0000001f0000001f 0000000140056140     DateTime.obj
 0002:0000b150       __xmm@0000001f0000001e0000001f0000001e 0000000140056150     DateTime.obj
 0002:0000b160       __xmm@3e22f9833e22f9833e22f9833e22f983 0000000140056160     StdAfx.obj
 0002:0000b170       __xmm@3f0000003f0000003f0000003f000000 0000000140056170     StdAfx.obj
 0002:0000b180       __xmm@3f8000003f8000003f8000003f800000 0000000140056180     StdAfx.obj
 0002:0000b190       __xmm@3fc90fdb3fc90fdb3fc90fdb3fc90fdb 0000000140056190     StdAfx.obj
 0002:0000b1a0       __xmm@40c90fdb40c90fdb40c90fdb40c90fdb 00000001400561a0     StdAfx.obj
 0002:0000b1b0       __xmm@bf800000bf800000bf800000bf800000 00000001400561b0     StdAfx.obj
 0002:0000c770       _load_config_used          0000000140057770     msvcrt:loadcfg.obj
 0002:0000c870       _tls_used                  0000000140057870     msvcrt:tlssup.obj
 0002:0000c8a0       ??_R4type_info@@6B@        00000001400578a0     msvcrt:std_type_info_static.obj
 0002:0000c8c8       ??_R3type_info@@8          00000001400578c8     msvcrt:std_type_info_static.obj
 0002:0000c8e0       ??_R2type_info@@8          00000001400578e0     msvcrt:std_type_info_static.obj
 0002:0000c8f0       ??_R1A@?0A@EA@type_info@@8 00000001400578f0     msvcrt:std_type_info_static.obj
 0002:0000c918       ??_R2CServerLog@@8         0000000140057918     LogMgmt.obj
 0002:0000c928       ??_R1A@?0A@EA@CServerLog@@8 0000000140057928     LogMgmt.obj
 0002:0000c950       ??_R3CServerLog@@8         0000000140057950     LogMgmt.obj
 0002:0000c968       ??_R4CServerLog@@6B@       0000000140057968     LogMgmt.obj
 0002:0000c990       ??_R2CReceiver@@8          0000000140057990     SGGMCallBackObj.obj
 0002:0000c9a8       ??_R2CSGGMCallBackObj@@8   00000001400579a8     SGGMCallBackObj.obj
 0002:0000c9c0       ??_R1A@?0A@EA@CReceiver@@8 00000001400579c0     SGGMCallBackObj.obj
 0002:0000c9e8       ??_R1A@?0A@EA@CSGGMCallBackObj@@8 00000001400579e8     SGGMCallBackObj.obj
 0002:0000ca10       ??_R3CReceiver@@8          0000000140057a10     SGGMCallBackObj.obj
 0002:0000ca28       ??_R3CSGGMCallBackObj@@8   0000000140057a28     SGGMCallBackObj.obj
 0002:0000ca40       ??_R4CReceiver@@6B@        0000000140057a40     SGGMCallBackObj.obj
 0002:0000ca68       ??_R4CSGGMCallBackObj@@6B@ 0000000140057a68     SGGMCallBackObj.obj
 0002:0000ca90       ??_R1A@?0A@EA@MultiReceiver@sggm_proxy@@8 0000000140057a90     SGGMCallBackObj.obj
 0002:0000cab8       ??_R2MultiReceiver@sggm_proxy@@8 0000000140057ab8     SGGMCallBackObj.obj
 0002:0000cac8       ??_R3MultiReceiver@sggm_proxy@@8 0000000140057ac8     SGGMCallBackObj.obj
 0002:0000cae0       ??_R4MultiReceiver@sggm_proxy@@6B@ 0000000140057ae0     SGGMCallBackObj.obj
 0002:0000cb08       ??_R1A@?0A@EA@EventReceiver@sggm@@8 0000000140057b08     SGGMCallBackObj.obj
 0002:0000cb30       ??_R2EventReceiver@sggm@@8 0000000140057b30     SGGMCallBackObj.obj
 0002:0000cb40       ??_R3EventReceiver@sggm@@8 0000000140057b40     SGGMCallBackObj.obj
 0002:0000cb58       ??_R2CClientLib@@8         0000000140057b58     ClientLib.obj
 0002:0000cb68       ??_R2?$CircuitQueue@E@@8   0000000140057b68     ClientLib.obj
 0002:0000cb78       ??_R2SendBuffer@@8         0000000140057b78     ClientLib.obj
 0002:0000cb88       ??_R1A@?0A@EA@CClientLib@@8 0000000140057b88     ClientLib.obj
 0002:0000cbb0       ??_R1A@?0A@EA@?$CircuitQueue@E@@8 0000000140057bb0     ClientLib.obj
 0002:0000cbd8       ??_R1A@?0A@EA@SendBuffer@@8 0000000140057bd8     ClientLib.obj
 0002:0000cc00       ??_R3CClientLib@@8         0000000140057c00     ClientLib.obj
 0002:0000cc18       ??_R3?$CircuitQueue@E@@8   0000000140057c18     ClientLib.obj
 0002:0000cc30       ??_R3SendBuffer@@8         0000000140057c30     ClientLib.obj
 0002:0000cc48       ??_R4CClientLib@@6B@       0000000140057c48     ClientLib.obj
 0002:0000cc70       ??_R4?$CircuitQueue@E@@6B@ 0000000140057c70     ClientLib.obj
 0002:0000cc98       ??_R4SendBuffer@@6B@       0000000140057c98     ClientLib.obj
 0002:0000ccc0       ??_R2CPacket@@8            0000000140057cc0     Packet.obj
 0002:0000ccd0       ??_R1A@?0A@EA@CPacket@@8   0000000140057cd0     Packet.obj
 0002:0000ccf8       ??_R3CPacket@@8            0000000140057cf8     Packet.obj
 0002:0000cd10       ??_R4CPacket@@6B@          0000000140057d10     Packet.obj
 0002:0000cd38       ??_R2CSFGameServerClientLib@@8 0000000140057d38     SFGameServerClientLib.obj
 0002:0000cd50       ??_R1A@?0A@EA@CSFGameServerClientLib@@8 0000000140057d50     SFGameServerClientLib.obj
 0002:0000cd78       ??_R3CSFGameServerClientLib@@8 0000000140057d78     SFGameServerClientLib.obj
 0002:0000cd90       ??_R4CSFGameServerClientLib@@6B@ 0000000140057d90     SFGameServerClientLib.obj
 0002:0000cdb8       ??_R2CDialog@@8            0000000140057db8     AppInfoDlg.obj
 0002:0000cde0       ??_R3CDialog@@8            0000000140057de0     AppInfoDlg.obj
 0002:0000cdf8       ??_R1A@?0A@EA@CDialog@@8   0000000140057df8     AppInfoDlg.obj
 0002:0000ce20       ??_R1A@?0A@EA@GAMEPROTO_SC_HOST_STAT@@8 0000000140057e20     AppInfoDlg.obj
 0002:0000ce48       ??_R2GAMEPROTO_SC_HOST_STAT@@8 0000000140057e48     AppInfoDlg.obj
 0002:0000ce68       ??_R3GAMEPROTO_SC_HOST_STAT@@8 0000000140057e68     AppInfoDlg.obj
 0002:0000ce80       ??_R4GAMEPROTO_SC_HOST_STAT@@6B@ 0000000140057e80     AppInfoDlg.obj
 0002:0000cea8       ??_R1A@?0A@EA@GAMEPROTO_SC_HOST_USER_STAT@@8 0000000140057ea8     AppInfoDlg.obj
 0002:0000ced0       ??_R2GAMEPROTO_SC_HOST_USER_STAT@@8 0000000140057ed0     AppInfoDlg.obj
 0002:0000cef0       ??_R3GAMEPROTO_SC_HOST_USER_STAT@@8 0000000140057ef0     AppInfoDlg.obj
 0002:0000cf08       ??_R4GAMEPROTO_SC_HOST_USER_STAT@@6B@ 0000000140057f08     AppInfoDlg.obj
 0002:0000cf30       ??_R1A@?0A@EA@GAMEPROTO_SC_REMOVECLIENT@@8 0000000140057f30     AppInfoDlg.obj
 0002:0000cf58       ??_R2GAMEPROTO_SC_REMOVECLIENT@@8 0000000140057f58     AppInfoDlg.obj
 0002:0000cf78       ??_R3GAMEPROTO_SC_REMOVECLIENT@@8 0000000140057f78     AppInfoDlg.obj
 0002:0000cf90       ??_R4GAMEPROTO_SC_REMOVECLIENT@@6B@ 0000000140057f90     AppInfoDlg.obj
 0002:0000cfb8       ??_R1A@?0A@EA@GAMEPROTO_CS_COMMON@@8 0000000140057fb8     AppInfoDlg.obj
 0002:0000cfe0       ??_R2GAMEPROTO_CS_COMMON@@8 0000000140057fe0     AppInfoDlg.obj
 0002:0000cff8       ??_R3GAMEPROTO_CS_COMMON@@8 0000000140057ff8     AppInfoDlg.obj
 0002:0000d010       ??_R1A@?0A@EA@GAMEPROTO_SS_GAMEEND@@8 0000000140058010     AppInfoDlg.obj
 0002:0000d038       ??_R2GAMEPROTO_SS_GAMEEND@@8 0000000140058038     AppInfoDlg.obj
 0002:0000d058       ??_R3GAMEPROTO_SS_GAMEEND@@8 0000000140058058     AppInfoDlg.obj
 0002:0000d070       ??_R4GAMEPROTO_SS_GAMEEND@@6B@ 0000000140058070     AppInfoDlg.obj
 0002:0000d098       ??_R1A@?0A@EA@exception@std@@8 0000000140058098     AppInfoDlg.obj
 0002:0000d0c0       ??_R2exception@std@@8      00000001400580c0     AppInfoDlg.obj
 0002:0000d0d0       ??_R3exception@std@@8      00000001400580d0     AppInfoDlg.obj
 0002:0000d0e8       ??_R4exception@std@@6B@    00000001400580e8     AppInfoDlg.obj
 0002:0000d110       ??_R1A@?0A@EA@GAMEPROTO_SC_SPY_CHANGE@@8 0000000140058110     AppInfoDlg.obj
 0002:0000d138       ??_R2GAMEPROTO_SC_SPY_CHANGE@@8 0000000140058138     AppInfoDlg.obj
 0002:0000d158       ??_R3GAMEPROTO_SC_SPY_CHANGE@@8 0000000140058158     AppInfoDlg.obj
 0002:0000d170       ??_R4GAMEPROTO_SC_SPY_CHANGE@@6B@ 0000000140058170     AppInfoDlg.obj
 0002:0000d198       ??_R1A@?0A@EA@GAMEPROTO_SC_COMMON@@8 0000000140058198     AppInfoDlg.obj
 0002:0000d1c0       ??_R2GAMEPROTO_COMMON@@8   00000001400581c0     AppInfoDlg.obj
 0002:0000d1d0       ??_R3GAMEPROTO_COMMON@@8   00000001400581d0     AppInfoDlg.obj
 0002:0000d1e8       ??_R1A@?0A@EA@GAMEPROTO_COMMON@@8 00000001400581e8     AppInfoDlg.obj
 0002:0000d210       ??_R2GAMEPROTO_SC_COMMON@@8 0000000140058210     AppInfoDlg.obj
 0002:0000d228       ??_R3GAMEPROTO_SC_COMMON@@8 0000000140058228     AppInfoDlg.obj
 0002:0000d240       ??_R1A@?0A@EA@CEdit@@8     0000000140058240     AppInfoDlg.obj
 0002:0000d268       ??_R2CWnd@@8               0000000140058268     AppInfoDlg.obj
 0002:0000d288       ??_R3CWnd@@8               0000000140058288     AppInfoDlg.obj
 0002:0000d2a0       ??_R1A@?0A@EA@CWnd@@8      00000001400582a0     AppInfoDlg.obj
 0002:0000d2c8       ??_R2CCmdTarget@@8         00000001400582c8     AppInfoDlg.obj
 0002:0000d2e0       ??_R3CCmdTarget@@8         00000001400582e0     AppInfoDlg.obj
 0002:0000d2f8       ??_R1A@?0A@EA@CCmdTarget@@8 00000001400582f8     AppInfoDlg.obj
 0002:0000d320       ??_R2CObject@@8            0000000140058320     AppInfoDlg.obj
 0002:0000d330       ??_R3CObject@@8            0000000140058330     AppInfoDlg.obj
 0002:0000d348       ??_R1A@?0A@EA@CObject@@8   0000000140058348     AppInfoDlg.obj
 0002:0000d370       ??_R2CEdit@@8              0000000140058370     AppInfoDlg.obj
 0002:0000d398       ??_R3CEdit@@8              0000000140058398     AppInfoDlg.obj
 0002:0000d3b0       ??_R4CEdit@@6B@            00000001400583b0     AppInfoDlg.obj
 0002:0000d3d8       ??_R2CGameServerManagerApp@@8 00000001400583d8     GameServerManager.obj
 0002:0000d408       ??_R2CWinApp@@8            0000000140058408     GameServerManager.obj
 0002:0000d430       ??_R2CWinThread@@8         0000000140058430     GameServerManager.obj
 0002:0000d450       ??_R1A@?0A@EA@CGameServerManagerApp@@8 0000000140058450     GameServerManager.obj
 0002:0000d478       ??_R1A@?0A@EA@CWinApp@@8   0000000140058478     GameServerManager.obj
 0002:0000d4a0       ??_R1A@?0A@EA@CWinThread@@8 00000001400584a0     GameServerManager.obj
 0002:0000d4c8       ??_R3CWinApp@@8            00000001400584c8     GameServerManager.obj
 0002:0000d4e0       ??_R3CWinThread@@8         00000001400584e0     GameServerManager.obj
 0002:0000d4f8       ??_R3CGameServerManagerApp@@8 00000001400584f8     GameServerManager.obj
 0002:0000d510       ??_R4CGameServerManagerApp@@6B@ 0000000140058510     GameServerManager.obj
 0002:0000d538       ??_R2?$_Ref_count@UGAMESERVERINFO@@@std@@8 0000000140058538     GameServerManagerDlg.obj
 0002:0000d550       ??_R2CGameServerManagerDlg@@8 0000000140058550     GameServerManagerDlg.obj
 0002:0000d588       ??_R2IClientHandler@@8     0000000140058588     GameServerManagerDlg.obj
 0002:0000d598       ??_R2_Ref_count_base@std@@8 0000000140058598     GameServerManagerDlg.obj
 0002:0000d5a8       ??_R3_Ref_count_base@std@@8 00000001400585a8     GameServerManagerDlg.obj
 0002:0000d5c0       ??_R1A@?0A@EA@_Ref_count_base@std@@8 00000001400585c0     GameServerManagerDlg.obj
 0002:0000d5e8       ??_R1A@?0A@EA@?$_Ref_count@UGAMESERVERINFO@@@std@@8 00000001400585e8     GameServerManagerDlg.obj
 0002:0000d610       ??_R1BDA@?0A@EA@IClientHandler@@8 0000000140058610     GameServerManagerDlg.obj
 0002:0000d638       ??_R1A@?0A@EA@CGameServerManagerDlg@@8 0000000140058638     GameServerManagerDlg.obj
 0002:0000d660       ??_R1A@?0A@EA@IClientHandler@@8 0000000140058660     GameServerManagerDlg.obj
 0002:0000d688       ??_R3?$_Ref_count@UGAMESERVERINFO@@@std@@8 0000000140058688     GameServerManagerDlg.obj
 0002:0000d6a0       ??_R3CGameServerManagerDlg@@8 00000001400586a0     GameServerManagerDlg.obj
 0002:0000d6b8       ??_R3IClientHandler@@8     00000001400586b8     GameServerManagerDlg.obj
 0002:0000d6d0       ??_R4?$_Ref_count@UGAMESERVERINFO@@@std@@6B@ 00000001400586d0     GameServerManagerDlg.obj
 0002:0000d6f8       ??_R4CGameServerManagerDlg@@6BIClientHandler@@@ 00000001400586f8     GameServerManagerDlg.obj
 0002:0000d720       ??_R4CGameServerManagerDlg@@6BCDialog@@@ 0000000140058720     GameServerManagerDlg.obj
 0002:0000d748       ??_R4IClientHandler@@6B@   0000000140058748     GameServerManagerDlg.obj
 0002:0000d770       ??_R2CHostStat@@8          0000000140058770     HostStat.obj
 0002:0000d780       ??_R1A@?0A@EA@CHostStat@@8 0000000140058780     HostStat.obj
 0002:0000d7a8       ??_R3CHostStat@@8          00000001400587a8     HostStat.obj
 0002:0000d7c0       ??_R4CHostStat@@6B@        00000001400587c0     HostStat.obj
 0002:0000d7e8       ??_R2?$basic_istream@DU?$char_traits@D@std@@@std@@8 00000001400587e8     mailer.obj
 0002:0000d810       ??_R2?$basic_ios@DU?$char_traits@D@std@@@std@@8 0000000140058810     mailer.obj
 0002:0000d830       ??_R2ios_base@std@@8       0000000140058830     mailer.obj
 0002:0000d848       ??_R2?$_Iosb@H@std@@8      0000000140058848     mailer.obj
 0002:0000d858       ??_R2?$basic_streambuf@DU?$char_traits@D@std@@@std@@8 0000000140058858     mailer.obj
 0002:0000d868       ??_R17A@3EA@?$_Iosb@H@std@@8 0000000140058868     mailer.obj
 0002:0000d890       ??_R1A@A@3EA@ios_base@std@@8 0000000140058890     mailer.obj
 0002:0000d8b8       ??_R1A@A@3FA@?$basic_ios@DU?$char_traits@D@std@@@std@@8 00000001400588b8     mailer.obj
 0002:0000d8e0       ??_R1A@?0A@EA@?$basic_istream@DU?$char_traits@D@std@@@std@@8 00000001400588e0     mailer.obj
 0002:0000d908       ??_R1A@?0A@EA@?$basic_ios@DU?$char_traits@D@std@@@std@@8 0000000140058908     mailer.obj
 0002:0000d930       ??_R17?0A@EA@?$_Iosb@H@std@@8 0000000140058930     mailer.obj
 0002:0000d958       ??_R1A@?0A@EA@ios_base@std@@8 0000000140058958     mailer.obj
 0002:0000d980       ??_R1A@?0A@EA@?$_Iosb@H@std@@8 0000000140058980     mailer.obj
 0002:0000d9a8       ??_R1A@?0A@EA@?$basic_streambuf@DU?$char_traits@D@std@@@std@@8 00000001400589a8     mailer.obj
 0002:0000d9d0       ??_R3?$basic_istream@DU?$char_traits@D@std@@@std@@8 00000001400589d0     mailer.obj
 0002:0000d9e8       ??_R3ios_base@std@@8       00000001400589e8     mailer.obj
 0002:0000da00       ??_R3?$_Iosb@H@std@@8      0000000140058a00     mailer.obj
 0002:0000da18       ??_R3?$basic_ios@DU?$char_traits@D@std@@@std@@8 0000000140058a18     mailer.obj
 0002:0000da30       ??_R3?$basic_streambuf@DU?$char_traits@D@std@@@std@@8 0000000140058a30     mailer.obj
 0002:0000da48       ??_R1A@?0A@EA@CMustSyncObjectLog@@8 0000000140058a48     HostLogger.obj
 0002:0000da70       ??_R1A@?0A@EA@_RTL_CRITICAL_SECTION@@8 0000000140058a70     HostLogger.obj
 0002:0000da98       ??_R2_RTL_CRITICAL_SECTION@@8 0000000140058a98     HostLogger.obj
 0002:0000daa8       ??_R3_RTL_CRITICAL_SECTION@@8 0000000140058aa8     HostLogger.obj
 0002:0000dac0       ??_R17?0A@EA@_RTL_CRITICAL_SECTION@@8 0000000140058ac0     HostLogger.obj
 0002:0000dae8       ??_R2CMustSyncObjectLog@@8 0000000140058ae8     HostLogger.obj
 0002:0000db00       ??_R3CMustSyncObjectLog@@8 0000000140058b00     HostLogger.obj
 0002:0000db18       ??_R4CMustSyncObjectLog@@6B@ 0000000140058b18     HostLogger.obj
 0002:0000db40       ??_R2FindXlsMsg@@8         0000000140058b40     LoadXlsMsg.obj
 0002:0000db50       ??_R1A@?0A@EA@FindXlsMsg@@8 0000000140058b50     LoadXlsMsg.obj
 0002:0000db78       ??_R3FindXlsMsg@@8         0000000140058b78     LoadXlsMsg.obj
 0002:0000db90       ??_R4FindXlsMsg@@6B@       0000000140058b90     LoadXlsMsg.obj
 0002:0000dbb8       ??_R3?$basic_iostream@DU?$char_traits@D@std@@@std@@8 0000000140058bb8     safe_string_x64:safe_string.obj
 0002:0000dbd0       ??_R2?$basic_stringbuf@DU?$char_traits@D@std@@V?$allocator@D@2@@std@@8 0000000140058bd0     safe_string_x64:safe_string.obj
 0002:0000dbe8       ??_R1A@?0A@EA@?$basic_stringstream@DU?$char_traits@D@std@@V?$allocator@D@2@@std@@8 0000000140058be8     safe_string_x64:safe_string.obj
 0002:0000dc10       ??_R3?$basic_stringbuf@DU?$char_traits@D@std@@V?$allocator@D@2@@std@@8 0000000140058c10     safe_string_x64:safe_string.obj
 0002:0000dc28       ??_R2?$basic_ostream@DU?$char_traits@D@std@@@std@@8 0000000140058c28     safe_string_x64:safe_string.obj
 0002:0000dc50       ??_R1BA@?0A@EA@?$basic_ostream@DU?$char_traits@D@std@@@std@@8 0000000140058c50     safe_string_x64:safe_string.obj
 0002:0000dc78       ??_R1A@?0A@EA@?$basic_ostream@DU?$char_traits@D@std@@@std@@8 0000000140058c78     safe_string_x64:safe_string.obj
 0002:0000dca0       ??_R1A@?0A@EA@?$basic_stringbuf@DU?$char_traits@D@std@@V?$allocator@D@2@@std@@8 0000000140058ca0     safe_string_x64:safe_string.obj
 0002:0000dcd0       ??_R2?$basic_iostream@DU?$char_traits@D@std@@@std@@8 0000000140058cd0     safe_string_x64:safe_string.obj
 0002:0000dd20       ??_R2?$basic_stringstream@DU?$char_traits@D@std@@V?$allocator@D@2@@std@@8 0000000140058d20     safe_string_x64:safe_string.obj
 0002:0000dd78       ??_R4?$basic_stringbuf@DU?$char_traits@D@std@@V?$allocator@D@2@@std@@6B@ 0000000140058d78     safe_string_x64:safe_string.obj
 0002:0000dda0       ??_R4?$basic_stringstream@DU?$char_traits@D@std@@V?$allocator@D@2@@std@@6B@ 0000000140058da0     safe_string_x64:safe_string.obj
 0002:0000ddc8       ??_R3?$basic_ostream@DU?$char_traits@D@std@@@std@@8 0000000140058dc8     safe_string_x64:safe_string.obj
 0002:0000dde0       ??_R1A@?0A@EA@?$basic_iostream@DU?$char_traits@D@std@@@std@@8 0000000140058de0     safe_string_x64:safe_string.obj
 0002:0000de08       ??_R3?$basic_stringstream@DU?$char_traits@D@std@@V?$allocator@D@2@@std@@8 0000000140058e08     safe_string_x64:safe_string.obj
 0002:0000e200       __rtc_iaa                  0000000140059200     msvcrt:initsect.obj
 0002:0000e208       __rtc_izz                  0000000140059208     msvcrt:initsect.obj
 0002:0000e210       __rtc_taa                  0000000140059210     msvcrt:initsect.obj
 0002:0000e218       __rtc_tzz                  0000000140059218     msvcrt:initsect.obj
 0002:0000e220       _tls_start                 0000000140059220     msvcrt:tlssup.obj
 0002:0000e230       _Init_thread_epoch         0000000140059230     msvcrt:thread_safe_statics.obj
 0002:0000e234       _tls_end                   0000000140059234     msvcrt:tlssup.obj
 0002:00013110       _CT??_R0?AVexception@std@@@8??0exception@std@@QEAA@AEBV01@@Z24 000000014005e110     AppInfoDlg.obj
 0002:00013138       _CTA1?AVexception@std@@    000000014005e138     AppInfoDlg.obj
 0002:00013148       _TI1?AVexception@std@@     000000014005e148     AppInfoDlg.obj
 0002:00013168       __IMPORT_DESCRIPTOR_PSAPI  000000014005e168     Psapi:PSAPI.DLL
 0002:0001317c       __IMPORT_DESCRIPTOR_mfc140 000000014005e17c     mfc140:mfc140.dll
 0002:00013190       __IMPORT_DESCRIPTOR_KERNEL32 000000014005e190     kernel32:KERNEL32.dll
 0002:000131a4       __IMPORT_DESCRIPTOR_USER32 000000014005e1a4     user32:USER32.dll
 0002:000131b8       __IMPORT_DESCRIPTOR_ADVAPI32 000000014005e1b8     advapi32:ADVAPI32.dll
 0002:000131cc       __IMPORT_DESCRIPTOR_SHELL32 000000014005e1cc     shell32:SHELL32.dll
 0002:000131e0       __IMPORT_DESCRIPTOR_SHLWAPI 000000014005e1e0     shlwapi:SHLWAPI.dll
 0002:000131f4       __IMPORT_DESCRIPTOR_MSVCP140 000000014005e1f4     msvcprt:MSVCP140.dll
 0002:00013208       __IMPORT_DESCRIPTOR_dbghelp 000000014005e208     DbgHelp:dbghelp.dll
 0002:0001321c       __IMPORT_DESCRIPTOR_WINMM  000000014005e21c     winmm:WINMM.dll
 0002:00013230       __IMPORT_DESCRIPTOR_WINHTTP 000000014005e230     winhttp:WINHTTP.dll
 0002:00013244       __IMPORT_DESCRIPTOR_WS2_32 000000014005e244     ws2_32:WS2_32.dll
 0002:00013258       __IMPORT_DESCRIPTOR_IPHLPAPI 000000014005e258     ipHlpapi:IPHLPAPI.DLL
 0002:0001326c       __IMPORT_DESCRIPTOR_VCRUNTIME140 000000014005e26c     vcruntime:VCRUNTIME140.dll
 0002:00013280       __IMPORT_DESCRIPTOR_api-ms-win-crt-runtime-l1-1-0 000000014005e280     ucrt:api-ms-win-crt-runtime-l1-1-0.dll
 0002:00013294       __IMPORT_DESCRIPTOR_api-ms-win-crt-stdio-l1-1-0 000000014005e294     ucrt:api-ms-win-crt-stdio-l1-1-0.dll
 0002:000132a8       __IMPORT_DESCRIPTOR_api-ms-win-crt-filesystem-l1-1-0 000000014005e2a8     ucrt:api-ms-win-crt-filesystem-l1-1-0.dll
 0002:000132bc       __IMPORT_DESCRIPTOR_api-ms-win-crt-string-l1-1-0 000000014005e2bc     ucrt:api-ms-win-crt-string-l1-1-0.dll
 0002:000132d0       __IMPORT_DESCRIPTOR_api-ms-win-crt-convert-l1-1-0 000000014005e2d0     ucrt:api-ms-win-crt-convert-l1-1-0.dll
 0002:000132e4       __IMPORT_DESCRIPTOR_api-ms-win-crt-time-l1-1-0 000000014005e2e4     ucrt:api-ms-win-crt-time-l1-1-0.dll
 0002:000132f8       __IMPORT_DESCRIPTOR_api-ms-win-crt-heap-l1-1-0 000000014005e2f8     ucrt:api-ms-win-crt-heap-l1-1-0.dll
 0002:0001330c       __IMPORT_DESCRIPTOR_api-ms-win-crt-multibyte-l1-1-0 000000014005e30c     ucrt:api-ms-win-crt-multibyte-l1-1-0.dll
 0002:00013320       __IMPORT_DESCRIPTOR_api-ms-win-crt-math-l1-1-0 000000014005e320     ucrt:api-ms-win-crt-math-l1-1-0.dll
 0002:00013334       __IMPORT_DESCRIPTOR_api-ms-win-crt-locale-l1-1-0 000000014005e334     ucrt:api-ms-win-crt-locale-l1-1-0.dll
 0002:00013348       __NULL_IMPORT_DESCRIPTOR   000000014005e348     Psapi:PSAPI.DLL
 0003:00000000       _Init_global_epoch         0000000140061000     msvcrt:thread_safe_statics.obj
 0003:00000004       __scrt_native_dllmain_reason 0000000140061004     msvcrt:utility.obj
 0003:00000008       __security_cookie_complement 0000000140061008     msvcrt:gs_cookie.obj
 0003:00000010       __security_cookie          0000000140061010     msvcrt:gs_cookie.obj
 0003:00000018       __isa_available            0000000140061018     msvcrt:cpu_disp.obj
 0003:0000001c       __isa_enabled              000000014006101c     msvcrt:cpu_disp.obj
 0003:00000020       __memcpy_nt_iters          0000000140061020     msvcrt:cpu_disp.obj
 0003:00000028       __scrt_default_matherr     0000000140061028     msvcrt:matherr.obj
 0003:00000030       __scrt_ucrt_dll_is_in_use  0000000140061030     msvcrt:ucrt_stubs.obj
 0003:00000040       ?command_list@@3PAUtagCommand_Entry@@A 0000000140061040     CSmtp.obj
 0003:00000180       ?m_LogLevel@CHLogger@@0IA  0000000140061180     HostLogger.obj
 0003:00000184       ?m_eSharedMemUsage@CLogMsgManager@@0W4ESHARED_MEM_USAGE_TYPE@1@A 0000000140061184     LogMsgManager.obj
 0003:00000190       ?g_cServerLog@@3VCServerLog@@A 0000000140061190     GameServerManagerDlg.obj
 0003:00000500       ?g_HostStat@@3VCHostStat@@A 0000000140061500     HostStat.obj
 0003:00001478       ?m_strFileFormat@CHLogger@@0V?$basic_string@DU?$char_traits@D@std@@V?$allocator@D@2@@std@@A 0000000140062478     HostLogger.obj
 0003:00001498       ?m_strBRFileFormat@CHLogger@@0V?$basic_string@DU?$char_traits@D@std@@V?$allocator@D@2@@std@@A 0000000140062498     HostLogger.obj
 0003:000014b8       ?m_strKernelFileFormat@CHLogger@@0V?$basic_string@DU?$char_traits@D@std@@V?$allocator@D@2@@std@@A 00000001400624b8     HostLogger.obj
 0003:000014d8       ?m_strEtcFileFormat@CHLogger@@0V?$basic_string@DU?$char_traits@D@std@@V?$allocator@D@2@@std@@A 00000001400624d8     HostLogger.obj
 0003:000014f8       ?m_strRWProcessMemoryFileFormat@CHLogger@@0V?$basic_string@DU?$char_traits@D@std@@V?$allocator@D@2@@std@@A 00000001400624f8     HostLogger.obj
 0003:00001518       ?m_strIPCMessageFileFormat@CHLogger@@0V?$basic_string@DU?$char_traits@D@std@@V?$allocator@D@2@@std@@A 0000000140062518     HostLogger.obj
 0003:00001538       ?m_strTimeOutFileFormat@CHLogger@@0V?$basic_string@DU?$char_traits@D@std@@V?$allocator@D@2@@std@@A 0000000140062538     HostLogger.obj
 0003:00001558       ?m_strPacketFileFormat@CHLogger@@0V?$basic_string@DU?$char_traits@D@std@@V?$allocator@D@2@@std@@A 0000000140062558     HostLogger.obj
 0003:00001578       ?m_strHostName@CHLogger@@0V?$basic_string@DU?$char_traits@D@std@@V?$allocator@D@2@@std@@A 0000000140062578     HostLogger.obj
 0003:00001598       ?m_strServerName@CHLogger@@0V?$basic_string@DU?$char_traits@D@std@@V?$allocator@D@2@@std@@A 0000000140062598     HostLogger.obj
 0003:000015b8       ?m_strLogFolder@CHLogger@@0V?$basic_string@DU?$char_traits@D@std@@V?$allocator@D@2@@std@@A 00000001400625b8     HostLogger.obj
 0003:000015d8       ?m_strModeUserCountFormat@CHLogger@@0V?$basic_string@DU?$char_traits@D@std@@V?$allocator@D@2@@std@@A 00000001400625d8     HostLogger.obj
 0003:000015f8       ?m_strServerAppUseCountFormat@CHLogger@@0V?$basic_string@DU?$char_traits@D@std@@V?$allocator@D@2@@std@@A 00000001400625f8     HostLogger.obj
 0003:00001618       ?m_LogLock@CHLogger@@0VCMustSyncObjectLog@@A 0000000140062618     HostLogger.obj
 0003:00001648       ?m_LogPacketLock@CHLogger@@0VCMustSyncObjectLog@@A 0000000140062648     HostLogger.obj
 0003:000016c0       _fltused                   00000001400626c0     msvcrt:fltused.obj
 0003:000016d0       ??_R0?AVtype_info@@@8      00000001400626d0     msvcrt:std_type_info_static.obj
 0003:000016f0       ??_R0?AVCServerLog@@@8     00000001400626f0     LogMgmt.obj
 0003:00001718       ??_R0?AVCReceiver@@@8      0000000140062718     SGGMCallBackObj.obj
 0003:00001738       ??_R0?AVCSGGMCallBackObj@@@8 0000000140062738     SGGMCallBackObj.obj
 0003:00001760       ??_R0?AVMultiReceiver@sggm_proxy@@@8 0000000140062760     SGGMCallBackObj.obj
 0003:00001790       ??_R0?AVEventReceiver@sggm@@@8 0000000140062790     SGGMCallBackObj.obj
 0003:000017c0       ??_R0?AVCClientLib@@@8     00000001400627c0     ClientLib.obj
 0003:000017e8       ??_R0?AV?$CircuitQueue@E@@@8 00000001400627e8     ClientLib.obj
 0003:00001810       ??_R0?AVSendBuffer@@@8     0000000140062810     ClientLib.obj
 0003:00001838       ??_R0?AVCPacket@@@8        0000000140062838     Packet.obj
 0003:00001858       ??_R0?AVCSFGameServerClientLib@@@8 0000000140062858     SFGameServerClientLib.obj
 0003:00001888       ??_R0?AVCDialog@@@8        0000000140062888     AppInfoDlg.obj
 0003:000018a8       ??_R0?AUGAMEPROTO_SC_HOST_STAT@@@8 00000001400628a8     AppInfoDlg.obj
 0003:000018d8       ??_R0?AUGAMEPROTO_SC_HOST_USER_STAT@@@8 00000001400628d8     AppInfoDlg.obj
 0003:00001910       ??_R0?AUGAMEPROTO_SC_REMOVECLIENT@@@8 0000000140062910     AppInfoDlg.obj
 0003:00001940       ??_R0?AUGAMEPROTO_CS_COMMON@@@8 0000000140062940     AppInfoDlg.obj
 0003:00001970       ??_R0?AUGAMEPROTO_SS_GAMEEND@@@8 0000000140062970     AppInfoDlg.obj
 0003:000019a0       ??_R0?AVexception@std@@@8  00000001400629a0     AppInfoDlg.obj
 0003:000019c8       ??_R0?AUGAMEPROTO_SC_SPY_CHANGE@@@8 00000001400629c8     AppInfoDlg.obj
 0003:000019f8       ??_R0?AUGAMEPROTO_SC_COMMON@@@8 00000001400629f8     AppInfoDlg.obj
 0003:00001a28       ??_R0?AUGAMEPROTO_COMMON@@@8 0000000140062a28     AppInfoDlg.obj
 0003:00001a50       ??_R0?AVCEdit@@@8          0000000140062a50     AppInfoDlg.obj
 0003:00001a70       ??_R0?AVCWnd@@@8           0000000140062a70     AppInfoDlg.obj
 0003:00001a90       ??_R0?AVCCmdTarget@@@8     0000000140062a90     AppInfoDlg.obj
 0003:00001ab8       ??_R0?AVCObject@@@8        0000000140062ab8     AppInfoDlg.obj
 0003:00001ad8       ??_R0?AVCWinApp@@@8        0000000140062ad8     GameServerManager.obj
 0003:00001af8       ??_R0?AVCWinThread@@@8     0000000140062af8     GameServerManager.obj
 0003:00001b20       ??_R0?AVCGameServerManagerApp@@@8 0000000140062b20     GameServerManager.obj
 0003:00001b50       ??_R0?AV_Ref_count_base@std@@@8 0000000140062b50     GameServerManagerDlg.obj
 0003:00001b80       ??_R0?AV?$_Ref_count@UGAMESERVERINFO@@@std@@@8 0000000140062b80     GameServerManagerDlg.obj
 0003:00001bc0       ??_R0?AVCGameServerManagerDlg@@@8 0000000140062bc0     GameServerManagerDlg.obj
 0003:00001bf0       ??_R0?AUIClientHandler@@@8 0000000140062bf0     GameServerManagerDlg.obj
 0003:00001c18       ??_R0?AVCHostStat@@@8      0000000140062c18     HostStat.obj
 0003:00001c40       ??_R0?AV?$basic_istream@DU?$char_traits@D@std@@@std@@@8 0000000140062c40     mailer.obj
 0003:00001c88       ??_R0?AVios_base@std@@@8   0000000140062c88     mailer.obj
 0003:00001cb0       ??_R0?AV?$_Iosb@H@std@@@8  0000000140062cb0     mailer.obj
 0003:00001cd8       ??_R0?AV?$basic_ios@DU?$char_traits@D@std@@@std@@@8 0000000140062cd8     mailer.obj
 0003:00001d20       ??_R0?AV?$basic_streambuf@DU?$char_traits@D@std@@@std@@@8 0000000140062d20     mailer.obj
 0003:00001d68       ??_R0?AVCMustSyncObjectLog@@@8 0000000140062d68     HostLogger.obj
 0003:00001d98       ??_R0?AU_RTL_CRITICAL_SECTION@@@8 0000000140062d98     HostLogger.obj
 0003:00001dc8       ??_R0?AVFindXlsMsg@@@8     0000000140062dc8     LoadXlsMsg.obj
 0003:00001df0       ??_R0?AV?$basic_stringstream@DU?$char_traits@D@std@@V?$allocator@D@2@@std@@@8 0000000140062df0     safe_string_x64:safe_string.obj
 0003:00001e50       ??_R0?AV?$basic_stringbuf@DU?$char_traits@D@std@@V?$allocator@D@2@@std@@@8 0000000140062e50     safe_string_x64:safe_string.obj
 0003:00001eb0       ??_R0?AV?$basic_iostream@DU?$char_traits@D@std@@@std@@@8 0000000140062eb0     safe_string_x64:safe_string.obj
 0003:00001f00       ??_R0?AV?$basic_ostream@DU?$char_traits@D@std@@@std@@@8 0000000140062f00     safe_string_x64:safe_string.obj
 0003:00001f50       __afxForceEXCLUDE          0000000140062f50     mfcs140:nolib.obj
 0003:00001f54       __afxForceSTDAFX           0000000140062f54     mfcs140:stdafx.obj
 0003:00001fa0       __scrt_current_native_startup_state 0000000140062fa0     msvcrt:utility.obj
 0003:00001fa8       __scrt_native_startup_lock 0000000140062fa8     msvcrt:utility.obj
 0003:00002560       __scrt_debugger_hook_flag  0000000140063560     msvcrt:utility_desktop.obj
 0003:00002564       _tls_index                 0000000140063564     msvcrt:tlssup.obj
 0003:00002568       __favor                    0000000140063568     msvcrt:cpu_disp.obj
 0003:00002570       ?__type_info_root_node@@3U__type_info_node@@A 0000000140063570     msvcrt:tncleanup.obj
 0003:00002580       ?_AtlBaseModule@ATL@@3VCAtlBaseModule@1@A 0000000140063580     atls:atlbase.obj
 0003:000025e0       __@@_PchSym_@00@UztvmgUPdlipUCUhUrmgvinvwrzgvUexgllohUzgohOmzgrevkilqPBACIAJCBDBUlyqiUznwGEUhgwzucOlyq@4B2008FD98C1DD4 00000001400635e0     atls:stdafx.obj
 0003:000025f8       ?_afxInitAppState@@3DA     00000001400635f8     mfcs140:appmodul.obj
 0003:00002600       ?_OptionsStorage@?1??__local_stdio_printf_options@@9@4_KA 0000000140063600     BugReporter.obj
 0003:00002610       ?m_szLogMailerFileName@CServerLog@@1PADA 0000000140063610     LogMgmt.obj
 0003:000029f9       ?m_isWriteLog_IPCMemory@CHLogger@@0_NA 00000001400639f9     HostLogger.obj
 0003:000029fa       ?m_isWriteLog_IPCMsg@CHLogger@@0_NA 00000001400639fa     HostLogger.obj
 0003:00002a00       ?m_szLogTryWeaponItemFileName@CServerLog@@1PADA 0000000140063a00     LogMgmt.obj
 0003:00002df0       ?m_szLogMgrDataFileName@CServerLog@@1PADA 0000000140063df0     LogMgmt.obj
 0003:000031e0       ?m_szLogKickUserFileName@CServerLog@@1PADA 00000001400641e0     LogMgmt.obj
 0003:000035d0       ?m_szLogServerSettingCheckFileName@CServerLog@@1PADA 00000001400645d0     LogMgmt.obj
 0003:000039c0       ?m_szLogCriticalErrorPath@CServerLog@@1PADA 00000001400649c0     LogMgmt.obj
 0003:00003db0       ?m_szLogInGameClanFileName@CServerLog@@1PADA 0000000140064db0     LogMgmt.obj
 0003:000041a0       ?m_szLogHackingFileName@CServerLog@@1PADA 00000001400651a0     LogMgmt.obj
 0003:00004590       ?m_szLogEmergencyStateFileName@CServerLog@@1PADA 0000000140065590     LogMgmt.obj
 0003:00004980       ?m_szLogMonitoringFileName@CServerLog@@1PADA 0000000140065980     LogMgmt.obj
 0003:00004d70       ?m_szLogMegaPhoneFileName@CServerLog@@1PADA 0000000140065d70     LogMgmt.obj
 0003:00005160       ?m_szLogCountFileName@CServerLog@@1PADA 0000000140066160     LogMgmt.obj
 0003:00005550       ?m_szLogHackFileName@CServerLog@@1PADA 0000000140066550     LogMgmt.obj
 0003:00005940       ?m_szLogTimeOutFileName@CServerLog@@1PADA 0000000140066940     LogMgmt.obj
 0003:00005d30       ?m_szLogTimeFileName@CServerLog@@1PADA 0000000140066d30     LogMgmt.obj
 0003:00006120       ?m_szLogEtcFileName@CServerLog@@1PADA 0000000140067120     LogMgmt.obj
 0003:00006510       ?m_szLogConnectCheckFileName@CServerLog@@1PADA 0000000140067510     LogMgmt.obj
 0003:00006900       ?m_szLogGachaFileName@CServerLog@@1PADA 0000000140067900     LogMgmt.obj
 0003:00006cf0       ?m_szLogUnknownDataFileName@CServerLog@@1PADA 0000000140067cf0     LogMgmt.obj
 0003:000070e0       ?m_szLogCashFileName@CServerLog@@1PADA 00000001400680e0     LogMgmt.obj
 0003:000074d0       ?m_szLogErrorFileName@CServerLog@@1PADA 00000001400684d0     LogMgmt.obj
 0003:000078c0       ?m_szLogFolder@CServerLog@@1PADA 00000001400688c0     LogMgmt.obj
 0003:00007a54       ?m_iLogLevel@CServerLog@@1HA 0000000140068a54     LogMgmt.obj
 0003:00007a58       ?pWnd@@3PEAVCWnd@@EA       0000000140068a58     GameServerManager.obj
 0003:00007a60       ?m_szServerName@CServerLog@@1PADA 0000000140068a60     LogMgmt.obj
 0003:00007ac8       ?g_NowState@@3KA           0000000140068ac8     GameServerManager.obj
 0003:00007ad0       ?m_szHostName@CServerLog@@1PADA 0000000140068ad0     LogMgmt.obj
 0003:00007b38       ?g_hSrv@@3PEAUSERVICE_STATUS_HANDLE__@@EA 0000000140068b38     GameServerManager.obj
 0003:00007b40       ?m_key@Seed@@0PAKA         0000000140068b40     Seed.obj
 0003:00007bc0       ?g_dwPrevGSMOnTimerTime@@3KA 0000000140068bc0     GameServerManagerDlg.obj
 0003:00007bc4       ?g_dwCurrGSMOnTimerTime@@3KA 0000000140068bc4     GameServerManagerDlg.obj
 0003:00007bc8       ?m_eLastError@CLogMsgManager@@0W4EERROR_TYPE@1@A 0000000140068bc8     LogMsgManager.obj
 0003:00007bd0       ?m_hSizeHandle@CLogMsgManager@@0PEAXEA 0000000140068bd0     LogMsgManager.obj
 0003:00007bd8       ?m_pXlsLoader@CLogMsgManager@@0PEAVFindXlsMsg@@EA 0000000140068bd8     LogMsgManager.obj
 0003:00007be0       ?handler@vars@cf@@2P6AXAEBV?$basic_string@DU?$char_traits@D@std@@V?$allocator@D@2@@std@@0@ZEA 0000000140068be0     safe_string_x64:safe_string.obj
 0003:00007be8       ?m_vectSharedMapHandles@CLogMsgManager@@0V?$vector@PEAXV?$allocator@PEAX@std@@@std@@A 0000000140068be8     LogMsgManager.obj
 0003:00007c00       ?theApp@@3VCGameServerManagerApp@@A 0000000140068c00     GameServerManager.obj
 0003:00008078       __iob_func                 0000000140069078     StdAfx.obj
 0003:00011098       ?_OptionsStorage@?1??__local_stdio_scanf_options@@9@4_KA 0000000140072098     GameServerManagerDlg.obj
 0003:000110ac       __@@_PchSym_@00@UdlipUhzPeCBAIUxorvmgUlyqUcGEUurmzoUtznvhvievinzmztviUhgwzucOlyq@4B2008FD98C1DD4 00000001400720ac     StdAfx.obj
 0003:000110b0       ?m_bInitFailed@CAtlBaseModule@ATL@@2_NA 00000001400720b0     StdAfx.obj
 0003:00011410       __dyn_tls_dtor_callback    0000000140072410     <common>
 0003:00011418       __dyn_tls_init_callback    0000000140072418     <common>

 entry point at        0001:00046a80

 Static symbols

 0000:fff88000       .debug$S                   0000000140000000     Psapi:PSAPI.DLL
 0000:fff88000       .debug$S                   0000000140000000     Psapi:PSAPI.DLL
 0000:fff88000       .debug$S                   0000000140000000     Psapi:PSAPI.DLL
 0000:fff88000       .debug$S                   0000000140000000     Psapi:PSAPI.DLL
 0000:fff88000       .debug$S                   0000000140000000     Psapi:PSAPI.DLL
 0000:fff88000       .debug$S                   0000000140000000     Psapi:PSAPI.DLL
 0000:fff88000       .debug$S                   0000000140000000     msvcprt:MSVCP140.dll
 0000:fff88000       .debug$S                   0000000140000000     ucrt:api-ms-win-crt-string-l1-1-0.dll
 0000:fff88000       .debug$S                   0000000140000000     ucrt:api-ms-win-crt-math-l1-1-0.dll
 0000:fff88000       .debug$S                   0000000140000000     ucrt:api-ms-win-crt-math-l1-1-0.dll
 0000:fff88000       .debug$S                   0000000140000000     vcruntime:VCRUNTIME140.dll
 0000:fff88000       .debug$S                   0000000140000000     vcruntime:VCRUNTIME140.dll
 0000:fff88000       .debug$S                   0000000140000000     vcruntime:VCRUNTIME140.dll
 0000:fff88000       .debug$S                   0000000140000000     vcruntime:VCRUNTIME140.dll
 0000:fff88000       .debug$S                   0000000140000000     msvcprt:MSVCP140.dll
 0000:fff88000       .debug$S                   0000000140000000     msvcprt:MSVCP140.dll
 0000:fff88000       .debug$S                   0000000140000000     libssl64MD:libssl-1_1-x64.dll
 0000:fff88000       .debug$S                   0000000140000000     msvcprt:MSVCP140.dll
 0000:fff88000       .debug$S                   0000000140000000     msvcprt:MSVCP140.dll
 0000:fff88000       .debug$S                   0000000140000000     msvcprt:MSVCP140.dll
 0000:fff88000       .debug$S                   0000000140000000     msvcprt:MSVCP140.dll
 0000:fff88000       .debug$S                   0000000140000000     msvcprt:MSVCP140.dll
 0000:fff88000       .debug$S                   0000000140000000     msvcprt:MSVCP140.dll
 0000:fff88000       .debug$S                   0000000140000000     msvcprt:MSVCP140.dll
 0000:fff88000       .debug$S                   0000000140000000     msvcprt:MSVCP140.dll
 0000:fff88000       .debug$S                   0000000140000000     msvcprt:MSVCP140.dll
 0000:fff88000       .debug$S                   0000000140000000     msvcprt:MSVCP140.dll
 0000:fff88000       .debug$S                   0000000140000000     msvcprt:MSVCP140.dll
 0000:fff88000       .debug$S                   0000000140000000     msvcprt:MSVCP140.dll
 0000:fff88000       .debug$S                   0000000140000000     msvcprt:MSVCP140.dll
 0000:fff88000       .debug$S                   0000000140000000     msvcprt:MSVCP140.dll
 0000:fff88000       .debug$S                   0000000140000000     msvcprt:MSVCP140.dll
 0000:fff88000       .debug$S                   0000000140000000     msvcprt:MSVCP140.dll
 0000:fff88000       .debug$S                   0000000140000000     msvcprt:MSVCP140.dll
 0000:fff88000       .debug$S                   0000000140000000     msvcprt:MSVCP140.dll
 0000:fff88000       .debug$S                   0000000140000000     msvcprt:MSVCP140.dll
 0000:fff88000       .debug$S                   0000000140000000     msvcprt:MSVCP140.dll
 0000:fff88000       .debug$S                   0000000140000000     msvcprt:MSVCP140.dll
 0000:fff88000       .debug$S                   0000000140000000     msvcprt:MSVCP140.dll
 0000:fff88000       .debug$S                   0000000140000000     msvcprt:MSVCP140.dll
 0000:fff88000       .debug$S                   0000000140000000     msvcprt:MSVCP140.dll
 0000:fff88000       .debug$S                   0000000140000000     msvcprt:MSVCP140.dll
 0000:fff88000       .debug$S                   0000000140000000     Wininet:WININET.dll
 0000:fff88000       .debug$S                   0000000140000000     Wininet:WININET.dll
 0000:fff88000       .debug$S                   0000000140000000     Wininet:WININET.dll
 0000:fff88000       .debug$S                   0000000140000000     Wininet:WININET.dll
 0000:fff88000       .debug$S                   0000000140000000     Wininet:WININET.dll
 0002:fffb5000       .idata$6                   0000000140000000     Wininet:WININET.dll
 0000:fff88000       .debug$S                   0000000140000000     DbgHelp:dbghelp.dll
 0000:fff88000       .debug$S                   0000000140000000     DbgHelp:dbghelp.dll
 0000:fff88000       .debug$S                   0000000140000000     DbgHelp:dbghelp.dll
 0000:fff88000       .debug$S                   0000000140000000     libssl64MD:libssl-1_1-x64.dll
 0000:fff88000       .debug$S                   0000000140000000     DbgHelp:dbghelp.dll
 0000:fff88000       .debug$S                   0000000140000000     DbgHelp:dbghelp.dll
 0000:fff88000       .debug$S                   0000000140000000     DbgHelp:dbghelp.dll
 0000:fff88000       .debug$S                   0000000140000000     DbgHelp:dbghelp.dll
 0000:fff88000       .debug$S                   0000000140000000     libssl64MD:libssl-1_1-x64.dll
 0000:fff88000       .debug$S                   0000000140000000     DbgHelp:dbghelp.dll
 0000:fff88000       .debug$S                   0000000140000000     libssl64MD:libssl-1_1-x64.dll
 0000:fff88000       .debug$S                   0000000140000000     winmm:WINMM.dll
 0000:fff88000       .debug$S                   0000000140000000     winhttp:WINHTTP.dll
 0000:fff88000       .debug$S                   0000000140000000     winhttp:WINHTTP.dll
 0000:fff88000       .debug$S                   0000000140000000     winhttp:WINHTTP.dll
 0000:fff88000       .debug$S                   0000000140000000     libssl64MD:libssl-1_1-x64.dll
 0000:fff88000       .debug$S                   0000000140000000     winhttp:WINHTTP.dll
 0000:fff88000       .debug$S                   0000000140000000     libssl64MD:libssl-1_1-x64.dll
 0000:fff88000       .debug$S                   0000000140000000     winhttp:WINHTTP.dll
 0000:fff88000       .debug$S                   0000000140000000     winhttp:WINHTTP.dll
 0000:fff88000       .debug$S                   0000000140000000     winhttp:WINHTTP.dll
 0000:fff88000       .debug$S                   0000000140000000     winhttp:WINHTTP.dll
 0000:fff88000       .debug$S                   0000000140000000     libssl64MD:libssl-1_1-x64.dll
 0000:fff88000       .debug$S                   0000000140000000     winhttp:WINHTTP.dll
 0000:fff88000       .debug$S                   0000000140000000     libssl64MD:libssl-1_1-x64.dll
 0000:fff88000       .debug$S                   0000000140000000     ws2_32:WS2_32.dll
 0000:fff88000       .debug$S                   0000000140000000     libssl64MD:libssl-1_1-x64.dll
 0000:fff88000       .debug$S                   0000000140000000     ws2_32:WS2_32.dll
 0000:fff88000       .debug$S                   0000000140000000     libssl64MD:libssl-1_1-x64.dll
 0000:fff88000       .debug$S                   0000000140000000     ws2_32:WS2_32.dll
 0000:fff88000       .debug$S                   0000000140000000     ws2_32:WS2_32.dll
 0000:fff88000       .debug$S                   0000000140000000     ws2_32:WS2_32.dll
 0000:fff88000       .debug$S                   0000000140000000     ws2_32:WS2_32.dll
 0000:fff88000       .debug$S                   0000000140000000     libssl64MD:libssl-1_1-x64.dll
 0000:fff88000       .debug$S                   0000000140000000     ws2_32:WS2_32.dll
 0000:fff88000       .debug$S                   0000000140000000     libssl64MD:libssl-1_1-x64.dll
 0000:fff88000       .debug$S                   0000000140000000     ws2_32:WS2_32.dll
 0000:fff88000       .debug$S                   0000000140000000     libssl64MD:libssl-1_1-x64.dll
 0000:fff88000       .debug$S                   0000000140000000     ws2_32:WS2_32.dll
 0000:fff88000       .debug$S                   0000000140000000     libssl64MD:libssl-1_1-x64.dll
 0000:fff88000       .debug$S                   0000000140000000     ws2_32:WS2_32.dll
 0002:fffb5000       .idata$6                   0000000140000000     libssl64MD:libssl-1_1-x64.dll
 0000:fff88000       .debug$S                   0000000140000000     ws2_32:WS2_32.dll
 0000:fff88000       .debug$S                   0000000140000000     mfc140:mfc140.dll
 0000:fff88000       .debug$S                   0000000140000000     ws2_32:WS2_32.dll
 0000:fff88000       .debug$S                   0000000140000000     mfc140:mfc140.dll
 0000:fff88000       .debug$S                   0000000140000000     ws2_32:WS2_32.dll
 0000:fff88000       .debug$S                   0000000140000000     ws2_32:WS2_32.dll
 0000:fff88000       .debug$S                   0000000140000000     ws2_32:WS2_32.dll
 0000:fff88000       .debug$S                   0000000140000000     ws2_32:WS2_32.dll
 0000:fff88000       .debug$S                   0000000140000000     ws2_32:WS2_32.dll
 0000:fff88000       .debug$S                   0000000140000000     ws2_32:WS2_32.dll
 0000:fff88000       .debug$S                   0000000140000000     ws2_32:WS2_32.dll
 0000:fff88000       .debug$S                   0000000140000000     ws2_32:WS2_32.dll
 0000:fff88000       .debug$S                   0000000140000000     ws2_32:WS2_32.dll
 0000:fff88000       .debug$S                   0000000140000000     ws2_32:WS2_32.dll
 0000:fff88000       .debug$S                   0000000140000000     ws2_32:WS2_32.dll
 0000:fff88000       .debug$S                   0000000140000000     ws2_32:WS2_32.dll
 0000:fff88000       .debug$S                   0000000140000000     ws2_32:WS2_32.dll
 0000:fff88000       .debug$S                   0000000140000000     ws2_32:WS2_32.dll
 0000:fff88000       .debug$S                   0000000140000000     ws2_32:WS2_32.dll
 0000:fff88000       .debug$S                   0000000140000000     ws2_32:WS2_32.dll
 0000:fff88000       .debug$S                   0000000140000000     mfc140:mfc140.dll
 0000:fff88000       .debug$S                   0000000140000000     ws2_32:WS2_32.dll
 0000:fff88000       .debug$S                   0000000140000000     mfc140:mfc140.dll
 0000:fff88000       .debug$S                   0000000140000000     ws2_32:WS2_32.dll
 0000:fff88000       .debug$S                   0000000140000000     mfc140:mfc140.dll
 0000:fff88000       .debug$S                   0000000140000000     ws2_32:WS2_32.dll
 0000:fff88000       .debug$S                   0000000140000000     Snmpapi:snmpapi.dll
 0000:fff88000       .debug$S                   0000000140000000     Snmpapi:snmpapi.dll
 0000:fff88000       .debug$S                   0000000140000000     Snmpapi:snmpapi.dll
 0000:fff88000       .debug$S                   0000000140000000     Snmpapi:snmpapi.dll
 0002:fffb5000       .idata$6                   0000000140000000     Snmpapi:snmpapi.dll
 0000:fff88000       .debug$S                   0000000140000000     mfc140:mfc140.dll
 0000:fff88000       .debug$S                   0000000140000000     ipHlpapi:IPHLPAPI.DLL
 0000:fff88000       .debug$S                   0000000140000000     mfc140:mfc140.dll
 0000:fff88000       .debug$S                   0000000140000000     vcruntime:VCRUNTIME140.dll
 0000:fff88000       .debug$S                   0000000140000000     vcruntime:VCRUNTIME140.dll
 0000:fff88000       .debug$S                   0000000140000000     vcruntime:VCRUNTIME140.dll
 0000:fff88000       .debug$S                   0000000140000000     vcruntime:VCRUNTIME140.dll
 0000:fff88000       .debug$S                   0000000140000000     mfc140:mfc140.dll
 0000:fff88000       .debug$S                   0000000140000000     vcruntime:VCRUNTIME140.dll
 0000:fff88000       .debug$S                   0000000140000000     mfc140:mfc140.dll
 0000:fff88000       .debug$S                   0000000140000000     vcruntime:VCRUNTIME140.dll
 0000:fff88000       .debug$S                   0000000140000000     vcruntime:VCRUNTIME140.dll
 0000:fff88000       .debug$S                   0000000140000000     vcruntime:VCRUNTIME140.dll
 0000:fff88000       .debug$S                   0000000140000000     vcruntime:VCRUNTIME140.dll
 0000:fff88000       .debug$S                   0000000140000000     mfc140:mfc140.dll
 0000:fff88000       .debug$S                   0000000140000000     vcruntime:VCRUNTIME140.dll
 0000:fff88000       .debug$S                   0000000140000000     mfc140:mfc140.dll
 0000:fff88000       .debug$S                   0000000140000000     vcruntime:VCRUNTIME140.dll
 0000:fff88000       .debug$S                   0000000140000000     vcruntime:VCRUNTIME140.dll
 0000:fff88000       .debug$S                   0000000140000000     ucrt:api-ms-win-crt-runtime-l1-1-0.dll
 0000:fff88000       .debug$S                   0000000140000000     ucrt:api-ms-win-crt-runtime-l1-1-0.dll
 0000:fff88000       .debug$S                   0000000140000000     ucrt:api-ms-win-crt-runtime-l1-1-0.dll
 0000:fff88000       .debug$S                   0000000140000000     ucrt:api-ms-win-crt-stdio-l1-1-0.dll
 0000:fff88000       .debug$S                   0000000140000000     ucrt:api-ms-win-crt-filesystem-l1-1-0.dll
 0000:fff88000       .debug$S                   0000000140000000     ucrt:api-ms-win-crt-string-l1-1-0.dll
 0000:fff88000       .debug$S                   0000000140000000     ucrt:api-ms-win-crt-filesystem-l1-1-0.dll
 0000:fff88000       .debug$S                   0000000140000000     ucrt:api-ms-win-crt-runtime-l1-1-0.dll
 0000:fff88000       .debug$S                   0000000140000000     ucrt:api-ms-win-crt-string-l1-1-0.dll
 0000:fff88000       .debug$S                   0000000140000000     ucrt:api-ms-win-crt-stdio-l1-1-0.dll
 0000:fff88000       .debug$S                   0000000140000000     ucrt:api-ms-win-crt-convert-l1-1-0.dll
 0000:fff88000       .debug$S                   0000000140000000     ucrt:api-ms-win-crt-string-l1-1-0.dll
 0000:fff88000       .debug$S                   0000000140000000     ucrt:api-ms-win-crt-stdio-l1-1-0.dll
 0000:fff88000       .debug$S                   0000000140000000     ucrt:api-ms-win-crt-stdio-l1-1-0.dll
 0000:fff88000       .debug$S                   0000000140000000     ucrt:api-ms-win-crt-stdio-l1-1-0.dll
 0000:fff88000       .debug$S                   0000000140000000     ucrt:api-ms-win-crt-stdio-l1-1-0.dll
 0000:fff88000       .debug$S                   0000000140000000     ucrt:api-ms-win-crt-stdio-l1-1-0.dll
 0000:fff88000       .debug$S                   0000000140000000     ucrt:api-ms-win-crt-string-l1-1-0.dll
 0000:fff88000       .debug$S                   0000000140000000     ucrt:api-ms-win-crt-string-l1-1-0.dll
 0000:fff88000       .debug$S                   0000000140000000     ucrt:api-ms-win-crt-stdio-l1-1-0.dll
 0000:fff88000       .debug$S                   0000000140000000     ucrt:api-ms-win-crt-stdio-l1-1-0.dll
 0000:fff88000       .debug$S                   0000000140000000     ucrt:api-ms-win-crt-stdio-l1-1-0.dll
 0000:fff88000       .debug$S                   0000000140000000     ucrt:api-ms-win-crt-time-l1-1-0.dll
 0000:fff88000       .debug$S                   0000000140000000     ucrt:api-ms-win-crt-string-l1-1-0.dll
 0000:fff88000       .debug$S                   0000000140000000     ucrt:api-ms-win-crt-string-l1-1-0.dll
 0000:fff88000       .debug$S                   0000000140000000     ucrt:api-ms-win-crt-stdio-l1-1-0.dll
 0000:fff88000       .debug$S                   0000000140000000     ucrt:api-ms-win-crt-convert-l1-1-0.dll
 0000:fff88000       .debug$S                   0000000140000000     ucrt:api-ms-win-crt-stdio-l1-1-0.dll
 0000:fff88000       .debug$S                   0000000140000000     ucrt:api-ms-win-crt-runtime-l1-1-0.dll
 0000:fff88000       .debug$S                   0000000140000000     ucrt:api-ms-win-crt-time-l1-1-0.dll
 0000:fff88000       .debug$S                   0000000140000000     ucrt:api-ms-win-crt-convert-l1-1-0.dll
 0000:fff88000       .debug$S                   0000000140000000     ucrt:api-ms-win-crt-string-l1-1-0.dll
 0000:fff88000       .debug$S                   0000000140000000     ucrt:api-ms-win-crt-string-l1-1-0.dll
 0000:fff88000       .debug$S                   0000000140000000     ucrt:api-ms-win-crt-stdio-l1-1-0.dll
 0000:fff88000       .debug$S                   0000000140000000     ucrt:api-ms-win-crt-stdio-l1-1-0.dll
 0000:fff88000       .debug$S                   0000000140000000     ucrt:api-ms-win-crt-time-l1-1-0.dll
 0000:fff88000       .debug$S                   0000000140000000     ucrt:api-ms-win-crt-string-l1-1-0.dll
 0000:fff88000       .debug$S                   0000000140000000     ucrt:api-ms-win-crt-heap-l1-1-0.dll
 0000:fff88000       .debug$S                   0000000140000000     ucrt:api-ms-win-crt-heap-l1-1-0.dll
 0000:fff88000       .debug$S                   0000000140000000     ucrt:api-ms-win-crt-string-l1-1-0.dll
 0000:fff88000       .debug$S                   0000000140000000     ucrt:api-ms-win-crt-multibyte-l1-1-0.dll
 0000:fff88000       .debug$S                   0000000140000000     ucrt:api-ms-win-crt-heap-l1-1-0.dll
 0000:fff88000       .debug$S                   0000000140000000     ucrt:api-ms-win-crt-multibyte-l1-1-0.dll
 0000:fff88000       .debug$S                   0000000140000000     ucrt:api-ms-win-crt-multibyte-l1-1-0.dll
 0000:fff88000       .debug$S                   0000000140000000     ucrt:api-ms-win-crt-stdio-l1-1-0.dll
 0000:fff88000       .debug$S                   0000000140000000     ucrt:api-ms-win-crt-convert-l1-1-0.dll
 0000:fff88000       .debug$S                   0000000140000000     ucrt:api-ms-win-crt-convert-l1-1-0.dll
 0000:fff88000       .debug$S                   0000000140000000     ucrt:api-ms-win-crt-string-l1-1-0.dll
 0000:fff88000       .debug$S                   0000000140000000     ucrt:api-ms-win-crt-multibyte-l1-1-0.dll
 0000:fff88000       .debug$S                   0000000140000000     ucrt:api-ms-win-crt-multibyte-l1-1-0.dll
 0000:fff88000       .debug$S                   0000000140000000     ucrt:api-ms-win-crt-stdio-l1-1-0.dll
 0000:fff88000       .debug$S                   0000000140000000     ucrt:api-ms-win-crt-stdio-l1-1-0.dll
 0000:fff88000       .debug$S                   0000000140000000     ucrt:api-ms-win-crt-stdio-l1-1-0.dll
 0000:fff88000       .debug$S                   0000000140000000     ucrt:api-ms-win-crt-time-l1-1-0.dll
 0000:fff88000       .debug$S                   0000000140000000     ucrt:api-ms-win-crt-string-l1-1-0.dll
 0000:fff88000       .debug$S                   0000000140000000     ucrt:api-ms-win-crt-stdio-l1-1-0.dll
 0000:fff88000       .debug$S                   0000000140000000     ucrt:api-ms-win-crt-stdio-l1-1-0.dll
 0000:fff88000       .debug$S                   0000000140000000     ucrt:api-ms-win-crt-stdio-l1-1-0.dll
 0000:fff88000       .debug$S                   0000000140000000     ucrt:api-ms-win-crt-stdio-l1-1-0.dll
 0000:fff88000       .debug$S                   0000000140000000     ucrt:api-ms-win-crt-stdio-l1-1-0.dll
 0000:fff88000       .debug$S                   0000000140000000     ucrt:api-ms-win-crt-filesystem-l1-1-0.dll
 0000:fff88000       .debug$S                   0000000140000000     ucrt:api-ms-win-crt-filesystem-l1-1-0.dll
 0000:fff88000       .debug$S                   0000000140000000     ucrt:api-ms-win-crt-stdio-l1-1-0.dll
 0000:fff88000       .debug$S                   0000000140000000     ucrt:api-ms-win-crt-stdio-l1-1-0.dll
 0000:fff88000       .debug$S                   0000000140000000     ucrt:api-ms-win-crt-stdio-l1-1-0.dll
 0000:fff88000       .debug$S                   0000000140000000     ucrt:api-ms-win-crt-stdio-l1-1-0.dll
 0000:fff88000       .debug$S                   0000000140000000     ucrt:api-ms-win-crt-runtime-l1-1-0.dll
 0000:fff88000       .debug$S                   0000000140000000     ucrt:api-ms-win-crt-runtime-l1-1-0.dll
 0000:fff88000       .debug$S                   0000000140000000     ucrt:api-ms-win-crt-runtime-l1-1-0.dll
 0000:fff88000       .debug$S                   0000000140000000     ucrt:api-ms-win-crt-runtime-l1-1-0.dll
 0000:fff88000       .debug$S                   0000000140000000     ucrt:api-ms-win-crt-runtime-l1-1-0.dll
 0000:fff88000       .debug$S                   0000000140000000     ucrt:api-ms-win-crt-runtime-l1-1-0.dll
 0000:fff88000       .debug$S                   0000000140000000     ucrt:api-ms-win-crt-runtime-l1-1-0.dll
 0000:fff88000       .debug$S                   0000000140000000     ucrt:api-ms-win-crt-runtime-l1-1-0.dll
 0000:fff88000       .debug$S                   0000000140000000     ucrt:api-ms-win-crt-runtime-l1-1-0.dll
 0000:fff88000       .debug$S                   0000000140000000     ucrt:api-ms-win-crt-runtime-l1-1-0.dll
 0000:fff88000       .debug$S                   0000000140000000     ucrt:api-ms-win-crt-runtime-l1-1-0.dll
 0000:fff88000       .debug$S                   0000000140000000     ucrt:api-ms-win-crt-runtime-l1-1-0.dll
 0000:fff88000       .debug$S                   0000000140000000     ucrt:api-ms-win-crt-math-l1-1-0.dll
 0000:fff88000       .debug$S                   0000000140000000     ucrt:api-ms-win-crt-runtime-l1-1-0.dll
 0000:fff88000       .debug$S                   0000000140000000     ucrt:api-ms-win-crt-runtime-l1-1-0.dll
 0000:fff88000       .debug$S                   0000000140000000     ucrt:api-ms-win-crt-runtime-l1-1-0.dll
 0000:fff88000       .debug$S                   0000000140000000     ucrt:api-ms-win-crt-runtime-l1-1-0.dll
 0000:fff88000       .debug$S                   0000000140000000     ucrt:api-ms-win-crt-runtime-l1-1-0.dll
 0000:fff88000       .debug$S                   0000000140000000     ucrt:api-ms-win-crt-stdio-l1-1-0.dll
 0000:fff88000       .debug$S                   0000000140000000     ucrt:api-ms-win-crt-runtime-l1-1-0.dll
 0000:fff88000       .debug$S                   0000000140000000     ucrt:api-ms-win-crt-runtime-l1-1-0.dll
 0000:fff88000       .debug$S                   0000000140000000     ucrt:api-ms-win-crt-locale-l1-1-0.dll
 0000:fff88000       .debug$S                   0000000140000000     ucrt:api-ms-win-crt-heap-l1-1-0.dll
 0000:fff88000       .debug$S                   0000000140000000     mfc140:mfc140.dll
 0000:fff88000       .debug$S                   0000000140000000     ucrt:api-ms-win-crt-stdio-l1-1-0.dll
 0000:fff88000       .debug$S                   0000000140000000     mfc140:mfc140.dll
 0000:fff88000       .debug$S                   0000000140000000     ucrt:api-ms-win-crt-heap-l1-1-0.dll
 0000:fff88000       .debug$S                   0000000140000000     ucrt:api-ms-win-crt-string-l1-1-0.dll
 0000:fff88000       .debug$S                   0000000140000000     ucrt:api-ms-win-crt-string-l1-1-0.dll
 0000:fff88000       .debug$S                   0000000140000000     ucrt:api-ms-win-crt-convert-l1-1-0.dll
 0000:fff88000       .debug$S                   0000000140000000     mfc140:mfc140.dll
 0000:fff88000       .debug$S                   0000000140000000     msvcprt:MSVCP140.dll
 0000:fff88000       .debug$S                   0000000140000000     mfc140:mfc140.dll
 0000:fff88000       .debug$S                   0000000140000000     kernel32:KERNEL32.dll
 0000:fff88000       .debug$S                   0000000140000000     mfc140:mfc140.dll
 0000:fff88000       .debug$S                   0000000140000000     msvcprt:MSVCP140.dll
 0000:fff88000       .debug$S                   0000000140000000     mfc140:mfc140.dll
 0000:fff88000       .debug$S                   0000000140000000     msvcprt:MSVCP140.dll
 0000:fff88000       .debug$S                   0000000140000000     mfc140:mfc140.dll
 0000:fff88000       .debug$S                   0000000140000000     msvcprt:MSVCP140.dll
 0000:fff88000       .debug$S                   0000000140000000     mfc140:mfc140.dll
 0000:fff88000       .debug$S                   0000000140000000     msvcprt:MSVCP140.dll
 0000:fff88000       .debug$S                   0000000140000000     msvcprt:MSVCP140.dll
 0000:fff88000       .debug$S                   0000000140000000     msvcprt:MSVCP140.dll
 0000:fff88000       .debug$S                   0000000140000000     msvcprt:MSVCP140.dll
 0000:fff88000       .debug$S                   0000000140000000     mfc140:mfc140.dll
 0000:fff88000       .debug$S                   0000000140000000     msvcprt:MSVCP140.dll
 0000:fff88000       .debug$S                   0000000140000000     mfc140:mfc140.dll
 0000:fff88000       .debug$S                   0000000140000000     msvcprt:MSVCP140.dll
 0000:fff88000       .debug$S                   0000000140000000     mfc140:mfc140.dll
 0000:fff88000       .debug$S                   0000000140000000     msvcprt:MSVCP140.dll
 0000:fff88000       .debug$S                   0000000140000000     mfc140:mfc140.dll
 0000:fff88000       .debug$S                   0000000140000000     msvcprt:MSVCP140.dll
 0000:fff88000       .debug$S                   0000000140000000     mfc140:mfc140.dll
 0000:fff88000       .debug$S                   0000000140000000     ucrt:api-ms-win-crt-locale-l1-1-0.dll
 0000:fff88000       .debug$S                   0000000140000000     mfc140:mfc140.dll
 0000:fff88000       .debug$S                   0000000140000000     msvcprt:MSVCP140.dll
 0000:fff88000       .debug$S                   0000000140000000     msvcprt:MSVCP140.dll
 0000:fff88000       .debug$S                   0000000140000000     msvcprt:MSVCP140.dll
 0000:fff88000       .debug$S                   0000000140000000     msvcprt:MSVCP140.dll
 0000:fff88000       .debug$S                   0000000140000000     mfc140:mfc140.dll
 0000:fff88000       .debug$S                   0000000140000000     msvcprt:MSVCP140.dll
 0000:fff88000       .debug$S                   0000000140000000     mfc140:mfc140.dll
 0000:fff88000       .debug$S                   0000000140000000     msvcprt:MSVCP140.dll
 0000:fff88000       .debug$S                   0000000140000000     mfc140:mfc140.dll
 0000:fff88000       .debug$S                   0000000140000000     msvcprt:MSVCP140.dll
 0000:fff88000       .debug$S                   0000000140000000     mfc140:mfc140.dll
 0000:fff88000       .debug$S                   0000000140000000     msvcprt:MSVCP140.dll
 0000:fff88000       .debug$S                   0000000140000000     mfc140:mfc140.dll
 0000:fff88000       .debug$S                   0000000140000000     msvcprt:MSVCP140.dll
 0000:fff88000       .debug$S                   0000000140000000     msvcprt:MSVCP140.dll
 0000:fff88000       .debug$S                   0000000140000000     msvcprt:MSVCP140.dll
 0000:fff88000       .debug$S                   0000000140000000     msvcprt:MSVCP140.dll
 0000:fff88000       .debug$S                   0000000140000000     msvcprt:MSVCP140.dll
 0000:fff88000       .debug$S                   0000000140000000     msvcprt:MSVCP140.dll
 0000:fff88000       .debug$S                   0000000140000000     mfc140:mfc140.dll
 0000:fff88000       .debug$S                   0000000140000000     msvcprt:MSVCP140.dll
 0000:fff88000       .debug$S                   0000000140000000     msvcprt:MSVCP140.dll
 0000:fff88000       .debug$S                   0000000140000000     msvcprt:MSVCP140.dll
 0000:fff88000       .debug$S                   0000000140000000     msvcprt:MSVCP140.dll
 0000:fff88000       .debug$S                   0000000140000000     msvcprt:MSVCP140.dll
 0000:fff88000       .debug$S                   0000000140000000     msvcprt:MSVCP140.dll
 0000:fff88000       .debug$S                   0000000140000000     mfc140:mfc140.dll
 0000:fff88000       .debug$S                   0000000140000000     msvcprt:MSVCP140.dll
 0000:fff88000       .debug$S                   0000000140000000     mfc140:mfc140.dll
 0000:fff88000       .debug$S                   0000000140000000     msvcprt:MSVCP140.dll
 0000:fff88000       .debug$S                   0000000140000000     mfc140:mfc140.dll
 0000:fff88000       .debug$S                   0000000140000000     msvcprt:MSVCP140.dll
 0000:fff88000       .debug$S                   0000000140000000     mfc140:mfc140.dll
 0000:fff88000       .debug$S                   0000000140000000     msvcprt:MSVCP140.dll
 0000:fff88000       .debug$S                   0000000140000000     mfc140:mfc140.dll
 0000:fff88000       .debug$S                   0000000140000000     msvcprt:MSVCP140.dll
 0000:fff88000       .debug$S                   0000000140000000     mfc140:mfc140.dll
 0000:fff88000       .debug$S                   0000000140000000     msvcprt:MSVCP140.dll
 0000:fff88000       .debug$S                   0000000140000000     mfc140:mfc140.dll
 0000:fff88000       .debug$S                   0000000140000000     msvcprt:MSVCP140.dll
 0000:fff88000       .debug$S                   0000000140000000     msvcprt:MSVCP140.dll
 0000:fff88000       .debug$S                   0000000140000000     msvcprt:MSVCP140.dll
 0000:fff88000       .debug$S                   0000000140000000     msvcprt:MSVCP140.dll
 0000:fff88000       .debug$S                   0000000140000000     mfc140:mfc140.dll
 0000:fff88000       .debug$S                   0000000140000000     msvcprt:MSVCP140.dll
 0000:fff88000       .debug$S                   0000000140000000     mfc140:mfc140.dll
 0000:fff88000       .debug$S                   0000000140000000     msvcprt:MSVCP140.dll
 0000:fff88000       .debug$S                   0000000140000000     msvcprt:MSVCP140.dll
 0002:fffb5000       .idata$6                   0000000140000000     oleaut32:OLEAUT32.dll
 0000:fff88000       .debug$S                   0000000140000000     oleaut32:OLEAUT32.dll
 0000:fff88000       .debug$S                   0000000140000000     mfc140:mfc140.dll
 0000:fff88000       .debug$S                   0000000140000000     shlwapi:SHLWAPI.dll
 0000:fff88000       .debug$S                   0000000140000000     mfc140:mfc140.dll
 0000:fff88000       .debug$S                   0000000140000000     shell32:SHELL32.dll
 0000:fff88000       .debug$S                   0000000140000000     mfc140:mfc140.dll
 0000:fff88000       .debug$S                   0000000140000000     shell32:SHELL32.dll
 0000:fff88000       .debug$S                   0000000140000000     mfc140:mfc140.dll
 0000:fff88000       .debug$S                   0000000140000000     advapi32:ADVAPI32.dll
 0000:fff88000       .debug$S                   0000000140000000     mfc140:mfc140.dll
 0000:fff88000       .debug$S                   0000000140000000     advapi32:ADVAPI32.dll
 0000:fff88000       .debug$S                   0000000140000000     mfc140:mfc140.dll
 0000:fff88000       .debug$S                   0000000140000000     advapi32:ADVAPI32.dll
 0000:fff88000       .debug$S                   0000000140000000     advapi32:ADVAPI32.dll
 0000:fff88000       .debug$S                   0000000140000000     advapi32:ADVAPI32.dll
 0000:fff88000       .debug$S                   0000000140000000     advapi32:ADVAPI32.dll
 0000:fff88000       .debug$S                   0000000140000000     advapi32:ADVAPI32.dll
 0000:fff88000       .debug$S                   0000000140000000     user32:USER32.dll
 0000:fff88000       .debug$S                   0000000140000000     user32:USER32.dll
 0000:fff88000       .debug$S                   0000000140000000     user32:USER32.dll
 0000:fff88000       .debug$S                   0000000140000000     mfc140:mfc140.dll
 0000:fff88000       .debug$S                   0000000140000000     user32:USER32.dll
 0000:fff88000       .debug$S                   0000000140000000     mfc140:mfc140.dll
 0000:fff88000       .debug$S                   0000000140000000     user32:USER32.dll
 0000:fff88000       .debug$S                   0000000140000000     mfc140:mfc140.dll
 0000:fff88000       .debug$S                   0000000140000000     user32:USER32.dll
 0000:fff88000       .debug$S                   0000000140000000     mfc140:mfc140.dll
 0000:fff88000       .debug$S                   0000000140000000     user32:USER32.dll
 0000:fff88000       .debug$S                   0000000140000000     mfc140:mfc140.dll
 0000:fff88000       .debug$S                   0000000140000000     user32:USER32.dll
 0000:fff88000       .debug$S                   0000000140000000     mfc140:mfc140.dll
 0000:fff88000       .debug$S                   0000000140000000     user32:USER32.dll
 0000:fff88000       .debug$S                   0000000140000000     user32:USER32.dll
 0000:fff88000       .debug$S                   0000000140000000     user32:USER32.dll
 0000:fff88000       .debug$S                   0000000140000000     user32:USER32.dll
 0000:fff88000       .debug$S                   0000000140000000     mfc140:mfc140.dll
 0000:fff88000       .debug$S                   0000000140000000     user32:USER32.dll
 0000:fff88000       .debug$S                   0000000140000000     mfc140:mfc140.dll
 0000:fff88000       .debug$S                   0000000140000000     user32:USER32.dll
 0000:fff88000       .debug$S                   0000000140000000     mfc140:mfc140.dll
 0000:fff88000       .debug$S                   0000000140000000     kernel32:KERNEL32.dll
 0000:fff88000       .debug$S                   0000000140000000     mfc140:mfc140.dll
 0000:fff88000       .debug$S                   0000000140000000     kernel32:KERNEL32.dll
 0000:fff88000       .debug$S                   0000000140000000     mfc140:mfc140.dll
 0000:fff88000       .debug$S                   0000000140000000     kernel32:KERNEL32.dll
 0000:fff88000       .debug$S                   0000000140000000     mfc140:mfc140.dll
 0000:fff88000       .debug$S                   0000000140000000     kernel32:KERNEL32.dll
 0000:fff88000       .debug$S                   0000000140000000     mfc140:mfc140.dll
 0000:fff88000       .debug$S                   0000000140000000     kernel32:KERNEL32.dll
 0000:fff88000       .debug$S                   0000000140000000     mfc140:mfc140.dll
 0000:fff88000       .debug$S                   0000000140000000     kernel32:KERNEL32.dll
 0000:fff88000       .debug$S                   0000000140000000     mfc140:mfc140.dll
 0000:fff88000       .debug$S                   0000000140000000     kernel32:KERNEL32.dll
 0000:fff88000       .debug$S                   0000000140000000     mfc140:mfc140.dll
 0000:fff88000       .debug$S                   0000000140000000     kernel32:KERNEL32.dll
 0000:fff88000       .debug$S                   0000000140000000     mfc140:mfc140.dll
 0000:fff88000       .debug$S                   0000000140000000     kernel32:KERNEL32.dll
 0000:fff88000       .debug$S                   0000000140000000     mfc140:mfc140.dll
 0000:fff88000       .debug$S                   0000000140000000     kernel32:KERNEL32.dll
 0000:fff88000       .debug$S                   0000000140000000     mfc140:mfc140.dll
 0000:fff88000       .debug$S                   0000000140000000     kernel32:KERNEL32.dll
 0000:fff88000       .debug$S                   0000000140000000     mfc140:mfc140.dll
 0000:fff88000       .debug$S                   0000000140000000     kernel32:KERNEL32.dll
 0000:fff88000       .debug$S                   0000000140000000     mfc140:mfc140.dll
 0000:fff88000       .debug$S                   0000000140000000     kernel32:KERNEL32.dll
 0000:fff88000       .debug$S                   0000000140000000     mfc140:mfc140.dll
 0000:fff88000       .debug$S                   0000000140000000     kernel32:KERNEL32.dll
 0000:fff88000       .debug$S                   0000000140000000     mfc140:mfc140.dll
 0000:fff88000       .debug$S                   0000000140000000     kernel32:KERNEL32.dll
 0000:fff88000       .debug$S                   0000000140000000     mfc140:mfc140.dll
 0000:fff88000       .debug$S                   0000000140000000     kernel32:KERNEL32.dll
 0000:fff88000       .debug$S                   0000000140000000     mfc140:mfc140.dll
 0000:fff88000       .debug$S                   0000000140000000     kernel32:KERNEL32.dll
 0000:fff88000       .debug$S                   0000000140000000     mfc140:mfc140.dll
 0000:fff88000       .debug$S                   0000000140000000     kernel32:KERNEL32.dll
 0000:fff88000       .debug$S                   0000000140000000     mfc140:mfc140.dll
 0000:fff88000       .debug$S                   0000000140000000     kernel32:KERNEL32.dll
 0000:fff88000       .debug$S                   0000000140000000     mfc140:mfc140.dll
 0000:fff88000       .debug$S                   0000000140000000     kernel32:KERNEL32.dll
 0000:fff88000       .debug$S                   0000000140000000     mfc140:mfc140.dll
 0000:fff88000       .debug$S                   0000000140000000     kernel32:KERNEL32.dll
 0000:fff88000       .debug$S                   0000000140000000     mfc140:mfc140.dll
 0000:fff88000       .debug$S                   0000000140000000     kernel32:KERNEL32.dll
 0000:fff88000       .debug$S                   0000000140000000     mfc140:mfc140.dll
 0000:fff88000       .debug$S                   0000000140000000     kernel32:KERNEL32.dll
 0000:fff88000       .debug$S                   0000000140000000     mfc140:mfc140.dll
 0000:fff88000       .debug$S                   0000000140000000     kernel32:KERNEL32.dll
 0000:fff88000       .debug$S                   0000000140000000     mfc140:mfc140.dll
 0000:fff88000       .debug$S                   0000000140000000     kernel32:KERNEL32.dll
 0000:fff88000       .debug$S                   0000000140000000     mfc140:mfc140.dll
 0000:fff88000       .debug$S                   0000000140000000     kernel32:KERNEL32.dll
 0000:fff88000       .debug$S                   0000000140000000     mfc140:mfc140.dll
 0000:fff88000       .debug$S                   0000000140000000     kernel32:KERNEL32.dll
 0000:fff88000       .debug$S                   0000000140000000     mfc140:mfc140.dll
 0000:fff88000       .debug$S                   0000000140000000     kernel32:KERNEL32.dll
 0000:fff88000       .debug$S                   0000000140000000     mfc140:mfc140.dll
 0000:fff88000       .debug$S                   0000000140000000     kernel32:KERNEL32.dll
 0000:fff88000       .debug$S                   0000000140000000     mfc140:mfc140.dll
 0000:fff88000       .debug$S                   0000000140000000     kernel32:KERNEL32.dll
 0000:fff88000       .debug$S                   0000000140000000     kernel32:KERNEL32.dll
 0000:fff88000       .debug$S                   0000000140000000     kernel32:KERNEL32.dll
 0000:fff88000       .debug$S                   0000000140000000     kernel32:KERNEL32.dll
 0000:fff88000       .debug$S                   0000000140000000     kernel32:KERNEL32.dll
 0000:fff88000       .debug$S                   0000000140000000     mfc140:mfc140.dll
 0000:fff88000       .debug$S                   0000000140000000     kernel32:KERNEL32.dll
 0000:fff88000       .debug$S                   0000000140000000     kernel32:KERNEL32.dll
 0000:fff88000       .debug$S                   0000000140000000     kernel32:KERNEL32.dll
 0000:fff88000       .debug$S                   0000000140000000     kernel32:KERNEL32.dll
 0000:fff88000       .debug$S                   0000000140000000     mfc140:mfc140.dll
 0000:fff88000       .debug$S                   0000000140000000     kernel32:KERNEL32.dll
 0000:fff88000       .debug$S                   0000000140000000     kernel32:KERNEL32.dll
 0000:fff88000       .debug$S                   0000000140000000     kernel32:KERNEL32.dll
 0000:fff88000       .debug$S                   0000000140000000     kernel32:KERNEL32.dll
 0000:fff88000       .debug$S                   0000000140000000     mfc140:mfc140.dll
 0000:fff88000       .debug$S                   0000000140000000     kernel32:KERNEL32.dll
 0000:fff88000       .debug$S                   0000000140000000     mfc140:mfc140.dll
 0000:fff88000       .debug$S                   0000000140000000     kernel32:KERNEL32.dll
 0000:fff88000       .debug$S                   0000000140000000     kernel32:KERNEL32.dll
 0000:fff88000       .debug$S                   0000000140000000     kernel32:KERNEL32.dll
 0000:fff88000       .debug$S                   0000000140000000     kernel32:KERNEL32.dll
 0000:fff88000       .debug$S                   0000000140000000     kernel32:KERNEL32.dll
 0000:fff88000       .debug$S                   0000000140000000     kernel32:KERNEL32.dll
 0000:fff88000       .debug$S                   0000000140000000     kernel32:KERNEL32.dll
 0000:fff88000       .debug$S                   0000000140000000     kernel32:KERNEL32.dll
 0000:fff88000       .debug$S                   0000000140000000     kernel32:KERNEL32.dll
 0000:fff88000       .debug$S                   0000000140000000     kernel32:KERNEL32.dll
 0000:fff88000       .debug$S                   0000000140000000     kernel32:KERNEL32.dll
 0000:fff88000       .debug$S                   0000000140000000     kernel32:KERNEL32.dll
 0000:fff88000       .debug$S                   0000000140000000     kernel32:KERNEL32.dll
 0000:fff88000       .debug$S                   0000000140000000     kernel32:KERNEL32.dll
 0000:fff88000       .debug$S                   0000000140000000     kernel32:KERNEL32.dll
 0000:fff88000       .debug$S                   0000000140000000     kernel32:KERNEL32.dll
 0000:fff88000       .debug$S                   0000000140000000     kernel32:KERNEL32.dll
 0000:fff88000       .debug$S                   0000000140000000     kernel32:KERNEL32.dll
 0000:fff88000       .debug$S                   0000000140000000     kernel32:KERNEL32.dll
 0000:fff88000       .debug$S                   0000000140000000     kernel32:KERNEL32.dll
 0000:fff88000       .debug$S                   0000000140000000     kernel32:KERNEL32.dll
 0000:fff88000       .debug$S                   0000000140000000     kernel32:KERNEL32.dll
 0000:fff88000       .debug$S                   0000000140000000     kernel32:KERNEL32.dll
 0000:fff88000       .debug$S                   0000000140000000     kernel32:KERNEL32.dll
 0000:fff88000       .debug$S                   0000000140000000     kernel32:KERNEL32.dll
 0000:fff88000       .debug$S                   0000000140000000     kernel32:KERNEL32.dll
 0000:fff88000       .debug$S                   0000000140000000     kernel32:KERNEL32.dll
 0000:fff88000       .debug$S                   0000000140000000     kernel32:KERNEL32.dll
 0000:fff88000       .debug$S                   0000000140000000     kernel32:KERNEL32.dll
 0000:fff88000       .debug$S                   0000000140000000     kernel32:KERNEL32.dll
 0000:fff88000       .debug$S                   0000000140000000     kernel32:KERNEL32.dll
 0000:fff88000       .debug$S                   0000000140000000     kernel32:KERNEL32.dll
 0000:fff88000       .debug$S                   0000000140000000     kernel32:KERNEL32.dll
 0000:fff88000       .debug$S                   0000000140000000     kernel32:KERNEL32.dll
 0000:fff88000       .debug$S                   0000000140000000     kernel32:KERNEL32.dll
 0000:fff88000       .debug$S                   0000000140000000     kernel32:KERNEL32.dll
 0000:fff88000       .debug$S                   0000000140000000     kernel32:KERNEL32.dll
 0000:fff88000       .debug$S                   0000000140000000     kernel32:KERNEL32.dll
 0000:fff88000       .debug$S                   0000000140000000     kernel32:KERNEL32.dll
 0000:fff88000       .debug$S                   0000000140000000     mfc140:mfc140.dll
 0000:fff88000       .debug$S                   0000000140000000     kernel32:KERNEL32.dll
 0000:fff88000       .debug$S                   0000000140000000     kernel32:KERNEL32.dll
 0000:fff88000       .debug$S                   0000000140000000     kernel32:KERNEL32.dll
 0000:fff88000       .debug$S                   0000000140000000     kernel32:KERNEL32.dll
 0000:fff88000       .debug$S                   0000000140000000     mfc140:mfc140.dll
 0000:fff88000       .debug$S                   0000000140000000     kernel32:KERNEL32.dll
 0000:fff88000       .debug$S                   0000000140000000     mfc140:mfc140.dll
 0000:fff88000       .debug$S                   0000000140000000     kernel32:KERNEL32.dll
 0000:fff88000       .debug$S                   0000000140000000     mfc140:mfc140.dll
 0000:fff88000       .debug$S                   0000000140000000     kernel32:KERNEL32.dll
 0000:fff88000       .debug$S                   0000000140000000     mfc140:mfc140.dll
 0000:fff88000       .debug$S                   0000000140000000     kernel32:KERNEL32.dll
 0000:fff88000       .debug$S                   0000000140000000     mfc140:mfc140.dll
 0000:fff88000       .debug$S                   0000000140000000     kernel32:KERNEL32.dll
 0000:fff88000       .debug$S                   0000000140000000     mfc140:mfc140.dll
 0000:fff88000       .debug$S                   0000000140000000     kernel32:KERNEL32.dll
 0000:fff88000       .debug$S                   0000000140000000     mfc140:mfc140.dll
 0000:fff88000       .debug$S                   0000000140000000     kernel32:KERNEL32.dll
 0000:fff88000       .debug$S                   0000000140000000     kernel32:KERNEL32.dll
 0000:fff88000       .debug$S                   0000000140000000     mfc140:mfc140.dll
 0000:fff88000       .debug$S                   0000000140000000     kernel32:KERNEL32.dll
 0000:fff88000       .debug$S                   0000000140000000     mfc140:mfc140.dll
 0000:fff88000       .debug$S                   0000000140000000     kernel32:KERNEL32.dll
 0000:fff88000       .debug$S                   0000000140000000     mfc140:mfc140.dll
 0000:fff88000       .debug$S                   0000000140000000     kernel32:KERNEL32.dll
 0000:fff88000       .debug$S                   0000000140000000     mfc140:mfc140.dll
 0000:fff88000       .debug$S                   0000000140000000     mfc140:mfc140.dll
 0000:fff88000       .debug$S                   0000000140000000     mfc140:mfc140.dll
 0000:fff88000       .debug$S                   0000000140000000     mfc140:mfc140.dll
 0000:fff88000       .debug$S                   0000000140000000     mfc140:mfc140.dll
 0000:fff88000       .debug$S                   0000000140000000     mfc140:mfc140.dll
 0000:fff88000       .debug$S                   0000000140000000     mfc140:mfc140.dll
 0000:fff88000       .debug$S                   0000000140000000     mfc140:mfc140.dll
 0000:fff88000       .debug$S                   0000000140000000     mfc140:mfc140.dll
 0000:fff88000       .debug$S                   0000000140000000     mfc140:mfc140.dll
 0000:fff88000       .debug$S                   0000000140000000     mfc140:mfc140.dll
 0000:fff88000       .debug$S                   0000000140000000     mfc140:mfc140.dll
 0000:fff88000       .debug$S                   0000000140000000     mfc140:mfc140.dll
 0000:fff88000       .debug$S                   0000000140000000     mfc140:mfc140.dll
 0000:fff88000       .debug$S                   0000000140000000     mfc140:mfc140.dll
 0000:fff88000       .debug$S                   0000000140000000     mfc140:mfc140.dll
 0000:fff88000       .debug$S                   0000000140000000     mfc140:mfc140.dll
 0000:fff88000       .debug$S                   0000000140000000     mfc140:mfc140.dll
 0000:fff88000       .debug$S                   0000000140000000     mfc140:mfc140.dll
 0000:fff88000       .debug$S                   0000000140000000     mfc140:mfc140.dll
 0000:fff88000       .debug$S                   0000000140000000     mfc140:mfc140.dll
 0000:fff88000       .debug$S                   0000000140000000     mfc140:mfc140.dll
 0000:fff88000       .debug$S                   0000000140000000     mfc140:mfc140.dll
 0000:fff88000       .debug$S                   0000000140000000     mfc140:mfc140.dll
 0000:fff88000       .debug$S                   0000000140000000     mfc140:mfc140.dll
 0000:fff88000       .debug$S                   0000000140000000     mfc140:mfc140.dll
 0000:fff88000       .debug$S                   0000000140000000     mfc140:mfc140.dll
 0000:fff88000       .debug$S                   0000000140000000     mfc140:mfc140.dll
 0000:fff88000       .debug$S                   0000000140000000     mfc140:mfc140.dll
 0000:fff88000       .debug$S                   0000000140000000     mfc140:mfc140.dll
 0000:fff88000       .debug$S                   0000000140000000     mfc140:mfc140.dll
 0000:fff88000       .debug$S                   0000000140000000     mfc140:mfc140.dll
 0000:fff88000       .debug$S                   0000000140000000     mfc140:mfc140.dll
 0000:fff88000       .debug$S                   0000000140000000     mfc140:mfc140.dll
 0000:fff88000       .debug$S                   0000000140000000     mfc140:mfc140.dll
 0000:fff88000       .debug$S                   0000000140000000     mfc140:mfc140.dll
 0000:fff88000       .debug$S                   0000000140000000     mfc140:mfc140.dll
 0000:fff88000       .debug$S                   0000000140000000     mfc140:mfc140.dll
 0000:fff88000       .debug$S                   0000000140000000     mfc140:mfc140.dll
 0000:fff88000       .debug$S                   0000000140000000     mfc140:mfc140.dll
 0000:fff88000       .debug$S                   0000000140000000     mfc140:mfc140.dll
 0000:fff88000       .debug$S                   0000000140000000     mfc140:mfc140.dll
 0000:fff88000       .debug$S                   0000000140000000     mfc140:mfc140.dll
 0000:fff88000       .debug$S                   0000000140000000     mfc140:mfc140.dll
 0000:fff88000       .debug$S                   0000000140000000     mfc140:mfc140.dll
 0000:fff88000       .debug$S                   0000000140000000     mfc140:mfc140.dll
 0000:fff88000       .debug$S                   0000000140000000     mfc140:mfc140.dll
 0000:fff88000       .debug$S                   0000000140000000     mfc140:mfc140.dll
 0000:fff88000       .debug$S                   0000000140000000     mfc140:mfc140.dll
 0000:fff88000       .debug$S                   0000000140000000     mfc140:mfc140.dll
 0000:fff88000       .debug$S                   0000000140000000     mfc140:mfc140.dll
 0000:fff88000       .debug$S                   0000000140000000     mfc140:mfc140.dll
 0000:fff88000       .debug$S                   0000000140000000     mfc140:mfc140.dll
 0000:fff88000       .debug$S                   0000000140000000     mfc140:mfc140.dll
 0000:fff88000       .debug$S                   0000000140000000     mfc140:mfc140.dll
 0000:fff88000       .debug$S                   0000000140000000     mfc140:mfc140.dll
 0000:fff88000       .debug$S                   0000000140000000     mfc140:mfc140.dll
 0000:fff88000       .debug$S                   0000000140000000     mfc140:mfc140.dll
 0000:fff88000       .debug$S                   0000000140000000     mfc140:mfc140.dll
 0000:fff88000       .debug$S                   0000000140000000     mfc140:mfc140.dll
 0000:fff88000       .debug$S                   0000000140000000     mfc140:mfc140.dll
 0000:fff88000       .debug$S                   0000000140000000     mfc140:mfc140.dll
 0000:fff88000       .debug$S                   0000000140000000     mfc140:mfc140.dll
 0000:fff88000       .debug$S                   0000000140000000     mfc140:mfc140.dll
 0000:fff88000       .debug$S                   0000000140000000     mfc140:mfc140.dll
 0000:fff88000       .debug$S                   0000000140000000     mfc140:mfc140.dll
 0000:fff88000       .debug$S                   0000000140000000     mfc140:mfc140.dll
 0000:fff88000       .debug$S                   0000000140000000     mfc140:mfc140.dll
 0000:fff88000       .debug$S                   0000000140000000     mfc140:mfc140.dll
 0000:fff88000       .debug$S                   0000000140000000     mfc140:mfc140.dll
 0000:fff88000       .debug$S                   0000000140000000     mfc140:mfc140.dll
 0000:fff88000       .debug$S                   0000000140000000     mfc140:mfc140.dll
 0000:fff88000       .debug$S                   0000000140000000     mfc140:mfc140.dll
 0000:fff88000       .debug$S                   0000000140000000     mfc140:mfc140.dll
 0000:fff88000       .debug$S                   0000000140000000     mfc140:mfc140.dll
 0000:fff88000       .debug$S                   0000000140000000     mfc140:mfc140.dll
 0000:fff88000       .debug$S                   0000000140000000     mfc140:mfc140.dll
 0000:fff88000       .debug$S                   0000000140000000     mfc140:mfc140.dll
 0000:fff88000       .debug$S                   0000000140000000     mfc140:mfc140.dll
 0000:fff88000       .debug$S                   0000000140000000     mfc140:mfc140.dll
 0000:fff88000       .debug$S                   0000000140000000     mfc140:mfc140.dll
 0000:fff88000       .debug$S                   0000000140000000     mfc140:mfc140.dll
 0000:fff88000       .debug$S                   0000000140000000     mfc140:mfc140.dll
 0000:fff88000       .debug$S                   0000000140000000     mfc140:mfc140.dll
 0000:fff88000       .debug$S                   0000000140000000     mfc140:mfc140.dll
 0000:fff88000       .debug$S                   0000000140000000     mfc140:mfc140.dll
 0000:fff88000       .debug$S                   0000000140000000     mfc140:mfc140.dll
 0000:fff88000       .debug$S                   0000000140000000     mfc140:mfc140.dll
 0000:fff88000       .debug$S                   0000000140000000     mfc140:mfc140.dll
 0000:fff88000       .debug$S                   0000000140000000     mfc140:mfc140.dll
 0000:fff88000       .debug$S                   0000000140000000     mfc140:mfc140.dll
 0000:fff88000       .debug$S                   0000000140000000     mfc140:mfc140.dll
 0000:fff88000       .debug$S                   0000000140000000     mfc140:mfc140.dll
 0000:fff88000       .debug$S                   0000000140000000     mfc140:mfc140.dll
 0000:fff88000       .debug$S                   0000000140000000     mfc140:mfc140.dll
 0000:fff88000       .debug$S                   0000000140000000     mfc140:mfc140.dll
 0000:fff88000       .debug$S                   0000000140000000     mfc140:mfc140.dll
 0000:fff88000       .debug$S                   0000000140000000     mfc140:mfc140.dll
 0000:fff88000       .debug$S                   0000000140000000     mfc140:mfc140.dll
 0000:fff88000       .debug$S                   0000000140000000     mfc140:mfc140.dll
 0000:fff88000       .debug$S                   0000000140000000     mfc140:mfc140.dll
 0000:fff88000       .debug$S                   0000000140000000     mfc140:mfc140.dll
 0000:fff88000       .debug$S                   0000000140000000     mfc140:mfc140.dll
 0000:fff88000       .debug$S                   0000000140000000     msvcprt:MSVCP140.dll
 0001:00000000       ??__EtheApp@@YAXXZ         0000000140001000 f   GameServerManager.obj
 0001:00000040       ??__Eg_cServerLog@@YAXXZ   0000000140001040 f   GameServerManagerDlg.obj
 0001:000001a0       ??__Ebase64_chars@@YAXXZ   00000001400011a0 f   base64.obj
 0001:000001d0       ??__Eg_HostStat@@YAXXZ     00000001400011d0 f   HostStat.obj
 0001:00000290       ??__E?m_strFileFormat@CHLogger@@0V?$basic_string@DU?$char_traits@D@std@@V?$allocator@D@2@@std@@A@@YAXXZ 0000000140001290 f   HostLogger.obj
 0001:000002a0       ??__E?m_strBRFileFormat@CHLogger@@0V?$basic_string@DU?$char_traits@D@std@@V?$allocator@D@2@@std@@A@@YAXXZ 00000001400012a0 f   HostLogger.obj
 0001:000002b0       ??__E?m_strKernelFileFormat@CHLogger@@0V?$basic_string@DU?$char_traits@D@std@@V?$allocator@D@2@@std@@A@@YAXXZ 00000001400012b0 f   HostLogger.obj
 0001:000002c0       ??__E?m_strEtcFileFormat@CHLogger@@0V?$basic_string@DU?$char_traits@D@std@@V?$allocator@D@2@@std@@A@@YAXXZ 00000001400012c0 f   HostLogger.obj
 0001:000002d0       ??__E?m_strRWProcessMemoryFileFormat@CHLogger@@0V?$basic_string@DU?$char_traits@D@std@@V?$allocator@D@2@@std@@A@@YAXXZ 00000001400012d0 f   HostLogger.obj
 0001:000002e0       ??__E?m_strIPCMessageFileFormat@CHLogger@@0V?$basic_string@DU?$char_traits@D@std@@V?$allocator@D@2@@std@@A@@YAXXZ 00000001400012e0 f   HostLogger.obj
 0001:000002f0       ??__E?m_strTimeOutFileFormat@CHLogger@@0V?$basic_string@DU?$char_traits@D@std@@V?$allocator@D@2@@std@@A@@YAXXZ 00000001400012f0 f   HostLogger.obj
 0001:00000300       ??__E?m_strPacketFileFormat@CHLogger@@0V?$basic_string@DU?$char_traits@D@std@@V?$allocator@D@2@@std@@A@@YAXXZ 0000000140001300 f   HostLogger.obj
 0001:00000310       ??__E?m_strHostName@CHLogger@@0V?$basic_string@DU?$char_traits@D@std@@V?$allocator@D@2@@std@@A@@YAXXZ 0000000140001310 f   HostLogger.obj
 0001:00000320       ??__E?m_strServerName@CHLogger@@0V?$basic_string@DU?$char_traits@D@std@@V?$allocator@D@2@@std@@A@@YAXXZ 0000000140001320 f   HostLogger.obj
 0001:00000330       ??__E?m_strLogFolder@CHLogger@@0V?$basic_string@DU?$char_traits@D@std@@V?$allocator@D@2@@std@@A@@YAXXZ 0000000140001330 f   HostLogger.obj
 0001:00000340       ??__E?m_strModeUserCountFormat@CHLogger@@0V?$basic_string@DU?$char_traits@D@std@@V?$allocator@D@2@@std@@A@@YAXXZ 0000000140001340 f   HostLogger.obj
 0001:00000350       ??__E?m_strServerAppUseCountFormat@CHLogger@@0V?$basic_string@DU?$char_traits@D@std@@V?$allocator@D@2@@std@@A@@YAXXZ 0000000140001350 f   HostLogger.obj
 0001:00000360       ??__E?m_LogLock@CHLogger@@0VCMustSyncObjectLog@@A@@YAXXZ 0000000140001360 f   HostLogger.obj
 0001:00000390       ??__E?m_LogPacketLock@CHLogger@@0VCMustSyncObjectLog@@A@@YAXXZ 0000000140001390 f   HostLogger.obj
 0001:000003c0       ??__E?m_vectSharedMapHandles@CLogMsgManager@@0V?$vector@PEAXV?$allocator@PEAX@std@@@std@@A@@YAXXZ 00000001400013c0 f   LogMsgManager.obj
 0001:000003d0       ??__EFloatOne@GlobalVectorConstants@@YAXXZ 00000001400013d0 f   StdAfx.obj
 0001:000003e0       ??__EFloatZero@GlobalVectorConstants@@YAXXZ 00000001400013e0 f   StdAfx.obj
 0001:000003f0       ??__EFloatMinusOne@GlobalVectorConstants@@YAXXZ 00000001400013f0 f   StdAfx.obj
 0001:00000400       ??__EFloatOneHalf@GlobalVectorConstants@@YAXXZ 0000000140001400 f   StdAfx.obj
 0001:00000410       ??__EXYZMask@GlobalVectorConstants@@YAXXZ 0000000140001410 f   StdAfx.obj
 0001:00000430       ??__ETwoPi@GlobalVectorConstants@@YAXXZ 0000000140001430 f   StdAfx.obj
 0001:00000440       ??__EPiByTwo@GlobalVectorConstants@@YAXXZ 0000000140001440 f   StdAfx.obj
 0001:00000450       ??__EOneOverTwoPi@GlobalVectorConstants@@YAXXZ 0000000140001450 f   StdAfx.obj
 0001:00000460       ??__Ea@VectorSinConstantsSSE@@YAXXZ 0000000140001460 f   StdAfx.obj
 0001:00000490       ??__Eb@VectorSinConstantsSSE@@YAXXZ 0000000140001490 f   StdAfx.obj
 0001:000004c0       ??__EA@VectorSinConstantsSSE@@YAXXZ 00000001400014c0 f   StdAfx.obj
 0001:000004e0       ??__EB@VectorSinConstantsSSE@@YAXXZ 00000001400014e0 f   StdAfx.obj
 0001:00000500       ??__EPI@@YAXXZ             0000000140001500 f   StdAfx.obj
 0001:00000530       ??__E__iob_func@@YAXXZ     0000000140001530 f   StdAfx.obj
 0001:00000558       ??__E_AtlBaseModule@ATL@@YAXXZ 0000000140001558 f   atls:atlbase.obj
 0001:00000578       ??__E_Fac_tidy_reg@std@@YAXXZ 0000000140001578 f   msvcprt:locale0_implib.obj
 0001:00000584       ??__E_afxInitAppState@@YAXXZ 0000000140001584 f   mfcs140:appmodul.obj
 0001:00000970       memcpy_s                   0000000140001970 f   DivisionPacket.obj
 0001:00001390       ?CRSUploader@@YAAEAVUploader@crs@@XZ 0000000140002390 f   BugReporter.obj
 0001:00003430       ?EnumModuleDetail@ModuleInfo@?1??makeExceptionLog@Uploader@crs@@QEAAXPEAU_EXCEPTION_POINTERS@@AEAVLogBuffer@4@@Z@SAHPEBD_KKPEAX@Z 0000000140004430 f   crs_uploader.obj
 0001:00015148       $LN1462                    0000000140016148     GameServerManagerDlg.obj
 0001:0001521c       $LN1459                    000000014001621c     GameServerManagerDlg.obj
 0001:00019278       $LN196                     000000014001a278     GameServerManagerDlg.obj
 0001:000192cc       $LN195                     000000014001a2cc     GameServerManagerDlg.obj
 0001:00020a54       $LN228                     0000000140021a54     GameServerManagerDlg.obj
 0001:00020a80       $LN227                     0000000140021a80     GameServerManagerDlg.obj
 0001:000260d0       ?RTIDUSNtoString@EXPAND_USN@@YA?AV?$basic_string@DU?$char_traits@D@std@@V?$allocator@D@2@@std@@HFF_J@Z 00000001400270d0 f   GameServerManagerDlg.obj
 0001:000262f0       ?USNtoStr@EXPAND_USN@@YA?AV?$basic_string@DU?$char_traits@D@std@@V?$allocator@D@2@@std@@_J@Z 00000001400272f0 f   GameServerManagerDlg.obj
 0001:000263a0       time                       00000001400273a0 f   GameServerManagerDlg.obj
 0001:000289a0       memcpy_s                   00000001400299a0 f   GameServerManagerDlg.obj
 0001:00033658       $LN106                     0000000140034658     iniReader.obj
 0001:00033688       $LN105                     0000000140034688     iniReader.obj
 0001:0003e0b0       des_key_schedule           000000014003f0b0 f   des.obj
 0001:0003fca0       ntlm_convert_key           0000000140040ca0 f   ntlmencrypt.obj
 0001:00043608       $LN70                      0000000140044608     base6409cee8549d9fd00dfa06fdadc87a8424.obj
 0001:00045de0       $$000000                   0000000140046de0     msvcrt:amdsecgs.obj
 0001:00045e1c       ?__scrt_initialize_thread_safe_statics@@YAHXZ 0000000140046e1c f   msvcrt:thread_safe_statics.obj
 0001:00045f7c       ?__scrt_uninitialize_thread_safe_statics@@YAXXZ 0000000140046f7c f   msvcrt:thread_safe_statics.obj
 0001:00046744       capture_current_context    0000000140047744 f   msvcrt:gs_report.obj
 0001:000467b4       capture_previous_context   00000001400477b4 f   msvcrt:gs_report.obj
 0001:00046828       ?pre_c_initialization@@YAHXZ 0000000140047828 f   msvcrt:exe_winmain.obj
 0001:000468e0       ?post_pgo_initialization@@YAHXZ 00000001400478e0 f   msvcrt:exe_winmain.obj
 0001:000468f0       ?pre_cpp_initialization@@YAXXZ 00000001400478f0 f   msvcrt:exe_winmain.obj
 0001:0004690c       ?__scrt_common_main_seh@@YAHXZ 000000014004790c f   msvcrt:exe_winmain.obj
 0001:00047340       $$000000                   0000000140048340     msvcrt:chkstk.obj
 0001:000473d0       $$000000                   00000001400483d0     msvcrt:guard_dispatch.obj
 0001:000473f0       ?dtor$0@?0??Instance@DivisionPacketReceiver@@SAPEAV1@XZ@4HA 00000001400483f0 f   DivisionPacketReceiver.obj
 0001:00047400       ?dtor$0@?0??GetPacketBuffer@DivisionPacketReceiver@@QEAA?BW4DIVISION_PACKET_RESULT@@EEEEEPEADG0H@Z@4HA 0000000140048400 f   DivisionPacketReceiver.obj
 0001:0004740c       ?dtor$1@?0??GetPacketBuffer@DivisionPacketReceiver@@QEAA?BW4DIVISION_PACKET_RESULT@@EEEEEPEADG0H@Z@4HA 000000014004840c f   DivisionPacketReceiver.obj
 0001:00047420       ?catch$2@?0???$_Buynode@U?$pair@_JVDivisionPacket@@@std@@@?$_Tree_comp_alloc@V?$_Tmap_traits@_JVDivisionPacket@@U?$less@_J@std@@V?$allocator@U?$pair@$$CB_JVDivisionPacket@@@std@@@3@$0A@@std@@@std@@QEAAPEAU?$_Tree_node@U?$pair@$$CB_JVDivisionPacket@@@std@@PEAX@1@$$QEAU?$pair@_JVDivisionPacket@@@1@@Z@4HA 0000000140048420 f   DivisionPacketReceiver.obj
 0001:0004742d       __catch$??$_Buynode@U?$pair@_JVDivisionPacket@@@std@@@?$_Tree_comp_alloc@V?$_Tmap_traits@_JVDivisionPacket@@U?$less@_J@std@@V?$allocator@U?$pair@$$CB_JVDivisionPacket@@@std@@@3@$0A@@std@@@std@@QEAAPEAU?$_Tree_node@U?$pair@$$CB_JVDivisionPacket@@@std@@PEAX@1@$$QEAU?$pair@_JVDivisionPacket@@@1@@Z$0 000000014004842d f   DivisionPacketReceiver.obj
 0001:00047440       ?catch$2@?0???$_Insert_nohint@AEAU?$pair@$$CB_JVDivisionPacket@@@std@@PEAU?$_Tree_node@U?$pair@$$CB_JVDivisionPacket@@@std@@PEAX@2@@?$_Tree@V?$_Tmap_traits@_JVDivisionPacket@@U?$less@_J@std@@V?$allocator@U?$pair@$$CB_JVDivisionPacket@@@std@@@3@$0A@@std@@@std@@IEAA?AU?$pair@V?$_Tree_iterator@V?$_Tree_val@U?$_Tree_simple_types@U?$pair@$$CB_JVDivisionPacket@@@std@@@std@@@std@@@std@@_N@1@_NAEAU?$pair@$$CB_JVDivisionPacket@@@1@PEAU?$_Tree_node@U?$pair@$$CB_JVDivisionPacket@@@std@@PEAX@1@@Z@4HA 0000000140048440 f   DivisionPacketReceiver.obj
 0001:0004744d       __catch$??$_Insert_nohint@AEAU?$pair@$$CB_JVDivisionPacket@@@std@@PEAU?$_Tree_node@U?$pair@$$CB_JVDivisionPacket@@@std@@PEAX@2@@?$_Tree@V?$_Tmap_traits@_JVDivisionPacket@@U?$less@_J@std@@V?$allocator@U?$pair@$$CB_JVDivisionPacket@@@std@@@3@$0A@@std@@@std@@IEAA?AU?$pair@V?$_Tree_iterator@V?$_Tree_val@U?$_Tree_simple_types@U?$pair@$$CB_JVDivisionPacket@@@std@@@std@@@std@@@std@@_N@1@_NAEAU?$pair@$$CB_JVDivisionPacket@@@1@PEAU?$_Tree_node@U?$pair@$$CB_JVDivisionPacket@@@std@@PEAX@1@@Z$0 000000014004844d f   DivisionPacketReceiver.obj
 0001:00047470       ?dtor$0@?0??CRSUploader@@YAAEAVUploader@crs@@XZ@4HA 0000000140048470 f   BugReporter.obj
 0001:0004747c       ?dtor$1@?0??CRSUploader@@YAAEAVUploader@crs@@XZ@4HA 000000014004847c f   BugReporter.obj
 0001:00047499       ?dtor$8@?0??CRSUploader@@YAAEAVUploader@crs@@XZ@4HA 0000000140048499 f   BugReporter.obj
 0001:000474b0       ?dtor$0@?0??threadCreateDumpFile@@YAKPEAX@Z@4HA 00000001400484b0 f   BugReporter.obj
 0001:000474c0       ?dtor$0@?0??readURL@Uploader@crs@@AEAAXAEAV?$basic_string@_WU?$char_traits@_W@std@@V?$allocator@_W@2@@std@@@Z@4HA 00000001400484c0 f   crs_uploader.obj
 0001:000474cc       ?dtor$1@?0??readURL@Uploader@crs@@AEAAXAEAV?$basic_string@_WU?$char_traits@_W@std@@V?$allocator@_W@2@@std@@@Z@4HA 00000001400484cc f   crs_uploader.obj
 0001:000474e0       ?dtor$0@?0??init@Uploader@crs@@QEAA_N_NPEAD1@Z@4HA 00000001400484e0 f   crs_uploader.obj
 0001:000474f0       ?dtor$0@?0??ProcessSocketEvent@CClientLib@@QEAAXXZ@4HA 00000001400484f0 f   ClientLib.obj
 0001:000474f0       ?dtor$0@?0??SendDiv@CGMSConnManager@@AEAAHEEEPEADK@Z@4HA 00000001400484f0 f   GMSConnManager.obj
 0001:00047500       ?dtor$0@?0??Connect@CSFGameServerClientLib@@QEAAHH@Z@4HA 0000000140048500 f   SFGameServerClientLib.obj
 0001:00047510       ?dtor$0@?0??ConnectToMatchMakingServer@CGameServerManagerDlg@@QEAAHXZ@4HA 0000000140048510 f   GameServerManagerDlg.obj
 0001:00047510       ?dtor$0@?0??GetProcessMemoryUsage@@YAKPEAXH@Z@4HA 0000000140048510 f   CheckMemUsage.obj
 0001:00047510       ?dtor$0@?0??EmptyWorkingset@CHECK_MEM_USAGE@@YA_NPEAXH@Z@4HA 0000000140048510 f   CheckMemUsage.obj
 0001:0004751c       ?dtor$1@?0??EmptyWorkingset@CHECK_MEM_USAGE@@YA_NPEAXH@Z@4HA 000000014004851c f   CheckMemUsage.obj
 0001:0004751c       ?dtor$1@?0??GetProcessMemoryUsage@@YAKPEAXH@Z@4HA 000000014004851c f   CheckMemUsage.obj
 0001:0004751c       ?dtor$1@?0??ConnectToMatchMakingServer@CGameServerManagerDlg@@QEAAHXZ@4HA 000000014004851c f   GameServerManagerDlg.obj
 0001:00047528       ?dtor$2@?0??ConnectToMatchMakingServer@CGameServerManagerDlg@@QEAAHXZ@4HA 0000000140048528 f   GameServerManagerDlg.obj
 0001:00047528       ?dtor$2@?0??EmptyWorkingset@CHECK_MEM_USAGE@@YA_NPEAXH@Z@4HA 0000000140048528 f   CheckMemUsage.obj
 0001:00047528       ?dtor$2@?0??GetProcessMemoryUsage@@YAKPEAXH@Z@4HA 0000000140048528 f   CheckMemUsage.obj
 0001:00047540       ?dtor$0@?0??MyServiceMain@@YAXKPEAPEAD@Z@4HA 0000000140048540 f   GameServerManager.obj
 0001:00047550       ?dtor$0@?0??KillRemoteProcess@@YA_NK@Z@4HA 0000000140048550 f   GameServerManagerDlg.obj
 0001:0004755c       ?dtor$1@?0??KillRemoteProcess@@YA_NK@Z@4HA 000000014004855c f   GameServerManagerDlg.obj
 0001:00047568       ?dtor$2@?0??KillRemoteProcess@@YA_NK@Z@4HA 0000000140048568 f   GameServerManagerDlg.obj
 0001:00047574       ?dtor$3@?0??KillRemoteProcess@@YA_NK@Z@4HA 0000000140048574 f   GameServerManagerDlg.obj
 0001:00047580       ?dtor$4@?0??KillRemoteProcess@@YA_NK@Z@4HA 0000000140048580 f   GameServerManagerDlg.obj
 0001:0004758c       ?dtor$5@?0??KillRemoteProcess@@YA_NK@Z@4HA 000000014004858c f   GameServerManagerDlg.obj
 0001:00047598       ?dtor$6@?0??KillRemoteProcess@@YA_NK@Z@4HA 0000000140048598 f   GameServerManagerDlg.obj
 0001:000475a4       ?dtor$7@?0??KillRemoteProcess@@YA_NK@Z@4HA 00000001400485a4 f   GameServerManagerDlg.obj
 0001:000475b0       ?dtor$0@?0???0CGameServerManagerDlg@@QEAA@PEAVCWnd@@@Z@4HA 00000001400485b0 f   GameServerManagerDlg.obj
 0001:000475be       ?dtor$1@?0???0CGameServerManagerDlg@@QEAA@PEAVCWnd@@@Z@4HA 00000001400485be f   GameServerManagerDlg.obj
 0001:000475d1       ?dtor$2@?0???0CGameServerManagerDlg@@QEAA@PEAVCWnd@@@Z@4HA 00000001400485d1 f   GameServerManagerDlg.obj
 0001:000475e6       ?dtor$3@?0???0CGameServerManagerDlg@@QEAA@PEAVCWnd@@@Z@4HA 00000001400485e6 f   GameServerManagerDlg.obj
 0001:000475fb       ?dtor$4@?0???0CGameServerManagerDlg@@QEAA@PEAVCWnd@@@Z@4HA 00000001400485fb f   GameServerManagerDlg.obj
 0001:0004760e       ?dtor$5@?0???0CGameServerManagerDlg@@QEAA@PEAVCWnd@@@Z@4HA 000000014004860e f   GameServerManagerDlg.obj
 0001:00047623       ?dtor$6@?0???0CGameServerManagerDlg@@QEAA@PEAVCWnd@@@Z@4HA 0000000140048623 f   GameServerManagerDlg.obj
 0001:00047636       ?dtor$7@?0???0CGameServerManagerDlg@@QEAA@PEAVCWnd@@@Z@4HA 0000000140048636 f   GameServerManagerDlg.obj
 0001:0004764b       ?dtor$17@?0???0CGameServerManagerDlg@@QEAA@PEAVCWnd@@@Z@4HA 000000014004864b f   GameServerManagerDlg.obj
 0001:0004765b       ?dtor$18@?0???0CGameServerManagerDlg@@QEAA@PEAVCWnd@@@Z@4HA 000000014004865b f   GameServerManagerDlg.obj
 0001:0004766b       ?dtor$8@?0???0CGameServerManagerDlg@@QEAA@PEAVCWnd@@@Z@4HA 000000014004866b f   GameServerManagerDlg.obj
 0001:0004767e       ?dtor$9@?0???0CGameServerManagerDlg@@QEAA@PEAVCWnd@@@Z@4HA 000000014004867e f   GameServerManagerDlg.obj
 0001:00047691       ?dtor$10@?0???0CGameServerManagerDlg@@QEAA@PEAVCWnd@@@Z@4HA 0000000140048691 f   GameServerManagerDlg.obj
 0001:000476a4       ?dtor$11@?0???0CGameServerManagerDlg@@QEAA@PEAVCWnd@@@Z@4HA 00000001400486a4 f   GameServerManagerDlg.obj
 0001:000476b7       ?dtor$12@?0???0CGameServerManagerDlg@@QEAA@PEAVCWnd@@@Z@4HA 00000001400486b7 f   GameServerManagerDlg.obj
 0001:000476ca       ?dtor$13@?0???0CGameServerManagerDlg@@QEAA@PEAVCWnd@@@Z@4HA 00000001400486ca f   GameServerManagerDlg.obj
 0001:000476f0       ?dtor$5@?0??InitializeManager@CGameServerManagerDlg@@QEAAHPEADKPEAPEAD@Z@4HA 00000001400486f0 f   GameServerManagerDlg.obj
 0001:0004772e       ?dtor$0@?0??InitializeManager@CGameServerManagerDlg@@QEAAHPEADKPEAPEAD@Z@4HA 000000014004872e f   GameServerManagerDlg.obj
 0001:0004773a       ?dtor$1@?0??InitializeManager@CGameServerManagerDlg@@QEAAHPEADKPEAPEAD@Z@4HA 000000014004873a f   GameServerManagerDlg.obj
 0001:00047757       ?dtor$10@?0??InitializeManager@CGameServerManagerDlg@@QEAAHPEADKPEAPEAD@Z@4HA 0000000140048757 f   GameServerManagerDlg.obj
 0001:00047763       ?dtor$2@?0??InitializeManager@CGameServerManagerDlg@@QEAAHPEADKPEAPEAD@Z@4HA 0000000140048763 f   GameServerManagerDlg.obj
 0001:0004776f       ?dtor$3@?0??InitializeManager@CGameServerManagerDlg@@QEAAHPEADKPEAPEAD@Z@4HA 000000014004876f f   GameServerManagerDlg.obj
 0001:0004777b       ?dtor$4@?0??InitializeManager@CGameServerManagerDlg@@QEAAHPEADKPEAPEAD@Z@4HA 000000014004877b f   GameServerManagerDlg.obj
 0001:00047790       ?dtor$0@?0??ReadSettings@CGameServerManagerDlg@@QEAAHXZ@4HA 0000000140048790 f   GameServerManagerDlg.obj
 0001:000477a0       ?dtor$0@?0??StartGameServer@CGameServerManagerDlg@@QEAAHF@Z@4HA 00000001400487a0 f   GameServerManagerDlg.obj
 0001:000477b0       ?dtor$0@?0??OnGameServerMsg@CGameServerManagerDlg@@IEAA_J_K_J@Z@4HA 00000001400487b0 f   GameServerManagerDlg.obj
 0001:000477bc       ?dtor$1@?0??OnGameServerMsg@CGameServerManagerDlg@@IEAA_J_K_J@Z@4HA 00000001400487bc f   GameServerManagerDlg.obj
 0001:000477c8       ?dtor$2@?0??OnGameServerMsg@CGameServerManagerDlg@@IEAA_J_K_J@Z@4HA 00000001400487c8 f   GameServerManagerDlg.obj
 0001:000477d4       ?dtor$3@?0??OnGameServerMsg@CGameServerManagerDlg@@IEAA_J_K_J@Z@4HA 00000001400487d4 f   GameServerManagerDlg.obj
 0001:000477e0       ?dtor$4@?0??OnGameServerMsg@CGameServerManagerDlg@@IEAA_J_K_J@Z@4HA 00000001400487e0 f   GameServerManagerDlg.obj
 0001:000477ec       ?dtor$5@?0??OnGameServerMsg@CGameServerManagerDlg@@IEAA_J_K_J@Z@4HA 00000001400487ec f   GameServerManagerDlg.obj
 0001:00047800       ?dtor$0@?0??KillServerApp@CGameServerManagerDlg@@IEAAXI_N@Z@4HA 0000000140048800 f   GameServerManagerDlg.obj
 0001:00047810       ?dtor$0@?0??OnTimer@CGameServerManagerDlg@@IEAAX_K@Z@4HA 0000000140048810 f   GameServerManagerDlg.obj
 0001:0004781c       ?dtor$1@?0??OnTimer@CGameServerManagerDlg@@IEAAX_K@Z@4HA 000000014004881c f   GameServerManagerDlg.obj
 0001:00047828       ?dtor$2@?0??OnTimer@CGameServerManagerDlg@@IEAAX_K@Z@4HA 0000000140048828 f   GameServerManagerDlg.obj
 0001:00047834       ?dtor$3@?0??OnTimer@CGameServerManagerDlg@@IEAAX_K@Z@4HA 0000000140048834 f   GameServerManagerDlg.obj
 0001:00047840       ?dtor$0@?0??OnButtonGo@CGameServerManagerDlg@@IEAAXXZ@4HA 0000000140048840 f   GameServerManagerDlg.obj
 0001:00047850       ?dtor$0@?0??TerminateGameServer@CGameServerManagerDlg@@QEAAXF@Z@4HA 0000000140048850 f   GameServerManagerDlg.obj
 0001:0004785c       ?dtor$1@?0??TerminateGameServer@CGameServerManagerDlg@@QEAAXF@Z@4HA 000000014004885c f   GameServerManagerDlg.obj
 0001:00047868       ?dtor$2@?0??TerminateGameServer@CGameServerManagerDlg@@QEAAXF@Z@4HA 0000000140048868 f   GameServerManagerDlg.obj
 0001:00047880       ?dtor$0@?0??VerifyServerAppTermination@CGameServerManagerDlg@@AEAAXXZ@4HA 0000000140048880 f   GameServerManagerDlg.obj
 0001:0004788c       ?dtor$1@?0??VerifyServerAppTermination@CGameServerManagerDlg@@AEAAXXZ@4HA 000000014004888c f   GameServerManagerDlg.obj
 0001:00047898       ?dtor$2@?0??VerifyServerAppTermination@CGameServerManagerDlg@@AEAAXXZ@4HA 0000000140048898 f   GameServerManagerDlg.obj
 0001:000478a4       ?dtor$3@?0??VerifyServerAppTermination@CGameServerManagerDlg@@AEAAXXZ@4HA 00000001400488a4 f   GameServerManagerDlg.obj
 0001:000478b0       ?dtor$4@?0??VerifyServerAppTermination@CGameServerManagerDlg@@AEAAXXZ@4HA 00000001400488b0 f   GameServerManagerDlg.obj
 0001:000478c0       ?dtor$0@?0??StringSplitToNumArray@CGameServerManagerDlg@@AEAAXV?$basic_string@DU?$char_traits@D@std@@V?$allocator@D@2@@std@@0PEAHAEAH@Z@4HA 00000001400488c0 f   GameServerManagerDlg.obj
 0001:000478cc       ?dtor$1@?0??StringSplitToNumArray@CGameServerManagerDlg@@AEAAXV?$basic_string@DU?$char_traits@D@std@@V?$allocator@D@2@@std@@0PEAHAEAH@Z@4HA 00000001400488cc f   GameServerManagerDlg.obj
 0001:000478d8       ?dtor$2@?0??StringSplitToNumArray@CGameServerManagerDlg@@AEAAXV?$basic_string@DU?$char_traits@D@std@@V?$allocator@D@2@@std@@0PEAHAEAH@Z@4HA 00000001400488d8 f   GameServerManagerDlg.obj
 0001:00047910       ?dtor$0@?0??FindFreePorts@CGameServerManagerDlg@@AEAA_NXZ@4HA 0000000140048910 f   GameServerManagerDlg.obj
 0001:0004791c       ?dtor$2@?0??FindFreePorts@CGameServerManagerDlg@@AEAA_NXZ@4HA 000000014004891c f   GameServerManagerDlg.obj
 0001:00047930       ?dtor$0@?0??LoadWMszFile@FindXlsMsg@@QEAA_NPEAD@Z@4HA 0000000140048930 f   LoadXlsMsg.obj
 0001:00047930       ?dtor$0@?0??RestoreFreePort@CGameServerManagerDlg@@AEAAXXZ@4HA 0000000140048930 f   GameServerManagerDlg.obj
 0001:00047930       ?dtor$0@?0??AssignServerApp@CGameServerManagerDlg@@AEAAXAEBUPROTO_AUTOMATCH_GAME_START_REQ@@F@Z@4HA 0000000140048930 f   GameServerManagerDlg.obj
 0001:00047940       ?dtor$0@?0???0CSharedMemoryLoader@@QEAA@XZ@4HA 0000000140048940 f   GameServerManagerDlg.obj
 0001:00047950       ?dtor$1@?0???0CSharedMemoryLoader@@QEAA@XZ@4HA 0000000140048950 f   GameServerManagerDlg.obj
 0001:00047960       ?dtor$2@?0???0CSharedMemoryLoader@@QEAA@XZ@4HA 0000000140048960 f   GameServerManagerDlg.obj
 0001:00047970       ?dtor$8@?0???0CSharedMemoryLoader@@QEAA@XZ@4HA 0000000140048970 f   GameServerManagerDlg.obj
 0001:00047996       ?dtor$14@?0???0CSharedMemoryLoader@@QEAA@XZ@4HA 0000000140048996 f   GameServerManagerDlg.obj
 0001:000479c0       ?dtor$0@?0??_PreLoad@CSharedMemoryLoader@@AEAA_NXZ@4HA 00000001400489c0 f   GameServerManagerDlg.obj
 0001:000479cc       ?dtor$1@?0??_PreLoad@CSharedMemoryLoader@@AEAA_NXZ@4HA 00000001400489cc f   GameServerManagerDlg.obj
 0001:000479e0       ?dtor$0@?0??_Load@CSharedMemoryLoader@@AEAA_NXZ@4HA 00000001400489e0 f   GameServerManagerDlg.obj
 0001:000479ec       ?dtor$1@?0??_Load@CSharedMemoryLoader@@AEAA_NXZ@4HA 00000001400489ec f   GameServerManagerDlg.obj
 0001:000479f8       ?dtor$2@?0??_Load@CSharedMemoryLoader@@AEAA_NXZ@4HA 00000001400489f8 f   GameServerManagerDlg.obj
 0001:00047a06       ?dtor$3@?0??_Load@CSharedMemoryLoader@@AEAA_NXZ@4HA 0000000140048a06 f   GameServerManagerDlg.obj
 0001:00047a14       ?dtor$4@?0??_Load@CSharedMemoryLoader@@AEAA_NXZ@4HA 0000000140048a14 f   GameServerManagerDlg.obj
 0001:00047a22       ?dtor$5@?0??_Load@CSharedMemoryLoader@@AEAA_NXZ@4HA 0000000140048a22 f   GameServerManagerDlg.obj
 0001:00047a30       ?dtor$6@?0??_Load@CSharedMemoryLoader@@AEAA_NXZ@4HA 0000000140048a30 f   GameServerManagerDlg.obj
 0001:00047a3e       ?dtor$7@?0??_Load@CSharedMemoryLoader@@AEAA_NXZ@4HA 0000000140048a3e f   GameServerManagerDlg.obj
 0001:00047a4a       ?dtor$8@?0??_Load@CSharedMemoryLoader@@AEAA_NXZ@4HA 0000000140048a4a f   GameServerManagerDlg.obj
 0001:00047a60       ?dtor$0@?0??Load@CSharedMemoryLoader@@QEAA_NXZ@4HA 0000000140048a60 f   GameServerManagerDlg.obj
 0001:00047a6c       ?dtor$1@?0??Load@CSharedMemoryLoader@@QEAA_NXZ@4HA 0000000140048a6c f   GameServerManagerDlg.obj
 0001:00047a80       ?dtor$0@?0??RECV_MSG_GAMEEND@CGameServerManagerDlg@@AEAAXFPEBUGAMEPROTO_SS_GAMEEND@@@Z@4HA 0000000140048a80 f   GameServerManagerDlg.obj
 0001:00047a90       ?dtor$0@?0??Send@CGMSConnManager@@AEAAHPEAVCPacket@@@Z@4HA 0000000140048a90 f   GMSConnManager.obj
 0001:00047a90       ?dtor$0@?0??RECV_MSG_AI_EXTRA_REWARD@CGameServerManagerDlg@@AEAAXFPEAUPROTO_AI_EXTRA_REWARD_REQ@@@Z@4HA 0000000140048a90 f   GameServerManagerDlg.obj
 0001:00047aa0       ?dtor$0@?0??OnReceiveFromGms@CGameServerManagerDlg@@AEAAXAEBUPROTO_STARTING_GAME_tag@@@Z@4HA 0000000140048aa0 f   GameServerManagerDlg.obj
 0001:00047aa0       ?dtor$0@?0??OnReceiveFromGms@CGameServerManagerDlg@@AEAAXAEBUPROTO_AUTOMATCH_GAME_START_REQ@@@Z@4HA 0000000140048aa0 f   GameServerManagerDlg.obj
 0001:00047aac       ?dtor$1@?0??OnReceiveFromGms@CGameServerManagerDlg@@AEAAXAEBUPROTO_AUTOMATCH_GAME_START_REQ@@@Z@4HA 0000000140048aac f   GameServerManagerDlg.obj
 0001:00047aac       ?dtor$1@?0??OnReceiveFromGms@CGameServerManagerDlg@@AEAAXAEBUPROTO_STARTING_GAME_tag@@@Z@4HA 0000000140048aac f   GameServerManagerDlg.obj
 0001:00047ac9       ?dtor$2@?0??OnReceiveFromGms@CGameServerManagerDlg@@AEAAXAEBUPROTO_STARTING_GAME_tag@@@Z@4HA 0000000140048ac9 f   GameServerManagerDlg.obj
 0001:00047ac9       ?dtor$2@?0??OnReceiveFromGms@CGameServerManagerDlg@@AEAAXAEBUPROTO_AUTOMATCH_GAME_START_REQ@@@Z@4HA 0000000140048ac9 f   GameServerManagerDlg.obj
 0001:00047ae0       ?dtor$0@?0??OnReceiveFromGms@CGameServerManagerDlg@@AEAAXAEBUPROTO_INSERT_CHARACTER_tag@@@Z@4HA 0000000140048ae0 f   GameServerManagerDlg.obj
 0001:00047aec       ?dtor$1@?0??OnReceiveFromGms@CGameServerManagerDlg@@AEAAXAEBUPROTO_INSERT_CHARACTER_tag@@@Z@4HA 0000000140048aec f   GameServerManagerDlg.obj
 0001:00047b00       ?dtor$0@?0??OnReceiveFromGms@CGameServerManagerDlg@@AEAAXAEBUPROTO_MMSERVER_TERMINATED_tag@@@Z@4HA 0000000140048b00 f   GameServerManagerDlg.obj
 0001:00047b10       ?dtor$0@?0??OnReceiveFromGms@CGameServerManagerDlg@@AEAAXAEBUPROTO_AUTOMATCH_GAME_ENTER_REQ@@@Z@4HA 0000000140048b10 f   GameServerManagerDlg.obj
 0001:00047b1c       ?dtor$1@?0??OnReceiveFromGms@CGameServerManagerDlg@@AEAAXAEBUPROTO_AUTOMATCH_GAME_ENTER_REQ@@@Z@4HA 0000000140048b1c f   GameServerManagerDlg.obj
 0001:00047b39       ?dtor$2@?0??OnReceiveFromGms@CGameServerManagerDlg@@AEAAXAEBUPROTO_AUTOMATCH_GAME_ENTER_REQ@@@Z@4HA 0000000140048b39 f   GameServerManagerDlg.obj
 0001:00047b50       ?dtor$0@?0??AssignServerApp@CGameServerManagerDlg@@AEAAXAEBUPROTO_STARTING_GAME_tag@@F@Z@4HA 0000000140048b50 f   GameServerManagerDlg.obj
 0001:00047b60       ?catch$1@?0???$_Setp@UGAMESERVERINFO@@@?$shared_ptr@UGAMESERVERINFO@@@std@@AEAAXPEAUGAMESERVERINFO@@U?$integral_constant@_N$0A@@1@@Z@4HA 0000000140048b60 f   GameServerManagerDlg.obj
 0001:00047b6d       __catch$??$_Setp@UGAMESERVERINFO@@@?$shared_ptr@UGAMESERVERINFO@@@std@@AEAAXPEAUGAMESERVERINFO@@U?$integral_constant@_N$0A@@1@@Z$0 0000000140048b6d f   GameServerManagerDlg.obj
 0001:00047b90       ?catch$0@?0???$_Insert_nohint@AEAU?$pair@$$CBIUPORTINFO@@@std@@PEAU?$_Tree_node@U?$pair@$$CBIUPORTINFO@@@std@@PEAX@2@@?$_Tree@V?$_Tmap_traits@IUPORTINFO@@U?$less@I@std@@V?$allocator@U?$pair@$$CBIUPORTINFO@@@std@@@3@$0A@@std@@@std@@IEAA?AU?$pair@V?$_Tree_iterator@V?$_Tree_val@U?$_Tree_simple_types@U?$pair@$$CBIUPORTINFO@@@std@@@std@@@std@@@std@@_N@1@_NAEAU?$pair@$$CBIUPORTINFO@@@1@PEAU?$_Tree_node@U?$pair@$$CBIUPORTINFO@@@std@@PEAX@1@@Z@4HA 0000000140048b90 f   GameServerManagerDlg.obj
 0001:00047b9d       __catch$??$_Insert_nohint@AEAU?$pair@$$CBIUPORTINFO@@@std@@PEAU?$_Tree_node@U?$pair@$$CBIUPORTINFO@@@std@@PEAX@2@@?$_Tree@V?$_Tmap_traits@IUPORTINFO@@U?$less@I@std@@V?$allocator@U?$pair@$$CBIUPORTINFO@@@std@@@3@$0A@@std@@@std@@IEAA?AU?$pair@V?$_Tree_iterator@V?$_Tree_val@U?$_Tree_simple_types@U?$pair@$$CBIUPORTINFO@@@std@@@std@@@std@@@std@@_N@1@_NAEAU?$pair@$$CBIUPORTINFO@@@1@PEAU?$_Tree_node@U?$pair@$$CBIUPORTINFO@@@std@@PEAX@1@@Z$0 0000000140048b9d f   GameServerManagerDlg.obj
 0001:00047bb0       ?catch$0@?0???$_Insert_hint@AEAU?$pair@$$CBIUPORTINFO@@@std@@PEAU?$_Tree_node@U?$pair@$$CBIUPORTINFO@@@std@@PEAX@2@@?$_Tree@V?$_Tmap_traits@IUPORTINFO@@U?$less@I@std@@V?$allocator@U?$pair@$$CBIUPORTINFO@@@std@@@3@$0A@@std@@@std@@IEAA?AV?$_Tree_iterator@V?$_Tree_val@U?$_Tree_simple_types@U?$pair@$$CBIUPORTINFO@@@std@@@std@@@std@@@1@V?$_Tree_const_iterator@V?$_Tree_val@U?$_Tree_simple_types@U?$pair@$$CBIUPORTINFO@@@std@@@std@@@std@@@1@AEAU?$pair@$$CBIUPORTINFO@@@1@PEAU?$_Tree_node@U?$pair@$$CBIUPORTINFO@@@std@@PEAX@1@@Z@4HA 0000000140048bb0 f   GameServerManagerDlg.obj
 0001:00047bbd       __catch$??$_Insert_hint@AEAU?$pair@$$CBIUPORTINFO@@@std@@PEAU?$_Tree_node@U?$pair@$$CBIUPORTINFO@@@std@@PEAX@2@@?$_Tree@V?$_Tmap_traits@IUPORTINFO@@U?$less@I@std@@V?$allocator@U?$pair@$$CBIUPORTINFO@@@std@@@3@$0A@@std@@@std@@IEAA?AV?$_Tree_iterator@V?$_Tree_val@U?$_Tree_simple_types@U?$pair@$$CBIUPORTINFO@@@std@@@std@@@std@@@1@V?$_Tree_const_iterator@V?$_Tree_val@U?$_Tree_simple_types@U?$pair@$$CBIUPORTINFO@@@std@@@std@@@std@@@1@AEAU?$pair@$$CBIUPORTINFO@@@1@PEAU?$_Tree_node@U?$pair@$$CBIUPORTINFO@@@std@@PEAX@1@@Z$0 0000000140048bbd f   GameServerManagerDlg.obj
 0001:00047be0       ?dtor$0@?0??RTIDUSNtoString@EXPAND_USN@@YA?AV?$basic_string@DU?$char_traits@D@std@@V?$allocator@D@2@@std@@HFF_J@Z@4HA 0000000140048be0 f   GameServerManagerDlg.obj
 0001:00047bf0       ?dtor$1@?0??init@SGGMProxyLoader@sggm_proxy@@QEAA_NPEAVMultiReceiver@2@@Z@4HA 0000000140048bf0 f   GameServerManagerDlg.obj
 0001:00047c20       ?dtor$0@?0??SendTeamDeathMatchKillCnt@CGMSConnManager@@QEAAHPEBUPROTO_GAMEGT_TEAM_DEATH_KILL_CNT_NTY@@@Z@4HA 0000000140048c20 f   GMSConnManager.obj
 0001:00047c20       ?dtor$0@?0??SendSpyChange@CGMSConnManager@@QEAAHPEAUPROTO_GAMEGT_SPY_CHANGE_NTY_tag@@@Z@4HA 0000000140048c20 f   GMSConnManager.obj
 0001:00047c20       ?dtor$0@?0??InsertCharacterResult@CGMSConnManager@@QEAAHUPROTO_INSERT_CHARACTER_RESULT_tag@@@Z@4HA 0000000140048c20 f   GMSConnManager.obj
 0001:00047c20       ?dtor$0@?0??SendPrevGameFinishNotify@CGMSConnManager@@QEAAHPEAUPROTO_FINISHED_GAME_PREV_tag@@@Z@4HA 0000000140048c20 f   GMSConnManager.obj
 0001:00047c20       ?dtor$0@?0??StartingGameResult@CGMSConnManager@@QEAAHUPROTO_STARTING_GAME_RESULT_tag@@W4START_HOST_RESULT@@@Z@4HA 0000000140048c20 f   GMSConnManager.obj
 0001:00047c20       ?dtor$0@?0??UpdateCharacterStat@CGMSConnManager@@QEAAHUPROTO_UPDATE_CHARACTER_STAT_tag@@@Z@4HA 0000000140048c20 f   GMSConnManager.obj
 0001:00047c20       ?dtor$0@?0??SendAI3BonusClearItemReq@CGMSConnManager@@QEAAHPEAUPROTO_GAMEGT_INGAME_AI3_BONUS_REWARD_ITEM_REQ@@@Z@4HA 0000000140048c20 f   GMSConnManager.obj
 0001:00047c20       ?dtor$0@?0??SendAIExtraMiddleRewardReq@CGMSConnManager@@QEAAHPEAUPROTO_AI_EXTRA_MIDDLE_REWARD_REQ@@@Z@4HA 0000000140048c20 f   GMSConnManager.obj
 0001:00047c20       ?dtor$0@?0??SendAIExtraRewardReq@CGMSConnManager@@QEAAHPEAUPROTO_AI_EXTRA_REWARD_REQ@@@Z@4HA 0000000140048c20 f   GMSConnManager.obj
 0001:00047c20       ?dtor$0@?0??SendRoundChange@CGMSConnManager@@QEAAHPEBUPROTO_GAMEGT_ROUND_CHANGE_NTY_tag@@@Z@4HA 0000000140048c20 f   GMSConnManager.obj
 0001:00047c20       ?dtor$0@?0??SendAIItemInsert@CGMSConnManager@@QEAAHPEAUPROTO_GAMEGT_INGAME_AIGACHA_ITEM_INSERT@@@Z@4HA 0000000140048c20 f   GMSConnManager.obj
 0001:00047c20       ?dtor$0@?0??SendAutoMatchIngameEnterNty@CGMSConnManager@@QEAAHAEBUPROTO_AUTOMATCH_INGAME_ENTER_NTY@@@Z@4HA 0000000140048c20 f   GMSConnManager.obj
 0001:00047c20       ?dtor$0@?0??SendKickUserInfo@CGMSConnManager@@QEAAHPEAUPROTO_GAMEMGT_KICK_USER@@@Z@4HA 0000000140048c20 f   GMSConnManager.obj
 0001:00047c20       ?dtor$0@?0??SendAutoMatchGameEnterRes@CGMSConnManager@@QEAAHAEBUPROTO_AUTOMATCH_GAME_ENTER_RES@@@Z@4HA 0000000140048c20 f   GMSConnManager.obj
 0001:00047c20       ?dtor$0@?0??SendIntrusionCoinDec@CGMSConnManager@@QEAAHPEAUPROTO_GAMEGT_MAPLOADING_COMPLETE_NTY_tag@@@Z@4HA 0000000140048c20 f   GMSConnManager.obj
 0001:00047c20       ?dtor$0@?0??SendIngameRewardReq@CGMSConnManager@@QEAAHPEAUPROTO_INGAME_RESULT_REQ@@@Z@4HA 0000000140048c20 f   GMSConnManager.obj
 0001:00047c20       ?dtor$0@?0??SendAutoMatchGameStartRes@CGMSConnManager@@QEAAHAEBUPROTO_AUTOMATCH_GAME_START_RES@@W4START_HOST_RESULT@@@Z@4HA 0000000140048c20 f   GMSConnManager.obj
 0001:00047c20       ?dtor$0@?0??SendGameStart@CGMSConnManager@@QEAAHPEBUPROTO_GAMEGT_GAME_START_NTY@@@Z@4HA 0000000140048c20 f   GMSConnManager.obj
 0001:00047c20       ?dtor$0@?0??SendSpectatorRecommendRoomData@CGMSConnManager@@QEAAHPEAUPROTO_SPECTATOR_RECOMMEND_ROOM_INGAME_DATA_NTY@@@Z@4HA 0000000140048c20 f   GMSConnManager.obj
 0001:00047c20       ?dtor$0@?0??SendAutoSideChangeTeamInfoNotify@CGMSConnManager@@QEAAHPEAUPROTO_GAMEGT_AUTO_SIDE_CHANGE_TEAM_INFO_NTY@@@Z@4HA 0000000140048c20 f   GMSConnManager.obj
 0001:00047c20       ?dtor$0@?0??SendBattleShipBonusCoinReq@CGMSConnManager@@QEAAHPEAUPROTOCOL_AI2_BONUSROUND_REWARD_REQ_tag@@@Z@4HA 0000000140048c20 f   GMSConnManager.obj
 0001:00047c20       ?dtor$0@?0??SendBossTowerRewardReq@CGMSConnManager@@QEAAHPEAUPROTO_AI_BOSS_TOWER_REWARD_REQ@@@Z@4HA 0000000140048c20 f   GMSConnManager.obj
 0001:00047c20       ?dtor$0@?0??SendFarmingItemReq@CGMSConnManager@@QEAAHPEAUPROTO_GAMEGT_INGAME_FARMING_ITEM_REQ@@@Z@4HA 0000000140048c20 f   GMSConnManager.obj
 0001:00047c20       ?dtor$0@?0??SendForceLeavePollResult@CGMSConnManager@@QEAAHPEBUPROTO_BAN_USER_tag@@@Z@4HA 0000000140048c20 f   GMSConnManager.obj
 0001:00047c30       ?dtor$0@?0??NotifyAllocableRoomCountChanged@CGMSConnManager@@QEAAHJHHHHHQEAHHH@Z@4HA 0000000140048c30 f   GMSConnManager.obj
 0001:00047c40       ?dtor$0@?0???$?HDU?$char_traits@D@std@@V?$allocator@D@1@@std@@YA?AV?$basic_string@DU?$char_traits@D@std@@V?$allocator@D@2@@0@QEBDAEBV10@@Z@4HA 0000000140048c40 f   CSmtp.obj
 0001:00047c70       ?dtor$1@?0???$?6U?$char_traits@D@std@@@std@@YAAEAV?$basic_ostream@DU?$char_traits@D@std@@@0@AEAV10@PEBD@Z@4HA 0000000140048c70 f   md5_csmtp.obj
 0001:00047c7c       ?dtor$0@?0???$?6U?$char_traits@D@std@@@std@@YAAEAV?$basic_ostream@DU?$char_traits@D@std@@@0@AEAV10@PEBD@Z@4HA 0000000140048c7c f   md5_csmtp.obj
 0001:00047c88       ?catch$4@?0???$?6U?$char_traits@D@std@@@std@@YAAEAV?$basic_ostream@DU?$char_traits@D@std@@@0@AEAV10@PEBD@Z@4HA 0000000140048c88 f   md5_csmtp.obj
 0001:00047c95       __catch$??$?6U?$char_traits@D@std@@@std@@YAAEAV?$basic_ostream@DU?$char_traits@D@std@@@0@AEAV10@PEBD@Z$0 0000000140048c95 f   md5_csmtp.obj
 0001:00047cc0       ?dtor$0@?0???__Eg_HostStat@@YAXXZ@4HA 0000000140048cc0 f   HostStat.obj
 0001:00047cd0       ?dtor$1@?0???__Eg_HostStat@@YAXXZ@4HA 0000000140048cd0 f   HostStat.obj
 0001:00047cf0       ?dtor$0@?0??setup@CHostStat@@QEAAXHH@Z@4HA 0000000140048cf0 f   HostStat.obj
 0001:00047cfc       ?dtor$2@?0??setup@CHostStat@@QEAAXHH@Z@4HA 0000000140048cfc f   HostStat.obj
 0001:00047d10       ?dtor$0@?0??thdMail@CHostStat@@KAIPEAX@Z@4HA 0000000140048d10 f   HostStat.obj
 0001:00047d1c       ?dtor$1@?0??thdMail@CHostStat@@KAIPEAX@Z@4HA 0000000140048d1c f   HostStat.obj
 0001:00047d28       ?dtor$2@?0??thdMail@CHostStat@@KAIPEAX@Z@4HA 0000000140048d28 f   HostStat.obj
 0001:00047d34       ?dtor$3@?0??thdMail@CHostStat@@KAIPEAX@Z@4HA 0000000140048d34 f   HostStat.obj
 0001:00047d40       ?dtor$4@?0??thdMail@CHostStat@@KAIPEAX@Z@4HA 0000000140048d40 f   HostStat.obj
 0001:00047d4c       ?dtor$5@?0??thdMail@CHostStat@@KAIPEAX@Z@4HA 0000000140048d4c f   HostStat.obj
 0001:00047d58       ?dtor$6@?0??thdMail@CHostStat@@KAIPEAX@Z@4HA 0000000140048d58 f   HostStat.obj
 0001:00047d64       ?dtor$7@?0??thdMail@CHostStat@@KAIPEAX@Z@4HA 0000000140048d64 f   HostStat.obj
 0001:00047d70       ?dtor$8@?0??thdMail@CHostStat@@KAIPEAX@Z@4HA 0000000140048d70 f   HostStat.obj
 0001:00047d80       ?dtor$0@?0??timer@CHostStat@@QEAAXXZ@4HA 0000000140048d80 f   HostStat.obj
 0001:00047d8c       ?dtor$1@?0??timer@CHostStat@@QEAAXXZ@4HA 0000000140048d8c f   HostStat.obj
 0001:00047d98       ?dtor$2@?0??timer@CHostStat@@QEAAXXZ@4HA 0000000140048d98 f   HostStat.obj
 0001:00047da4       ?dtor$3@?0??timer@CHostStat@@QEAAXXZ@4HA 0000000140048da4 f   HostStat.obj
 0001:00047db0       ?dtor$0@?0??addData@CHostStat@@QEAAXGEEG@Z@4HA 0000000140048db0 f   HostStat.obj
 0001:00047db0       ?dtor$0@?0??setData64@CHostStat@@QEAAXGEEG_J@Z@4HA 0000000140048db0 f   HostStat.obj
 0001:00047db0       ?dtor$0@?0??getData64@CHostStat@@QEAA_JGEEG@Z@4HA 0000000140048db0 f   HostStat.obj
 0001:00047db0       ?dtor$0@?0??addExtraData@CHostStat@@QEAAXGE@Z@4HA 0000000140048db0 f   HostStat.obj
 0001:00047db0       ?dtor$0@?0??addExtraData@CHostStat@@QEAAXGEEGIII@Z@4HA 0000000140048db0 f   HostStat.obj
 0001:00047dc0       ?dtor$0@?0??send@CHostStat@@IEAA_NPEAD0@Z@4HA 0000000140048dc0 f   HostStat.obj
 0001:00047dcc       ?dtor$1@?0??send@CHostStat@@IEAA_NPEAD0@Z@4HA 0000000140048dcc f   HostStat.obj
 0001:00047dd8       ?dtor$2@?0??send@CHostStat@@IEAA_NPEAD0@Z@4HA 0000000140048dd8 f   HostStat.obj
 0001:00047de4       ?dtor$3@?0??send@CHostStat@@IEAA_NPEAD0@Z@4HA 0000000140048de4 f   HostStat.obj
 0001:00047df0       ?dtor$4@?0??send@CHostStat@@IEAA_NPEAD0@Z@4HA 0000000140048df0 f   HostStat.obj
 0001:00047dfc       ?dtor$5@?0??send@CHostStat@@IEAA_NPEAD0@Z@4HA 0000000140048dfc f   HostStat.obj
 0001:00047e08       ?dtor$6@?0??send@CHostStat@@IEAA_NPEAD0@Z@4HA 0000000140048e08 f   HostStat.obj
 0001:00047e14       ?dtor$7@?0??send@CHostStat@@IEAA_NPEAD0@Z@4HA 0000000140048e14 f   HostStat.obj
 0001:00047e20       ?dtor$8@?0??send@CHostStat@@IEAA_NPEAD0@Z@4HA 0000000140048e20 f   HostStat.obj
 0001:00047e2c       ?dtor$9@?0??send@CHostStat@@IEAA_NPEAD0@Z@4HA 0000000140048e2c f   HostStat.obj
 0001:00047e40       ?dtor$0@?0??GatherFiles@CHostStat@@QEAAXPEAD@Z@4HA 0000000140048e40 f   HostStat.obj
 0001:00047e50       ?catch$0@?0???$_Insert_nohint@AEAU?$pair@$$CBGUExtraStatsFPSVerify@CHostStat@@@std@@PEAU?$_Tree_node@U?$pair@$$CBGUExtraStatsFPSVerify@CHostStat@@@std@@PEAX@2@@?$_Tree@V?$_Tmap_traits@GUExtraStatsFPSVerify@CHostStat@@U?$less@G@std@@V?$allocator@U?$pair@$$CBGUExtraStatsFPSVerify@CHostStat@@@std@@@4@$0A@@std@@@std@@IEAA?AU?$pair@V?$_Tree_iterator@V?$_Tree_val@U?$_Tree_simple_types@U?$pair@$$CBGUExtraStatsFPSVerify@CHostStat@@@std@@@std@@@std@@@std@@_N@1@_NAEAU?$pair@$$CBGUExtraStatsFPSVerify@CHostStat@@@1@PEAU?$_Tree_node@U?$pair@$$CBGUExtraStatsFPSVerify@CHostStat@@@std@@PEAX@1@@Z@4HA 0000000140048e50 f   HostStat.obj
 0001:00047e50       ?catch$0@?0???$_Insert_nohint@AEAU?$pair@$$CBGUExtraStatsMemVerify@CHostStat@@@std@@PEAU?$_Tree_node@U?$pair@$$CBGUExtraStatsMemVerify@CHostStat@@@std@@PEAX@2@@?$_Tree@V?$_Tmap_traits@GUExtraStatsMemVerify@CHostStat@@U?$less@G@std@@V?$allocator@U?$pair@$$CBGUExtraStatsMemVerify@CHostStat@@@std@@@4@$0A@@std@@@std@@IEAA?AU?$pair@V?$_Tree_iterator@V?$_Tree_val@U?$_Tree_simple_types@U?$pair@$$CBGUExtraStatsMemVerify@CHostStat@@@std@@@std@@@std@@@std@@_N@1@_NAEAU?$pair@$$CBGUExtraStatsMemVerify@CHostStat@@@1@PEAU?$_Tree_node@U?$pair@$$CBGUExtraStatsMemVerify@CHostStat@@@std@@PEAX@1@@Z@4HA 0000000140048e50 f   HostStat.obj
 0001:00047e5d       __catch$??$_Insert_nohint@AEAU?$pair@$$CBGUExtraStatsMemVerify@CHostStat@@@std@@PEAU?$_Tree_node@U?$pair@$$CBGUExtraStatsMemVerify@CHostStat@@@std@@PEAX@2@@?$_Tree@V?$_Tmap_traits@GUExtraStatsMemVerify@CHostStat@@U?$less@G@std@@V?$allocator@U?$pair@$$CBGUExtraStatsMemVerify@CHostStat@@@std@@@4@$0A@@std@@@std@@IEAA?AU?$pair@V?$_Tree_iterator@V?$_Tree_val@U?$_Tree_simple_types@U?$pair@$$CBGUExtraStatsMemVerify@CHostStat@@@std@@@std@@@std@@@std@@_N@1@_NAEAU?$pair@$$CBGUExtraStatsMemVerify@CHostStat@@@1@PEAU?$_Tree_node@U?$pair@$$CBGUExtraStatsMemVerify@CHostStat@@@std@@PEAX@1@@Z$0 0000000140048e5d f   HostStat.obj
 0001:00047e5d       __catch$??$_Insert_nohint@AEAU?$pair@$$CBGUExtraStatsFPSVerify@CHostStat@@@std@@PEAU?$_Tree_node@U?$pair@$$CBGUExtraStatsFPSVerify@CHostStat@@@std@@PEAX@2@@?$_Tree@V?$_Tmap_traits@GUExtraStatsFPSVerify@CHostStat@@U?$less@G@std@@V?$allocator@U?$pair@$$CBGUExtraStatsFPSVerify@CHostStat@@@std@@@4@$0A@@std@@@std@@IEAA?AU?$pair@V?$_Tree_iterator@V?$_Tree_val@U?$_Tree_simple_types@U?$pair@$$CBGUExtraStatsFPSVerify@CHostStat@@@std@@@std@@@std@@@std@@_N@1@_NAEAU?$pair@$$CBGUExtraStatsFPSVerify@CHostStat@@@1@PEAU?$_Tree_node@U?$pair@$$CBGUExtraStatsFPSVerify@CHostStat@@@std@@PEAX@1@@Z$0 0000000140048e5d f   HostStat.obj
 0001:00047e70       ?dtor$3@?0??write@CIniSection@CIniReader@@QEAAKPEAX@Z@4HA 0000000140048e70 f   iniReader.obj
 0001:00047e99       ?dtor$1@?0??write@CIniSection@CIniReader@@QEAAKPEAX@Z@4HA 0000000140048e99 f   iniReader.obj
 0001:00047eb0       ?dtor$0@?0??setString@CIniSection@CIniReader@@QEAAXPEBD0@Z@4HA 0000000140048eb0 f   iniReader.obj
 0001:00047ebc       ?dtor$1@?0??setString@CIniSection@CIniReader@@QEAAXPEBD0@Z@4HA 0000000140048ebc f   iniReader.obj
 0001:00047ed0       ?dtor$3@?0??write@CIniReader@@QEAAKPEBD@Z@4HA 0000000140048ed0 f   iniReader.obj
 0001:00047ef6       ?dtor$1@?0??write@CIniReader@@QEAAKPEBD@Z@4HA 0000000140048ef6 f   iniReader.obj
 0001:00047f02       ?dtor$2@?0??write@CIniReader@@QEAAKPEBD@Z@4HA 0000000140048f02 f   iniReader.obj
 0001:00047f10       ?dtor$1@?0??setString@CIniReader@@QEAAXPEBD00@Z@4HA 0000000140048f10 f   iniReader.obj
 0001:00047f30       ?catch$1@?0???$_Buynode@U?$pair@PEADPEAVCIniSection@CIniReader@@@std@@@?$_Tree_comp_alloc@V?$_Tmap_traits@V?$basic_string@DU?$char_traits@D@std@@V?$allocator@D@2@@std@@PEAVCIniSection@CIniReader@@U?$less@V?$basic_string@DU?$char_traits@D@std@@V?$allocator@D@2@@std@@@2@V?$allocator@U?$pair@$$CBV?$basic_string@DU?$char_traits@D@std@@V?$allocator@D@2@@std@@PEAVCIniSection@CIniReader@@@std@@@2@$0A@@std@@@std@@QEAAPEAU?$_Tree_node@U?$pair@$$CBV?$basic_string@DU?$char_traits@D@std@@V?$allocator@D@2@@std@@PEAVCIniSection@CIniReader@@@std@@PEAX@1@$$QEAU?$pair@PEADPEAVCIniSection@CIniReader@@@1@@Z@4HA 0000000140048f30 f   iniReader.obj
 0001:00047f3d       __catch$??$_Buynode@U?$pair@PEADPEAVCIniSection@CIniReader@@@std@@@?$_Tree_comp_alloc@V?$_Tmap_traits@V?$basic_string@DU?$char_traits@D@std@@V?$allocator@D@2@@std@@PEAVCIniSection@CIniReader@@U?$less@V?$basic_string@DU?$char_traits@D@std@@V?$allocator@D@2@@std@@@2@V?$allocator@U?$pair@$$CBV?$basic_string@DU?$char_traits@D@std@@V?$allocator@D@2@@std@@PEAVCIniSection@CIniReader@@@std@@@2@$0A@@std@@@std@@QEAAPEAU?$_Tree_node@U?$pair@$$CBV?$basic_string@DU?$char_traits@D@std@@V?$allocator@D@2@@std@@PEAVCIniSection@CIniReader@@@std@@PEAX@1@$$QEAU?$pair@PEADPEAVCIniSection@CIniReader@@@1@@Z$0 0000000140048f3d f   iniReader.obj
 0001:00047f50       ?catch$0@?0???$_Insert_nohint@AEAU?$pair@$$CBV?$basic_string@DU?$char_traits@D@std@@V?$allocator@D@2@@std@@PEAVCIniSection@CIniReader@@@std@@PEAU?$_Tree_node@U?$pair@$$CBV?$basic_string@DU?$char_traits@D@std@@V?$allocator@D@2@@std@@PEAVCIniSection@CIniReader@@@std@@PEAX@2@@?$_Tree@V?$_Tmap_traits@V?$basic_string@DU?$char_traits@D@std@@V?$allocator@D@2@@std@@PEAVCIniSection@CIniReader@@U?$less@V?$basic_string@DU?$char_traits@D@std@@V?$allocator@D@2@@std@@@2@V?$allocator@U?$pair@$$CBV?$basic_string@DU?$char_traits@D@std@@V?$allocator@D@2@@std@@PEAVCIniSection@CIniReader@@@std@@@2@$0A@@std@@@std@@IEAA?AU?$pair@V?$_Tree_iterator@V?$_Tree_val@U?$_Tree_simple_types@U?$pair@$$CBV?$basic_string@DU?$char_traits@D@std@@V?$allocator@D@2@@std@@PEAVCIniSection@CIniReader@@@std@@@std@@@std@@@std@@_N@1@_NAEAU?$pair@$$CBV?$basic_string@DU?$char_traits@D@std@@V?$allocator@D@2@@std@@PEAVCIniSection@CIniReader@@@1@PEAU?$_Tree_node@U?$pair@$$CBV?$basic_string@DU?$char_traits@D@std@@V?$allocator@D@2@@std@@PEAVCIniSection@CIniReader@@@std@@PEAX@1@@Z@4HA 0000000140048f50 f   iniReader.obj
 0001:00047f5d       __catch$??$_Insert_nohint@AEAU?$pair@$$CBV?$basic_string@DU?$char_traits@D@std@@V?$allocator@D@2@@std@@PEAVCIniSection@CIniReader@@@std@@PEAU?$_Tree_node@U?$pair@$$CBV?$basic_string@DU?$char_traits@D@std@@V?$allocator@D@2@@std@@PEAVCIniSection@CIniReader@@@std@@PEAX@2@@?$_Tree@V?$_Tmap_traits@V?$basic_string@DU?$char_traits@D@std@@V?$allocator@D@2@@std@@PEAVCIniSection@CIniReader@@U?$less@V?$basic_string@DU?$char_traits@D@std@@V?$allocator@D@2@@std@@@2@V?$allocator@U?$pair@$$CBV?$basic_string@DU?$char_traits@D@std@@V?$allocator@D@2@@std@@PEAVCIniSection@CIniReader@@@std@@@2@$0A@@std@@@std@@IEAA?AU?$pair@V?$_Tree_iterator@V?$_Tree_val@U?$_Tree_simple_types@U?$pair@$$CBV?$basic_string@DU?$char_traits@D@std@@V?$allocator@D@2@@std@@PEAVCIniSection@CIniReader@@@std@@@std@@@std@@@std@@_N@1@_NAEAU?$pair@$$CBV?$basic_string@DU?$char_traits@D@std@@V?$allocator@D@2@@std@@PEAVCIniSection@CIniReader@@@1@PEAU?$_Tree_node@U?$pair@$$CBV?$basic_string@DU?$char_traits@D@std@@V?$allocator@D@2@@std@@PEAVCIniSection@CIniReader@@@std@@PEAX@1@@Z$0 0000000140048f5d f   iniReader.obj
 0001:00047f80       ?catch$0@?0???$_Insert_hint@AEAU?$pair@$$CBV?$basic_string@DU?$char_traits@D@std@@V?$allocator@D@2@@std@@V12@@std@@PEAU?$_Tree_node@U?$pair@$$CBV?$basic_string@DU?$char_traits@D@std@@V?$allocator@D@2@@std@@V12@@std@@PEAX@2@@?$_Tree@V?$_Tmap_traits@V?$basic_string@DU?$char_traits@D@std@@V?$allocator@D@2@@std@@V12@U?$less@V?$basic_string@DU?$char_traits@D@std@@V?$allocator@D@2@@std@@@2@V?$allocator@U?$pair@$$CBV?$basic_string@DU?$char_traits@D@std@@V?$allocator@D@2@@std@@V12@@std@@@2@$0A@@std@@@std@@IEAA?AV?$_Tree_iterator@V?$_Tree_val@U?$_Tree_simple_types@U?$pair@$$CBV?$basic_string@DU?$char_traits@D@std@@V?$allocator@D@2@@std@@V12@@std@@@std@@@std@@@1@V?$_Tree_const_iterator@V?$_Tree_val@U?$_Tree_simple_types@U?$pair@$$CBV?$basic_string@DU?$char_traits@D@std@@V?$allocator@D@2@@std@@V12@@std@@@std@@@std@@@1@AEAU?$pair@$$CBV?$basic_string@DU?$char_traits@D@std@@V?$allocator@D@2@@std@@V12@@1@PEAU?$_Tree_node@U?$pair@$$CBV?$basic_string@DU?$char_traits@D@std@@V?$allocator@D@2@@std@@V12@@std@@PEAX@1@@Z@4HA 0000000140048f80 f   iniReader.obj
 0001:00047f8d       __catch$??$_Insert_hint@AEAU?$pair@$$CBV?$basic_string@DU?$char_traits@D@std@@V?$allocator@D@2@@std@@V12@@std@@PEAU?$_Tree_node@U?$pair@$$CBV?$basic_string@DU?$char_traits@D@std@@V?$allocator@D@2@@std@@V12@@std@@PEAX@2@@?$_Tree@V?$_Tmap_traits@V?$basic_string@DU?$char_traits@D@std@@V?$allocator@D@2@@std@@V12@U?$less@V?$basic_string@DU?$char_traits@D@std@@V?$allocator@D@2@@std@@@2@V?$allocator@U?$pair@$$CBV?$basic_string@DU?$char_traits@D@std@@V?$allocator@D@2@@std@@V12@@std@@@2@$0A@@std@@@std@@IEAA?AV?$_Tree_iterator@V?$_Tree_val@U?$_Tree_simple_types@U?$pair@$$CBV?$basic_string@DU?$char_traits@D@std@@V?$allocator@D@2@@std@@V12@@std@@@std@@@std@@@1@V?$_Tree_const_iterator@V?$_Tree_val@U?$_Tree_simple_types@U?$pair@$$CBV?$basic_string@DU?$char_traits@D@std@@V?$allocator@D@2@@std@@V12@@std@@@std@@@std@@@1@AEAU?$pair@$$CBV?$basic_string@DU?$char_traits@D@std@@V?$allocator@D@2@@std@@V12@@1@PEAU?$_Tree_node@U?$pair@$$CBV?$basic_string@DU?$char_traits@D@std@@V?$allocator@D@2@@std@@V12@@std@@PEAX@1@@Z$0 0000000140048f8d f   iniReader.obj
 0001:00047fb0       ?catch$0@?0???$_Insert_nohint@AEAU?$pair@$$CBV?$basic_string@DU?$char_traits@D@std@@V?$allocator@D@2@@std@@V12@@std@@PEAU?$_Tree_node@U?$pair@$$CBV?$basic_string@DU?$char_traits@D@std@@V?$allocator@D@2@@std@@V12@@std@@PEAX@2@@?$_Tree@V?$_Tmap_traits@V?$basic_string@DU?$char_traits@D@std@@V?$allocator@D@2@@std@@V12@U?$less@V?$basic_string@DU?$char_traits@D@std@@V?$allocator@D@2@@std@@@2@V?$allocator@U?$pair@$$CBV?$basic_string@DU?$char_traits@D@std@@V?$allocator@D@2@@std@@V12@@std@@@2@$0A@@std@@@std@@IEAA?AU?$pair@V?$_Tree_iterator@V?$_Tree_val@U?$_Tree_simple_types@U?$pair@$$CBV?$basic_string@DU?$char_traits@D@std@@V?$allocator@D@2@@std@@V12@@std@@@std@@@std@@@std@@_N@1@_NAEAU?$pair@$$CBV?$basic_string@DU?$char_traits@D@std@@V?$allocator@D@2@@std@@V12@@1@PEAU?$_Tree_node@U?$pair@$$CBV?$basic_string@DU?$char_traits@D@std@@V?$allocator@D@2@@std@@V12@@std@@PEAX@1@@Z@4HA 0000000140048fb0 f   iniReader.obj
 0001:00047fbd       __catch$??$_Insert_nohint@AEAU?$pair@$$CBV?$basic_string@DU?$char_traits@D@std@@V?$allocator@D@2@@std@@V12@@std@@PEAU?$_Tree_node@U?$pair@$$CBV?$basic_string@DU?$char_traits@D@std@@V?$allocator@D@2@@std@@V12@@std@@PEAX@2@@?$_Tree@V?$_Tmap_traits@V?$basic_string@DU?$char_traits@D@std@@V?$allocator@D@2@@std@@V12@U?$less@V?$basic_string@DU?$char_traits@D@std@@V?$allocator@D@2@@std@@@2@V?$allocator@U?$pair@$$CBV?$basic_string@DU?$char_traits@D@std@@V?$allocator@D@2@@std@@V12@@std@@@2@$0A@@std@@@std@@IEAA?AU?$pair@V?$_Tree_iterator@V?$_Tree_val@U?$_Tree_simple_types@U?$pair@$$CBV?$basic_string@DU?$char_traits@D@std@@V?$allocator@D@2@@std@@V12@@std@@@std@@@std@@@std@@_N@1@_NAEAU?$pair@$$CBV?$basic_string@DU?$char_traits@D@std@@V?$allocator@D@2@@std@@V12@@1@PEAU?$_Tree_node@U?$pair@$$CBV?$basic_string@DU?$char_traits@D@std@@V?$allocator@D@2@@std@@V12@@std@@PEAX@1@@Z$0 0000000140048fbd f   iniReader.obj
 0001:00047fe0       ?dtor$0@?0??auth_NTLM@mailer@jwsmtp@@AEAA_NAEBV?$basic_string@DU?$char_traits@D@std@@V?$allocator@D@2@@std@@AEB_K@Z@4HA 0000000140048fe0 f   auth.obj
 0001:00047fec       ?dtor$13@?0??auth_NTLM@mailer@jwsmtp@@AEAA_NAEBV?$basic_string@DU?$char_traits@D@std@@V?$allocator@D@2@@std@@AEB_K@Z@4HA 0000000140048fec f   auth.obj
 0001:00047ff8       ?dtor$14@?0??auth_NTLM@mailer@jwsmtp@@AEAA_NAEBV?$basic_string@DU?$char_traits@D@std@@V?$allocator@D@2@@std@@AEB_K@Z@4HA 0000000140048ff8 f   auth.obj
 0001:00048010       ?dtor$0@?0???0mailer@jwsmtp@@QEAA@PEBD0000G_N@Z@4HA 0000000140049010 f   mailer.obj
 0001:00048020       ?dtor$1@?0???0mailer@jwsmtp@@QEAA@PEBD0000G_N@Z@4HA 0000000140049020 f   mailer.obj
 0001:00048030       ?dtor$2@?0???0mailer@jwsmtp@@QEAA@PEBD0000G_N@Z@4HA 0000000140049030 f   mailer.obj
 0001:00048040       ?dtor$3@?0???0mailer@jwsmtp@@QEAA@PEBD0000G_N@Z@4HA 0000000140049040 f   mailer.obj
 0001:00048053       ?dtor$4@?0???0mailer@jwsmtp@@QEAA@PEBD0000G_N@Z@4HA 0000000140049053 f   mailer.obj
 0001:00048066       ?dtor$5@?0???0mailer@jwsmtp@@QEAA@PEBD0000G_N@Z@4HA 0000000140049066 f   mailer.obj
 0001:00048079       ?dtor$6@?0???0mailer@jwsmtp@@QEAA@PEBD0000G_N@Z@4HA 0000000140049079 f   mailer.obj
 0001:00048085       ?dtor$7@?0???0mailer@jwsmtp@@QEAA@PEBD0000G_N@Z@4HA 0000000140049085 f   mailer.obj
 0001:00048098       ?dtor$8@?0???0mailer@jwsmtp@@QEAA@PEBD0000G_N@Z@4HA 0000000140049098 f   mailer.obj
 0001:000480ab       ?dtor$9@?0???0mailer@jwsmtp@@QEAA@PEBD0000G_N@Z@4HA 00000001400490ab f   mailer.obj
 0001:000480be       ?dtor$10@?0???0mailer@jwsmtp@@QEAA@PEBD0000G_N@Z@4HA 00000001400490be f   mailer.obj
 0001:000480d1       ?dtor$11@?0???0mailer@jwsmtp@@QEAA@PEBD0000G_N@Z@4HA 00000001400490d1 f   mailer.obj
 0001:000480e4       ?dtor$12@?0???0mailer@jwsmtp@@QEAA@PEBD0000G_N@Z@4HA 00000001400490e4 f   mailer.obj
 0001:000480f7       ?dtor$13@?0???0mailer@jwsmtp@@QEAA@PEBD0000G_N@Z@4HA 00000001400490f7 f   mailer.obj
 0001:0004810a       ?dtor$14@?0???0mailer@jwsmtp@@QEAA@PEBD0000G_N@Z@4HA 000000014004910a f   mailer.obj
 0001:00048116       ?dtor$15@?0???0mailer@jwsmtp@@QEAA@PEBD0000G_N@Z@4HA 0000000140049116 f   mailer.obj
 0001:00048122       ?dtor$16@?0???0mailer@jwsmtp@@QEAA@PEBD0000G_N@Z@4HA 0000000140049122 f   mailer.obj
 0001:00048130       ?dtor$0@?0??setsender@mailer@jwsmtp@@QEAA_NAEBV?$basic_string@DU?$char_traits@D@std@@V?$allocator@D@2@@std@@@Z@4HA 0000000140049130 f   mailer.obj
 0001:00048140       ?dtor$1@?0??addrecipient@mailer@jwsmtp@@QEAA_NAEBV?$basic_string@DU?$char_traits@D@std@@V?$allocator@D@2@@std@@F@Z@4HA 0000000140049140 f   mailer.obj
 0001:0004814c       ?dtor$10@?0??addrecipient@mailer@jwsmtp@@QEAA_NAEBV?$basic_string@DU?$char_traits@D@std@@V?$allocator@D@2@@std@@F@Z@4HA 000000014004914c f   mailer.obj
 0001:00048158       ?dtor$2@?0??addrecipient@mailer@jwsmtp@@QEAA_NAEBV?$basic_string@DU?$char_traits@D@std@@V?$allocator@D@2@@std@@F@Z@4HA 0000000140049158 f   mailer.obj
 0001:00048170       ?dtor$0@?0???Rmailer@jwsmtp@@QEAAXXZ@4HA 0000000140049170 f   mailer.obj
 0001:0004817c       ?dtor$1@?0???Rmailer@jwsmtp@@QEAAXXZ@4HA 000000014004917c f   mailer.obj
 0001:00048188       ?dtor$2@?0???Rmailer@jwsmtp@@QEAAXXZ@4HA 0000000140049188 f   mailer.obj
 0001:00048194       ?dtor$3@?0???Rmailer@jwsmtp@@QEAAXXZ@4HA 0000000140049194 f   mailer.obj
 0001:000481a0       ?dtor$4@?0???Rmailer@jwsmtp@@QEAAXXZ@4HA 00000001400491a0 f   mailer.obj
 0001:000481ac       ?dtor$5@?0???Rmailer@jwsmtp@@QEAAXXZ@4HA 00000001400491ac f   mailer.obj
 0001:000481b8       ?dtor$6@?0???Rmailer@jwsmtp@@QEAAXXZ@4HA 00000001400491b8 f   mailer.obj
 0001:000481c4       ?dtor$7@?0???Rmailer@jwsmtp@@QEAAXXZ@4HA 00000001400491c4 f   mailer.obj
 0001:000481d0       ?dtor$10@?0???Rmailer@jwsmtp@@QEAAXXZ@4HA 00000001400491d0 f   mailer.obj
 0001:000481dc       ?dtor$11@?0???Rmailer@jwsmtp@@QEAAXXZ@4HA 00000001400491dc f   mailer.obj
 0001:000481e8       ?dtor$12@?0???Rmailer@jwsmtp@@QEAAXXZ@4HA 00000001400491e8 f   mailer.obj
 0001:000481f4       ?dtor$13@?0???Rmailer@jwsmtp@@QEAAXXZ@4HA 00000001400491f4 f   mailer.obj
 0001:00048200       ?dtor$137@?0???Rmailer@jwsmtp@@QEAAXXZ@4HA 0000000140049200 f   mailer.obj
 0001:00048229       ?dtor$178@?0???Rmailer@jwsmtp@@QEAAXXZ@4HA 0000000140049229 f   mailer.obj
 0001:00048260       ?dtor$0@?0??makesmtpmessage@mailer@jwsmtp@@AEBA?AV?$vector@DV?$allocator@D@std@@@std@@XZ@4HA 0000000140049260 f   mailer.obj
 0001:0004826c       ?dtor$2@?0??makesmtpmessage@mailer@jwsmtp@@AEBA?AV?$vector@DV?$allocator@D@std@@@std@@XZ@4HA 000000014004926c f   mailer.obj
 0001:00048295       ?dtor$3@?0??makesmtpmessage@mailer@jwsmtp@@AEBA?AV?$vector@DV?$allocator@D@std@@@std@@XZ@4HA 0000000140049295 f   mailer.obj
 0001:000482a1       ?dtor$54@?0??makesmtpmessage@mailer@jwsmtp@@AEBA?AV?$vector@DV?$allocator@D@std@@@std@@XZ@4HA 00000001400492a1 f   mailer.obj
 0001:000482ca       ?dtor$5@?0??makesmtpmessage@mailer@jwsmtp@@AEBA?AV?$vector@DV?$allocator@D@std@@@std@@XZ@4HA 00000001400492ca f   mailer.obj
 0001:000482d6       ?dtor$6@?0??makesmtpmessage@mailer@jwsmtp@@AEBA?AV?$vector@DV?$allocator@D@std@@@std@@XZ@4HA 00000001400492d6 f   mailer.obj
 0001:000482e2       ?dtor$7@?0??makesmtpmessage@mailer@jwsmtp@@AEBA?AV?$vector@DV?$allocator@D@std@@@std@@XZ@4HA 00000001400492e2 f   mailer.obj
 0001:000482ee       ?dtor$8@?0??makesmtpmessage@mailer@jwsmtp@@AEBA?AV?$vector@DV?$allocator@D@std@@@std@@XZ@4HA 00000001400492ee f   mailer.obj
 0001:000482fa       ?dtor$90@?0??makesmtpmessage@mailer@jwsmtp@@AEBA?AV?$vector@DV?$allocator@D@std@@@std@@XZ@4HA 00000001400492fa f   mailer.obj
 0001:00048328       ?dtor$11@?0??makesmtpmessage@mailer@jwsmtp@@AEBA?AV?$vector@DV?$allocator@D@std@@@std@@XZ@4HA 0000000140049328 f   mailer.obj
 0001:00048334       ?dtor$12@?0??makesmtpmessage@mailer@jwsmtp@@AEBA?AV?$vector@DV?$allocator@D@std@@@std@@XZ@4HA 0000000140049334 f   mailer.obj
 0001:00048340       ?dtor$14@?0??makesmtpmessage@mailer@jwsmtp@@AEBA?AV?$vector@DV?$allocator@D@std@@@std@@XZ@4HA 0000000140049340 f   mailer.obj
 0001:0004834c       ?dtor$15@?0??makesmtpmessage@mailer@jwsmtp@@AEBA?AV?$vector@DV?$allocator@D@std@@@std@@XZ@4HA 000000014004934c f   mailer.obj
 0001:00048358       ?dtor$16@?0??makesmtpmessage@mailer@jwsmtp@@AEBA?AV?$vector@DV?$allocator@D@std@@@std@@XZ@4HA 0000000140049358 f   mailer.obj
 0001:00048364       ?dtor$17@?0??makesmtpmessage@mailer@jwsmtp@@AEBA?AV?$vector@DV?$allocator@D@std@@@std@@XZ@4HA 0000000140049364 f   mailer.obj
 0001:00048370       ?dtor$114@?0??makesmtpmessage@mailer@jwsmtp@@AEBA?AV?$vector@DV?$allocator@D@std@@@std@@XZ@4HA 0000000140049370 f   mailer.obj
 0001:0004839e       ?dtor$126@?0??makesmtpmessage@mailer@jwsmtp@@AEBA?AV?$vector@DV?$allocator@D@std@@@std@@XZ@4HA 000000014004939e f   mailer.obj
 0001:000483cc       ?dtor$138@?0??makesmtpmessage@mailer@jwsmtp@@AEBA?AV?$vector@DV?$allocator@D@std@@@std@@XZ@4HA 00000001400493cc f   mailer.obj
 0001:000483fa       ?dtor$23@?0??makesmtpmessage@mailer@jwsmtp@@AEBA?AV?$vector@DV?$allocator@D@std@@@std@@XZ@4HA 00000001400493fa f   mailer.obj
 0001:00048406       ?dtor$150@?0??makesmtpmessage@mailer@jwsmtp@@AEBA?AV?$vector@DV?$allocator@D@std@@@std@@XZ@4HA 0000000140049406 f   mailer.obj
 0001:00048434       ?dtor$26@?0??makesmtpmessage@mailer@jwsmtp@@AEBA?AV?$vector@DV?$allocator@D@std@@@std@@XZ@4HA 0000000140049434 f   mailer.obj
 0001:00048440       ?dtor$27@?0??makesmtpmessage@mailer@jwsmtp@@AEBA?AV?$vector@DV?$allocator@D@std@@@std@@XZ@4HA 0000000140049440 f   mailer.obj
 0001:0004844c       ?dtor$28@?0??makesmtpmessage@mailer@jwsmtp@@AEBA?AV?$vector@DV?$allocator@D@std@@@std@@XZ@4HA 000000014004944c f   mailer.obj
 0001:00048458       ?dtor$29@?0??makesmtpmessage@mailer@jwsmtp@@AEBA?AV?$vector@DV?$allocator@D@std@@@std@@XZ@4HA 0000000140049458 f   mailer.obj
 0001:00048464       ?dtor$30@?0??makesmtpmessage@mailer@jwsmtp@@AEBA?AV?$vector@DV?$allocator@D@std@@@std@@XZ@4HA 0000000140049464 f   mailer.obj
 0001:00048470       ?dtor$31@?0??makesmtpmessage@mailer@jwsmtp@@AEBA?AV?$vector@DV?$allocator@D@std@@@std@@XZ@4HA 0000000140049470 f   mailer.obj
 0001:0004847c       ?dtor$33@?0??makesmtpmessage@mailer@jwsmtp@@AEBA?AV?$vector@DV?$allocator@D@std@@@std@@XZ@4HA 000000014004947c f   mailer.obj
 0001:00048488       ?dtor$35@?0??makesmtpmessage@mailer@jwsmtp@@AEBA?AV?$vector@DV?$allocator@D@std@@@std@@XZ@4HA 0000000140049488 f   mailer.obj
 0001:00048494       ?dtor$36@?0??makesmtpmessage@mailer@jwsmtp@@AEBA?AV?$vector@DV?$allocator@D@std@@@std@@XZ@4HA 0000000140049494 f   mailer.obj
 0001:000484a0       ?dtor$37@?0??makesmtpmessage@mailer@jwsmtp@@AEBA?AV?$vector@DV?$allocator@D@std@@@std@@XZ@4HA 00000001400494a0 f   mailer.obj
 0001:000484ac       ?dtor$38@?0??makesmtpmessage@mailer@jwsmtp@@AEBA?AV?$vector@DV?$allocator@D@std@@@std@@XZ@4HA 00000001400494ac f   mailer.obj
 0001:000484b8       ?dtor$39@?0??makesmtpmessage@mailer@jwsmtp@@AEBA?AV?$vector@DV?$allocator@D@std@@@std@@XZ@4HA 00000001400494b8 f   mailer.obj
 0001:000484c4       ?dtor$40@?0??makesmtpmessage@mailer@jwsmtp@@AEBA?AV?$vector@DV?$allocator@D@std@@@std@@XZ@4HA 00000001400494c4 f   mailer.obj
 0001:000484d0       ?dtor$41@?0??makesmtpmessage@mailer@jwsmtp@@AEBA?AV?$vector@DV?$allocator@D@std@@@std@@XZ@4HA 00000001400494d0 f   mailer.obj
 0001:000484dc       ?dtor$42@?0??makesmtpmessage@mailer@jwsmtp@@AEBA?AV?$vector@DV?$allocator@D@std@@@std@@XZ@4HA 00000001400494dc f   mailer.obj
 0001:000484e8       ?dtor$43@?0??makesmtpmessage@mailer@jwsmtp@@AEBA?AV?$vector@DV?$allocator@D@std@@@std@@XZ@4HA 00000001400494e8 f   mailer.obj
 0001:000484f4       ?dtor$44@?0??makesmtpmessage@mailer@jwsmtp@@AEBA?AV?$vector@DV?$allocator@D@std@@@std@@XZ@4HA 00000001400494f4 f   mailer.obj
 0001:00048500       ?dtor$45@?0??makesmtpmessage@mailer@jwsmtp@@AEBA?AV?$vector@DV?$allocator@D@std@@@std@@XZ@4HA 0000000140049500 f   mailer.obj
 0001:0004850c       ?dtor$46@?0??makesmtpmessage@mailer@jwsmtp@@AEBA?AV?$vector@DV?$allocator@D@std@@@std@@XZ@4HA 000000014004950c f   mailer.obj
 0001:00048518       ?dtor$47@?0??makesmtpmessage@mailer@jwsmtp@@AEBA?AV?$vector@DV?$allocator@D@std@@@std@@XZ@4HA 0000000140049518 f   mailer.obj
 0001:00048530       ?dtor$0@?0??gethostaddresses@mailer@jwsmtp@@AEAA_NAEAV?$vector@USOCKADDR_IN@jwsmtp@@V?$allocator@USOCKADDR_IN@jwsmtp@@@std@@@std@@@Z@4HA 0000000140049530 f   mailer.obj
 0001:0004853c       ?dtor$2@?0??gethostaddresses@mailer@jwsmtp@@AEAA_NAEAV?$vector@USOCKADDR_IN@jwsmtp@@V?$allocator@USOCKADDR_IN@jwsmtp@@@std@@@std@@@Z@4HA 000000014004953c f   mailer.obj
 0001:00048548       ?dtor$3@?0??gethostaddresses@mailer@jwsmtp@@AEAA_NAEAV?$vector@USOCKADDR_IN@jwsmtp@@V?$allocator@USOCKADDR_IN@jwsmtp@@@std@@@std@@@Z@4HA 0000000140049548 f   mailer.obj
 0001:00048554       ?dtor$4@?0??gethostaddresses@mailer@jwsmtp@@AEAA_NAEAV?$vector@USOCKADDR_IN@jwsmtp@@V?$allocator@USOCKADDR_IN@jwsmtp@@@std@@@std@@@Z@4HA 0000000140049554 f   mailer.obj
 0001:00048560       ?dtor$0@?0??parseaddress@mailer@jwsmtp@@AEAA?AUAddress@12@AEBV?$basic_string@DU?$char_traits@D@std@@V?$allocator@D@2@@std@@@Z@4HA 0000000140049560 f   mailer.obj
 0001:00048570       ?dtor$0@?0??authenticate@mailer@jwsmtp@@AEAA_NAEBV?$basic_string@DU?$char_traits@D@std@@V?$allocator@D@2@@std@@AEB_K@Z@4HA 0000000140049570 f   mailer.obj
 0001:0004857c       ?dtor$1@?0??authenticate@mailer@jwsmtp@@AEAA_NAEBV?$basic_string@DU?$char_traits@D@std@@V?$allocator@D@2@@std@@AEB_K@Z@4HA 000000014004957c f   mailer.obj
 0001:00048588       ?dtor$29@?0??authenticate@mailer@jwsmtp@@AEAA_NAEBV?$basic_string@DU?$char_traits@D@std@@V?$allocator@D@2@@std@@AEB_K@Z@4HA 0000000140049588 f   mailer.obj
 0001:000485ae       ?dtor$41@?0??authenticate@mailer@jwsmtp@@AEAA_NAEBV?$basic_string@DU?$char_traits@D@std@@V?$allocator@D@2@@std@@AEB_K@Z@4HA 00000001400495ae f   mailer.obj
 0001:000485d4       ?dtor$7@?0??authenticate@mailer@jwsmtp@@AEAA_NAEBV?$basic_string@DU?$char_traits@D@std@@V?$allocator@D@2@@std@@AEB_K@Z@4HA 00000001400495d4 f   mailer.obj
 0001:000485e0       ?dtor$10@?0??authenticate@mailer@jwsmtp@@AEAA_NAEBV?$basic_string@DU?$char_traits@D@std@@V?$allocator@D@2@@std@@AEB_K@Z@4HA 00000001400495e0 f   mailer.obj
 0001:000485ec       ?dtor$13@?0??authenticate@mailer@jwsmtp@@AEAA_NAEBV?$basic_string@DU?$char_traits@D@std@@V?$allocator@D@2@@std@@AEB_K@Z@4HA 00000001400495ec f   mailer.obj
 0001:00048600       ?catch$3@?0???$_Emplace_reallocate@AEBV?$basic_string@DU?$char_traits@D@std@@V?$allocator@D@2@@std@@@?$vector@V?$basic_string@DU?$char_traits@D@std@@V?$allocator@D@2@@std@@V?$allocator@V?$basic_string@DU?$char_traits@D@std@@V?$allocator@D@2@@std@@@2@@std@@QEAAPEAV?$basic_string@DU?$char_traits@D@std@@V?$allocator@D@2@@1@QEAV21@AEBV21@@Z@4HA 0000000140049600 f   mailer.obj
 0001:0004860d       __catch$??$_Emplace_reallocate@AEBV?$basic_string@DU?$char_traits@D@std@@V?$allocator@D@2@@std@@@?$vector@V?$basic_string@DU?$char_traits@D@std@@V?$allocator@D@2@@std@@V?$allocator@V?$basic_string@DU?$char_traits@D@std@@V?$allocator@D@2@@std@@@2@@std@@QEAAPEAV?$basic_string@DU?$char_traits@D@std@@V?$allocator@D@2@@1@QEAV21@AEBV21@@Z$0 000000014004960d f   mailer.obj
 0001:00048640       ?dtor$0@?0??getHashFromFile@md5wrapper@@QEAA?AV?$basic_string@DU?$char_traits@D@std@@V?$allocator@D@2@@std@@V23@@Z@4HA 0000000140049640 f   md5wrapper.obj
 0001:00048650       ?dtor$0@?0??LogPacket@CHLogger@@SAXPEBDZZ@4HA 0000000140049650 f   HostLogger.obj
 0001:00048660       ?dtor$0@?0??_BuildDirectory@CHLogger@@CAXAEBU_SYSTEMTIME@@@Z@4HA 0000000140049660 f   HostLogger.obj
 0001:0004866c       ?dtor$1@?0??_BuildDirectory@CHLogger@@CAXAEBU_SYSTEMTIME@@@Z@4HA 000000014004966c f   HostLogger.obj
 0001:00048678       ?dtor$2@?0??_BuildDirectory@CHLogger@@CAXAEBU_SYSTEMTIME@@@Z@4HA 0000000140049678 f   HostLogger.obj
 0001:00048690       ?dtor$0@?0??_DoLogWithLevel@CHLogger@@CAXPEBDW4ELOG_LEVEL@1@0PEAD@Z@4HA 0000000140049690 f   HostLogger.obj
 0001:000486a0       ?dtor$0@?0??Init@CLogMsgManager@@SA_NW4ESHARED_MEM_USAGE_TYPE@1@@Z@4HA 00000001400496a0 f   LogMsgManager.obj
 0001:000486bd       ?dtor$1@?0??Init@CLogMsgManager@@SA_NW4ESHARED_MEM_USAGE_TYPE@1@@Z@4HA 00000001400496bd f   LogMsgManager.obj
 0001:000486e0       ?dtor$0@?0??_WriteXlsDataToSharedMemory@CLogMsgManager@@CA_NXZ@4HA 00000001400496e0 f   LogMsgManager.obj
 0001:000486f0       ?catch$0@?0???$_Insert_hint@AEAU?$pair@$$CB_JV?$basic_string@DU?$char_traits@D@std@@V?$allocator@D@2@@std@@@std@@PEAU?$_Tree_node@U?$pair@$$CB_JV?$basic_string@DU?$char_traits@D@std@@V?$allocator@D@2@@std@@@std@@PEAX@2@@?$_Tree@V?$_Tmap_traits@_JV?$basic_string@DU?$char_traits@D@std@@V?$allocator@D@2@@std@@U?$less@_J@2@V?$allocator@U?$pair@$$CB_JV?$basic_string@DU?$char_traits@D@std@@V?$allocator@D@2@@std@@@std@@@2@$0A@@std@@@std@@IEAA?AV?$_Tree_iterator@V?$_Tree_val@U?$_Tree_simple_types@U?$pair@$$CB_JV?$basic_string@DU?$char_traits@D@std@@V?$allocator@D@2@@std@@@std@@@std@@@std@@@1@V?$_Tree_const_iterator@V?$_Tree_val@U?$_Tree_simple_types@U?$pair@$$CB_JV?$basic_string@DU?$char_traits@D@std@@V?$allocator@D@2@@std@@@std@@@std@@@std@@@1@AEAU?$pair@$$CB_JV?$basic_string@DU?$char_traits@D@std@@V?$allocator@D@2@@std@@@1@PEAU?$_Tree_node@U?$pair@$$CB_JV?$basic_string@DU?$char_traits@D@std@@V?$allocator@D@2@@std@@@std@@PEAX@1@@Z@4HA 00000001400496f0 f   LoadXlsMsg.obj
 0001:000486fd       __catch$??$_Insert_hint@AEAU?$pair@$$CB_JV?$basic_string@DU?$char_traits@D@std@@V?$allocator@D@2@@std@@@std@@PEAU?$_Tree_node@U?$pair@$$CB_JV?$basic_string@DU?$char_traits@D@std@@V?$allocator@D@2@@std@@@std@@PEAX@2@@?$_Tree@V?$_Tmap_traits@_JV?$basic_string@DU?$char_traits@D@std@@V?$allocator@D@2@@std@@U?$less@_J@2@V?$allocator@U?$pair@$$CB_JV?$basic_string@DU?$char_traits@D@std@@V?$allocator@D@2@@std@@@std@@@2@$0A@@std@@@std@@IEAA?AV?$_Tree_iterator@V?$_Tree_val@U?$_Tree_simple_types@U?$pair@$$CB_JV?$basic_string@DU?$char_traits@D@std@@V?$allocator@D@2@@std@@@std@@@std@@@std@@@1@V?$_Tree_const_iterator@V?$_Tree_val@U?$_Tree_simple_types@U?$pair@$$CB_JV?$basic_string@DU?$char_traits@D@std@@V?$allocator@D@2@@std@@@std@@@std@@@std@@@1@AEAU?$pair@$$CB_JV?$basic_string@DU?$char_traits@D@std@@V?$allocator@D@2@@std@@@1@PEAU?$_Tree_node@U?$pair@$$CB_JV?$basic_string@DU?$char_traits@D@std@@V?$allocator@D@2@@std@@@std@@PEAX@1@@Z$0 00000001400496fd f   LoadXlsMsg.obj
 0001:00048720       ?catch$0@?0???$_Insert_nohint@AEAU?$pair@$$CB_JV?$basic_string@DU?$char_traits@D@std@@V?$allocator@D@2@@std@@@std@@PEAU?$_Tree_node@U?$pair@$$CB_JV?$basic_string@DU?$char_traits@D@std@@V?$allocator@D@2@@std@@@std@@PEAX@2@@?$_Tree@V?$_Tmap_traits@_JV?$basic_string@DU?$char_traits@D@std@@V?$allocator@D@2@@std@@U?$less@_J@2@V?$allocator@U?$pair@$$CB_JV?$basic_string@DU?$char_traits@D@std@@V?$allocator@D@2@@std@@@std@@@2@$0A@@std@@@std@@IEAA?AU?$pair@V?$_Tree_iterator@V?$_Tree_val@U?$_Tree_simple_types@U?$pair@$$CB_JV?$basic_string@DU?$char_traits@D@std@@V?$allocator@D@2@@std@@@std@@@std@@@std@@@std@@_N@1@_NAEAU?$pair@$$CB_JV?$basic_string@DU?$char_traits@D@std@@V?$allocator@D@2@@std@@@1@PEAU?$_Tree_node@U?$pair@$$CB_JV?$basic_string@DU?$char_traits@D@std@@V?$allocator@D@2@@std@@@std@@PEAX@1@@Z@4HA 0000000140049720 f   LoadXlsMsg.obj
 0001:0004872d       __catch$??$_Insert_nohint@AEAU?$pair@$$CB_JV?$basic_string@DU?$char_traits@D@std@@V?$allocator@D@2@@std@@@std@@PEAU?$_Tree_node@U?$pair@$$CB_JV?$basic_string@DU?$char_traits@D@std@@V?$allocator@D@2@@std@@@std@@PEAX@2@@?$_Tree@V?$_Tmap_traits@_JV?$basic_string@DU?$char_traits@D@std@@V?$allocator@D@2@@std@@U?$less@_J@2@V?$allocator@U?$pair@$$CB_JV?$basic_string@DU?$char_traits@D@std@@V?$allocator@D@2@@std@@@std@@@2@$0A@@std@@@std@@IEAA?AU?$pair@V?$_Tree_iterator@V?$_Tree_val@U?$_Tree_simple_types@U?$pair@$$CB_JV?$basic_string@DU?$char_traits@D@std@@V?$allocator@D@2@@std@@@std@@@std@@@std@@@std@@_N@1@_NAEAU?$pair@$$CB_JV?$basic_string@DU?$char_traits@D@std@@V?$allocator@D@2@@std@@@1@PEAU?$_Tree_node@U?$pair@$$CB_JV?$basic_string@DU?$char_traits@D@std@@V?$allocator@D@2@@std@@@std@@PEAX@1@@Z$0 000000014004972d f   LoadXlsMsg.obj
 0001:00048740       ?dtor$0@?0??base64encode@jwsmtp@@YA?AV?$vector@DV?$allocator@D@std@@@std@@AEBV23@_N@Z@4HA 0000000140049740 f   base6409cee8549d9fd00dfa06fdadc87a8424.obj
 0001:00048770       ?dtor$0@?0??base64encode@jwsmtp@@YA?AV?$basic_string@DU?$char_traits@D@std@@V?$allocator@D@2@@std@@AEBV23@_N@Z@4HA 0000000140049770 f   base6409cee8549d9fd00dfa06fdadc87a8424.obj
 0001:0004877c       ?dtor$1@?0??base64encode@jwsmtp@@YA?AV?$basic_string@DU?$char_traits@D@std@@V?$allocator@D@2@@std@@AEBV23@_N@Z@4HA 000000014004977c f   base6409cee8549d9fd00dfa06fdadc87a8424.obj
 0001:00048788       ?dtor$3@?0??base64encode@jwsmtp@@YA?AV?$basic_string@DU?$char_traits@D@std@@V?$allocator@D@2@@std@@AEBV23@_N@Z@4HA 0000000140049788 f   base6409cee8549d9fd00dfa06fdadc87a8424.obj
 0001:000487c0       ?dtor$0@?0??base64encode@jwsmtp@@YAXPEBDHPEAD_N@Z@4HA 00000001400497c0 f   base6409cee8549d9fd00dfa06fdadc87a8424.obj
 0001:000487cc       ?dtor$1@?0??base64encode@jwsmtp@@YAXPEBDHPEAD_N@Z@4HA 00000001400497cc f   base6409cee8549d9fd00dfa06fdadc87a8424.obj
 0001:000487e0       ?dtor$0@?0??sprintf_s@internal@cf@@YAHPEAD_KPEBDAEAPEAD@Z@4HA 00000001400497e0 f   safe_string_x64:safe_string.obj
 0001:000487ec       ?dtor$1@?0??sprintf_s@internal@cf@@YAHPEAD_KPEBDAEAPEAD@Z@4HA 00000001400497ec f   safe_string_x64:safe_string.obj
 0001:000487f8       ?dtor$4@?0??sprintf_s@internal@cf@@YAHPEAD_KPEBDAEAPEAD@Z@4HA 00000001400497f8 f   safe_string_x64:safe_string.obj
 0001:00048821       ?dtor$2@?0??sprintf_s@internal@cf@@YAHPEAD_KPEBDAEAPEAD@Z@4HA 0000000140049821 f   safe_string_x64:safe_string.obj
 0001:00048830       ?dtor$0@?0??strncpy_s@cf@@YAHPEAD_KPEBD1@Z@4HA 0000000140049830 f   safe_string_x64:safe_string.obj
 0001:00048830       ?dtor$0@?0??strcpy_s@cf@@YAHPEAD_KPEBD@Z@4HA 0000000140049830 f   safe_string_x64:safe_string.obj
 0001:0004883c       ?dtor$1@?0??strcpy_s@cf@@YAHPEAD_KPEBD@Z@4HA 000000014004983c f   safe_string_x64:safe_string.obj
 0001:0004883c       ?dtor$1@?0??strncpy_s@cf@@YAHPEAD_KPEBD1@Z@4HA 000000014004983c f   safe_string_x64:safe_string.obj
 0001:00048848       ?dtor$4@?0??strncpy_s@cf@@YAHPEAD_KPEBD1@Z@4HA 0000000140049848 f   safe_string_x64:safe_string.obj
 0001:00048848       ?dtor$4@?0??strcpy_s@cf@@YAHPEAD_KPEBD@Z@4HA 0000000140049848 f   safe_string_x64:safe_string.obj
 0001:00048871       ?dtor$2@?0??strncpy_s@cf@@YAHPEAD_KPEBD1@Z@4HA 0000000140049871 f   safe_string_x64:safe_string.obj
 0001:00048871       ?dtor$2@?0??strcpy_s@cf@@YAHPEAD_KPEBD@Z@4HA 0000000140049871 f   safe_string_x64:safe_string.obj
 0001:00048880       ?dtor$0@?0???0?$basic_stringstream@DU?$char_traits@D@std@@V?$allocator@D@2@@std@@QEAA@H@Z@4HA 0000000140049880 f   safe_string_x64:safe_string.obj
 0001:000488ae       ?dtor$1@?0???0?$basic_stringstream@DU?$char_traits@D@std@@V?$allocator@D@2@@std@@QEAA@H@Z@4HA 00000001400498ae f   safe_string_x64:safe_string.obj
 0001:000488c0       __scrt_is_nonwritable_in_current_image$filt$0 00000001400498c0 f   msvcrt:utility.obj
 0001:000488d8       ?fin$0@?0???_L@YAXPEAX_K1P6AX0@Z2@Z@4HA 00000001400498d8 f   msvcrt:ehvecctr.obj
 0001:00048904       ?fin$0@?0???_M@YAXPEAX_K1P6AX0@Z@Z@4HA 0000000140049904 f   msvcrt:ehvecdtr.obj
 0001:00048930       ?filt$0@?0??__ArrayUnwind@@YAXPEAX_K1P6AX0@Z@Z@4HA 0000000140049930 f   msvcrt:ehvecdtr.obj
 0001:00048971       ?filt$0@?0??__scrt_common_main_seh@@YAHXZ@4HA 0000000140049971 f   msvcrt:exe_winmain.obj
 0001:00048990       ??__Fthis_instance_@?1??Instance@DivisionPacketReceiver@@SAPEAV1@XZ@YAXXZ 0000000140049990 f   DivisionPacketReceiver.obj
 0001:00048a40       ??__Fcrs_uploader@?1??CRSUploader@@YAAEAVUploader@crs@@XZ@YAXXZ 0000000140049a40 f   BugReporter.obj
 0001:00048a50       ??__FtheApp@@YAXXZ         0000000140049a50 f   GameServerManager.obj
 0001:00048a60       ??__Fg_cServerLog@@YAXXZ   0000000140049a60 f   GameServerManagerDlg.obj
 0001:00048a70       ??__Fbase64_chars@@YAXXZ   0000000140049a70 f   base64.obj
 0001:00048ae0       ??__Fg_HostStat@@YAXXZ     0000000140049ae0 f   HostStat.obj
 0001:00048af0       ??__Fs@?1??initNetworking@jwsmtp@@YAXXZ@YAXXZ 0000000140049af0 f   compat.obj
 0001:00048b10       ??__F?m_strEtcFileFormat@CHLogger@@0V?$basic_string@DU?$char_traits@D@std@@V?$allocator@D@2@@std@@A@@YAXXZ 0000000140049b10 f   HostLogger.obj
 0001:00048b80       ??__F?m_strKernelFileFormat@CHLogger@@0V?$basic_string@DU?$char_traits@D@std@@V?$allocator@D@2@@std@@A@@YAXXZ 0000000140049b80 f   HostLogger.obj
 0001:00048bf0       ??__F?m_strBRFileFormat@CHLogger@@0V?$basic_string@DU?$char_traits@D@std@@V?$allocator@D@2@@std@@A@@YAXXZ 0000000140049bf0 f   HostLogger.obj
 0001:00048c60       ??__F?m_strFileFormat@CHLogger@@0V?$basic_string@DU?$char_traits@D@std@@V?$allocator@D@2@@std@@A@@YAXXZ 0000000140049c60 f   HostLogger.obj
 0001:00048cd0       ??__F?m_strRWProcessMemoryFileFormat@CHLogger@@0V?$basic_string@DU?$char_traits@D@std@@V?$allocator@D@2@@std@@A@@YAXXZ 0000000140049cd0 f   HostLogger.obj
 0001:00048d40       ??__F?m_strIPCMessageFileFormat@CHLogger@@0V?$basic_string@DU?$char_traits@D@std@@V?$allocator@D@2@@std@@A@@YAXXZ 0000000140049d40 f   HostLogger.obj
 0001:00048db0       ??__F?m_strPacketFileFormat@CHLogger@@0V?$basic_string@DU?$char_traits@D@std@@V?$allocator@D@2@@std@@A@@YAXXZ 0000000140049db0 f   HostLogger.obj
 0001:00048e20       ??__F?m_strTimeOutFileFormat@CHLogger@@0V?$basic_string@DU?$char_traits@D@std@@V?$allocator@D@2@@std@@A@@YAXXZ 0000000140049e20 f   HostLogger.obj
 0001:00048e90       ??__F?m_strHostName@CHLogger@@0V?$basic_string@DU?$char_traits@D@std@@V?$allocator@D@2@@std@@A@@YAXXZ 0000000140049e90 f   HostLogger.obj
 0001:00048f00       ??__F?m_strServerName@CHLogger@@0V?$basic_string@DU?$char_traits@D@std@@V?$allocator@D@2@@std@@A@@YAXXZ 0000000140049f00 f   HostLogger.obj
 0001:00048f70       ??__F?m_strLogFolder@CHLogger@@0V?$basic_string@DU?$char_traits@D@std@@V?$allocator@D@2@@std@@A@@YAXXZ 0000000140049f70 f   HostLogger.obj
 0001:00048fe0       ??__F?m_strModeUserCountFormat@CHLogger@@0V?$basic_string@DU?$char_traits@D@std@@V?$allocator@D@2@@std@@A@@YAXXZ 0000000140049fe0 f   HostLogger.obj
 0001:00049050       ??__F?m_strServerAppUseCountFormat@CHLogger@@0V?$basic_string@DU?$char_traits@D@std@@V?$allocator@D@2@@std@@A@@YAXXZ 000000014004a050 f   HostLogger.obj
 0001:000490c0       ??__F?m_LogLock@CHLogger@@0VCMustSyncObjectLog@@A@@YAXXZ 000000014004a0c0 f   HostLogger.obj
 0001:000490e0       ??__F?m_LogPacketLock@CHLogger@@0VCMustSyncObjectLog@@A@@YAXXZ 000000014004a0e0 f   HostLogger.obj
 0001:00049100       ??__F?m_vectSharedMapHandles@CLogMsgManager@@0V?$vector@PEAXV?$allocator@PEAX@std@@@std@@A@@YAXXZ 000000014004a100 f   LogMsgManager.obj
 0001:00049168       ??__F_AtlBaseModule@ATL@@YAXXZ 000000014004a168 f   atls:atlbase.obj
 0001:00049174       ??__F_Fac_tidy_reg@std@@YAXXZ 000000014004a174 f   msvcprt:locale0_implib.obj
 0002:00000f08       ?pre_cpp_initializer@@3P6AXXZEA 000000014004bf08     msvcrt:exe_winmain.obj
 0002:00000f10       ?_AtlBaseModule$initializer$@ATL@@3P6AXXZEA 000000014004bf10     atls:atlbase.obj
 0002:00000f18       ?_Fac_tidy_reg$initializer$@std@@3P6AXXZEA 000000014004bf18     msvcprt:locale0_implib.obj
 0002:00000f20       ?_afxInitAppState$initializer$@@3P6AXXZEA 000000014004bf20     mfcs140:appmodul.obj
 0002:00000f28       ?theApp$initializer$@@3P6AXXZEA 000000014004bf28     GameServerManager.obj
 0002:00000f30       ?g_cServerLog$initializer$@@3P6AXXZEA 000000014004bf30     GameServerManagerDlg.obj
 0002:00000f38       ?base64_chars$initializer$@@3P6AXXZEA 000000014004bf38     base64.obj
 0002:00000f40       ?g_HostStat$initializer$@@3P6AXXZEA 000000014004bf40     HostStat.obj
 0002:00000f48       ??m_strFileFormat$initializer$@CHLogger@@0P6AXXZEA@@3P6AXXZEA 000000014004bf48     HostLogger.obj
 0002:00000f50       ??m_strBRFileFormat$initializer$@CHLogger@@0P6AXXZEA@@3P6AXXZEA 000000014004bf50     HostLogger.obj
 0002:00000f58       ??m_strKernelFileFormat$initializer$@CHLogger@@0P6AXXZEA@@3P6AXXZEA 000000014004bf58     HostLogger.obj
 0002:00000f60       ??m_strEtcFileFormat$initializer$@CHLogger@@0P6AXXZEA@@3P6AXXZEA 000000014004bf60     HostLogger.obj
 0002:00000f68       ??m_strRWProcessMemoryFileFormat$initializer$@CHLogger@@0P6AXXZEA@@3P6AXXZEA 000000014004bf68     HostLogger.obj
 0002:00000f70       ??m_strIPCMessageFileFormat$initializer$@CHLogger@@0P6AXXZEA@@3P6AXXZEA 000000014004bf70     HostLogger.obj
 0002:00000f78       ??m_strTimeOutFileFormat$initializer$@CHLogger@@0P6AXXZEA@@3P6AXXZEA 000000014004bf78     HostLogger.obj
 0002:00000f80       ??m_strPacketFileFormat$initializer$@CHLogger@@0P6AXXZEA@@3P6AXXZEA 000000014004bf80     HostLogger.obj
 0002:00000f88       ??m_strHostName$initializer$@CHLogger@@0P6AXXZEA@@3P6AXXZEA 000000014004bf88     HostLogger.obj
 0002:00000f90       ??m_strServerName$initializer$@CHLogger@@0P6AXXZEA@@3P6AXXZEA 000000014004bf90     HostLogger.obj
 0002:00000f98       ??m_strLogFolder$initializer$@CHLogger@@0P6AXXZEA@@3P6AXXZEA 000000014004bf98     HostLogger.obj
 0002:00000fa0       ??m_strModeUserCountFormat$initializer$@CHLogger@@0P6AXXZEA@@3P6AXXZEA 000000014004bfa0     HostLogger.obj
 0002:00000fa8       ??m_strServerAppUseCountFormat$initializer$@CHLogger@@0P6AXXZEA@@3P6AXXZEA 000000014004bfa8     HostLogger.obj
 0002:00000fb0       ??m_LogLock$initializer$@CHLogger@@0P6AXXZEA@@3P6AXXZEA 000000014004bfb0     HostLogger.obj
 0002:00000fb8       ??m_LogPacketLock$initializer$@CHLogger@@0P6AXXZEA@@3P6AXXZEA 000000014004bfb8     HostLogger.obj
 0002:00000fc0       ??m_vectSharedMapHandles$initializer$@CLogMsgManager@@0P6AXXZEA@@3P6AXXZEA 000000014004bfc0     LogMsgManager.obj
 0002:00000fc8       ?FloatOne$initializer$@GlobalVectorConstants@@3P6AXXZEA 000000014004bfc8     StdAfx.obj
 0002:00000fd0       ?FloatZero$initializer$@GlobalVectorConstants@@3P6AXXZEA 000000014004bfd0     StdAfx.obj
 0002:00000fd8       ?FloatMinusOne$initializer$@GlobalVectorConstants@@3P6AXXZEA 000000014004bfd8     StdAfx.obj
 0002:00000fe0       ?FloatOneHalf$initializer$@GlobalVectorConstants@@3P6AXXZEA 000000014004bfe0     StdAfx.obj
 0002:00000fe8       ?XYZMask$initializer$@GlobalVectorConstants@@3P6AXXZEA 000000014004bfe8     StdAfx.obj
 0002:00000ff0       ?TwoPi$initializer$@GlobalVectorConstants@@3P6AXXZEA 000000014004bff0     StdAfx.obj
 0002:00000ff8       ?PiByTwo$initializer$@GlobalVectorConstants@@3P6AXXZEA 000000014004bff8     StdAfx.obj
 0002:00001000       ?OneOverTwoPi$initializer$@GlobalVectorConstants@@3P6AXXZEA 000000014004c000     StdAfx.obj
 0002:00001008       ?a$initializer$@VectorSinConstantsSSE@@3P6AXXZEA 000000014004c008     StdAfx.obj
 0002:00001010       ?b$initializer$@VectorSinConstantsSSE@@3P6AXXZEA 000000014004c010     StdAfx.obj
 0002:00001018       ?A$initializer$@VectorSinConstantsSSE@@3P6AXXZEA 000000014004c018     StdAfx.obj
 0002:00001020       ?B$initializer$@VectorSinConstantsSSE@@3P6AXXZEA 000000014004c020     StdAfx.obj
 0002:00001028       ?PI$initializer$@@3P6AXXZEA 000000014004c028     StdAfx.obj
 0002:00001030       ?__iob_func$initializer$@@3P6AXXZEA 000000014004c030     StdAfx.obj
 0002:00001048       ?pre_c_initializer@@3P6AHXZEA 000000014004c048     msvcrt:exe_winmain.obj
 0002:00001050       ?post_pgo_initializer@@3P6AHXZEA 000000014004c050     msvcrt:exe_winmain.obj
 0002:00001058       ?__scrt_initialize_tss_var@@3P6AHXZEA 000000014004c058     msvcrt:thread_safe_statics.obj
 0002:000010a0       $cppxdata$?__scrt_initialize_thread_safe_statics@@YAHXZ 000000014004c0a0     msvcrt:thread_safe_statics.obj
 0002:000011a8       GS_ExceptionPointers       000000014004c1a8     msvcrt:gs_report.obj
 0002:00001258       $cppxdata$??1_Fac_tidy_reg_t@std@@QEAA@XZ 000000014004c258     msvcprt:locale0_implib.obj
 0002:000013e0       ?g_szDmp_FileName_Format@@3PEADEA 000000014004c3e0     BugReporter.obj
 0002:000013e8       ?szDmp_ErrorFile@@3PEADEA  000000014004c3e8     BugReporter.obj
 0002:000013f0       ?szDmp_Folder@@3PEADEA     000000014004c3f0     BugReporter.obj
 0002:000013f8       ?piecewise_construct@std@@3Upiecewise_construct_t@1@B 000000014004c3f8     AppInfoDlg.obj
 0002:000013f9       ?piecewise_construct@std@@3Upiecewise_construct_t@1@B 000000014004c3f9     GameServerManagerDlg.obj
 0002:000013fa       ?piecewise_construct@std@@3Upiecewise_construct_t@1@B 000000014004c3fa     iniReader.obj
 0002:000013fb       ?piecewise_construct@std@@3Upiecewise_construct_t@1@B 000000014004c3fb     LoadXlsMsg.obj
 0002:00001400       ?BOUNDARY_TEXT@@3QBDB      000000014004c400     CSmtp.obj
 0002:00001420       sbox7                      000000014004c420     des.obj
 0002:00001520       sbox4                      000000014004c520     des.obj
 0002:00001620       encrypt_rotate_tab         000000014004c620     des.obj
 0002:00001630       sbox5                      000000014004c630     des.obj
 0002:00001730       sbox8                      000000014004c730     des.obj
 0002:00001830       sbox1                      000000014004c830     des.obj
 0002:00001930       sbox3                      000000014004c930     des.obj
 0002:00001a30       sbox2                      000000014004ca30     des.obj
 0002:00001b30       rightkey_swap              000000014004cb30     des.obj
 0002:00001b70       leftkey_swap               000000014004cb70     des.obj
 0002:00001bb0       weak_keys                  000000014004cbb0     des.obj
 0002:00001db0       sbox6                      000000014004cdb0     des.obj
 0002:00001eb0       fillbuf                    000000014004ceb0     md4.obj
 0002:00001ef0       ?magic@?1??LMOWFv1@@9@9    000000014004cef0     ntlmencrypt.obj
 0002:00001ef8       ?AlmostTwoBits@GlobalVectorConstants@@3IB 000000014004cef8     StdAfx.obj
 0002:00001f00       ?g_szCommonAnimNames@@3QAY0IA@$$CBDA 000000014004cf00     StdAfx.obj
 0002:00005f00       ?WORLD_FORWARD@@3V?$LTVector3@M@@B 0000000140050f00     StdAfx.obj
 0002:00005f10       ?WORLD_RIGHT@@3V?$LTVector3@M@@B 0000000140050f10     StdAfx.obj
 0002:00005f20       ?WORLD_UP@@3V?$LTVector3@M@@B 0000000140050f20     StdAfx.obj
 0002:000071d0       ?messageMap@?1??GetThisMessageMap@CGameServerManagerApp@@KAPEBUAFX_MSGMAP@@XZ@4U3@B 00000001400521d0     GameServerManager.obj
 0002:000071e0       ?_messageEntries@?1??GetThisMessageMap@CGameServerManagerApp@@KAPEBUAFX_MSGMAP@@XZ@4QBUAFX_MSGMAP_ENTRY@@B 00000001400521e0     GameServerManager.obj
 0002:000096e8       ?messageMap@?1??GetThisMessageMap@CGameServerManagerDlg@@KAPEBUAFX_MSGMAP@@XZ@4U3@B 00000001400546e8     GameServerManagerDlg.obj
 0002:00009700       ?_messageEntries@?1??GetThisMessageMap@CGameServerManagerDlg@@KAPEBUAFX_MSGMAP@@XZ@4QBUAFX_MSGMAP_ENTRY@@B 0000000140054700     GameServerManagerDlg.obj
 0002:0000b1c0       $cppxdata$??$_Insert_nohint@AEAU?$pair@$$CB_JVDivisionPacket@@@std@@PEAU?$_Tree_node@U?$pair@$$CB_JVDivisionPacket@@@std@@PEAX@2@@?$_Tree@V?$_Tmap_traits@_JVDivisionPacket@@U?$less@_J@std@@V?$allocator@U?$pair@$$CB_JVDivisionPacket@@@std@@@3@$0A@@std@@@std@@IEAA?AU?$pair@V?$_Tree_iterator@V?$_Tree_val@U?$_Tree_simple_types@U?$pair@$$CB_JVDivisionPacket@@@std@@@std@@@std@@@std@@_N@1@_NAEAU?$pair@$$CB_JVDivisionPacket@@@1@PEAU?$_Tree_node@U?$pair@$$CB_JVDivisionPacket@@@std@@PEAX@1@@Z 00000001400561c0     DivisionPacketReceiver.obj
 0002:0000b1e8       $cppxdata$??$_Buynode@U?$pair@_JVDivisionPacket@@@std@@@?$_Tree_comp_alloc@V?$_Tmap_traits@_JVDivisionPacket@@U?$less@_J@std@@V?$allocator@U?$pair@$$CB_JVDivisionPacket@@@std@@@3@$0A@@std@@@std@@QEAAPEAU?$_Tree_node@U?$pair@$$CB_JVDivisionPacket@@@std@@PEAX@1@$$QEAU?$pair@_JVDivisionPacket@@@1@@Z 00000001400561e8     DivisionPacketReceiver.obj
 0002:0000b210       $cppxdata$?GetPacketBuffer@DivisionPacketReceiver@@QEAA?BW4DIVISION_PACKET_RESULT@@EEEEEPEADG0H@Z 0000000140056210     DivisionPacketReceiver.obj
 0002:0000b238       $cppxdata$??__Fthis_instance_@?1??Instance@DivisionPacketReceiver@@SAPEAV1@XZ@YAXXZ 0000000140056238     DivisionPacketReceiver.obj
 0002:0000b260       $cppxdata$?Instance@DivisionPacketReceiver@@SAPEAV1@XZ 0000000140056260     DivisionPacketReceiver.obj
 0002:0000b288       $cppxdata$?threadCreateDumpFile@@YAKPEAX@Z 0000000140056288     BugReporter.obj
 0002:0000b2b0       $cppxdata$?CRSUploader@@YAAEAVUploader@crs@@XZ 00000001400562b0     BugReporter.obj
 0002:0000b2d8       $cppxdata$?readURL@Uploader@crs@@AEAAXAEAV?$basic_string@_WU?$char_traits@_W@std@@V?$allocator@_W@2@@std@@@Z 00000001400562d8     crs_uploader.obj
 0002:0000b300       $cppxdata$?init@Uploader@crs@@QEAA_N_NPEAD1@Z 0000000140056300     crs_uploader.obj
 0002:0000b328       $cppxdata$?ProcessSocketEvent@CClientLib@@QEAAXXZ 0000000140056328     ClientLib.obj
 0002:0000b350       $cppxdata$?Connect@CSFGameServerClientLib@@QEAAHH@Z 0000000140056350     SFGameServerClientLib.obj
 0002:0000b378       $cppxdata$?GetProcessMemoryUsage@@YAKPEAXH@Z 0000000140056378     CheckMemUsage.obj
 0002:0000b3a0       $cppxdata$?EmptyWorkingset@CHECK_MEM_USAGE@@YA_NPEAXH@Z 00000001400563a0     CheckMemUsage.obj
 0002:0000b3c8       $cppxdata$?clear@?$_Tree@V?$_Tmap_traits@GPEAUtagIP4Address@@U?$less@G@std@@V?$allocator@U?$pair@$$CBGPEAUtagIP4Address@@@std@@@3@$0A@@std@@@std@@QEAAXXZ 00000001400563c8     cSnmpEX.obj
 0002:0000b3c8       $cppxdata$?clear@?$_Tree@V?$_Tmap_traits@GUExtraStatsMemVerify@CHostStat@@U?$less@G@std@@V?$allocator@U?$pair@$$CBGUExtraStatsMemVerify@CHostStat@@@std@@@4@$0A@@std@@@std@@QEAAXXZ 00000001400563c8     HostStat.obj
 0002:0000b3c8       $cppxdata$?clear@?$_Tree@V?$_Tmap_traits@GUExtraStatsFPSVerify@CHostStat@@U?$less@G@std@@V?$allocator@U?$pair@$$CBGUExtraStatsFPSVerify@CHostStat@@@std@@@4@$0A@@std@@@std@@QEAAXXZ 00000001400563c8     HostStat.obj
 0002:0000b3f0       $cppxdata$?MyServiceMain@@YAXKPEAPEAD@Z 00000001400563f0     GameServerManager.obj
 0002:0000b418       $cppxdata$??1SGGMProxyLoader@sggm_proxy@@QEAA@XZ 0000000140056418     GameServerManagerDlg.obj
 0002:0000b440       $cppxdata$?init@SGGMProxyLoader@sggm_proxy@@QEAA_NPEAVMultiReceiver@2@@Z 0000000140056440     GameServerManagerDlg.obj
 0002:0000b468       $cppxdata$?RTIDUSNtoString@EXPAND_USN@@YA?AV?$basic_string@DU?$char_traits@D@std@@V?$allocator@D@2@@std@@HFF_J@Z 0000000140056468     GameServerManagerDlg.obj
 0002:0000b490       $cppxdata$??$_Insert_hint@AEAU?$pair@$$CBIUPORTINFO@@@std@@PEAU?$_Tree_node@U?$pair@$$CBIUPORTINFO@@@std@@PEAX@2@@?$_Tree@V?$_Tmap_traits@IUPORTINFO@@U?$less@I@std@@V?$allocator@U?$pair@$$CBIUPORTINFO@@@std@@@3@$0A@@std@@@std@@IEAA?AV?$_Tree_iterator@V?$_Tree_val@U?$_Tree_simple_types@U?$pair@$$CBIUPORTINFO@@@std@@@std@@@std@@@1@V?$_Tree_const_iterator@V?$_Tree_val@U?$_Tree_simple_types@U?$pair@$$CBIUPORTINFO@@@std@@@std@@@std@@@1@AEAU?$pair@$$CBIUPORTINFO@@@1@PEAU?$_Tree_node@U?$pair@$$CBIUPORTINFO@@@std@@PEAX@1@@Z 0000000140056490     GameServerManagerDlg.obj
 0002:0000b4b8       $cppxdata$??$_Insert_nohint@AEAU?$pair@$$CBIUPORTINFO@@@std@@PEAU?$_Tree_node@U?$pair@$$CBIUPORTINFO@@@std@@PEAX@2@@?$_Tree@V?$_Tmap_traits@IUPORTINFO@@U?$less@I@std@@V?$allocator@U?$pair@$$CBIUPORTINFO@@@std@@@3@$0A@@std@@@std@@IEAA?AU?$pair@V?$_Tree_iterator@V?$_Tree_val@U?$_Tree_simple_types@U?$pair@$$CBIUPORTINFO@@@std@@@std@@@std@@@std@@_N@1@_NAEAU?$pair@$$CBIUPORTINFO@@@1@PEAU?$_Tree_node@U?$pair@$$CBIUPORTINFO@@@std@@PEAX@1@@Z 00000001400564b8     GameServerManagerDlg.obj
 0002:0000b4e0       $cppxdata$??$_Setp@UGAMESERVERINFO@@@?$shared_ptr@UGAMESERVERINFO@@@std@@AEAAXPEAUGAMESERVERINFO@@U?$integral_constant@_N$0A@@1@@Z 00000001400564e0     GameServerManagerDlg.obj
 0002:0000b508       $cppxdata$?clear@?$_Tree@V?$_Tmap_traits@IUPORTINFO@@U?$less@I@std@@V?$allocator@U?$pair@$$CBIUPORTINFO@@@std@@@3@$0A@@std@@@std@@QEAAXXZ 0000000140056508     GameServerManagerDlg.obj
 0002:0000b530       $cppxdata$??1?$shared_ptr@UGAMESERVERINFO@@@std@@QEAA@XZ 0000000140056530     GameServerManagerDlg.obj
 0002:0000b558       $cppxdata$?AssignServerApp@CGameServerManagerDlg@@AEAAXAEBUPROTO_AUTOMATCH_GAME_START_REQ@@F@Z 0000000140056558     GameServerManagerDlg.obj
 0002:0000b580       $cppxdata$?AssignServerApp@CGameServerManagerDlg@@AEAAXAEBUPROTO_STARTING_GAME_tag@@F@Z 0000000140056580     GameServerManagerDlg.obj
 0002:0000b5a8       $cppxdata$?OnReceiveFromGms@CGameServerManagerDlg@@AEAAXAEBUPROTO_AUTOMATCH_GAME_ENTER_REQ@@@Z 00000001400565a8     GameServerManagerDlg.obj
 0002:0000b5d0       $cppxdata$?OnReceiveFromGms@CGameServerManagerDlg@@AEAAXAEBUPROTO_AUTOMATCH_GAME_START_REQ@@@Z 00000001400565d0     GameServerManagerDlg.obj
 0002:0000b5f8       $cppxdata$?OnReceiveFromGms@CGameServerManagerDlg@@AEAAXAEBUPROTO_MMSERVER_TERMINATED_tag@@@Z 00000001400565f8     GameServerManagerDlg.obj
 0002:0000b620       $cppxdata$?OnReceiveFromGms@CGameServerManagerDlg@@AEAAXAEBUPROTO_INSERT_CHARACTER_tag@@@Z 0000000140056620     GameServerManagerDlg.obj
 0002:0000b648       $cppxdata$?OnReceiveFromGms@CGameServerManagerDlg@@AEAAXAEBUPROTO_STARTING_GAME_tag@@@Z 0000000140056648     GameServerManagerDlg.obj
 0002:0000b670       $cppxdata$?RECV_MSG_AI_EXTRA_REWARD@CGameServerManagerDlg@@AEAAXFPEAUPROTO_AI_EXTRA_REWARD_REQ@@@Z 0000000140056670     GameServerManagerDlg.obj
 0002:0000b698       $cppxdata$?RECV_MSG_GAMEEND@CGameServerManagerDlg@@AEAAXFPEBUGAMEPROTO_SS_GAMEEND@@@Z 0000000140056698     GameServerManagerDlg.obj
 0002:0000b6c0       $cppxdata$?Load@CSharedMemoryLoader@@QEAA_NXZ 00000001400566c0     GameServerManagerDlg.obj
 0002:0000b6e8       $cppxdata$?_Load@CSharedMemoryLoader@@AEAA_NXZ 00000001400566e8     GameServerManagerDlg.obj
 0002:0000b710       $cppxdata$?_PreLoad@CSharedMemoryLoader@@AEAA_NXZ 0000000140056710     GameServerManagerDlg.obj
 0002:0000b738       $cppxdata$??0CSharedMemoryLoader@@QEAA@XZ 0000000140056738     GameServerManagerDlg.obj
 0002:0000b760       $cppxdata$?RestoreFreePort@CGameServerManagerDlg@@AEAAXXZ 0000000140056760     GameServerManagerDlg.obj
 0002:0000b788       $cppxdata$?FindFreePorts@CGameServerManagerDlg@@AEAA_NXZ 0000000140056788     GameServerManagerDlg.obj
 0002:0000b7b0       $cppxdata$?StringSplitToNumArray@CGameServerManagerDlg@@AEAAXV?$basic_string@DU?$char_traits@D@std@@V?$allocator@D@2@@std@@0PEAHAEAH@Z 00000001400567b0     GameServerManagerDlg.obj
 0002:0000b7d8       $cppxdata$?VerifyServerAppTermination@CGameServerManagerDlg@@AEAAXXZ 00000001400567d8     GameServerManagerDlg.obj
 0002:0000b800       $cppxdata$?TerminateGameServer@CGameServerManagerDlg@@QEAAXF@Z 0000000140056800     GameServerManagerDlg.obj
 0002:0000b828       $cppxdata$?OnButtonGo@CGameServerManagerDlg@@IEAAXXZ 0000000140056828     GameServerManagerDlg.obj
 0002:0000b850       $cppxdata$?OnTimer@CGameServerManagerDlg@@IEAAX_K@Z 0000000140056850     GameServerManagerDlg.obj
 0002:0000b878       $cppxdata$?KillServerApp@CGameServerManagerDlg@@IEAAXI_N@Z 0000000140056878     GameServerManagerDlg.obj
 0002:0000b8a0       $cppxdata$?OnGameServerMsg@CGameServerManagerDlg@@IEAA_J_K_J@Z 00000001400568a0     GameServerManagerDlg.obj
 0002:0000b8c8       $cppxdata$?StartGameServer@CGameServerManagerDlg@@QEAAHF@Z 00000001400568c8     GameServerManagerDlg.obj
 0002:0000b8f0       $cppxdata$?ConnectToMatchMakingServer@CGameServerManagerDlg@@QEAAHXZ 00000001400568f0     GameServerManagerDlg.obj
 0002:0000b918       $cppxdata$?ReadSettings@CGameServerManagerDlg@@QEAAHXZ 0000000140056918     GameServerManagerDlg.obj
 0002:0000b940       $cppxdata$?InitializeManager@CGameServerManagerDlg@@QEAAHPEADKPEAPEAD@Z 0000000140056940     GameServerManagerDlg.obj
 0002:0000b968       $cppxdata$?KillRemoteProcess@@YA_NK@Z 0000000140056968     GameServerManagerDlg.obj
 0002:0000b990       $cppxdata$??0CGameServerManagerDlg@@QEAA@PEAVCWnd@@@Z 0000000140056990     GameServerManagerDlg.obj
 0002:0000b9b8       $cppxdata$??1CGameServerManagerDlg@@UEAA@XZ 00000001400569b8     GameServerManagerDlg.obj
 0002:0000b9e0       $cppxdata$?SendDiv@CGMSConnManager@@AEAAHEEEPEADK@Z 00000001400569e0     GMSConnManager.obj
 0002:0000ba08       $cppxdata$?Send@CGMSConnManager@@AEAAHPEAVCPacket@@@Z 0000000140056a08     GMSConnManager.obj
 0002:0000ba30       $cppxdata$?SendRoundChange@CGMSConnManager@@QEAAHPEBUPROTO_GAMEGT_ROUND_CHANGE_NTY_tag@@@Z 0000000140056a30     GMSConnManager.obj
 0002:0000ba58       $cppxdata$?SendGameStart@CGMSConnManager@@QEAAHPEBUPROTO_GAMEGT_GAME_START_NTY@@@Z 0000000140056a58     GMSConnManager.obj
 0002:0000ba80       $cppxdata$?SendTeamDeathMatchKillCnt@CGMSConnManager@@QEAAHPEBUPROTO_GAMEGT_TEAM_DEATH_KILL_CNT_NTY@@@Z 0000000140056a80     GMSConnManager.obj
 0002:0000baa8       $cppxdata$?InsertCharacterResult@CGMSConnManager@@QEAAHUPROTO_INSERT_CHARACTER_RESULT_tag@@@Z 0000000140056aa8     GMSConnManager.obj
 0002:0000bad0       $cppxdata$?NotifyAllocableRoomCountChanged@CGMSConnManager@@QEAAHJHHHHHQEAHHH@Z 0000000140056ad0     GMSConnManager.obj
 0002:0000baf8       $cppxdata$?SendBossTowerRewardReq@CGMSConnManager@@QEAAHPEAUPROTO_AI_BOSS_TOWER_REWARD_REQ@@@Z 0000000140056af8     GMSConnManager.obj
 0002:0000bb20       $cppxdata$?SendIngameRewardReq@CGMSConnManager@@QEAAHPEAUPROTO_INGAME_RESULT_REQ@@@Z 0000000140056b20     GMSConnManager.obj
 0002:0000bb48       $cppxdata$?SendAIExtraMiddleRewardReq@CGMSConnManager@@QEAAHPEAUPROTO_AI_EXTRA_MIDDLE_REWARD_REQ@@@Z 0000000140056b48     GMSConnManager.obj
 0002:0000bb70       $cppxdata$?SendKickUserInfo@CGMSConnManager@@QEAAHPEAUPROTO_GAMEMGT_KICK_USER@@@Z 0000000140056b70     GMSConnManager.obj
 0002:0000bb98       $cppxdata$?UpdateCharacterStat@CGMSConnManager@@QEAAHUPROTO_UPDATE_CHARACTER_STAT_tag@@@Z 0000000140056b98     GMSConnManager.obj
 0002:0000bbc0       $cppxdata$?SendForceLeavePollResult@CGMSConnManager@@QEAAHPEBUPROTO_BAN_USER_tag@@@Z 0000000140056bc0     GMSConnManager.obj
 0002:0000bbe8       $cppxdata$?SendAIItemInsert@CGMSConnManager@@QEAAHPEAUPROTO_GAMEGT_INGAME_AIGACHA_ITEM_INSERT@@@Z 0000000140056be8     GMSConnManager.obj
 0002:0000bc10       $cppxdata$?SendIntrusionCoinDec@CGMSConnManager@@QEAAHPEAUPROTO_GAMEGT_MAPLOADING_COMPLETE_NTY_tag@@@Z 0000000140056c10     GMSConnManager.obj
 0002:0000bc38       $cppxdata$?SendSpyChange@CGMSConnManager@@QEAAHPEAUPROTO_GAMEGT_SPY_CHANGE_NTY_tag@@@Z 0000000140056c38     GMSConnManager.obj
 0002:0000bc60       $cppxdata$?SendFarmingItemReq@CGMSConnManager@@QEAAHPEAUPROTO_GAMEGT_INGAME_FARMING_ITEM_REQ@@@Z 0000000140056c60     GMSConnManager.obj
 0002:0000bc88       $cppxdata$?SendBattleShipBonusCoinReq@CGMSConnManager@@QEAAHPEAUPROTOCOL_AI2_BONUSROUND_REWARD_REQ_tag@@@Z 0000000140056c88     GMSConnManager.obj
 0002:0000bcb0       $cppxdata$?SendAI3BonusClearItemReq@CGMSConnManager@@QEAAHPEAUPROTO_GAMEGT_INGAME_AI3_BONUS_REWARD_ITEM_REQ@@@Z 0000000140056cb0     GMSConnManager.obj
 0002:0000bcd8       $cppxdata$?SendAIExtraRewardReq@CGMSConnManager@@QEAAHPEAUPROTO_AI_EXTRA_REWARD_REQ@@@Z 0000000140056cd8     GMSConnManager.obj
 0002:0000bd00       $cppxdata$?SendPrevGameFinishNotify@CGMSConnManager@@QEAAHPEAUPROTO_FINISHED_GAME_PREV_tag@@@Z 0000000140056d00     GMSConnManager.obj
 0002:0000bd28       $cppxdata$?SendSpectatorRecommendRoomData@CGMSConnManager@@QEAAHPEAUPROTO_SPECTATOR_RECOMMEND_ROOM_INGAME_DATA_NTY@@@Z 0000000140056d28     GMSConnManager.obj
 0002:0000bd50       $cppxdata$?SendAutoSideChangeTeamInfoNotify@CGMSConnManager@@QEAAHPEAUPROTO_GAMEGT_AUTO_SIDE_CHANGE_TEAM_INFO_NTY@@@Z 0000000140056d50     GMSConnManager.obj
 0002:0000bd78       $cppxdata$?StartingGameResult@CGMSConnManager@@QEAAHUPROTO_STARTING_GAME_RESULT_tag@@W4START_HOST_RESULT@@@Z 0000000140056d78     GMSConnManager.obj
 0002:0000bda0       $cppxdata$?SendAutoMatchGameStartRes@CGMSConnManager@@QEAAHAEBUPROTO_AUTOMATCH_GAME_START_RES@@W4START_HOST_RESULT@@@Z 0000000140056da0     GMSConnManager.obj
 0002:0000bdc8       $cppxdata$?SendAutoMatchGameEnterRes@CGMSConnManager@@QEAAHAEBUPROTO_AUTOMATCH_GAME_ENTER_RES@@@Z 0000000140056dc8     GMSConnManager.obj
 0002:0000bdf0       $cppxdata$?SendAutoMatchIngameEnterNty@CGMSConnManager@@QEAAHAEBUPROTO_AUTOMATCH_INGAME_ENTER_NTY@@@Z 0000000140056df0     GMSConnManager.obj
 0002:0000be18       $cppxdata$??_ECSFGameServerClientLib@@UEAAPEAXI@Z 0000000140056e18     GMSConnManager.obj
 0002:0000be40       $cppxdata$??$?HDU?$char_traits@D@std@@V?$allocator@D@1@@std@@YA?AV?$basic_string@DU?$char_traits@D@std@@V?$allocator@D@2@@0@QEBDAEBV10@@Z 0000000140056e40     CSmtp.obj
 0002:0000be68       $cppxdata$??$?6U?$char_traits@D@std@@@std@@YAAEAV?$basic_ostream@DU?$char_traits@D@std@@@0@AEAV10@PEBD@Z 0000000140056e68     md5_csmtp.obj
 0002:0000be90       $cppxdata$??1_Sentry_base@?$basic_ostream@DU?$char_traits@D@std@@@std@@QEAA@XZ 0000000140056e90     md5_csmtp.obj
 0002:0000beb8       $cppxdata$??1sentry@?$basic_ostream@DU?$char_traits@D@std@@@std@@QEAA@XZ 0000000140056eb8     md5_csmtp.obj
 0002:0000bee0       $cppxdata$??$_Insert_nohint@AEAU?$pair@$$CBGUExtraStatsMemVerify@CHostStat@@@std@@PEAU?$_Tree_node@U?$pair@$$CBGUExtraStatsMemVerify@CHostStat@@@std@@PEAX@2@@?$_Tree@V?$_Tmap_traits@GUExtraStatsMemVerify@CHostStat@@U?$less@G@std@@V?$allocator@U?$pair@$$CBGUExtraStatsMemVerify@CHostStat@@@std@@@4@$0A@@std@@@std@@IEAA?AU?$pair@V?$_Tree_iterator@V?$_Tree_val@U?$_Tree_simple_types@U?$pair@$$CBGUExtraStatsMemVerify@CHostStat@@@std@@@std@@@std@@@std@@_N@1@_NAEAU?$pair@$$CBGUExtraStatsMemVerify@CHostStat@@@1@PEAU?$_Tree_node@U?$pair@$$CBGUExtraStatsMemVerify@CHostStat@@@std@@PEAX@1@@Z 0000000140056ee0     HostStat.obj
 0002:0000bee0       $cppxdata$??$_Insert_nohint@AEAU?$pair@$$CBGUExtraStatsFPSVerify@CHostStat@@@std@@PEAU?$_Tree_node@U?$pair@$$CBGUExtraStatsFPSVerify@CHostStat@@@std@@PEAX@2@@?$_Tree@V?$_Tmap_traits@GUExtraStatsFPSVerify@CHostStat@@U?$less@G@std@@V?$allocator@U?$pair@$$CBGUExtraStatsFPSVerify@CHostStat@@@std@@@4@$0A@@std@@@std@@IEAA?AU?$pair@V?$_Tree_iterator@V?$_Tree_val@U?$_Tree_simple_types@U?$pair@$$CBGUExtraStatsFPSVerify@CHostStat@@@std@@@std@@@std@@@std@@_N@1@_NAEAU?$pair@$$CBGUExtraStatsFPSVerify@CHostStat@@@1@PEAU?$_Tree_node@U?$pair@$$CBGUExtraStatsFPSVerify@CHostStat@@@std@@PEAX@1@@Z 0000000140056ee0     HostStat.obj
 0002:0000bf08       $cppxdata$?GatherFiles@CHostStat@@QEAAXPEAD@Z 0000000140056f08     HostStat.obj
 0002:0000bf30       $cppxdata$?send@CHostStat@@IEAA_NPEAD0@Z 0000000140056f30     HostStat.obj
 0002:0000bf58       $cppxdata$?addExtraData@CHostStat@@QEAAXGE@Z 0000000140056f58     HostStat.obj
 0002:0000bf80       $cppxdata$?setData64@CHostStat@@QEAAXGEEG_J@Z 0000000140056f80     HostStat.obj
 0002:0000bfa8       $cppxdata$?getData64@CHostStat@@QEAA_JGEEG@Z 0000000140056fa8     HostStat.obj
 0002:0000bfd0       $cppxdata$?thdMail@CHostStat@@KAIPEAX@Z 0000000140056fd0     HostStat.obj
 0002:0000bff8       $cppxdata$??1CHostStat@@UEAA@XZ 0000000140056ff8     HostStat.obj
 0002:0000c020       $cppxdata$??__Eg_HostStat@@YAXXZ 0000000140057020     HostStat.obj
 0002:0000c048       $cppxdata$?setup@CHostStat@@QEAAXHH@Z 0000000140057048     HostStat.obj
 0002:0000c070       $cppxdata$?timer@CHostStat@@QEAAXXZ 0000000140057070     HostStat.obj
 0002:0000c098       $cppxdata$?addExtraData@CHostStat@@QEAAXGEEGIII@Z 0000000140057098     HostStat.obj
 0002:0000c0c0       $cppxdata$?addData@CHostStat@@QEAAXGEEG@Z 00000001400570c0     HostStat.obj
 0002:0000c0e8       $cppxdata$??$_Insert_nohint@AEAU?$pair@$$CBV?$basic_string@DU?$char_traits@D@std@@V?$allocator@D@2@@std@@V12@@std@@PEAU?$_Tree_node@U?$pair@$$CBV?$basic_string@DU?$char_traits@D@std@@V?$allocator@D@2@@std@@V12@@std@@PEAX@2@@?$_Tree@V?$_Tmap_traits@V?$basic_string@DU?$char_traits@D@std@@V?$allocator@D@2@@std@@V12@U?$less@V?$basic_string@DU?$char_traits@D@std@@V?$allocator@D@2@@std@@@2@V?$allocator@U?$pair@$$CBV?$basic_string@DU?$char_traits@D@std@@V?$allocator@D@2@@std@@V12@@std@@@2@$0A@@std@@@std@@IEAA?AU?$pair@V?$_Tree_iterator@V?$_Tree_val@U?$_Tree_simple_types@U?$pair@$$CBV?$basic_string@DU?$char_traits@D@std@@V?$allocator@D@2@@std@@V12@@std@@@std@@@std@@@std@@_N@1@_NAEAU?$pair@$$CBV?$basic_string@DU?$char_traits@D@std@@V?$allocator@D@2@@std@@V12@@1@PEAU?$_Tree_node@U?$pair@$$CBV?$basic_string@DU?$char_traits@D@std@@V?$allocator@D@2@@std@@V12@@std@@PEAX@1@@Z 00000001400570e8     iniReader.obj
 0002:0000c110       $cppxdata$??$_Insert_hint@AEAU?$pair@$$CBV?$basic_string@DU?$char_traits@D@std@@V?$allocator@D@2@@std@@V12@@std@@PEAU?$_Tree_node@U?$pair@$$CBV?$basic_string@DU?$char_traits@D@std@@V?$allocator@D@2@@std@@V12@@std@@PEAX@2@@?$_Tree@V?$_Tmap_traits@V?$basic_string@DU?$char_traits@D@std@@V?$allocator@D@2@@std@@V12@U?$less@V?$basic_string@DU?$char_traits@D@std@@V?$allocator@D@2@@std@@@2@V?$allocator@U?$pair@$$CBV?$basic_string@DU?$char_traits@D@std@@V?$allocator@D@2@@std@@V12@@std@@@2@$0A@@std@@@std@@IEAA?AV?$_Tree_iterator@V?$_Tree_val@U?$_Tree_simple_types@U?$pair@$$CBV?$basic_string@DU?$char_traits@D@std@@V?$allocator@D@2@@std@@V12@@std@@@std@@@std@@@1@V?$_Tree_const_iterator@V?$_Tree_val@U?$_Tree_simple_types@U?$pair@$$CBV?$basic_string@DU?$char_traits@D@std@@V?$allocator@D@2@@std@@V12@@std@@@std@@@std@@@1@AEAU?$pair@$$CBV?$basic_string@DU?$char_traits@D@std@@V?$allocator@D@2@@std@@V12@@1@PEAU?$_Tree_node@U?$pair@$$CBV?$basic_string@DU?$char_traits@D@std@@V?$allocator@D@2@@std@@V12@@std@@PEAX@1@@Z 0000000140057110     iniReader.obj
 0002:0000c138       $cppxdata$??$_Insert_nohint@AEAU?$pair@$$CBV?$basic_string@DU?$char_traits@D@std@@V?$allocator@D@2@@std@@PEAVCIniSection@CIniReader@@@std@@PEAU?$_Tree_node@U?$pair@$$CBV?$basic_string@DU?$char_traits@D@std@@V?$allocator@D@2@@std@@PEAVCIniSection@CIniReader@@@std@@PEAX@2@@?$_Tree@V?$_Tmap_traits@V?$basic_string@DU?$char_traits@D@std@@V?$allocator@D@2@@std@@PEAVCIniSection@CIniReader@@U?$less@V?$basic_string@DU?$char_traits@D@std@@V?$allocator@D@2@@std@@@2@V?$allocator@U?$pair@$$CBV?$basic_string@DU?$char_traits@D@std@@V?$allocator@D@2@@std@@PEAVCIniSection@CIniReader@@@std@@@2@$0A@@std@@@std@@IEAA?AU?$pair@V?$_Tree_iterator@V?$_Tree_val@U?$_Tree_simple_types@U?$pair@$$CBV?$basic_string@DU?$char_traits@D@std@@V?$allocator@D@2@@std@@PEAVCIniSection@CIniReader@@@std@@@std@@@std@@@std@@_N@1@_NAEAU?$pair@$$CBV?$basic_string@DU?$char_traits@D@std@@V?$allocator@D@2@@std@@PEAVCIniSection@CIniReader@@@1@PEAU?$_Tree_node@U?$pair@$$CBV?$basic_string@DU?$char_traits@D@std@@V?$allocator@D@2@@std@@PEAVCIniSection@CIniReader@@@std@@PEAX@1@@Z 0000000140057138     iniReader.obj
 0002:0000c160       $cppxdata$??$_Buynode@U?$pair@PEADPEAVCIniSection@CIniReader@@@std@@@?$_Tree_comp_alloc@V?$_Tmap_traits@V?$basic_string@DU?$char_traits@D@std@@V?$allocator@D@2@@std@@PEAVCIniSection@CIniReader@@U?$less@V?$basic_string@DU?$char_traits@D@std@@V?$allocator@D@2@@std@@@2@V?$allocator@U?$pair@$$CBV?$basic_string@DU?$char_traits@D@std@@V?$allocator@D@2@@std@@PEAVCIniSection@CIniReader@@@std@@@2@$0A@@std@@@std@@QEAAPEAU?$_Tree_node@U?$pair@$$CBV?$basic_string@DU?$char_traits@D@std@@V?$allocator@D@2@@std@@PEAVCIniSection@CIniReader@@@std@@PEAX@1@$$QEAU?$pair@PEADPEAVCIniSection@CIniReader@@@1@@Z 0000000140057160     iniReader.obj
 0002:0000c188       $cppxdata$?erase@?$_Tree@V?$_Tmap_traits@V?$basic_string@DU?$char_traits@D@std@@V?$allocator@D@2@@std@@V12@U?$less@V?$basic_string@DU?$char_traits@D@std@@V?$allocator@D@2@@std@@@2@V?$allocator@U?$pair@$$CBV?$basic_string@DU?$char_traits@D@std@@V?$allocator@D@2@@std@@V12@@std@@@2@$0A@@std@@@std@@QEAA?AV?$_Tree_iterator@V?$_Tree_val@U?$_Tree_simple_types@U?$pair@$$CBV?$basic_string@DU?$char_traits@D@std@@V?$allocator@D@2@@std@@V12@@std@@@std@@@std@@@2@V?$_Tree_const_iterator@V?$_Tree_val@U?$_Tree_simple_types@U?$pair@$$CBV?$basic_string@DU?$char_traits@D@std@@V?$allocator@D@2@@std@@V12@@std@@@std@@@std@@@2@0@Z 0000000140057188     iniReader.obj
 0002:0000c1b0       $cppxdata$?erase@?$_Tree@V?$_Tmap_traits@V?$basic_string@DU?$char_traits@D@std@@V?$allocator@D@2@@std@@PEAVCIniSection@CIniReader@@U?$less@V?$basic_string@DU?$char_traits@D@std@@V?$allocator@D@2@@std@@@2@V?$allocator@U?$pair@$$CBV?$basic_string@DU?$char_traits@D@std@@V?$allocator@D@2@@std@@PEAVCIniSection@CIniReader@@@std@@@2@$0A@@std@@@std@@QEAA?AV?$_Tree_iterator@V?$_Tree_val@U?$_Tree_simple_types@U?$pair@$$CBV?$basic_string@DU?$char_traits@D@std@@V?$allocator@D@2@@std@@PEAVCIniSection@CIniReader@@@std@@@std@@@std@@@2@V?$_Tree_const_iterator@V?$_Tree_val@U?$_Tree_simple_types@U?$pair@$$CBV?$basic_string@DU?$char_traits@D@std@@V?$allocator@D@2@@std@@PEAVCIniSection@CIniReader@@@std@@@std@@@std@@@2@0@Z 00000001400571b0     iniReader.obj
 0002:0000c1d8       $cppxdata$?setString@CIniSection@CIniReader@@QEAAXPEBD0@Z 00000001400571d8     iniReader.obj
 0002:0000c200       $cppxdata$?write@CIniSection@CIniReader@@QEAAKPEAX@Z 0000000140057200     iniReader.obj
 0002:0000c228       $cppxdata$?clear@CIniReader@@QEAAXXZ 0000000140057228     iniReader.obj
 0002:0000c250       $cppxdata$?setString@CIniReader@@QEAAXPEBD00@Z 0000000140057250     iniReader.obj
 0002:0000c278       $cppxdata$?write@CIniReader@@QEAAKPEBD@Z 0000000140057278     iniReader.obj
 0002:0000c2a0       $cppxdata$?auth_NTLM@mailer@jwsmtp@@AEAA_NAEBV?$basic_string@DU?$char_traits@D@std@@V?$allocator@D@2@@std@@AEB_K@Z 00000001400572a0     auth.obj
 0002:0000c2c8       $cppxdata$??$_Emplace_reallocate@AEBV?$basic_string@DU?$char_traits@D@std@@V?$allocator@D@2@@std@@@?$vector@V?$basic_string@DU?$char_traits@D@std@@V?$allocator@D@2@@std@@V?$allocator@V?$basic_string@DU?$char_traits@D@std@@V?$allocator@D@2@@std@@@2@@std@@QEAAPEAV?$basic_string@DU?$char_traits@D@std@@V?$allocator@D@2@@1@QEAV21@AEBV21@@Z 00000001400572c8     mailer.obj
 0002:0000c2f0       $cppxdata$?authenticate@mailer@jwsmtp@@AEAA_NAEBV?$basic_string@DU?$char_traits@D@std@@V?$allocator@D@2@@std@@AEB_K@Z 00000001400572f0     mailer.obj
 0002:0000c318       $cppxdata$?parseaddress@mailer@jwsmtp@@AEAA?AUAddress@12@AEBV?$basic_string@DU?$char_traits@D@std@@V?$allocator@D@2@@std@@@Z 0000000140057318     mailer.obj
 0002:0000c340       $cppxdata$?gethostaddresses@mailer@jwsmtp@@AEAA_NAEAV?$vector@USOCKADDR_IN@jwsmtp@@V?$allocator@USOCKADDR_IN@jwsmtp@@@std@@@std@@@Z 0000000140057340     mailer.obj
 0002:0000c368       $cppxdata$?makesmtpmessage@mailer@jwsmtp@@AEBA?AV?$vector@DV?$allocator@D@std@@@std@@XZ 0000000140057368     mailer.obj
 0002:0000c390       $cppxdata$??Rmailer@jwsmtp@@QEAAXXZ 0000000140057390     mailer.obj
 0002:0000c3b8       $cppxdata$?addrecipient@mailer@jwsmtp@@QEAA_NAEBV?$basic_string@DU?$char_traits@D@std@@V?$allocator@D@2@@std@@F@Z 00000001400573b8     mailer.obj
 0002:0000c3e0       $cppxdata$?setsender@mailer@jwsmtp@@QEAA_NAEBV?$basic_string@DU?$char_traits@D@std@@V?$allocator@D@2@@std@@@Z 00000001400573e0     mailer.obj
 0002:0000c408       $cppxdata$??0mailer@jwsmtp@@QEAA@PEBD0000G_N@Z 0000000140057408     mailer.obj
 0002:0000c430       $cppxdata$?getHashFromFile@md5wrapper@@QEAA?AV?$basic_string@DU?$char_traits@D@std@@V?$allocator@D@2@@std@@V23@@Z 0000000140057430     md5wrapper.obj
 0002:0000c458       $cppxdata$?_DoLogWithLevel@CHLogger@@CAXPEBDW4ELOG_LEVEL@1@0PEAD@Z 0000000140057458     HostLogger.obj
 0002:0000c480       $cppxdata$?_BuildDirectory@CHLogger@@CAXAEBU_SYSTEMTIME@@@Z 0000000140057480     HostLogger.obj
 0002:0000c4a8       $cppxdata$?LogPacket@CHLogger@@SAXPEBDZZ 00000001400574a8     HostLogger.obj
 0002:0000c4d0       $cppxdata$?_WriteXlsDataToSharedMemory@CLogMsgManager@@CA_NXZ 00000001400574d0     LogMsgManager.obj
 0002:0000c4f8       $cppxdata$?Init@CLogMsgManager@@SA_NW4ESHARED_MEM_USAGE_TYPE@1@@Z 00000001400574f8     LogMsgManager.obj
 0002:0000c520       $cppxdata$??$_Insert_nohint@AEAU?$pair@$$CB_JV?$basic_string@DU?$char_traits@D@std@@V?$allocator@D@2@@std@@@std@@PEAU?$_Tree_node@U?$pair@$$CB_JV?$basic_string@DU?$char_traits@D@std@@V?$allocator@D@2@@std@@@std@@PEAX@2@@?$_Tree@V?$_Tmap_traits@_JV?$basic_string@DU?$char_traits@D@std@@V?$allocator@D@2@@std@@U?$less@_J@2@V?$allocator@U?$pair@$$CB_JV?$basic_string@DU?$char_traits@D@std@@V?$allocator@D@2@@std@@@std@@@2@$0A@@std@@@std@@IEAA?AU?$pair@V?$_Tree_iterator@V?$_Tree_val@U?$_Tree_simple_types@U?$pair@$$CB_JV?$basic_string@DU?$char_traits@D@std@@V?$allocator@D@2@@std@@@std@@@std@@@std@@@std@@_N@1@_NAEAU?$pair@$$CB_JV?$basic_string@DU?$char_traits@D@std@@V?$allocator@D@2@@std@@@1@PEAU?$_Tree_node@U?$pair@$$CB_JV?$basic_string@DU?$char_traits@D@std@@V?$allocator@D@2@@std@@@std@@PEAX@1@@Z 0000000140057520     LoadXlsMsg.obj
 0002:0000c548       $cppxdata$??$_Insert_hint@AEAU?$pair@$$CB_JV?$basic_string@DU?$char_traits@D@std@@V?$allocator@D@2@@std@@@std@@PEAU?$_Tree_node@U?$pair@$$CB_JV?$basic_string@DU?$char_traits@D@std@@V?$allocator@D@2@@std@@@std@@PEAX@2@@?$_Tree@V?$_Tmap_traits@_JV?$basic_string@DU?$char_traits@D@std@@V?$allocator@D@2@@std@@U?$less@_J@2@V?$allocator@U?$pair@$$CB_JV?$basic_string@DU?$char_traits@D@std@@V?$allocator@D@2@@std@@@std@@@2@$0A@@std@@@std@@IEAA?AV?$_Tree_iterator@V?$_Tree_val@U?$_Tree_simple_types@U?$pair@$$CB_JV?$basic_string@DU?$char_traits@D@std@@V?$allocator@D@2@@std@@@std@@@std@@@std@@@1@V?$_Tree_const_iterator@V?$_Tree_val@U?$_Tree_simple_types@U?$pair@$$CB_JV?$basic_string@DU?$char_traits@D@std@@V?$allocator@D@2@@std@@@std@@@std@@@std@@@1@AEAU?$pair@$$CB_JV?$basic_string@DU?$char_traits@D@std@@V?$allocator@D@2@@std@@@1@PEAU?$_Tree_node@U?$pair@$$CB_JV?$basic_string@DU?$char_traits@D@std@@V?$allocator@D@2@@std@@@std@@PEAX@1@@Z 0000000140057548     LoadXlsMsg.obj
 0002:0000c570       $cppxdata$?erase@?$_Tree@V?$_Tmap_traits@_JV?$basic_string@DU?$char_traits@D@std@@V?$allocator@D@2@@std@@U?$less@_J@2@V?$allocator@U?$pair@$$CB_JV?$basic_string@DU?$char_traits@D@std@@V?$allocator@D@2@@std@@@std@@@2@$0A@@std@@@std@@QEAA?AV?$_Tree_iterator@V?$_Tree_val@U?$_Tree_simple_types@U?$pair@$$CB_JV?$basic_string@DU?$char_traits@D@std@@V?$allocator@D@2@@std@@@std@@@std@@@std@@@2@V?$_Tree_const_iterator@V?$_Tree_val@U?$_Tree_simple_types@U?$pair@$$CB_JV?$basic_string@DU?$char_traits@D@std@@V?$allocator@D@2@@std@@@std@@@std@@@std@@@2@0@Z 0000000140057570     LoadXlsMsg.obj
 0002:0000c598       $cppxdata$??_GFindXlsMsg@@UEAAPEAXI@Z 0000000140057598     LoadXlsMsg.obj
 0002:0000c5c0       $cppxdata$?LoadWMszFile@FindXlsMsg@@QEAA_NPEAD@Z 00000001400575c0     LoadXlsMsg.obj
 0002:0000c5e8       $cppxdata$?base64encode@jwsmtp@@YA?AV?$vector@DV?$allocator@D@std@@@std@@AEBV23@_N@Z 00000001400575e8     base6409cee8549d9fd00dfa06fdadc87a8424.obj
 0002:0000c610       $cppxdata$?base64encode@jwsmtp@@YA?AV?$basic_string@DU?$char_traits@D@std@@V?$allocator@D@2@@std@@AEBV23@_N@Z 0000000140057610     base6409cee8549d9fd00dfa06fdadc87a8424.obj
 0002:0000c638       $cppxdata$?base64encode@jwsmtp@@YAXPEBDHPEAD_N@Z 0000000140057638     base6409cee8549d9fd00dfa06fdadc87a8424.obj
 0002:0000c660       $cppxdata$??0?$basic_stringstream@DU?$char_traits@D@std@@V?$allocator@D@2@@std@@QEAA@H@Z 0000000140057660     safe_string_x64:safe_string.obj
 0002:0000c688       $cppxdata$?strncpy_s@cf@@YAHPEAD_KPEBD1@Z 0000000140057688     safe_string_x64:safe_string.obj
 0002:0000c6b0       $cppxdata$?sprintf_s@internal@cf@@YAHPEAD_KPEBDAEAPEAD@Z 00000001400576b0     safe_string_x64:safe_string.obj
 0002:0000c6d8       $cppxdata$?strcpy_s@cf@@YAHPEAD_KPEBD@Z 00000001400576d8     safe_string_x64:safe_string.obj
 0002:0000e240       $unwind$?AppendPacket@DivisionPacket@@AEAA?BW4DIVISION_PACKET_RESULT@@PEADG@Z 0000000140059240     DivisionPacket.obj
 0002:0000e258       $unwind$?_Buynode0@?$_Tree_comp_alloc@V?$_Tmap_traits@IUPORTINFO@@U?$less@I@std@@V?$allocator@U?$pair@$$CBIUPORTINFO@@@std@@@3@$0A@@std@@@std@@QEAAPEAU?$_Tree_node@U?$pair@$$CBIUPORTINFO@@@std@@PEAX@2@XZ 0000000140059258     GameServerManagerDlg.obj
 0002:0000e258       $unwind$_onexit            0000000140059258     msvcrt:utility.obj
 0002:0000e258       $unwind$??_GCReceiver@@UEAAPEAXI@Z 0000000140059258     SGGMCallBackObj.obj
 0002:0000e258       $unwind$??$_Buynode@U?$pair@IUPORTINFO@@@std@@@?$_Tree_comp_alloc@V?$_Tmap_traits@IUPORTINFO@@U?$less@I@std@@V?$allocator@U?$pair@$$CBIUPORTINFO@@@std@@@3@$0A@@std@@@std@@QEAAPEAU?$_Tree_node@U?$pair@$$CBIUPORTINFO@@@std@@PEAX@1@$$QEAU?$pair@IUPORTINFO@@@1@@Z 0000000140059258     GameServerManagerDlg.obj
 0002:0000e258       $unwind$??1?$pair@$$CBV?$basic_string@DU?$char_traits@D@std@@V?$allocator@D@2@@std@@V12@@std@@QEAA@XZ 0000000140059258     iniReader.obj
 0002:0000e258       $unwind$__scrt_initialize_crt 0000000140059258     msvcrt:utility.obj
 0002:0000e258       $unwind$??1?$map@GPEAUtagIP4Address@@U?$less@G@std@@V?$allocator@U?$pair@$$CBGPEAUtagIP4Address@@@std@@@3@@std@@QEAA@XZ 0000000140059258     cSnmpEX.obj
 0002:0000e258       $unwind$?pre_c_initialization@@YAHXZ 0000000140059258     msvcrt:exe_winmain.obj
 0002:0000e258       $unwind$__scrt_uninitialize_crt 0000000140059258     msvcrt:utility.obj
 0002:0000e258       $unwind$?_Tidy@?$vector@DV?$allocator@D@std@@@std@@AEAAXXZ 0000000140059258     mailer.obj
 0002:0000e258       $unwind$?_Tidy@?$vector@UPART_PACKET@@V?$allocator@UPART_PACKET@@@std@@@std@@AEAAXXZ 0000000140059258     DivisionPacket.obj
 0002:0000e258       $unwind$??$_Buynode@AEBUpiecewise_construct_t@std@@V?$tuple@AEBI@2@V?$tuple@$$V@2@@?$_Tree_comp_alloc@V?$_Tmap_traits@IUPORTINFO@@U?$less@I@std@@V?$allocator@U?$pair@$$CBIUPORTINFO@@@std@@@3@$0A@@std@@@std@@QEAAPEAU?$_Tree_node@U?$pair@$$CBIUPORTINFO@@@std@@PEAX@1@AEBUpiecewise_construct_t@1@$$QEAV?$tuple@AEBI@1@$$QEAV?$tuple@$$V@1@@Z 0000000140059258     GameServerManagerDlg.obj
 0002:0000e258       $unwind$__scrt_release_startup_lock 0000000140059258     msvcrt:utility.obj
 0002:0000e258       $unwind$??0BATTLE_ROYAL_RESULT@@QEAA@XZ 0000000140059258     GameServerManagerDlg.obj
 0002:0000e258       $unwind$?_Tidy_deallocate@?$basic_string@_WU?$char_traits@_W@std@@V?$allocator@_W@2@@std@@QEAAXXZ 0000000140059258     crs_uploader.obj
 0002:0000e258       $unwind$?_Buynode0@?$_Tree_comp_alloc@V?$_Tmap_traits@V?$basic_string@DU?$char_traits@D@std@@V?$allocator@D@2@@std@@PEAVCIniSection@CIniReader@@U?$less@V?$basic_string@DU?$char_traits@D@std@@V?$allocator@D@2@@std@@@2@V?$allocator@U?$pair@$$CBV?$basic_string@DU?$char_traits@D@std@@V?$allocator@D@2@@std@@PEAVCIniSection@CIniReader@@@std@@@2@$0A@@std@@@std@@QEAAPEAU?$_Tree_node@U?$pair@$$CBV?$basic_string@DU?$char_traits@D@std@@V?$allocator@D@2@@std@@PEAVCIniSection@CIniReader@@@std@@PEAX@2@XZ 0000000140059258     iniReader.obj
 0002:0000e258       $unwind$?OnDisconnect@CGameServerManagerDlg@@UEAAXXZ 0000000140059258     GameServerManagerDlg.obj
 0002:0000e258       $unwind$??$?HDU?$char_traits@D@std@@V?$allocator@D@1@@std@@YA?AV?$basic_string@DU?$char_traits@D@std@@V?$allocator@D@2@@0@$$QEAV10@QEBD@Z 0000000140059258     iniReader.obj
 0002:0000e258       $unwind$??_D?$basic_stringstream@DU?$char_traits@D@std@@V?$allocator@D@2@@std@@QEAAXXZ 0000000140059258     safe_string_x64:safe_string.obj
 0002:0000e258       $unwind$??1?$basic_string@_WU?$char_traits@_W@std@@V?$allocator@_W@2@@std@@QEAA@XZ 0000000140059258     crs_uploader.obj
 0002:0000e258       $unwind$??$_Buynode@AEBUpiecewise_construct_t@std@@V?$tuple@$$QEAV?$basic_string@DU?$char_traits@D@std@@V?$allocator@D@2@@std@@@2@V?$tuple@$$V@2@@?$_Tree_comp_alloc@V?$_Tmap_traits@V?$basic_string@DU?$char_traits@D@std@@V?$allocator@D@2@@std@@V12@U?$less@V?$basic_string@DU?$char_traits@D@std@@V?$allocator@D@2@@std@@@2@V?$allocator@U?$pair@$$CBV?$basic_string@DU?$char_traits@D@std@@V?$allocator@D@2@@std@@V12@@std@@@2@$0A@@std@@@std@@QEAAPEAU?$_Tree_node@U?$pair@$$CBV?$basic_string@DU?$char_traits@D@std@@V?$allocator@D@2@@std@@V12@@std@@PEAX@1@AEBUpiecewise_construct_t@1@$$QEAV?$tuple@$$QEAV?$basic_string@DU?$char_traits@D@std@@V?$allocator@D@2@@std@@@1@$$QEAV?$tuple@$$V@1@@Z 0000000140059258     iniReader.obj
 0002:0000e258       $unwind$??_GIClientHandler@@UEAAPEAXI@Z 0000000140059258     GameServerManagerDlg.obj
 0002:0000e258       $unwind$?_Tidy@?$vector@USOCKADDR_IN@jwsmtp@@V?$allocator@USOCKADDR_IN@jwsmtp@@@std@@@std@@AEAAXXZ 0000000140059258     mailer.obj
 0002:0000e258       $unwind$??_Gtype_info@@UEAAPEAXI@Z 0000000140059258     msvcrt:std_type_info_static.obj
 0002:0000e258       $unwind$?_Extract@?$_Tree_val@U?$_Tree_simple_types@U?$pair@$$CBIUPORTINFO@@@std@@@std@@@std@@QEAAPEAU?$_Tree_node@U?$pair@$$CBIUPORTINFO@@@std@@PEAX@2@V?$_Tree_const_iterator@V?$_Tree_val@U?$_Tree_simple_types@U?$pair@$$CBIUPORTINFO@@@std@@@std@@@std@@@2@@Z 0000000140059258     GameServerManagerDlg.obj
 0002:0000e258       $unwind$??1CIniReader@@QEAA@XZ 0000000140059258     iniReader.obj
 0002:0000e258       $unwind$??$_Buynode@AEBUpiecewise_construct_t@std@@V?$tuple@AEB_J@2@V?$tuple@$$V@2@@?$_Tree_comp_alloc@V?$_Tmap_traits@_JV?$basic_string@DU?$char_traits@D@std@@V?$allocator@D@2@@std@@U?$less@_J@2@V?$allocator@U?$pair@$$CB_JV?$basic_string@DU?$char_traits@D@std@@V?$allocator@D@2@@std@@@std@@@2@$0A@@std@@@std@@QEAAPEAU?$_Tree_node@U?$pair@$$CB_JV?$basic_string@DU?$char_traits@D@std@@V?$allocator@D@2@@std@@@std@@PEAX@1@AEBUpiecewise_construct_t@1@$$QEAV?$tuple@AEB_J@1@$$QEAV?$tuple@$$V@1@@Z 0000000140059258     LoadXlsMsg.obj
 0002:0000e258       $unwind$?_Buynode0@?$_Tree_comp_alloc@V?$_Tmap_traits@GUExtraStatsFPSVerify@CHostStat@@U?$less@G@std@@V?$allocator@U?$pair@$$CBGUExtraStatsFPSVerify@CHostStat@@@std@@@4@$0A@@std@@@std@@QEAAPEAU?$_Tree_node@U?$pair@$$CBGUExtraStatsFPSVerify@CHostStat@@@std@@PEAX@2@XZ 0000000140059258     HostStat.obj
 0002:0000e258       $unwind$?_Destroy_if_node@?$_Tree@V?$_Tmap_traits@_JVDivisionPacket@@U?$less@_J@std@@V?$allocator@U?$pair@$$CB_JVDivisionPacket@@@std@@@3@$0A@@std@@@std@@IEAAXPEAU?$_Tree_node@U?$pair@$$CB_JVDivisionPacket@@@std@@PEAX@2@@Z 0000000140059258     DivisionPacketReceiver.obj
 0002:0000e258       $unwind$?_Tidy_deallocate@?$basic_string@DU?$char_traits@D@std@@V?$allocator@D@2@@std@@QEAAXXZ 0000000140059258     BugReporter.obj
 0002:0000e258       $unwind$??0exception@std@@QEAA@AEBV01@@Z 0000000140059258     AppInfoDlg.obj
 0002:0000e258       $unwind$??1?$vector@DV?$allocator@D@std@@@std@@QEAA@XZ 0000000140059258     mailer.obj
 0002:0000e258       $unwind$??$_Buynode@AEBUverifyTerminationStatus_t@@@?$_List_buy@UverifyTerminationStatus_t@@V?$allocator@UverifyTerminationStatus_t@@@std@@@std@@QEAAPEAU?$_List_node@UverifyTerminationStatus_t@@PEAX@1@PEAU21@0AEBUverifyTerminationStatus_t@@@Z 0000000140059258     GameServerManagerDlg.obj
 0002:0000e258       $unwind$?_Buynode0@?$_Tree_comp_alloc@V?$_Tmap_traits@GUExtraStatsMemVerify@CHostStat@@U?$less@G@std@@V?$allocator@U?$pair@$$CBGUExtraStatsMemVerify@CHostStat@@@std@@@4@$0A@@std@@@std@@QEAAPEAU?$_Tree_node@U?$pair@$$CBGUExtraStatsMemVerify@CHostStat@@@std@@PEAX@2@XZ 0000000140059258     HostStat.obj
 0002:0000e258       $unwind$??1?$map@IUPORTINFO@@U?$less@I@std@@V?$allocator@U?$pair@$$CBIUPORTINFO@@@std@@@3@@std@@QEAA@XZ 0000000140059258     GameServerManagerDlg.obj
 0002:0000e258       $unwind$?Release@CSharedMemoryLoader@@QEAA_NXZ 0000000140059258     GameServerManagerDlg.obj
 0002:0000e258       $unwind$?_Destroy_if_node@?$_Tree@V?$_Tmap_traits@_JV?$basic_string@DU?$char_traits@D@std@@V?$allocator@D@2@@std@@U?$less@_J@2@V?$allocator@U?$pair@$$CB_JV?$basic_string@DU?$char_traits@D@std@@V?$allocator@D@2@@std@@@std@@@2@$0A@@std@@@std@@IEAAXPEAU?$_Tree_node@U?$pair@$$CB_JV?$basic_string@DU?$char_traits@D@std@@V?$allocator@D@2@@std@@@std@@PEAX@2@@Z 0000000140059258     LoadXlsMsg.obj
 0002:0000e258       $unwind$??1Uploader@crs@@QEAA@XZ 0000000140059258     crs_uploader.obj
 0002:0000e258       $unwind$?_Buynode0@?$_Tree_comp_alloc@V?$_Tmap_traits@_JVDivisionPacket@@U?$less@_J@std@@V?$allocator@U?$pair@$$CB_JVDivisionPacket@@@std@@@3@$0A@@std@@@std@@QEAAPEAU?$_Tree_node@U?$pair@$$CB_JVDivisionPacket@@@std@@PEAX@2@XZ 0000000140059258     DivisionPacketReceiver.obj
 0002:0000e258       $unwind$?_Destroy_if_node@?$_Tree@V?$_Tmap_traits@V?$basic_string@DU?$char_traits@D@std@@V?$allocator@D@2@@std@@PEAVCIniSection@CIniReader@@U?$less@V?$basic_string@DU?$char_traits@D@std@@V?$allocator@D@2@@std@@@2@V?$allocator@U?$pair@$$CBV?$basic_string@DU?$char_traits@D@std@@V?$allocator@D@2@@std@@PEAVCIniSection@CIniReader@@@std@@@2@$0A@@std@@@std@@IEAAXPEAU?$_Tree_node@U?$pair@$$CBV?$basic_string@DU?$char_traits@D@std@@V?$allocator@D@2@@std@@PEAVCIniSection@CIniReader@@@std@@PEAX@2@@Z 0000000140059258     iniReader.obj
 0002:0000e258       $unwind$_Init_thread_wait  0000000140059258     msvcrt:thread_safe_statics.obj
 0002:0000e258       $unwind$??_G?$_Ref_count@UGAMESERVERINFO@@@std@@UEAAPEAXI@Z 0000000140059258     GameServerManagerDlg.obj
 0002:0000e258       $unwind$??1CServerLog@@UEAA@XZ 0000000140059258     LogMgmt.obj
 0002:0000e258       $unwind$??$_Buynode@U?$pair@GUExtraStatsMemVerify@CHostStat@@@std@@@?$_Tree_comp_alloc@V?$_Tmap_traits@GUExtraStatsMemVerify@CHostStat@@U?$less@G@std@@V?$allocator@U?$pair@$$CBGUExtraStatsMemVerify@CHostStat@@@std@@@4@$0A@@std@@@std@@QEAAPEAU?$_Tree_node@U?$pair@$$CBGUExtraStatsMemVerify@CHostStat@@@std@@PEAX@1@$$QEAU?$pair@GUExtraStatsMemVerify@CHostStat@@@1@@Z 0000000140059258     HostStat.obj
 0002:0000e258       $unwind$??1Address@mailer@jwsmtp@@QEAA@XZ 0000000140059258     mailer.obj
 0002:0000e258       $unwind$??1?$vector@USOCKADDR_IN@jwsmtp@@V?$allocator@USOCKADDR_IN@jwsmtp@@@std@@@std@@QEAA@XZ 0000000140059258     mailer.obj
 0002:0000e258       $unwind$?_Buynode0@?$_Tree_comp_alloc@V?$_Tmap_traits@V?$basic_string@DU?$char_traits@D@std@@V?$allocator@D@2@@std@@V12@U?$less@V?$basic_string@DU?$char_traits@D@std@@V?$allocator@D@2@@std@@@2@V?$allocator@U?$pair@$$CBV?$basic_string@DU?$char_traits@D@std@@V?$allocator@D@2@@std@@V12@@std@@@2@$0A@@std@@@std@@QEAAPEAU?$_Tree_node@U?$pair@$$CBV?$basic_string@DU?$char_traits@D@std@@V?$allocator@D@2@@std@@V12@@std@@PEAX@2@XZ 0000000140059258     iniReader.obj
 0002:0000e258       $unwind$??_GCPacket@@UEAAPEAXI@Z 0000000140059258     Packet.obj
 0002:0000e258       $unwind$??1?$auto_ptr@VUrl@crs@@@std@@QEAA@XZ 0000000140059258     crs_uploader.obj
 0002:0000e258       $unwind$??1?$basic_string@DU?$char_traits@D@std@@V?$allocator@D@2@@std@@QEAA@XZ 0000000140059258     BugReporter.obj
 0002:0000e258       $unwind$?substr@?$basic_string@DU?$char_traits@D@std@@V?$allocator@D@2@@std@@QEBA?AV12@_K0@Z 0000000140059258     GameServerManagerDlg.obj
 0002:0000e258       $unwind$??1CSharedMemoryLoader@@QEAA@XZ 0000000140059258     GameServerManagerDlg.obj
 0002:0000e258       $unwind$??1?$map@GUExtraStatsFPSVerify@CHostStat@@U?$less@G@std@@V?$allocator@U?$pair@$$CBGUExtraStatsFPSVerify@CHostStat@@@std@@@4@@std@@QEAA@XZ 0000000140059258     HostStat.obj
 0002:0000e258       $unwind$?_Destroy_if_node@?$_Tree@V?$_Tmap_traits@V?$basic_string@DU?$char_traits@D@std@@V?$allocator@D@2@@std@@V12@U?$less@V?$basic_string@DU?$char_traits@D@std@@V?$allocator@D@2@@std@@@2@V?$allocator@U?$pair@$$CBV?$basic_string@DU?$char_traits@D@std@@V?$allocator@D@2@@std@@V12@@std@@@2@$0A@@std@@@std@@IEAAXPEAU?$_Tree_node@U?$pair@$$CBV?$basic_string@DU?$char_traits@D@std@@V?$allocator@D@2@@std@@V12@@std@@PEAX@2@@Z 0000000140059258     iniReader.obj
 0002:0000e258       $unwind$_Init_thread_footer 0000000140059258     msvcrt:thread_safe_statics.obj
 0002:0000e258       $unwind$??1CAtlBaseModule@ATL@@QEAA@XZ 0000000140059258     atls:atlbase.obj
 0002:0000e258       $unwind$??1?$basic_stringbuf@DU?$char_traits@D@std@@V?$allocator@D@2@@std@@UEAA@XZ 0000000140059258     safe_string_x64:safe_string.obj
 0002:0000e258       $unwind$?TerminateGSThread@CGameServerManagerDlg@@SAIPEAX@Z 0000000140059258     GameServerManagerDlg.obj
 0002:0000e258       $unwind$??$_Buynode@U?$pair@GUExtraStatsFPSVerify@CHostStat@@@std@@@?$_Tree_comp_alloc@V?$_Tmap_traits@GUExtraStatsFPSVerify@CHostStat@@U?$less@G@std@@V?$allocator@U?$pair@$$CBGUExtraStatsFPSVerify@CHostStat@@@std@@@4@$0A@@std@@@std@@QEAAPEAU?$_Tree_node@U?$pair@$$CBGUExtraStatsFPSVerify@CHostStat@@@std@@PEAX@1@$$QEAU?$pair@GUExtraStatsFPSVerify@CHostStat@@@1@@Z 0000000140059258     HostStat.obj
 0002:0000e258       $unwind$__raise_securityfailure 0000000140059258     msvcrt:gs_report.obj
 0002:0000e258       $unwind$??1CSFGameServerClientLib@@UEAA@XZ 0000000140059258     SFGameServerClientLib.obj
 0002:0000e258       $unwind$_Init_thread_abort 0000000140059258     msvcrt:thread_safe_statics.obj
 0002:0000e258       $unwind$?_Buynode0@?$_Tree_comp_alloc@V?$_Tmap_traits@_JV?$basic_string@DU?$char_traits@D@std@@V?$allocator@D@2@@std@@U?$less@_J@2@V?$allocator@U?$pair@$$CB_JV?$basic_string@DU?$char_traits@D@std@@V?$allocator@D@2@@std@@@std@@@2@$0A@@std@@@std@@QEAAPEAU?$_Tree_node@U?$pair@$$CB_JV?$basic_string@DU?$char_traits@D@std@@V?$allocator@D@2@@std@@@std@@PEAX@2@XZ 0000000140059258     LoadXlsMsg.obj
 0002:0000e258       $unwind$??$endl@DU?$char_traits@D@std@@@std@@YAAEAV?$basic_ostream@DU?$char_traits@D@std@@@0@AEAV10@@Z 0000000140059258     md5_csmtp.obj
 0002:0000e258       $unwind$??0?$basic_string@DU?$char_traits@D@std@@V?$allocator@D@2@@std@@QEAA@QEBD@Z 0000000140059258     BugReporter.obj
 0002:0000e258       $unwind$?_Tidy@?$vector@V?$basic_string@DU?$char_traits@D@std@@V?$allocator@D@2@@std@@V?$allocator@V?$basic_string@DU?$char_traits@D@std@@V?$allocator@D@2@@std@@@2@@std@@AEAAXXZ 0000000140059258     CSmtp.obj
 0002:0000e258       $unwind$_Init_thread_header 0000000140059258     msvcrt:thread_safe_statics.obj
 0002:0000e258       $unwind$?OnInitDialog@CGameServerManagerDlg@@MEAAHXZ 0000000140059258     GameServerManagerDlg.obj
 0002:0000e258       $unwind$??1?$vector@V?$basic_string@DU?$char_traits@D@std@@V?$allocator@D@2@@std@@V?$allocator@V?$basic_string@DU?$char_traits@D@std@@V?$allocator@D@2@@std@@@2@@std@@QEAA@XZ 0000000140059258     CSmtp.obj
 0002:0000e258       $unwind$??0PROTO_USER_STAT_tag@@QEAA@XZ 0000000140059258     GameServerManagerDlg.obj
 0002:0000e260       $unwind$??$_Emplace_reallocate@AEBUPART_PACKET@@@?$vector@UPART_PACKET@@V?$allocator@UPART_PACKET@@@std@@@std@@QEAAPEAUPART_PACKET@@QEAU2@AEBU2@@Z 0000000140059260     DivisionPacket.obj
 0002:0000e270       $chain$3$??$_Emplace_reallocate@AEBUPART_PACKET@@@?$vector@UPART_PACKET@@V?$allocator@UPART_PACKET@@@std@@@std@@QEAAPEAUPART_PACKET@@QEAU2@AEBU2@@Z 0000000140059270     DivisionPacket.obj
 0002:0000e290       $chain$5$??$_Emplace_reallocate@AEBUPART_PACKET@@@?$vector@UPART_PACKET@@V?$allocator@UPART_PACKET@@@std@@@std@@QEAAPEAUPART_PACKET@@QEAU2@AEBU2@@Z 0000000140059290     DivisionPacket.obj
 0002:0000e2b0       $chain$6$??$_Emplace_reallocate@AEBUPART_PACKET@@@?$vector@UPART_PACKET@@V?$allocator@UPART_PACKET@@@std@@@std@@QEAAPEAUPART_PACKET@@QEAU2@AEBU2@@Z 00000001400592b0     DivisionPacket.obj
 0002:0000e2c0       $unwind$__report_rangecheckfailure 00000001400592c0     msvcrt:gs_report.obj
 0002:0000e2c0       $unwind$??__E?m_LogPacketLock@CHLogger@@0VCMustSyncObjectLog@@A@@YAXXZ 00000001400592c0     HostLogger.obj
 0002:0000e2c0       $unwind$?_Buyheadnode@?$_Tree_comp_alloc@V?$_Tmap_traits@_JVDivisionPacket@@U?$less@_J@std@@V?$allocator@U?$pair@$$CB_JVDivisionPacket@@@std@@@3@$0A@@std@@@std@@QEAAPEAU?$_Tree_node@U?$pair@$$CB_JVDivisionPacket@@@std@@PEAX@2@XZ 00000001400592c0     DivisionPacketReceiver.obj
 0002:0000e2c0       $unwind$?post_pgo_initialization@@YAHXZ 00000001400592c0     msvcrt:exe_winmain.obj
 0002:0000e2c0       $unwind$??__EtheApp@@YAXXZ 00000001400592c0     GameServerManager.obj
 0002:0000e2c0       $unwind$?_Xlength@?$vector@U?$pair@UAddress@mailer@jwsmtp@@F@std@@V?$allocator@U?$pair@UAddress@mailer@jwsmtp@@F@std@@@2@@std@@CAXXZ 00000001400592c0     mailer.obj
 0002:0000e2c0       $unwind$?pre_cpp_initialization@@YAXXZ 00000001400592c0     msvcrt:exe_winmain.obj
 0002:0000e2c0       $unwind$?_Xlength@?$vector@PEAXV?$allocator@PEAX@std@@@std@@CAXXZ 00000001400592c0     LogMsgManager.obj
 0002:0000e2c0       $unwind$WinMainCRTStartup  00000001400592c0     msvcrt:exe_winmain.obj
 0002:0000e2c0       $unwind$?_Xlength@?$vector@USOCKADDR_IN@jwsmtp@@V?$allocator@USOCKADDR_IN@jwsmtp@@@std@@@std@@CAXXZ 00000001400592c0     mailer.obj
 0002:0000e2c0       $unwind$?_Xlength@?$vector@DV?$allocator@D@std@@@std@@CAXXZ 00000001400592c0     mailer.obj
 0002:0000e2c0       $unwind$?_Xlen@?$basic_string@_WU?$char_traits@_W@std@@V?$allocator@_W@2@@std@@SAXXZ 00000001400592c0     crs_uploader.obj
 0002:0000e2c0       $unwind$??$?9DU?$char_traits@D@std@@V?$allocator@D@1@@std@@YA_NAEBV?$basic_string@DU?$char_traits@D@std@@V?$allocator@D@2@@0@0@Z 00000001400592c0     mailer.obj
 0002:0000e2c0       $unwind$?_Buyheadnode@?$_Tree_comp_alloc@V?$_Tmap_traits@_JV?$basic_string@DU?$char_traits@D@std@@V?$allocator@D@2@@std@@U?$less@_J@2@V?$allocator@U?$pair@$$CB_JV?$basic_string@DU?$char_traits@D@std@@V?$allocator@D@2@@std@@@std@@@2@$0A@@std@@@std@@QEAAPEAU?$_Tree_node@U?$pair@$$CB_JV?$basic_string@DU?$char_traits@D@std@@V?$allocator@D@2@@std@@@std@@PEAX@2@XZ 00000001400592c0     LoadXlsMsg.obj
 0002:0000e2c0       $unwind$??__F?m_strModeUserCountFormat@CHLogger@@0V?$basic_string@DU?$char_traits@D@std@@V?$allocator@D@2@@std@@A@@YAXXZ 00000001400592c0     HostLogger.obj
 0002:0000e2c0       $unwind$?_Buyheadnode@?$_Tree_comp_alloc@V?$_Tmap_traits@GUExtraStatsMemVerify@CHostStat@@U?$less@G@std@@V?$allocator@U?$pair@$$CBGUExtraStatsMemVerify@CHostStat@@@std@@@4@$0A@@std@@@std@@QEAAPEAU?$_Tree_node@U?$pair@$$CBGUExtraStatsMemVerify@CHostStat@@@std@@PEAX@2@XZ 00000001400592c0     HostStat.obj
 0002:0000e2c0       $unwind$?_Equal@?$basic_string@DU?$char_traits@D@std@@V?$allocator@D@2@@std@@QEBA_NQEBD@Z 00000001400592c0     mailer.obj
 0002:0000e2c0       $unwind$?_Xran@?$_String_val@U?$_Simple_types@D@std@@@std@@SAXXZ 00000001400592c0     GameServerManagerDlg.obj
 0002:0000e2c0       $unwind$?_Buyheadnode@?$_Tree_comp_alloc@V?$_Tmap_traits@GUExtraStatsFPSVerify@CHostStat@@U?$less@G@std@@V?$allocator@U?$pair@$$CBGUExtraStatsFPSVerify@CHostStat@@@std@@@4@$0A@@std@@@std@@QEAAPEAU?$_Tree_node@U?$pair@$$CBGUExtraStatsFPSVerify@CHostStat@@@std@@PEAX@2@XZ 00000001400592c0     HostStat.obj
 0002:0000e2c0       $unwind$??$?9DU?$char_traits@D@std@@V?$allocator@D@1@@std@@YA_NAEBV?$basic_string@DU?$char_traits@D@std@@V?$allocator@D@2@@0@QEBD@Z 00000001400592c0     mailer.obj
 0002:0000e2c0       $unwind$??__F?m_strLogFolder@CHLogger@@0V?$basic_string@DU?$char_traits@D@std@@V?$allocator@D@2@@std@@A@@YAXXZ 00000001400592c0     HostLogger.obj
 0002:0000e2c0       $unwind$??__F?m_strServerName@CHLogger@@0V?$basic_string@DU?$char_traits@D@std@@V?$allocator@D@2@@std@@A@@YAXXZ 00000001400592c0     HostLogger.obj
 0002:0000e2c0       $unwind$??__F?m_strHostName@CHLogger@@0V?$basic_string@DU?$char_traits@D@std@@V?$allocator@D@2@@std@@A@@YAXXZ 00000001400592c0     HostLogger.obj
 0002:0000e2c0       $unwind$__scrt_is_managed_app 00000001400592c0     msvcrt:utility_desktop.obj
 0002:0000e2c0       $unwind$??__F?m_strTimeOutFileFormat@CHLogger@@0V?$basic_string@DU?$char_traits@D@std@@V?$allocator@D@2@@std@@A@@YAXXZ 00000001400592c0     HostLogger.obj
 0002:0000e2c0       $unwind$?_Xlen@?$basic_string@DU?$char_traits@D@std@@V?$allocator@D@2@@std@@SAXXZ 00000001400592c0     BugReporter.obj
 0002:0000e2c0       $unwind$??__E?m_LogLock@CHLogger@@0VCMustSyncObjectLog@@A@@YAXXZ 00000001400592c0     HostLogger.obj
 0002:0000e2c0       $unwind$??__Ebase64_chars@@YAXXZ 00000001400592c0     base64.obj
 0002:0000e2c0       $unwind$??__F?m_strPacketFileFormat@CHLogger@@0V?$basic_string@DU?$char_traits@D@std@@V?$allocator@D@2@@std@@A@@YAXXZ 00000001400592c0     HostLogger.obj
 0002:0000e2c0       $unwind$??__F?m_strIPCMessageFileFormat@CHLogger@@0V?$basic_string@DU?$char_traits@D@std@@V?$allocator@D@2@@std@@A@@YAXXZ 00000001400592c0     HostLogger.obj
 0002:0000e2c0       $unwind$__scrt_unhandled_exception_filter 00000001400592c0     msvcrt:utility_desktop.obj
 0002:0000e2c0       $unwind$??__F?m_strRWProcessMemoryFileFormat@CHLogger@@0V?$basic_string@DU?$char_traits@D@std@@V?$allocator@D@2@@std@@A@@YAXXZ 00000001400592c0     HostLogger.obj
 0002:0000e2c0       $unwind$?_Xlength@?$vector@V?$basic_string@DU?$char_traits@D@std@@V?$allocator@D@2@@std@@V?$allocator@V?$basic_string@DU?$char_traits@D@std@@V?$allocator@D@2@@std@@@2@@std@@CAXXZ 00000001400592c0     CSmtp.obj
 0002:0000e2c0       $unwind$??__F?m_strFileFormat@CHLogger@@0V?$basic_string@DU?$char_traits@D@std@@V?$allocator@D@2@@std@@A@@YAXXZ 00000001400592c0     HostLogger.obj
 0002:0000e2c0       $unwind$??__F?m_strBRFileFormat@CHLogger@@0V?$basic_string@DU?$char_traits@D@std@@V?$allocator@D@2@@std@@A@@YAXXZ 00000001400592c0     HostLogger.obj
 0002:0000e2c0       $unwind$??__F?m_strKernelFileFormat@CHLogger@@0V?$basic_string@DU?$char_traits@D@std@@V?$allocator@D@2@@std@@A@@YAXXZ 00000001400592c0     HostLogger.obj
 0002:0000e2c0       $unwind$__scrt_initialize_default_local_stdio_options 00000001400592c0     msvcrt:default_local_stdio_options.obj
 0002:0000e2c0       $unwind$??__F?m_strEtcFileFormat@CHLogger@@0V?$basic_string@DU?$char_traits@D@std@@V?$allocator@D@2@@std@@A@@YAXXZ 00000001400592c0     HostLogger.obj
 0002:0000e2c0       $unwind$??__F?m_vectSharedMapHandles@CLogMsgManager@@0V?$vector@PEAXV?$allocator@PEAX@std@@@std@@A@@YAXXZ 00000001400592c0     LogMsgManager.obj
 0002:0000e2c0       $unwind$??__Ea@VectorSinConstantsSSE@@YAXXZ 00000001400592c0     StdAfx.obj
 0002:0000e2c0       $unwind$??__Eb@VectorSinConstantsSSE@@YAXXZ 00000001400592c0     StdAfx.obj
 0002:0000e2c0       $unwind$?deallocate@?$allocator@V?$basic_string@DU?$char_traits@D@std@@V?$allocator@D@2@@std@@@std@@QEAAXQEAV?$basic_string@DU?$char_traits@D@std@@V?$allocator@D@2@@2@_K@Z 00000001400592c0     CSmtp.obj
 0002:0000e2c0       $unwind$??__E_afxInitAppState@@YAXXZ 00000001400592c0     mfcs140:appmodul.obj
 0002:0000e2c0       $unwind$??__EPI@@YAXXZ     00000001400592c0     StdAfx.obj
 0002:0000e2c0       $unwind$??__E__iob_func@@YAXXZ 00000001400592c0     StdAfx.obj
 0002:0000e2c0       $unwind$__GSHandlerCheck   00000001400592c0     msvcrt:gshandler.obj
 0002:0000e2c0       $unwind$_Init_thread_notify 00000001400592c0     msvcrt:thread_safe_statics.obj
 0002:0000e2c0       $unwind$?_Buyheadnode@?$_Tree_comp_alloc@V?$_Tmap_traits@IUPORTINFO@@U?$less@I@std@@V?$allocator@U?$pair@$$CBIUPORTINFO@@@std@@@3@$0A@@std@@@std@@QEAAPEAU?$_Tree_node@U?$pair@$$CBIUPORTINFO@@@std@@PEAX@2@XZ 00000001400592c0     GameServerManagerDlg.obj
 0002:0000e2c0       $unwind$??__F?m_strServerAppUseCountFormat@CHLogger@@0V?$basic_string@DU?$char_traits@D@std@@V?$allocator@D@2@@std@@A@@YAXXZ 00000001400592c0     HostLogger.obj
 0002:0000e2c0       $unwind$?__scrt_uninitialize_thread_safe_statics@@YAXXZ 00000001400592c0     msvcrt:thread_safe_statics.obj
 0002:0000e2c0       $unwind$?MyServiceHandler@@YAXK@Z 00000001400592c0     GameServerManager.obj
 0002:0000e2c0       $unwind$??__E_AtlBaseModule@ATL@@YAXXZ 00000001400592c0     atls:atlbase.obj
 0002:0000e2c0       $unwind$?_Buyheadnode@?$_Tree_comp_alloc@V?$_Tmap_traits@GPEAUtagIP4Address@@U?$less@G@std@@V?$allocator@U?$pair@$$CBGPEAUtagIP4Address@@@std@@@3@$0A@@std@@@std@@QEAAPEAU?$_Tree_node@U?$pair@$$CBGPEAUtagIP4Address@@@std@@PEAX@2@XZ 00000001400592c0     cSnmpEX.obj
 0002:0000e2c0       $unwind$memcpy_s           00000001400592c0     GameServerManagerDlg.obj
 0002:0000e2c0       $unwind$??__Fbase64_chars@@YAXXZ 00000001400592c0     base64.obj
 0002:0000e2c0       $unwind$?_Xlength@?$vector@UPART_PACKET@@V?$allocator@UPART_PACKET@@@std@@@std@@CAXXZ 00000001400592c0     DivisionPacket.obj
 0002:0000e2c0       $unwind$__scrt_acquire_startup_lock 00000001400592c0     msvcrt:utility.obj
 0002:0000e2c0       $unwind$?_Buyheadnode@?$_Tree_comp_alloc@V?$_Tmap_traits@V?$basic_string@DU?$char_traits@D@std@@V?$allocator@D@2@@std@@PEAVCIniSection@CIniReader@@U?$less@V?$basic_string@DU?$char_traits@D@std@@V?$allocator@D@2@@std@@@2@V?$allocator@U?$pair@$$CBV?$basic_string@DU?$char_traits@D@std@@V?$allocator@D@2@@std@@PEAVCIniSection@CIniReader@@@std@@@2@$0A@@std@@@std@@QEAAPEAU?$_Tree_node@U?$pair@$$CBV?$basic_string@DU?$char_traits@D@std@@V?$allocator@D@2@@std@@PEAVCIniSection@CIniReader@@@std@@PEAX@2@XZ 00000001400592c0     iniReader.obj
 0002:0000e2c0       $unwind$atexit             00000001400592c0     msvcrt:utility.obj
 0002:0000e2c0       $unwind$?_Buyheadnode@?$_Tree_comp_alloc@V?$_Tmap_traits@V?$basic_string@DU?$char_traits@D@std@@V?$allocator@D@2@@std@@V12@U?$less@V?$basic_string@DU?$char_traits@D@std@@V?$allocator@D@2@@std@@@2@V?$allocator@U?$pair@$$CBV?$basic_string@DU?$char_traits@D@std@@V?$allocator@D@2@@std@@V12@@std@@@2@$0A@@std@@@std@@QEAAPEAU?$_Tree_node@U?$pair@$$CBV?$basic_string@DU?$char_traits@D@std@@V?$allocator@D@2@@std@@V12@@std@@PEAX@2@XZ 00000001400592c0     iniReader.obj
 0002:0000e2c8       $unwind$?ReleaseTCPPortAddressMap@cSnmpEX@@QEAAXXZ 00000001400592c8     cSnmpEX.obj
 0002:0000e2c8       $unwind$?ReleaseUDPPortAddressMap@cSnmpEX@@QEAAXXZ 00000001400592c8     cSnmpEX.obj
 0002:0000e2c8       $unwind$?_Erase@?$_Tree@V?$_Tmap_traits@V?$basic_string@DU?$char_traits@D@std@@V?$allocator@D@2@@std@@V12@U?$less@V?$basic_string@DU?$char_traits@D@std@@V?$allocator@D@2@@std@@@2@V?$allocator@U?$pair@$$CBV?$basic_string@DU?$char_traits@D@std@@V?$allocator@D@2@@std@@V12@@std@@@2@$0A@@std@@@std@@IEAAXPEAU?$_Tree_node@U?$pair@$$CBV?$basic_string@DU?$char_traits@D@std@@V?$allocator@D@2@@std@@V12@@std@@PEAX@2@@Z 00000001400592c8     iniReader.obj
 0002:0000e2c8       $unwind$memcpy_s           00000001400592c8     DivisionPacket.obj
 0002:0000e2c8       $unwind$??0GAMESERVERINFO@@QEAA@XZ 00000001400592c8     GameServerManagerDlg.obj
 0002:0000e2c8       $unwind$?CloseSocket@CClientLib@@MEAAHXZ 00000001400592c8     ClientLib.obj
 0002:0000e2c8       $unwind$??0PROTO_START_HOST_tag@@QEAA@XZ 00000001400592c8     DividePacket.obj
 0002:0000e2c8       $unwind$??0PROTO_GAME_ENDED_tag@@QEAA@XZ 00000001400592c8     GameServerManagerDlg.obj
 0002:0000e2c8       $unwind$?_Erase@?$_Tree@V?$_Tmap_traits@GUExtraStatsMemVerify@CHostStat@@U?$less@G@std@@V?$allocator@U?$pair@$$CBGUExtraStatsMemVerify@CHostStat@@@std@@@4@$0A@@std@@@std@@IEAAXPEAU?$_Tree_node@U?$pair@$$CBGUExtraStatsMemVerify@CHostStat@@@std@@PEAX@2@@Z 00000001400592c8     HostStat.obj
 0002:0000e2c8       $unwind$?_Erase@?$_Tree@V?$_Tmap_traits@GUExtraStatsFPSVerify@CHostStat@@U?$less@G@std@@V?$allocator@U?$pair@$$CBGUExtraStatsFPSVerify@CHostStat@@@std@@@4@$0A@@std@@@std@@IEAAXPEAU?$_Tree_node@U?$pair@$$CBGUExtraStatsFPSVerify@CHostStat@@@std@@PEAX@2@@Z 00000001400592c8     HostStat.obj
 0002:0000e2c8       $unwind$?_Erase@?$_Tree@V?$_Tmap_traits@GPEAUtagIP4Address@@U?$less@G@std@@V?$allocator@U?$pair@$$CBGPEAUtagIP4Address@@@std@@@3@$0A@@std@@@std@@IEAAXPEAU?$_Tree_node@U?$pair@$$CBGPEAUtagIP4Address@@@std@@PEAX@2@@Z 00000001400592c8     cSnmpEX.obj
 0002:0000e2c8       $unwind$?regulate@datetime@@QEAAXXZ 00000001400592c8     DateTime.obj
 0002:0000e2c8       $unwind$?DestroyManager@CGameServerManagerDlg@@QEAAXXZ 00000001400592c8     GameServerManagerDlg.obj
 0002:0000e2c8       $unwind$?_Erase@?$_Tree@V?$_Tmap_traits@IUPORTINFO@@U?$less@I@std@@V?$allocator@U?$pair@$$CBIUPORTINFO@@@std@@@3@$0A@@std@@@std@@IEAAXPEAU?$_Tree_node@U?$pair@$$CBIUPORTINFO@@@std@@PEAX@2@@Z 00000001400592c8     GameServerManagerDlg.obj
 0002:0000e2c8       $unwind$??_G?$basic_stringstream@DU?$char_traits@D@std@@V?$allocator@D@2@@std@@UEAAPEAXI@Z 00000001400592c8     safe_string_x64:safe_string.obj
 0002:0000e2c8       $unwind$?Recv@jwsmtp@@YA_NAEAH_KPEAD1H@Z 00000001400592c8     compat.obj
 0002:0000e2d8       $unwind$?Instance@DivisionPacketReceiver@@SAPEAV1@XZ 00000001400592d8     DivisionPacketReceiver.obj
 0002:0000e2e8       $stateUnwindMap$?Instance@DivisionPacketReceiver@@SAPEAV1@XZ 00000001400592e8     DivisionPacketReceiver.obj
 0002:0000e2f0       $ip2state$?Instance@DivisionPacketReceiver@@SAPEAV1@XZ 00000001400592f0     DivisionPacketReceiver.obj
 0002:0000e2f8       $unwind$??__Fthis_instance_@?1??Instance@DivisionPacketReceiver@@SAPEAV1@XZ@YAXXZ 00000001400592f8     DivisionPacketReceiver.obj
 0002:0000e310       $stateUnwindMap$??1_Fac_tidy_reg_t@std@@QEAA@XZ 0000000140059310     msvcprt:locale0_implib.obj
 0002:0000e310       $stateUnwindMap$?erase@?$_Tree@V?$_Tmap_traits@V?$basic_string@DU?$char_traits@D@std@@V?$allocator@D@2@@std@@PEAVCIniSection@CIniReader@@U?$less@V?$basic_string@DU?$char_traits@D@std@@V?$allocator@D@2@@std@@@2@V?$allocator@U?$pair@$$CBV?$basic_string@DU?$char_traits@D@std@@V?$allocator@D@2@@std@@PEAVCIniSection@CIniReader@@@std@@@2@$0A@@std@@@std@@QEAA?AV?$_Tree_iterator@V?$_Tree_val@U?$_Tree_simple_types@U?$pair@$$CBV?$basic_string@DU?$char_traits@D@std@@V?$allocator@D@2@@std@@PEAVCIniSection@CIniReader@@@std@@@std@@@std@@@2@V?$_Tree_const_iterator@V?$_Tree_val@U?$_Tree_simple_types@U?$pair@$$CBV?$basic_string@DU?$char_traits@D@std@@V?$allocator@D@2@@std@@PEAVCIniSection@CIniReader@@@std@@@std@@@std@@@2@0@Z 0000000140059310     iniReader.obj
 0002:0000e310       $stateUnwindMap$?__scrt_initialize_thread_safe_statics@@YAHXZ 0000000140059310     msvcrt:thread_safe_statics.obj
 0002:0000e310       $stateUnwindMap$??1CGameServerManagerDlg@@UEAA@XZ 0000000140059310     GameServerManagerDlg.obj
 0002:0000e310       $stateUnwindMap$?clear@CIniReader@@QEAAXXZ 0000000140059310     iniReader.obj
 0002:0000e310       $stateUnwindMap$?erase@?$_Tree@V?$_Tmap_traits@V?$basic_string@DU?$char_traits@D@std@@V?$allocator@D@2@@std@@V12@U?$less@V?$basic_string@DU?$char_traits@D@std@@V?$allocator@D@2@@std@@@2@V?$allocator@U?$pair@$$CBV?$basic_string@DU?$char_traits@D@std@@V?$allocator@D@2@@std@@V12@@std@@@2@$0A@@std@@@std@@QEAA?AV?$_Tree_iterator@V?$_Tree_val@U?$_Tree_simple_types@U?$pair@$$CBV?$basic_string@DU?$char_traits@D@std@@V?$allocator@D@2@@std@@V12@@std@@@std@@@std@@@2@V?$_Tree_const_iterator@V?$_Tree_val@U?$_Tree_simple_types@U?$pair@$$CBV?$basic_string@DU?$char_traits@D@std@@V?$allocator@D@2@@std@@V12@@std@@@std@@@std@@@2@0@Z 0000000140059310     iniReader.obj
 0002:0000e310       $stateUnwindMap$??1sentry@?$basic_ostream@DU?$char_traits@D@std@@@std@@QEAA@XZ 0000000140059310     md5_csmtp.obj
 0002:0000e310       $stateUnwindMap$??__Fthis_instance_@?1??Instance@DivisionPacketReceiver@@SAPEAV1@XZ@YAXXZ 0000000140059310     DivisionPacketReceiver.obj
 0002:0000e310       $stateUnwindMap$?erase@?$_Tree@V?$_Tmap_traits@_JV?$basic_string@DU?$char_traits@D@std@@V?$allocator@D@2@@std@@U?$less@_J@2@V?$allocator@U?$pair@$$CB_JV?$basic_string@DU?$char_traits@D@std@@V?$allocator@D@2@@std@@@std@@@2@$0A@@std@@@std@@QEAA?AV?$_Tree_iterator@V?$_Tree_val@U?$_Tree_simple_types@U?$pair@$$CB_JV?$basic_string@DU?$char_traits@D@std@@V?$allocator@D@2@@std@@@std@@@std@@@std@@@2@V?$_Tree_const_iterator@V?$_Tree_val@U?$_Tree_simple_types@U?$pair@$$CB_JV?$basic_string@DU?$char_traits@D@std@@V?$allocator@D@2@@std@@@std@@@std@@@std@@@2@0@Z 0000000140059310     LoadXlsMsg.obj
 0002:0000e310       $stateUnwindMap$??_GFindXlsMsg@@UEAAPEAXI@Z 0000000140059310     LoadXlsMsg.obj
 0002:0000e318       $ip2state$??__Fthis_instance_@?1??Instance@DivisionPacketReceiver@@SAPEAV1@XZ@YAXXZ 0000000140059318     DivisionPacketReceiver.obj
 0002:0000e320       $unwind$?GetPacketBuffer@DivisionPacketReceiver@@QEAA?BW4DIVISION_PACKET_RESULT@@EEEEEPEADG0H@Z 0000000140059320     DivisionPacketReceiver.obj
 0002:0000e33c       $stateUnwindMap$?GetPacketBuffer@DivisionPacketReceiver@@QEAA?BW4DIVISION_PACKET_RESULT@@EEEEEPEADG0H@Z 000000014005933c     DivisionPacketReceiver.obj
 0002:0000e350       $ip2state$?GetPacketBuffer@DivisionPacketReceiver@@QEAA?BW4DIVISION_PACKET_RESULT@@EEEEEPEADG0H@Z 0000000140059350     DivisionPacketReceiver.obj
 0002:0000e370       $unwind$?_Buynode0@?$_List_alloc@U?$_List_base_types@UverifyTerminationStatus_t@@V?$allocator@UverifyTerminationStatus_t@@@std@@@std@@@std@@QEAAPEAU?$_List_node@UverifyTerminationStatus_t@@PEAX@2@PEAU32@0@Z 0000000140059370     GameServerManagerDlg.obj
 0002:0000e370       $unwind$??1?$pair@V?$vector@DV?$allocator@D@std@@@std@@V?$basic_string@DU?$char_traits@D@std@@V?$allocator@D@2@@2@@std@@QEAA@XZ 0000000140059370     mailer.obj
 0002:0000e370       $unwind$??_GCEdit@@UEAAPEAXI@Z 0000000140059370     AppInfoDlg.obj
 0002:0000e370       $unwind$?WriteData@GAMEPROTO_SC_HOST_STAT@@UEAA_NPEAVILTMessage_Write@@@Z 0000000140059370     AppInfoDlg.obj
 0002:0000e370       $unwind$??_GMultiReceiver@sggm_proxy@@UEAAPEAXI@Z 0000000140059370     SGGMCallBackObj.obj
 0002:0000e370       $unwind$??_GCSGGMCallBackObj@@UEAAPEAXI@Z 0000000140059370     SGGMCallBackObj.obj
 0002:0000e370       $unwind$_RTC_Initialize    0000000140059370     msvcrt:initsect.obj
 0002:0000e370       $unwind$?DoDataExchange@CGameServerManagerDlg@@MEAAXPEAVCDataExchange@@@Z 0000000140059370     GameServerManagerDlg.obj
 0002:0000e370       $unwind$??_G?$basic_stringbuf@DU?$char_traits@D@std@@V?$allocator@D@2@@std@@UEAAPEAXI@Z 0000000140059370     safe_string_x64:safe_string.obj
 0002:0000e370       $unwind$?addcarry@datetime@@IEAAHAEAHHHH@Z 0000000140059370     DateTime.obj
 0002:0000e370       $unwind$??1cSnmpEX@@QEAA@XZ 0000000140059370     cSnmpEX.obj
 0002:0000e370       $unwind$??0CAtlBaseModule@ATL@@QEAA@XZ 0000000140059370     atls:atlbase.obj
 0002:0000e370       $unwind$??4?$basic_string@DU?$char_traits@D@std@@V?$allocator@D@2@@std@@QEAAAEAV01@$$QEAV01@@Z 0000000140059370     GameServerManagerDlg.obj
 0002:0000e370       $unwind$?Send@jwsmtp@@YA_NAEAH_KPEBD1H@Z 0000000140059370     compat.obj
 0002:0000e370       $unwind$??_GCGameServerManagerDlg@@UEAAPEAXI@Z 0000000140059370     GameServerManagerDlg.obj
 0002:0000e370       $unwind$??_GSendBuffer@@UEAAPEAXI@Z 0000000140059370     ClientLib.obj
 0002:0000e370       $unwind$?WriteData@GAMEPROTO_SC_REMOVECLIENT@@UEAA_NPEAVILTMessage_Write@@@Z 0000000140059370     AppInfoDlg.obj
 0002:0000e370       $unwind$?PostWriteData@GAMEPROTO_SC_COMMON@@UEAA_NPEAVILTMessage_Write@@@Z 0000000140059370     AppInfoDlg.obj
 0002:0000e370       $unwind$??_GCHostStat@@UEAAPEAXI@Z 0000000140059370     HostStat.obj
 0002:0000e370       $unwind$?PreReadData@GAMEPROTO_CS_COMMON@@UEAA_NPEAVILTMessage_Read@@@Z 0000000140059370     AppInfoDlg.obj
 0002:0000e370       $unwind$??0GAMEPROTO_SC_HOST_USER_STAT@@QEAA@XZ 0000000140059370     GameServerManagerDlg.obj
 0002:0000e370       $unwind$?PreWriteData@GAMEPROTO_CS_COMMON@@UEAA_NPEAVILTMessage_Write@@@Z 0000000140059370     AppInfoDlg.obj
 0002:0000e370       $unwind$?AfxInitialize@@YAHHK@Z 0000000140059370     mfcs140:appmodul.obj
 0002:0000e370       $unwind$?PostWriteData@GAMEPROTO_CS_COMMON@@UEAA_NPEAVILTMessage_Write@@@Z 0000000140059370     AppInfoDlg.obj
 0002:0000e370       $unwind$?ProcessSocketEventThread@CGameServerManagerDlg@@CAIPEAX@Z 0000000140059370     GameServerManagerDlg.obj
 0002:0000e370       $unwind$_RTC_Terminate     0000000140059370     msvcrt:initsect.obj
 0002:0000e370       $unwind$??_GCGameServerManagerApp@@UEAAPEAXI@Z 0000000140059370     GameServerManager.obj
 0002:0000e370       $unwind$?Init@GAMESERVERINFO@@QEAAXXZ 0000000140059370     GameServerManagerDlg.obj
 0002:0000e370       $unwind$??_GCClientLib@@UEAAPEAXI@Z 0000000140059370     ClientLib.obj
 0002:0000e370       $unwind$??_GCServerLog@@UEAAPEAXI@Z 0000000140059370     LogMgmt.obj
 0002:0000e370       $unwind$?_Erase@?$_Tree@V?$_Tmap_traits@_JVDivisionPacket@@U?$less@_J@std@@V?$allocator@U?$pair@$$CB_JVDivisionPacket@@@std@@@3@$0A@@std@@@std@@IEAAXPEAU?$_Tree_node@U?$pair@$$CB_JVDivisionPacket@@@std@@PEAX@2@@Z 0000000140059370     DivisionPacketReceiver.obj
 0002:0000e370       $unwind$??_Gexception@std@@UEAAPEAXI@Z 0000000140059370     AppInfoDlg.obj
 0002:0000e370       $unwind$??_GCMustSyncObjectLog@@UEAAPEAXI@Z 0000000140059370     HostLogger.obj
 0002:0000e370       $unwind$??_G?$CircuitQueue@E@@UEAAPEAXI@Z 0000000140059370     ClientLib.obj
 0002:0000e37c       $unwind$??0?$vector@UPART_PACKET@@V?$allocator@UPART_PACKET@@@std@@@std@@QEAA@AEBV01@@Z 000000014005937c     DivisionPacketReceiver.obj
 0002:0000e38c       $chain$0$??0?$vector@UPART_PACKET@@V?$allocator@UPART_PACKET@@@std@@@std@@QEAA@AEBV01@@Z 000000014005938c     DivisionPacketReceiver.obj
 0002:0000e3a0       $chain$1$??0?$vector@UPART_PACKET@@V?$allocator@UPART_PACKET@@@std@@@std@@QEAA@AEBV01@@Z 00000001400593a0     DivisionPacketReceiver.obj
 0002:0000e3b0       $unwind$??$_Buynode@U?$pair@_JVDivisionPacket@@@std@@@?$_Tree_comp_alloc@V?$_Tmap_traits@_JVDivisionPacket@@U?$less@_J@std@@V?$allocator@U?$pair@$$CB_JVDivisionPacket@@@std@@@3@$0A@@std@@@std@@QEAAPEAU?$_Tree_node@U?$pair@$$CB_JVDivisionPacket@@@std@@PEAX@1@$$QEAU?$pair@_JVDivisionPacket@@@1@@Z 00000001400593b0     DivisionPacketReceiver.obj
 0002:0000e3c4       $stateUnwindMap$??$_Insert_hint@AEAU?$pair@$$CB_JV?$basic_string@DU?$char_traits@D@std@@V?$allocator@D@2@@std@@@std@@PEAU?$_Tree_node@U?$pair@$$CB_JV?$basic_string@DU?$char_traits@D@std@@V?$allocator@D@2@@std@@@std@@PEAX@2@@?$_Tree@V?$_Tmap_traits@_JV?$basic_string@DU?$char_traits@D@std@@V?$allocator@D@2@@std@@U?$less@_J@2@V?$allocator@U?$pair@$$CB_JV?$basic_string@DU?$char_traits@D@std@@V?$allocator@D@2@@std@@@std@@@2@$0A@@std@@@std@@IEAA?AV?$_Tree_iterator@V?$_Tree_val@U?$_Tree_simple_types@U?$pair@$$CB_JV?$basic_string@DU?$char_traits@D@std@@V?$allocator@D@2@@std@@@std@@@std@@@std@@@1@V?$_Tree_const_iterator@V?$_Tree_val@U?$_Tree_simple_types@U?$pair@$$CB_JV?$basic_string@DU?$char_traits@D@std@@V?$allocator@D@2@@std@@@std@@@std@@@std@@@1@AEAU?$pair@$$CB_JV?$basic_string@DU?$char_traits@D@std@@V?$allocator@D@2@@std@@@1@PEAU?$_Tree_node@U?$pair@$$CB_JV?$basic_string@DU?$char_traits@D@std@@V?$allocator@D@2@@std@@@std@@PEAX@1@@Z 00000001400593c4     LoadXlsMsg.obj
 0002:0000e3c4       $stateUnwindMap$??$_Insert_nohint@AEAU?$pair@$$CBV?$basic_string@DU?$char_traits@D@std@@V?$allocator@D@2@@std@@V12@@std@@PEAU?$_Tree_node@U?$pair@$$CBV?$basic_string@DU?$char_traits@D@std@@V?$allocator@D@2@@std@@V12@@std@@PEAX@2@@?$_Tree@V?$_Tmap_traits@V?$basic_string@DU?$char_traits@D@std@@V?$allocator@D@2@@std@@V12@U?$less@V?$basic_string@DU?$char_traits@D@std@@V?$allocator@D@2@@std@@@2@V?$allocator@U?$pair@$$CBV?$basic_string@DU?$char_traits@D@std@@V?$allocator@D@2@@std@@V12@@std@@@2@$0A@@std@@@std@@IEAA?AU?$pair@V?$_Tree_iterator@V?$_Tree_val@U?$_Tree_simple_types@U?$pair@$$CBV?$basic_string@DU?$char_traits@D@std@@V?$allocator@D@2@@std@@V12@@std@@@std@@@std@@@std@@_N@1@_NAEAU?$pair@$$CBV?$basic_string@DU?$char_traits@D@std@@V?$allocator@D@2@@std@@V12@@1@PEAU?$_Tree_node@U?$pair@$$CBV?$basic_string@DU?$char_traits@D@std@@V?$allocator@D@2@@std@@V12@@std@@PEAX@1@@Z 00000001400593c4     iniReader.obj
 0002:0000e3c4       $stateUnwindMap$??$_Setp@UGAMESERVERINFO@@@?$shared_ptr@UGAMESERVERINFO@@@std@@AEAAXPEAUGAMESERVERINFO@@U?$integral_constant@_N$0A@@1@@Z 00000001400593c4     GameServerManagerDlg.obj
 0002:0000e3c4       $stateUnwindMap$??$_Insert_nohint@AEAU?$pair@$$CB_JV?$basic_string@DU?$char_traits@D@std@@V?$allocator@D@2@@std@@@std@@PEAU?$_Tree_node@U?$pair@$$CB_JV?$basic_string@DU?$char_traits@D@std@@V?$allocator@D@2@@std@@@std@@PEAX@2@@?$_Tree@V?$_Tmap_traits@_JV?$basic_string@DU?$char_traits@D@std@@V?$allocator@D@2@@std@@U?$less@_J@2@V?$allocator@U?$pair@$$CB_JV?$basic_string@DU?$char_traits@D@std@@V?$allocator@D@2@@std@@@std@@@2@$0A@@std@@@std@@IEAA?AU?$pair@V?$_Tree_iterator@V?$_Tree_val@U?$_Tree_simple_types@U?$pair@$$CB_JV?$basic_string@DU?$char_traits@D@std@@V?$allocator@D@2@@std@@@std@@@std@@@std@@@std@@_N@1@_NAEAU?$pair@$$CB_JV?$basic_string@DU?$char_traits@D@std@@V?$allocator@D@2@@std@@@1@PEAU?$_Tree_node@U?$pair@$$CB_JV?$basic_string@DU?$char_traits@D@std@@V?$allocator@D@2@@std@@@std@@PEAX@1@@Z 00000001400593c4     LoadXlsMsg.obj
 0002:0000e3c4       $stateUnwindMap$??$_Insert_hint@AEAU?$pair@$$CBIUPORTINFO@@@std@@PEAU?$_Tree_node@U?$pair@$$CBIUPORTINFO@@@std@@PEAX@2@@?$_Tree@V?$_Tmap_traits@IUPORTINFO@@U?$less@I@std@@V?$allocator@U?$pair@$$CBIUPORTINFO@@@std@@@3@$0A@@std@@@std@@IEAA?AV?$_Tree_iterator@V?$_Tree_val@U?$_Tree_simple_types@U?$pair@$$CBIUPORTINFO@@@std@@@std@@@std@@@1@V?$_Tree_const_iterator@V?$_Tree_val@U?$_Tree_simple_types@U?$pair@$$CBIUPORTINFO@@@std@@@std@@@std@@@1@AEAU?$pair@$$CBIUPORTINFO@@@1@PEAU?$_Tree_node@U?$pair@$$CBIUPORTINFO@@@std@@PEAX@1@@Z 00000001400593c4     GameServerManagerDlg.obj
 0002:0000e3c4       $stateUnwindMap$??$_Buynode@U?$pair@_JVDivisionPacket@@@std@@@?$_Tree_comp_alloc@V?$_Tmap_traits@_JVDivisionPacket@@U?$less@_J@std@@V?$allocator@U?$pair@$$CB_JVDivisionPacket@@@std@@@3@$0A@@std@@@std@@QEAAPEAU?$_Tree_node@U?$pair@$$CB_JVDivisionPacket@@@std@@PEAX@1@$$QEAU?$pair@_JVDivisionPacket@@@1@@Z 00000001400593c4     DivisionPacketReceiver.obj
 0002:0000e3c4       $stateUnwindMap$??$_Insert_nohint@AEAU?$pair@$$CBGUExtraStatsFPSVerify@CHostStat@@@std@@PEAU?$_Tree_node@U?$pair@$$CBGUExtraStatsFPSVerify@CHostStat@@@std@@PEAX@2@@?$_Tree@V?$_Tmap_traits@GUExtraStatsFPSVerify@CHostStat@@U?$less@G@std@@V?$allocator@U?$pair@$$CBGUExtraStatsFPSVerify@CHostStat@@@std@@@4@$0A@@std@@@std@@IEAA?AU?$pair@V?$_Tree_iterator@V?$_Tree_val@U?$_Tree_simple_types@U?$pair@$$CBGUExtraStatsFPSVerify@CHostStat@@@std@@@std@@@std@@@std@@_N@1@_NAEAU?$pair@$$CBGUExtraStatsFPSVerify@CHostStat@@@1@PEAU?$_Tree_node@U?$pair@$$CBGUExtraStatsFPSVerify@CHostStat@@@std@@PEAX@1@@Z 00000001400593c4     HostStat.obj
 0002:0000e3c4       $stateUnwindMap$??$_Insert_nohint@AEAU?$pair@$$CB_JVDivisionPacket@@@std@@PEAU?$_Tree_node@U?$pair@$$CB_JVDivisionPacket@@@std@@PEAX@2@@?$_Tree@V?$_Tmap_traits@_JVDivisionPacket@@U?$less@_J@std@@V?$allocator@U?$pair@$$CB_JVDivisionPacket@@@std@@@3@$0A@@std@@@std@@IEAA?AU?$pair@V?$_Tree_iterator@V?$_Tree_val@U?$_Tree_simple_types@U?$pair@$$CB_JVDivisionPacket@@@std@@@std@@@std@@@std@@_N@1@_NAEAU?$pair@$$CB_JVDivisionPacket@@@1@PEAU?$_Tree_node@U?$pair@$$CB_JVDivisionPacket@@@std@@PEAX@1@@Z 00000001400593c4     DivisionPacketReceiver.obj
 0002:0000e3c4       $stateUnwindMap$??$_Insert_hint@AEAU?$pair@$$CBV?$basic_string@DU?$char_traits@D@std@@V?$allocator@D@2@@std@@V12@@std@@PEAU?$_Tree_node@U?$pair@$$CBV?$basic_string@DU?$char_traits@D@std@@V?$allocator@D@2@@std@@V12@@std@@PEAX@2@@?$_Tree@V?$_Tmap_traits@V?$basic_string@DU?$char_traits@D@std@@V?$allocator@D@2@@std@@V12@U?$less@V?$basic_string@DU?$char_traits@D@std@@V?$allocator@D@2@@std@@@2@V?$allocator@U?$pair@$$CBV?$basic_string@DU?$char_traits@D@std@@V?$allocator@D@2@@std@@V12@@std@@@2@$0A@@std@@@std@@IEAA?AV?$_Tree_iterator@V?$_Tree_val@U?$_Tree_simple_types@U?$pair@$$CBV?$basic_string@DU?$char_traits@D@std@@V?$allocator@D@2@@std@@V12@@std@@@std@@@std@@@1@V?$_Tree_const_iterator@V?$_Tree_val@U?$_Tree_simple_types@U?$pair@$$CBV?$basic_string@DU?$char_traits@D@std@@V?$allocator@D@2@@std@@V12@@std@@@std@@@std@@@1@AEAU?$pair@$$CBV?$basic_string@DU?$char_traits@D@std@@V?$allocator@D@2@@std@@V12@@1@PEAU?$_Tree_node@U?$pair@$$CBV?$basic_string@DU?$char_traits@D@std@@V?$allocator@D@2@@std@@V12@@std@@PEAX@1@@Z 00000001400593c4     iniReader.obj
 0002:0000e3c4       $stateUnwindMap$??$_Insert_nohint@AEAU?$pair@$$CBGUExtraStatsMemVerify@CHostStat@@@std@@PEAU?$_Tree_node@U?$pair@$$CBGUExtraStatsMemVerify@CHostStat@@@std@@PEAX@2@@?$_Tree@V?$_Tmap_traits@GUExtraStatsMemVerify@CHostStat@@U?$less@G@std@@V?$allocator@U?$pair@$$CBGUExtraStatsMemVerify@CHostStat@@@std@@@4@$0A@@std@@@std@@IEAA?AU?$pair@V?$_Tree_iterator@V?$_Tree_val@U?$_Tree_simple_types@U?$pair@$$CBGUExtraStatsMemVerify@CHostStat@@@std@@@std@@@std@@@std@@_N@1@_NAEAU?$pair@$$CBGUExtraStatsMemVerify@CHostStat@@@1@PEAU?$_Tree_node@U?$pair@$$CBGUExtraStatsMemVerify@CHostStat@@@std@@PEAX@1@@Z 00000001400593c4     HostStat.obj
 0002:0000e3c4       $stateUnwindMap$??$_Emplace_reallocate@AEBV?$basic_string@DU?$char_traits@D@std@@V?$allocator@D@2@@std@@@?$vector@V?$basic_string@DU?$char_traits@D@std@@V?$allocator@D@2@@std@@V?$allocator@V?$basic_string@DU?$char_traits@D@std@@V?$allocator@D@2@@std@@@2@@std@@QEAAPEAV?$basic_string@DU?$char_traits@D@std@@V?$allocator@D@2@@1@QEAV21@AEBV21@@Z 00000001400593c4     mailer.obj
 0002:0000e3c4       $stateUnwindMap$??$_Insert_nohint@AEAU?$pair@$$CBV?$basic_string@DU?$char_traits@D@std@@V?$allocator@D@2@@std@@PEAVCIniSection@CIniReader@@@std@@PEAU?$_Tree_node@U?$pair@$$CBV?$basic_string@DU?$char_traits@D@std@@V?$allocator@D@2@@std@@PEAVCIniSection@CIniReader@@@std@@PEAX@2@@?$_Tree@V?$_Tmap_traits@V?$basic_string@DU?$char_traits@D@std@@V?$allocator@D@2@@std@@PEAVCIniSection@CIniReader@@U?$less@V?$basic_string@DU?$char_traits@D@std@@V?$allocator@D@2@@std@@@2@V?$allocator@U?$pair@$$CBV?$basic_string@DU?$char_traits@D@std@@V?$allocator@D@2@@std@@PEAVCIniSection@CIniReader@@@std@@@2@$0A@@std@@@std@@IEAA?AU?$pair@V?$_Tree_iterator@V?$_Tree_val@U?$_Tree_simple_types@U?$pair@$$CBV?$basic_string@DU?$char_traits@D@std@@V?$allocator@D@2@@std@@PEAVCIniSection@CIniReader@@@std@@@std@@@std@@@std@@_N@1@_NAEAU?$pair@$$CBV?$basic_string@DU?$char_traits@D@std@@V?$allocator@D@2@@std@@PEAVCIniSection@CIniReader@@@1@PEAU?$_Tree_node@U?$pair@$$CBV?$basic_string@DU?$char_traits@D@std@@V?$allocator@D@2@@std@@PEAVCIniSection@CIniReader@@@std@@PEAX@1@@Z 00000001400593c4     iniReader.obj
 0002:0000e3c4       $stateUnwindMap$??$_Insert_nohint@AEAU?$pair@$$CBIUPORTINFO@@@std@@PEAU?$_Tree_node@U?$pair@$$CBIUPORTINFO@@@std@@PEAX@2@@?$_Tree@V?$_Tmap_traits@IUPORTINFO@@U?$less@I@std@@V?$allocator@U?$pair@$$CBIUPORTINFO@@@std@@@3@$0A@@std@@@std@@IEAA?AU?$pair@V?$_Tree_iterator@V?$_Tree_val@U?$_Tree_simple_types@U?$pair@$$CBIUPORTINFO@@@std@@@std@@@std@@@std@@_N@1@_NAEAU?$pair@$$CBIUPORTINFO@@@1@PEAU?$_Tree_node@U?$pair@$$CBIUPORTINFO@@@std@@PEAX@1@@Z 00000001400593c4     GameServerManagerDlg.obj
 0002:0000e3c4       $stateUnwindMap$??$_Buynode@U?$pair@PEADPEAVCIniSection@CIniReader@@@std@@@?$_Tree_comp_alloc@V?$_Tmap_traits@V?$basic_string@DU?$char_traits@D@std@@V?$allocator@D@2@@std@@PEAVCIniSection@CIniReader@@U?$less@V?$basic_string@DU?$char_traits@D@std@@V?$allocator@D@2@@std@@@2@V?$allocator@U?$pair@$$CBV?$basic_string@DU?$char_traits@D@std@@V?$allocator@D@2@@std@@PEAVCIniSection@CIniReader@@@std@@@2@$0A@@std@@@std@@QEAAPEAU?$_Tree_node@U?$pair@$$CBV?$basic_string@DU?$char_traits@D@std@@V?$allocator@D@2@@std@@PEAVCIniSection@CIniReader@@@std@@PEAX@1@$$QEAU?$pair@PEADPEAVCIniSection@CIniReader@@@1@@Z 00000001400593c4     iniReader.obj
 0002:0000e3d4       $tryMap$??$_Buynode@U?$pair@_JVDivisionPacket@@@std@@@?$_Tree_comp_alloc@V?$_Tmap_traits@_JVDivisionPacket@@U?$less@_J@std@@V?$allocator@U?$pair@$$CB_JVDivisionPacket@@@std@@@3@$0A@@std@@@std@@QEAAPEAU?$_Tree_node@U?$pair@$$CB_JVDivisionPacket@@@std@@PEAX@1@$$QEAU?$pair@_JVDivisionPacket@@@1@@Z 00000001400593d4     DivisionPacketReceiver.obj
 0002:0000e3e8       $handlerMap$0$??$_Buynode@U?$pair@_JVDivisionPacket@@@std@@@?$_Tree_comp_alloc@V?$_Tmap_traits@_JVDivisionPacket@@U?$less@_J@std@@V?$allocator@U?$pair@$$CB_JVDivisionPacket@@@std@@@3@$0A@@std@@@std@@QEAAPEAU?$_Tree_node@U?$pair@$$CB_JVDivisionPacket@@@std@@PEAX@1@$$QEAU?$pair@_JVDivisionPacket@@@1@@Z 00000001400593e8     DivisionPacketReceiver.obj
 0002:0000e400       $ip2state$??$_Buynode@U?$pair@_JVDivisionPacket@@@std@@@?$_Tree_comp_alloc@V?$_Tmap_traits@_JVDivisionPacket@@U?$less@_J@std@@V?$allocator@U?$pair@$$CB_JVDivisionPacket@@@std@@@3@$0A@@std@@@std@@QEAAPEAU?$_Tree_node@U?$pair@$$CB_JVDivisionPacket@@@std@@PEAX@1@$$QEAU?$pair@_JVDivisionPacket@@@1@@Z 0000000140059400     DivisionPacketReceiver.obj
 0002:0000e418       $unwind$?catch$2@?0???$_Buynode@U?$pair@_JVDivisionPacket@@@std@@@?$_Tree_comp_alloc@V?$_Tmap_traits@_JVDivisionPacket@@U?$less@_J@std@@V?$allocator@U?$pair@$$CB_JVDivisionPacket@@@std@@@3@$0A@@std@@@std@@QEAAPEAU?$_Tree_node@U?$pair@$$CB_JVDivisionPacket@@@std@@PEAX@1@$$QEAU?$pair@_JVDivisionPacket@@@1@@Z@4HA 0000000140059418     DivisionPacketReceiver.obj
 0002:0000e428       $unwind$??$_Insert_nohint@AEAU?$pair@$$CB_JVDivisionPacket@@@std@@PEAU?$_Tree_node@U?$pair@$$CB_JVDivisionPacket@@@std@@PEAX@2@@?$_Tree@V?$_Tmap_traits@_JVDivisionPacket@@U?$less@_J@std@@V?$allocator@U?$pair@$$CB_JVDivisionPacket@@@std@@@3@$0A@@std@@@std@@IEAA?AU?$pair@V?$_Tree_iterator@V?$_Tree_val@U?$_Tree_simple_types@U?$pair@$$CB_JVDivisionPacket@@@std@@@std@@@std@@@std@@_N@1@_NAEAU?$pair@$$CB_JVDivisionPacket@@@1@PEAU?$_Tree_node@U?$pair@$$CB_JVDivisionPacket@@@std@@PEAX@1@@Z 0000000140059428     DivisionPacketReceiver.obj
 0002:0000e444       $tryMap$??$_Insert_nohint@AEAU?$pair@$$CB_JVDivisionPacket@@@std@@PEAU?$_Tree_node@U?$pair@$$CB_JVDivisionPacket@@@std@@PEAX@2@@?$_Tree@V?$_Tmap_traits@_JVDivisionPacket@@U?$less@_J@std@@V?$allocator@U?$pair@$$CB_JVDivisionPacket@@@std@@@3@$0A@@std@@@std@@IEAA?AU?$pair@V?$_Tree_iterator@V?$_Tree_val@U?$_Tree_simple_types@U?$pair@$$CB_JVDivisionPacket@@@std@@@std@@@std@@@std@@_N@1@_NAEAU?$pair@$$CB_JVDivisionPacket@@@1@PEAU?$_Tree_node@U?$pair@$$CB_JVDivisionPacket@@@std@@PEAX@1@@Z 0000000140059444     DivisionPacketReceiver.obj
 0002:0000e458       $handlerMap$0$??$_Insert_nohint@AEAU?$pair@$$CB_JVDivisionPacket@@@std@@PEAU?$_Tree_node@U?$pair@$$CB_JVDivisionPacket@@@std@@PEAX@2@@?$_Tree@V?$_Tmap_traits@_JVDivisionPacket@@U?$less@_J@std@@V?$allocator@U?$pair@$$CB_JVDivisionPacket@@@std@@@3@$0A@@std@@@std@@IEAA?AU?$pair@V?$_Tree_iterator@V?$_Tree_val@U?$_Tree_simple_types@U?$pair@$$CB_JVDivisionPacket@@@std@@@std@@@std@@@std@@_N@1@_NAEAU?$pair@$$CB_JVDivisionPacket@@@1@PEAU?$_Tree_node@U?$pair@$$CB_JVDivisionPacket@@@std@@PEAX@1@@Z 0000000140059458     DivisionPacketReceiver.obj
 0002:0000e470       $ip2state$??$_Insert_nohint@AEAU?$pair@$$CB_JVDivisionPacket@@@std@@PEAU?$_Tree_node@U?$pair@$$CB_JVDivisionPacket@@@std@@PEAX@2@@?$_Tree@V?$_Tmap_traits@_JVDivisionPacket@@U?$less@_J@std@@V?$allocator@U?$pair@$$CB_JVDivisionPacket@@@std@@@3@$0A@@std@@@std@@IEAA?AU?$pair@V?$_Tree_iterator@V?$_Tree_val@U?$_Tree_simple_types@U?$pair@$$CB_JVDivisionPacket@@@std@@@std@@@std@@@std@@_N@1@_NAEAU?$pair@$$CB_JVDivisionPacket@@@1@PEAU?$_Tree_node@U?$pair@$$CB_JVDivisionPacket@@@std@@PEAX@1@@Z 0000000140059470     DivisionPacketReceiver.obj
 0002:0000e480       $unwind$?catch$2@?0???$_Insert_nohint@AEAU?$pair@$$CB_JVDivisionPacket@@@std@@PEAU?$_Tree_node@U?$pair@$$CB_JVDivisionPacket@@@std@@PEAX@2@@?$_Tree@V?$_Tmap_traits@_JVDivisionPacket@@U?$less@_J@std@@V?$allocator@U?$pair@$$CB_JVDivisionPacket@@@std@@@3@$0A@@std@@@std@@IEAA?AU?$pair@V?$_Tree_iterator@V?$_Tree_val@U?$_Tree_simple_types@U?$pair@$$CB_JVDivisionPacket@@@std@@@std@@@std@@@std@@_N@1@_NAEAU?$pair@$$CB_JVDivisionPacket@@@1@PEAU?$_Tree_node@U?$pair@$$CB_JVDivisionPacket@@@std@@PEAX@1@@Z@4HA 0000000140059480     DivisionPacketReceiver.obj
 0002:0000e490       $unwind$??$_Insert_at@AEAU?$pair@$$CBGUExtraStatsMemVerify@CHostStat@@@std@@PEAU?$_Tree_node@U?$pair@$$CBGUExtraStatsMemVerify@CHostStat@@@std@@PEAX@2@@?$_Tree@V?$_Tmap_traits@GUExtraStatsMemVerify@CHostStat@@U?$less@G@std@@V?$allocator@U?$pair@$$CBGUExtraStatsMemVerify@CHostStat@@@std@@@4@$0A@@std@@@std@@IEAA?AV?$_Tree_iterator@V?$_Tree_val@U?$_Tree_simple_types@U?$pair@$$CBGUExtraStatsMemVerify@CHostStat@@@std@@@std@@@std@@@1@_NPEAU?$_Tree_node@U?$pair@$$CBGUExtraStatsMemVerify@CHostStat@@@std@@PEAX@1@AEAU?$pair@$$CBGUExtraStatsMemVerify@CHostStat@@@1@1@Z 0000000140059490     HostStat.obj
 0002:0000e490       $unwind$??$_Insert_at@AEAU?$pair@$$CB_JV?$basic_string@DU?$char_traits@D@std@@V?$allocator@D@2@@std@@@std@@PEAU?$_Tree_node@U?$pair@$$CB_JV?$basic_string@DU?$char_traits@D@std@@V?$allocator@D@2@@std@@@std@@PEAX@2@@?$_Tree@V?$_Tmap_traits@_JV?$basic_string@DU?$char_traits@D@std@@V?$allocator@D@2@@std@@U?$less@_J@2@V?$allocator@U?$pair@$$CB_JV?$basic_string@DU?$char_traits@D@std@@V?$allocator@D@2@@std@@@std@@@2@$0A@@std@@@std@@IEAA?AV?$_Tree_iterator@V?$_Tree_val@U?$_Tree_simple_types@U?$pair@$$CB_JV?$basic_string@DU?$char_traits@D@std@@V?$allocator@D@2@@std@@@std@@@std@@@std@@@1@_NPEAU?$_Tree_node@U?$pair@$$CB_JV?$basic_string@DU?$char_traits@D@std@@V?$allocator@D@2@@std@@@std@@PEAX@1@AEAU?$pair@$$CB_JV?$basic_string@DU?$char_traits@D@std@@V?$allocator@D@2@@std@@@1@1@Z 0000000140059490     LoadXlsMsg.obj
 0002:0000e490       $unwind$??$_Insert_at@AEAU?$pair@$$CBIUPORTINFO@@@std@@PEAU?$_Tree_node@U?$pair@$$CBIUPORTINFO@@@std@@PEAX@2@@?$_Tree@V?$_Tmap_traits@IUPORTINFO@@U?$less@I@std@@V?$allocator@U?$pair@$$CBIUPORTINFO@@@std@@@3@$0A@@std@@@std@@IEAA?AV?$_Tree_iterator@V?$_Tree_val@U?$_Tree_simple_types@U?$pair@$$CBIUPORTINFO@@@std@@@std@@@std@@@1@_NPEAU?$_Tree_node@U?$pair@$$CBIUPORTINFO@@@std@@PEAX@1@AEAU?$pair@$$CBIUPORTINFO@@@1@1@Z 0000000140059490     GameServerManagerDlg.obj
 0002:0000e490       $unwind$??$_Insert_at@AEAU?$pair@$$CBV?$basic_string@DU?$char_traits@D@std@@V?$allocator@D@2@@std@@PEAVCIniSection@CIniReader@@@std@@PEAU?$_Tree_node@U?$pair@$$CBV?$basic_string@DU?$char_traits@D@std@@V?$allocator@D@2@@std@@PEAVCIniSection@CIniReader@@@std@@PEAX@2@@?$_Tree@V?$_Tmap_traits@V?$basic_string@DU?$char_traits@D@std@@V?$allocator@D@2@@std@@PEAVCIniSection@CIniReader@@U?$less@V?$basic_string@DU?$char_traits@D@std@@V?$allocator@D@2@@std@@@2@V?$allocator@U?$pair@$$CBV?$basic_string@DU?$char_traits@D@std@@V?$allocator@D@2@@std@@PEAVCIniSection@CIniReader@@@std@@@2@$0A@@std@@@std@@IEAA?AV?$_Tree_iterator@V?$_Tree_val@U?$_Tree_simple_types@U?$pair@$$CBV?$basic_string@DU?$char_traits@D@std@@V?$allocator@D@2@@std@@PEAVCIniSection@CIniReader@@@std@@@std@@@std@@@1@_NPEAU?$_Tree_node@U?$pair@$$CBV?$basic_string@DU?$char_traits@D@std@@V?$allocator@D@2@@std@@PEAVCIniSection@CIniReader@@@std@@PEAX@1@AEAU?$pair@$$CBV?$basic_string@DU?$char_traits@D@std@@V?$allocator@D@2@@std@@PEAVCIniSection@CIniReader@@@1@1@Z 0000000140059490     iniReader.obj
 0002:0000e490       $unwind$??$_Insert_at@AEAU?$pair@$$CBGUExtraStatsFPSVerify@CHostStat@@@std@@PEAU?$_Tree_node@U?$pair@$$CBGUExtraStatsFPSVerify@CHostStat@@@std@@PEAX@2@@?$_Tree@V?$_Tmap_traits@GUExtraStatsFPSVerify@CHostStat@@U?$less@G@std@@V?$allocator@U?$pair@$$CBGUExtraStatsFPSVerify@CHostStat@@@std@@@4@$0A@@std@@@std@@IEAA?AV?$_Tree_iterator@V?$_Tree_val@U?$_Tree_simple_types@U?$pair@$$CBGUExtraStatsFPSVerify@CHostStat@@@std@@@std@@@std@@@1@_NPEAU?$_Tree_node@U?$pair@$$CBGUExtraStatsFPSVerify@CHostStat@@@std@@PEAX@1@AEAU?$pair@$$CBGUExtraStatsFPSVerify@CHostStat@@@1@1@Z 0000000140059490     HostStat.obj
 0002:0000e490       $unwind$??$_Insert_at@AEAU?$pair@$$CBV?$basic_string@DU?$char_traits@D@std@@V?$allocator@D@2@@std@@V12@@std@@PEAU?$_Tree_node@U?$pair@$$CBV?$basic_string@DU?$char_traits@D@std@@V?$allocator@D@2@@std@@V12@@std@@PEAX@2@@?$_Tree@V?$_Tmap_traits@V?$basic_string@DU?$char_traits@D@std@@V?$allocator@D@2@@std@@V12@U?$less@V?$basic_string@DU?$char_traits@D@std@@V?$allocator@D@2@@std@@@2@V?$allocator@U?$pair@$$CBV?$basic_string@DU?$char_traits@D@std@@V?$allocator@D@2@@std@@V12@@std@@@2@$0A@@std@@@std@@IEAA?AV?$_Tree_iterator@V?$_Tree_val@U?$_Tree_simple_types@U?$pair@$$CBV?$basic_string@DU?$char_traits@D@std@@V?$allocator@D@2@@std@@V12@@std@@@std@@@std@@@1@_NPEAU?$_Tree_node@U?$pair@$$CBV?$basic_string@DU?$char_traits@D@std@@V?$allocator@D@2@@std@@V12@@std@@PEAX@1@AEAU?$pair@$$CBV?$basic_string@DU?$char_traits@D@std@@V?$allocator@D@2@@std@@V12@@1@1@Z 0000000140059490     iniReader.obj
 0002:0000e490       $unwind$??$_Insert_at@AEAU?$pair@$$CB_JVDivisionPacket@@@std@@PEAU?$_Tree_node@U?$pair@$$CB_JVDivisionPacket@@@std@@PEAX@2@@?$_Tree@V?$_Tmap_traits@_JVDivisionPacket@@U?$less@_J@std@@V?$allocator@U?$pair@$$CB_JVDivisionPacket@@@std@@@3@$0A@@std@@@std@@IEAA?AV?$_Tree_iterator@V?$_Tree_val@U?$_Tree_simple_types@U?$pair@$$CB_JVDivisionPacket@@@std@@@std@@@std@@@1@_NPEAU?$_Tree_node@U?$pair@$$CB_JVDivisionPacket@@@std@@PEAX@1@AEAU?$pair@$$CB_JVDivisionPacket@@@1@1@Z 0000000140059490     DivisionPacketReceiver.obj
 0002:0000e49c       $unwind$?CRSUploader@@YAAEAVUploader@crs@@XZ 000000014005949c     BugReporter.obj
 0002:0000e4b0       $stateUnwindMap$?CRSUploader@@YAAEAVUploader@crs@@XZ 00000001400594b0     BugReporter.obj
 0002:0000e4c8       $ip2state$?CRSUploader@@YAAEAVUploader@crs@@XZ 00000001400594c8     BugReporter.obj
 0002:0000e4d8       $unwind$?dtor$90@?0??makesmtpmessage@mailer@jwsmtp@@AEBA?AV?$vector@DV?$allocator@D@std@@@std@@XZ@4HA 00000001400594d8     mailer.obj
 0002:0000e4d8       $unwind$?dtor$54@?0??makesmtpmessage@mailer@jwsmtp@@AEBA?AV?$vector@DV?$allocator@D@std@@@std@@XZ@4HA 00000001400594d8     mailer.obj
 0002:0000e4d8       $unwind$?filt$0@?0??__ArrayUnwind@@YAXPEAX_K1P6AX0@Z@Z@4HA 00000001400594d8     msvcrt:ehvecdtr.obj
 0002:0000e4d8       $unwind$?dtor$1@?0??OnReceiveFromGms@CGameServerManagerDlg@@AEAAXAEBUPROTO_STARTING_GAME_tag@@@Z@4HA 00000001400594d8     GameServerManagerDlg.obj
 0002:0000e4d8       $unwind$?dtor$4@?0??strcpy_s@cf@@YAHPEAD_KPEBD@Z@4HA 00000001400594d8     safe_string_x64:safe_string.obj
 0002:0000e4d8       $unwind$?dtor$4@?0??sprintf_s@internal@cf@@YAHPEAD_KPEBDAEAPEAD@Z@4HA 00000001400594d8     safe_string_x64:safe_string.obj
 0002:0000e4d8       $unwind$?dtor$2@?0??makesmtpmessage@mailer@jwsmtp@@AEBA?AV?$vector@DV?$allocator@D@std@@@std@@XZ@4HA 00000001400594d8     mailer.obj
 0002:0000e4d8       $unwind$?fin$0@?0???_M@YAXPEAX_K1P6AX0@Z@Z@4HA 00000001400594d8     msvcrt:ehvecdtr.obj
 0002:0000e4d8       $unwind$?dtor$41@?0??authenticate@mailer@jwsmtp@@AEAA_NAEBV?$basic_string@DU?$char_traits@D@std@@V?$allocator@D@2@@std@@AEB_K@Z@4HA 00000001400594d8     mailer.obj
 0002:0000e4d8       $unwind$?dtor$114@?0??makesmtpmessage@mailer@jwsmtp@@AEBA?AV?$vector@DV?$allocator@D@std@@@std@@XZ@4HA 00000001400594d8     mailer.obj
 0002:0000e4d8       $unwind$?dtor$29@?0??authenticate@mailer@jwsmtp@@AEAA_NAEBV?$basic_string@DU?$char_traits@D@std@@V?$allocator@D@2@@std@@AEB_K@Z@4HA 00000001400594d8     mailer.obj
 0002:0000e4d8       $unwind$?dtor$126@?0??makesmtpmessage@mailer@jwsmtp@@AEBA?AV?$vector@DV?$allocator@D@std@@@std@@XZ@4HA 00000001400594d8     mailer.obj
 0002:0000e4d8       $unwind$?dtor$5@?0??InitializeManager@CGameServerManagerDlg@@QEAAHPEADKPEAPEAD@Z@4HA 00000001400594d8     GameServerManagerDlg.obj
 0002:0000e4d8       $unwind$?fin$0@?0???_L@YAXPEAX_K1P6AX0@Z2@Z@4HA 00000001400594d8     msvcrt:ehvecctr.obj
 0002:0000e4d8       $unwind$?dtor$138@?0??makesmtpmessage@mailer@jwsmtp@@AEBA?AV?$vector@DV?$allocator@D@std@@@std@@XZ@4HA 00000001400594d8     mailer.obj
 0002:0000e4d8       $unwind$?dtor$4@?0??strncpy_s@cf@@YAHPEAD_KPEBD1@Z@4HA 00000001400594d8     safe_string_x64:safe_string.obj
 0002:0000e4d8       $unwind$?dtor$0@?0??Init@CLogMsgManager@@SA_NW4ESHARED_MEM_USAGE_TYPE@1@@Z@4HA 00000001400594d8     LogMsgManager.obj
 0002:0000e4d8       $unwind$?dtor$13@?0???0CGameServerManagerDlg@@QEAA@PEAVCWnd@@@Z@4HA 00000001400594d8     GameServerManagerDlg.obj
 0002:0000e4d8       $unwind$?dtor$1@?0??InitializeManager@CGameServerManagerDlg@@QEAAHPEADKPEAPEAD@Z@4HA 00000001400594d8     GameServerManagerDlg.obj
 0002:0000e4d8       $unwind$?dtor$150@?0??makesmtpmessage@mailer@jwsmtp@@AEBA?AV?$vector@DV?$allocator@D@std@@@std@@XZ@4HA 00000001400594d8     mailer.obj
 0002:0000e4d8       $unwind$?dtor$8@?0???0CSharedMemoryLoader@@QEAA@XZ@4HA 00000001400594d8     GameServerManagerDlg.obj
 0002:0000e4d8       $unwind$?dtor$0@?0???$?HDU?$char_traits@D@std@@V?$allocator@D@1@@std@@YA?AV?$basic_string@DU?$char_traits@D@std@@V?$allocator@D@2@@0@QEBDAEBV10@@Z@4HA 00000001400594d8     CSmtp.obj
 0002:0000e4d8       $unwind$?dtor$1@?0??OnReceiveFromGms@CGameServerManagerDlg@@AEAAXAEBUPROTO_AUTOMATCH_GAME_START_REQ@@@Z@4HA 00000001400594d8     GameServerManagerDlg.obj
 0002:0000e4d8       $unwind$?dtor$2@?0??StringSplitToNumArray@CGameServerManagerDlg@@AEAAXV?$basic_string@DU?$char_traits@D@std@@V?$allocator@D@2@@std@@0PEAHAEAH@Z@4HA 00000001400594d8     GameServerManagerDlg.obj
 0002:0000e4d8       $unwind$?dtor$0@?0???0?$basic_stringstream@DU?$char_traits@D@std@@V?$allocator@D@2@@std@@QEAA@H@Z@4HA 00000001400594d8     safe_string_x64:safe_string.obj
 0002:0000e4d8       $unwind$?filt$0@?0??__scrt_common_main_seh@@YAHXZ@4HA 00000001400594d8     msvcrt:exe_winmain.obj
 0002:0000e4d8       $unwind$?dtor$3@?0??write@CIniSection@CIniReader@@QEAAKPEAX@Z@4HA 00000001400594d8     iniReader.obj
 0002:0000e4d8       $unwind$?dtor$1@?0??CRSUploader@@YAAEAVUploader@crs@@XZ@4HA 00000001400594d8     BugReporter.obj
 0002:0000e4d8       $unwind$?dtor$1@?0??Init@CLogMsgManager@@SA_NW4ESHARED_MEM_USAGE_TYPE@1@@Z@4HA 00000001400594d8     LogMsgManager.obj
 0002:0000e4d8       $unwind$?dtor$137@?0???Rmailer@jwsmtp@@QEAAXXZ@4HA 00000001400594d8     mailer.obj
 0002:0000e4d8       $unwind$?dtor$178@?0???Rmailer@jwsmtp@@QEAAXXZ@4HA 00000001400594d8     mailer.obj
 0002:0000e4d8       $unwind$?dtor$14@?0???0CSharedMemoryLoader@@QEAA@XZ@4HA 00000001400594d8     GameServerManagerDlg.obj
 0002:0000e4d8       $unwind$?dtor$1@?0??OnReceiveFromGms@CGameServerManagerDlg@@AEAAXAEBUPROTO_AUTOMATCH_GAME_ENTER_REQ@@@Z@4HA 00000001400594d8     GameServerManagerDlg.obj
 0002:0000e4d8       $unwind$?dtor$1@?0??init@SGGMProxyLoader@sggm_proxy@@QEAA_NPEAVMultiReceiver@2@@Z@4HA 00000001400594d8     GameServerManagerDlg.obj
 0002:0000e4d8       $unwind$?dtor$3@?0??base64encode@jwsmtp@@YA?AV?$basic_string@DU?$char_traits@D@std@@V?$allocator@D@2@@std@@AEBV23@_N@Z@4HA 00000001400594d8     base6409cee8549d9fd00dfa06fdadc87a8424.obj
 0002:0000e4d8       $unwind$?dtor$1@?0??setString@CIniReader@@QEAAXPEBD00@Z@4HA 00000001400594d8     iniReader.obj
 0002:0000e4d8       $unwind$?dtor$3@?0??write@CIniReader@@QEAAKPEBD@Z@4HA 00000001400594d8     iniReader.obj
 0002:0000e4d8       $unwind$?dtor$0@?0??base64encode@jwsmtp@@YA?AV?$vector@DV?$allocator@D@std@@@std@@AEBV23@_N@Z@4HA 00000001400594d8     base6409cee8549d9fd00dfa06fdadc87a8424.obj
 0002:0000e4e0       $unwind$?threadCreateDumpFile@@YAKPEAX@Z 00000001400594e0     BugReporter.obj
 0002:0000e508       $stateUnwindMap$?threadCreateDumpFile@@YAKPEAX@Z 0000000140059508     BugReporter.obj
 0002:0000e510       $ip2state$?threadCreateDumpFile@@YAKPEAX@Z 0000000140059510     BugReporter.obj
 0002:0000e528       $unwind$?CrashExceptionDump@@YAJPEAU_EXCEPTION_POINTERS@@@Z 0000000140059528     BugReporter.obj
 0002:0000e530       $chain$0$?CrashExceptionDump@@YAJPEAU_EXCEPTION_POINTERS@@@Z 0000000140059530     BugReporter.obj
 0002:0000e544       $chain$1$?CrashExceptionDump@@YAJPEAU_EXCEPTION_POINTERS@@@Z 0000000140059544     BugReporter.obj
 0002:0000e554       $unwind$?InitBugReporter@@YAXPEAD0000@Z 0000000140059554     BugReporter.obj
 0002:0000e574       $unwind$??$sprintf_s@$0PP@@cf@@YAHAEAY0PP@DPEBDZZ 0000000140059574     GameServerManagerDlg.obj
 0002:0000e574       $unwind$??$sprintf_s@$0EBA@@cf@@YAHAEAY0EBA@DPEBDZZ 0000000140059574     GMSConnManager.obj
 0002:0000e574       $unwind$??$sprintf_s@$0BAA@@cf@@YAHAEAY0BAA@DPEBDZZ 0000000140059574     BugReporter.obj
 0002:0000e574       $unwind$??$sprintf_s@$0BJB@@cf@@YAHAEAY0BJB@DPEBDZZ 0000000140059574     BugReporter.obj
 0002:0000e574       $unwind$??$sprintf_s@$0GE@@cf@@YAHAEAY0GE@DPEBDZZ 0000000140059574     GameServerManagerDlg.obj
 0002:0000e574       $unwind$??$sprintf_s@$0BE@@cf@@YAHAEAY0BE@DPEBDZZ 0000000140059574     BugReporter.obj
 0002:0000e574       $unwind$??$sprintf_s@$0EA@@cf@@YAHAEAY0EA@DPEBDZZ 0000000140059574     RWPMLog.obj
 0002:0000e574       $unwind$??$sprintf_s@$0CA@@cf@@YAHAEAY0CA@DPEBDZZ 0000000140059574     LogMsgManager.obj
 0002:0000e574       $unwind$??$sprintf_s@$0CAA@@cf@@YAHAEAY0CAA@DPEBDZZ 0000000140059574     HostStat.obj
 0002:0000e574       $unwind$??$sprintf_s@$0DOJ@@cf@@YAHAEAY0DOJ@DPEBDZZ 0000000140059574     BugReporter.obj
 0002:0000e574       $unwind$??$sprintf_s@$0BAE@@cf@@YAHAEAY0BAE@DPEBDZZ 0000000140059574     BugReporter.obj
 0002:0000e57c       $unwind$?assign@?$basic_string@DU?$char_traits@D@std@@V?$allocator@D@2@@std@@QEAAAEAV12@QEBD_K@Z 000000014005957c     BugReporter.obj
 0002:0000e57c       $unwind$?Write@SendBuffer@@QEAAHPEAEG@Z 000000014005957c     ClientLib.obj
 0002:0000e590       $chain$0$?assign@?$basic_string@DU?$char_traits@D@std@@V?$allocator@D@2@@std@@QEAAAEAV12@QEBD_K@Z 0000000140059590     BugReporter.obj
 0002:0000e5a4       $chain$3$?assign@?$basic_string@DU?$char_traits@D@std@@V?$allocator@D@2@@std@@QEAAAEAV12@QEBD_K@Z 00000001400595a4     BugReporter.obj
 0002:0000e5a4       $chain$1$?assign@?$basic_string@DU?$char_traits@D@std@@V?$allocator@D@2@@std@@QEAAAEAV12@QEBD_K@Z 00000001400595a4     BugReporter.obj
 0002:0000e5b4       $chain$2$?assign@?$basic_string@DU?$char_traits@D@std@@V?$allocator@D@2@@std@@QEAAAEAV12@QEBD_K@Z 00000001400595b4     BugReporter.obj
 0002:0000e5c8       $unwind$_snwprintf_s       00000001400595c8     crs_uploader.obj
 0002:0000e5c8       $unwind$_snprintf_s        00000001400595c8     BugReporter.obj
 0002:0000e5d8       $unwind$?recordExceptionLog@Uploader@crs@@QEAAXAEAVLogBuffer@2@PEBDZZ 00000001400595d8     crs_uploader.obj
 0002:0000e5ec       $chain$0$?recordExceptionLog@Uploader@crs@@QEAAXAEAVLogBuffer@2@PEBDZZ 00000001400595ec     crs_uploader.obj
 0002:0000e600       $chain$1$?recordExceptionLog@Uploader@crs@@QEAAXAEAVLogBuffer@2@PEBDZZ 0000000140059600     crs_uploader.obj
 0002:0000e610       $unwind$?readURL@Uploader@crs@@AEAAXAEAV?$basic_string@_WU?$char_traits@_W@std@@V?$allocator@_W@2@@std@@@Z 0000000140059610     crs_uploader.obj
 0002:0000e62c       $stateUnwindMap$?readURL@Uploader@crs@@AEAAXAEAV?$basic_string@_WU?$char_traits@_W@std@@V?$allocator@_W@2@@std@@@Z 000000014005962c     crs_uploader.obj
 0002:0000e648       $ip2state$?readURL@Uploader@crs@@AEAAXAEAV?$basic_string@_WU?$char_traits@_W@std@@V?$allocator@_W@2@@std@@@Z 0000000140059648     crs_uploader.obj
 0002:0000e668       $unwind$?iniPath@Uploader@crs@@AEAA?AV?$basic_string@_WU?$char_traits@_W@std@@V?$allocator@_W@2@@std@@AEBV34@@Z 0000000140059668     crs_uploader.obj
 0002:0000e684       $chain$1$?iniPath@Uploader@crs@@AEAA?AV?$basic_string@_WU?$char_traits@_W@std@@V?$allocator@_W@2@@std@@AEBV34@@Z 0000000140059684     crs_uploader.obj
 0002:0000e698       $chain$2$?iniPath@Uploader@crs@@AEAA?AV?$basic_string@_WU?$char_traits@_W@std@@V?$allocator@_W@2@@std@@AEBV34@@Z 0000000140059698     crs_uploader.obj
 0002:0000e6a8       $unwind$?makeBaseInfo@Uploader@crs@@AEAAXPEAD0@Z 00000001400596a8     crs_uploader.obj
 0002:0000e6c4       $unwind$?error@Uploader@crs@@AEAA_NPEBDZZ 00000001400596c4     crs_uploader.obj
 0002:0000e6d0       $unwind$?init@Uploader@crs@@QEAA_N_NPEAD1@Z 00000001400596d0     crs_uploader.obj
 0002:0000e6f4       $stateUnwindMap$?init@Uploader@crs@@QEAA_N_NPEAD1@Z 00000001400596f4     crs_uploader.obj
 0002:0000e700       $ip2state$?init@Uploader@crs@@QEAA_N_NPEAD1@Z 0000000140059700     crs_uploader.obj
 0002:0000e710       $unwind$?upload@Uploader@crs@@QEAA_N_NAEBV?$basic_string@DU?$char_traits@D@std@@V?$allocator@D@2@@std@@AEAVLogBuffer@2@@Z 0000000140059710     crs_uploader.obj
 0002:0000e72c       $unwind$?makeExceptionLog@Uploader@crs@@QEAAXPEAU_EXCEPTION_POINTERS@@AEAVLogBuffer@2@@Z 000000014005972c     crs_uploader.obj
 0002:0000e744       $chain$3$?makeExceptionLog@Uploader@crs@@QEAAXPEAU_EXCEPTION_POINTERS@@AEAVLogBuffer@2@@Z 0000000140059744     crs_uploader.obj
 0002:0000e764       $chain$4$?makeExceptionLog@Uploader@crs@@QEAAXPEAU_EXCEPTION_POINTERS@@AEAVLogBuffer@2@@Z 0000000140059764     crs_uploader.obj
 0002:0000e774       $unwind$?EnumModuleDetail@ModuleInfo@?1??makeExceptionLog@Uploader@crs@@QEAAXPEAU_EXCEPTION_POINTERS@@AEAVLogBuffer@4@@Z@SAHPEBD_KKPEAX@Z 0000000140059774     crs_uploader.obj
 0002:0000e788       $chain$0$?EnumModuleDetail@ModuleInfo@?1??makeExceptionLog@Uploader@crs@@QEAAXPEAU_EXCEPTION_POINTERS@@AEAVLogBuffer@4@@Z@SAHPEBD_KKPEAX@Z 0000000140059788     crs_uploader.obj
 0002:0000e79c       $chain$1$?EnumModuleDetail@ModuleInfo@?1??makeExceptionLog@Uploader@crs@@QEAAXPEAU_EXCEPTION_POINTERS@@AEAVLogBuffer@4@@Z@SAHPEBD_KKPEAX@Z 000000014005979c     crs_uploader.obj
 0002:0000e7ac       $unwind$?prepare@Uploader@crs@@AEAA_NAEAVHttpHandles@2@@Z 00000001400597ac     crs_uploader.obj
 0002:0000e7c0       $unwind$?uploadHTTP@Uploader@crs@@AEAA_NAEAVHttpHandle@2@PEBDPEB_W2@Z 00000001400597c0     crs_uploader.obj
 0002:0000e7dc       $unwind$?uploadLOG@Uploader@crs@@AEAA_NAEAVHttpHandle@2@AEAU_SYSTEMTIME@@AEAVLogBuffer@2@@Z 00000001400597dc     crs_uploader.obj
 0002:0000e7f8       $chain$0$?uploadLOG@Uploader@crs@@AEAA_NAEAVHttpHandle@2@AEAU_SYSTEMTIME@@AEAVLogBuffer@2@@Z 00000001400597f8     crs_uploader.obj
 0002:0000e80c       $chain$1$?uploadLOG@Uploader@crs@@AEAA_NAEAVHttpHandle@2@AEAU_SYSTEMTIME@@AEAVLogBuffer@2@@Z 000000014005980c     crs_uploader.obj
 0002:0000e820       $chain$2$?uploadLOG@Uploader@crs@@AEAA_NAEAVHttpHandle@2@AEAU_SYSTEMTIME@@AEAVLogBuffer@2@@Z 0000000140059820     crs_uploader.obj
 0002:0000e830       $chain$3$?uploadLOG@Uploader@crs@@AEAA_NAEAVHttpHandle@2@AEAU_SYSTEMTIME@@AEAVLogBuffer@2@@Z 0000000140059830     crs_uploader.obj
 0002:0000e840       $unwind$?success@Uploader@crs@@AEAA_NPEBDAEAVHttpHandle@2@@Z 0000000140059840     crs_uploader.obj
 0002:0000e840       $unwind$?PostMessageToWriteLogFile@CGameServerManagerDlg@@AEAA_NFPEAUHWND__@@_K_J@Z 0000000140059840     GameServerManagerDlg.obj
 0002:0000e840       $unwind$??$insert@V?$_String_iterator@V?$_String_val@U?$_Simple_types@D@std@@@std@@@std@@X@?$vector@DV?$allocator@D@std@@@std@@QEAA?AV?$_Vector_iterator@V?$_Vector_val@U?$_Simple_types@D@std@@@std@@@1@V?$_Vector_const_iterator@V?$_Vector_val@U?$_Simple_types@D@std@@@std@@@1@V?$_String_iterator@V?$_String_val@U?$_Simple_types@D@std@@@std@@@1@1@Z 0000000140059840     mailer.obj
 0002:0000e840       $unwind$??$insert@V?$_Vector_const_iterator@V?$_Vector_val@U?$_Simple_types@D@std@@@std@@@std@@X@?$vector@DV?$allocator@D@std@@@std@@QEAA?AV?$_Vector_iterator@V?$_Vector_val@U?$_Simple_types@D@std@@@std@@@1@V?$_Vector_const_iterator@V?$_Vector_val@U?$_Simple_types@D@std@@@std@@@1@00@Z 0000000140059840     mailer.obj
 0002:0000e850       $chain$0$??1?$auto_ptr@VUrl@crs@@@std@@QEAA@XZ 0000000140059850     crs_uploader.obj
 0002:0000e864       $chain$1$??1?$auto_ptr@VUrl@crs@@@std@@QEAA@XZ 0000000140059864     crs_uploader.obj
 0002:0000e874       $chain$2$??1?$auto_ptr@VUrl@crs@@@std@@QEAA@XZ 0000000140059874     crs_uploader.obj
 0002:0000e888       $unwind$??$_snprintf_s@$0IA@@@YAHAEAY0IA@D_KPEBDZZ 0000000140059888     crs_uploader.obj
 0002:0000e898       $unwind$??$_Reallocate_grow_by@V<lambda_65e615be2a453ca0576c979606f46740>@@PEBD_K@?$basic_string@DU?$char_traits@D@std@@V?$allocator@D@2@@std@@QEAAAEAV01@_KV<lambda_65e615be2a453ca0576c979606f46740>@@PEBD_K@Z 0000000140059898     GameServerManagerDlg.obj
 0002:0000e898       $unwind$??$_Reallocate_grow_by@V<lambda_1dfe18491bcca09701d8ccb01d0b0af4>@@PEB_W_K@?$basic_string@_WU?$char_traits@_W@std@@V?$allocator@_W@2@@std@@QEAAAEAV01@_KV<lambda_1dfe18491bcca09701d8ccb01d0b0af4>@@PEB_W_K@Z 0000000140059898     crs_uploader.obj
 0002:0000e8a8       $chain$3$??$_Reallocate_grow_by@V<lambda_1dfe18491bcca09701d8ccb01d0b0af4>@@PEB_W_K@?$basic_string@_WU?$char_traits@_W@std@@V?$allocator@_W@2@@std@@QEAAAEAV01@_KV<lambda_1dfe18491bcca09701d8ccb01d0b0af4>@@PEB_W_K@Z 00000001400598a8     crs_uploader.obj
 0002:0000e8c8       $chain$4$??$_Reallocate_grow_by@V<lambda_1dfe18491bcca09701d8ccb01d0b0af4>@@PEB_W_K@?$basic_string@_WU?$char_traits@_W@std@@V?$allocator@_W@2@@std@@QEAAAEAV01@_KV<lambda_1dfe18491bcca09701d8ccb01d0b0af4>@@PEB_W_K@Z 00000001400598c8     crs_uploader.obj
 0002:0000e8d8       $unwind$??0exception@std@@QEAA@QEBD@Z 00000001400598d8     AppInfoDlg.obj
 0002:0000e8d8       $unwind$?append@?$basic_string@_WU?$char_traits@_W@std@@V?$allocator@_W@2@@std@@QEAAAEAV12@QEB_W_K@Z 00000001400598d8     crs_uploader.obj
 0002:0000e8d8       $unwind$?Add@datetime@@QEAAXV1@@Z 00000001400598d8     DateTime.obj
 0002:0000e8e0       $chain$1$?append@?$basic_string@_WU?$char_traits@_W@std@@V?$allocator@_W@2@@std@@QEAAAEAV12@QEB_W_K@Z 00000001400598e0     crs_uploader.obj
 0002:0000e8f8       $chain$2$?append@?$basic_string@_WU?$char_traits@_W@std@@V?$allocator@_W@2@@std@@QEAAAEAV12@QEB_W_K@Z 00000001400598f8     crs_uploader.obj
 0002:0000e908       $unwind$?overflow@?$basic_stringbuf@DU?$char_traits@D@std@@V?$allocator@D@2@@std@@MEAAHH@Z 0000000140059908     safe_string_x64:safe_string.obj
 0002:0000e908       $unwind$?assign@?$basic_string@_WU?$char_traits@_W@std@@V?$allocator@_W@2@@std@@QEAAAEAV12@QEB_W_K@Z 0000000140059908     crs_uploader.obj
 0002:0000e924       $unwind$?LOG_MAILER@CServerLog@@QEAAXHPEBD@Z 0000000140059924     LogMgmt.obj
 0002:0000e938       $chain$0$?LOG_MAILER@CServerLog@@QEAAXHPEBD@Z 0000000140059938     LogMgmt.obj
 0002:0000e94c       $chain$1$?LOG_MAILER@CServerLog@@QEAAXHPEBD@Z 000000014005994c     LogMgmt.obj
 0002:0000e95c       $unwind$fprintf            000000014005995c     LogMgmt.obj
 0002:0000e95c       $unwind$sprintf            000000014005995c     LogMgmt.obj
 0002:0000e95c       $unwind$sscanf             000000014005995c     GameServerManagerDlg.obj
 0002:0000e968       $unwind$?Log@rwpmlog@@YAXPEBDFPEBUCLANSTATREPORTDATA@@@Z 0000000140059968     RWPMLog.obj
 0002:0000e968       $unwind$?Log@rwpmlog@@YAXPEBDFPEBUGAMEPROTO_SC_REMOVECLIENT@@@Z 0000000140059968     RWPMLog.obj
 0002:0000e968       $unwind$?Log@rwpmlog@@YAXPEBDFPEBUGAMEPROTO_SC_HOST_STAT@@@Z 0000000140059968     RWPMLog.obj
 0002:0000e984       $unwind$?Log@rwpmlog@@YAXPEBDFPEBUGAMEPROTO_SS_GAMEEND@@@Z 0000000140059984     RWPMLog.obj
 0002:0000e9a8       $unwind$?Log@rwpmlog@@YAXPEBDFPEBUGAMEPROTO_SC_HOST_USER_STAT@@@Z 00000001400599a8     RWPMLog.obj
 0002:0000e9c8       $unwind$?Log@rwpmlog@@YAXPEBDFPEBUPROTO_GAMEGT_INGAME_AIGACHA_ITEM_INSERT@@@Z 00000001400599c8     RWPMLog.obj
 0002:0000e9e4       $chain$0$?Log@rwpmlog@@YAXPEBDFPEBUPROTO_GAMEGT_INGAME_AIGACHA_ITEM_INSERT@@@Z 00000001400599e4     RWPMLog.obj
 0002:0000e9f8       $chain$1$?Log@rwpmlog@@YAXPEBDFPEBUPROTO_GAMEGT_INGAME_AIGACHA_ITEM_INSERT@@@Z 00000001400599f8     RWPMLog.obj
 0002:0000ea08       $unwind$?Log@rwpmlog@@YAXPEBDFPEBUPROTO_SPEC_RECOMMENDROOM_INGAME_DATA@@@Z 0000000140059a08     RWPMLog.obj
 0002:0000ea24       $unwind$?Log@rwpmlog@@YAXPEBDFPEBUPROTO_GAMEGT_AUTO_SIDE_CHANGE_TEAM_INFO_NTY@@@Z 0000000140059a24     RWPMLog.obj
 0002:0000ea40       $unwind$?GetSendParam@SendBuffer@@QEAAHPEAPEAEAEAH@Z 0000000140059a40     ClientLib.obj
 0002:0000ea54       $chain$0$?GetSendParam@SendBuffer@@QEAAHPEAPEAEAEAH@Z 0000000140059a54     ClientLib.obj
 0002:0000ea68       $chain$1$?GetSendParam@SendBuffer@@QEAAHPEAPEAEAEAH@Z 0000000140059a68     ClientLib.obj
 0002:0000ea78       $chain$0$?Write@SendBuffer@@QEAAHPEAEG@Z 0000000140059a78     ClientLib.obj
 0002:0000ea8c       $chain$1$?Write@SendBuffer@@QEAAHPEAEG@Z 0000000140059a8c     ClientLib.obj
 0002:0000ea9c       $unwind$?ProcessSend@CClientLib@@QEAAHXZ 0000000140059a9c     ClientLib.obj
 0002:0000eaa8       $chain$0$?ProcessSend@CClientLib@@QEAAHXZ 0000000140059aa8     ClientLib.obj
 0002:0000eabc       $chain$3$?ProcessSend@CClientLib@@QEAAHXZ 0000000140059abc     ClientLib.obj
 0002:0000ead8       $chain$4$?ProcessSend@CClientLib@@QEAAHXZ 0000000140059ad8     ClientLib.obj
 0002:0000eae8       $chain$5$?ProcessSend@CClientLib@@QEAAHXZ 0000000140059ae8     ClientLib.obj
 0002:0000eaf8       $unwind$?CopySendBuffer@CClientLib@@QEAAHPEAVSendBuffer@@@Z 0000000140059af8     ClientLib.obj
 0002:0000eb00       $chain$2$?CopySendBuffer@CClientLib@@QEAAHPEAVSendBuffer@@@Z 0000000140059b00     ClientLib.obj
 0002:0000eb1c       $chain$3$?CopySendBuffer@CClientLib@@QEAAHPEAVSendBuffer@@@Z 0000000140059b1c     ClientLib.obj
 0002:0000eb2c       $unwind$?ProcessSocketEvent@CClientLib@@QEAAXXZ 0000000140059b2c     ClientLib.obj
 0002:0000eb50       $stateUnwindMap$?SendDiv@CGMSConnManager@@AEAAHEEEPEADK@Z 0000000140059b50     GMSConnManager.obj
 0002:0000eb50       $stateUnwindMap$?ProcessSocketEvent@CClientLib@@QEAAXXZ 0000000140059b50     ClientLib.obj
 0002:0000eb58       $ip2state$?ProcessSocketEvent@CClientLib@@QEAAXXZ 0000000140059b58     ClientLib.obj
 0002:0000eb70       $unwind$?CopyFromUserDataArea@CPacket@@QEAAHPEAXK@Z 0000000140059b70     Packet.obj
 0002:0000eb80       $chain$3$?CopyFromUserDataArea@CPacket@@QEAAHPEAXK@Z 0000000140059b80     Packet.obj
 0002:0000eba0       $chain$4$?CopyFromUserDataArea@CPacket@@QEAAHPEAXK@Z 0000000140059ba0     Packet.obj
 0002:0000ebb0       $unwind$??0CSFGameServerClientLib@@QEAA@XZ 0000000140059bb0     SFGameServerClientLib.obj
 0002:0000ebc4       $unwind$?Connect@CSFGameServerClientLib@@QEAAHH@Z 0000000140059bc4     SFGameServerClientLib.obj
 0002:0000ebf0       $stateUnwindMap$?Connect@CSFGameServerClientLib@@QEAAHH@Z 0000000140059bf0     SFGameServerClientLib.obj
 0002:0000ebf8       $ip2state$?Connect@CSFGameServerClientLib@@QEAAHH@Z 0000000140059bf8     SFGameServerClientLib.obj
 0002:0000ec10       $unwind$??1mailer@jwsmtp@@QEAA@XZ 0000000140059c10     mailer.obj
 0002:0000ec10       $unwind$?CloseSocket@CSFGameServerClientLib@@UEAAHXZ 0000000140059c10     SFGameServerClientLib.obj
 0002:0000ec10       $unwind$?RECV_MSG_BAN_USER@CGameServerManagerDlg@@AEAAXFPEAUPROTO_BAN_USER_tag@@@Z 0000000140059c10     GameServerManagerDlg.obj
 0002:0000ec10       $unwind$?_Change_array@?$vector@DV?$allocator@D@std@@@std@@AEAAXQEAD_K1@Z 0000000140059c10     mailer.obj
 0002:0000ec10       $unwind$?MD5Update@MD5@@QEAAXPEAUMD5_CTX@@PEAEI@Z 0000000140059c10     md55d7732e46e8b0b019ace15d3c50ded71.obj
 0002:0000ec10       $unwind$??0PROTO_GAME_USER_INFO_tag@@QEAA@XZ 0000000140059c10     DividePacket.obj
 0002:0000ec24       $unwind$?ReadData@GAMEPROTO_SC_REMOVECLIENT@@UEAA_NPEAVILTMessage_Read@@@Z 0000000140059c24     AppInfoDlg.obj
 0002:0000ec24       $unwind$?ReadData@GAMEPROTO_SC_HOST_STAT@@UEAA_NPEAVILTMessage_Read@@@Z 0000000140059c24     AppInfoDlg.obj
 0002:0000ec30       $unwind$?ReadData@GAMEPROTO_SC_HOST_USER_STAT@@UEAA_NPEAVILTMessage_Read@@@Z 0000000140059c30     AppInfoDlg.obj
 0002:0000ec3c       $chain$2$?ReadData@GAMEPROTO_SC_HOST_USER_STAT@@UEAA_NPEAVILTMessage_Read@@@Z 0000000140059c3c     AppInfoDlg.obj
 0002:0000ec58       $chain$3$?ReadData@GAMEPROTO_SC_HOST_USER_STAT@@UEAA_NPEAVILTMessage_Read@@@Z 0000000140059c58     AppInfoDlg.obj
 0002:0000ec68       $chain$4$?ReadData@GAMEPROTO_SC_HOST_USER_STAT@@UEAA_NPEAVILTMessage_Read@@@Z 0000000140059c68     AppInfoDlg.obj
 0002:0000ec80       $chain$5$?ReadData@GAMEPROTO_SC_HOST_USER_STAT@@UEAA_NPEAVILTMessage_Read@@@Z 0000000140059c80     AppInfoDlg.obj
 0002:0000ec9c       $unwind$?IsProcessInTrouble@CHECK_MEM_USAGE@@YA_NPEAXHH@Z 0000000140059c9c     CheckMemUsage.obj
 0002:0000ec9c       $unwind$?WriteData@GAMEPROTO_SC_HOST_USER_STAT@@UEAA_NPEAVILTMessage_Write@@@Z 0000000140059c9c     AppInfoDlg.obj
 0002:0000ecb4       $unwind$?ReadData@GAMEPROTO_SS_GAMEEND@@UEAA_NPEAVILTMessage_Read@@@Z 0000000140059cb4     AppInfoDlg.obj
 0002:0000eccc       $unwind$?WriteData@GAMEPROTO_SS_GAMEEND@@UEAA_NPEAVILTMessage_Write@@@Z 0000000140059ccc     AppInfoDlg.obj
 0002:0000ece4       $unwind$?PostReadData@GAMEPROTO_COMMON@@UEAA_NPEAVILTMessage_Read@@@Z 0000000140059ce4     AppInfoDlg.obj
 0002:0000ecf0       $chain$0$?PostReadData@GAMEPROTO_COMMON@@UEAA_NPEAVILTMessage_Read@@@Z 0000000140059cf0     AppInfoDlg.obj
 0002:0000ed04       $chain$1$?PostReadData@GAMEPROTO_COMMON@@UEAA_NPEAVILTMessage_Read@@@Z 0000000140059d04     AppInfoDlg.obj
 0002:0000ed14       $unwind$?EmptyWorkingset@CHECK_MEM_USAGE@@YA_NPEAXH@Z 0000000140059d14     CheckMemUsage.obj
 0002:0000ed30       $stateUnwindMap$?ConnectToMatchMakingServer@CGameServerManagerDlg@@QEAAHXZ 0000000140059d30     GameServerManagerDlg.obj
 0002:0000ed30       $stateUnwindMap$?GetProcessMemoryUsage@@YAKPEAXH@Z 0000000140059d30     CheckMemUsage.obj
 0002:0000ed30       $stateUnwindMap$?EmptyWorkingset@CHECK_MEM_USAGE@@YA_NPEAXH@Z 0000000140059d30     CheckMemUsage.obj
 0002:0000ed48       $ip2state$?EmptyWorkingset@CHECK_MEM_USAGE@@YA_NPEAXH@Z 0000000140059d48     CheckMemUsage.obj
 0002:0000ed80       $unwind$?GetProcessMemoryUsage@@YAKPEAXH@Z 0000000140059d80     CheckMemUsage.obj
 0002:0000eda0       $ip2state$?GetProcessMemoryUsage@@YAKPEAXH@Z 0000000140059da0     CheckMemUsage.obj
 0002:0000edd8       $unwind$?clear@?$_Tree@V?$_Tmap_traits@GUExtraStatsMemVerify@CHostStat@@U?$less@G@std@@V?$allocator@U?$pair@$$CBGUExtraStatsMemVerify@CHostStat@@@std@@@4@$0A@@std@@@std@@QEAAXXZ 0000000140059dd8     HostStat.obj
 0002:0000edd8       $unwind$?clear@?$_Tree@V?$_Tmap_traits@GPEAUtagIP4Address@@U?$less@G@std@@V?$allocator@U?$pair@$$CBGPEAUtagIP4Address@@@std@@@3@$0A@@std@@@std@@QEAAXXZ 0000000140059dd8     cSnmpEX.obj
 0002:0000edd8       $unwind$?clear@?$_Tree@V?$_Tmap_traits@GUExtraStatsFPSVerify@CHostStat@@U?$less@G@std@@V?$allocator@U?$pair@$$CBGUExtraStatsFPSVerify@CHostStat@@@std@@@4@$0A@@std@@@std@@QEAAXXZ 0000000140059dd8     HostStat.obj
 0002:0000edf8       $ip2state$?clear@?$_Tree@V?$_Tmap_traits@GUExtraStatsFPSVerify@CHostStat@@U?$less@G@std@@V?$allocator@U?$pair@$$CBGUExtraStatsFPSVerify@CHostStat@@@std@@@4@$0A@@std@@@std@@QEAAXXZ 0000000140059df8     HostStat.obj
 0002:0000edf8       $ip2state$?clear@?$_Tree@V?$_Tmap_traits@GPEAUtagIP4Address@@U?$less@G@std@@V?$allocator@U?$pair@$$CBGPEAUtagIP4Address@@@std@@@3@$0A@@std@@@std@@QEAAXXZ 0000000140059df8     cSnmpEX.obj
 0002:0000edf8       $ip2state$?clear@?$_Tree@V?$_Tmap_traits@GUExtraStatsMemVerify@CHostStat@@U?$less@G@std@@V?$allocator@U?$pair@$$CBGUExtraStatsMemVerify@CHostStat@@@std@@@4@$0A@@std@@@std@@QEAAXXZ 0000000140059df8     HostStat.obj
 0002:0000ee00       $unwind$?SetMyServiceStatus@@YAXKK@Z 0000000140059e00     GameServerManager.obj
 0002:0000ee00       $unwind$?KillServiceWithErrorcode@@YAXPEAUSERVICE_STATUS_HANDLE__@@K@Z 0000000140059e00     GameServerManager.obj
 0002:0000ee10       $unwind$?InitInstance@CGameServerManagerApp@@UEAAHXZ 0000000140059e10     GameServerManager.obj
 0002:0000ee18       $unwind$?MyServiceMain@@YAXKPEAPEAD@Z 0000000140059e18     GameServerManager.obj
 0002:0000ee44       $stateUnwindMap$?MyServiceMain@@YAXKPEAPEAD@Z 0000000140059e44     GameServerManager.obj
 0002:0000ee50       $ip2state$?MyServiceMain@@YAXKPEAPEAD@Z 0000000140059e50     GameServerManager.obj
 0002:0000ee68       $unwind$?Init@GameServerIPCMemory@@QEAAXXZ 0000000140059e68     GameServerManagerDlg.obj
 0002:0000ee84       $unwind$?getDay@datetime@@IEAAHHH@Z 0000000140059e84     DateTime.obj
 0002:0000ee84       $unwind$??__Eg_cServerLog@@YAXXZ 0000000140059e84     GameServerManagerDlg.obj
 0002:0000ee94       $unwind$?GetGAME_MGMT_SETTING_FILE_PATH@@YAPEBDXZ 0000000140059e94     GameServerManagerDlg.obj
 0002:0000eea8       $unwind$?GetStringFormat@@YA?AV?$basic_string@DU?$char_traits@D@std@@V?$allocator@D@2@@std@@PEADZZ 0000000140059ea8     GameServerManagerDlg.obj
 0002:0000eec0       $unwind$?KillRemoteProcess@@YA_NK@Z 0000000140059ec0     GameServerManagerDlg.obj
 0002:0000eee0       $stateUnwindMap$?KillRemoteProcess@@YA_NK@Z 0000000140059ee0     GameServerManagerDlg.obj
 0002:0000ef20       $ip2state$?KillRemoteProcess@@YA_NK@Z 0000000140059f20     GameServerManagerDlg.obj
 0002:0000efa8       $unwind$??0CGameServerManagerDlg@@QEAA@PEAVCWnd@@@Z 0000000140059fa8     GameServerManagerDlg.obj
 0002:0000efc0       $stateUnwindMap$??0CGameServerManagerDlg@@QEAA@PEAVCWnd@@@Z 0000000140059fc0     GameServerManagerDlg.obj
 0002:0000f040       $ip2state$??0CGameServerManagerDlg@@QEAA@PEAVCWnd@@@Z 000000014005a040     GameServerManagerDlg.obj
 0002:0000f0a0       $unwind$??0GameServerIPCMemory@@QEAA@XZ 000000014005a0a0     GameServerManagerDlg.obj
 0002:0000f0a0       $unwind$??$_Traits_find@U?$char_traits@D@std@@@std@@YA_KQEBD_K101@Z 000000014005a0a0     CSmtp.obj
 0002:0000f0b8       $unwind$??1CGameServerManagerDlg@@UEAA@XZ 000000014005a0b8     GameServerManagerDlg.obj
 0002:0000f0d8       $ip2state$??1CGameServerManagerDlg@@UEAA@XZ 000000014005a0d8     GameServerManagerDlg.obj
 0002:0000f0f0       $unwind$?OnPaint@CGameServerManagerDlg@@IEAAXXZ 000000014005a0f0     GameServerManagerDlg.obj
 0002:0000f104       $chain$1$?OnPaint@CGameServerManagerDlg@@IEAAXXZ 000000014005a104     GameServerManagerDlg.obj
 0002:0000f11c       $chain$2$?OnPaint@CGameServerManagerDlg@@IEAAXXZ 000000014005a11c     GameServerManagerDlg.obj
 0002:0000f12c       $unwind$?InitializeManager@CGameServerManagerDlg@@QEAAHPEADKPEAPEAD@Z 000000014005a12c     GameServerManagerDlg.obj
 0002:0000f154       $stateUnwindMap$?InitializeManager@CGameServerManagerDlg@@QEAAHPEADKPEAPEAD@Z 000000014005a154     GameServerManagerDlg.obj
 0002:0000f190       $ip2state$?InitializeManager@CGameServerManagerDlg@@QEAAHPEADKPEAPEAD@Z 000000014005a190     GameServerManagerDlg.obj
 0002:0000f200       $unwind$?ReadSettings@CGameServerManagerDlg@@QEAAHXZ 000000014005a200     GameServerManagerDlg.obj
 0002:0000f22c       $stateUnwindMap$?ReadSettings@CGameServerManagerDlg@@QEAAHXZ 000000014005a22c     GameServerManagerDlg.obj
 0002:0000f238       $ip2state$?ReadSettings@CGameServerManagerDlg@@QEAAHXZ 000000014005a238     GameServerManagerDlg.obj
 0002:0000f250       $unwind$?ConnectToMatchMakingServer@CGameServerManagerDlg@@QEAAHXZ 000000014005a250     GameServerManagerDlg.obj
 0002:0000f278       $ip2state$?ConnectToMatchMakingServer@CGameServerManagerDlg@@QEAAHXZ 000000014005a278     GameServerManagerDlg.obj
 0002:0000f2b0       $unwind$?StartGameServer@CGameServerManagerDlg@@QEAAHF@Z 000000014005a2b0     GameServerManagerDlg.obj
 0002:0000f2d4       $stateUnwindMap$?StartGameServer@CGameServerManagerDlg@@QEAAHF@Z 000000014005a2d4     GameServerManagerDlg.obj
 0002:0000f2e0       $ip2state$?StartGameServer@CGameServerManagerDlg@@QEAAHF@Z 000000014005a2e0     GameServerManagerDlg.obj
 0002:0000f2f8       $unwind$?OnGameServerMsg@CGameServerManagerDlg@@IEAA_J_K_J@Z 000000014005a2f8     GameServerManagerDlg.obj
 0002:0000f320       $stateUnwindMap$?OnGameServerMsg@CGameServerManagerDlg@@IEAA_J_K_J@Z 000000014005a320     GameServerManagerDlg.obj
 0002:0000f350       $ip2state$?OnGameServerMsg@CGameServerManagerDlg@@IEAA_J_K_J@Z 000000014005a350     GameServerManagerDlg.obj
 0002:0000f3d0       $unwind$?KillServerApp@CGameServerManagerDlg@@IEAAXI_N@Z 000000014005a3d0     GameServerManagerDlg.obj
 0002:0000f3f8       $stateUnwindMap$?KillServerApp@CGameServerManagerDlg@@IEAAXI_N@Z 000000014005a3f8     GameServerManagerDlg.obj
 0002:0000f400       $ip2state$?KillServerApp@CGameServerManagerDlg@@IEAAXI_N@Z 000000014005a400     GameServerManagerDlg.obj
 0002:0000f418       $unwind$?OnTimer@CGameServerManagerDlg@@IEAAX_K@Z 000000014005a418     GameServerManagerDlg.obj
 0002:0000f440       $stateUnwindMap$?OnTimer@CGameServerManagerDlg@@IEAAX_K@Z 000000014005a440     GameServerManagerDlg.obj
 0002:0000f460       $ip2state$?OnTimer@CGameServerManagerDlg@@IEAAX_K@Z 000000014005a460     GameServerManagerDlg.obj
 0002:0000f4a8       $unwind$?OnButtonGo@CGameServerManagerDlg@@IEAAXXZ 000000014005a4a8     GameServerManagerDlg.obj
 0002:0000f4c0       $stateUnwindMap$?OnButtonGo@CGameServerManagerDlg@@IEAAXXZ 000000014005a4c0     GameServerManagerDlg.obj
 0002:0000f4c8       $ip2state$?OnButtonGo@CGameServerManagerDlg@@IEAAXXZ 000000014005a4c8     GameServerManagerDlg.obj
 0002:0000f4e0       $unwind$?TerminateGameServer@CGameServerManagerDlg@@QEAAXF@Z 000000014005a4e0     GameServerManagerDlg.obj
 0002:0000f504       $stateUnwindMap$?TerminateGameServer@CGameServerManagerDlg@@QEAAXF@Z 000000014005a504     GameServerManagerDlg.obj
 0002:0000f520       $ip2state$?TerminateGameServer@CGameServerManagerDlg@@QEAAXF@Z 000000014005a520     GameServerManagerDlg.obj
 0002:0000f558       $unwind$?SendMessageToWriteLogFile@CGameServerManagerDlg@@QEAAXFPEAUHWND__@@0AEAUtagCOPYDATASTRUCT@@@Z 000000014005a558     GameServerManagerDlg.obj
 0002:0000f568       $unwind$?VerifyServerAppTermination@CGameServerManagerDlg@@AEAAXXZ 000000014005a568     GameServerManagerDlg.obj
 0002:0000f590       $stateUnwindMap$?VerifyServerAppTermination@CGameServerManagerDlg@@AEAAXXZ 000000014005a590     GameServerManagerDlg.obj
 0002:0000f5c0       $ip2state$?VerifyServerAppTermination@CGameServerManagerDlg@@AEAAXXZ 000000014005a5c0     GameServerManagerDlg.obj
 0002:0000f618       $unwind$?StringSplitToNumArray@CGameServerManagerDlg@@AEAAXV?$basic_string@DU?$char_traits@D@std@@V?$allocator@D@2@@std@@0PEAHAEAH@Z 000000014005a618     GameServerManagerDlg.obj
 0002:0000f640       $stateUnwindMap$?StringSplitToNumArray@CGameServerManagerDlg@@AEAAXV?$basic_string@DU?$char_traits@D@std@@V?$allocator@D@2@@std@@0PEAHAEAH@Z 000000014005a640     GameServerManagerDlg.obj
 0002:0000f658       $ip2state$?StringSplitToNumArray@CGameServerManagerDlg@@AEAAXV?$basic_string@DU?$char_traits@D@std@@V?$allocator@D@2@@std@@0PEAHAEAH@Z 000000014005a658     GameServerManagerDlg.obj
 0002:0000f688       $unwind$?FindFreePorts@CGameServerManagerDlg@@AEAA_NXZ 000000014005a688     GameServerManagerDlg.obj
 0002:0000f6b4       $stateUnwindMap$?FindFreePorts@CGameServerManagerDlg@@AEAA_NXZ 000000014005a6b4     GameServerManagerDlg.obj
 0002:0000f6c8       $ip2state$?FindFreePorts@CGameServerManagerDlg@@AEAA_NXZ 000000014005a6c8     GameServerManagerDlg.obj
 0002:0000f6f0       $unwind$?RestoreFreePort@CGameServerManagerDlg@@AEAAXXZ 000000014005a6f0     GameServerManagerDlg.obj
 0002:0000f718       $stateUnwindMap$?LoadWMszFile@FindXlsMsg@@QEAA_NPEAD@Z 000000014005a718     LoadXlsMsg.obj
 0002:0000f718       $stateUnwindMap$?AssignServerApp@CGameServerManagerDlg@@AEAAXAEBUPROTO_AUTOMATCH_GAME_START_REQ@@F@Z 000000014005a718     GameServerManagerDlg.obj
 0002:0000f718       $stateUnwindMap$?RestoreFreePort@CGameServerManagerDlg@@AEAAXXZ 000000014005a718     GameServerManagerDlg.obj
 0002:0000f720       $ip2state$?RestoreFreePort@CGameServerManagerDlg@@AEAAXXZ 000000014005a720     GameServerManagerDlg.obj
 0002:0000f738       $unwind$?ReservePort@CGameServerManagerDlg@@AEAAXIF@Z 000000014005a738     GameServerManagerDlg.obj
 0002:0000f744       $chain$0$?ReservePort@CGameServerManagerDlg@@AEAAXIF@Z 000000014005a744     GameServerManagerDlg.obj
 0002:0000f758       $chain$1$?ReservePort@CGameServerManagerDlg@@AEAAXIF@Z 000000014005a758     GameServerManagerDlg.obj
 0002:0000f768       $unwind$?ChangeNumRoomsReserved@CGameServerManagerDlg@@QEAAXHH_N@Z 000000014005a768     GameServerManagerDlg.obj
 0002:0000f768       $unwind$?ChangeNumActiveServers@CGameServerManagerDlg@@QEAAXH@Z 000000014005a768     GameServerManagerDlg.obj
 0002:0000f770       $unwind$?ServerAppUseCountLog@CGameServerManagerDlg@@AEAAXXZ 000000014005a770     GameServerManagerDlg.obj
 0002:0000f788       $unwind$??0CSharedMemoryLoader@@QEAA@XZ 000000014005a788     GameServerManagerDlg.obj
 0002:0000f7ac       $stateUnwindMap$??0CSharedMemoryLoader@@QEAA@XZ 000000014005a7ac     GameServerManagerDlg.obj
 0002:0000f7d8       $ip2state$??0CSharedMemoryLoader@@QEAA@XZ 000000014005a7d8     GameServerManagerDlg.obj
 0002:0000f808       $unwind$?_PreLoad@CSharedMemoryLoader@@AEAA_NXZ 000000014005a808     GameServerManagerDlg.obj
 0002:0000f820       $stateUnwindMap$?_PreLoad@CSharedMemoryLoader@@AEAA_NXZ 000000014005a820     GameServerManagerDlg.obj
 0002:0000f830       $ip2state$?_PreLoad@CSharedMemoryLoader@@AEAA_NXZ 000000014005a830     GameServerManagerDlg.obj
 0002:0000f858       $unwind$?_Load@CSharedMemoryLoader@@AEAA_NXZ 000000014005a858     GameServerManagerDlg.obj
 0002:0000f87c       $stateUnwindMap$?_Load@CSharedMemoryLoader@@AEAA_NXZ 000000014005a87c     GameServerManagerDlg.obj
 0002:0000f8d0       $ip2state$?_Load@CSharedMemoryLoader@@AEAA_NXZ 000000014005a8d0     GameServerManagerDlg.obj
 0002:0000f958       $unwind$?Load@CSharedMemoryLoader@@QEAA_NXZ 000000014005a958     GameServerManagerDlg.obj
 0002:0000f970       $stateUnwindMap$?Load@CSharedMemoryLoader@@QEAA_NXZ 000000014005a970     GameServerManagerDlg.obj
 0002:0000f980       $ip2state$?Load@CSharedMemoryLoader@@QEAA_NXZ 000000014005a980     GameServerManagerDlg.obj
 0002:0000f9a8       $unwind$?ProcessThread@CGameServerManagerDlg@@CAIPEAX@Z 000000014005a9a8     GameServerManagerDlg.obj
 0002:0000f9bc       $unwind$?OnCopyData@CGameServerManagerDlg@@IEAAHPEAVCWnd@@PEAUtagCOPYDATASTRUCT@@@Z 000000014005a9bc     GameServerManagerDlg.obj
 0002:0000f9d8       $unwind$?RECV_MSG_REMOVE_CLIENT@CGameServerManagerDlg@@AEAAXFPEBUGAMEPROTO_SC_REMOVECLIENT@@@Z 000000014005a9d8     GameServerManagerDlg.obj
 0002:0000f9e8       $unwind$?RECV_MSG_GAMEEND@CGameServerManagerDlg@@AEAAXFPEBUGAMEPROTO_SS_GAMEEND@@@Z 000000014005a9e8     GameServerManagerDlg.obj
 0002:0000fa10       $stateUnwindMap$?RECV_MSG_GAMEEND@CGameServerManagerDlg@@AEAAXFPEBUGAMEPROTO_SS_GAMEEND@@@Z 000000014005aa10     GameServerManagerDlg.obj
 0002:0000fa20       $ip2state$?RECV_MSG_GAMEEND@CGameServerManagerDlg@@AEAAXFPEBUGAMEPROTO_SS_GAMEEND@@@Z 000000014005aa20     GameServerManagerDlg.obj
 0002:0000fa40       $unwind$?RECV_MSG_HOST_USER_STAT@CGameServerManagerDlg@@AEAAXFPEBUGAMEPROTO_SC_HOST_USER_STAT@@@Z 000000014005aa40     GameServerManagerDlg.obj
 0002:0000fa5c       $chain$2$?RECV_MSG_HOST_USER_STAT@CGameServerManagerDlg@@AEAAXFPEBUGAMEPROTO_SC_HOST_USER_STAT@@@Z 000000014005aa5c     GameServerManagerDlg.obj
 0002:0000fa78       $chain$3$?RECV_MSG_HOST_USER_STAT@CGameServerManagerDlg@@AEAAXFPEBUGAMEPROTO_SC_HOST_USER_STAT@@@Z 000000014005aa78     GameServerManagerDlg.obj
 0002:0000fa88       $unwind$?RECV_MSG_HOST_STAT@CGameServerManagerDlg@@AEAAXFPEBUGAMEPROTO_SC_HOST_STAT@@@Z 000000014005aa88     GameServerManagerDlg.obj
 0002:0000faa0       $unwind$?RECV_MSG_MAPLOADING_COMPLETE_NTY@CGameServerManagerDlg@@AEAAXFPEAUPROTO_GAMEGT_MAPLOADING_COMPLETE_NTY_tag@@@Z 000000014005aaa0     GameServerManagerDlg.obj
 0002:0000faa0       $unwind$?RECV_MSG_AI2_BONUSROUND_REWARD@CGameServerManagerDlg@@AEAAXFPEAUPROTOCOL_AI2_BONUSROUND_REWARD_REQ_tag@@@Z 000000014005aaa0     GameServerManagerDlg.obj
 0002:0000faa0       $unwind$?RECV_MSG_AI3_BONUS_REWARD_ITEM@CGameServerManagerDlg@@AEAAXFPEAUPROTO_GAMEGT_INGAME_AI3_BONUS_REWARD_ITEM_REQ@@@Z 000000014005aaa0     GameServerManagerDlg.obj
 0002:0000faa0       $unwind$?RECV_MSG_FINISHED_GAME_PREV@CGameServerManagerDlg@@AEAAXFPEAUPROTO_FINISHED_GAME_PREV_tag@@@Z 000000014005aaa0     GameServerManagerDlg.obj
 0002:0000faa0       $unwind$?RECV_MSG_INGAME_AIGACHA_ITEM_INSERT@CGameServerManagerDlg@@AEAAXFPEAUPROTO_GAMEGT_INGAME_AIGACHA_ITEM_INSERT@@@Z 000000014005aaa0     GameServerManagerDlg.obj
 0002:0000faa0       $unwind$md4_finish_ctx     000000014005aaa0     md4.obj
 0002:0000faa0       $unwind$?RECV_MSG_INGAME_FARMING_ITEM_REQ@CGameServerManagerDlg@@AEAAXFPEAUPROTO_GAMEGT_INGAME_FARMING_ITEM_REQ@@@Z 000000014005aaa0     GameServerManagerDlg.obj
 0002:0000fab4       $unwind$?RECV_MSG_SPY_CHANGE@CGameServerManagerDlg@@AEAAXFPEAUGAMEPROTO_SC_SPY_CHANGE@@@Z 000000014005aab4     GameServerManagerDlg.obj
 0002:0000facc       $unwind$?RECV_MSG_AI_EXTRA_REWARD@CGameServerManagerDlg@@AEAAXFPEAUPROTO_AI_EXTRA_REWARD_REQ@@@Z 000000014005aacc     GameServerManagerDlg.obj
 0002:0000faf0       $stateUnwindMap$?Send@CGMSConnManager@@AEAAHPEAVCPacket@@@Z 000000014005aaf0     GMSConnManager.obj
 0002:0000faf0       $stateUnwindMap$?RECV_MSG_AI_EXTRA_REWARD@CGameServerManagerDlg@@AEAAXFPEAUPROTO_AI_EXTRA_REWARD_REQ@@@Z 000000014005aaf0     GameServerManagerDlg.obj
 0002:0000faf8       $ip2state$?RECV_MSG_AI_EXTRA_REWARD@CGameServerManagerDlg@@AEAAXFPEAUPROTO_AI_EXTRA_REWARD_REQ@@@Z 000000014005aaf8     GameServerManagerDlg.obj
 0002:0000fb10       $unwind$?RECV_MSG_SPEC_RECOMMENDROOM_INGAME_DATA@CGameServerManagerDlg@@AEAAXFPEBUPROTO_SPEC_RECOMMENDROOM_INGAME_DATA@@@Z 000000014005ab10     GameServerManagerDlg.obj
 0002:0000fb28       $unwind$?RECV_MSG_AUTO_SIDE_CHANGE_TEAM_INFO_NTY@CGameServerManagerDlg@@AEAAXFPEAUPROTO_GAMEGT_AUTO_SIDE_CHANGE_TEAM_INFO_NTY@@@Z 000000014005ab28     GameServerManagerDlg.obj
 0002:0000fb3c       $unwind$?SendToGmsStartingGameRes@CGameServerManagerDlg@@AEAAXAEBUGAMESERVERINFO@@FW4START_HOST_RESULT@@@Z 000000014005ab3c     GameServerManagerDlg.obj
 0002:0000fb3c       $unwind$?RECV_MSG_INSERTCHARACTER_ACK@CGameServerManagerDlg@@AEAAXFPEBUPROTO_INSERT_CHARACTER_RESULT_tag@@@Z 000000014005ab3c     GameServerManagerDlg.obj
 0002:0000fb50       $unwind$?OnReceive@CGameServerManagerDlg@@UEAAXPEAVCPacket@@@Z 000000014005ab50     GameServerManagerDlg.obj
 0002:0000fb58       $chain$1$?OnReceive@CGameServerManagerDlg@@UEAAXPEAVCPacket@@@Z 000000014005ab58     GameServerManagerDlg.obj
 0002:0000fb70       $chain$7$?OnReceive@CGameServerManagerDlg@@UEAAXPEAVCPacket@@@Z 000000014005ab70     GameServerManagerDlg.obj
 0002:0000fb98       $chain$8$?OnReceive@CGameServerManagerDlg@@UEAAXPEAVCPacket@@@Z 000000014005ab98     GameServerManagerDlg.obj
 0002:0000fba8       $chain$9$?OnReceive@CGameServerManagerDlg@@UEAAXPEAVCPacket@@@Z 000000014005aba8     GameServerManagerDlg.obj
 0002:0000fbb8       $unwind$?OnReceiveFromGms@CGameServerManagerDlg@@AEAAXPEAVCPacket@@@Z 000000014005abb8     GameServerManagerDlg.obj
 0002:0000fbd0       $chain$4$?OnReceiveFromGms@CGameServerManagerDlg@@AEAAXPEAVCPacket@@@Z 000000014005abd0     GameServerManagerDlg.obj
 0002:0000fbf4       $chain$5$?OnReceiveFromGms@CGameServerManagerDlg@@AEAAXPEAVCPacket@@@Z 000000014005abf4     GameServerManagerDlg.obj
 0002:0000fc04       $unwind$?OnReceiveFromGms@CGameServerManagerDlg@@AEAAXAEBUPROTO_STARTING_GAME_tag@@@Z 000000014005ac04     GameServerManagerDlg.obj
 0002:0000fc2c       $stateUnwindMap$?OnReceiveFromGms@CGameServerManagerDlg@@AEAAXAEBUPROTO_STARTING_GAME_tag@@@Z 000000014005ac2c     GameServerManagerDlg.obj
 0002:0000fc2c       $stateUnwindMap$?OnReceiveFromGms@CGameServerManagerDlg@@AEAAXAEBUPROTO_AUTOMATCH_GAME_START_REQ@@@Z 000000014005ac2c     GameServerManagerDlg.obj
 0002:0000fc50       $ip2state$?OnReceiveFromGms@CGameServerManagerDlg@@AEAAXAEBUPROTO_STARTING_GAME_tag@@@Z 000000014005ac50     GameServerManagerDlg.obj
 0002:0000fc90       $unwind$?OnReceiveFromGms@CGameServerManagerDlg@@AEAAXAEBUPROTO_INSERT_CHARACTER_tag@@@Z 000000014005ac90     GameServerManagerDlg.obj
 0002:0000fcb8       $stateUnwindMap$?OnReceiveFromGms@CGameServerManagerDlg@@AEAAXAEBUPROTO_INSERT_CHARACTER_tag@@@Z 000000014005acb8     GameServerManagerDlg.obj
 0002:0000fcc8       $ip2state$?OnReceiveFromGms@CGameServerManagerDlg@@AEAAXAEBUPROTO_INSERT_CHARACTER_tag@@@Z 000000014005acc8     GameServerManagerDlg.obj
 0002:0000fcf0       $unwind$?OnReceiveFromGms@CGameServerManagerDlg@@AEAAXAEBUPROTO_MMSERVER_TERMINATED_tag@@@Z 000000014005acf0     GameServerManagerDlg.obj
 0002:0000fd14       $stateUnwindMap$?OnReceiveFromGms@CGameServerManagerDlg@@AEAAXAEBUPROTO_MMSERVER_TERMINATED_tag@@@Z 000000014005ad14     GameServerManagerDlg.obj
 0002:0000fd20       $ip2state$?OnReceiveFromGms@CGameServerManagerDlg@@AEAAXAEBUPROTO_MMSERVER_TERMINATED_tag@@@Z 000000014005ad20     GameServerManagerDlg.obj
 0002:0000fd38       $unwind$?OnReceiveFromGms@CGameServerManagerDlg@@AEAAXAEBUPROTO_USER_DISCONNECTED_tag@@@Z 000000014005ad38     GameServerManagerDlg.obj
 0002:0000fd4c       $chain$1$?OnReceiveFromGms@CGameServerManagerDlg@@AEAAXAEBUPROTO_USER_DISCONNECTED_tag@@@Z 000000014005ad4c     GameServerManagerDlg.obj
 0002:0000fd64       $chain$2$?OnReceiveFromGms@CGameServerManagerDlg@@AEAAXAEBUPROTO_USER_DISCONNECTED_tag@@@Z 000000014005ad64     GameServerManagerDlg.obj
 0002:0000fd74       $unwind$?OnReceiveFromGms@CGameServerManagerDlg@@AEAAXAEBUPROTO_GAMEGT_INGAME_AIGACHA_ITEM_INSERT_RESULT@@@Z 000000014005ad74     GameServerManagerDlg.obj
 0002:0000fd8c       $unwind$?OnReceiveFromGms@CGameServerManagerDlg@@AEAAXAEBUPROTO_AUTOMATCH_GAME_START_REQ@@@Z 000000014005ad8c     GameServerManagerDlg.obj
 0002:0000fdc0       $ip2state$?OnReceiveFromGms@CGameServerManagerDlg@@AEAAXAEBUPROTO_AUTOMATCH_GAME_START_REQ@@@Z 000000014005adc0     GameServerManagerDlg.obj
 0002:0000fe00       $unwind$?OnReceiveFromGms@CGameServerManagerDlg@@AEAAXAEBUPROTO_AUTOMATCH_GAME_ENTER_REQ@@@Z 000000014005ae00     GameServerManagerDlg.obj
 0002:0000fe28       $stateUnwindMap$?OnReceiveFromGms@CGameServerManagerDlg@@AEAAXAEBUPROTO_AUTOMATCH_GAME_ENTER_REQ@@@Z 000000014005ae28     GameServerManagerDlg.obj
 0002:0000fe50       $ip2state$?OnReceiveFromGms@CGameServerManagerDlg@@AEAAXAEBUPROTO_AUTOMATCH_GAME_ENTER_REQ@@@Z 000000014005ae50     GameServerManagerDlg.obj
 0002:0000fe90       $unwind$?FindServerApp@CGameServerManagerDlg@@AEAA?B_NFKAEAF@Z 000000014005ae90     GameServerManagerDlg.obj
 0002:0000fea4       $unwind$?AssignServerApp@CGameServerManagerDlg@@AEAAXAEBUPROTO_STARTING_GAME_tag@@F@Z 000000014005aea4     GameServerManagerDlg.obj
 0002:0000fec8       $stateUnwindMap$?AssignServerApp@CGameServerManagerDlg@@AEAAXAEBUPROTO_STARTING_GAME_tag@@F@Z 000000014005aec8     GameServerManagerDlg.obj
 0002:0000fed0       $ip2state$?AssignServerApp@CGameServerManagerDlg@@AEAAXAEBUPROTO_STARTING_GAME_tag@@F@Z 000000014005aed0     GameServerManagerDlg.obj
 0002:0000fee8       $unwind$?AssignServerApp@CGameServerManagerDlg@@AEAAXAEBUPROTO_AUTOMATCH_GAME_START_REQ@@F@Z 000000014005aee8     GameServerManagerDlg.obj
 0002:0000ff10       $ip2state$?AssignServerApp@CGameServerManagerDlg@@AEAAXAEBUPROTO_AUTOMATCH_GAME_START_REQ@@F@Z 000000014005af10     GameServerManagerDlg.obj
 0002:0000ff28       $unwind$?SendToGmsAutoMatchGameStartRes@CGameServerManagerDlg@@AEAAXAEBUGAMESERVERINFO@@FW4START_HOST_RESULT@@@Z 000000014005af28     GameServerManagerDlg.obj
 0002:0000ff44       $unwind$?SendToGmsAutoMatchGameEnterNty@CGameServerManagerDlg@@AEAAXF@Z 000000014005af44     GameServerManagerDlg.obj
 0002:0000ff5c       $chain$0$?SendToGmsAutoMatchGameEnterNty@CGameServerManagerDlg@@AEAAXF@Z 000000014005af5c     GameServerManagerDlg.obj
 0002:0000ff70       $chain$1$?SendToGmsAutoMatchGameEnterNty@CGameServerManagerDlg@@AEAAXF@Z 000000014005af70     GameServerManagerDlg.obj
 0002:0000ff80       $unwind$?SendToServerAppAutoMatchGameEnterNty@CGameServerManagerDlg@@AEAAXF@Z 000000014005af80     GameServerManagerDlg.obj
 0002:0000ff8c       $chain$0$?SendToServerAppAutoMatchGameEnterNty@CGameServerManagerDlg@@AEAAXF@Z 000000014005af8c     GameServerManagerDlg.obj
 0002:0000ffa0       $chain$1$?SendToServerAppAutoMatchGameEnterNty@CGameServerManagerDlg@@AEAAXF@Z 000000014005afa0     GameServerManagerDlg.obj
 0002:0000ffb0       $unwind$??1?$shared_ptr@UGAMESERVERINFO@@@std@@QEAA@XZ 000000014005afb0     GameServerManagerDlg.obj
 0002:0000ffc8       $ip2state$??1?$shared_ptr@UGAMESERVERINFO@@@std@@QEAA@XZ 000000014005afc8     GameServerManagerDlg.obj
 0002:0000ffd0       $unwind$??1?$list@UverifyTerminationStatus_t@@V?$allocator@UverifyTerminationStatus_t@@@std@@@std@@QEAA@XZ 000000014005afd0     GameServerManagerDlg.obj
 0002:0000ffd8       $chain$0$??1?$list@UverifyTerminationStatus_t@@V?$allocator@UverifyTerminationStatus_t@@@std@@@std@@QEAA@XZ 000000014005afd8     GameServerManagerDlg.obj
 0002:0000ffec       $chain$1$??1?$list@UverifyTerminationStatus_t@@V?$allocator@UverifyTerminationStatus_t@@@std@@@std@@QEAA@XZ 000000014005afec     GameServerManagerDlg.obj
 0002:0000fffc       $unwind$?clear@?$_Tree@V?$_Tmap_traits@IUPORTINFO@@U?$less@I@std@@V?$allocator@U?$pair@$$CBIUPORTINFO@@@std@@@3@$0A@@std@@@std@@QEAAXXZ 000000014005affc     GameServerManagerDlg.obj
 0002:00010018       $ip2state$?clear@?$_Tree@V?$_Tmap_traits@IUPORTINFO@@U?$less@I@std@@V?$allocator@U?$pair@$$CBIUPORTINFO@@@std@@@3@$0A@@std@@@std@@QEAAXXZ 000000014005b018     GameServerManagerDlg.obj
 0002:00010020       $unwind$?find_first_of@?$basic_string@DU?$char_traits@D@std@@V?$allocator@D@2@@std@@QEBA_KAEBV12@_K@Z 000000014005b020     GameServerManagerDlg.obj
 0002:00010040       $unwind$?reserve@?$basic_string@DU?$char_traits@D@std@@V?$allocator@D@2@@std@@QEAAX_K@Z 000000014005b040     GameServerManagerDlg.obj
 0002:0001004c       $chain$0$?reserve@?$basic_string@DU?$char_traits@D@std@@V?$allocator@D@2@@std@@QEAAX_K@Z 000000014005b04c     GameServerManagerDlg.obj
 0002:00010060       $chain$2$?reserve@?$basic_string@DU?$char_traits@D@std@@V?$allocator@D@2@@std@@QEAAX_K@Z 000000014005b060     GameServerManagerDlg.obj
 0002:00010078       $chain$3$?reserve@?$basic_string@DU?$char_traits@D@std@@V?$allocator@D@2@@std@@QEAAX_K@Z 000000014005b078     GameServerManagerDlg.obj
 0002:00010088       $chain$4$?reserve@?$basic_string@DU?$char_traits@D@std@@V?$allocator@D@2@@std@@QEAAX_K@Z 000000014005b088     GameServerManagerDlg.obj
 0002:00010098       $chain$5$?reserve@?$basic_string@DU?$char_traits@D@std@@V?$allocator@D@2@@std@@QEAAX_K@Z 000000014005b098     GameServerManagerDlg.obj
 0002:000100b4       $unwind$??$_Setp@UGAMESERVERINFO@@@?$shared_ptr@UGAMESERVERINFO@@@std@@AEAAXPEAUGAMESERVERINFO@@U?$integral_constant@_N$0A@@1@@Z 000000014005b0b4     GameServerManagerDlg.obj
 0002:000100c8       $tryMap$??$_Setp@UGAMESERVERINFO@@@?$shared_ptr@UGAMESERVERINFO@@@std@@AEAAXPEAUGAMESERVERINFO@@U?$integral_constant@_N$0A@@1@@Z 000000014005b0c8     GameServerManagerDlg.obj
 0002:000100dc       $handlerMap$0$??$_Setp@UGAMESERVERINFO@@@?$shared_ptr@UGAMESERVERINFO@@@std@@AEAAXPEAUGAMESERVERINFO@@U?$integral_constant@_N$0A@@1@@Z 000000014005b0dc     GameServerManagerDlg.obj
 0002:000100f0       $ip2state$??$_Setp@UGAMESERVERINFO@@@?$shared_ptr@UGAMESERVERINFO@@@std@@AEAAXPEAUGAMESERVERINFO@@U?$integral_constant@_N$0A@@1@@Z 000000014005b0f0     GameServerManagerDlg.obj
 0002:00010100       $unwind$?catch$1@?0???$_Setp@UGAMESERVERINFO@@@?$shared_ptr@UGAMESERVERINFO@@@std@@AEAAXPEAUGAMESERVERINFO@@U?$integral_constant@_N$0A@@1@@Z@4HA 000000014005b100     GameServerManagerDlg.obj
 0002:00010110       $unwind$??$_Insert_nohint@AEAU?$pair@$$CBIUPORTINFO@@@std@@PEAU?$_Tree_node@U?$pair@$$CBIUPORTINFO@@@std@@PEAX@2@@?$_Tree@V?$_Tmap_traits@IUPORTINFO@@U?$less@I@std@@V?$allocator@U?$pair@$$CBIUPORTINFO@@@std@@@3@$0A@@std@@@std@@IEAA?AU?$pair@V?$_Tree_iterator@V?$_Tree_val@U?$_Tree_simple_types@U?$pair@$$CBIUPORTINFO@@@std@@@std@@@std@@@std@@_N@1@_NAEAU?$pair@$$CBIUPORTINFO@@@1@PEAU?$_Tree_node@U?$pair@$$CBIUPORTINFO@@@std@@PEAX@1@@Z 000000014005b110     GameServerManagerDlg.obj
 0002:0001012c       $tryMap$??$_Insert_nohint@AEAU?$pair@$$CBIUPORTINFO@@@std@@PEAU?$_Tree_node@U?$pair@$$CBIUPORTINFO@@@std@@PEAX@2@@?$_Tree@V?$_Tmap_traits@IUPORTINFO@@U?$less@I@std@@V?$allocator@U?$pair@$$CBIUPORTINFO@@@std@@@3@$0A@@std@@@std@@IEAA?AU?$pair@V?$_Tree_iterator@V?$_Tree_val@U?$_Tree_simple_types@U?$pair@$$CBIUPORTINFO@@@std@@@std@@@std@@@std@@_N@1@_NAEAU?$pair@$$CBIUPORTINFO@@@1@PEAU?$_Tree_node@U?$pair@$$CBIUPORTINFO@@@std@@PEAX@1@@Z 000000014005b12c     GameServerManagerDlg.obj
 0002:00010140       $handlerMap$0$??$_Insert_nohint@AEAU?$pair@$$CBIUPORTINFO@@@std@@PEAU?$_Tree_node@U?$pair@$$CBIUPORTINFO@@@std@@PEAX@2@@?$_Tree@V?$_Tmap_traits@IUPORTINFO@@U?$less@I@std@@V?$allocator@U?$pair@$$CBIUPORTINFO@@@std@@@3@$0A@@std@@@std@@IEAA?AU?$pair@V?$_Tree_iterator@V?$_Tree_val@U?$_Tree_simple_types@U?$pair@$$CBIUPORTINFO@@@std@@@std@@@std@@@std@@_N@1@_NAEAU?$pair@$$CBIUPORTINFO@@@1@PEAU?$_Tree_node@U?$pair@$$CBIUPORTINFO@@@std@@PEAX@1@@Z 000000014005b140     GameServerManagerDlg.obj
 0002:00010158       $ip2state$??$_Insert_nohint@AEAU?$pair@$$CBIUPORTINFO@@@std@@PEAU?$_Tree_node@U?$pair@$$CBIUPORTINFO@@@std@@PEAX@2@@?$_Tree@V?$_Tmap_traits@IUPORTINFO@@U?$less@I@std@@V?$allocator@U?$pair@$$CBIUPORTINFO@@@std@@@3@$0A@@std@@@std@@IEAA?AU?$pair@V?$_Tree_iterator@V?$_Tree_val@U?$_Tree_simple_types@U?$pair@$$CBIUPORTINFO@@@std@@@std@@@std@@@std@@_N@1@_NAEAU?$pair@$$CBIUPORTINFO@@@1@PEAU?$_Tree_node@U?$pair@$$CBIUPORTINFO@@@std@@PEAX@1@@Z 000000014005b158     GameServerManagerDlg.obj
 0002:00010168       $unwind$?catch$0@?0???$_Insert_nohint@AEAU?$pair@$$CBIUPORTINFO@@@std@@PEAU?$_Tree_node@U?$pair@$$CBIUPORTINFO@@@std@@PEAX@2@@?$_Tree@V?$_Tmap_traits@IUPORTINFO@@U?$less@I@std@@V?$allocator@U?$pair@$$CBIUPORTINFO@@@std@@@3@$0A@@std@@@std@@IEAA?AU?$pair@V?$_Tree_iterator@V?$_Tree_val@U?$_Tree_simple_types@U?$pair@$$CBIUPORTINFO@@@std@@@std@@@std@@@std@@_N@1@_NAEAU?$pair@$$CBIUPORTINFO@@@1@PEAU?$_Tree_node@U?$pair@$$CBIUPORTINFO@@@std@@PEAX@1@@Z@4HA 000000014005b168     GameServerManagerDlg.obj
 0002:00010178       $unwind$??$_Insert_hint@AEAU?$pair@$$CBIUPORTINFO@@@std@@PEAU?$_Tree_node@U?$pair@$$CBIUPORTINFO@@@std@@PEAX@2@@?$_Tree@V?$_Tmap_traits@IUPORTINFO@@U?$less@I@std@@V?$allocator@U?$pair@$$CBIUPORTINFO@@@std@@@3@$0A@@std@@@std@@IEAA?AV?$_Tree_iterator@V?$_Tree_val@U?$_Tree_simple_types@U?$pair@$$CBIUPORTINFO@@@std@@@std@@@std@@@1@V?$_Tree_const_iterator@V?$_Tree_val@U?$_Tree_simple_types@U?$pair@$$CBIUPORTINFO@@@std@@@std@@@std@@@1@AEAU?$pair@$$CBIUPORTINFO@@@1@PEAU?$_Tree_node@U?$pair@$$CBIUPORTINFO@@@std@@PEAX@1@@Z 000000014005b178     GameServerManagerDlg.obj
 0002:00010190       $tryMap$??$_Insert_hint@AEAU?$pair@$$CBIUPORTINFO@@@std@@PEAU?$_Tree_node@U?$pair@$$CBIUPORTINFO@@@std@@PEAX@2@@?$_Tree@V?$_Tmap_traits@IUPORTINFO@@U?$less@I@std@@V?$allocator@U?$pair@$$CBIUPORTINFO@@@std@@@3@$0A@@std@@@std@@IEAA?AV?$_Tree_iterator@V?$_Tree_val@U?$_Tree_simple_types@U?$pair@$$CBIUPORTINFO@@@std@@@std@@@std@@@1@V?$_Tree_const_iterator@V?$_Tree_val@U?$_Tree_simple_types@U?$pair@$$CBIUPORTINFO@@@std@@@std@@@std@@@1@AEAU?$pair@$$CBIUPORTINFO@@@1@PEAU?$_Tree_node@U?$pair@$$CBIUPORTINFO@@@std@@PEAX@1@@Z 000000014005b190     GameServerManagerDlg.obj
 0002:000101a4       $handlerMap$0$??$_Insert_hint@AEAU?$pair@$$CBIUPORTINFO@@@std@@PEAU?$_Tree_node@U?$pair@$$CBIUPORTINFO@@@std@@PEAX@2@@?$_Tree@V?$_Tmap_traits@IUPORTINFO@@U?$less@I@std@@V?$allocator@U?$pair@$$CBIUPORTINFO@@@std@@@3@$0A@@std@@@std@@IEAA?AV?$_Tree_iterator@V?$_Tree_val@U?$_Tree_simple_types@U?$pair@$$CBIUPORTINFO@@@std@@@std@@@std@@@1@V?$_Tree_const_iterator@V?$_Tree_val@U?$_Tree_simple_types@U?$pair@$$CBIUPORTINFO@@@std@@@std@@@std@@@1@AEAU?$pair@$$CBIUPORTINFO@@@1@PEAU?$_Tree_node@U?$pair@$$CBIUPORTINFO@@@std@@PEAX@1@@Z 000000014005b1a4     GameServerManagerDlg.obj
 0002:000101b8       $ip2state$??$_Insert_hint@AEAU?$pair@$$CBIUPORTINFO@@@std@@PEAU?$_Tree_node@U?$pair@$$CBIUPORTINFO@@@std@@PEAX@2@@?$_Tree@V?$_Tmap_traits@IUPORTINFO@@U?$less@I@std@@V?$allocator@U?$pair@$$CBIUPORTINFO@@@std@@@3@$0A@@std@@@std@@IEAA?AV?$_Tree_iterator@V?$_Tree_val@U?$_Tree_simple_types@U?$pair@$$CBIUPORTINFO@@@std@@@std@@@std@@@1@V?$_Tree_const_iterator@V?$_Tree_val@U?$_Tree_simple_types@U?$pair@$$CBIUPORTINFO@@@std@@@std@@@std@@@1@AEAU?$pair@$$CBIUPORTINFO@@@1@PEAU?$_Tree_node@U?$pair@$$CBIUPORTINFO@@@std@@PEAX@1@@Z 000000014005b1b8     GameServerManagerDlg.obj
 0002:000101d8       $unwind$?catch$0@?0???$_Insert_hint@AEAU?$pair@$$CBIUPORTINFO@@@std@@PEAU?$_Tree_node@U?$pair@$$CBIUPORTINFO@@@std@@PEAX@2@@?$_Tree@V?$_Tmap_traits@IUPORTINFO@@U?$less@I@std@@V?$allocator@U?$pair@$$CBIUPORTINFO@@@std@@@3@$0A@@std@@@std@@IEAA?AV?$_Tree_iterator@V?$_Tree_val@U?$_Tree_simple_types@U?$pair@$$CBIUPORTINFO@@@std@@@std@@@std@@@1@V?$_Tree_const_iterator@V?$_Tree_val@U?$_Tree_simple_types@U?$pair@$$CBIUPORTINFO@@@std@@@std@@@std@@@1@AEAU?$pair@$$CBIUPORTINFO@@@1@PEAU?$_Tree_node@U?$pair@$$CBIUPORTINFO@@@std@@PEAX@1@@Z@4HA 000000014005b1d8     GameServerManagerDlg.obj
 0002:000101e8       $unwind$?RTIDUSNtoString@EXPAND_USN@@YA?AV?$basic_string@DU?$char_traits@D@std@@V?$allocator@D@2@@std@@HFF_J@Z 000000014005b1e8     GameServerManagerDlg.obj
 0002:00010208       $stateUnwindMap$?RTIDUSNtoString@EXPAND_USN@@YA?AV?$basic_string@DU?$char_traits@D@std@@V?$allocator@D@2@@std@@HFF_J@Z 000000014005b208     GameServerManagerDlg.obj
 0002:00010210       $ip2state$?RTIDUSNtoString@EXPAND_USN@@YA?AV?$basic_string@DU?$char_traits@D@std@@V?$allocator@D@2@@std@@HFF_J@Z 000000014005b210     GameServerManagerDlg.obj
 0002:00010228       $unwind$?_Extract@?$_Tree_val@U?$_Tree_simple_types@U?$pair@$$CBV?$basic_string@DU?$char_traits@D@std@@V?$allocator@D@2@@std@@PEAVCIniSection@CIniReader@@@std@@@std@@@std@@QEAAPEAU?$_Tree_node@U?$pair@$$CBV?$basic_string@DU?$char_traits@D@std@@V?$allocator@D@2@@std@@PEAVCIniSection@CIniReader@@@std@@PEAX@2@V?$_Tree_const_iterator@V?$_Tree_val@U?$_Tree_simple_types@U?$pair@$$CBV?$basic_string@DU?$char_traits@D@std@@V?$allocator@D@2@@std@@PEAVCIniSection@CIniReader@@@std@@@std@@@std@@@2@@Z 000000014005b228     iniReader.obj
 0002:00010228       $unwind$?_Extract@?$_Tree_val@U?$_Tree_simple_types@U?$pair@$$CB_JV?$basic_string@DU?$char_traits@D@std@@V?$allocator@D@2@@std@@@std@@@std@@@std@@QEAAPEAU?$_Tree_node@U?$pair@$$CB_JV?$basic_string@DU?$char_traits@D@std@@V?$allocator@D@2@@std@@@std@@PEAX@2@V?$_Tree_const_iterator@V?$_Tree_val@U?$_Tree_simple_types@U?$pair@$$CB_JV?$basic_string@DU?$char_traits@D@std@@V?$allocator@D@2@@std@@@std@@@std@@@std@@@2@@Z 000000014005b228     LoadXlsMsg.obj
 0002:00010228       $unwind$?StringCchCopyA@@YAJPEAD_KPEBD@Z 000000014005b228     GameServerManagerDlg.obj
 0002:00010228       $unwind$?_Extract@?$_Tree_val@U?$_Tree_simple_types@U?$pair@$$CBV?$basic_string@DU?$char_traits@D@std@@V?$allocator@D@2@@std@@V12@@std@@@std@@@std@@QEAAPEAU?$_Tree_node@U?$pair@$$CBV?$basic_string@DU?$char_traits@D@std@@V?$allocator@D@2@@std@@V12@@std@@PEAX@2@V?$_Tree_const_iterator@V?$_Tree_val@U?$_Tree_simple_types@U?$pair@$$CBV?$basic_string@DU?$char_traits@D@std@@V?$allocator@D@2@@std@@V12@@std@@@std@@@std@@@2@@Z 000000014005b228     iniReader.obj
 0002:00010228       $unwind$??4WEAPON_INFO@@QEAAAEAU0@AEBU0@@Z 000000014005b228     GameServerManagerDlg.obj
 0002:00010230       $unwind$?USNtoStr@EXPAND_USN@@YA?AV?$basic_string@DU?$char_traits@D@std@@V?$allocator@D@2@@std@@_J@Z 000000014005b230     GameServerManagerDlg.obj
 0002:00010240       $unwind$?find_last_of@?$basic_string@DU?$char_traits@D@std@@V?$allocator@D@2@@std@@QEBA_KQEBD_K@Z 000000014005b240     GameServerManagerDlg.obj
 0002:00010258       $chain$3$??$_Reallocate_grow_by@V<lambda_65e615be2a453ca0576c979606f46740>@@PEBD_K@?$basic_string@DU?$char_traits@D@std@@V?$allocator@D@2@@std@@QEAAAEAV01@_KV<lambda_65e615be2a453ca0576c979606f46740>@@PEBD_K@Z 000000014005b258     GameServerManagerDlg.obj
 0002:00010278       $chain$4$??$_Reallocate_grow_by@V<lambda_65e615be2a453ca0576c979606f46740>@@PEBD_K@?$basic_string@DU?$char_traits@D@std@@V?$allocator@D@2@@std@@QEAAAEAV01@_KV<lambda_65e615be2a453ca0576c979606f46740>@@PEBD_K@Z 000000014005b278     GameServerManagerDlg.obj
 0002:00010288       $unwind$?append@?$basic_string@DU?$char_traits@D@std@@V?$allocator@D@2@@std@@QEAAAEAV12@QEBD_K@Z 000000014005b288     GameServerManagerDlg.obj
 0002:00010294       $chain$0$?append@?$basic_string@DU?$char_traits@D@std@@V?$allocator@D@2@@std@@QEAAAEAV12@QEBD_K@Z 000000014005b294     GameServerManagerDlg.obj
 0002:000102a8       $chain$1$?append@?$basic_string@DU?$char_traits@D@std@@V?$allocator@D@2@@std@@QEAAAEAV12@QEBD_K@Z 000000014005b2a8     GameServerManagerDlg.obj
 0002:000102b8       $unwind$?init@SGGMProxyLoader@sggm_proxy@@QEAA_NPEAVMultiReceiver@2@@Z 000000014005b2b8     GameServerManagerDlg.obj
 0002:000102d8       $stateUnwindMap$?init@SGGMProxyLoader@sggm_proxy@@QEAA_NPEAVMultiReceiver@2@@Z 000000014005b2d8     GameServerManagerDlg.obj
 0002:000102e0       $ip2state$?init@SGGMProxyLoader@sggm_proxy@@QEAA_NPEAVMultiReceiver@2@@Z 000000014005b2e0     GameServerManagerDlg.obj
 0002:000102f0       $unwind$??0GAMEPROTO_SS_GAMEEND@@QEAA@XZ 000000014005b2f0     GameServerManagerDlg.obj
 0002:00010308       $unwind$??1SGGMProxyLoader@sggm_proxy@@QEAA@XZ 000000014005b308     GameServerManagerDlg.obj
 0002:00010318       $ip2state$??1SGGMProxyLoader@sggm_proxy@@QEAA@XZ 000000014005b318     GameServerManagerDlg.obj
 0002:00010320       $unwind$?Send@CGMSConnManager@@AEAAHPEAVCPacket@@@Z 000000014005b320     GMSConnManager.obj
 0002:00010340       $ip2state$?Send@CGMSConnManager@@AEAAHPEAVCPacket@@@Z 000000014005b340     GMSConnManager.obj
 0002:00010358       $unwind$?SendDiv@CGMSConnManager@@AEAAHEEEPEADK@Z 000000014005b358     GMSConnManager.obj
 0002:00010388       $ip2state$?SendDiv@CGMSConnManager@@AEAAHEEEPEADK@Z 000000014005b388     GMSConnManager.obj
 0002:000103a0       $unwind$?SortFinishedGameUserInfo@CGMSConnManager@@AEAAXAEAUPROTO_FINISHED_GAME_tag@@@Z 000000014005b3a0     GMSConnManager.obj
 0002:000103c4       $unwind$??4PROTO_USER_STAT_tag@@QEAAAEAU0@AEBU0@@Z 000000014005b3c4     GMSConnManager.obj
 0002:000103d0       $unwind$??_ECSFGameServerClientLib@@UEAAPEAXI@Z 000000014005b3d0     GMSConnManager.obj
 0002:000103e8       $ip2state$??_ECSFGameServerClientLib@@UEAAPEAXI@Z 000000014005b3e8     GMSConnManager.obj
 0002:000103f0       $unwind$?StartingReport@CGMSConnManager@@QEAAHFHHHHHHHQEAHHH@Z 000000014005b3f0     GMSConnManager.obj
 0002:0001040c       $unwind$?StartingGameResult@CGMSConnManager@@QEAAHUPROTO_STARTING_GAME_RESULT_tag@@W4START_HOST_RESULT@@@Z 000000014005b40c     GMSConnManager.obj
 0002:0001042c       $stateUnwindMap$?SendTeamDeathMatchKillCnt@CGMSConnManager@@QEAAHPEBUPROTO_GAMEGT_TEAM_DEATH_KILL_CNT_NTY@@@Z 000000014005b42c     GMSConnManager.obj
 0002:0001042c       $stateUnwindMap$?SendAI3BonusClearItemReq@CGMSConnManager@@QEAAHPEAUPROTO_GAMEGT_INGAME_AI3_BONUS_REWARD_ITEM_REQ@@@Z 000000014005b42c     GMSConnManager.obj
 0002:0001042c       $stateUnwindMap$?SendAIExtraMiddleRewardReq@CGMSConnManager@@QEAAHPEAUPROTO_AI_EXTRA_MIDDLE_REWARD_REQ@@@Z 000000014005b42c     GMSConnManager.obj
 0002:0001042c       $stateUnwindMap$?SendKickUserInfo@CGMSConnManager@@QEAAHPEAUPROTO_GAMEMGT_KICK_USER@@@Z 000000014005b42c     GMSConnManager.obj
 0002:0001042c       $stateUnwindMap$?SendAIExtraRewardReq@CGMSConnManager@@QEAAHPEAUPROTO_AI_EXTRA_REWARD_REQ@@@Z 000000014005b42c     GMSConnManager.obj
 0002:0001042c       $stateUnwindMap$?SendIntrusionCoinDec@CGMSConnManager@@QEAAHPEAUPROTO_GAMEGT_MAPLOADING_COMPLETE_NTY_tag@@@Z 000000014005b42c     GMSConnManager.obj
 0002:0001042c       $stateUnwindMap$?InsertCharacterResult@CGMSConnManager@@QEAAHUPROTO_INSERT_CHARACTER_RESULT_tag@@@Z 000000014005b42c     GMSConnManager.obj
 0002:0001042c       $stateUnwindMap$?UpdateCharacterStat@CGMSConnManager@@QEAAHUPROTO_UPDATE_CHARACTER_STAT_tag@@@Z 000000014005b42c     GMSConnManager.obj
 0002:0001042c       $stateUnwindMap$?SendPrevGameFinishNotify@CGMSConnManager@@QEAAHPEAUPROTO_FINISHED_GAME_PREV_tag@@@Z 000000014005b42c     GMSConnManager.obj
 0002:0001042c       $stateUnwindMap$?SendRoundChange@CGMSConnManager@@QEAAHPEBUPROTO_GAMEGT_ROUND_CHANGE_NTY_tag@@@Z 000000014005b42c     GMSConnManager.obj
 0002:0001042c       $stateUnwindMap$?SendBattleShipBonusCoinReq@CGMSConnManager@@QEAAHPEAUPROTOCOL_AI2_BONUSROUND_REWARD_REQ_tag@@@Z 000000014005b42c     GMSConnManager.obj
 0002:0001042c       $stateUnwindMap$?SendAutoMatchIngameEnterNty@CGMSConnManager@@QEAAHAEBUPROTO_AUTOMATCH_INGAME_ENTER_NTY@@@Z 000000014005b42c     GMSConnManager.obj
 0002:0001042c       $stateUnwindMap$?SendAutoMatchGameEnterRes@CGMSConnManager@@QEAAHAEBUPROTO_AUTOMATCH_GAME_ENTER_RES@@@Z 000000014005b42c     GMSConnManager.obj
 0002:0001042c       $stateUnwindMap$?SendAutoMatchGameStartRes@CGMSConnManager@@QEAAHAEBUPROTO_AUTOMATCH_GAME_START_RES@@W4START_HOST_RESULT@@@Z 000000014005b42c     GMSConnManager.obj
 0002:0001042c       $stateUnwindMap$?SendSpectatorRecommendRoomData@CGMSConnManager@@QEAAHPEAUPROTO_SPECTATOR_RECOMMEND_ROOM_INGAME_DATA_NTY@@@Z 000000014005b42c     GMSConnManager.obj
 0002:0001042c       $stateUnwindMap$?StartingGameResult@CGMSConnManager@@QEAAHUPROTO_STARTING_GAME_RESULT_tag@@W4START_HOST_RESULT@@@Z 000000014005b42c     GMSConnManager.obj
 0002:0001042c       $stateUnwindMap$?SendFarmingItemReq@CGMSConnManager@@QEAAHPEAUPROTO_GAMEGT_INGAME_FARMING_ITEM_REQ@@@Z 000000014005b42c     GMSConnManager.obj
 0002:0001042c       $stateUnwindMap$?SendSpyChange@CGMSConnManager@@QEAAHPEAUPROTO_GAMEGT_SPY_CHANGE_NTY_tag@@@Z 000000014005b42c     GMSConnManager.obj
 0002:0001042c       $stateUnwindMap$?SendForceLeavePollResult@CGMSConnManager@@QEAAHPEBUPROTO_BAN_USER_tag@@@Z 000000014005b42c     GMSConnManager.obj
 0002:0001042c       $stateUnwindMap$?SendBossTowerRewardReq@CGMSConnManager@@QEAAHPEAUPROTO_AI_BOSS_TOWER_REWARD_REQ@@@Z 000000014005b42c     GMSConnManager.obj
 0002:0001042c       $stateUnwindMap$?SendIngameRewardReq@CGMSConnManager@@QEAAHPEAUPROTO_INGAME_RESULT_REQ@@@Z 000000014005b42c     GMSConnManager.obj
 0002:0001042c       $stateUnwindMap$?SendAutoSideChangeTeamInfoNotify@CGMSConnManager@@QEAAHPEAUPROTO_GAMEGT_AUTO_SIDE_CHANGE_TEAM_INFO_NTY@@@Z 000000014005b42c     GMSConnManager.obj
 0002:0001042c       $stateUnwindMap$?SendAIItemInsert@CGMSConnManager@@QEAAHPEAUPROTO_GAMEGT_INGAME_AIGACHA_ITEM_INSERT@@@Z 000000014005b42c     GMSConnManager.obj
 0002:0001042c       $stateUnwindMap$?SendGameStart@CGMSConnManager@@QEAAHPEBUPROTO_GAMEGT_GAME_START_NTY@@@Z 000000014005b42c     GMSConnManager.obj
 0002:00010438       $ip2state$?StartingGameResult@CGMSConnManager@@QEAAHUPROTO_STARTING_GAME_RESULT_tag@@W4START_HOST_RESULT@@@Z 000000014005b438     GMSConnManager.obj
 0002:00010450       $unwind$?FinishedGame@CGMSConnManager@@QEAAHUPROTO_FINISHED_GAME_tag@@@Z 000000014005b450     GMSConnManager.obj
 0002:0001045c       $unwind$?UpdateCharacterStat@CGMSConnManager@@QEAAHUPROTO_UPDATE_CHARACTER_STAT_tag@@@Z 000000014005b45c     GMSConnManager.obj
 0002:00010478       $ip2state$?UpdateCharacterStat@CGMSConnManager@@QEAAHUPROTO_UPDATE_CHARACTER_STAT_tag@@@Z 000000014005b478     GMSConnManager.obj
 0002:00010490       $unwind$?InsertCharacterResult@CGMSConnManager@@QEAAHUPROTO_INSERT_CHARACTER_RESULT_tag@@@Z 000000014005b490     GMSConnManager.obj
 0002:000104b0       $ip2state$?InsertCharacterResult@CGMSConnManager@@QEAAHUPROTO_INSERT_CHARACTER_RESULT_tag@@@Z 000000014005b4b0     GMSConnManager.obj
 0002:000104c8       $unwind$?SendHeartBeat@CGMSConnManager@@QEAAHH@Z 000000014005b4c8     GMSConnManager.obj
 0002:000104e4       $unwind$?SendForceLeavePollResult@CGMSConnManager@@QEAAHPEBUPROTO_BAN_USER_tag@@@Z 000000014005b4e4     GMSConnManager.obj
 0002:00010500       $ip2state$?SendForceLeavePollResult@CGMSConnManager@@QEAAHPEBUPROTO_BAN_USER_tag@@@Z 000000014005b500     GMSConnManager.obj
 0002:00010518       $unwind$?NotifyAllocableRoomCountChanged@CGMSConnManager@@QEAAHJHHHHHQEAHHH@Z 000000014005b518     GMSConnManager.obj
 0002:00010538       $stateUnwindMap$?NotifyAllocableRoomCountChanged@CGMSConnManager@@QEAAHJHHHHHQEAHHH@Z 000000014005b538     GMSConnManager.obj
 0002:00010540       $ip2state$?NotifyAllocableRoomCountChanged@CGMSConnManager@@QEAAHJHHHHHQEAHHH@Z 000000014005b540     GMSConnManager.obj
 0002:00010558       $unwind$?SendRoundChange@CGMSConnManager@@QEAAHPEBUPROTO_GAMEGT_ROUND_CHANGE_NTY_tag@@@Z 000000014005b558     GMSConnManager.obj
 0002:00010578       $ip2state$?SendRoundChange@CGMSConnManager@@QEAAHPEBUPROTO_GAMEGT_ROUND_CHANGE_NTY_tag@@@Z 000000014005b578     GMSConnManager.obj
 0002:00010590       $unwind$?SendGameStart@CGMSConnManager@@QEAAHPEBUPROTO_GAMEGT_GAME_START_NTY@@@Z 000000014005b590     GMSConnManager.obj
 0002:000105b0       $ip2state$?SendGameStart@CGMSConnManager@@QEAAHPEBUPROTO_GAMEGT_GAME_START_NTY@@@Z 000000014005b5b0     GMSConnManager.obj
 0002:000105c8       $unwind$?SendTeamDeathMatchKillCnt@CGMSConnManager@@QEAAHPEBUPROTO_GAMEGT_TEAM_DEATH_KILL_CNT_NTY@@@Z 000000014005b5c8     GMSConnManager.obj
 0002:000105e8       $ip2state$?SendTeamDeathMatchKillCnt@CGMSConnManager@@QEAAHPEBUPROTO_GAMEGT_TEAM_DEATH_KILL_CNT_NTY@@@Z 000000014005b5e8     GMSConnManager.obj
 0002:00010600       $unwind$?SendAIItemInsert@CGMSConnManager@@QEAAHPEAUPROTO_GAMEGT_INGAME_AIGACHA_ITEM_INSERT@@@Z 000000014005b600     GMSConnManager.obj
 0002:00010620       $ip2state$?SendAIItemInsert@CGMSConnManager@@QEAAHPEAUPROTO_GAMEGT_INGAME_AIGACHA_ITEM_INSERT@@@Z 000000014005b620     GMSConnManager.obj
 0002:00010638       $unwind$?SendIntrusionCoinDec@CGMSConnManager@@QEAAHPEAUPROTO_GAMEGT_MAPLOADING_COMPLETE_NTY_tag@@@Z 000000014005b638     GMSConnManager.obj
 0002:00010658       $ip2state$?SendIntrusionCoinDec@CGMSConnManager@@QEAAHPEAUPROTO_GAMEGT_MAPLOADING_COMPLETE_NTY_tag@@@Z 000000014005b658     GMSConnManager.obj
 0002:00010670       $unwind$?SendSpyChange@CGMSConnManager@@QEAAHPEAUPROTO_GAMEGT_SPY_CHANGE_NTY_tag@@@Z 000000014005b670     GMSConnManager.obj
 0002:00010690       $ip2state$?SendSpyChange@CGMSConnManager@@QEAAHPEAUPROTO_GAMEGT_SPY_CHANGE_NTY_tag@@@Z 000000014005b690     GMSConnManager.obj
 0002:000106a8       $unwind$?SendFarmingItemReq@CGMSConnManager@@QEAAHPEAUPROTO_GAMEGT_INGAME_FARMING_ITEM_REQ@@@Z 000000014005b6a8     GMSConnManager.obj
 0002:000106c8       $ip2state$?SendFarmingItemReq@CGMSConnManager@@QEAAHPEAUPROTO_GAMEGT_INGAME_FARMING_ITEM_REQ@@@Z 000000014005b6c8     GMSConnManager.obj
 0002:000106e0       $unwind$?SendBattleShipBonusCoinReq@CGMSConnManager@@QEAAHPEAUPROTOCOL_AI2_BONUSROUND_REWARD_REQ_tag@@@Z 000000014005b6e0     GMSConnManager.obj
 0002:00010700       $ip2state$?SendBattleShipBonusCoinReq@CGMSConnManager@@QEAAHPEAUPROTOCOL_AI2_BONUSROUND_REWARD_REQ_tag@@@Z 000000014005b700     GMSConnManager.obj
 0002:00010718       $unwind$?SendAI3BonusClearItemReq@CGMSConnManager@@QEAAHPEAUPROTO_GAMEGT_INGAME_AI3_BONUS_REWARD_ITEM_REQ@@@Z 000000014005b718     GMSConnManager.obj
 0002:00010738       $ip2state$?SendAI3BonusClearItemReq@CGMSConnManager@@QEAAHPEAUPROTO_GAMEGT_INGAME_AI3_BONUS_REWARD_ITEM_REQ@@@Z 000000014005b738     GMSConnManager.obj
 0002:00010750       $unwind$?SendAIExtraRewardReq@CGMSConnManager@@QEAAHPEAUPROTO_AI_EXTRA_REWARD_REQ@@@Z 000000014005b750     GMSConnManager.obj
 0002:00010770       $ip2state$?SendAIExtraRewardReq@CGMSConnManager@@QEAAHPEAUPROTO_AI_EXTRA_REWARD_REQ@@@Z 000000014005b770     GMSConnManager.obj
 0002:00010788       $unwind$?SendBossTowerRewardReq@CGMSConnManager@@QEAAHPEAUPROTO_AI_BOSS_TOWER_REWARD_REQ@@@Z 000000014005b788     GMSConnManager.obj
 0002:000107a8       $ip2state$?SendBossTowerRewardReq@CGMSConnManager@@QEAAHPEAUPROTO_AI_BOSS_TOWER_REWARD_REQ@@@Z 000000014005b7a8     GMSConnManager.obj
 0002:000107c0       $unwind$?SendIngameRewardReq@CGMSConnManager@@QEAAHPEAUPROTO_INGAME_RESULT_REQ@@@Z 000000014005b7c0     GMSConnManager.obj
 0002:000107e0       $ip2state$?SendIngameRewardReq@CGMSConnManager@@QEAAHPEAUPROTO_INGAME_RESULT_REQ@@@Z 000000014005b7e0     GMSConnManager.obj
 0002:000107f8       $unwind$?SendKickUserInfo@CGMSConnManager@@QEAAHPEAUPROTO_GAMEMGT_KICK_USER@@@Z 000000014005b7f8     GMSConnManager.obj
 0002:00010818       $ip2state$?SendKickUserInfo@CGMSConnManager@@QEAAHPEAUPROTO_GAMEMGT_KICK_USER@@@Z 000000014005b818     GMSConnManager.obj
 0002:00010830       $unwind$?SendSpectatorRecommendRoomData@CGMSConnManager@@QEAAHPEAUPROTO_SPECTATOR_RECOMMEND_ROOM_INGAME_DATA_NTY@@@Z 000000014005b830     GMSConnManager.obj
 0002:00010850       $ip2state$?SendSpectatorRecommendRoomData@CGMSConnManager@@QEAAHPEAUPROTO_SPECTATOR_RECOMMEND_ROOM_INGAME_DATA_NTY@@@Z 000000014005b850     GMSConnManager.obj
 0002:00010868       $unwind$?SendPrevGameFinishNotify@CGMSConnManager@@QEAAHPEAUPROTO_FINISHED_GAME_PREV_tag@@@Z 000000014005b868     GMSConnManager.obj
 0002:00010888       $ip2state$?SendPrevGameFinishNotify@CGMSConnManager@@QEAAHPEAUPROTO_FINISHED_GAME_PREV_tag@@@Z 000000014005b888     GMSConnManager.obj
 0002:000108a0       $unwind$?SendAutoSideChangeTeamInfoNotify@CGMSConnManager@@QEAAHPEAUPROTO_GAMEGT_AUTO_SIDE_CHANGE_TEAM_INFO_NTY@@@Z 000000014005b8a0     GMSConnManager.obj
 0002:000108c0       $ip2state$?SendAutoSideChangeTeamInfoNotify@CGMSConnManager@@QEAAHPEAUPROTO_GAMEGT_AUTO_SIDE_CHANGE_TEAM_INFO_NTY@@@Z 000000014005b8c0     GMSConnManager.obj
 0002:000108d8       $unwind$?SendAIExtraMiddleRewardReq@CGMSConnManager@@QEAAHPEAUPROTO_AI_EXTRA_MIDDLE_REWARD_REQ@@@Z 000000014005b8d8     GMSConnManager.obj
 0002:000108f8       $ip2state$?SendAIExtraMiddleRewardReq@CGMSConnManager@@QEAAHPEAUPROTO_AI_EXTRA_MIDDLE_REWARD_REQ@@@Z 000000014005b8f8     GMSConnManager.obj
 0002:00010910       $unwind$?SendAutoMatchGameStartRes@CGMSConnManager@@QEAAHAEBUPROTO_AUTOMATCH_GAME_START_RES@@W4START_HOST_RESULT@@@Z 000000014005b910     GMSConnManager.obj
 0002:00010930       $ip2state$?SendAutoMatchGameStartRes@CGMSConnManager@@QEAAHAEBUPROTO_AUTOMATCH_GAME_START_RES@@W4START_HOST_RESULT@@@Z 000000014005b930     GMSConnManager.obj
 0002:00010948       $unwind$?SendAutoMatchGameEnterRes@CGMSConnManager@@QEAAHAEBUPROTO_AUTOMATCH_GAME_ENTER_RES@@@Z 000000014005b948     GMSConnManager.obj
 0002:00010968       $ip2state$?SendAutoMatchGameEnterRes@CGMSConnManager@@QEAAHAEBUPROTO_AUTOMATCH_GAME_ENTER_RES@@@Z 000000014005b968     GMSConnManager.obj
 0002:00010980       $unwind$?SendAutoMatchIngameEnterNty@CGMSConnManager@@QEAAHAEBUPROTO_AUTOMATCH_INGAME_ENTER_NTY@@@Z 000000014005b980     GMSConnManager.obj
 0002:000109a0       $ip2state$?SendAutoMatchIngameEnterNty@CGMSConnManager@@QEAAHAEBUPROTO_AUTOMATCH_INGAME_ENTER_NTY@@@Z 000000014005b9a0     GMSConnManager.obj
 0002:000109b8       $unwind$??$_Reallocate_grow_by@V<lambda_319d5e083f45f90dcdce5dce53cbb275>@@D@?$basic_string@DU?$char_traits@D@std@@V?$allocator@D@2@@std@@QEAAAEAV01@_KV<lambda_319d5e083f45f90dcdce5dce53cbb275>@@D@Z 000000014005b9b8     base64.obj
 0002:000109c8       $chain$2$??$_Reallocate_grow_by@V<lambda_319d5e083f45f90dcdce5dce53cbb275>@@D@?$basic_string@DU?$char_traits@D@std@@V?$allocator@D@2@@std@@QEAAAEAV01@_KV<lambda_319d5e083f45f90dcdce5dce53cbb275>@@D@Z 000000014005b9c8     base64.obj
 0002:000109e4       $chain$3$??$_Reallocate_grow_by@V<lambda_319d5e083f45f90dcdce5dce53cbb275>@@D@?$basic_string@DU?$char_traits@D@std@@V?$allocator@D@2@@std@@QEAAAEAV01@_KV<lambda_319d5e083f45f90dcdce5dce53cbb275>@@D@Z 000000014005b9e4     base64.obj
 0002:000109f4       $unwind$??$?HDU?$char_traits@D@std@@V?$allocator@D@1@@std@@YA?AV?$basic_string@DU?$char_traits@D@std@@V?$allocator@D@2@@0@QEBDAEBV10@@Z 000000014005b9f4     CSmtp.obj
 0002:00010a10       $stateUnwindMap$??$?HDU?$char_traits@D@std@@V?$allocator@D@1@@std@@YA?AV?$basic_string@DU?$char_traits@D@std@@V?$allocator@D@2@@0@QEBDAEBV10@@Z 000000014005ba10     CSmtp.obj
 0002:00010a18       $ip2state$??$?HDU?$char_traits@D@std@@V?$allocator@D@1@@std@@YA?AV?$basic_string@DU?$char_traits@D@std@@V?$allocator@D@2@@0@QEBDAEBV10@@Z 000000014005ba18     CSmtp.obj
 0002:00010a20       $unwind$??$_Destroy_range@V?$allocator@V?$basic_string@DU?$char_traits@D@std@@V?$allocator@D@2@@std@@@std@@@std@@YAXPEAV?$basic_string@DU?$char_traits@D@std@@V?$allocator@D@2@@0@0AEAV?$allocator@V?$basic_string@DU?$char_traits@D@std@@V?$allocator@D@2@@std@@@0@@Z 000000014005ba20     CSmtp.obj
 0002:00010a2c       $chain$0$??$_Destroy_range@V?$allocator@V?$basic_string@DU?$char_traits@D@std@@V?$allocator@D@2@@std@@@std@@@std@@YAXPEAV?$basic_string@DU?$char_traits@D@std@@V?$allocator@D@2@@0@0AEAV?$allocator@V?$basic_string@DU?$char_traits@D@std@@V?$allocator@D@2@@std@@@0@@Z 000000014005ba2c     CSmtp.obj
 0002:00010a40       $chain$1$??$_Destroy_range@V?$allocator@V?$basic_string@DU?$char_traits@D@std@@V?$allocator@D@2@@std@@@std@@@std@@YAXPEAV?$basic_string@DU?$char_traits@D@std@@V?$allocator@D@2@@0@0AEAV?$allocator@V?$basic_string@DU?$char_traits@D@std@@V?$allocator@D@2@@std@@@0@@Z 000000014005ba40     CSmtp.obj
 0002:00010a50       $chain$2$??$_Destroy_range@V?$allocator@V?$basic_string@DU?$char_traits@D@std@@V?$allocator@D@2@@std@@@std@@@std@@YAXPEAV?$basic_string@DU?$char_traits@D@std@@V?$allocator@D@2@@0@0AEAV?$allocator@V?$basic_string@DU?$char_traits@D@std@@V?$allocator@D@2@@std@@@0@@Z 000000014005ba50     CSmtp.obj
 0002:00010a64       $unwind$??0?$basic_string@DU?$char_traits@D@std@@V?$allocator@D@2@@std@@QEAA@AEBV01@@Z 000000014005ba64     CSmtp.obj
 0002:00010a78       $unwind$??1sentry@?$basic_ostream@DU?$char_traits@D@std@@@std@@QEAA@XZ 000000014005ba78     md5_csmtp.obj
 0002:00010a88       $ip2state$??1sentry@?$basic_ostream@DU?$char_traits@D@std@@@std@@QEAA@XZ 000000014005ba88     md5_csmtp.obj
 0002:00010a98       $unwind$??1_Sentry_base@?$basic_ostream@DU?$char_traits@D@std@@@std@@QEAA@XZ 000000014005ba98     md5_csmtp.obj
 0002:00010aa8       $ip2state$??1_Sentry_base@?$basic_ostream@DU?$char_traits@D@std@@@std@@QEAA@XZ 000000014005baa8     md5_csmtp.obj
 0002:00010ab0       $unwind$??$?6U?$char_traits@D@std@@@std@@YAAEAV?$basic_ostream@DU?$char_traits@D@std@@@0@AEAV10@PEBD@Z 000000014005bab0     md5_csmtp.obj
 0002:00010acc       $stateUnwindMap$??$?6U?$char_traits@D@std@@@std@@YAAEAV?$basic_ostream@DU?$char_traits@D@std@@@0@AEAV10@PEBD@Z 000000014005bacc     md5_csmtp.obj
 0002:00010afc       $tryMap$??$?6U?$char_traits@D@std@@@std@@YAAEAV?$basic_ostream@DU?$char_traits@D@std@@@0@AEAV10@PEBD@Z 000000014005bafc     md5_csmtp.obj
 0002:00010b10       $handlerMap$0$??$?6U?$char_traits@D@std@@@std@@YAAEAV?$basic_ostream@DU?$char_traits@D@std@@@0@AEAV10@PEBD@Z 000000014005bb10     md5_csmtp.obj
 0002:00010b30       $ip2state$??$?6U?$char_traits@D@std@@@std@@YAAEAV?$basic_ostream@DU?$char_traits@D@std@@@0@AEAV10@PEBD@Z 000000014005bb30     md5_csmtp.obj
 0002:00010b70       $unwind$?catch$4@?0???$?6U?$char_traits@D@std@@@std@@YAAEAV?$basic_ostream@DU?$char_traits@D@std@@@0@AEAV10@PEBD@Z@4HA 000000014005bb70     md5_csmtp.obj
 0002:00010b80       $unwind$?a2toi@@YAHPEADHH@Z 000000014005bb80     DateTime.obj
 0002:00010b90       $chain$0$?a2toi@@YAHPEADHH@Z 000000014005bb90     DateTime.obj
 0002:00010ba4       $chain$1$?a2toi@@YAHPEADHH@Z 000000014005bba4     DateTime.obj
 0002:00010bb4       $chain$2$?a2toi@@YAHPEADHH@Z 000000014005bbb4     DateTime.obj
 0002:00010bc8       $unwind$?GetCurrentLocalTime@datetime@@QEAAXXZ 000000014005bbc8     DateTime.obj
 0002:00010bd8       $unwind$??__Eg_HostStat@@YAXXZ 000000014005bbd8     HostStat.obj
 0002:00010be8       $stateUnwindMap$??__Eg_HostStat@@YAXXZ 000000014005bbe8     HostStat.obj
 0002:00010bf8       $ip2state$??__Eg_HostStat@@YAXXZ 000000014005bbf8     HostStat.obj
 0002:00010c10       $unwind$??1CHostStat@@UEAA@XZ 000000014005bc10     HostStat.obj
 0002:00010c28       $ip2state$??1CHostStat@@UEAA@XZ 000000014005bc28     HostStat.obj
 0002:00010c30       $unwind$?setup@CHostStat@@QEAAXHH@Z 000000014005bc30     HostStat.obj
 0002:00010c54       $stateUnwindMap$?setup@CHostStat@@QEAAXHH@Z 000000014005bc54     HostStat.obj
 0002:00010c68       $ip2state$?setup@CHostStat@@QEAAXHH@Z 000000014005bc68     HostStat.obj
 0002:00010c90       $unwind$?thdMail@CHostStat@@KAIPEAX@Z 000000014005bc90     HostStat.obj
 0002:00010cc0       $stateUnwindMap$?thdMail@CHostStat@@KAIPEAX@Z 000000014005bcc0     HostStat.obj
 0002:00010d10       $ip2state$?thdMail@CHostStat@@KAIPEAX@Z 000000014005bd10     HostStat.obj
 0002:00010da8       $unwind$?timer@CHostStat@@QEAAXXZ 000000014005bda8     HostStat.obj
 0002:00010dd0       $stateUnwindMap$?timer@CHostStat@@QEAAXXZ 000000014005bdd0     HostStat.obj
 0002:00010df0       $ip2state$?timer@CHostStat@@QEAAXXZ 000000014005bdf0     HostStat.obj
 0002:00010e38       $unwind$?getData64@CHostStat@@QEAA_JGEEG@Z 000000014005be38     HostStat.obj
 0002:00010e5c       $stateUnwindMap$?getData64@CHostStat@@QEAA_JGEEG@Z 000000014005be5c     HostStat.obj
 0002:00010e5c       $stateUnwindMap$?setData64@CHostStat@@QEAAXGEEG_J@Z 000000014005be5c     HostStat.obj
 0002:00010e5c       $stateUnwindMap$?addData@CHostStat@@QEAAXGEEG@Z 000000014005be5c     HostStat.obj
 0002:00010e5c       $stateUnwindMap$?addExtraData@CHostStat@@QEAAXGEEGIII@Z 000000014005be5c     HostStat.obj
 0002:00010e68       $ip2state$?getData64@CHostStat@@QEAA_JGEEG@Z 000000014005be68     HostStat.obj
 0002:00010e80       $unwind$?setData64@CHostStat@@QEAAXGEEG_J@Z 000000014005be80     HostStat.obj
 0002:00010ea8       $ip2state$?setData64@CHostStat@@QEAAXGEEG_J@Z 000000014005bea8     HostStat.obj
 0002:00010ec0       $unwind$?addData@CHostStat@@QEAAXGEEG@Z 000000014005bec0     HostStat.obj
 0002:00010ee8       $ip2state$?addData@CHostStat@@QEAAXGEEG@Z 000000014005bee8     HostStat.obj
 0002:00010f00       $unwind$?addExtraData@CHostStat@@QEAAXGE@Z 000000014005bf00     HostStat.obj
 0002:00010f28       $stateUnwindMap$?addExtraData@CHostStat@@QEAAXGE@Z 000000014005bf28     HostStat.obj
 0002:00010f38       $ip2state$?addExtraData@CHostStat@@QEAAXGE@Z 000000014005bf38     HostStat.obj
 0002:00010f60       $unwind$?addExtraData@CHostStat@@QEAAXGEEGIII@Z 000000014005bf60     HostStat.obj
 0002:00010f88       $ip2state$?addExtraData@CHostStat@@QEAAXGEEGIII@Z 000000014005bf88     HostStat.obj
 0002:00010fa0       $unwind$?send@CHostStat@@IEAA_NPEAD0@Z 000000014005bfa0     HostStat.obj
 0002:00010fc8       $stateUnwindMap$?send@CHostStat@@IEAA_NPEAD0@Z 000000014005bfc8     HostStat.obj
 0002:00011020       $ip2state$?send@CHostStat@@IEAA_NPEAD0@Z 000000014005c020     HostStat.obj
 0002:000110c8       $unwind$?timerPerfMem@CHostStat@@QEAAXXZ 000000014005c0c8     HostStat.obj
 0002:000110dc       $chain$3$?timerPerfMem@CHostStat@@QEAAXXZ 000000014005c0dc     HostStat.obj
 0002:000110fc       $chain$6$?timerPerfMem@CHostStat@@QEAAXXZ 000000014005c0fc     HostStat.obj
 0002:00011118       $chain$7$?timerPerfMem@CHostStat@@QEAAXXZ 000000014005c118     HostStat.obj
 0002:00011130       $chain$8$?timerPerfMem@CHostStat@@QEAAXXZ 000000014005c130     HostStat.obj
 0002:00011144       $chain$9$?timerPerfMem@CHostStat@@QEAAXXZ 000000014005c144     HostStat.obj
 0002:00011154       $chain$10$?timerPerfMem@CHostStat@@QEAAXXZ 000000014005c154     HostStat.obj
 0002:00011164       $unwind$?timerLogUser@CHostStat@@QEAAXHHHHH@Z 000000014005c164     HostStat.obj
 0002:0001117c       $chain$3$?timerLogUser@CHostStat@@QEAAXHHHHH@Z 000000014005c17c     HostStat.obj
 0002:0001119c       $chain$4$?timerLogUser@CHostStat@@QEAAXHHHHH@Z 000000014005c19c     HostStat.obj
 0002:000111ac       $unwind$?AddLog@CHostStat@@QEAAXPEBDZZ 000000014005c1ac     HostStat.obj
 0002:000111c4       $chain$4$?AddLog@CHostStat@@QEAAXPEBDZZ 000000014005c1c4     HostStat.obj
 0002:000111e8       $chain$5$?AddLog@CHostStat@@QEAAXPEBDZZ 000000014005c1e8     HostStat.obj
 0002:000111f8       $unwind$?GatherFiles@CHostStat@@QEAAXPEAD@Z 000000014005c1f8     HostStat.obj
 0002:0001121c       $stateUnwindMap$?GatherFiles@CHostStat@@QEAAXPEAD@Z 000000014005c21c     HostStat.obj
 0002:00011228       $ip2state$?GatherFiles@CHostStat@@QEAAXPEAD@Z 000000014005c228     HostStat.obj
 0002:00011248       $unwind$?GetDataFolder@CHostStat@@QEAAXPEAD_K@Z 000000014005c248     HostStat.obj
 0002:00011260       $unwind$?AddUserPCSpec@CHostStat@@QEAAXGPEBD00I@Z 000000014005c260     HostStat.obj
 0002:00011274       $chain$5$?AddUserPCSpec@CHostStat@@QEAAXGPEBD00I@Z 000000014005c274     HostStat.obj
 0002:0001129c       $chain$6$?AddUserPCSpec@CHostStat@@QEAAXGPEBD00I@Z 000000014005c29c     HostStat.obj
 0002:000112ac       $unwind$??$_Insert_nohint@AEAU?$pair@$$CBGUExtraStatsMemVerify@CHostStat@@@std@@PEAU?$_Tree_node@U?$pair@$$CBGUExtraStatsMemVerify@CHostStat@@@std@@PEAX@2@@?$_Tree@V?$_Tmap_traits@GUExtraStatsMemVerify@CHostStat@@U?$less@G@std@@V?$allocator@U?$pair@$$CBGUExtraStatsMemVerify@CHostStat@@@std@@@4@$0A@@std@@@std@@IEAA?AU?$pair@V?$_Tree_iterator@V?$_Tree_val@U?$_Tree_simple_types@U?$pair@$$CBGUExtraStatsMemVerify@CHostStat@@@std@@@std@@@std@@@std@@_N@1@_NAEAU?$pair@$$CBGUExtraStatsMemVerify@CHostStat@@@1@PEAU?$_Tree_node@U?$pair@$$CBGUExtraStatsMemVerify@CHostStat@@@std@@PEAX@1@@Z 000000014005c2ac     HostStat.obj
 0002:000112ac       $unwind$??$_Insert_nohint@AEAU?$pair@$$CBGUExtraStatsFPSVerify@CHostStat@@@std@@PEAU?$_Tree_node@U?$pair@$$CBGUExtraStatsFPSVerify@CHostStat@@@std@@PEAX@2@@?$_Tree@V?$_Tmap_traits@GUExtraStatsFPSVerify@CHostStat@@U?$less@G@std@@V?$allocator@U?$pair@$$CBGUExtraStatsFPSVerify@CHostStat@@@std@@@4@$0A@@std@@@std@@IEAA?AU?$pair@V?$_Tree_iterator@V?$_Tree_val@U?$_Tree_simple_types@U?$pair@$$CBGUExtraStatsFPSVerify@CHostStat@@@std@@@std@@@std@@@std@@_N@1@_NAEAU?$pair@$$CBGUExtraStatsFPSVerify@CHostStat@@@1@PEAU?$_Tree_node@U?$pair@$$CBGUExtraStatsFPSVerify@CHostStat@@@std@@PEAX@1@@Z 000000014005c2ac     HostStat.obj
 0002:000112c8       $tryMap$??$_Insert_nohint@AEAU?$pair@$$CBGUExtraStatsMemVerify@CHostStat@@@std@@PEAU?$_Tree_node@U?$pair@$$CBGUExtraStatsMemVerify@CHostStat@@@std@@PEAX@2@@?$_Tree@V?$_Tmap_traits@GUExtraStatsMemVerify@CHostStat@@U?$less@G@std@@V?$allocator@U?$pair@$$CBGUExtraStatsMemVerify@CHostStat@@@std@@@4@$0A@@std@@@std@@IEAA?AU?$pair@V?$_Tree_iterator@V?$_Tree_val@U?$_Tree_simple_types@U?$pair@$$CBGUExtraStatsMemVerify@CHostStat@@@std@@@std@@@std@@@std@@_N@1@_NAEAU?$pair@$$CBGUExtraStatsMemVerify@CHostStat@@@1@PEAU?$_Tree_node@U?$pair@$$CBGUExtraStatsMemVerify@CHostStat@@@std@@PEAX@1@@Z 000000014005c2c8     HostStat.obj
 0002:000112c8       $tryMap$??$_Insert_nohint@AEAU?$pair@$$CBGUExtraStatsFPSVerify@CHostStat@@@std@@PEAU?$_Tree_node@U?$pair@$$CBGUExtraStatsFPSVerify@CHostStat@@@std@@PEAX@2@@?$_Tree@V?$_Tmap_traits@GUExtraStatsFPSVerify@CHostStat@@U?$less@G@std@@V?$allocator@U?$pair@$$CBGUExtraStatsFPSVerify@CHostStat@@@std@@@4@$0A@@std@@@std@@IEAA?AU?$pair@V?$_Tree_iterator@V?$_Tree_val@U?$_Tree_simple_types@U?$pair@$$CBGUExtraStatsFPSVerify@CHostStat@@@std@@@std@@@std@@@std@@_N@1@_NAEAU?$pair@$$CBGUExtraStatsFPSVerify@CHostStat@@@1@PEAU?$_Tree_node@U?$pair@$$CBGUExtraStatsFPSVerify@CHostStat@@@std@@PEAX@1@@Z 000000014005c2c8     HostStat.obj
 0002:000112dc       $handlerMap$0$??$_Insert_nohint@AEAU?$pair@$$CBGUExtraStatsFPSVerify@CHostStat@@@std@@PEAU?$_Tree_node@U?$pair@$$CBGUExtraStatsFPSVerify@CHostStat@@@std@@PEAX@2@@?$_Tree@V?$_Tmap_traits@GUExtraStatsFPSVerify@CHostStat@@U?$less@G@std@@V?$allocator@U?$pair@$$CBGUExtraStatsFPSVerify@CHostStat@@@std@@@4@$0A@@std@@@std@@IEAA?AU?$pair@V?$_Tree_iterator@V?$_Tree_val@U?$_Tree_simple_types@U?$pair@$$CBGUExtraStatsFPSVerify@CHostStat@@@std@@@std@@@std@@@std@@_N@1@_NAEAU?$pair@$$CBGUExtraStatsFPSVerify@CHostStat@@@1@PEAU?$_Tree_node@U?$pair@$$CBGUExtraStatsFPSVerify@CHostStat@@@std@@PEAX@1@@Z 000000014005c2dc     HostStat.obj
 0002:000112dc       $handlerMap$0$??$_Insert_nohint@AEAU?$pair@$$CBGUExtraStatsMemVerify@CHostStat@@@std@@PEAU?$_Tree_node@U?$pair@$$CBGUExtraStatsMemVerify@CHostStat@@@std@@PEAX@2@@?$_Tree@V?$_Tmap_traits@GUExtraStatsMemVerify@CHostStat@@U?$less@G@std@@V?$allocator@U?$pair@$$CBGUExtraStatsMemVerify@CHostStat@@@std@@@4@$0A@@std@@@std@@IEAA?AU?$pair@V?$_Tree_iterator@V?$_Tree_val@U?$_Tree_simple_types@U?$pair@$$CBGUExtraStatsMemVerify@CHostStat@@@std@@@std@@@std@@@std@@_N@1@_NAEAU?$pair@$$CBGUExtraStatsMemVerify@CHostStat@@@1@PEAU?$_Tree_node@U?$pair@$$CBGUExtraStatsMemVerify@CHostStat@@@std@@PEAX@1@@Z 000000014005c2dc     HostStat.obj
 0002:000112f0       $ip2state$??$_Insert_nohint@AEAU?$pair@$$CBGUExtraStatsMemVerify@CHostStat@@@std@@PEAU?$_Tree_node@U?$pair@$$CBGUExtraStatsMemVerify@CHostStat@@@std@@PEAX@2@@?$_Tree@V?$_Tmap_traits@GUExtraStatsMemVerify@CHostStat@@U?$less@G@std@@V?$allocator@U?$pair@$$CBGUExtraStatsMemVerify@CHostStat@@@std@@@4@$0A@@std@@@std@@IEAA?AU?$pair@V?$_Tree_iterator@V?$_Tree_val@U?$_Tree_simple_types@U?$pair@$$CBGUExtraStatsMemVerify@CHostStat@@@std@@@std@@@std@@@std@@_N@1@_NAEAU?$pair@$$CBGUExtraStatsMemVerify@CHostStat@@@1@PEAU?$_Tree_node@U?$pair@$$CBGUExtraStatsMemVerify@CHostStat@@@std@@PEAX@1@@Z 000000014005c2f0     HostStat.obj
 0002:000112f0       $ip2state$??$_Insert_nohint@AEAU?$pair@$$CBGUExtraStatsFPSVerify@CHostStat@@@std@@PEAU?$_Tree_node@U?$pair@$$CBGUExtraStatsFPSVerify@CHostStat@@@std@@PEAX@2@@?$_Tree@V?$_Tmap_traits@GUExtraStatsFPSVerify@CHostStat@@U?$less@G@std@@V?$allocator@U?$pair@$$CBGUExtraStatsFPSVerify@CHostStat@@@std@@@4@$0A@@std@@@std@@IEAA?AU?$pair@V?$_Tree_iterator@V?$_Tree_val@U?$_Tree_simple_types@U?$pair@$$CBGUExtraStatsFPSVerify@CHostStat@@@std@@@std@@@std@@@std@@_N@1@_NAEAU?$pair@$$CBGUExtraStatsFPSVerify@CHostStat@@@1@PEAU?$_Tree_node@U?$pair@$$CBGUExtraStatsFPSVerify@CHostStat@@@std@@PEAX@1@@Z 000000014005c2f0     HostStat.obj
 0002:00011300       $unwind$?catch$0@?0???$_Insert_nohint@AEAU?$pair@$$CBGUExtraStatsFPSVerify@CHostStat@@@std@@PEAU?$_Tree_node@U?$pair@$$CBGUExtraStatsFPSVerify@CHostStat@@@std@@PEAX@2@@?$_Tree@V?$_Tmap_traits@GUExtraStatsFPSVerify@CHostStat@@U?$less@G@std@@V?$allocator@U?$pair@$$CBGUExtraStatsFPSVerify@CHostStat@@@std@@@4@$0A@@std@@@std@@IEAA?AU?$pair@V?$_Tree_iterator@V?$_Tree_val@U?$_Tree_simple_types@U?$pair@$$CBGUExtraStatsFPSVerify@CHostStat@@@std@@@std@@@std@@@std@@_N@1@_NAEAU?$pair@$$CBGUExtraStatsFPSVerify@CHostStat@@@1@PEAU?$_Tree_node@U?$pair@$$CBGUExtraStatsFPSVerify@CHostStat@@@std@@PEAX@1@@Z@4HA 000000014005c300     HostStat.obj
 0002:00011300       $unwind$?catch$0@?0???$_Insert_nohint@AEAU?$pair@$$CBGUExtraStatsMemVerify@CHostStat@@@std@@PEAU?$_Tree_node@U?$pair@$$CBGUExtraStatsMemVerify@CHostStat@@@std@@PEAX@2@@?$_Tree@V?$_Tmap_traits@GUExtraStatsMemVerify@CHostStat@@U?$less@G@std@@V?$allocator@U?$pair@$$CBGUExtraStatsMemVerify@CHostStat@@@std@@@4@$0A@@std@@@std@@IEAA?AU?$pair@V?$_Tree_iterator@V?$_Tree_val@U?$_Tree_simple_types@U?$pair@$$CBGUExtraStatsMemVerify@CHostStat@@@std@@@std@@@std@@@std@@_N@1@_NAEAU?$pair@$$CBGUExtraStatsMemVerify@CHostStat@@@1@PEAU?$_Tree_node@U?$pair@$$CBGUExtraStatsMemVerify@CHostStat@@@std@@PEAX@1@@Z@4HA 000000014005c300     HostStat.obj
 0002:00011310       $unwind$?write@CIniSection@CIniReader@@QEAAKPEAX@Z 000000014005c310     iniReader.obj
 0002:0001133c       $stateUnwindMap$?write@CIniSection@CIniReader@@QEAAKPEAX@Z 000000014005c33c     iniReader.obj
 0002:00011350       $ip2state$?write@CIniSection@CIniReader@@QEAAKPEAX@Z 000000014005c350     iniReader.obj
 0002:00011370       $unwind$?setString@CIniSection@CIniReader@@QEAAXPEBD0@Z 000000014005c370     iniReader.obj
 0002:00011398       $stateUnwindMap$?setString@CIniSection@CIniReader@@QEAAXPEBD0@Z 000000014005c398     iniReader.obj
 0002:000113a8       $ip2state$?setString@CIniSection@CIniReader@@QEAAXPEBD0@Z 000000014005c3a8     iniReader.obj
 0002:000113d0       $unwind$?getString@CIniSection@CIniReader@@QEAA_KPEBDPEAD_K@Z 000000014005c3d0     iniReader.obj
 0002:000113f0       $chain$0$?getString@CIniSection@CIniReader@@QEAA_KPEBDPEAD_K@Z 000000014005c3f0     iniReader.obj
 0002:00011404       $chain$1$?getString@CIniSection@CIniReader@@QEAA_KPEBDPEAD_K@Z 000000014005c404     iniReader.obj
 0002:00011414       $unwind$?clear@CIniReader@@QEAAXXZ 000000014005c414     iniReader.obj
 0002:00011430       $ip2state$?clear@CIniReader@@QEAAXXZ 000000014005c430     iniReader.obj
 0002:00011438       $unwind$?read@CIniReader@@QEAAKPEBD@Z 000000014005c438     iniReader.obj
 0002:0001144c       $chain$2$?read@CIniReader@@QEAAKPEBD@Z 000000014005c44c     iniReader.obj
 0002:00011460       $chain$3$?read@CIniReader@@QEAAKPEBD@Z 000000014005c460     iniReader.obj
 0002:00011474       $chain$4$?read@CIniReader@@QEAAKPEBD@Z 000000014005c474     iniReader.obj
 0002:00011484       $chain$5$?read@CIniReader@@QEAAKPEBD@Z 000000014005c484     iniReader.obj
 0002:00011494       $unwind$?write@CIniReader@@QEAAKPEBD@Z 000000014005c494     iniReader.obj
 0002:000114c0       $stateUnwindMap$?write@CIniReader@@QEAAKPEBD@Z 000000014005c4c0     iniReader.obj
 0002:000114e8       $ip2state$?write@CIniReader@@QEAAKPEBD@Z 000000014005c4e8     iniReader.obj
 0002:00011510       $unwind$?parse@CIniReader@@QEAAKPEBD@Z 000000014005c510     iniReader.obj
 0002:00011534       $unwind$?getInt@CIniReader@@QEAAHPEBD0H@Z 000000014005c534     iniReader.obj
 0002:00011550       $unwind$?getString@CIniReader@@QEAA_KPEBD0PEAD_K@Z 000000014005c550     iniReader.obj
 0002:0001156c       $unwind$?getIntArray@CIniReader@@QEAA_KPEBD0PEAH_K@Z 000000014005c56c     iniReader.obj
 0002:00011584       $chain$1$?getIntArray@CIniReader@@QEAA_KPEBD0PEAH_K@Z 000000014005c584     iniReader.obj
 0002:0001159c       $chain$2$?getIntArray@CIniReader@@QEAA_KPEBD0PEAH_K@Z 000000014005c59c     iniReader.obj
 0002:000115ac       $chain$3$?getIntArray@CIniReader@@QEAA_KPEBD0PEAH_K@Z 000000014005c5ac     iniReader.obj
 0002:000115c4       $unwind$?setString@CIniReader@@QEAAXPEBD00@Z 000000014005c5c4     iniReader.obj
 0002:000115e4       $stateUnwindMap$?setString@CIniReader@@QEAAXPEBD00@Z 000000014005c5e4     iniReader.obj
 0002:000115f0       $ip2state$?setString@CIniReader@@QEAAXPEBD00@Z 000000014005c5f0     iniReader.obj
 0002:00011608       $unwind$?find@?$_Tree@V?$_Tmap_traits@V?$basic_string@DU?$char_traits@D@std@@V?$allocator@D@2@@std@@PEAVCIniSection@CIniReader@@U?$less@V?$basic_string@DU?$char_traits@D@std@@V?$allocator@D@2@@std@@@2@V?$allocator@U?$pair@$$CBV?$basic_string@DU?$char_traits@D@std@@V?$allocator@D@2@@std@@PEAVCIniSection@CIniReader@@@std@@@2@$0A@@std@@@std@@QEAA?AV?$_Tree_iterator@V?$_Tree_val@U?$_Tree_simple_types@U?$pair@$$CBV?$basic_string@DU?$char_traits@D@std@@V?$allocator@D@2@@std@@PEAVCIniSection@CIniReader@@@std@@@std@@@std@@@2@AEBV?$basic_string@DU?$char_traits@D@std@@V?$allocator@D@2@@2@@Z 000000014005c608     iniReader.obj
 0002:0001161c       $chain$1$?find@?$_Tree@V?$_Tmap_traits@V?$basic_string@DU?$char_traits@D@std@@V?$allocator@D@2@@std@@PEAVCIniSection@CIniReader@@U?$less@V?$basic_string@DU?$char_traits@D@std@@V?$allocator@D@2@@std@@@2@V?$allocator@U?$pair@$$CBV?$basic_string@DU?$char_traits@D@std@@V?$allocator@D@2@@std@@PEAVCIniSection@CIniReader@@@std@@@2@$0A@@std@@@std@@QEAA?AV?$_Tree_iterator@V?$_Tree_val@U?$_Tree_simple_types@U?$pair@$$CBV?$basic_string@DU?$char_traits@D@std@@V?$allocator@D@2@@std@@PEAVCIniSection@CIniReader@@@std@@@std@@@std@@@2@AEBV?$basic_string@DU?$char_traits@D@std@@V?$allocator@D@2@@2@@Z 000000014005c61c     iniReader.obj
 0002:00011634       $chain$4$?find@?$_Tree@V?$_Tmap_traits@V?$basic_string@DU?$char_traits@D@std@@V?$allocator@D@2@@std@@PEAVCIniSection@CIniReader@@U?$less@V?$basic_string@DU?$char_traits@D@std@@V?$allocator@D@2@@std@@@2@V?$allocator@U?$pair@$$CBV?$basic_string@DU?$char_traits@D@std@@V?$allocator@D@2@@std@@PEAVCIniSection@CIniReader@@@std@@@2@$0A@@std@@@std@@QEAA?AV?$_Tree_iterator@V?$_Tree_val@U?$_Tree_simple_types@U?$pair@$$CBV?$basic_string@DU?$char_traits@D@std@@V?$allocator@D@2@@std@@PEAVCIniSection@CIniReader@@@std@@@std@@@std@@@2@AEBV?$basic_string@DU?$char_traits@D@std@@V?$allocator@D@2@@2@@Z 000000014005c634     iniReader.obj
 0002:00011634       $chain$2$?find@?$_Tree@V?$_Tmap_traits@V?$basic_string@DU?$char_traits@D@std@@V?$allocator@D@2@@std@@PEAVCIniSection@CIniReader@@U?$less@V?$basic_string@DU?$char_traits@D@std@@V?$allocator@D@2@@std@@@2@V?$allocator@U?$pair@$$CBV?$basic_string@DU?$char_traits@D@std@@V?$allocator@D@2@@std@@PEAVCIniSection@CIniReader@@@std@@@2@$0A@@std@@@std@@QEAA?AV?$_Tree_iterator@V?$_Tree_val@U?$_Tree_simple_types@U?$pair@$$CBV?$basic_string@DU?$char_traits@D@std@@V?$allocator@D@2@@std@@PEAVCIniSection@CIniReader@@@std@@@std@@@std@@@2@AEBV?$basic_string@DU?$char_traits@D@std@@V?$allocator@D@2@@2@@Z 000000014005c634     iniReader.obj
 0002:00011644       $chain$3$?find@?$_Tree@V?$_Tmap_traits@V?$basic_string@DU?$char_traits@D@std@@V?$allocator@D@2@@std@@PEAVCIniSection@CIniReader@@U?$less@V?$basic_string@DU?$char_traits@D@std@@V?$allocator@D@2@@std@@@2@V?$allocator@U?$pair@$$CBV?$basic_string@DU?$char_traits@D@std@@V?$allocator@D@2@@std@@PEAVCIniSection@CIniReader@@@std@@@2@$0A@@std@@@std@@QEAA?AV?$_Tree_iterator@V?$_Tree_val@U?$_Tree_simple_types@U?$pair@$$CBV?$basic_string@DU?$char_traits@D@std@@V?$allocator@D@2@@std@@PEAVCIniSection@CIniReader@@@std@@@std@@@std@@@2@AEBV?$basic_string@DU?$char_traits@D@std@@V?$allocator@D@2@@2@@Z 000000014005c644     iniReader.obj
 0002:0001165c       $unwind$?_Erase@?$_Tree@V?$_Tmap_traits@_JV?$basic_string@DU?$char_traits@D@std@@V?$allocator@D@2@@std@@U?$less@_J@2@V?$allocator@U?$pair@$$CB_JV?$basic_string@DU?$char_traits@D@std@@V?$allocator@D@2@@std@@@std@@@2@$0A@@std@@@std@@IEAAXPEAU?$_Tree_node@U?$pair@$$CB_JV?$basic_string@DU?$char_traits@D@std@@V?$allocator@D@2@@std@@@std@@PEAX@2@@Z 000000014005c65c     LoadXlsMsg.obj
 0002:0001165c       $unwind$?_Erase@?$_Tree@V?$_Tmap_traits@V?$basic_string@DU?$char_traits@D@std@@V?$allocator@D@2@@std@@PEAVCIniSection@CIniReader@@U?$less@V?$basic_string@DU?$char_traits@D@std@@V?$allocator@D@2@@std@@@2@V?$allocator@U?$pair@$$CBV?$basic_string@DU?$char_traits@D@std@@V?$allocator@D@2@@std@@PEAVCIniSection@CIniReader@@@std@@@2@$0A@@std@@@std@@IEAAXPEAU?$_Tree_node@U?$pair@$$CBV?$basic_string@DU?$char_traits@D@std@@V?$allocator@D@2@@std@@PEAVCIniSection@CIniReader@@@std@@PEAX@2@@Z 000000014005c65c     iniReader.obj
 0002:0001166c       $chain$0$?_Erase@?$_Tree@V?$_Tmap_traits@V?$basic_string@DU?$char_traits@D@std@@V?$allocator@D@2@@std@@PEAVCIniSection@CIniReader@@U?$less@V?$basic_string@DU?$char_traits@D@std@@V?$allocator@D@2@@std@@@2@V?$allocator@U?$pair@$$CBV?$basic_string@DU?$char_traits@D@std@@V?$allocator@D@2@@std@@PEAVCIniSection@CIniReader@@@std@@@2@$0A@@std@@@std@@IEAAXPEAU?$_Tree_node@U?$pair@$$CBV?$basic_string@DU?$char_traits@D@std@@V?$allocator@D@2@@std@@PEAVCIniSection@CIniReader@@@std@@PEAX@2@@Z 000000014005c66c     iniReader.obj
 0002:00011680       $chain$1$?_Erase@?$_Tree@V?$_Tmap_traits@V?$basic_string@DU?$char_traits@D@std@@V?$allocator@D@2@@std@@PEAVCIniSection@CIniReader@@U?$less@V?$basic_string@DU?$char_traits@D@std@@V?$allocator@D@2@@std@@@2@V?$allocator@U?$pair@$$CBV?$basic_string@DU?$char_traits@D@std@@V?$allocator@D@2@@std@@PEAVCIniSection@CIniReader@@@std@@@2@$0A@@std@@@std@@IEAAXPEAU?$_Tree_node@U?$pair@$$CBV?$basic_string@DU?$char_traits@D@std@@V?$allocator@D@2@@std@@PEAVCIniSection@CIniReader@@@std@@PEAX@2@@Z 000000014005c680     iniReader.obj
 0002:00011690       $chain$2$?_Erase@?$_Tree@V?$_Tmap_traits@V?$basic_string@DU?$char_traits@D@std@@V?$allocator@D@2@@std@@PEAVCIniSection@CIniReader@@U?$less@V?$basic_string@DU?$char_traits@D@std@@V?$allocator@D@2@@std@@@2@V?$allocator@U?$pair@$$CBV?$basic_string@DU?$char_traits@D@std@@V?$allocator@D@2@@std@@PEAVCIniSection@CIniReader@@@std@@@2@$0A@@std@@@std@@IEAAXPEAU?$_Tree_node@U?$pair@$$CBV?$basic_string@DU?$char_traits@D@std@@V?$allocator@D@2@@std@@PEAVCIniSection@CIniReader@@@std@@PEAX@2@@Z 000000014005c690     iniReader.obj
 0002:000116a4       $unwind$?lower_bound@?$_Tree@V?$_Tmap_traits@V?$basic_string@DU?$char_traits@D@std@@V?$allocator@D@2@@std@@V12@U?$less@V?$basic_string@DU?$char_traits@D@std@@V?$allocator@D@2@@std@@@2@V?$allocator@U?$pair@$$CBV?$basic_string@DU?$char_traits@D@std@@V?$allocator@D@2@@std@@V12@@std@@@2@$0A@@std@@@std@@QEAA?AV?$_Tree_iterator@V?$_Tree_val@U?$_Tree_simple_types@U?$pair@$$CBV?$basic_string@DU?$char_traits@D@std@@V?$allocator@D@2@@std@@V12@@std@@@std@@@std@@@2@AEBV?$basic_string@DU?$char_traits@D@std@@V?$allocator@D@2@@2@@Z 000000014005c6a4     iniReader.obj
 0002:000116b4       $chain$2$?lower_bound@?$_Tree@V?$_Tmap_traits@V?$basic_string@DU?$char_traits@D@std@@V?$allocator@D@2@@std@@V12@U?$less@V?$basic_string@DU?$char_traits@D@std@@V?$allocator@D@2@@std@@@2@V?$allocator@U?$pair@$$CBV?$basic_string@DU?$char_traits@D@std@@V?$allocator@D@2@@std@@V12@@std@@@2@$0A@@std@@@std@@QEAA?AV?$_Tree_iterator@V?$_Tree_val@U?$_Tree_simple_types@U?$pair@$$CBV?$basic_string@DU?$char_traits@D@std@@V?$allocator@D@2@@std@@V12@@std@@@std@@@std@@@2@AEBV?$basic_string@DU?$char_traits@D@std@@V?$allocator@D@2@@2@@Z 000000014005c6b4     iniReader.obj
 0002:000116d0       $chain$4$?lower_bound@?$_Tree@V?$_Tmap_traits@V?$basic_string@DU?$char_traits@D@std@@V?$allocator@D@2@@std@@V12@U?$less@V?$basic_string@DU?$char_traits@D@std@@V?$allocator@D@2@@std@@@2@V?$allocator@U?$pair@$$CBV?$basic_string@DU?$char_traits@D@std@@V?$allocator@D@2@@std@@V12@@std@@@2@$0A@@std@@@std@@QEAA?AV?$_Tree_iterator@V?$_Tree_val@U?$_Tree_simple_types@U?$pair@$$CBV?$basic_string@DU?$char_traits@D@std@@V?$allocator@D@2@@std@@V12@@std@@@std@@@std@@@2@AEBV?$basic_string@DU?$char_traits@D@std@@V?$allocator@D@2@@2@@Z 000000014005c6d0     iniReader.obj
 0002:000116ec       $chain$5$?lower_bound@?$_Tree@V?$_Tmap_traits@V?$basic_string@DU?$char_traits@D@std@@V?$allocator@D@2@@std@@V12@U?$less@V?$basic_string@DU?$char_traits@D@std@@V?$allocator@D@2@@std@@@2@V?$allocator@U?$pair@$$CBV?$basic_string@DU?$char_traits@D@std@@V?$allocator@D@2@@std@@V12@@std@@@2@$0A@@std@@@std@@QEAA?AV?$_Tree_iterator@V?$_Tree_val@U?$_Tree_simple_types@U?$pair@$$CBV?$basic_string@DU?$char_traits@D@std@@V?$allocator@D@2@@std@@V12@@std@@@std@@@std@@@2@AEBV?$basic_string@DU?$char_traits@D@std@@V?$allocator@D@2@@2@@Z 000000014005c6ec     iniReader.obj
 0002:000116fc       $unwind$?erase@?$_Tree@V?$_Tmap_traits@V?$basic_string@DU?$char_traits@D@std@@V?$allocator@D@2@@std@@PEAVCIniSection@CIniReader@@U?$less@V?$basic_string@DU?$char_traits@D@std@@V?$allocator@D@2@@std@@@2@V?$allocator@U?$pair@$$CBV?$basic_string@DU?$char_traits@D@std@@V?$allocator@D@2@@std@@PEAVCIniSection@CIniReader@@@std@@@2@$0A@@std@@@std@@QEAA?AV?$_Tree_iterator@V?$_Tree_val@U?$_Tree_simple_types@U?$pair@$$CBV?$basic_string@DU?$char_traits@D@std@@V?$allocator@D@2@@std@@PEAVCIniSection@CIniReader@@@std@@@std@@@std@@@2@V?$_Tree_const_iterator@V?$_Tree_val@U?$_Tree_simple_types@U?$pair@$$CBV?$basic_string@DU?$char_traits@D@std@@V?$allocator@D@2@@std@@PEAVCIniSection@CIniReader@@@std@@@std@@@std@@@2@0@Z 000000014005c6fc     iniReader.obj
 0002:00011720       $ip2state$?erase@?$_Tree@V?$_Tmap_traits@V?$basic_string@DU?$char_traits@D@std@@V?$allocator@D@2@@std@@PEAVCIniSection@CIniReader@@U?$less@V?$basic_string@DU?$char_traits@D@std@@V?$allocator@D@2@@std@@@2@V?$allocator@U?$pair@$$CBV?$basic_string@DU?$char_traits@D@std@@V?$allocator@D@2@@std@@PEAVCIniSection@CIniReader@@@std@@@2@$0A@@std@@@std@@QEAA?AV?$_Tree_iterator@V?$_Tree_val@U?$_Tree_simple_types@U?$pair@$$CBV?$basic_string@DU?$char_traits@D@std@@V?$allocator@D@2@@std@@PEAVCIniSection@CIniReader@@@std@@@std@@@std@@@2@V?$_Tree_const_iterator@V?$_Tree_val@U?$_Tree_simple_types@U?$pair@$$CBV?$basic_string@DU?$char_traits@D@std@@V?$allocator@D@2@@std@@PEAVCIniSection@CIniReader@@@std@@@std@@@std@@@2@0@Z 000000014005c720     iniReader.obj
 0002:00011728       $unwind$?erase@?$_Tree@V?$_Tmap_traits@V?$basic_string@DU?$char_traits@D@std@@V?$allocator@D@2@@std@@V12@U?$less@V?$basic_string@DU?$char_traits@D@std@@V?$allocator@D@2@@std@@@2@V?$allocator@U?$pair@$$CBV?$basic_string@DU?$char_traits@D@std@@V?$allocator@D@2@@std@@V12@@std@@@2@$0A@@std@@@std@@QEAA?AV?$_Tree_iterator@V?$_Tree_val@U?$_Tree_simple_types@U?$pair@$$CBV?$basic_string@DU?$char_traits@D@std@@V?$allocator@D@2@@std@@V12@@std@@@std@@@std@@@2@V?$_Tree_const_iterator@V?$_Tree_val@U?$_Tree_simple_types@U?$pair@$$CBV?$basic_string@DU?$char_traits@D@std@@V?$allocator@D@2@@std@@V12@@std@@@std@@@std@@@2@0@Z 000000014005c728     iniReader.obj
 0002:00011748       $ip2state$?erase@?$_Tree@V?$_Tmap_traits@V?$basic_string@DU?$char_traits@D@std@@V?$allocator@D@2@@std@@V12@U?$less@V?$basic_string@DU?$char_traits@D@std@@V?$allocator@D@2@@std@@@2@V?$allocator@U?$pair@$$CBV?$basic_string@DU?$char_traits@D@std@@V?$allocator@D@2@@std@@V12@@std@@@2@$0A@@std@@@std@@QEAA?AV?$_Tree_iterator@V?$_Tree_val@U?$_Tree_simple_types@U?$pair@$$CBV?$basic_string@DU?$char_traits@D@std@@V?$allocator@D@2@@std@@V12@@std@@@std@@@std@@@2@V?$_Tree_const_iterator@V?$_Tree_val@U?$_Tree_simple_types@U?$pair@$$CBV?$basic_string@DU?$char_traits@D@std@@V?$allocator@D@2@@std@@V12@@std@@@std@@@std@@@2@0@Z 000000014005c748     iniReader.obj
 0002:00011750       $unwind$??$_Buynode@U?$pair@PEADPEAVCIniSection@CIniReader@@@std@@@?$_Tree_comp_alloc@V?$_Tmap_traits@V?$basic_string@DU?$char_traits@D@std@@V?$allocator@D@2@@std@@PEAVCIniSection@CIniReader@@U?$less@V?$basic_string@DU?$char_traits@D@std@@V?$allocator@D@2@@std@@@2@V?$allocator@U?$pair@$$CBV?$basic_string@DU?$char_traits@D@std@@V?$allocator@D@2@@std@@PEAVCIniSection@CIniReader@@@std@@@2@$0A@@std@@@std@@QEAAPEAU?$_Tree_node@U?$pair@$$CBV?$basic_string@DU?$char_traits@D@std@@V?$allocator@D@2@@std@@PEAVCIniSection@CIniReader@@@std@@PEAX@1@$$QEAU?$pair@PEADPEAVCIniSection@CIniReader@@@1@@Z 000000014005c750     iniReader.obj
 0002:00011768       $tryMap$??$_Buynode@U?$pair@PEADPEAVCIniSection@CIniReader@@@std@@@?$_Tree_comp_alloc@V?$_Tmap_traits@V?$basic_string@DU?$char_traits@D@std@@V?$allocator@D@2@@std@@PEAVCIniSection@CIniReader@@U?$less@V?$basic_string@DU?$char_traits@D@std@@V?$allocator@D@2@@std@@@2@V?$allocator@U?$pair@$$CBV?$basic_string@DU?$char_traits@D@std@@V?$allocator@D@2@@std@@PEAVCIniSection@CIniReader@@@std@@@2@$0A@@std@@@std@@QEAAPEAU?$_Tree_node@U?$pair@$$CBV?$basic_string@DU?$char_traits@D@std@@V?$allocator@D@2@@std@@PEAVCIniSection@CIniReader@@@std@@PEAX@1@$$QEAU?$pair@PEADPEAVCIniSection@CIniReader@@@1@@Z 000000014005c768     iniReader.obj
 0002:0001177c       $handlerMap$0$??$_Buynode@U?$pair@PEADPEAVCIniSection@CIniReader@@@std@@@?$_Tree_comp_alloc@V?$_Tmap_traits@V?$basic_string@DU?$char_traits@D@std@@V?$allocator@D@2@@std@@PEAVCIniSection@CIniReader@@U?$less@V?$basic_string@DU?$char_traits@D@std@@V?$allocator@D@2@@std@@@2@V?$allocator@U?$pair@$$CBV?$basic_string@DU?$char_traits@D@std@@V?$allocator@D@2@@std@@PEAVCIniSection@CIniReader@@@std@@@2@$0A@@std@@@std@@QEAAPEAU?$_Tree_node@U?$pair@$$CBV?$basic_string@DU?$char_traits@D@std@@V?$allocator@D@2@@std@@PEAVCIniSection@CIniReader@@@std@@PEAX@1@$$QEAU?$pair@PEADPEAVCIniSection@CIniReader@@@1@@Z 000000014005c77c     iniReader.obj
 0002:00011790       $ip2state$??$_Buynode@U?$pair@PEADPEAVCIniSection@CIniReader@@@std@@@?$_Tree_comp_alloc@V?$_Tmap_traits@V?$basic_string@DU?$char_traits@D@std@@V?$allocator@D@2@@std@@PEAVCIniSection@CIniReader@@U?$less@V?$basic_string@DU?$char_traits@D@std@@V?$allocator@D@2@@std@@@2@V?$allocator@U?$pair@$$CBV?$basic_string@DU?$char_traits@D@std@@V?$allocator@D@2@@std@@PEAVCIniSection@CIniReader@@@std@@@2@$0A@@std@@@std@@QEAAPEAU?$_Tree_node@U?$pair@$$CBV?$basic_string@DU?$char_traits@D@std@@V?$allocator@D@2@@std@@PEAVCIniSection@CIniReader@@@std@@PEAX@1@$$QEAU?$pair@PEADPEAVCIniSection@CIniReader@@@1@@Z 000000014005c790     iniReader.obj
 0002:000117a8       $unwind$?catch$1@?0???$_Buynode@U?$pair@PEADPEAVCIniSection@CIniReader@@@std@@@?$_Tree_comp_alloc@V?$_Tmap_traits@V?$basic_string@DU?$char_traits@D@std@@V?$allocator@D@2@@std@@PEAVCIniSection@CIniReader@@U?$less@V?$basic_string@DU?$char_traits@D@std@@V?$allocator@D@2@@std@@@2@V?$allocator@U?$pair@$$CBV?$basic_string@DU?$char_traits@D@std@@V?$allocator@D@2@@std@@PEAVCIniSection@CIniReader@@@std@@@2@$0A@@std@@@std@@QEAAPEAU?$_Tree_node@U?$pair@$$CBV?$basic_string@DU?$char_traits@D@std@@V?$allocator@D@2@@std@@PEAVCIniSection@CIniReader@@@std@@PEAX@1@$$QEAU?$pair@PEADPEAVCIniSection@CIniReader@@@1@@Z@4HA 000000014005c7a8     iniReader.obj
 0002:000117b8       $unwind$??$_Insert_nohint@AEAU?$pair@$$CBV?$basic_string@DU?$char_traits@D@std@@V?$allocator@D@2@@std@@PEAVCIniSection@CIniReader@@@std@@PEAU?$_Tree_node@U?$pair@$$CBV?$basic_string@DU?$char_traits@D@std@@V?$allocator@D@2@@std@@PEAVCIniSection@CIniReader@@@std@@PEAX@2@@?$_Tree@V?$_Tmap_traits@V?$basic_string@DU?$char_traits@D@std@@V?$allocator@D@2@@std@@PEAVCIniSection@CIniReader@@U?$less@V?$basic_string@DU?$char_traits@D@std@@V?$allocator@D@2@@std@@@2@V?$allocator@U?$pair@$$CBV?$basic_string@DU?$char_traits@D@std@@V?$allocator@D@2@@std@@PEAVCIniSection@CIniReader@@@std@@@2@$0A@@std@@@std@@IEAA?AU?$pair@V?$_Tree_iterator@V?$_Tree_val@U?$_Tree_simple_types@U?$pair@$$CBV?$basic_string@DU?$char_traits@D@std@@V?$allocator@D@2@@std@@PEAVCIniSection@CIniReader@@@std@@@std@@@std@@@std@@_N@1@_NAEAU?$pair@$$CBV?$basic_string@DU?$char_traits@D@std@@V?$allocator@D@2@@std@@PEAVCIniSection@CIniReader@@@1@PEAU?$_Tree_node@U?$pair@$$CBV?$basic_string@DU?$char_traits@D@std@@V?$allocator@D@2@@std@@PEAVCIniSection@CIniReader@@@std@@PEAX@1@@Z 000000014005c7b8     iniReader.obj
 0002:000117d8       $tryMap$??$_Insert_nohint@AEAU?$pair@$$CBV?$basic_string@DU?$char_traits@D@std@@V?$allocator@D@2@@std@@PEAVCIniSection@CIniReader@@@std@@PEAU?$_Tree_node@U?$pair@$$CBV?$basic_string@DU?$char_traits@D@std@@V?$allocator@D@2@@std@@PEAVCIniSection@CIniReader@@@std@@PEAX@2@@?$_Tree@V?$_Tmap_traits@V?$basic_string@DU?$char_traits@D@std@@V?$allocator@D@2@@std@@PEAVCIniSection@CIniReader@@U?$less@V?$basic_string@DU?$char_traits@D@std@@V?$allocator@D@2@@std@@@2@V?$allocator@U?$pair@$$CBV?$basic_string@DU?$char_traits@D@std@@V?$allocator@D@2@@std@@PEAVCIniSection@CIniReader@@@std@@@2@$0A@@std@@@std@@IEAA?AU?$pair@V?$_Tree_iterator@V?$_Tree_val@U?$_Tree_simple_types@U?$pair@$$CBV?$basic_string@DU?$char_traits@D@std@@V?$allocator@D@2@@std@@PEAVCIniSection@CIniReader@@@std@@@std@@@std@@@std@@_N@1@_NAEAU?$pair@$$CBV?$basic_string@DU?$char_traits@D@std@@V?$allocator@D@2@@std@@PEAVCIniSection@CIniReader@@@1@PEAU?$_Tree_node@U?$pair@$$CBV?$basic_string@DU?$char_traits@D@std@@V?$allocator@D@2@@std@@PEAVCIniSection@CIniReader@@@std@@PEAX@1@@Z 000000014005c7d8     iniReader.obj
 0002:000117ec       $handlerMap$0$??$_Insert_nohint@AEAU?$pair@$$CBV?$basic_string@DU?$char_traits@D@std@@V?$allocator@D@2@@std@@PEAVCIniSection@CIniReader@@@std@@PEAU?$_Tree_node@U?$pair@$$CBV?$basic_string@DU?$char_traits@D@std@@V?$allocator@D@2@@std@@PEAVCIniSection@CIniReader@@@std@@PEAX@2@@?$_Tree@V?$_Tmap_traits@V?$basic_string@DU?$char_traits@D@std@@V?$allocator@D@2@@std@@PEAVCIniSection@CIniReader@@U?$less@V?$basic_string@DU?$char_traits@D@std@@V?$allocator@D@2@@std@@@2@V?$allocator@U?$pair@$$CBV?$basic_string@DU?$char_traits@D@std@@V?$allocator@D@2@@std@@PEAVCIniSection@CIniReader@@@std@@@2@$0A@@std@@@std@@IEAA?AU?$pair@V?$_Tree_iterator@V?$_Tree_val@U?$_Tree_simple_types@U?$pair@$$CBV?$basic_string@DU?$char_traits@D@std@@V?$allocator@D@2@@std@@PEAVCIniSection@CIniReader@@@std@@@std@@@std@@@std@@_N@1@_NAEAU?$pair@$$CBV?$basic_string@DU?$char_traits@D@std@@V?$allocator@D@2@@std@@PEAVCIniSection@CIniReader@@@1@PEAU?$_Tree_node@U?$pair@$$CBV?$basic_string@DU?$char_traits@D@std@@V?$allocator@D@2@@std@@PEAVCIniSection@CIniReader@@@std@@PEAX@1@@Z 000000014005c7ec     iniReader.obj
 0002:00011800       $ip2state$??$_Insert_nohint@AEAU?$pair@$$CBV?$basic_string@DU?$char_traits@D@std@@V?$allocator@D@2@@std@@PEAVCIniSection@CIniReader@@@std@@PEAU?$_Tree_node@U?$pair@$$CBV?$basic_string@DU?$char_traits@D@std@@V?$allocator@D@2@@std@@PEAVCIniSection@CIniReader@@@std@@PEAX@2@@?$_Tree@V?$_Tmap_traits@V?$basic_string@DU?$char_traits@D@std@@V?$allocator@D@2@@std@@PEAVCIniSection@CIniReader@@U?$less@V?$basic_string@DU?$char_traits@D@std@@V?$allocator@D@2@@std@@@2@V?$allocator@U?$pair@$$CBV?$basic_string@DU?$char_traits@D@std@@V?$allocator@D@2@@std@@PEAVCIniSection@CIniReader@@@std@@@2@$0A@@std@@@std@@IEAA?AU?$pair@V?$_Tree_iterator@V?$_Tree_val@U?$_Tree_simple_types@U?$pair@$$CBV?$basic_string@DU?$char_traits@D@std@@V?$allocator@D@2@@std@@PEAVCIniSection@CIniReader@@@std@@@std@@@std@@@std@@_N@1@_NAEAU?$pair@$$CBV?$basic_string@DU?$char_traits@D@std@@V?$allocator@D@2@@std@@PEAVCIniSection@CIniReader@@@1@PEAU?$_Tree_node@U?$pair@$$CBV?$basic_string@DU?$char_traits@D@std@@V?$allocator@D@2@@std@@PEAVCIniSection@CIniReader@@@std@@PEAX@1@@Z 000000014005c800     iniReader.obj
 0002:00011810       $unwind$?catch$0@?0???$_Insert_nohint@AEAU?$pair@$$CBV?$basic_string@DU?$char_traits@D@std@@V?$allocator@D@2@@std@@PEAVCIniSection@CIniReader@@@std@@PEAU?$_Tree_node@U?$pair@$$CBV?$basic_string@DU?$char_traits@D@std@@V?$allocator@D@2@@std@@PEAVCIniSection@CIniReader@@@std@@PEAX@2@@?$_Tree@V?$_Tmap_traits@V?$basic_string@DU?$char_traits@D@std@@V?$allocator@D@2@@std@@PEAVCIniSection@CIniReader@@U?$less@V?$basic_string@DU?$char_traits@D@std@@V?$allocator@D@2@@std@@@2@V?$allocator@U?$pair@$$CBV?$basic_string@DU?$char_traits@D@std@@V?$allocator@D@2@@std@@PEAVCIniSection@CIniReader@@@std@@@2@$0A@@std@@@std@@IEAA?AU?$pair@V?$_Tree_iterator@V?$_Tree_val@U?$_Tree_simple_types@U?$pair@$$CBV?$basic_string@DU?$char_traits@D@std@@V?$allocator@D@2@@std@@PEAVCIniSection@CIniReader@@@std@@@std@@@std@@@std@@_N@1@_NAEAU?$pair@$$CBV?$basic_string@DU?$char_traits@D@std@@V?$allocator@D@2@@std@@PEAVCIniSection@CIniReader@@@1@PEAU?$_Tree_node@U?$pair@$$CBV?$basic_string@DU?$char_traits@D@std@@V?$allocator@D@2@@std@@PEAVCIniSection@CIniReader@@@std@@PEAX@1@@Z@4HA 000000014005c810     iniReader.obj
 0002:00011820       $unwind$??$_Insert_hint@AEAU?$pair@$$CBV?$basic_string@DU?$char_traits@D@std@@V?$allocator@D@2@@std@@V12@@std@@PEAU?$_Tree_node@U?$pair@$$CBV?$basic_string@DU?$char_traits@D@std@@V?$allocator@D@2@@std@@V12@@std@@PEAX@2@@?$_Tree@V?$_Tmap_traits@V?$basic_string@DU?$char_traits@D@std@@V?$allocator@D@2@@std@@V12@U?$less@V?$basic_string@DU?$char_traits@D@std@@V?$allocator@D@2@@std@@@2@V?$allocator@U?$pair@$$CBV?$basic_string@DU?$char_traits@D@std@@V?$allocator@D@2@@std@@V12@@std@@@2@$0A@@std@@@std@@IEAA?AV?$_Tree_iterator@V?$_Tree_val@U?$_Tree_simple_types@U?$pair@$$CBV?$basic_string@DU?$char_traits@D@std@@V?$allocator@D@2@@std@@V12@@std@@@std@@@std@@@1@V?$_Tree_const_iterator@V?$_Tree_val@U?$_Tree_simple_types@U?$pair@$$CBV?$basic_string@DU?$char_traits@D@std@@V?$allocator@D@2@@std@@V12@@std@@@std@@@std@@@1@AEAU?$pair@$$CBV?$basic_string@DU?$char_traits@D@std@@V?$allocator@D@2@@std@@V12@@1@PEAU?$_Tree_node@U?$pair@$$CBV?$basic_string@DU?$char_traits@D@std@@V?$allocator@D@2@@std@@V12@@std@@PEAX@1@@Z 000000014005c820     iniReader.obj
 0002:00011840       $tryMap$??$_Insert_hint@AEAU?$pair@$$CBV?$basic_string@DU?$char_traits@D@std@@V?$allocator@D@2@@std@@V12@@std@@PEAU?$_Tree_node@U?$pair@$$CBV?$basic_string@DU?$char_traits@D@std@@V?$allocator@D@2@@std@@V12@@std@@PEAX@2@@?$_Tree@V?$_Tmap_traits@V?$basic_string@DU?$char_traits@D@std@@V?$allocator@D@2@@std@@V12@U?$less@V?$basic_string@DU?$char_traits@D@std@@V?$allocator@D@2@@std@@@2@V?$allocator@U?$pair@$$CBV?$basic_string@DU?$char_traits@D@std@@V?$allocator@D@2@@std@@V12@@std@@@2@$0A@@std@@@std@@IEAA?AV?$_Tree_iterator@V?$_Tree_val@U?$_Tree_simple_types@U?$pair@$$CBV?$basic_string@DU?$char_traits@D@std@@V?$allocator@D@2@@std@@V12@@std@@@std@@@std@@@1@V?$_Tree_const_iterator@V?$_Tree_val@U?$_Tree_simple_types@U?$pair@$$CBV?$basic_string@DU?$char_traits@D@std@@V?$allocator@D@2@@std@@V12@@std@@@std@@@std@@@1@AEAU?$pair@$$CBV?$basic_string@DU?$char_traits@D@std@@V?$allocator@D@2@@std@@V12@@1@PEAU?$_Tree_node@U?$pair@$$CBV?$basic_string@DU?$char_traits@D@std@@V?$allocator@D@2@@std@@V12@@std@@PEAX@1@@Z 000000014005c840     iniReader.obj
 0002:00011854       $handlerMap$0$??$_Insert_hint@AEAU?$pair@$$CBV?$basic_string@DU?$char_traits@D@std@@V?$allocator@D@2@@std@@V12@@std@@PEAU?$_Tree_node@U?$pair@$$CBV?$basic_string@DU?$char_traits@D@std@@V?$allocator@D@2@@std@@V12@@std@@PEAX@2@@?$_Tree@V?$_Tmap_traits@V?$basic_string@DU?$char_traits@D@std@@V?$allocator@D@2@@std@@V12@U?$less@V?$basic_string@DU?$char_traits@D@std@@V?$allocator@D@2@@std@@@2@V?$allocator@U?$pair@$$CBV?$basic_string@DU?$char_traits@D@std@@V?$allocator@D@2@@std@@V12@@std@@@2@$0A@@std@@@std@@IEAA?AV?$_Tree_iterator@V?$_Tree_val@U?$_Tree_simple_types@U?$pair@$$CBV?$basic_string@DU?$char_traits@D@std@@V?$allocator@D@2@@std@@V12@@std@@@std@@@std@@@1@V?$_Tree_const_iterator@V?$_Tree_val@U?$_Tree_simple_types@U?$pair@$$CBV?$basic_string@DU?$char_traits@D@std@@V?$allocator@D@2@@std@@V12@@std@@@std@@@std@@@1@AEAU?$pair@$$CBV?$basic_string@DU?$char_traits@D@std@@V?$allocator@D@2@@std@@V12@@1@PEAU?$_Tree_node@U?$pair@$$CBV?$basic_string@DU?$char_traits@D@std@@V?$allocator@D@2@@std@@V12@@std@@PEAX@1@@Z 000000014005c854     iniReader.obj
 0002:00011868       $ip2state$??$_Insert_hint@AEAU?$pair@$$CBV?$basic_string@DU?$char_traits@D@std@@V?$allocator@D@2@@std@@V12@@std@@PEAU?$_Tree_node@U?$pair@$$CBV?$basic_string@DU?$char_traits@D@std@@V?$allocator@D@2@@std@@V12@@std@@PEAX@2@@?$_Tree@V?$_Tmap_traits@V?$basic_string@DU?$char_traits@D@std@@V?$allocator@D@2@@std@@V12@U?$less@V?$basic_string@DU?$char_traits@D@std@@V?$allocator@D@2@@std@@@2@V?$allocator@U?$pair@$$CBV?$basic_string@DU?$char_traits@D@std@@V?$allocator@D@2@@std@@V12@@std@@@2@$0A@@std@@@std@@IEAA?AV?$_Tree_iterator@V?$_Tree_val@U?$_Tree_simple_types@U?$pair@$$CBV?$basic_string@DU?$char_traits@D@std@@V?$allocator@D@2@@std@@V12@@std@@@std@@@std@@@1@V?$_Tree_const_iterator@V?$_Tree_val@U?$_Tree_simple_types@U?$pair@$$CBV?$basic_string@DU?$char_traits@D@std@@V?$allocator@D@2@@std@@V12@@std@@@std@@@std@@@1@AEAU?$pair@$$CBV?$basic_string@DU?$char_traits@D@std@@V?$allocator@D@2@@std@@V12@@1@PEAU?$_Tree_node@U?$pair@$$CBV?$basic_string@DU?$char_traits@D@std@@V?$allocator@D@2@@std@@V12@@std@@PEAX@1@@Z 000000014005c868     iniReader.obj
 0002:00011888       $unwind$?catch$0@?0???$_Insert_hint@AEAU?$pair@$$CBV?$basic_string@DU?$char_traits@D@std@@V?$allocator@D@2@@std@@V12@@std@@PEAU?$_Tree_node@U?$pair@$$CBV?$basic_string@DU?$char_traits@D@std@@V?$allocator@D@2@@std@@V12@@std@@PEAX@2@@?$_Tree@V?$_Tmap_traits@V?$basic_string@DU?$char_traits@D@std@@V?$allocator@D@2@@std@@V12@U?$less@V?$basic_string@DU?$char_traits@D@std@@V?$allocator@D@2@@std@@@2@V?$allocator@U?$pair@$$CBV?$basic_string@DU?$char_traits@D@std@@V?$allocator@D@2@@std@@V12@@std@@@2@$0A@@std@@@std@@IEAA?AV?$_Tree_iterator@V?$_Tree_val@U?$_Tree_simple_types@U?$pair@$$CBV?$basic_string@DU?$char_traits@D@std@@V?$allocator@D@2@@std@@V12@@std@@@std@@@std@@@1@V?$_Tree_const_iterator@V?$_Tree_val@U?$_Tree_simple_types@U?$pair@$$CBV?$basic_string@DU?$char_traits@D@std@@V?$allocator@D@2@@std@@V12@@std@@@std@@@std@@@1@AEAU?$pair@$$CBV?$basic_string@DU?$char_traits@D@std@@V?$allocator@D@2@@std@@V12@@1@PEAU?$_Tree_node@U?$pair@$$CBV?$basic_string@DU?$char_traits@D@std@@V?$allocator@D@2@@std@@V12@@std@@PEAX@1@@Z@4HA 000000014005c888     iniReader.obj
 0002:00011898       $unwind$??$_Insert_nohint@AEAU?$pair@$$CBV?$basic_string@DU?$char_traits@D@std@@V?$allocator@D@2@@std@@V12@@std@@PEAU?$_Tree_node@U?$pair@$$CBV?$basic_string@DU?$char_traits@D@std@@V?$allocator@D@2@@std@@V12@@std@@PEAX@2@@?$_Tree@V?$_Tmap_traits@V?$basic_string@DU?$char_traits@D@std@@V?$allocator@D@2@@std@@V12@U?$less@V?$basic_string@DU?$char_traits@D@std@@V?$allocator@D@2@@std@@@2@V?$allocator@U?$pair@$$CBV?$basic_string@DU?$char_traits@D@std@@V?$allocator@D@2@@std@@V12@@std@@@2@$0A@@std@@@std@@IEAA?AU?$pair@V?$_Tree_iterator@V?$_Tree_val@U?$_Tree_simple_types@U?$pair@$$CBV?$basic_string@DU?$char_traits@D@std@@V?$allocator@D@2@@std@@V12@@std@@@std@@@std@@@std@@_N@1@_NAEAU?$pair@$$CBV?$basic_string@DU?$char_traits@D@std@@V?$allocator@D@2@@std@@V12@@1@PEAU?$_Tree_node@U?$pair@$$CBV?$basic_string@DU?$char_traits@D@std@@V?$allocator@D@2@@std@@V12@@std@@PEAX@1@@Z 000000014005c898     iniReader.obj
 0002:000118b8       $tryMap$??$_Insert_nohint@AEAU?$pair@$$CBV?$basic_string@DU?$char_traits@D@std@@V?$allocator@D@2@@std@@V12@@std@@PEAU?$_Tree_node@U?$pair@$$CBV?$basic_string@DU?$char_traits@D@std@@V?$allocator@D@2@@std@@V12@@std@@PEAX@2@@?$_Tree@V?$_Tmap_traits@V?$basic_string@DU?$char_traits@D@std@@V?$allocator@D@2@@std@@V12@U?$less@V?$basic_string@DU?$char_traits@D@std@@V?$allocator@D@2@@std@@@2@V?$allocator@U?$pair@$$CBV?$basic_string@DU?$char_traits@D@std@@V?$allocator@D@2@@std@@V12@@std@@@2@$0A@@std@@@std@@IEAA?AU?$pair@V?$_Tree_iterator@V?$_Tree_val@U?$_Tree_simple_types@U?$pair@$$CBV?$basic_string@DU?$char_traits@D@std@@V?$allocator@D@2@@std@@V12@@std@@@std@@@std@@@std@@_N@1@_NAEAU?$pair@$$CBV?$basic_string@DU?$char_traits@D@std@@V?$allocator@D@2@@std@@V12@@1@PEAU?$_Tree_node@U?$pair@$$CBV?$basic_string@DU?$char_traits@D@std@@V?$allocator@D@2@@std@@V12@@std@@PEAX@1@@Z 000000014005c8b8     iniReader.obj
 0002:000118cc       $handlerMap$0$??$_Insert_nohint@AEAU?$pair@$$CBV?$basic_string@DU?$char_traits@D@std@@V?$allocator@D@2@@std@@V12@@std@@PEAU?$_Tree_node@U?$pair@$$CBV?$basic_string@DU?$char_traits@D@std@@V?$allocator@D@2@@std@@V12@@std@@PEAX@2@@?$_Tree@V?$_Tmap_traits@V?$basic_string@DU?$char_traits@D@std@@V?$allocator@D@2@@std@@V12@U?$less@V?$basic_string@DU?$char_traits@D@std@@V?$allocator@D@2@@std@@@2@V?$allocator@U?$pair@$$CBV?$basic_string@DU?$char_traits@D@std@@V?$allocator@D@2@@std@@V12@@std@@@2@$0A@@std@@@std@@IEAA?AU?$pair@V?$_Tree_iterator@V?$_Tree_val@U?$_Tree_simple_types@U?$pair@$$CBV?$basic_string@DU?$char_traits@D@std@@V?$allocator@D@2@@std@@V12@@std@@@std@@@std@@@std@@_N@1@_NAEAU?$pair@$$CBV?$basic_string@DU?$char_traits@D@std@@V?$allocator@D@2@@std@@V12@@1@PEAU?$_Tree_node@U?$pair@$$CBV?$basic_string@DU?$char_traits@D@std@@V?$allocator@D@2@@std@@V12@@std@@PEAX@1@@Z 000000014005c8cc     iniReader.obj
 0002:000118e0       $ip2state$??$_Insert_nohint@AEAU?$pair@$$CBV?$basic_string@DU?$char_traits@D@std@@V?$allocator@D@2@@std@@V12@@std@@PEAU?$_Tree_node@U?$pair@$$CBV?$basic_string@DU?$char_traits@D@std@@V?$allocator@D@2@@std@@V12@@std@@PEAX@2@@?$_Tree@V?$_Tmap_traits@V?$basic_string@DU?$char_traits@D@std@@V?$allocator@D@2@@std@@V12@U?$less@V?$basic_string@DU?$char_traits@D@std@@V?$allocator@D@2@@std@@@2@V?$allocator@U?$pair@$$CBV?$basic_string@DU?$char_traits@D@std@@V?$allocator@D@2@@std@@V12@@std@@@2@$0A@@std@@@std@@IEAA?AU?$pair@V?$_Tree_iterator@V?$_Tree_val@U?$_Tree_simple_types@U?$pair@$$CBV?$basic_string@DU?$char_traits@D@std@@V?$allocator@D@2@@std@@V12@@std@@@std@@@std@@@std@@_N@1@_NAEAU?$pair@$$CBV?$basic_string@DU?$char_traits@D@std@@V?$allocator@D@2@@std@@V12@@1@PEAU?$_Tree_node@U?$pair@$$CBV?$basic_string@DU?$char_traits@D@std@@V?$allocator@D@2@@std@@V12@@std@@PEAX@1@@Z 000000014005c8e0     iniReader.obj
 0002:000118f0       $unwind$?catch$0@?0???$_Insert_nohint@AEAU?$pair@$$CBV?$basic_string@DU?$char_traits@D@std@@V?$allocator@D@2@@std@@V12@@std@@PEAU?$_Tree_node@U?$pair@$$CBV?$basic_string@DU?$char_traits@D@std@@V?$allocator@D@2@@std@@V12@@std@@PEAX@2@@?$_Tree@V?$_Tmap_traits@V?$basic_string@DU?$char_traits@D@std@@V?$allocator@D@2@@std@@V12@U?$less@V?$basic_string@DU?$char_traits@D@std@@V?$allocator@D@2@@std@@@2@V?$allocator@U?$pair@$$CBV?$basic_string@DU?$char_traits@D@std@@V?$allocator@D@2@@std@@V12@@std@@@2@$0A@@std@@@std@@IEAA?AU?$pair@V?$_Tree_iterator@V?$_Tree_val@U?$_Tree_simple_types@U?$pair@$$CBV?$basic_string@DU?$char_traits@D@std@@V?$allocator@D@2@@std@@V12@@std@@@std@@@std@@@std@@_N@1@_NAEAU?$pair@$$CBV?$basic_string@DU?$char_traits@D@std@@V?$allocator@D@2@@std@@V12@@1@PEAU?$_Tree_node@U?$pair@$$CBV?$basic_string@DU?$char_traits@D@std@@V?$allocator@D@2@@std@@V12@@std@@PEAX@1@@Z@4HA 000000014005c8f0     iniReader.obj
 0002:00011900       $unwind$?auth_NTLM@mailer@jwsmtp@@AEAA_NAEBV?$basic_string@DU?$char_traits@D@std@@V?$allocator@D@2@@std@@AEB_K@Z 000000014005c900     auth.obj
 0002:00011924       $stateUnwindMap$?auth_NTLM@mailer@jwsmtp@@AEAA_NAEBV?$basic_string@DU?$char_traits@D@std@@V?$allocator@D@2@@std@@AEB_K@Z 000000014005c924     auth.obj
 0002:00011940       $ip2state$?auth_NTLM@mailer@jwsmtp@@AEAA_NAEBV?$basic_string@DU?$char_traits@D@std@@V?$allocator@D@2@@std@@AEB_K@Z 000000014005c940     auth.obj
 0002:00011980       $unwind$?initNetworking@jwsmtp@@YAXXZ 000000014005c980     compat.obj
 0002:00011990       $unwind$??0mailer@jwsmtp@@QEAA@PEBD0000G_N@Z 000000014005c990     mailer.obj
 0002:000119b4       $stateUnwindMap$??0mailer@jwsmtp@@QEAA@PEBD0000G_N@Z 000000014005c9b4     mailer.obj
 0002:00011a50       $ip2state$??0mailer@jwsmtp@@QEAA@PEBD0000G_N@Z 000000014005ca50     mailer.obj
 0002:00011ab8       $unwind$?checkRFCcompat@mailer@jwsmtp@@AEAAXXZ 000000014005cab8     mailer.obj
 0002:00011ac8       $chain$0$?checkRFCcompat@mailer@jwsmtp@@AEAAXXZ 000000014005cac8     mailer.obj
 0002:00011adc       $chain$1$?checkRFCcompat@mailer@jwsmtp@@AEAAXXZ 000000014005cadc     mailer.obj
 0002:00011aec       $unwind$?setsender@mailer@jwsmtp@@QEAA_NAEBV?$basic_string@DU?$char_traits@D@std@@V?$allocator@D@2@@std@@@Z 000000014005caec     mailer.obj
 0002:00011b00       $stateUnwindMap$?setsender@mailer@jwsmtp@@QEAA_NAEBV?$basic_string@DU?$char_traits@D@std@@V?$allocator@D@2@@std@@@Z 000000014005cb00     mailer.obj
 0002:00011b08       $ip2state$?setsender@mailer@jwsmtp@@QEAA_NAEBV?$basic_string@DU?$char_traits@D@std@@V?$allocator@D@2@@std@@@Z 000000014005cb08     mailer.obj
 0002:00011b20       $unwind$?addrecipient@mailer@jwsmtp@@QEAA_NAEBV?$basic_string@DU?$char_traits@D@std@@V?$allocator@D@2@@std@@F@Z 000000014005cb20     mailer.obj
 0002:00011b44       $stateUnwindMap$?addrecipient@mailer@jwsmtp@@QEAA_NAEBV?$basic_string@DU?$char_traits@D@std@@V?$allocator@D@2@@std@@F@Z 000000014005cb44     mailer.obj
 0002:00011b60       $ip2state$?addrecipient@mailer@jwsmtp@@QEAA_NAEBV?$basic_string@DU?$char_traits@D@std@@V?$allocator@D@2@@std@@F@Z 000000014005cb60     mailer.obj
 0002:00011b90       $unwind$??Rmailer@jwsmtp@@QEAAXXZ 000000014005cb90     mailer.obj
 0002:00011bc4       $stateUnwindMap$??Rmailer@jwsmtp@@QEAAXXZ 000000014005cbc4     mailer.obj
 0002:00011c70       $ip2state$??Rmailer@jwsmtp@@QEAAXXZ 000000014005cc70     mailer.obj
 0002:00011dc0       $unwind$?makesmtpmessage@mailer@jwsmtp@@AEBA?AV?$vector@DV?$allocator@D@std@@@std@@XZ 000000014005cdc0     mailer.obj
 0002:00011df0       $stateUnwindMap$?makesmtpmessage@mailer@jwsmtp@@AEBA?AV?$vector@DV?$allocator@D@std@@@std@@XZ 000000014005cdf0     mailer.obj
 0002:00011f30       $ip2state$?makesmtpmessage@mailer@jwsmtp@@AEBA?AV?$vector@DV?$allocator@D@std@@@std@@XZ 000000014005cf30     mailer.obj
 0002:00012128       $unwind$?gethostaddresses@mailer@jwsmtp@@AEAA_NAEAV?$vector@USOCKADDR_IN@jwsmtp@@V?$allocator@USOCKADDR_IN@jwsmtp@@@std@@@std@@@Z 000000014005d128     mailer.obj
 0002:00012150       $stateUnwindMap$?gethostaddresses@mailer@jwsmtp@@AEAA_NAEAV?$vector@USOCKADDR_IN@jwsmtp@@V?$allocator@USOCKADDR_IN@jwsmtp@@@std@@@std@@@Z 000000014005d150     mailer.obj
 0002:00012170       $ip2state$?gethostaddresses@mailer@jwsmtp@@AEAA_NAEAV?$vector@USOCKADDR_IN@jwsmtp@@V?$allocator@USOCKADDR_IN@jwsmtp@@@std@@@std@@@Z 000000014005d170     mailer.obj
 0002:000121b8       $unwind$?parsename@mailer@jwsmtp@@AEAAXAEAHQEBEAEAV?$basic_string@DU?$char_traits@D@std@@V?$allocator@D@2@@std@@@Z 000000014005d1b8     mailer.obj
 0002:000121cc       $unwind$?parseaddress@mailer@jwsmtp@@AEAA?AUAddress@12@AEBV?$basic_string@DU?$char_traits@D@std@@V?$allocator@D@2@@std@@@Z 000000014005d1cc     mailer.obj
 0002:000121f8       $stateUnwindMap$?parseaddress@mailer@jwsmtp@@AEAA?AUAddress@12@AEBV?$basic_string@DU?$char_traits@D@std@@V?$allocator@D@2@@std@@@Z 000000014005d1f8     mailer.obj
 0002:00012200       $ip2state$?parseaddress@mailer@jwsmtp@@AEAA?AUAddress@12@AEBV?$basic_string@DU?$char_traits@D@std@@V?$allocator@D@2@@std@@@Z 000000014005d200     mailer.obj
 0002:00012218       $unwind$?authenticate@mailer@jwsmtp@@AEAA_NAEBV?$basic_string@DU?$char_traits@D@std@@V?$allocator@D@2@@std@@AEB_K@Z 000000014005d218     mailer.obj
 0002:00012248       $stateUnwindMap$?authenticate@mailer@jwsmtp@@AEAA_NAEBV?$basic_string@DU?$char_traits@D@std@@V?$allocator@D@2@@std@@AEB_K@Z 000000014005d248     mailer.obj
 0002:00012280       $ip2state$?authenticate@mailer@jwsmtp@@AEAA_NAEBV?$basic_string@DU?$char_traits@D@std@@V?$allocator@D@2@@std@@AEB_K@Z 000000014005d280     mailer.obj
 0002:00012300       $unwind$??1?$vector@U?$pair@V?$vector@DV?$allocator@D@std@@@std@@V?$basic_string@DU?$char_traits@D@std@@V?$allocator@D@2@@2@@std@@V?$allocator@U?$pair@V?$vector@DV?$allocator@D@std@@@std@@V?$basic_string@DU?$char_traits@D@std@@V?$allocator@D@2@@2@@std@@@2@@std@@QEAA@XZ 000000014005d300     mailer.obj
 0002:00012300       $unwind$??1?$vector@U?$pair@UAddress@mailer@jwsmtp@@F@std@@V?$allocator@U?$pair@UAddress@mailer@jwsmtp@@F@std@@@2@@std@@QEAA@XZ 000000014005d300     mailer.obj
 0002:00012300       $unwind$??0FindXlsMsg@@QEAA@XZ 000000014005d300     LoadXlsMsg.obj
 0002:0001230c       $chain$0$??1?$vector@U?$pair@UAddress@mailer@jwsmtp@@F@std@@V?$allocator@U?$pair@UAddress@mailer@jwsmtp@@F@std@@@2@@std@@QEAA@XZ 000000014005d30c     mailer.obj
 0002:00012320       $chain$1$??1?$vector@U?$pair@UAddress@mailer@jwsmtp@@F@std@@V?$allocator@U?$pair@UAddress@mailer@jwsmtp@@F@std@@@2@@std@@QEAA@XZ 000000014005d320     mailer.obj
 0002:00012330       $chain$0$??1?$vector@U?$pair@V?$vector@DV?$allocator@D@std@@@std@@V?$basic_string@DU?$char_traits@D@std@@V?$allocator@D@2@@2@@std@@V?$allocator@U?$pair@V?$vector@DV?$allocator@D@std@@@std@@V?$basic_string@DU?$char_traits@D@std@@V?$allocator@D@2@@2@@std@@@2@@std@@QEAA@XZ 000000014005d330     mailer.obj
 0002:00012344       $chain$1$??1?$vector@U?$pair@V?$vector@DV?$allocator@D@std@@@std@@V?$basic_string@DU?$char_traits@D@std@@V?$allocator@D@2@@2@@std@@V?$allocator@U?$pair@V?$vector@DV?$allocator@D@std@@@std@@V?$basic_string@DU?$char_traits@D@std@@V?$allocator@D@2@@2@@std@@@2@@std@@QEAA@XZ 000000014005d344     mailer.obj
 0002:00012354       $unwind$??$?HDU?$char_traits@D@std@@V?$allocator@D@1@@std@@YA?AV?$basic_string@DU?$char_traits@D@std@@V?$allocator@D@2@@0@$$QEAV10@0@Z 000000014005d354     mailer.obj
 0002:00012368       $chain$1$??$?HDU?$char_traits@D@std@@V?$allocator@D@1@@std@@YA?AV?$basic_string@DU?$char_traits@D@std@@V?$allocator@D@2@@0@$$QEAV10@0@Z 000000014005d368     mailer.obj
 0002:00012380       $chain$2$??$?HDU?$char_traits@D@std@@V?$allocator@D@1@@std@@YA?AV?$basic_string@DU?$char_traits@D@std@@V?$allocator@D@2@@0@$$QEAV10@0@Z 000000014005d380     mailer.obj
 0002:00012390       $unwind$??$_Emplace_reallocate@AEBV?$basic_string@DU?$char_traits@D@std@@V?$allocator@D@2@@std@@@?$vector@V?$basic_string@DU?$char_traits@D@std@@V?$allocator@D@2@@std@@V?$allocator@V?$basic_string@DU?$char_traits@D@std@@V?$allocator@D@2@@std@@@2@@std@@QEAAPEAV?$basic_string@DU?$char_traits@D@std@@V?$allocator@D@2@@1@QEAV21@AEBV21@@Z 000000014005d390     mailer.obj
 0002:000123ac       $tryMap$??$_Emplace_reallocate@AEBV?$basic_string@DU?$char_traits@D@std@@V?$allocator@D@2@@std@@@?$vector@V?$basic_string@DU?$char_traits@D@std@@V?$allocator@D@2@@std@@V?$allocator@V?$basic_string@DU?$char_traits@D@std@@V?$allocator@D@2@@std@@@2@@std@@QEAAPEAV?$basic_string@DU?$char_traits@D@std@@V?$allocator@D@2@@1@QEAV21@AEBV21@@Z 000000014005d3ac     mailer.obj
 0002:000123c0       $handlerMap$0$??$_Emplace_reallocate@AEBV?$basic_string@DU?$char_traits@D@std@@V?$allocator@D@2@@std@@@?$vector@V?$basic_string@DU?$char_traits@D@std@@V?$allocator@D@2@@std@@V?$allocator@V?$basic_string@DU?$char_traits@D@std@@V?$allocator@D@2@@std@@@2@@std@@QEAAPEAV?$basic_string@DU?$char_traits@D@std@@V?$allocator@D@2@@1@QEAV21@AEBV21@@Z 000000014005d3c0     mailer.obj
 0002:000123d8       $ip2state$??$_Emplace_reallocate@AEBV?$basic_string@DU?$char_traits@D@std@@V?$allocator@D@2@@std@@@?$vector@V?$basic_string@DU?$char_traits@D@std@@V?$allocator@D@2@@std@@V?$allocator@V?$basic_string@DU?$char_traits@D@std@@V?$allocator@D@2@@std@@@2@@std@@QEAAPEAV?$basic_string@DU?$char_traits@D@std@@V?$allocator@D@2@@1@QEAV21@AEBV21@@Z 000000014005d3d8     mailer.obj
 0002:000123f8       $unwind$?catch$3@?0???$_Emplace_reallocate@AEBV?$basic_string@DU?$char_traits@D@std@@V?$allocator@D@2@@std@@@?$vector@V?$basic_string@DU?$char_traits@D@std@@V?$allocator@D@2@@std@@V?$allocator@V?$basic_string@DU?$char_traits@D@std@@V?$allocator@D@2@@std@@@2@@std@@QEAAPEAV?$basic_string@DU?$char_traits@D@std@@V?$allocator@D@2@@1@QEAV21@AEBV21@@Z@4HA 000000014005d3f8     mailer.obj
 0002:00012408       $unwind$??$_Emplace_reallocate@U?$pair@UAddress@mailer@jwsmtp@@F@std@@@?$vector@U?$pair@UAddress@mailer@jwsmtp@@F@std@@V?$allocator@U?$pair@UAddress@mailer@jwsmtp@@F@std@@@2@@std@@QEAAPEAU?$pair@UAddress@mailer@jwsmtp@@F@1@QEAU21@$$QEAU21@@Z 000000014005d408     mailer.obj
 0002:00012418       $chain$3$??$_Emplace_reallocate@U?$pair@UAddress@mailer@jwsmtp@@F@std@@@?$vector@U?$pair@UAddress@mailer@jwsmtp@@F@std@@V?$allocator@U?$pair@UAddress@mailer@jwsmtp@@F@std@@@2@@std@@QEAAPEAU?$pair@UAddress@mailer@jwsmtp@@F@1@QEAU21@$$QEAU21@@Z 000000014005d418     mailer.obj
 0002:00012438       $chain$5$??$_Emplace_reallocate@U?$pair@UAddress@mailer@jwsmtp@@F@std@@@?$vector@U?$pair@UAddress@mailer@jwsmtp@@F@std@@V?$allocator@U?$pair@UAddress@mailer@jwsmtp@@F@std@@@2@@std@@QEAAPEAU?$pair@UAddress@mailer@jwsmtp@@F@1@QEAU21@$$QEAU21@@Z 000000014005d438     mailer.obj
 0002:00012458       $chain$6$??$_Emplace_reallocate@U?$pair@UAddress@mailer@jwsmtp@@F@std@@@?$vector@U?$pair@UAddress@mailer@jwsmtp@@F@std@@V?$allocator@U?$pair@UAddress@mailer@jwsmtp@@F@std@@@2@@std@@QEAAPEAU?$pair@UAddress@mailer@jwsmtp@@F@1@QEAU21@$$QEAU21@@Z 000000014005d458     mailer.obj
 0002:00012468       $unwind$??$_Emplace_reallocate@AEBUSOCKADDR_IN@jwsmtp@@@?$vector@USOCKADDR_IN@jwsmtp@@V?$allocator@USOCKADDR_IN@jwsmtp@@@std@@@std@@QEAAPEAUSOCKADDR_IN@jwsmtp@@QEAU23@AEBU23@@Z 000000014005d468     mailer.obj
 0002:00012478       $chain$2$??$_Emplace_reallocate@AEBUSOCKADDR_IN@jwsmtp@@@?$vector@USOCKADDR_IN@jwsmtp@@V?$allocator@USOCKADDR_IN@jwsmtp@@@std@@@std@@QEAAPEAUSOCKADDR_IN@jwsmtp@@QEAU23@AEBU23@@Z 000000014005d478     mailer.obj
 0002:00012494       $chain$4$??$_Emplace_reallocate@AEBUSOCKADDR_IN@jwsmtp@@@?$vector@USOCKADDR_IN@jwsmtp@@V?$allocator@USOCKADDR_IN@jwsmtp@@@std@@@std@@QEAAPEAUSOCKADDR_IN@jwsmtp@@QEAU23@AEBU23@@Z 000000014005d494     mailer.obj
 0002:000124b0       $chain$5$??$_Emplace_reallocate@AEBUSOCKADDR_IN@jwsmtp@@@?$vector@USOCKADDR_IN@jwsmtp@@V?$allocator@USOCKADDR_IN@jwsmtp@@@std@@@std@@QEAAPEAUSOCKADDR_IN@jwsmtp@@QEAU23@AEBU23@@Z 000000014005d4b0     mailer.obj
 0002:000124c0       $unwind$??$_Emplace_reallocate@AEBD@?$vector@DV?$allocator@D@std@@@std@@QEAAPEADQEADAEBD@Z 000000014005d4c0     mailer.obj
 0002:000124c0       $unwind$??$_Emplace_reallocate@D@?$vector@DV?$allocator@D@std@@@std@@QEAAPEADQEAD$$QEAD@Z 000000014005d4c0     mailer.obj
 0002:000124d4       $chain$1$??$_Emplace_reallocate@AEBD@?$vector@DV?$allocator@D@std@@@std@@QEAAPEADQEADAEBD@Z 000000014005d4d4     mailer.obj
 0002:000124d4       $chain$1$??$_Emplace_reallocate@D@?$vector@DV?$allocator@D@std@@@std@@QEAAPEADQEAD$$QEAD@Z 000000014005d4d4     mailer.obj
 0002:000124ec       $chain$2$??$_Emplace_reallocate@AEBD@?$vector@DV?$allocator@D@std@@@std@@QEAAPEADQEADAEBD@Z 000000014005d4ec     mailer.obj
 0002:000124ec       $chain$2$??$_Emplace_reallocate@D@?$vector@DV?$allocator@D@std@@@std@@QEAAPEADQEAD$$QEAD@Z 000000014005d4ec     mailer.obj
 0002:000124fc       $unwind$??$_Insert_range@PEBD@?$vector@DV?$allocator@D@std@@@std@@AEAAXV?$_Vector_const_iterator@V?$_Vector_val@U?$_Simple_types@D@std@@@std@@@1@PEBD1Uforward_iterator_tag@1@@Z 000000014005d4fc     mailer.obj
 0002:000124fc       $unwind$??$_Insert_range@PEAD@?$vector@DV?$allocator@D@std@@@std@@AEAAXV?$_Vector_const_iterator@V?$_Vector_val@U?$_Simple_types@D@std@@@std@@@1@PEAD1Uforward_iterator_tag@1@@Z 000000014005d4fc     mailer.obj
 0002:00012510       $chain$1$??$_Insert_range@PEAD@?$vector@DV?$allocator@D@std@@@std@@AEAAXV?$_Vector_const_iterator@V?$_Vector_val@U?$_Simple_types@D@std@@@std@@@1@PEAD1Uforward_iterator_tag@1@@Z 000000014005d510     mailer.obj
 0002:00012510       $chain$1$??$_Insert_range@PEBD@?$vector@DV?$allocator@D@std@@@std@@AEAAXV?$_Vector_const_iterator@V?$_Vector_val@U?$_Simple_types@D@std@@@std@@@1@PEBD1Uforward_iterator_tag@1@@Z 000000014005d510     mailer.obj
 0002:00012528       $chain$2$??$_Insert_range@PEAD@?$vector@DV?$allocator@D@std@@@std@@AEAAXV?$_Vector_const_iterator@V?$_Vector_val@U?$_Simple_types@D@std@@@std@@@1@PEAD1Uforward_iterator_tag@1@@Z 000000014005d528     mailer.obj
 0002:00012528       $chain$2$??$_Insert_range@PEBD@?$vector@DV?$allocator@D@std@@@std@@AEAAXV?$_Vector_const_iterator@V?$_Vector_val@U?$_Simple_types@D@std@@@std@@@1@PEBD1Uforward_iterator_tag@1@@Z 000000014005d528     mailer.obj
 0002:00012538       $chain$3$??$_Insert_range@PEAD@?$vector@DV?$allocator@D@std@@@std@@AEAAXV?$_Vector_const_iterator@V?$_Vector_val@U?$_Simple_types@D@std@@@std@@@1@PEAD1Uforward_iterator_tag@1@@Z 000000014005d538     mailer.obj
 0002:00012538       $chain$3$??$_Insert_range@PEBD@?$vector@DV?$allocator@D@std@@@std@@AEAAXV?$_Vector_const_iterator@V?$_Vector_val@U?$_Simple_types@D@std@@@std@@@1@PEBD1Uforward_iterator_tag@1@@Z 000000014005d538     mailer.obj
 0002:00012550       $unwind$??$_Reallocate_grow_by@V<lambda_f3a66ab6a0570788f31503db83886f49>@@_KPEBD_K@?$basic_string@DU?$char_traits@D@std@@V?$allocator@D@2@@std@@QEAAAEAV01@_KV<lambda_f3a66ab6a0570788f31503db83886f49>@@_KPEBD2@Z 000000014005d550     mailer.obj
 0002:0001255c       $chain$2$??$_Reallocate_grow_by@V<lambda_f3a66ab6a0570788f31503db83886f49>@@_KPEBD_K@?$basic_string@DU?$char_traits@D@std@@V?$allocator@D@2@@std@@QEAAAEAV01@_KV<lambda_f3a66ab6a0570788f31503db83886f49>@@_KPEBD2@Z 000000014005d55c     mailer.obj
 0002:00012578       $chain$3$??$_Reallocate_grow_by@V<lambda_f3a66ab6a0570788f31503db83886f49>@@_KPEBD_K@?$basic_string@DU?$char_traits@D@std@@V?$allocator@D@2@@std@@QEAAAEAV01@_KV<lambda_f3a66ab6a0570788f31503db83886f49>@@_KPEBD2@Z 000000014005d578     mailer.obj
 0002:00012588       $unwind$des_key_schedule   000000014005d588     des.obj
 0002:00012588       $unwind$gl_des_ecb_crypt   000000014005d588     des.obj
 0002:00012598       $unwind$md4_process_bytes  000000014005d598     md4.obj
 0002:000125a8       $chain$0$md4_process_bytes 000000014005d5a8     md4.obj
 0002:000125bc       $chain$1$md4_process_bytes 000000014005d5bc     md4.obj
 0002:000125d0       $chain$2$md4_process_bytes 000000014005d5d0     md4.obj
 0002:000125e0       $chain$3$md4_process_bytes 000000014005d5e0     md4.obj
 0002:000125f0       $unwind$md4_process_block  000000014005d5f0     md4.obj
 0002:000125f8       $chain$7$md4_process_block 000000014005d5f8     md4.obj
 0002:00012628       $chain$8$md4_process_block 000000014005d628     md4.obj
 0002:00012638       $unwind$ntlm_convert_key   000000014005d638     ntlmencrypt.obj
 0002:00012648       $unwind$buildSmbNtlmAuthResponse 000000014005d648     smbutil.obj
 0002:00012664       $chain$0$buildSmbNtlmAuthResponse 000000014005d664     smbutil.obj
 0002:00012678       $chain$1$buildSmbNtlmAuthResponse 000000014005d678     smbutil.obj
 0002:0001268c       $chain$2$buildSmbNtlmAuthResponse 000000014005d68c     smbutil.obj
 0002:0001269c       $chain$3$buildSmbNtlmAuthResponse 000000014005d69c     smbutil.obj
 0002:000126ac       $chain$4$buildSmbNtlmAuthResponse 000000014005d6ac     smbutil.obj
 0002:000126c0       $unwind$?getHashFromFile@md5wrapper@@QEAA?AV?$basic_string@DU?$char_traits@D@std@@V?$allocator@D@2@@std@@V23@@Z 000000014005d6c0     md5wrapper.obj
 0002:000126e8       $stateUnwindMap$?getHashFromFile@md5wrapper@@QEAA?AV?$basic_string@DU?$char_traits@D@std@@V?$allocator@D@2@@std@@V23@@Z 000000014005d6e8     md5wrapper.obj
 0002:000126f0       $ip2state$?getHashFromFile@md5wrapper@@QEAA?AV?$basic_string@DU?$char_traits@D@std@@V?$allocator@D@2@@std@@V23@@Z 000000014005d6f0     md5wrapper.obj
 0002:00012700       $unwind$?_InitPathNameInfo@CHLogger@@CAXPEBD000@Z 000000014005d700     HostLogger.obj
 0002:00012724       $unwind$?Log@CHLogger@@SAXW4ELOG_LEVEL@1@PEBDZZ 000000014005d724     HostLogger.obj
 0002:0001272c       $unwind$?LogTimeOut@CHLogger@@SAXPEBDZZ 000000014005d72c     HostLogger.obj
 0002:00012740       $chain$0$?LogTimeOut@CHLogger@@SAXPEBDZZ 000000014005d740     HostLogger.obj
 0002:00012754       $chain$3$?LogTimeOut@CHLogger@@SAXPEBDZZ 000000014005d754     HostLogger.obj
 0002:00012770       $chain$4$?LogTimeOut@CHLogger@@SAXPEBDZZ 000000014005d770     HostLogger.obj
 0002:00012780       $chain$5$?LogTimeOut@CHLogger@@SAXPEBDZZ 000000014005d780     HostLogger.obj
 0002:00012790       $unwind$?LogPacket@CHLogger@@SAXPEBDZZ 000000014005d790     HostLogger.obj
 0002:000127b0       $stateUnwindMap$?LogPacket@CHLogger@@SAXPEBDZZ 000000014005d7b0     HostLogger.obj
 0002:000127b8       $ip2state$?LogPacket@CHLogger@@SAXPEBDZZ 000000014005d7b8     HostLogger.obj
 0002:000127c8       $unwind$?LogModeUserCount@CHLogger@@SAXPEBDZZ 000000014005d7c8     HostLogger.obj
 0002:000127dc       $chain$0$?LogModeUserCount@CHLogger@@SAXPEBDZZ 000000014005d7dc     HostLogger.obj
 0002:000127f0       $chain$1$?LogModeUserCount@CHLogger@@SAXPEBDZZ 000000014005d7f0     HostLogger.obj
 0002:00012804       $chain$2$?LogModeUserCount@CHLogger@@SAXPEBDZZ 000000014005d804     HostLogger.obj
 0002:00012814       $chain$3$?LogModeUserCount@CHLogger@@SAXPEBDZZ 000000014005d814     HostLogger.obj
 0002:00012824       $unwind$?LogServerAppUseCount@CHLogger@@SAXPEBDZZ 000000014005d824     HostLogger.obj
 0002:00012838       $chain$0$?LogServerAppUseCount@CHLogger@@SAXPEBDZZ 000000014005d838     HostLogger.obj
 0002:0001284c       $chain$1$?LogServerAppUseCount@CHLogger@@SAXPEBDZZ 000000014005d84c     HostLogger.obj
 0002:0001285c       $unwind$?LogIPCMessage@CHLogger@@SAXPEBDZZ 000000014005d85c     HostLogger.obj
 0002:0001285c       $unwind$?LogRWProcessMemory@CHLogger@@SAXPEBDZZ 000000014005d85c     HostLogger.obj
 0002:00012870       $chain$0$?LogRWProcessMemory@CHLogger@@SAXPEBDZZ 000000014005d870     HostLogger.obj
 0002:00012884       $chain$1$?LogRWProcessMemory@CHLogger@@SAXPEBDZZ 000000014005d884     HostLogger.obj
 0002:00012898       $chain$2$?LogRWProcessMemory@CHLogger@@SAXPEBDZZ 000000014005d898     HostLogger.obj
 0002:000128a8       $chain$3$?LogRWProcessMemory@CHLogger@@SAXPEBDZZ 000000014005d8a8     HostLogger.obj
 0002:000128b8       $chain$0$?LogIPCMessage@CHLogger@@SAXPEBDZZ 000000014005d8b8     HostLogger.obj
 0002:000128cc       $chain$1$?LogIPCMessage@CHLogger@@SAXPEBDZZ 000000014005d8cc     HostLogger.obj
 0002:000128e0       $chain$2$?LogIPCMessage@CHLogger@@SAXPEBDZZ 000000014005d8e0     HostLogger.obj
 0002:000128f0       $chain$3$?LogIPCMessage@CHLogger@@SAXPEBDZZ 000000014005d8f0     HostLogger.obj
 0002:00012900       $unwind$?_BuildDirectory@CHLogger@@CAXAEBU_SYSTEMTIME@@@Z 000000014005d900     HostLogger.obj
 0002:0001292c       $stateUnwindMap$?_BuildDirectory@CHLogger@@CAXAEBU_SYSTEMTIME@@@Z 000000014005d92c     HostLogger.obj
 0002:00012948       $ip2state$?_BuildDirectory@CHLogger@@CAXAEBU_SYSTEMTIME@@@Z 000000014005d948     HostLogger.obj
 0002:00012978       $unwind$?_DoLogWithLevel@CHLogger@@CAXPEBDW4ELOG_LEVEL@1@0PEAD@Z 000000014005d978     HostLogger.obj
 0002:00012998       $stateUnwindMap$?_DoLogWithLevel@CHLogger@@CAXPEBDW4ELOG_LEVEL@1@0PEAD@Z 000000014005d998     HostLogger.obj
 0002:000129a0       $ip2state$?_DoLogWithLevel@CHLogger@@CAXPEBDW4ELOG_LEVEL@1@0PEAD@Z 000000014005d9a0     HostLogger.obj
 0002:000129b0       $unwind$?Init@CLogMsgManager@@SA_NW4ESHARED_MEM_USAGE_TYPE@1@@Z 000000014005d9b0     LogMsgManager.obj
 0002:000129c8       $stateUnwindMap$?Init@CLogMsgManager@@SA_NW4ESHARED_MEM_USAGE_TYPE@1@@Z 000000014005d9c8     LogMsgManager.obj
 0002:000129d8       $ip2state$?Init@CLogMsgManager@@SA_NW4ESHARED_MEM_USAGE_TYPE@1@@Z 000000014005d9d8     LogMsgManager.obj
 0002:00012a00       $unwind$?GetString@CLogMsgManager@@SA?BV?$basic_string@DU?$char_traits@D@std@@V?$allocator@D@2@@std@@I@Z 000000014005da00     LogMsgManager.obj
 0002:00012a10       $chain$0$?GetString@CLogMsgManager@@SA?BV?$basic_string@DU?$char_traits@D@std@@V?$allocator@D@2@@std@@I@Z 000000014005da10     LogMsgManager.obj
 0002:00012a24       $chain$1$?GetString@CLogMsgManager@@SA?BV?$basic_string@DU?$char_traits@D@std@@V?$allocator@D@2@@std@@I@Z 000000014005da24     LogMsgManager.obj
 0002:00012a24       $chain$3$?GetString@CLogMsgManager@@SA?BV?$basic_string@DU?$char_traits@D@std@@V?$allocator@D@2@@std@@I@Z 000000014005da24     LogMsgManager.obj
 0002:00012a34       $chain$2$?GetString@CLogMsgManager@@SA?BV?$basic_string@DU?$char_traits@D@std@@V?$allocator@D@2@@std@@I@Z 000000014005da34     LogMsgManager.obj
 0002:00012a48       $unwind$?_WriteXlsDataToSharedMemory@CLogMsgManager@@CA_NXZ 000000014005da48     LogMsgManager.obj
 0002:00012a70       $stateUnwindMap$?_WriteXlsDataToSharedMemory@CLogMsgManager@@CA_NXZ 000000014005da70     LogMsgManager.obj
 0002:00012a78       $ip2state$?_WriteXlsDataToSharedMemory@CLogMsgManager@@CA_NXZ 000000014005da78     LogMsgManager.obj
 0002:00012a98       $unwind$??$_Emplace_reallocate@AEBQEAX@?$vector@PEAXV?$allocator@PEAX@std@@@std@@QEAAPEAPEAXQEAPEAXAEBQEAX@Z 000000014005da98     LogMsgManager.obj
 0002:00012aa4       $chain$2$??$_Emplace_reallocate@AEBQEAX@?$vector@PEAXV?$allocator@PEAX@std@@@std@@QEAAPEAPEAXQEAPEAXAEBQEAX@Z 000000014005daa4     LogMsgManager.obj
 0002:00012ac0       $chain$4$??$_Emplace_reallocate@AEBQEAX@?$vector@PEAXV?$allocator@PEAX@std@@@std@@QEAAPEAPEAXQEAPEAXAEBQEAX@Z 000000014005dac0     LogMsgManager.obj
 0002:00012adc       $chain$5$??$_Emplace_reallocate@AEBQEAX@?$vector@PEAXV?$allocator@PEAX@std@@@std@@QEAAPEAPEAXQEAPEAXAEBQEAX@Z 000000014005dadc     LogMsgManager.obj
 0002:00012aec       $unwind$??_GFindXlsMsg@@UEAAPEAXI@Z 000000014005daec     LoadXlsMsg.obj
 0002:00012b08       $ip2state$??_GFindXlsMsg@@UEAAPEAXI@Z 000000014005db08     LoadXlsMsg.obj
 0002:00012b10       $unwind$?LoadWMszFile@FindXlsMsg@@QEAA_NPEAD@Z 000000014005db10     LoadXlsMsg.obj
 0002:00012b40       $ip2state$?LoadWMszFile@FindXlsMsg@@QEAA_NPEAD@Z 000000014005db40     LoadXlsMsg.obj
 0002:00012b58       $unwind$??A?$map@_JV?$basic_string@DU?$char_traits@D@std@@V?$allocator@D@2@@std@@U?$less@_J@2@V?$allocator@U?$pair@$$CB_JV?$basic_string@DU?$char_traits@D@std@@V?$allocator@D@2@@std@@@std@@@2@@std@@QEAAAEAV?$basic_string@DU?$char_traits@D@std@@V?$allocator@D@2@@1@AEB_J@Z 000000014005db58     LoadXlsMsg.obj
 0002:00012b64       $chain$0$?_Erase@?$_Tree@V?$_Tmap_traits@_JV?$basic_string@DU?$char_traits@D@std@@V?$allocator@D@2@@std@@U?$less@_J@2@V?$allocator@U?$pair@$$CB_JV?$basic_string@DU?$char_traits@D@std@@V?$allocator@D@2@@std@@@std@@@2@$0A@@std@@@std@@IEAAXPEAU?$_Tree_node@U?$pair@$$CB_JV?$basic_string@DU?$char_traits@D@std@@V?$allocator@D@2@@std@@@std@@PEAX@2@@Z 000000014005db64     LoadXlsMsg.obj
 0002:00012b78       $chain$1$?_Erase@?$_Tree@V?$_Tmap_traits@_JV?$basic_string@DU?$char_traits@D@std@@V?$allocator@D@2@@std@@U?$less@_J@2@V?$allocator@U?$pair@$$CB_JV?$basic_string@DU?$char_traits@D@std@@V?$allocator@D@2@@std@@@std@@@2@$0A@@std@@@std@@IEAAXPEAU?$_Tree_node@U?$pair@$$CB_JV?$basic_string@DU?$char_traits@D@std@@V?$allocator@D@2@@std@@@std@@PEAX@2@@Z 000000014005db78     LoadXlsMsg.obj
 0002:00012b88       $chain$2$?_Erase@?$_Tree@V?$_Tmap_traits@_JV?$basic_string@DU?$char_traits@D@std@@V?$allocator@D@2@@std@@U?$less@_J@2@V?$allocator@U?$pair@$$CB_JV?$basic_string@DU?$char_traits@D@std@@V?$allocator@D@2@@std@@@std@@@2@$0A@@std@@@std@@IEAAXPEAU?$_Tree_node@U?$pair@$$CB_JV?$basic_string@DU?$char_traits@D@std@@V?$allocator@D@2@@std@@@std@@PEAX@2@@Z 000000014005db88     LoadXlsMsg.obj
 0002:00012b9c       $unwind$?erase@?$_Tree@V?$_Tmap_traits@_JV?$basic_string@DU?$char_traits@D@std@@V?$allocator@D@2@@std@@U?$less@_J@2@V?$allocator@U?$pair@$$CB_JV?$basic_string@DU?$char_traits@D@std@@V?$allocator@D@2@@std@@@std@@@2@$0A@@std@@@std@@QEAA?AV?$_Tree_iterator@V?$_Tree_val@U?$_Tree_simple_types@U?$pair@$$CB_JV?$basic_string@DU?$char_traits@D@std@@V?$allocator@D@2@@std@@@std@@@std@@@std@@@2@V?$_Tree_const_iterator@V?$_Tree_val@U?$_Tree_simple_types@U?$pair@$$CB_JV?$basic_string@DU?$char_traits@D@std@@V?$allocator@D@2@@std@@@std@@@std@@@std@@@2@0@Z 000000014005db9c     LoadXlsMsg.obj
 0002:00012bc0       $ip2state$?erase@?$_Tree@V?$_Tmap_traits@_JV?$basic_string@DU?$char_traits@D@std@@V?$allocator@D@2@@std@@U?$less@_J@2@V?$allocator@U?$pair@$$CB_JV?$basic_string@DU?$char_traits@D@std@@V?$allocator@D@2@@std@@@std@@@2@$0A@@std@@@std@@QEAA?AV?$_Tree_iterator@V?$_Tree_val@U?$_Tree_simple_types@U?$pair@$$CB_JV?$basic_string@DU?$char_traits@D@std@@V?$allocator@D@2@@std@@@std@@@std@@@std@@@2@V?$_Tree_const_iterator@V?$_Tree_val@U?$_Tree_simple_types@U?$pair@$$CB_JV?$basic_string@DU?$char_traits@D@std@@V?$allocator@D@2@@std@@@std@@@std@@@std@@@2@0@Z 000000014005dbc0     LoadXlsMsg.obj
 0002:00012bc8       $unwind$??$_Insert_hint@AEAU?$pair@$$CB_JV?$basic_string@DU?$char_traits@D@std@@V?$allocator@D@2@@std@@@std@@PEAU?$_Tree_node@U?$pair@$$CB_JV?$basic_string@DU?$char_traits@D@std@@V?$allocator@D@2@@std@@@std@@PEAX@2@@?$_Tree@V?$_Tmap_traits@_JV?$basic_string@DU?$char_traits@D@std@@V?$allocator@D@2@@std@@U?$less@_J@2@V?$allocator@U?$pair@$$CB_JV?$basic_string@DU?$char_traits@D@std@@V?$allocator@D@2@@std@@@std@@@2@$0A@@std@@@std@@IEAA?AV?$_Tree_iterator@V?$_Tree_val@U?$_Tree_simple_types@U?$pair@$$CB_JV?$basic_string@DU?$char_traits@D@std@@V?$allocator@D@2@@std@@@std@@@std@@@std@@@1@V?$_Tree_const_iterator@V?$_Tree_val@U?$_Tree_simple_types@U?$pair@$$CB_JV?$basic_string@DU?$char_traits@D@std@@V?$allocator@D@2@@std@@@std@@@std@@@std@@@1@AEAU?$pair@$$CB_JV?$basic_string@DU?$char_traits@D@std@@V?$allocator@D@2@@std@@@1@PEAU?$_Tree_node@U?$pair@$$CB_JV?$basic_string@DU?$char_traits@D@std@@V?$allocator@D@2@@std@@@std@@PEAX@1@@Z 000000014005dbc8     LoadXlsMsg.obj
 0002:00012be0       $tryMap$??$_Insert_hint@AEAU?$pair@$$CB_JV?$basic_string@DU?$char_traits@D@std@@V?$allocator@D@2@@std@@@std@@PEAU?$_Tree_node@U?$pair@$$CB_JV?$basic_string@DU?$char_traits@D@std@@V?$allocator@D@2@@std@@@std@@PEAX@2@@?$_Tree@V?$_Tmap_traits@_JV?$basic_string@DU?$char_traits@D@std@@V?$allocator@D@2@@std@@U?$less@_J@2@V?$allocator@U?$pair@$$CB_JV?$basic_string@DU?$char_traits@D@std@@V?$allocator@D@2@@std@@@std@@@2@$0A@@std@@@std@@IEAA?AV?$_Tree_iterator@V?$_Tree_val@U?$_Tree_simple_types@U?$pair@$$CB_JV?$basic_string@DU?$char_traits@D@std@@V?$allocator@D@2@@std@@@std@@@std@@@std@@@1@V?$_Tree_const_iterator@V?$_Tree_val@U?$_Tree_simple_types@U?$pair@$$CB_JV?$basic_string@DU?$char_traits@D@std@@V?$allocator@D@2@@std@@@std@@@std@@@std@@@1@AEAU?$pair@$$CB_JV?$basic_string@DU?$char_traits@D@std@@V?$allocator@D@2@@std@@@1@PEAU?$_Tree_node@U?$pair@$$CB_JV?$basic_string@DU?$char_traits@D@std@@V?$allocator@D@2@@std@@@std@@PEAX@1@@Z 000000014005dbe0     LoadXlsMsg.obj
 0002:00012bf4       $handlerMap$0$??$_Insert_hint@AEAU?$pair@$$CB_JV?$basic_string@DU?$char_traits@D@std@@V?$allocator@D@2@@std@@@std@@PEAU?$_Tree_node@U?$pair@$$CB_JV?$basic_string@DU?$char_traits@D@std@@V?$allocator@D@2@@std@@@std@@PEAX@2@@?$_Tree@V?$_Tmap_traits@_JV?$basic_string@DU?$char_traits@D@std@@V?$allocator@D@2@@std@@U?$less@_J@2@V?$allocator@U?$pair@$$CB_JV?$basic_string@DU?$char_traits@D@std@@V?$allocator@D@2@@std@@@std@@@2@$0A@@std@@@std@@IEAA?AV?$_Tree_iterator@V?$_Tree_val@U?$_Tree_simple_types@U?$pair@$$CB_JV?$basic_string@DU?$char_traits@D@std@@V?$allocator@D@2@@std@@@std@@@std@@@std@@@1@V?$_Tree_const_iterator@V?$_Tree_val@U?$_Tree_simple_types@U?$pair@$$CB_JV?$basic_string@DU?$char_traits@D@std@@V?$allocator@D@2@@std@@@std@@@std@@@std@@@1@AEAU?$pair@$$CB_JV?$basic_string@DU?$char_traits@D@std@@V?$allocator@D@2@@std@@@1@PEAU?$_Tree_node@U?$pair@$$CB_JV?$basic_string@DU?$char_traits@D@std@@V?$allocator@D@2@@std@@@std@@PEAX@1@@Z 000000014005dbf4     LoadXlsMsg.obj
 0002:00012c08       $ip2state$??$_Insert_hint@AEAU?$pair@$$CB_JV?$basic_string@DU?$char_traits@D@std@@V?$allocator@D@2@@std@@@std@@PEAU?$_Tree_node@U?$pair@$$CB_JV?$basic_string@DU?$char_traits@D@std@@V?$allocator@D@2@@std@@@std@@PEAX@2@@?$_Tree@V?$_Tmap_traits@_JV?$basic_string@DU?$char_traits@D@std@@V?$allocator@D@2@@std@@U?$less@_J@2@V?$allocator@U?$pair@$$CB_JV?$basic_string@DU?$char_traits@D@std@@V?$allocator@D@2@@std@@@std@@@2@$0A@@std@@@std@@IEAA?AV?$_Tree_iterator@V?$_Tree_val@U?$_Tree_simple_types@U?$pair@$$CB_JV?$basic_string@DU?$char_traits@D@std@@V?$allocator@D@2@@std@@@std@@@std@@@std@@@1@V?$_Tree_const_iterator@V?$_Tree_val@U?$_Tree_simple_types@U?$pair@$$CB_JV?$basic_string@DU?$char_traits@D@std@@V?$allocator@D@2@@std@@@std@@@std@@@std@@@1@AEAU?$pair@$$CB_JV?$basic_string@DU?$char_traits@D@std@@V?$allocator@D@2@@std@@@1@PEAU?$_Tree_node@U?$pair@$$CB_JV?$basic_string@DU?$char_traits@D@std@@V?$allocator@D@2@@std@@@std@@PEAX@1@@Z 000000014005dc08     LoadXlsMsg.obj
 0002:00012c28       $unwind$?catch$0@?0???$_Insert_hint@AEAU?$pair@$$CB_JV?$basic_string@DU?$char_traits@D@std@@V?$allocator@D@2@@std@@@std@@PEAU?$_Tree_node@U?$pair@$$CB_JV?$basic_string@DU?$char_traits@D@std@@V?$allocator@D@2@@std@@@std@@PEAX@2@@?$_Tree@V?$_Tmap_traits@_JV?$basic_string@DU?$char_traits@D@std@@V?$allocator@D@2@@std@@U?$less@_J@2@V?$allocator@U?$pair@$$CB_JV?$basic_string@DU?$char_traits@D@std@@V?$allocator@D@2@@std@@@std@@@2@$0A@@std@@@std@@IEAA?AV?$_Tree_iterator@V?$_Tree_val@U?$_Tree_simple_types@U?$pair@$$CB_JV?$basic_string@DU?$char_traits@D@std@@V?$allocator@D@2@@std@@@std@@@std@@@std@@@1@V?$_Tree_const_iterator@V?$_Tree_val@U?$_Tree_simple_types@U?$pair@$$CB_JV?$basic_string@DU?$char_traits@D@std@@V?$allocator@D@2@@std@@@std@@@std@@@std@@@1@AEAU?$pair@$$CB_JV?$basic_string@DU?$char_traits@D@std@@V?$allocator@D@2@@std@@@1@PEAU?$_Tree_node@U?$pair@$$CB_JV?$basic_string@DU?$char_traits@D@std@@V?$allocator@D@2@@std@@@std@@PEAX@1@@Z@4HA 000000014005dc28     LoadXlsMsg.obj
 0002:00012c38       $unwind$??$_Insert_nohint@AEAU?$pair@$$CB_JV?$basic_string@DU?$char_traits@D@std@@V?$allocator@D@2@@std@@@std@@PEAU?$_Tree_node@U?$pair@$$CB_JV?$basic_string@DU?$char_traits@D@std@@V?$allocator@D@2@@std@@@std@@PEAX@2@@?$_Tree@V?$_Tmap_traits@_JV?$basic_string@DU?$char_traits@D@std@@V?$allocator@D@2@@std@@U?$less@_J@2@V?$allocator@U?$pair@$$CB_JV?$basic_string@DU?$char_traits@D@std@@V?$allocator@D@2@@std@@@std@@@2@$0A@@std@@@std@@IEAA?AU?$pair@V?$_Tree_iterator@V?$_Tree_val@U?$_Tree_simple_types@U?$pair@$$CB_JV?$basic_string@DU?$char_traits@D@std@@V?$allocator@D@2@@std@@@std@@@std@@@std@@@std@@_N@1@_NAEAU?$pair@$$CB_JV?$basic_string@DU?$char_traits@D@std@@V?$allocator@D@2@@std@@@1@PEAU?$_Tree_node@U?$pair@$$CB_JV?$basic_string@DU?$char_traits@D@std@@V?$allocator@D@2@@std@@@std@@PEAX@1@@Z 000000014005dc38     LoadXlsMsg.obj
 0002:00012c54       $tryMap$??$_Insert_nohint@AEAU?$pair@$$CB_JV?$basic_string@DU?$char_traits@D@std@@V?$allocator@D@2@@std@@@std@@PEAU?$_Tree_node@U?$pair@$$CB_JV?$basic_string@DU?$char_traits@D@std@@V?$allocator@D@2@@std@@@std@@PEAX@2@@?$_Tree@V?$_Tmap_traits@_JV?$basic_string@DU?$char_traits@D@std@@V?$allocator@D@2@@std@@U?$less@_J@2@V?$allocator@U?$pair@$$CB_JV?$basic_string@DU?$char_traits@D@std@@V?$allocator@D@2@@std@@@std@@@2@$0A@@std@@@std@@IEAA?AU?$pair@V?$_Tree_iterator@V?$_Tree_val@U?$_Tree_simple_types@U?$pair@$$CB_JV?$basic_string@DU?$char_traits@D@std@@V?$allocator@D@2@@std@@@std@@@std@@@std@@@std@@_N@1@_NAEAU?$pair@$$CB_JV?$basic_string@DU?$char_traits@D@std@@V?$allocator@D@2@@std@@@1@PEAU?$_Tree_node@U?$pair@$$CB_JV?$basic_string@DU?$char_traits@D@std@@V?$allocator@D@2@@std@@@std@@PEAX@1@@Z 000000014005dc54     LoadXlsMsg.obj
 0002:00012c68       $handlerMap$0$??$_Insert_nohint@AEAU?$pair@$$CB_JV?$basic_string@DU?$char_traits@D@std@@V?$allocator@D@2@@std@@@std@@PEAU?$_Tree_node@U?$pair@$$CB_JV?$basic_string@DU?$char_traits@D@std@@V?$allocator@D@2@@std@@@std@@PEAX@2@@?$_Tree@V?$_Tmap_traits@_JV?$basic_string@DU?$char_traits@D@std@@V?$allocator@D@2@@std@@U?$less@_J@2@V?$allocator@U?$pair@$$CB_JV?$basic_string@DU?$char_traits@D@std@@V?$allocator@D@2@@std@@@std@@@2@$0A@@std@@@std@@IEAA?AU?$pair@V?$_Tree_iterator@V?$_Tree_val@U?$_Tree_simple_types@U?$pair@$$CB_JV?$basic_string@DU?$char_traits@D@std@@V?$allocator@D@2@@std@@@std@@@std@@@std@@@std@@_N@1@_NAEAU?$pair@$$CB_JV?$basic_string@DU?$char_traits@D@std@@V?$allocator@D@2@@std@@@1@PEAU?$_Tree_node@U?$pair@$$CB_JV?$basic_string@DU?$char_traits@D@std@@V?$allocator@D@2@@std@@@std@@PEAX@1@@Z 000000014005dc68     LoadXlsMsg.obj
 0002:00012c80       $ip2state$??$_Insert_nohint@AEAU?$pair@$$CB_JV?$basic_string@DU?$char_traits@D@std@@V?$allocator@D@2@@std@@@std@@PEAU?$_Tree_node@U?$pair@$$CB_JV?$basic_string@DU?$char_traits@D@std@@V?$allocator@D@2@@std@@@std@@PEAX@2@@?$_Tree@V?$_Tmap_traits@_JV?$basic_string@DU?$char_traits@D@std@@V?$allocator@D@2@@std@@U?$less@_J@2@V?$allocator@U?$pair@$$CB_JV?$basic_string@DU?$char_traits@D@std@@V?$allocator@D@2@@std@@@std@@@2@$0A@@std@@@std@@IEAA?AU?$pair@V?$_Tree_iterator@V?$_Tree_val@U?$_Tree_simple_types@U?$pair@$$CB_JV?$basic_string@DU?$char_traits@D@std@@V?$allocator@D@2@@std@@@std@@@std@@@std@@@std@@_N@1@_NAEAU?$pair@$$CB_JV?$basic_string@DU?$char_traits@D@std@@V?$allocator@D@2@@std@@@1@PEAU?$_Tree_node@U?$pair@$$CB_JV?$basic_string@DU?$char_traits@D@std@@V?$allocator@D@2@@std@@@std@@PEAX@1@@Z 000000014005dc80     LoadXlsMsg.obj
 0002:00012c90       $unwind$?catch$0@?0???$_Insert_nohint@AEAU?$pair@$$CB_JV?$basic_string@DU?$char_traits@D@std@@V?$allocator@D@2@@std@@@std@@PEAU?$_Tree_node@U?$pair@$$CB_JV?$basic_string@DU?$char_traits@D@std@@V?$allocator@D@2@@std@@@std@@PEAX@2@@?$_Tree@V?$_Tmap_traits@_JV?$basic_string@DU?$char_traits@D@std@@V?$allocator@D@2@@std@@U?$less@_J@2@V?$allocator@U?$pair@$$CB_JV?$basic_string@DU?$char_traits@D@std@@V?$allocator@D@2@@std@@@std@@@2@$0A@@std@@@std@@IEAA?AU?$pair@V?$_Tree_iterator@V?$_Tree_val@U?$_Tree_simple_types@U?$pair@$$CB_JV?$basic_string@DU?$char_traits@D@std@@V?$allocator@D@2@@std@@@std@@@std@@@std@@@std@@_N@1@_NAEAU?$pair@$$CB_JV?$basic_string@DU?$char_traits@D@std@@V?$allocator@D@2@@std@@@1@PEAU?$_Tree_node@U?$pair@$$CB_JV?$basic_string@DU?$char_traits@D@std@@V?$allocator@D@2@@std@@@std@@PEAX@1@@Z@4HA 000000014005dc90     LoadXlsMsg.obj
 0002:00012ca0       $unwind$?base64encode@jwsmtp@@YA?AV?$vector@DV?$allocator@D@std@@@std@@AEBV23@_N@Z 000000014005dca0     base6409cee8549d9fd00dfa06fdadc87a8424.obj
 0002:00012cc0       $stateUnwindMap$?base64encode@jwsmtp@@YA?AV?$vector@DV?$allocator@D@std@@@std@@AEBV23@_N@Z 000000014005dcc0     base6409cee8549d9fd00dfa06fdadc87a8424.obj
 0002:00012cc8       $ip2state$?base64encode@jwsmtp@@YA?AV?$vector@DV?$allocator@D@std@@@std@@AEBV23@_N@Z 000000014005dcc8     base6409cee8549d9fd00dfa06fdadc87a8424.obj
 0002:00012cd0       $unwind$?base64encode@jwsmtp@@YA?AV?$basic_string@DU?$char_traits@D@std@@V?$allocator@D@2@@std@@AEBV23@_N@Z 000000014005dcd0     base6409cee8549d9fd00dfa06fdadc87a8424.obj
 0002:00012cf0       $stateUnwindMap$?base64encode@jwsmtp@@YA?AV?$basic_string@DU?$char_traits@D@std@@V?$allocator@D@2@@std@@AEBV23@_N@Z 000000014005dcf0     base6409cee8549d9fd00dfa06fdadc87a8424.obj
 0002:00012d08       $ip2state$?base64encode@jwsmtp@@YA?AV?$basic_string@DU?$char_traits@D@std@@V?$allocator@D@2@@std@@AEBV23@_N@Z 000000014005dd08     base6409cee8549d9fd00dfa06fdadc87a8424.obj
 0002:00012d18       $unwind$?base64encode@jwsmtp@@YAXPEBDHPEAD_N@Z 000000014005dd18     base6409cee8549d9fd00dfa06fdadc87a8424.obj
 0002:00012d38       $stateUnwindMap$?base64encode@jwsmtp@@YAXPEBDHPEAD_N@Z 000000014005dd38     base6409cee8549d9fd00dfa06fdadc87a8424.obj
 0002:00012d48       $ip2state$?base64encode@jwsmtp@@YAXPEBDHPEAD_N@Z 000000014005dd48     base6409cee8549d9fd00dfa06fdadc87a8424.obj
 0002:00012d58       $unwind$?base64decode@jwsmtp@@YAXAEBV?$vector@DV?$allocator@D@std@@@std@@AEAV23@@Z 000000014005dd58     base6409cee8549d9fd00dfa06fdadc87a8424.obj
 0002:00012d78       $unwind$?MD5Final@MD5@@QEAAXQEAEPEAUMD5_CTX@@@Z 000000014005dd78     md55d7732e46e8b0b019ace15d3c50ded71.obj
 0002:00012d90       $unwind$?MD5Transform@MD5@@AEAAXQEAKQEAE@Z 000000014005dd90     md55d7732e46e8b0b019ace15d3c50ded71.obj
 0002:00012db4       $unwind$?sprintf_s@internal@cf@@YAHPEAD_KPEBDAEAPEAD@Z 000000014005ddb4     safe_string_x64:safe_string.obj
 0002:00012dd8       $stateUnwindMap$?sprintf_s@internal@cf@@YAHPEAD_KPEBDAEAPEAD@Z 000000014005ddd8     safe_string_x64:safe_string.obj
 0002:00012df8       $ip2state$?sprintf_s@internal@cf@@YAHPEAD_KPEBDAEAPEAD@Z 000000014005ddf8     safe_string_x64:safe_string.obj
 0002:00012e28       $unwind$?strcpy_s@cf@@YAHPEAD_KPEBD@Z 000000014005de28     safe_string_x64:safe_string.obj
 0002:00012e48       $stateUnwindMap$?strcpy_s@cf@@YAHPEAD_KPEBD@Z 000000014005de48     safe_string_x64:safe_string.obj
 0002:00012e48       $stateUnwindMap$?strncpy_s@cf@@YAHPEAD_KPEBD1@Z 000000014005de48     safe_string_x64:safe_string.obj
 0002:00012e68       $ip2state$?strcpy_s@cf@@YAHPEAD_KPEBD@Z 000000014005de68     safe_string_x64:safe_string.obj
 0002:00012e98       $unwind$?strncpy_s@cf@@YAHPEAD_KPEBD1@Z 000000014005de98     safe_string_x64:safe_string.obj
 0002:00012eb8       $ip2state$?strncpy_s@cf@@YAHPEAD_KPEBD1@Z 000000014005deb8     safe_string_x64:safe_string.obj
 0002:00012ee8       $unwind$?sprintf_s@cf@@YAHPEAD_KPEBDZZ 000000014005dee8     safe_string_x64:safe_string.obj
 0002:00012ef0       $unwind$??0?$basic_stringstream@DU?$char_traits@D@std@@V?$allocator@D@2@@std@@QEAA@H@Z 000000014005def0     safe_string_x64:safe_string.obj
 0002:00012f04       $stateUnwindMap$??0?$basic_stringstream@DU?$char_traits@D@std@@V?$allocator@D@2@@std@@QEAA@H@Z 000000014005df04     safe_string_x64:safe_string.obj
 0002:00012f18       $ip2state$??0?$basic_stringstream@DU?$char_traits@D@std@@V?$allocator@D@2@@std@@QEAA@H@Z 000000014005df18     safe_string_x64:safe_string.obj
 0002:00012f30       $unwind$?seekpos@?$basic_stringbuf@DU?$char_traits@D@std@@V?$allocator@D@2@@std@@MEAA?AV?$fpos@U_Mbstatet@@@2@V32@H@Z 000000014005df30     safe_string_x64:safe_string.obj
 0002:00012f44       $unwind$?seekoff@?$basic_stringbuf@DU?$char_traits@D@std@@V?$allocator@D@2@@std@@MEAA?AV?$fpos@U_Mbstatet@@@2@_JHH@Z 000000014005df44     safe_string_x64:safe_string.obj
 0002:00012f60       $xdatasym                  000000014005df60     msvcrt:amdsecgs.obj
 0002:00012f64       $unwind$?__scrt_initialize_thread_safe_statics@@YAHXZ 000000014005df64     msvcrt:thread_safe_statics.obj
 0002:00012f80       $ip2state$?__scrt_initialize_thread_safe_statics@@YAHXZ 000000014005df80     msvcrt:thread_safe_statics.obj
 0002:00012f88       $unwind$__scrt_is_nonwritable_in_current_image 000000014005df88     msvcrt:utility.obj
 0002:00012fa8       $unwind$__scrt_is_nonwritable_in_current_image$filt$0 000000014005dfa8     msvcrt:utility.obj
 0002:00012fb0       $unwind$__scrt_initialize_onexit_tables 000000014005dfb0     msvcrt:utility.obj
 0002:00012fb8       $unwind$??_L@YAXPEAX_K1P6AX0@Z2@Z 000000014005dfb8     msvcrt:ehvecctr.obj
 0002:00012fe4       $unwind$??_M@YAXPEAX_K1P6AX0@Z@Z 000000014005dfe4     msvcrt:ehvecdtr.obj
 0002:0001300c       $unwind$?__ArrayUnwind@@YAXPEAX_K1P6AX0@Z@Z 000000014005e00c     msvcrt:ehvecdtr.obj
 0002:00013038       $unwind$__report_securityfailure 000000014005e038     msvcrt:gs_report.obj
 0002:00013040       $unwind$__report_gsfailure 000000014005e040     msvcrt:gs_report.obj
 0002:00013048       $unwind$capture_current_context 000000014005e048     msvcrt:gs_report.obj
 0002:00013054       $unwind$capture_previous_context 000000014005e054     msvcrt:gs_report.obj
 0002:00013060       $unwind$?__scrt_common_main_seh@@YAHXZ 000000014005e060     msvcrt:exe_winmain.obj
 0002:00013094       $unwind$__scrt_get_show_window_mode 000000014005e094     msvcrt:utility_desktop.obj
 0002:0001309c       $unwind$__scrt_fastfail    000000014005e09c     msvcrt:utility_desktop.obj
 0002:000130ac       $unwind$__isa_available_init 000000014005e0ac     msvcrt:cpu_disp.obj
 0002:000130bc       $unwind$__security_init_cookie 000000014005e0bc     msvcrt:gs_support.obj
 0002:000130c8       $unwind$__GSHandlerCheckCommon 000000014005e0c8     msvcrt:gshandler.obj
 0002:000130d0       $xdatasym                  000000014005e0d0     msvcrt:guard_dispatch.obj
 0002:000130d4       $unwind$??1_Fac_tidy_reg_t@std@@QEAA@XZ 000000014005e0d4     msvcprt:locale0_implib.obj
 0002:000130e8       $ip2state$??1_Fac_tidy_reg_t@std@@QEAA@XZ 000000014005e0e8     msvcprt:locale0_implib.obj
 0002:000130f0       $unwind$__GSHandlerCheck_EH 000000014005e0f0     msvcrt:gshandlereh.obj
 0002:00013108       $xdatasym                  000000014005e108     msvcrt:chkstk.obj
 0002:000142d2       .idata$6                   000000014005f2d2     Psapi:PSAPI.DLL
 0002:000142dc       .idata$6                   000000014005f2dc     mfc140:mfc140.dll
 0002:000148ce       .idata$6                   000000014005f8ce     kernel32:KERNEL32.dll
 0002:0001498e       .idata$6                   000000014005f98e     user32:USER32.dll
 0002:00014a3a       .idata$6                   000000014005fa3a     advapi32:ADVAPI32.dll
 0002:00014a72       .idata$6                   000000014005fa72     shell32:SHELL32.dll
 0002:00014a90       .idata$6                   000000014005fa90     shlwapi:SHLWAPI.dll
 0002:00014f20       .idata$6                   000000014005ff20     msvcprt:MSVCP140.dll
 0002:00014fcc       .idata$6                   000000014005ffcc     DbgHelp:dbghelp.dll
 0002:00014fe6       .idata$6                   000000014005ffe6     winmm:WINMM.dll
 0002:000150a8       .idata$6                   00000001400600a8     winhttp:WINHTTP.dll
 0002:0001515a       .idata$6                   000000014006015a     ws2_32:WS2_32.dll
 0002:00015178       .idata$6                   0000000140060178     ipHlpapi:IPHLPAPI.DLL
 0002:00015236       .idata$6                   0000000140060236     vcruntime:VCRUNTIME140.dll
 0002:00015694       .idata$6                   0000000140060694     ucrt:api-ms-win-crt-runtime-l1-1-0.dll
 0002:000156b6       .idata$6                   00000001400606b6     ucrt:api-ms-win-crt-stdio-l1-1-0.dll
 0002:000156d6       .idata$6                   00000001400606d6     ucrt:api-ms-win-crt-filesystem-l1-1-0.dll
 0002:000156fc       .idata$6                   00000001400606fc     ucrt:api-ms-win-crt-string-l1-1-0.dll
 0002:0001571e       .idata$6                   000000014006071e     ucrt:api-ms-win-crt-convert-l1-1-0.dll
 0002:00015740       .idata$6                   0000000140060740     ucrt:api-ms-win-crt-time-l1-1-0.dll
 0002:00015760       .idata$6                   0000000140060760     ucrt:api-ms-win-crt-heap-l1-1-0.dll
 0002:00015780       .idata$6                   0000000140060780     ucrt:api-ms-win-crt-multibyte-l1-1-0.dll
 0002:000157a4       .idata$6                   00000001400607a4     ucrt:api-ms-win-crt-math-l1-1-0.dll
 0002:000157c4       .idata$6                   00000001400607c4     ucrt:api-ms-win-crt-locale-l1-1-0.dll
 0003:00000034       ?prefix@?1??uploadLOG@Uploader@crs@@AEAA_NAEAVHttpHandle@3@AEAU_SYSTEMTIME@@AEAVLogBuffer@3@@Z@4PADA 0000000140061034     crs_uploader.obj
 0003:00000188       ?version@?1??buildVersion@@9@9 0000000140061188     smbutil.obj
 0003:000004e0       ?base64_chars@@3V?$basic_string@DU?$char_traits@D@std@@V?$allocator@D@2@@std@@B 00000001400614e0     base64.obj
 0003:00001470       ?defVersion@?1??buildVersion@@9@9 0000000140062470     smbutil.obj
 0003:00001680       ?PADDING@@3PAEA            0000000140062680     md55d7732e46e8b0b019ace15d3c50ded71.obj
 0003:00001f58       ?_Tss_mutex@@3U_RTL_CRITICAL_SECTION@@A 0000000140062f58     msvcrt:thread_safe_statics.obj
 0003:00001f80       ?_Tss_cv@@3U_RTL_CONDITION_VARIABLE@@A 0000000140062f80     msvcrt:thread_safe_statics.obj
 0003:00001f88       ?_Tss_event@@3PEAXEA       0000000140062f88     msvcrt:thread_safe_statics.obj
 0003:00001f90       ?encoded_sleep_condition_variable_cs@@3P6AHPEAU_RTL_CONDITION_VARIABLE@@PEAU_RTL_CRITICAL_SECTION@@K@ZEA 0000000140062f90     msvcrt:thread_safe_statics.obj
 0003:00001f98       ?encoded_wake_all_condition_variable@@3P6AXPEAU_RTL_CONDITION_VARIABLE@@@ZEA 0000000140062f98     msvcrt:thread_safe_statics.obj
 0003:00001fb0       ?is_initialized_as_dll@@3_NA 0000000140062fb0     msvcrt:utility.obj
 0003:00001fb1       ?module_local_atexit_table_initialized@@3_NA 0000000140062fb1     msvcrt:utility.obj
 0003:00001fb8       ?module_local_atexit_table@@3U_onexit_table_t@@A 0000000140062fb8     msvcrt:utility.obj
 0003:00001fd0       ?module_local_at_quick_exit_table@@3U_onexit_table_t@@A 0000000140062fd0     msvcrt:utility.obj
 0003:00001ff0       GS_ExceptionRecord         0000000140062ff0     msvcrt:gs_report.obj
 0003:00002090       GS_ContextRecord           0000000140063090     msvcrt:gs_report.obj
 0003:000025e8       ?_Fac_tidy_reg@std@@3U_Fac_tidy_reg_t@1@B 00000001400635e8     msvcprt:locale0_implib.obj
 0003:000025f0       ?_Fac_head@std@@3PEAU_Fac_node@1@EA 00000001400635f0     msvcprt:locale0_implib.obj
 0003:00007d78       ?a@VectorSinConstantsSSE@@3MB 0000000140068d78     StdAfx.obj
 0003:00007d7c       ?RADIANS_PER_DEGREE@@3MB   0000000140068d7c     StdAfx.obj
 0003:00007d80       ?PiByTwo@GlobalVectorConstants@@3T__m128@@B 0000000140068d80     StdAfx.obj
 0003:00007d90       ?FloatMinusOneHalf@GlobalVectorConstants@@3T__m128@@B 0000000140068d90     StdAfx.obj
 0003:00007da0       ?IntAllMask@GlobalVectorConstants@@3T__m128i@@B 0000000140068da0     StdAfx.obj
 0003:00007db0       ?TwoPi@GlobalVectorConstants@@3T__m128@@B 0000000140068db0     StdAfx.obj
 0003:00007dc0       ?SmallLengthThreshold@GlobalVectorConstants@@3T__m128@@B 0000000140068dc0     StdAfx.obj
 0003:00007dd0       ?OneOverPi@GlobalVectorConstants@@3T__m128@@B 0000000140068dd0     StdAfx.obj
 0003:00007de0       ?AllMask@GlobalVectorConstants@@3T__m128@@B 0000000140068de0     StdAfx.obj
 0003:00007df0       ?ThreshQuatNormalized@GlobalVectorConstants@@3T__m128@@B 0000000140068df0     StdAfx.obj
 0003:00007e00       ?SignBit@GlobalVectorConstants@@3T__m128@@B 0000000140068e00     StdAfx.obj
 0003:00007e10       ?Float360@GlobalVectorConstants@@3T__m128@@B 0000000140068e10     StdAfx.obj
 0003:00007e20       ?QMULTI_SIGN_MASK0@GlobalVectorConstants@@3T__m128@@B 0000000140068e20     StdAfx.obj
 0003:00007e30       ?OneOverTwoPi@GlobalVectorConstants@@3T__m128@@B 0000000140068e30     StdAfx.obj
 0003:00007e40       ?DEG_TO_RAD@GlobalVectorConstants@@3T__m128@@B 0000000140068e40     StdAfx.obj
 0003:00007e50       ?BigNumber@GlobalVectorConstants@@3T__m128@@B 0000000140068e50     StdAfx.obj
 0003:00007e60       ?FloatOneHundredth@GlobalVectorConstants@@3T__m128@@B 0000000140068e60     StdAfx.obj
 0003:00007e70       ?FloatTwo@GlobalVectorConstants@@3T__m128@@B 0000000140068e70     StdAfx.obj
 0003:00007e80       ?Float0001@GlobalVectorConstants@@3T__m128@@B 0000000140068e80     StdAfx.obj
 0003:00007e90       ?FloatAlmostTwo@GlobalVectorConstants@@3T__m128@@B 0000000140068e90     StdAfx.obj
 0003:00007ea0       ?QMULTI_SIGN_MASK2@GlobalVectorConstants@@3T__m128@@B 0000000140068ea0     StdAfx.obj
 0003:00007eb0       ?SignMask@GlobalVectorConstants@@3T__m128@@B 0000000140068eb0     StdAfx.obj
 0003:00007ec0       ?FloatMinus1_111@GlobalVectorConstants@@3T__m128@@B 0000000140068ec0     StdAfx.obj
 0003:00007ed0       ?QMULTI_SIGN_MASK1@GlobalVectorConstants@@3T__m128@@B 0000000140068ed0     StdAfx.obj
 0003:00007ee0       ?IntMinusOne@GlobalVectorConstants@@3T__m128i@@B 0000000140068ee0     StdAfx.obj
 0003:00007ef0       ?FloatOneHalf@GlobalVectorConstants@@3T__m128@@B 0000000140068ef0     StdAfx.obj
 0003:00007f00       ?FloatZero@GlobalVectorConstants@@3T__m128@@B 0000000140068f00     StdAfx.obj
 0003:00007f10       ?B@VectorSinConstantsSSE@@3T__m128@@B 0000000140068f10     StdAfx.obj
 0003:00007f20       ?Float255@GlobalVectorConstants@@3T__m128@@B 0000000140068f20     StdAfx.obj
 0003:00007f30       ?Float127@GlobalVectorConstants@@3T__m128@@B 0000000140068f30     StdAfx.obj
 0003:00007f40       ?QINV_SIGN_MASK@GlobalVectorConstants@@3T__m128@@B 0000000140068f40     StdAfx.obj
 0003:00007f50       ?DEG_TO_RAD_HALF@GlobalVectorConstants@@3T__m128@@B 0000000140068f50     StdAfx.obj
 0003:00007f60       ?b@VectorSinConstantsSSE@@3MB 0000000140068f60     StdAfx.obj
 0003:00007f64       ?PI_3@@3MB                 0000000140068f64     StdAfx.obj
 0003:00007f68       ?DEGREES_PER_RADIAN@@3MB   0000000140068f68     StdAfx.obj
 0003:00007f6c       ?PI@@3MB                   0000000140068f6c     StdAfx.obj
 0003:00007f70       ?FloatOne@GlobalVectorConstants@@3T__m128@@B 0000000140068f70     StdAfx.obj
 0003:00007f80       ?A@VectorSinConstantsSSE@@3T__m128@@B 0000000140068f80     StdAfx.obj
 0003:00007f90       ?IntSignBit@GlobalVectorConstants@@3T__m128i@@B 0000000140068f90     StdAfx.obj
 0003:00007fa0       ?FloatMinusOne@GlobalVectorConstants@@3T__m128@@B 0000000140068fa0     StdAfx.obj
 0003:00007fb0       ?FloatNeg127@GlobalVectorConstants@@3T__m128@@B 0000000140068fb0     StdAfx.obj
 0003:00007fc0       ?Float111_Minus1@GlobalVectorConstants@@3T__m128@@B 0000000140068fc0     StdAfx.obj
 0003:00007fd0       ?XYZMask@GlobalVectorConstants@@3T__m128@@B 0000000140068fd0     StdAfx.obj
 0003:00007fe0       ?KindaSmallNumber@GlobalVectorConstants@@3T__m128@@B 0000000140068fe0     StdAfx.obj
 0003:00007ff0       ?IntOne@GlobalVectorConstants@@3T__m128i@@B 0000000140068ff0     StdAfx.obj
 0003:00008000       ?SmallNumber@GlobalVectorConstants@@3T__m128@@B 0000000140069000     StdAfx.obj
 0003:00008010       ?PiByFour@GlobalVectorConstants@@3T__m128@@B 0000000140069010     StdAfx.obj
 0003:00008020       ?Pi@GlobalVectorConstants@@3T__m128@@B 0000000140069020     StdAfx.obj
 0003:00008030       ?FloatInfinity@GlobalVectorConstants@@3T__m128@@B 0000000140069030     StdAfx.obj
 0003:00008040       ?IntZero@GlobalVectorConstants@@3T__m128i@@B 0000000140069040     StdAfx.obj
 0003:00008050       ?IntSignMask@GlobalVectorConstants@@3T__m128i@@B 0000000140069050     StdAfx.obj
 0003:00008060       ?RAD_TO_DEG@GlobalVectorConstants@@3T__m128@@B 0000000140069060     StdAfx.obj
 0003:00008070       ?PI_4@@3MB                 0000000140069070     StdAfx.obj
 0003:00008074       ?PI_2@@3MB                 0000000140069074     StdAfx.obj
 0003:00008090       ?Float180@GlobalVectorConstants@@3T__m128@@B 0000000140069090     StdAfx.obj
 0003:000080a0       ?g_szHostName@@3PADA       00000001400690a0     BugReporter.obj
 0003:00008110       ?g_szServerName@@3PADA     0000000140069110     BugReporter.obj
 0003:00008180       ?g_szDmpFolder@@3PADA      0000000140069180     BugReporter.obj
 0003:00008320       ?g_szDmpFileName@@3PADA    0000000140069320     BugReporter.obj
 0003:00008710       ?g_szSubDir@@3PADA         0000000140069710     BugReporter.obj
 0003:00008780       ?settingPath@@3PADA        0000000140069780     GameServerManagerDlg.obj
 0003:00008890       ?buffer@?7??ProcessSocketEvent@CClientLib@@QEAAXXZ@4PADA 0000000140069890     ClientLib.obj
 0003:00011090       ?dwVal@?8??OnTimer@CGameServerManagerDlg@@IEAAX_K@Z@4KA 0000000140072090     GameServerManagerDlg.obj
 0003:000110a0       ?count@?1??timerLogUser@CHostStat@@QEAAXHHHHH@Z@4HA 00000001400720a0     HostStat.obj
 0003:000110a4       ?count@?1??timerPerfMem@CHostStat@@QEAAXXZ@4HA 00000001400720a4     HostStat.obj
 0003:000110a8       ?count@?1??timerPerfCpu@CHostStat@@QEAAXXZ@4HA 00000001400720a8     HostStat.obj
 0003:000110b4       ?$TSS0@?1??Instance@DivisionPacketReceiver@@SAPEAV2@XZ@4HA 00000001400720b4     DivisionPacketReceiver.obj
 0003:000110b8       ?this_instance_@?1??Instance@DivisionPacketReceiver@@SAPEAV2@XZ@4V2@A 00000001400720b8     DivisionPacketReceiver.obj
 0003:000110c8       ?$TSS0@?1??CRSUploader@@YAAEAVUploader@crs@@XZ@4HA 00000001400720c8     BugReporter.obj
 0003:000110d0       ?crs_uploader@?1??CRSUploader@@YAAEAVUploader@crs@@XZ@4V23@A 00000001400720d0     BugReporter.obj
 0003:00011208       ?$TSS0@?1??initNetworking@jwsmtp@@YAXXZ@4HA 0000000140072208     compat.obj
 0003:0001120c       ?s@?1??initNetworking@jwsmtp@@YAXXZ@4Vsocks@?1??12@YAXXZ@A 000000014007220c     compat.obj
 0003:00011210       ?inalphabet@?1??base64decode@jwsmtp@@YAXAEBV?$vector@DV?$allocator@D@std@@@std@@AEAV34@@Z@4PADA 0000000140072210     base6409cee8549d9fd00dfa06fdadc87a8424.obj
 0003:00011310       ?decoder@?1??base64decode@jwsmtp@@YAXAEBV?$vector@DV?$allocator@D@std@@@std@@AEAV34@@Z@4PADA 0000000140072310     base6409cee8549d9fd00dfa06fdadc87a8424.obj
 0004:00000000       $pdata$??__EtheApp@@YAXXZ  0000000140073000     GameServerManager.obj
 0004:0000000c       $pdata$??__Eg_cServerLog@@YAXXZ 000000014007300c     GameServerManagerDlg.obj
 0004:00000018       $pdata$??__Ebase64_chars@@YAXXZ 0000000140073018     base64.obj
 0004:00000024       $pdata$??__Eg_HostStat@@YAXXZ 0000000140073024     HostStat.obj
 0004:00000030       $pdata$??__E?m_LogLock@CHLogger@@0VCMustSyncObjectLog@@A@@YAXXZ 0000000140073030     HostLogger.obj
 0004:0000003c       $pdata$??__E?m_LogPacketLock@CHLogger@@0VCMustSyncObjectLog@@A@@YAXXZ 000000014007303c     HostLogger.obj
 0004:00000048       $pdata$??__Ea@VectorSinConstantsSSE@@YAXXZ 0000000140073048     StdAfx.obj
 0004:00000054       $pdata$??__Eb@VectorSinConstantsSSE@@YAXXZ 0000000140073054     StdAfx.obj
 0004:00000060       $pdata$??__EPI@@YAXXZ      0000000140073060     StdAfx.obj
 0004:0000006c       $pdata$??__E__iob_func@@YAXXZ 000000014007306c     StdAfx.obj
 0004:00000078       $pdata$??__E_AtlBaseModule@ATL@@YAXXZ 0000000140073078     atls:atlbase.obj
 0004:00000084       $pdata$??__E_afxInitAppState@@YAXXZ 0000000140073084     mfcs140:appmodul.obj
 0004:00000090       $pdata$?AppendPacket@DivisionPacket@@AEAA?BW4DIVISION_PACKET_RESULT@@PEADG@Z 0000000140073090     DivisionPacket.obj
 0004:0000009c       $pdata$?_Tidy@?$vector@UPART_PACKET@@V?$allocator@UPART_PACKET@@@std@@@std@@AEAAXXZ 000000014007309c     DivisionPacket.obj
 0004:000000a8       $pdata$??$_Emplace_reallocate@AEBUPART_PACKET@@@?$vector@UPART_PACKET@@V?$allocator@UPART_PACKET@@@std@@@std@@QEAAPEAUPART_PACKET@@QEAU2@AEBU2@@Z 00000001400730a8     DivisionPacket.obj
 0004:000000b4       $pdata$3$??$_Emplace_reallocate@AEBUPART_PACKET@@@?$vector@UPART_PACKET@@V?$allocator@UPART_PACKET@@@std@@@std@@QEAAPEAUPART_PACKET@@QEAU2@AEBU2@@Z 00000001400730b4     DivisionPacket.obj
 0004:000000c0       $pdata$5$??$_Emplace_reallocate@AEBUPART_PACKET@@@?$vector@UPART_PACKET@@V?$allocator@UPART_PACKET@@@std@@@std@@QEAAPEAUPART_PACKET@@QEAU2@AEBU2@@Z 00000001400730c0     DivisionPacket.obj
 0004:000000cc       $pdata$6$??$_Emplace_reallocate@AEBUPART_PACKET@@@?$vector@UPART_PACKET@@V?$allocator@UPART_PACKET@@@std@@@std@@QEAAPEAUPART_PACKET@@QEAU2@AEBU2@@Z 00000001400730cc     DivisionPacket.obj
 0004:000000d8       $pdata$?_Xlength@?$vector@UPART_PACKET@@V?$allocator@UPART_PACKET@@@std@@@std@@CAXXZ 00000001400730d8     DivisionPacket.obj
 0004:000000d8       $pdata$?_Xlength@?$vector@DV?$allocator@D@std@@@std@@CAXXZ 00000001400730d8     mailer.obj
 0004:000000d8       $pdata$?_Xlength@?$vector@PEAXV?$allocator@PEAX@std@@@std@@CAXXZ 00000001400730d8     LogMsgManager.obj
 0004:000000d8       $pdata$?_Xlength@?$vector@U?$pair@UAddress@mailer@jwsmtp@@F@std@@V?$allocator@U?$pair@UAddress@mailer@jwsmtp@@F@std@@@2@@std@@CAXXZ 00000001400730d8     mailer.obj
 0004:000000d8       $pdata$?_Xlength@?$vector@USOCKADDR_IN@jwsmtp@@V?$allocator@USOCKADDR_IN@jwsmtp@@@std@@@std@@CAXXZ 00000001400730d8     mailer.obj
 0004:000000d8       $pdata$?_Xlength@?$vector@V?$basic_string@DU?$char_traits@D@std@@V?$allocator@D@2@@std@@V?$allocator@V?$basic_string@DU?$char_traits@D@std@@V?$allocator@D@2@@std@@@2@@std@@CAXXZ 00000001400730d8     CSmtp.obj
 0004:000000e4       $pdata$memcpy_s            00000001400730e4     DivisionPacket.obj
 0004:000000f0       $pdata$?Instance@DivisionPacketReceiver@@SAPEAV1@XZ 00000001400730f0     DivisionPacketReceiver.obj
 0004:000000fc       $pdata$?GetPacketBuffer@DivisionPacketReceiver@@QEAA?BW4DIVISION_PACKET_RESULT@@EEEEEPEADG0H@Z 00000001400730fc     DivisionPacketReceiver.obj
 0004:00000108       $pdata$?_Buyheadnode@?$_Tree_comp_alloc@V?$_Tmap_traits@_JVDivisionPacket@@U?$less@_J@std@@V?$allocator@U?$pair@$$CB_JVDivisionPacket@@@std@@@3@$0A@@std@@@std@@QEAAPEAU?$_Tree_node@U?$pair@$$CB_JVDivisionPacket@@@std@@PEAX@2@XZ 0000000140073108     DivisionPacketReceiver.obj
 0004:00000114       $pdata$?_Erase@?$_Tree@V?$_Tmap_traits@_JVDivisionPacket@@U?$less@_J@std@@V?$allocator@U?$pair@$$CB_JVDivisionPacket@@@std@@@3@$0A@@std@@@std@@IEAAXPEAU?$_Tree_node@U?$pair@$$CB_JVDivisionPacket@@@std@@PEAX@2@@Z 0000000140073114     DivisionPacketReceiver.obj
 0004:00000120       $pdata$??0?$vector@UPART_PACKET@@V?$allocator@UPART_PACKET@@@std@@@std@@QEAA@AEBV01@@Z 0000000140073120     DivisionPacketReceiver.obj
 0004:0000012c       $pdata$0$??0?$vector@UPART_PACKET@@V?$allocator@UPART_PACKET@@@std@@@std@@QEAA@AEBV01@@Z 000000014007312c     DivisionPacketReceiver.obj
 0004:00000138       $pdata$1$??0?$vector@UPART_PACKET@@V?$allocator@UPART_PACKET@@@std@@@std@@QEAA@AEBV01@@Z 0000000140073138     DivisionPacketReceiver.obj
 0004:00000144       $pdata$??$_Buynode@U?$pair@_JVDivisionPacket@@@std@@@?$_Tree_comp_alloc@V?$_Tmap_traits@_JVDivisionPacket@@U?$less@_J@std@@V?$allocator@U?$pair@$$CB_JVDivisionPacket@@@std@@@3@$0A@@std@@@std@@QEAAPEAU?$_Tree_node@U?$pair@$$CB_JVDivisionPacket@@@std@@PEAX@1@$$QEAU?$pair@_JVDivisionPacket@@@1@@Z 0000000140073144     DivisionPacketReceiver.obj
 0004:00000150       $pdata$??$_Insert_nohint@AEAU?$pair@$$CB_JVDivisionPacket@@@std@@PEAU?$_Tree_node@U?$pair@$$CB_JVDivisionPacket@@@std@@PEAX@2@@?$_Tree@V?$_Tmap_traits@_JVDivisionPacket@@U?$less@_J@std@@V?$allocator@U?$pair@$$CB_JVDivisionPacket@@@std@@@3@$0A@@std@@@std@@IEAA?AU?$pair@V?$_Tree_iterator@V?$_Tree_val@U?$_Tree_simple_types@U?$pair@$$CB_JVDivisionPacket@@@std@@@std@@@std@@@std@@_N@1@_NAEAU?$pair@$$CB_JVDivisionPacket@@@1@PEAU?$_Tree_node@U?$pair@$$CB_JVDivisionPacket@@@std@@PEAX@1@@Z 0000000140073150     DivisionPacketReceiver.obj
 0004:0000015c       $pdata$?_Buynode0@?$_Tree_comp_alloc@V?$_Tmap_traits@_JVDivisionPacket@@U?$less@_J@std@@V?$allocator@U?$pair@$$CB_JVDivisionPacket@@@std@@@3@$0A@@std@@@std@@QEAAPEAU?$_Tree_node@U?$pair@$$CB_JVDivisionPacket@@@std@@PEAX@2@XZ 000000014007315c     DivisionPacketReceiver.obj
 0004:00000168       $pdata$?_Destroy_if_node@?$_Tree@V?$_Tmap_traits@_JVDivisionPacket@@U?$less@_J@std@@V?$allocator@U?$pair@$$CB_JVDivisionPacket@@@std@@@3@$0A@@std@@@std@@IEAAXPEAU?$_Tree_node@U?$pair@$$CB_JVDivisionPacket@@@std@@PEAX@2@@Z 0000000140073168     DivisionPacketReceiver.obj
 0004:00000174       $pdata$??$_Insert_at@AEAU?$pair@$$CB_JVDivisionPacket@@@std@@PEAU?$_Tree_node@U?$pair@$$CB_JVDivisionPacket@@@std@@PEAX@2@@?$_Tree@V?$_Tmap_traits@_JVDivisionPacket@@U?$less@_J@std@@V?$allocator@U?$pair@$$CB_JVDivisionPacket@@@std@@@3@$0A@@std@@@std@@IEAA?AV?$_Tree_iterator@V?$_Tree_val@U?$_Tree_simple_types@U?$pair@$$CB_JVDivisionPacket@@@std@@@std@@@std@@@1@_NPEAU?$_Tree_node@U?$pair@$$CB_JVDivisionPacket@@@std@@PEAX@1@AEAU?$pair@$$CB_JVDivisionPacket@@@1@1@Z 0000000140073174     DivisionPacketReceiver.obj
 0004:00000180       $pdata$?CRSUploader@@YAAEAVUploader@crs@@XZ 0000000140073180     BugReporter.obj
 0004:0000018c       $pdata$?threadCreateDumpFile@@YAKPEAX@Z 000000014007318c     BugReporter.obj
 0004:00000198       $pdata$?CrashExceptionDump@@YAJPEAU_EXCEPTION_POINTERS@@@Z 0000000140073198     BugReporter.obj
 0004:000001a4       $pdata$0$?CrashExceptionDump@@YAJPEAU_EXCEPTION_POINTERS@@@Z 00000001400731a4     BugReporter.obj
 0004:000001b0       $pdata$1$?CrashExceptionDump@@YAJPEAU_EXCEPTION_POINTERS@@@Z 00000001400731b0     BugReporter.obj
 0004:000001bc       $pdata$?InitBugReporter@@YAXPEAD0000@Z 00000001400731bc     BugReporter.obj
 0004:000001c8       $pdata$??$sprintf_s@$0BAA@@cf@@YAHAEAY0BAA@DPEBDZZ 00000001400731c8     BugReporter.obj
 0004:000001d4       $pdata$??$sprintf_s@$0BJB@@cf@@YAHAEAY0BJB@DPEBDZZ 00000001400731d4     BugReporter.obj
 0004:000001e0       $pdata$??$sprintf_s@$0BE@@cf@@YAHAEAY0BE@DPEBDZZ 00000001400731e0     BugReporter.obj
 0004:000001ec       $pdata$??$sprintf_s@$0DOJ@@cf@@YAHAEAY0DOJ@DPEBDZZ 00000001400731ec     BugReporter.obj
 0004:000001f8       $pdata$??$sprintf_s@$0BAE@@cf@@YAHAEAY0BAE@DPEBDZZ 00000001400731f8     BugReporter.obj
 0004:00000204       $pdata$??1?$basic_string@DU?$char_traits@D@std@@V?$allocator@D@2@@std@@QEAA@XZ 0000000140073204     BugReporter.obj
 0004:00000204       $pdata$?_Tidy_deallocate@?$basic_string@DU?$char_traits@D@std@@V?$allocator@D@2@@std@@QEAAXXZ 0000000140073204     BugReporter.obj
 0004:00000210       $pdata$?_Xlen@?$basic_string@DU?$char_traits@D@std@@V?$allocator@D@2@@std@@SAXXZ 0000000140073210     BugReporter.obj
 0004:00000210       $pdata$?_Xlen@?$basic_string@_WU?$char_traits@_W@std@@V?$allocator@_W@2@@std@@SAXXZ 0000000140073210     crs_uploader.obj
 0004:0000021c       $pdata$?assign@?$basic_string@DU?$char_traits@D@std@@V?$allocator@D@2@@std@@QEAAAEAV12@QEBD_K@Z 000000014007321c     BugReporter.obj
 0004:00000228       $pdata$0$?assign@?$basic_string@DU?$char_traits@D@std@@V?$allocator@D@2@@std@@QEAAAEAV12@QEBD_K@Z 0000000140073228     BugReporter.obj
 0004:00000234       $pdata$1$?assign@?$basic_string@DU?$char_traits@D@std@@V?$allocator@D@2@@std@@QEAAAEAV12@QEBD_K@Z 0000000140073234     BugReporter.obj
 0004:00000240       $pdata$2$?assign@?$basic_string@DU?$char_traits@D@std@@V?$allocator@D@2@@std@@QEAAAEAV12@QEBD_K@Z 0000000140073240     BugReporter.obj
 0004:0000024c       $pdata$3$?assign@?$basic_string@DU?$char_traits@D@std@@V?$allocator@D@2@@std@@QEAAAEAV12@QEBD_K@Z 000000014007324c     BugReporter.obj
 0004:00000258       $pdata$??0?$basic_string@DU?$char_traits@D@std@@V?$allocator@D@2@@std@@QEAA@QEBD@Z 0000000140073258     BugReporter.obj
 0004:00000264       $pdata$_snprintf_s         0000000140073264     BugReporter.obj
 0004:00000270       $pdata$?recordExceptionLog@Uploader@crs@@QEAAXAEAVLogBuffer@2@PEBDZZ 0000000140073270     crs_uploader.obj
 0004:0000027c       $pdata$0$?recordExceptionLog@Uploader@crs@@QEAAXAEAVLogBuffer@2@PEBDZZ 000000014007327c     crs_uploader.obj
 0004:00000288       $pdata$1$?recordExceptionLog@Uploader@crs@@QEAAXAEAVLogBuffer@2@PEBDZZ 0000000140073288     crs_uploader.obj
 0004:00000294       $pdata$?readURL@Uploader@crs@@AEAAXAEAV?$basic_string@_WU?$char_traits@_W@std@@V?$allocator@_W@2@@std@@@Z 0000000140073294     crs_uploader.obj
 0004:000002a0       $pdata$?iniPath@Uploader@crs@@AEAA?AV?$basic_string@_WU?$char_traits@_W@std@@V?$allocator@_W@2@@std@@AEBV34@@Z 00000001400732a0     crs_uploader.obj
 0004:000002ac       $pdata$1$?iniPath@Uploader@crs@@AEAA?AV?$basic_string@_WU?$char_traits@_W@std@@V?$allocator@_W@2@@std@@AEBV34@@Z 00000001400732ac     crs_uploader.obj
 0004:000002b8       $pdata$2$?iniPath@Uploader@crs@@AEAA?AV?$basic_string@_WU?$char_traits@_W@std@@V?$allocator@_W@2@@std@@AEBV34@@Z 00000001400732b8     crs_uploader.obj
 0004:000002c4       $pdata$?makeBaseInfo@Uploader@crs@@AEAAXPEAD0@Z 00000001400732c4     crs_uploader.obj
 0004:000002d0       $pdata$?error@Uploader@crs@@AEAA_NPEBDZZ 00000001400732d0     crs_uploader.obj
 0004:000002dc       $pdata$??1Uploader@crs@@QEAA@XZ 00000001400732dc     crs_uploader.obj
 0004:000002e8       $pdata$?init@Uploader@crs@@QEAA_N_NPEAD1@Z 00000001400732e8     crs_uploader.obj
 0004:000002f4       $pdata$?upload@Uploader@crs@@QEAA_N_NAEBV?$basic_string@DU?$char_traits@D@std@@V?$allocator@D@2@@std@@AEAVLogBuffer@2@@Z 00000001400732f4     crs_uploader.obj
 0004:00000300       $pdata$?makeExceptionLog@Uploader@crs@@QEAAXPEAU_EXCEPTION_POINTERS@@AEAVLogBuffer@2@@Z 0000000140073300     crs_uploader.obj
 0004:0000030c       $pdata$3$?makeExceptionLog@Uploader@crs@@QEAAXPEAU_EXCEPTION_POINTERS@@AEAVLogBuffer@2@@Z 000000014007330c     crs_uploader.obj
 0004:00000318       $pdata$4$?makeExceptionLog@Uploader@crs@@QEAAXPEAU_EXCEPTION_POINTERS@@AEAVLogBuffer@2@@Z 0000000140073318     crs_uploader.obj
 0004:00000324       $pdata$?EnumModuleDetail@ModuleInfo@?1??makeExceptionLog@Uploader@crs@@QEAAXPEAU_EXCEPTION_POINTERS@@AEAVLogBuffer@4@@Z@SAHPEBD_KKPEAX@Z 0000000140073324     crs_uploader.obj
 0004:00000330       $pdata$0$?EnumModuleDetail@ModuleInfo@?1??makeExceptionLog@Uploader@crs@@QEAAXPEAU_EXCEPTION_POINTERS@@AEAVLogBuffer@4@@Z@SAHPEBD_KKPEAX@Z 0000000140073330     crs_uploader.obj
 0004:0000033c       $pdata$1$?EnumModuleDetail@ModuleInfo@?1??makeExceptionLog@Uploader@crs@@QEAAXPEAU_EXCEPTION_POINTERS@@AEAVLogBuffer@4@@Z@SAHPEBD_KKPEAX@Z 000000014007333c     crs_uploader.obj
 0004:00000348       $pdata$?prepare@Uploader@crs@@AEAA_NAEAVHttpHandles@2@@Z 0000000140073348     crs_uploader.obj
 0004:00000354       $pdata$?uploadHTTP@Uploader@crs@@AEAA_NAEAVHttpHandle@2@PEBDPEB_W2@Z 0000000140073354     crs_uploader.obj
 0004:00000360       $pdata$?uploadLOG@Uploader@crs@@AEAA_NAEAVHttpHandle@2@AEAU_SYSTEMTIME@@AEAVLogBuffer@2@@Z 0000000140073360     crs_uploader.obj
 0004:0000036c       $pdata$0$?uploadLOG@Uploader@crs@@AEAA_NAEAVHttpHandle@2@AEAU_SYSTEMTIME@@AEAVLogBuffer@2@@Z 000000014007336c     crs_uploader.obj
 0004:00000378       $pdata$1$?uploadLOG@Uploader@crs@@AEAA_NAEAVHttpHandle@2@AEAU_SYSTEMTIME@@AEAVLogBuffer@2@@Z 0000000140073378     crs_uploader.obj
 0004:00000384       $pdata$2$?uploadLOG@Uploader@crs@@AEAA_NAEAVHttpHandle@2@AEAU_SYSTEMTIME@@AEAVLogBuffer@2@@Z 0000000140073384     crs_uploader.obj
 0004:00000390       $pdata$3$?uploadLOG@Uploader@crs@@AEAA_NAEAVHttpHandle@2@AEAU_SYSTEMTIME@@AEAVLogBuffer@2@@Z 0000000140073390     crs_uploader.obj
 0004:0000039c       $pdata$?success@Uploader@crs@@AEAA_NPEBDAEAVHttpHandle@2@@Z 000000014007339c     crs_uploader.obj
 0004:000003a8       $pdata$??1?$auto_ptr@VUrl@crs@@@std@@QEAA@XZ 00000001400733a8     crs_uploader.obj
 0004:000003b4       $pdata$0$??1?$auto_ptr@VUrl@crs@@@std@@QEAA@XZ 00000001400733b4     crs_uploader.obj
 0004:000003c0       $pdata$1$??1?$auto_ptr@VUrl@crs@@@std@@QEAA@XZ 00000001400733c0     crs_uploader.obj
 0004:000003cc       $pdata$2$??1?$auto_ptr@VUrl@crs@@@std@@QEAA@XZ 00000001400733cc     crs_uploader.obj
 0004:000003d8       $pdata$??$_snprintf_s@$0IA@@@YAHAEAY0IA@D_KPEBDZZ 00000001400733d8     crs_uploader.obj
 0004:000003e4       $pdata$??$_Reallocate_grow_by@V<lambda_1dfe18491bcca09701d8ccb01d0b0af4>@@PEB_W_K@?$basic_string@_WU?$char_traits@_W@std@@V?$allocator@_W@2@@std@@QEAAAEAV01@_KV<lambda_1dfe18491bcca09701d8ccb01d0b0af4>@@PEB_W_K@Z 00000001400733e4     crs_uploader.obj
 0004:000003f0       $pdata$3$??$_Reallocate_grow_by@V<lambda_1dfe18491bcca09701d8ccb01d0b0af4>@@PEB_W_K@?$basic_string@_WU?$char_traits@_W@std@@V?$allocator@_W@2@@std@@QEAAAEAV01@_KV<lambda_1dfe18491bcca09701d8ccb01d0b0af4>@@PEB_W_K@Z 00000001400733f0     crs_uploader.obj
 0004:000003fc       $pdata$4$??$_Reallocate_grow_by@V<lambda_1dfe18491bcca09701d8ccb01d0b0af4>@@PEB_W_K@?$basic_string@_WU?$char_traits@_W@std@@V?$allocator@_W@2@@std@@QEAAAEAV01@_KV<lambda_1dfe18491bcca09701d8ccb01d0b0af4>@@PEB_W_K@Z 00000001400733fc     crs_uploader.obj
 0004:00000408       $pdata$?append@?$basic_string@_WU?$char_traits@_W@std@@V?$allocator@_W@2@@std@@QEAAAEAV12@QEB_W_K@Z 0000000140073408     crs_uploader.obj
 0004:00000414       $pdata$1$?append@?$basic_string@_WU?$char_traits@_W@std@@V?$allocator@_W@2@@std@@QEAAAEAV12@QEB_W_K@Z 0000000140073414     crs_uploader.obj
 0004:00000420       $pdata$2$?append@?$basic_string@_WU?$char_traits@_W@std@@V?$allocator@_W@2@@std@@QEAAAEAV12@QEB_W_K@Z 0000000140073420     crs_uploader.obj
 0004:0000042c       $pdata$_snwprintf_s        000000014007342c     crs_uploader.obj
 0004:00000438       $pdata$??1?$basic_string@_WU?$char_traits@_W@std@@V?$allocator@_W@2@@std@@QEAA@XZ 0000000140073438     crs_uploader.obj
 0004:00000438       $pdata$?_Tidy_deallocate@?$basic_string@_WU?$char_traits@_W@std@@V?$allocator@_W@2@@std@@QEAAXXZ 0000000140073438     crs_uploader.obj
 0004:00000444       $pdata$?assign@?$basic_string@_WU?$char_traits@_W@std@@V?$allocator@_W@2@@std@@QEAAAEAV12@QEB_W_K@Z 0000000140073444     crs_uploader.obj
 0004:00000450       $pdata$??_GCServerLog@@UEAAPEAXI@Z 0000000140073450     LogMgmt.obj
 0004:0000045c       $pdata$??1CServerLog@@UEAA@XZ 000000014007345c     LogMgmt.obj
 0004:00000468       $pdata$?LOG_MAILER@CServerLog@@QEAAXHPEBD@Z 0000000140073468     LogMgmt.obj
 0004:00000474       $pdata$0$?LOG_MAILER@CServerLog@@QEAAXHPEBD@Z 0000000140073474     LogMgmt.obj
 0004:00000480       $pdata$1$?LOG_MAILER@CServerLog@@QEAAXHPEBD@Z 0000000140073480     LogMgmt.obj
 0004:0000048c       $pdata$fprintf             000000014007348c     LogMgmt.obj
 0004:00000498       $pdata$sprintf             0000000140073498     LogMgmt.obj
 0004:000004a4       $pdata$?Log@rwpmlog@@YAXPEBDFPEBUGAMEPROTO_SC_REMOVECLIENT@@@Z 00000001400734a4     RWPMLog.obj
 0004:000004b0       $pdata$?Log@rwpmlog@@YAXPEBDFPEBUGAMEPROTO_SS_GAMEEND@@@Z 00000001400734b0     RWPMLog.obj
 0004:000004bc       $pdata$?Log@rwpmlog@@YAXPEBDFPEBUGAMEPROTO_SC_HOST_USER_STAT@@@Z 00000001400734bc     RWPMLog.obj
 0004:000004c8       $pdata$?Log@rwpmlog@@YAXPEBDFPEBUCLANSTATREPORTDATA@@@Z 00000001400734c8     RWPMLog.obj
 0004:000004d4       $pdata$?Log@rwpmlog@@YAXPEBDFPEBUGAMEPROTO_SC_HOST_STAT@@@Z 00000001400734d4     RWPMLog.obj
 0004:000004e0       $pdata$?Log@rwpmlog@@YAXPEBDFPEBUPROTO_GAMEGT_INGAME_AIGACHA_ITEM_INSERT@@@Z 00000001400734e0     RWPMLog.obj
 0004:000004ec       $pdata$0$?Log@rwpmlog@@YAXPEBDFPEBUPROTO_GAMEGT_INGAME_AIGACHA_ITEM_INSERT@@@Z 00000001400734ec     RWPMLog.obj
 0004:000004f8       $pdata$1$?Log@rwpmlog@@YAXPEBDFPEBUPROTO_GAMEGT_INGAME_AIGACHA_ITEM_INSERT@@@Z 00000001400734f8     RWPMLog.obj
 0004:00000504       $pdata$?Log@rwpmlog@@YAXPEBDFPEBUPROTO_SPEC_RECOMMENDROOM_INGAME_DATA@@@Z 0000000140073504     RWPMLog.obj
 0004:00000510       $pdata$?Log@rwpmlog@@YAXPEBDFPEBUPROTO_GAMEGT_AUTO_SIDE_CHANGE_TEAM_INFO_NTY@@@Z 0000000140073510     RWPMLog.obj
 0004:0000051c       $pdata$??$sprintf_s@$0EA@@cf@@YAHAEAY0EA@DPEBDZZ 000000014007351c     RWPMLog.obj
 0004:00000528       $pdata$??_GCReceiver@@UEAAPEAXI@Z 0000000140073528     SGGMCallBackObj.obj
 0004:00000534       $pdata$??_GCSGGMCallBackObj@@UEAAPEAXI@Z 0000000140073534     SGGMCallBackObj.obj
 0004:00000540       $pdata$??_GMultiReceiver@sggm_proxy@@UEAAPEAXI@Z 0000000140073540     SGGMCallBackObj.obj
 0004:0000054c       $pdata$?GetSendParam@SendBuffer@@QEAAHPEAPEAEAEAH@Z 000000014007354c     ClientLib.obj
 0004:00000558       $pdata$0$?GetSendParam@SendBuffer@@QEAAHPEAPEAEAEAH@Z 0000000140073558     ClientLib.obj
 0004:00000564       $pdata$1$?GetSendParam@SendBuffer@@QEAAHPEAPEAEAEAH@Z 0000000140073564     ClientLib.obj
 0004:00000570       $pdata$?Write@SendBuffer@@QEAAHPEAEG@Z 0000000140073570     ClientLib.obj
 0004:0000057c       $pdata$0$?Write@SendBuffer@@QEAAHPEAEG@Z 000000014007357c     ClientLib.obj
 0004:00000588       $pdata$1$?Write@SendBuffer@@QEAAHPEAEG@Z 0000000140073588     ClientLib.obj
 0004:00000594       $pdata$??_GSendBuffer@@UEAAPEAXI@Z 0000000140073594     ClientLib.obj
 0004:000005a0       $pdata$??_GCClientLib@@UEAAPEAXI@Z 00000001400735a0     ClientLib.obj
 0004:000005ac       $pdata$?CloseSocket@CClientLib@@MEAAHXZ 00000001400735ac     ClientLib.obj
 0004:000005b8       $pdata$?ProcessSend@CClientLib@@QEAAHXZ 00000001400735b8     ClientLib.obj
 0004:000005c4       $pdata$0$?ProcessSend@CClientLib@@QEAAHXZ 00000001400735c4     ClientLib.obj
 0004:000005d0       $pdata$3$?ProcessSend@CClientLib@@QEAAHXZ 00000001400735d0     ClientLib.obj
 0004:000005dc       $pdata$4$?ProcessSend@CClientLib@@QEAAHXZ 00000001400735dc     ClientLib.obj
 0004:000005e8       $pdata$5$?ProcessSend@CClientLib@@QEAAHXZ 00000001400735e8     ClientLib.obj
 0004:000005f4       $pdata$?CopySendBuffer@CClientLib@@QEAAHPEAVSendBuffer@@@Z 00000001400735f4     ClientLib.obj
 0004:00000600       $pdata$2$?CopySendBuffer@CClientLib@@QEAAHPEAVSendBuffer@@@Z 0000000140073600     ClientLib.obj
 0004:0000060c       $pdata$3$?CopySendBuffer@CClientLib@@QEAAHPEAVSendBuffer@@@Z 000000014007360c     ClientLib.obj
 0004:00000618       $pdata$?ProcessSocketEvent@CClientLib@@QEAAXXZ 0000000140073618     ClientLib.obj
 0004:00000624       $pdata$??_G?$CircuitQueue@E@@UEAAPEAXI@Z 0000000140073624     ClientLib.obj
 0004:00000630       $pdata$??_GCPacket@@UEAAPEAXI@Z 0000000140073630     Packet.obj
 0004:0000063c       $pdata$?CopyFromUserDataArea@CPacket@@QEAAHPEAXK@Z 000000014007363c     Packet.obj
 0004:00000648       $pdata$3$?CopyFromUserDataArea@CPacket@@QEAAHPEAXK@Z 0000000140073648     Packet.obj
 0004:00000654       $pdata$4$?CopyFromUserDataArea@CPacket@@QEAAHPEAXK@Z 0000000140073654     Packet.obj
 0004:00000660       $pdata$??0CSFGameServerClientLib@@QEAA@XZ 0000000140073660     SFGameServerClientLib.obj
 0004:0000066c       $pdata$??1CSFGameServerClientLib@@UEAA@XZ 000000014007366c     SFGameServerClientLib.obj
 0004:00000678       $pdata$?Connect@CSFGameServerClientLib@@QEAAHH@Z 0000000140073678     SFGameServerClientLib.obj
 0004:00000684       $pdata$?CloseSocket@CSFGameServerClientLib@@UEAAHXZ 0000000140073684     SFGameServerClientLib.obj
 0004:00000690       $pdata$?ReadData@GAMEPROTO_SC_HOST_STAT@@UEAA_NPEAVILTMessage_Read@@@Z 0000000140073690     AppInfoDlg.obj
 0004:0000069c       $pdata$?WriteData@GAMEPROTO_SC_HOST_STAT@@UEAA_NPEAVILTMessage_Write@@@Z 000000014007369c     AppInfoDlg.obj
 0004:000006a8       $pdata$?ReadData@GAMEPROTO_SC_HOST_USER_STAT@@UEAA_NPEAVILTMessage_Read@@@Z 00000001400736a8     AppInfoDlg.obj
 0004:000006b4       $pdata$2$?ReadData@GAMEPROTO_SC_HOST_USER_STAT@@UEAA_NPEAVILTMessage_Read@@@Z 00000001400736b4     AppInfoDlg.obj
 0004:000006c0       $pdata$3$?ReadData@GAMEPROTO_SC_HOST_USER_STAT@@UEAA_NPEAVILTMessage_Read@@@Z 00000001400736c0     AppInfoDlg.obj
 0004:000006cc       $pdata$4$?ReadData@GAMEPROTO_SC_HOST_USER_STAT@@UEAA_NPEAVILTMessage_Read@@@Z 00000001400736cc     AppInfoDlg.obj
 0004:000006d8       $pdata$5$?ReadData@GAMEPROTO_SC_HOST_USER_STAT@@UEAA_NPEAVILTMessage_Read@@@Z 00000001400736d8     AppInfoDlg.obj
 0004:000006e4       $pdata$?WriteData@GAMEPROTO_SC_HOST_USER_STAT@@UEAA_NPEAVILTMessage_Write@@@Z 00000001400736e4     AppInfoDlg.obj
 0004:000006f0       $pdata$?ReadData@GAMEPROTO_SC_REMOVECLIENT@@UEAA_NPEAVILTMessage_Read@@@Z 00000001400736f0     AppInfoDlg.obj
 0004:000006fc       $pdata$?WriteData@GAMEPROTO_SC_REMOVECLIENT@@UEAA_NPEAVILTMessage_Write@@@Z 00000001400736fc     AppInfoDlg.obj
 0004:00000708       $pdata$?PreReadData@GAMEPROTO_CS_COMMON@@UEAA_NPEAVILTMessage_Read@@@Z 0000000140073708     AppInfoDlg.obj
 0004:00000714       $pdata$?PreWriteData@GAMEPROTO_CS_COMMON@@UEAA_NPEAVILTMessage_Write@@@Z 0000000140073714     AppInfoDlg.obj
 0004:00000720       $pdata$?PostWriteData@GAMEPROTO_CS_COMMON@@UEAA_NPEAVILTMessage_Write@@@Z 0000000140073720     AppInfoDlg.obj
 0004:00000720       $pdata$?PostWriteData@GAMEPROTO_SC_COMMON@@UEAA_NPEAVILTMessage_Write@@@Z 0000000140073720     AppInfoDlg.obj
 0004:0000072c       $pdata$??0exception@std@@QEAA@QEBD@Z 000000014007372c     AppInfoDlg.obj
 0004:00000738       $pdata$??_Gexception@std@@UEAAPEAXI@Z 0000000140073738     AppInfoDlg.obj
 0004:00000744       $pdata$??0exception@std@@QEAA@AEBV01@@Z 0000000140073744     AppInfoDlg.obj
 0004:00000750       $pdata$?ReadData@GAMEPROTO_SS_GAMEEND@@UEAA_NPEAVILTMessage_Read@@@Z 0000000140073750     AppInfoDlg.obj
 0004:0000075c       $pdata$?WriteData@GAMEPROTO_SS_GAMEEND@@UEAA_NPEAVILTMessage_Write@@@Z 000000014007375c     AppInfoDlg.obj
 0004:00000768       $pdata$?PostReadData@GAMEPROTO_COMMON@@UEAA_NPEAVILTMessage_Read@@@Z 0000000140073768     AppInfoDlg.obj
 0004:00000774       $pdata$0$?PostReadData@GAMEPROTO_COMMON@@UEAA_NPEAVILTMessage_Read@@@Z 0000000140073774     AppInfoDlg.obj
 0004:00000780       $pdata$1$?PostReadData@GAMEPROTO_COMMON@@UEAA_NPEAVILTMessage_Read@@@Z 0000000140073780     AppInfoDlg.obj
 0004:0000078c       $pdata$??_GCEdit@@UEAAPEAXI@Z 000000014007378c     AppInfoDlg.obj
 0004:00000798       $pdata$?IsProcessInTrouble@CHECK_MEM_USAGE@@YA_NPEAXHH@Z 0000000140073798     CheckMemUsage.obj
 0004:000007a4       $pdata$?EmptyWorkingset@CHECK_MEM_USAGE@@YA_NPEAXH@Z 00000001400737a4     CheckMemUsage.obj
 0004:000007b0       $pdata$?GetProcessMemoryUsage@@YAKPEAXH@Z 00000001400737b0     CheckMemUsage.obj
 0004:000007bc       $pdata$??1?$map@GUExtraStatsFPSVerify@CHostStat@@U?$less@G@std@@V?$allocator@U?$pair@$$CBGUExtraStatsFPSVerify@CHostStat@@@std@@@4@@std@@QEAA@XZ 00000001400737bc     HostStat.obj
 0004:000007bc       $pdata$??1?$map@GPEAUtagIP4Address@@U?$less@G@std@@V?$allocator@U?$pair@$$CBGPEAUtagIP4Address@@@std@@@3@@std@@QEAA@XZ 00000001400737bc     cSnmpEX.obj
 0004:000007c8       $pdata$??1cSnmpEX@@QEAA@XZ 00000001400737c8     cSnmpEX.obj
 0004:000007d4       $pdata$?ReleaseUDPPortAddressMap@cSnmpEX@@QEAAXXZ 00000001400737d4     cSnmpEX.obj
 0004:000007e0       $pdata$?ReleaseTCPPortAddressMap@cSnmpEX@@QEAAXXZ 00000001400737e0     cSnmpEX.obj
 0004:000007ec       $pdata$?clear@?$_Tree@V?$_Tmap_traits@GUExtraStatsFPSVerify@CHostStat@@U?$less@G@std@@V?$allocator@U?$pair@$$CBGUExtraStatsFPSVerify@CHostStat@@@std@@@4@$0A@@std@@@std@@QEAAXXZ 00000001400737ec     HostStat.obj
 0004:000007ec       $pdata$?clear@?$_Tree@V?$_Tmap_traits@GPEAUtagIP4Address@@U?$less@G@std@@V?$allocator@U?$pair@$$CBGPEAUtagIP4Address@@@std@@@3@$0A@@std@@@std@@QEAAXXZ 00000001400737ec     cSnmpEX.obj
 0004:000007ec       $pdata$?clear@?$_Tree@V?$_Tmap_traits@GUExtraStatsMemVerify@CHostStat@@U?$less@G@std@@V?$allocator@U?$pair@$$CBGUExtraStatsMemVerify@CHostStat@@@std@@@4@$0A@@std@@@std@@QEAAXXZ 00000001400737ec     HostStat.obj
 0004:000007f8       $pdata$?_Erase@?$_Tree@V?$_Tmap_traits@GUExtraStatsMemVerify@CHostStat@@U?$less@G@std@@V?$allocator@U?$pair@$$CBGUExtraStatsMemVerify@CHostStat@@@std@@@4@$0A@@std@@@std@@IEAAXPEAU?$_Tree_node@U?$pair@$$CBGUExtraStatsMemVerify@CHostStat@@@std@@PEAX@2@@Z 00000001400737f8     HostStat.obj
 0004:000007f8       $pdata$?_Erase@?$_Tree@V?$_Tmap_traits@GUExtraStatsFPSVerify@CHostStat@@U?$less@G@std@@V?$allocator@U?$pair@$$CBGUExtraStatsFPSVerify@CHostStat@@@std@@@4@$0A@@std@@@std@@IEAAXPEAU?$_Tree_node@U?$pair@$$CBGUExtraStatsFPSVerify@CHostStat@@@std@@PEAX@2@@Z 00000001400737f8     HostStat.obj
 0004:000007f8       $pdata$?_Erase@?$_Tree@V?$_Tmap_traits@GPEAUtagIP4Address@@U?$less@G@std@@V?$allocator@U?$pair@$$CBGPEAUtagIP4Address@@@std@@@3@$0A@@std@@@std@@IEAAXPEAU?$_Tree_node@U?$pair@$$CBGPEAUtagIP4Address@@@std@@PEAX@2@@Z 00000001400737f8     cSnmpEX.obj
 0004:00000804       $pdata$?_Buyheadnode@?$_Tree_comp_alloc@V?$_Tmap_traits@GUExtraStatsFPSVerify@CHostStat@@U?$less@G@std@@V?$allocator@U?$pair@$$CBGUExtraStatsFPSVerify@CHostStat@@@std@@@4@$0A@@std@@@std@@QEAAPEAU?$_Tree_node@U?$pair@$$CBGUExtraStatsFPSVerify@CHostStat@@@std@@PEAX@2@XZ 0000000140073804     HostStat.obj
 0004:00000804       $pdata$?_Buyheadnode@?$_Tree_comp_alloc@V?$_Tmap_traits@GPEAUtagIP4Address@@U?$less@G@std@@V?$allocator@U?$pair@$$CBGPEAUtagIP4Address@@@std@@@3@$0A@@std@@@std@@QEAAPEAU?$_Tree_node@U?$pair@$$CBGPEAUtagIP4Address@@@std@@PEAX@2@XZ 0000000140073804     cSnmpEX.obj
 0004:00000804       $pdata$?_Buyheadnode@?$_Tree_comp_alloc@V?$_Tmap_traits@GUExtraStatsMemVerify@CHostStat@@U?$less@G@std@@V?$allocator@U?$pair@$$CBGUExtraStatsMemVerify@CHostStat@@@std@@@4@$0A@@std@@@std@@QEAAPEAU?$_Tree_node@U?$pair@$$CBGUExtraStatsMemVerify@CHostStat@@@std@@PEAX@2@XZ 0000000140073804     HostStat.obj
 0004:00000810       $pdata$??0PROTO_GAME_USER_INFO_tag@@QEAA@XZ 0000000140073810     DividePacket.obj
 0004:0000081c       $pdata$??0PROTO_START_HOST_tag@@QEAA@XZ 000000014007381c     DividePacket.obj
 0004:00000828       $pdata$?KillServiceWithErrorcode@@YAXPEAUSERVICE_STATUS_HANDLE__@@K@Z 0000000140073828     GameServerManager.obj
 0004:00000834       $pdata$??_GCGameServerManagerApp@@UEAAPEAXI@Z 0000000140073834     GameServerManager.obj
 0004:00000840       $pdata$?InitInstance@CGameServerManagerApp@@UEAAHXZ 0000000140073840     GameServerManager.obj
 0004:0000084c       $pdata$?SetMyServiceStatus@@YAXKK@Z 000000014007384c     GameServerManager.obj
 0004:00000858       $pdata$?MyServiceMain@@YAXKPEAPEAD@Z 0000000140073858     GameServerManager.obj
 0004:00000864       $pdata$?MyServiceHandler@@YAXK@Z 0000000140073864     GameServerManager.obj
 0004:00000870       $pdata$??_GIClientHandler@@UEAAPEAXI@Z 0000000140073870     GameServerManagerDlg.obj
 0004:0000087c       $pdata$?Init@GameServerIPCMemory@@QEAAXXZ 000000014007387c     GameServerManagerDlg.obj
 0004:00000888       $pdata$?Init@GAMESERVERINFO@@QEAAXXZ 0000000140073888     GameServerManagerDlg.obj
 0004:00000894       $pdata$?GetGAME_MGMT_SETTING_FILE_PATH@@YAPEBDXZ 0000000140073894     GameServerManagerDlg.obj
 0004:000008a0       $pdata$?GetStringFormat@@YA?AV?$basic_string@DU?$char_traits@D@std@@V?$allocator@D@2@@std@@PEADZZ 00000001400738a0     GameServerManagerDlg.obj
 0004:000008ac       $pdata$?KillRemoteProcess@@YA_NK@Z 00000001400738ac     GameServerManagerDlg.obj
 0004:000008b8       $pdata$??0CGameServerManagerDlg@@QEAA@PEAVCWnd@@@Z 00000001400738b8     GameServerManagerDlg.obj
 0004:000008c4       $pdata$??_GCGameServerManagerDlg@@UEAAPEAXI@Z 00000001400738c4     GameServerManagerDlg.obj
 0004:000008d0       $pdata$??1?$map@IUPORTINFO@@U?$less@I@std@@V?$allocator@U?$pair@$$CBIUPORTINFO@@@std@@@3@@std@@QEAA@XZ 00000001400738d0     GameServerManagerDlg.obj
 0004:000008dc       $pdata$??0GAMESERVERINFO@@QEAA@XZ 00000001400738dc     GameServerManagerDlg.obj
 0004:000008e8       $pdata$??0GameServerIPCMemory@@QEAA@XZ 00000001400738e8     GameServerManagerDlg.obj
 0004:000008f4       $pdata$??1CGameServerManagerDlg@@UEAA@XZ 00000001400738f4     GameServerManagerDlg.obj
 0004:00000900       $pdata$?DoDataExchange@CGameServerManagerDlg@@MEAAXPEAVCDataExchange@@@Z 0000000140073900     GameServerManagerDlg.obj
 0004:0000090c       $pdata$?OnInitDialog@CGameServerManagerDlg@@MEAAHXZ 000000014007390c     GameServerManagerDlg.obj
 0004:00000918       $pdata$?OnPaint@CGameServerManagerDlg@@IEAAXXZ 0000000140073918     GameServerManagerDlg.obj
 0004:00000924       $pdata$1$?OnPaint@CGameServerManagerDlg@@IEAAXXZ 0000000140073924     GameServerManagerDlg.obj
 0004:00000930       $pdata$2$?OnPaint@CGameServerManagerDlg@@IEAAXXZ 0000000140073930     GameServerManagerDlg.obj
 0004:0000093c       $pdata$?InitializeManager@CGameServerManagerDlg@@QEAAHPEADKPEAPEAD@Z 000000014007393c     GameServerManagerDlg.obj
 0004:00000948       $pdata$?DestroyManager@CGameServerManagerDlg@@QEAAXXZ 0000000140073948     GameServerManagerDlg.obj
 0004:00000954       $pdata$?ReadSettings@CGameServerManagerDlg@@QEAAHXZ 0000000140073954     GameServerManagerDlg.obj
 0004:00000960       $pdata$?ConnectToMatchMakingServer@CGameServerManagerDlg@@QEAAHXZ 0000000140073960     GameServerManagerDlg.obj
 0004:0000096c       $pdata$?StartGameServer@CGameServerManagerDlg@@QEAAHF@Z 000000014007396c     GameServerManagerDlg.obj
 0004:00000978       $pdata$?OnGameServerMsg@CGameServerManagerDlg@@IEAA_J_K_J@Z 0000000140073978     GameServerManagerDlg.obj
 0004:00000984       $pdata$?KillServerApp@CGameServerManagerDlg@@IEAAXI_N@Z 0000000140073984     GameServerManagerDlg.obj
 0004:00000990       $pdata$??0PROTO_GAME_ENDED_tag@@QEAA@XZ 0000000140073990     GameServerManagerDlg.obj
 0004:0000099c       $pdata$??0PROTO_USER_STAT_tag@@QEAA@XZ 000000014007399c     GameServerManagerDlg.obj
 0004:000009a8       $pdata$?OnTimer@CGameServerManagerDlg@@IEAAX_K@Z 00000001400739a8     GameServerManagerDlg.obj
 0004:000009b4       $pdata$?OnButtonGo@CGameServerManagerDlg@@IEAAXXZ 00000001400739b4     GameServerManagerDlg.obj
 0004:000009c0       $pdata$?OnDisconnect@CGameServerManagerDlg@@UEAAXXZ 00000001400739c0     GameServerManagerDlg.obj
 0004:000009cc       $pdata$?TerminateGameServer@CGameServerManagerDlg@@QEAAXF@Z 00000001400739cc     GameServerManagerDlg.obj
 0004:000009d8       $pdata$?TerminateGSThread@CGameServerManagerDlg@@SAIPEAX@Z 00000001400739d8     GameServerManagerDlg.obj
 0004:000009e4       $pdata$?SendMessageToWriteLogFile@CGameServerManagerDlg@@QEAAXFPEAUHWND__@@0AEAUtagCOPYDATASTRUCT@@@Z 00000001400739e4     GameServerManagerDlg.obj
 0004:000009f0       $pdata$?VerifyServerAppTermination@CGameServerManagerDlg@@AEAAXXZ 00000001400739f0     GameServerManagerDlg.obj
 0004:000009fc       $pdata$?StringSplitToNumArray@CGameServerManagerDlg@@AEAAXV?$basic_string@DU?$char_traits@D@std@@V?$allocator@D@2@@std@@0PEAHAEAH@Z 00000001400739fc     GameServerManagerDlg.obj
 0004:00000a08       $pdata$?FindFreePorts@CGameServerManagerDlg@@AEAA_NXZ 0000000140073a08     GameServerManagerDlg.obj
 0004:00000a14       $pdata$?RestoreFreePort@CGameServerManagerDlg@@AEAAXXZ 0000000140073a14     GameServerManagerDlg.obj
 0004:00000a20       $pdata$?ReservePort@CGameServerManagerDlg@@AEAAXIF@Z 0000000140073a20     GameServerManagerDlg.obj
 0004:00000a2c       $pdata$0$?ReservePort@CGameServerManagerDlg@@AEAAXIF@Z 0000000140073a2c     GameServerManagerDlg.obj
 0004:00000a38       $pdata$1$?ReservePort@CGameServerManagerDlg@@AEAAXIF@Z 0000000140073a38     GameServerManagerDlg.obj
 0004:00000a44       $pdata$?ChangeNumRoomsReserved@CGameServerManagerDlg@@QEAAXHH_N@Z 0000000140073a44     GameServerManagerDlg.obj
 0004:00000a50       $pdata$?ChangeNumActiveServers@CGameServerManagerDlg@@QEAAXH@Z 0000000140073a50     GameServerManagerDlg.obj
 0004:00000a5c       $pdata$?ServerAppUseCountLog@CGameServerManagerDlg@@AEAAXXZ 0000000140073a5c     GameServerManagerDlg.obj
 0004:00000a68       $pdata$??0CSharedMemoryLoader@@QEAA@XZ 0000000140073a68     GameServerManagerDlg.obj
 0004:00000a74       $pdata$??1CSharedMemoryLoader@@QEAA@XZ 0000000140073a74     GameServerManagerDlg.obj
 0004:00000a80       $pdata$?_PreLoad@CSharedMemoryLoader@@AEAA_NXZ 0000000140073a80     GameServerManagerDlg.obj
 0004:00000a8c       $pdata$?_Load@CSharedMemoryLoader@@AEAA_NXZ 0000000140073a8c     GameServerManagerDlg.obj
 0004:00000a98       $pdata$?Load@CSharedMemoryLoader@@QEAA_NXZ 0000000140073a98     GameServerManagerDlg.obj
 0004:00000aa4       $pdata$?Release@CSharedMemoryLoader@@QEAA_NXZ 0000000140073aa4     GameServerManagerDlg.obj
 0004:00000ab0       $pdata$?ProcessThread@CGameServerManagerDlg@@CAIPEAX@Z 0000000140073ab0     GameServerManagerDlg.obj
 0004:00000abc       $pdata$?ProcessSocketEventThread@CGameServerManagerDlg@@CAIPEAX@Z 0000000140073abc     GameServerManagerDlg.obj
 0004:00000ac8       $pdata$?PostMessageToWriteLogFile@CGameServerManagerDlg@@AEAA_NFPEAUHWND__@@_K_J@Z 0000000140073ac8     GameServerManagerDlg.obj
 0004:00000ad4       $pdata$?OnCopyData@CGameServerManagerDlg@@IEAAHPEAVCWnd@@PEAUtagCOPYDATASTRUCT@@@Z 0000000140073ad4     GameServerManagerDlg.obj
 0004:00000ae0       $pdata$?RECV_MSG_REMOVE_CLIENT@CGameServerManagerDlg@@AEAAXFPEBUGAMEPROTO_SC_REMOVECLIENT@@@Z 0000000140073ae0     GameServerManagerDlg.obj
 0004:00000aec       $pdata$?RECV_MSG_GAMEEND@CGameServerManagerDlg@@AEAAXFPEBUGAMEPROTO_SS_GAMEEND@@@Z 0000000140073aec     GameServerManagerDlg.obj
 0004:00000af8       $pdata$?RECV_MSG_HOST_USER_STAT@CGameServerManagerDlg@@AEAAXFPEBUGAMEPROTO_SC_HOST_USER_STAT@@@Z 0000000140073af8     GameServerManagerDlg.obj
 0004:00000b04       $pdata$2$?RECV_MSG_HOST_USER_STAT@CGameServerManagerDlg@@AEAAXFPEBUGAMEPROTO_SC_HOST_USER_STAT@@@Z 0000000140073b04     GameServerManagerDlg.obj
 0004:00000b10       $pdata$3$?RECV_MSG_HOST_USER_STAT@CGameServerManagerDlg@@AEAAXFPEBUGAMEPROTO_SC_HOST_USER_STAT@@@Z 0000000140073b10     GameServerManagerDlg.obj
 0004:00000b1c       $pdata$?RECV_MSG_BAN_USER@CGameServerManagerDlg@@AEAAXFPEAUPROTO_BAN_USER_tag@@@Z 0000000140073b1c     GameServerManagerDlg.obj
 0004:00000b28       $pdata$?RECV_MSG_HOST_STAT@CGameServerManagerDlg@@AEAAXFPEBUGAMEPROTO_SC_HOST_STAT@@@Z 0000000140073b28     GameServerManagerDlg.obj
 0004:00000b34       $pdata$?RECV_MSG_INGAME_AIGACHA_ITEM_INSERT@CGameServerManagerDlg@@AEAAXFPEAUPROTO_GAMEGT_INGAME_AIGACHA_ITEM_INSERT@@@Z 0000000140073b34     GameServerManagerDlg.obj
 0004:00000b40       $pdata$?RECV_MSG_MAPLOADING_COMPLETE_NTY@CGameServerManagerDlg@@AEAAXFPEAUPROTO_GAMEGT_MAPLOADING_COMPLETE_NTY_tag@@@Z 0000000140073b40     GameServerManagerDlg.obj
 0004:00000b4c       $pdata$?RECV_MSG_SPY_CHANGE@CGameServerManagerDlg@@AEAAXFPEAUGAMEPROTO_SC_SPY_CHANGE@@@Z 0000000140073b4c     GameServerManagerDlg.obj
 0004:00000b58       $pdata$?RECV_MSG_INGAME_FARMING_ITEM_REQ@CGameServerManagerDlg@@AEAAXFPEAUPROTO_GAMEGT_INGAME_FARMING_ITEM_REQ@@@Z 0000000140073b58     GameServerManagerDlg.obj
 0004:00000b64       $pdata$?RECV_MSG_AI2_BONUSROUND_REWARD@CGameServerManagerDlg@@AEAAXFPEAUPROTOCOL_AI2_BONUSROUND_REWARD_REQ_tag@@@Z 0000000140073b64     GameServerManagerDlg.obj
 0004:00000b70       $pdata$?RECV_MSG_AI3_BONUS_REWARD_ITEM@CGameServerManagerDlg@@AEAAXFPEAUPROTO_GAMEGT_INGAME_AI3_BONUS_REWARD_ITEM_REQ@@@Z 0000000140073b70     GameServerManagerDlg.obj
 0004:00000b7c       $pdata$?RECV_MSG_AI_EXTRA_REWARD@CGameServerManagerDlg@@AEAAXFPEAUPROTO_AI_EXTRA_REWARD_REQ@@@Z 0000000140073b7c     GameServerManagerDlg.obj
 0004:00000b88       $pdata$?RECV_MSG_FINISHED_GAME_PREV@CGameServerManagerDlg@@AEAAXFPEAUPROTO_FINISHED_GAME_PREV_tag@@@Z 0000000140073b88     GameServerManagerDlg.obj
 0004:00000b94       $pdata$?RECV_MSG_SPEC_RECOMMENDROOM_INGAME_DATA@CGameServerManagerDlg@@AEAAXFPEBUPROTO_SPEC_RECOMMENDROOM_INGAME_DATA@@@Z 0000000140073b94     GameServerManagerDlg.obj
 0004:00000ba0       $pdata$?RECV_MSG_AUTO_SIDE_CHANGE_TEAM_INFO_NTY@CGameServerManagerDlg@@AEAAXFPEAUPROTO_GAMEGT_AUTO_SIDE_CHANGE_TEAM_INFO_NTY@@@Z 0000000140073ba0     GameServerManagerDlg.obj
 0004:00000bac       $pdata$?RECV_MSG_INSERTCHARACTER_ACK@CGameServerManagerDlg@@AEAAXFPEBUPROTO_INSERT_CHARACTER_RESULT_tag@@@Z 0000000140073bac     GameServerManagerDlg.obj
 0004:00000bb8       $pdata$?OnReceive@CGameServerManagerDlg@@UEAAXPEAVCPacket@@@Z 0000000140073bb8     GameServerManagerDlg.obj
 0004:00000bc4       $pdata$1$?OnReceive@CGameServerManagerDlg@@UEAAXPEAVCPacket@@@Z 0000000140073bc4     GameServerManagerDlg.obj
 0004:00000bd0       $pdata$7$?OnReceive@CGameServerManagerDlg@@UEAAXPEAVCPacket@@@Z 0000000140073bd0     GameServerManagerDlg.obj
 0004:00000bdc       $pdata$8$?OnReceive@CGameServerManagerDlg@@UEAAXPEAVCPacket@@@Z 0000000140073bdc     GameServerManagerDlg.obj
 0004:00000be8       $pdata$9$?OnReceive@CGameServerManagerDlg@@UEAAXPEAVCPacket@@@Z 0000000140073be8     GameServerManagerDlg.obj
 0004:00000bf4       $pdata$?OnReceiveFromGms@CGameServerManagerDlg@@AEAAXPEAVCPacket@@@Z 0000000140073bf4     GameServerManagerDlg.obj
 0004:00000c00       $pdata$4$?OnReceiveFromGms@CGameServerManagerDlg@@AEAAXPEAVCPacket@@@Z 0000000140073c00     GameServerManagerDlg.obj
 0004:00000c0c       $pdata$5$?OnReceiveFromGms@CGameServerManagerDlg@@AEAAXPEAVCPacket@@@Z 0000000140073c0c     GameServerManagerDlg.obj
 0004:00000c18       $pdata$?OnReceiveFromGms@CGameServerManagerDlg@@AEAAXAEBUPROTO_STARTING_GAME_tag@@@Z 0000000140073c18     GameServerManagerDlg.obj
 0004:00000c24       $pdata$?OnReceiveFromGms@CGameServerManagerDlg@@AEAAXAEBUPROTO_INSERT_CHARACTER_tag@@@Z 0000000140073c24     GameServerManagerDlg.obj
 0004:00000c30       $pdata$?OnReceiveFromGms@CGameServerManagerDlg@@AEAAXAEBUPROTO_MMSERVER_TERMINATED_tag@@@Z 0000000140073c30     GameServerManagerDlg.obj
 0004:00000c3c       $pdata$?OnReceiveFromGms@CGameServerManagerDlg@@AEAAXAEBUPROTO_USER_DISCONNECTED_tag@@@Z 0000000140073c3c     GameServerManagerDlg.obj
 0004:00000c48       $pdata$1$?OnReceiveFromGms@CGameServerManagerDlg@@AEAAXAEBUPROTO_USER_DISCONNECTED_tag@@@Z 0000000140073c48     GameServerManagerDlg.obj
 0004:00000c54       $pdata$2$?OnReceiveFromGms@CGameServerManagerDlg@@AEAAXAEBUPROTO_USER_DISCONNECTED_tag@@@Z 0000000140073c54     GameServerManagerDlg.obj
 0004:00000c60       $pdata$?OnReceiveFromGms@CGameServerManagerDlg@@AEAAXAEBUPROTO_GAMEGT_INGAME_AIGACHA_ITEM_INSERT_RESULT@@@Z 0000000140073c60     GameServerManagerDlg.obj
 0004:00000c6c       $pdata$?OnReceiveFromGms@CGameServerManagerDlg@@AEAAXAEBUPROTO_AUTOMATCH_GAME_START_REQ@@@Z 0000000140073c6c     GameServerManagerDlg.obj
 0004:00000c78       $pdata$?OnReceiveFromGms@CGameServerManagerDlg@@AEAAXAEBUPROTO_AUTOMATCH_GAME_ENTER_REQ@@@Z 0000000140073c78     GameServerManagerDlg.obj
 0004:00000c84       $pdata$?FindServerApp@CGameServerManagerDlg@@AEAA?B_NFKAEAF@Z 0000000140073c84     GameServerManagerDlg.obj
 0004:00000c90       $pdata$?AssignServerApp@CGameServerManagerDlg@@AEAAXAEBUPROTO_STARTING_GAME_tag@@F@Z 0000000140073c90     GameServerManagerDlg.obj
 0004:00000c9c       $pdata$?AssignServerApp@CGameServerManagerDlg@@AEAAXAEBUPROTO_AUTOMATCH_GAME_START_REQ@@F@Z 0000000140073c9c     GameServerManagerDlg.obj
 0004:00000ca8       $pdata$?SendToGmsStartingGameRes@CGameServerManagerDlg@@AEAAXAEBUGAMESERVERINFO@@FW4START_HOST_RESULT@@@Z 0000000140073ca8     GameServerManagerDlg.obj
 0004:00000cb4       $pdata$?SendToGmsAutoMatchGameStartRes@CGameServerManagerDlg@@AEAAXAEBUGAMESERVERINFO@@FW4START_HOST_RESULT@@@Z 0000000140073cb4     GameServerManagerDlg.obj
 0004:00000cc0       $pdata$?SendToGmsAutoMatchGameEnterNty@CGameServerManagerDlg@@AEAAXF@Z 0000000140073cc0     GameServerManagerDlg.obj
 0004:00000ccc       $pdata$0$?SendToGmsAutoMatchGameEnterNty@CGameServerManagerDlg@@AEAAXF@Z 0000000140073ccc     GameServerManagerDlg.obj
 0004:00000cd8       $pdata$1$?SendToGmsAutoMatchGameEnterNty@CGameServerManagerDlg@@AEAAXF@Z 0000000140073cd8     GameServerManagerDlg.obj
 0004:00000ce4       $pdata$?SendToServerAppAutoMatchGameEnterNty@CGameServerManagerDlg@@AEAAXF@Z 0000000140073ce4     GameServerManagerDlg.obj
 0004:00000cf0       $pdata$0$?SendToServerAppAutoMatchGameEnterNty@CGameServerManagerDlg@@AEAAXF@Z 0000000140073cf0     GameServerManagerDlg.obj
 0004:00000cfc       $pdata$1$?SendToServerAppAutoMatchGameEnterNty@CGameServerManagerDlg@@AEAAXF@Z 0000000140073cfc     GameServerManagerDlg.obj
 0004:00000d08       $pdata$??1?$shared_ptr@UGAMESERVERINFO@@@std@@QEAA@XZ 0000000140073d08     GameServerManagerDlg.obj
 0004:00000d14       $pdata$??1?$list@UverifyTerminationStatus_t@@V?$allocator@UverifyTerminationStatus_t@@@std@@@std@@QEAA@XZ 0000000140073d14     GameServerManagerDlg.obj
 0004:00000d20       $pdata$0$??1?$list@UverifyTerminationStatus_t@@V?$allocator@UverifyTerminationStatus_t@@@std@@@std@@QEAA@XZ 0000000140073d20     GameServerManagerDlg.obj
 0004:00000d2c       $pdata$1$??1?$list@UverifyTerminationStatus_t@@V?$allocator@UverifyTerminationStatus_t@@@std@@@std@@QEAA@XZ 0000000140073d2c     GameServerManagerDlg.obj
 0004:00000d38       $pdata$?clear@?$_Tree@V?$_Tmap_traits@IUPORTINFO@@U?$less@I@std@@V?$allocator@U?$pair@$$CBIUPORTINFO@@@std@@@3@$0A@@std@@@std@@QEAAXXZ 0000000140073d38     GameServerManagerDlg.obj
 0004:00000d44       $pdata$?find_first_of@?$basic_string@DU?$char_traits@D@std@@V?$allocator@D@2@@std@@QEBA_KAEBV12@_K@Z 0000000140073d44     GameServerManagerDlg.obj
 0004:00000d50       $pdata$?_Erase@?$_Tree@V?$_Tmap_traits@IUPORTINFO@@U?$less@I@std@@V?$allocator@U?$pair@$$CBIUPORTINFO@@@std@@@3@$0A@@std@@@std@@IEAAXPEAU?$_Tree_node@U?$pair@$$CBIUPORTINFO@@@std@@PEAX@2@@Z 0000000140073d50     GameServerManagerDlg.obj
 0004:00000d5c       $pdata$?_Buynode0@?$_List_alloc@U?$_List_base_types@UverifyTerminationStatus_t@@V?$allocator@UverifyTerminationStatus_t@@@std@@@std@@@std@@QEAAPEAU?$_List_node@UverifyTerminationStatus_t@@PEAX@2@PEAU32@0@Z 0000000140073d5c     GameServerManagerDlg.obj
 0004:00000d68       $pdata$?_Extract@?$_Tree_val@U?$_Tree_simple_types@U?$pair@$$CBIUPORTINFO@@@std@@@std@@@std@@QEAAPEAU?$_Tree_node@U?$pair@$$CBIUPORTINFO@@@std@@PEAX@2@V?$_Tree_const_iterator@V?$_Tree_val@U?$_Tree_simple_types@U?$pair@$$CBIUPORTINFO@@@std@@@std@@@std@@@2@@Z 0000000140073d68     GameServerManagerDlg.obj
 0004:00000d74       $pdata$?_Buyheadnode@?$_Tree_comp_alloc@V?$_Tmap_traits@IUPORTINFO@@U?$less@I@std@@V?$allocator@U?$pair@$$CBIUPORTINFO@@@std@@@3@$0A@@std@@@std@@QEAAPEAU?$_Tree_node@U?$pair@$$CBIUPORTINFO@@@std@@PEAX@2@XZ 0000000140073d74     GameServerManagerDlg.obj
 0004:00000d80       $pdata$??$sprintf_s@$0GE@@cf@@YAHAEAY0GE@DPEBDZZ 0000000140073d80     GameServerManagerDlg.obj
 0004:00000d8c       $pdata$??$sprintf_s@$0PP@@cf@@YAHAEAY0PP@DPEBDZZ 0000000140073d8c     GameServerManagerDlg.obj
 0004:00000d98       $pdata$?reserve@?$basic_string@DU?$char_traits@D@std@@V?$allocator@D@2@@std@@QEAAX_K@Z 0000000140073d98     GameServerManagerDlg.obj
 0004:00000da4       $pdata$0$?reserve@?$basic_string@DU?$char_traits@D@std@@V?$allocator@D@2@@std@@QEAAX_K@Z 0000000140073da4     GameServerManagerDlg.obj
 0004:00000db0       $pdata$2$?reserve@?$basic_string@DU?$char_traits@D@std@@V?$allocator@D@2@@std@@QEAAX_K@Z 0000000140073db0     GameServerManagerDlg.obj
 0004:00000dbc       $pdata$3$?reserve@?$basic_string@DU?$char_traits@D@std@@V?$allocator@D@2@@std@@QEAAX_K@Z 0000000140073dbc     GameServerManagerDlg.obj
 0004:00000dc8       $pdata$4$?reserve@?$basic_string@DU?$char_traits@D@std@@V?$allocator@D@2@@std@@QEAAX_K@Z 0000000140073dc8     GameServerManagerDlg.obj
 0004:00000dd4       $pdata$5$?reserve@?$basic_string@DU?$char_traits@D@std@@V?$allocator@D@2@@std@@QEAAX_K@Z 0000000140073dd4     GameServerManagerDlg.obj
 0004:00000de0       $pdata$??$_Setp@UGAMESERVERINFO@@@?$shared_ptr@UGAMESERVERINFO@@@std@@AEAAXPEAUGAMESERVERINFO@@U?$integral_constant@_N$0A@@1@@Z 0000000140073de0     GameServerManagerDlg.obj
 0004:00000dec       $pdata$??$_Buynode@AEBUverifyTerminationStatus_t@@@?$_List_buy@UverifyTerminationStatus_t@@V?$allocator@UverifyTerminationStatus_t@@@std@@@std@@QEAAPEAU?$_List_node@UverifyTerminationStatus_t@@PEAX@1@PEAU21@0AEBUverifyTerminationStatus_t@@@Z 0000000140073dec     GameServerManagerDlg.obj
 0004:00000df8       $pdata$??_G?$_Ref_count@UGAMESERVERINFO@@@std@@UEAAPEAXI@Z 0000000140073df8     GameServerManagerDlg.obj
 0004:00000e04       $pdata$??$_Buynode@U?$pair@IUPORTINFO@@@std@@@?$_Tree_comp_alloc@V?$_Tmap_traits@IUPORTINFO@@U?$less@I@std@@V?$allocator@U?$pair@$$CBIUPORTINFO@@@std@@@3@$0A@@std@@@std@@QEAAPEAU?$_Tree_node@U?$pair@$$CBIUPORTINFO@@@std@@PEAX@1@$$QEAU?$pair@IUPORTINFO@@@1@@Z 0000000140073e04     GameServerManagerDlg.obj
 0004:00000e10       $pdata$??$_Insert_nohint@AEAU?$pair@$$CBIUPORTINFO@@@std@@PEAU?$_Tree_node@U?$pair@$$CBIUPORTINFO@@@std@@PEAX@2@@?$_Tree@V?$_Tmap_traits@IUPORTINFO@@U?$less@I@std@@V?$allocator@U?$pair@$$CBIUPORTINFO@@@std@@@3@$0A@@std@@@std@@IEAA?AU?$pair@V?$_Tree_iterator@V?$_Tree_val@U?$_Tree_simple_types@U?$pair@$$CBIUPORTINFO@@@std@@@std@@@std@@@std@@_N@1@_NAEAU?$pair@$$CBIUPORTINFO@@@1@PEAU?$_Tree_node@U?$pair@$$CBIUPORTINFO@@@std@@PEAX@1@@Z 0000000140073e10     GameServerManagerDlg.obj
 0004:00000e1c       $pdata$?_Buynode0@?$_Tree_comp_alloc@V?$_Tmap_traits@IUPORTINFO@@U?$less@I@std@@V?$allocator@U?$pair@$$CBIUPORTINFO@@@std@@@3@$0A@@std@@@std@@QEAAPEAU?$_Tree_node@U?$pair@$$CBIUPORTINFO@@@std@@PEAX@2@XZ 0000000140073e1c     GameServerManagerDlg.obj
 0004:00000e28       $pdata$??$_Insert_at@AEAU?$pair@$$CBIUPORTINFO@@@std@@PEAU?$_Tree_node@U?$pair@$$CBIUPORTINFO@@@std@@PEAX@2@@?$_Tree@V?$_Tmap_traits@IUPORTINFO@@U?$less@I@std@@V?$allocator@U?$pair@$$CBIUPORTINFO@@@std@@@3@$0A@@std@@@std@@IEAA?AV?$_Tree_iterator@V?$_Tree_val@U?$_Tree_simple_types@U?$pair@$$CBIUPORTINFO@@@std@@@std@@@std@@@1@_NPEAU?$_Tree_node@U?$pair@$$CBIUPORTINFO@@@std@@PEAX@1@AEAU?$pair@$$CBIUPORTINFO@@@1@1@Z 0000000140073e28     GameServerManagerDlg.obj
 0004:00000e34       $pdata$??$_Buynode@AEBUpiecewise_construct_t@std@@V?$tuple@AEBI@2@V?$tuple@$$V@2@@?$_Tree_comp_alloc@V?$_Tmap_traits@IUPORTINFO@@U?$less@I@std@@V?$allocator@U?$pair@$$CBIUPORTINFO@@@std@@@3@$0A@@std@@@std@@QEAAPEAU?$_Tree_node@U?$pair@$$CBIUPORTINFO@@@std@@PEAX@1@AEBUpiecewise_construct_t@1@$$QEAV?$tuple@AEBI@1@$$QEAV?$tuple@$$V@1@@Z 0000000140073e34     GameServerManagerDlg.obj
 0004:00000e40       $pdata$??$_Insert_hint@AEAU?$pair@$$CBIUPORTINFO@@@std@@PEAU?$_Tree_node@U?$pair@$$CBIUPORTINFO@@@std@@PEAX@2@@?$_Tree@V?$_Tmap_traits@IUPORTINFO@@U?$less@I@std@@V?$allocator@U?$pair@$$CBIUPORTINFO@@@std@@@3@$0A@@std@@@std@@IEAA?AV?$_Tree_iterator@V?$_Tree_val@U?$_Tree_simple_types@U?$pair@$$CBIUPORTINFO@@@std@@@std@@@std@@@1@V?$_Tree_const_iterator@V?$_Tree_val@U?$_Tree_simple_types@U?$pair@$$CBIUPORTINFO@@@std@@@std@@@std@@@1@AEAU?$pair@$$CBIUPORTINFO@@@1@PEAU?$_Tree_node@U?$pair@$$CBIUPORTINFO@@@std@@PEAX@1@@Z 0000000140073e40     GameServerManagerDlg.obj
 0004:00000e4c       $pdata$?RTIDUSNtoString@EXPAND_USN@@YA?AV?$basic_string@DU?$char_traits@D@std@@V?$allocator@D@2@@std@@HFF_J@Z 0000000140073e4c     GameServerManagerDlg.obj
 0004:00000e58       $pdata$??4WEAPON_INFO@@QEAAAEAU0@AEBU0@@Z 0000000140073e58     GameServerManagerDlg.obj
 0004:00000e64       $pdata$?USNtoStr@EXPAND_USN@@YA?AV?$basic_string@DU?$char_traits@D@std@@V?$allocator@D@2@@std@@_J@Z 0000000140073e64     GameServerManagerDlg.obj
 0004:00000e70       $pdata$?find_last_of@?$basic_string@DU?$char_traits@D@std@@V?$allocator@D@2@@std@@QEBA_KQEBD_K@Z 0000000140073e70     GameServerManagerDlg.obj
 0004:00000e7c       $pdata$??4?$basic_string@DU?$char_traits@D@std@@V?$allocator@D@2@@std@@QEAAAEAV01@$$QEAV01@@Z 0000000140073e7c     GameServerManagerDlg.obj
 0004:00000e88       $pdata$?_Xran@?$_String_val@U?$_Simple_types@D@std@@@std@@SAXXZ 0000000140073e88     GameServerManagerDlg.obj
 0004:00000e94       $pdata$?substr@?$basic_string@DU?$char_traits@D@std@@V?$allocator@D@2@@std@@QEBA?AV12@_K0@Z 0000000140073e94     GameServerManagerDlg.obj
 0004:00000ea0       $pdata$??$_Reallocate_grow_by@V<lambda_65e615be2a453ca0576c979606f46740>@@PEBD_K@?$basic_string@DU?$char_traits@D@std@@V?$allocator@D@2@@std@@QEAAAEAV01@_KV<lambda_65e615be2a453ca0576c979606f46740>@@PEBD_K@Z 0000000140073ea0     GameServerManagerDlg.obj
 0004:00000eac       $pdata$3$??$_Reallocate_grow_by@V<lambda_65e615be2a453ca0576c979606f46740>@@PEBD_K@?$basic_string@DU?$char_traits@D@std@@V?$allocator@D@2@@std@@QEAAAEAV01@_KV<lambda_65e615be2a453ca0576c979606f46740>@@PEBD_K@Z 0000000140073eac     GameServerManagerDlg.obj
 0004:00000eb8       $pdata$4$??$_Reallocate_grow_by@V<lambda_65e615be2a453ca0576c979606f46740>@@PEBD_K@?$basic_string@DU?$char_traits@D@std@@V?$allocator@D@2@@std@@QEAAAEAV01@_KV<lambda_65e615be2a453ca0576c979606f46740>@@PEBD_K@Z 0000000140073eb8     GameServerManagerDlg.obj
 0004:00000ec4       $pdata$?append@?$basic_string@DU?$char_traits@D@std@@V?$allocator@D@2@@std@@QEAAAEAV12@QEBD_K@Z 0000000140073ec4     GameServerManagerDlg.obj
 0004:00000ed0       $pdata$0$?append@?$basic_string@DU?$char_traits@D@std@@V?$allocator@D@2@@std@@QEAAAEAV12@QEBD_K@Z 0000000140073ed0     GameServerManagerDlg.obj
 0004:00000edc       $pdata$1$?append@?$basic_string@DU?$char_traits@D@std@@V?$allocator@D@2@@std@@QEAAAEAV12@QEBD_K@Z 0000000140073edc     GameServerManagerDlg.obj
 0004:00000ee8       $pdata$?init@SGGMProxyLoader@sggm_proxy@@QEAA_NPEAVMultiReceiver@2@@Z 0000000140073ee8     GameServerManagerDlg.obj
 0004:00000ef4       $pdata$sscanf              0000000140073ef4     GameServerManagerDlg.obj
 0004:00000f00       $pdata$??0BATTLE_ROYAL_RESULT@@QEAA@XZ 0000000140073f00     GameServerManagerDlg.obj
 0004:00000f0c       $pdata$??0GAMEPROTO_SC_HOST_USER_STAT@@QEAA@XZ 0000000140073f0c     GameServerManagerDlg.obj
 0004:00000f18       $pdata$??0GAMEPROTO_SS_GAMEEND@@QEAA@XZ 0000000140073f18     GameServerManagerDlg.obj
 0004:00000f24       $pdata$??1SGGMProxyLoader@sggm_proxy@@QEAA@XZ 0000000140073f24     GameServerManagerDlg.obj
 0004:00000f30       $pdata$memcpy_s            0000000140073f30     GameServerManagerDlg.obj
 0004:00000f3c       $pdata$?StringCchCopyA@@YAJPEAD_KPEBD@Z 0000000140073f3c     GameServerManagerDlg.obj
 0004:00000f48       $pdata$?Send@CGMSConnManager@@AEAAHPEAVCPacket@@@Z 0000000140073f48     GMSConnManager.obj
 0004:00000f54       $pdata$?SendDiv@CGMSConnManager@@AEAAHEEEPEADK@Z 0000000140073f54     GMSConnManager.obj
 0004:00000f60       $pdata$?SortFinishedGameUserInfo@CGMSConnManager@@AEAAXAEAUPROTO_FINISHED_GAME_tag@@@Z 0000000140073f60     GMSConnManager.obj
 0004:00000f6c       $pdata$??4PROTO_USER_STAT_tag@@QEAAAEAU0@AEBU0@@Z 0000000140073f6c     GMSConnManager.obj
 0004:00000f78       $pdata$??_ECSFGameServerClientLib@@UEAAPEAXI@Z 0000000140073f78     GMSConnManager.obj
 0004:00000f84       $pdata$?StartingReport@CGMSConnManager@@QEAAHFHHHHHHHQEAHHH@Z 0000000140073f84     GMSConnManager.obj
 0004:00000f90       $pdata$?StartingGameResult@CGMSConnManager@@QEAAHUPROTO_STARTING_GAME_RESULT_tag@@W4START_HOST_RESULT@@@Z 0000000140073f90     GMSConnManager.obj
 0004:00000f9c       $pdata$?FinishedGame@CGMSConnManager@@QEAAHUPROTO_FINISHED_GAME_tag@@@Z 0000000140073f9c     GMSConnManager.obj
 0004:00000fa8       $pdata$?UpdateCharacterStat@CGMSConnManager@@QEAAHUPROTO_UPDATE_CHARACTER_STAT_tag@@@Z 0000000140073fa8     GMSConnManager.obj
 0004:00000fb4       $pdata$?InsertCharacterResult@CGMSConnManager@@QEAAHUPROTO_INSERT_CHARACTER_RESULT_tag@@@Z 0000000140073fb4     GMSConnManager.obj
 0004:00000fc0       $pdata$?SendHeartBeat@CGMSConnManager@@QEAAHH@Z 0000000140073fc0     GMSConnManager.obj
 0004:00000fcc       $pdata$?SendForceLeavePollResult@CGMSConnManager@@QEAAHPEBUPROTO_BAN_USER_tag@@@Z 0000000140073fcc     GMSConnManager.obj
 0004:00000fd8       $pdata$?NotifyAllocableRoomCountChanged@CGMSConnManager@@QEAAHJHHHHHQEAHHH@Z 0000000140073fd8     GMSConnManager.obj
 0004:00000fe4       $pdata$?SendRoundChange@CGMSConnManager@@QEAAHPEBUPROTO_GAMEGT_ROUND_CHANGE_NTY_tag@@@Z 0000000140073fe4     GMSConnManager.obj
 0004:00000ff0       $pdata$?SendGameStart@CGMSConnManager@@QEAAHPEBUPROTO_GAMEGT_GAME_START_NTY@@@Z 0000000140073ff0     GMSConnManager.obj
 0004:00000ffc       $pdata$?SendTeamDeathMatchKillCnt@CGMSConnManager@@QEAAHPEBUPROTO_GAMEGT_TEAM_DEATH_KILL_CNT_NTY@@@Z 0000000140073ffc     GMSConnManager.obj
 0004:00001008       $pdata$?SendAIItemInsert@CGMSConnManager@@QEAAHPEAUPROTO_GAMEGT_INGAME_AIGACHA_ITEM_INSERT@@@Z 0000000140074008     GMSConnManager.obj
 0004:00001014       $pdata$?SendIntrusionCoinDec@CGMSConnManager@@QEAAHPEAUPROTO_GAMEGT_MAPLOADING_COMPLETE_NTY_tag@@@Z 0000000140074014     GMSConnManager.obj
 0004:00001020       $pdata$?SendSpyChange@CGMSConnManager@@QEAAHPEAUPROTO_GAMEGT_SPY_CHANGE_NTY_tag@@@Z 0000000140074020     GMSConnManager.obj
 0004:0000102c       $pdata$?SendFarmingItemReq@CGMSConnManager@@QEAAHPEAUPROTO_GAMEGT_INGAME_FARMING_ITEM_REQ@@@Z 000000014007402c     GMSConnManager.obj
 0004:00001038       $pdata$?SendBattleShipBonusCoinReq@CGMSConnManager@@QEAAHPEAUPROTOCOL_AI2_BONUSROUND_REWARD_REQ_tag@@@Z 0000000140074038     GMSConnManager.obj
 0004:00001044       $pdata$?SendAI3BonusClearItemReq@CGMSConnManager@@QEAAHPEAUPROTO_GAMEGT_INGAME_AI3_BONUS_REWARD_ITEM_REQ@@@Z 0000000140074044     GMSConnManager.obj
 0004:00001050       $pdata$?SendAIExtraRewardReq@CGMSConnManager@@QEAAHPEAUPROTO_AI_EXTRA_REWARD_REQ@@@Z 0000000140074050     GMSConnManager.obj
 0004:0000105c       $pdata$?SendBossTowerRewardReq@CGMSConnManager@@QEAAHPEAUPROTO_AI_BOSS_TOWER_REWARD_REQ@@@Z 000000014007405c     GMSConnManager.obj
 0004:00001068       $pdata$?SendIngameRewardReq@CGMSConnManager@@QEAAHPEAUPROTO_INGAME_RESULT_REQ@@@Z 0000000140074068     GMSConnManager.obj
 0004:00001074       $pdata$?SendKickUserInfo@CGMSConnManager@@QEAAHPEAUPROTO_GAMEMGT_KICK_USER@@@Z 0000000140074074     GMSConnManager.obj
 0004:00001080       $pdata$?SendSpectatorRecommendRoomData@CGMSConnManager@@QEAAHPEAUPROTO_SPECTATOR_RECOMMEND_ROOM_INGAME_DATA_NTY@@@Z 0000000140074080     GMSConnManager.obj
 0004:0000108c       $pdata$?SendPrevGameFinishNotify@CGMSConnManager@@QEAAHPEAUPROTO_FINISHED_GAME_PREV_tag@@@Z 000000014007408c     GMSConnManager.obj
 0004:00001098       $pdata$?SendAutoSideChangeTeamInfoNotify@CGMSConnManager@@QEAAHPEAUPROTO_GAMEGT_AUTO_SIDE_CHANGE_TEAM_INFO_NTY@@@Z 0000000140074098     GMSConnManager.obj
 0004:000010a4       $pdata$?SendAIExtraMiddleRewardReq@CGMSConnManager@@QEAAHPEAUPROTO_AI_EXTRA_MIDDLE_REWARD_REQ@@@Z 00000001400740a4     GMSConnManager.obj
 0004:000010b0       $pdata$?SendAutoMatchGameStartRes@CGMSConnManager@@QEAAHAEBUPROTO_AUTOMATCH_GAME_START_RES@@W4START_HOST_RESULT@@@Z 00000001400740b0     GMSConnManager.obj
 0004:000010bc       $pdata$?SendAutoMatchGameEnterRes@CGMSConnManager@@QEAAHAEBUPROTO_AUTOMATCH_GAME_ENTER_RES@@@Z 00000001400740bc     GMSConnManager.obj
 0004:000010c8       $pdata$?SendAutoMatchIngameEnterNty@CGMSConnManager@@QEAAHAEBUPROTO_AUTOMATCH_INGAME_ENTER_NTY@@@Z 00000001400740c8     GMSConnManager.obj
 0004:000010d4       $pdata$??$sprintf_s@$0EBA@@cf@@YAHAEAY0EBA@DPEBDZZ 00000001400740d4     GMSConnManager.obj
 0004:000010e0       $pdata$??$_Reallocate_grow_by@V<lambda_319d5e083f45f90dcdce5dce53cbb275>@@D@?$basic_string@DU?$char_traits@D@std@@V?$allocator@D@2@@std@@QEAAAEAV01@_KV<lambda_319d5e083f45f90dcdce5dce53cbb275>@@D@Z 00000001400740e0     base64.obj
 0004:000010ec       $pdata$2$??$_Reallocate_grow_by@V<lambda_319d5e083f45f90dcdce5dce53cbb275>@@D@?$basic_string@DU?$char_traits@D@std@@V?$allocator@D@2@@std@@QEAAAEAV01@_KV<lambda_319d5e083f45f90dcdce5dce53cbb275>@@D@Z 00000001400740ec     base64.obj
 0004:000010f8       $pdata$3$??$_Reallocate_grow_by@V<lambda_319d5e083f45f90dcdce5dce53cbb275>@@D@?$basic_string@DU?$char_traits@D@std@@V?$allocator@D@2@@std@@QEAAAEAV01@_KV<lambda_319d5e083f45f90dcdce5dce53cbb275>@@D@Z 00000001400740f8     base64.obj
 0004:00001104       $pdata$?_Tidy@?$vector@V?$basic_string@DU?$char_traits@D@std@@V?$allocator@D@2@@std@@V?$allocator@V?$basic_string@DU?$char_traits@D@std@@V?$allocator@D@2@@std@@@2@@std@@AEAAXXZ 0000000140074104     CSmtp.obj
 0004:00001104       $pdata$??1?$vector@V?$basic_string@DU?$char_traits@D@std@@V?$allocator@D@2@@std@@V?$allocator@V?$basic_string@DU?$char_traits@D@std@@V?$allocator@D@2@@std@@@2@@std@@QEAA@XZ 0000000140074104     CSmtp.obj
 0004:00001110       $pdata$?deallocate@?$allocator@V?$basic_string@DU?$char_traits@D@std@@V?$allocator@D@2@@std@@@std@@QEAAXQEAV?$basic_string@DU?$char_traits@D@std@@V?$allocator@D@2@@2@_K@Z 0000000140074110     CSmtp.obj
 0004:0000111c       $pdata$??$?HDU?$char_traits@D@std@@V?$allocator@D@1@@std@@YA?AV?$basic_string@DU?$char_traits@D@std@@V?$allocator@D@2@@0@QEBDAEBV10@@Z 000000014007411c     CSmtp.obj
 0004:00001128       $pdata$??$_Traits_find@U?$char_traits@D@std@@@std@@YA_KQEBD_K101@Z 0000000140074128     CSmtp.obj
 0004:00001134       $pdata$??$_Destroy_range@V?$allocator@V?$basic_string@DU?$char_traits@D@std@@V?$allocator@D@2@@std@@@std@@@std@@YAXPEAV?$basic_string@DU?$char_traits@D@std@@V?$allocator@D@2@@0@0AEAV?$allocator@V?$basic_string@DU?$char_traits@D@std@@V?$allocator@D@2@@std@@@0@@Z 0000000140074134     CSmtp.obj
 0004:00001140       $pdata$0$??$_Destroy_range@V?$allocator@V?$basic_string@DU?$char_traits@D@std@@V?$allocator@D@2@@std@@@std@@@std@@YAXPEAV?$basic_string@DU?$char_traits@D@std@@V?$allocator@D@2@@0@0AEAV?$allocator@V?$basic_string@DU?$char_traits@D@std@@V?$allocator@D@2@@std@@@0@@Z 0000000140074140     CSmtp.obj
 0004:0000114c       $pdata$1$??$_Destroy_range@V?$allocator@V?$basic_string@DU?$char_traits@D@std@@V?$allocator@D@2@@std@@@std@@@std@@YAXPEAV?$basic_string@DU?$char_traits@D@std@@V?$allocator@D@2@@0@0AEAV?$allocator@V?$basic_string@DU?$char_traits@D@std@@V?$allocator@D@2@@std@@@0@@Z 000000014007414c     CSmtp.obj
 0004:00001158       $pdata$2$??$_Destroy_range@V?$allocator@V?$basic_string@DU?$char_traits@D@std@@V?$allocator@D@2@@std@@@std@@@std@@YAXPEAV?$basic_string@DU?$char_traits@D@std@@V?$allocator@D@2@@0@0AEAV?$allocator@V?$basic_string@DU?$char_traits@D@std@@V?$allocator@D@2@@std@@@0@@Z 0000000140074158     CSmtp.obj
 0004:00001164       $pdata$??0?$basic_string@DU?$char_traits@D@std@@V?$allocator@D@2@@std@@QEAA@AEBV01@@Z 0000000140074164     CSmtp.obj
 0004:00001170       $pdata$??1sentry@?$basic_ostream@DU?$char_traits@D@std@@@std@@QEAA@XZ 0000000140074170     md5_csmtp.obj
 0004:0000117c       $pdata$??1_Sentry_base@?$basic_ostream@DU?$char_traits@D@std@@@std@@QEAA@XZ 000000014007417c     md5_csmtp.obj
 0004:00001188       $pdata$??$?6U?$char_traits@D@std@@@std@@YAAEAV?$basic_ostream@DU?$char_traits@D@std@@@0@AEAV10@PEBD@Z 0000000140074188     md5_csmtp.obj
 0004:00001194       $pdata$??$endl@DU?$char_traits@D@std@@@std@@YAAEAV?$basic_ostream@DU?$char_traits@D@std@@@0@AEAV10@@Z 0000000140074194     md5_csmtp.obj
 0004:000011a0       $pdata$?a2toi@@YAHPEADHH@Z 00000001400741a0     DateTime.obj
 0004:000011ac       $pdata$0$?a2toi@@YAHPEADHH@Z 00000001400741ac     DateTime.obj
 0004:000011b8       $pdata$1$?a2toi@@YAHPEADHH@Z 00000001400741b8     DateTime.obj
 0004:000011c4       $pdata$2$?a2toi@@YAHPEADHH@Z 00000001400741c4     DateTime.obj
 0004:000011d0       $pdata$?Add@datetime@@QEAAXV1@@Z 00000001400741d0     DateTime.obj
 0004:000011dc       $pdata$?GetCurrentLocalTime@datetime@@QEAAXXZ 00000001400741dc     DateTime.obj
 0004:000011e8       $pdata$?regulate@datetime@@QEAAXXZ 00000001400741e8     DateTime.obj
 0004:000011f4       $pdata$?addcarry@datetime@@IEAAHAEAHHHH@Z 00000001400741f4     DateTime.obj
 0004:00001200       $pdata$?getDay@datetime@@IEAAHHH@Z 0000000140074200     DateTime.obj
 0004:0000120c       $pdata$??_GCHostStat@@UEAAPEAXI@Z 000000014007420c     HostStat.obj
 0004:00001218       $pdata$??1CHostStat@@UEAA@XZ 0000000140074218     HostStat.obj
 0004:00001224       $pdata$?setup@CHostStat@@QEAAXHH@Z 0000000140074224     HostStat.obj
 0004:00001230       $pdata$?thdMail@CHostStat@@KAIPEAX@Z 0000000140074230     HostStat.obj
 0004:0000123c       $pdata$?timer@CHostStat@@QEAAXXZ 000000014007423c     HostStat.obj
 0004:00001248       $pdata$?getData64@CHostStat@@QEAA_JGEEG@Z 0000000140074248     HostStat.obj
 0004:00001254       $pdata$?setData64@CHostStat@@QEAAXGEEG_J@Z 0000000140074254     HostStat.obj
 0004:00001260       $pdata$?addData@CHostStat@@QEAAXGEEG@Z 0000000140074260     HostStat.obj
 0004:0000126c       $pdata$?addExtraData@CHostStat@@QEAAXGE@Z 000000014007426c     HostStat.obj
 0004:00001278       $pdata$?addExtraData@CHostStat@@QEAAXGEEGIII@Z 0000000140074278     HostStat.obj
 0004:00001284       $pdata$?send@CHostStat@@IEAA_NPEAD0@Z 0000000140074284     HostStat.obj
 0004:00001290       $pdata$?timerPerfMem@CHostStat@@QEAAXXZ 0000000140074290     HostStat.obj
 0004:0000129c       $pdata$3$?timerPerfMem@CHostStat@@QEAAXXZ 000000014007429c     HostStat.obj
 0004:000012a8       $pdata$6$?timerPerfMem@CHostStat@@QEAAXXZ 00000001400742a8     HostStat.obj
 0004:000012b4       $pdata$7$?timerPerfMem@CHostStat@@QEAAXXZ 00000001400742b4     HostStat.obj
 0004:000012c0       $pdata$8$?timerPerfMem@CHostStat@@QEAAXXZ 00000001400742c0     HostStat.obj
 0004:000012cc       $pdata$9$?timerPerfMem@CHostStat@@QEAAXXZ 00000001400742cc     HostStat.obj
 0004:000012d8       $pdata$10$?timerPerfMem@CHostStat@@QEAAXXZ 00000001400742d8     HostStat.obj
 0004:000012e4       $pdata$?timerLogUser@CHostStat@@QEAAXHHHHH@Z 00000001400742e4     HostStat.obj
 0004:000012f0       $pdata$3$?timerLogUser@CHostStat@@QEAAXHHHHH@Z 00000001400742f0     HostStat.obj
 0004:000012fc       $pdata$4$?timerLogUser@CHostStat@@QEAAXHHHHH@Z 00000001400742fc     HostStat.obj
 0004:00001308       $pdata$?AddLog@CHostStat@@QEAAXPEBDZZ 0000000140074308     HostStat.obj
 0004:00001314       $pdata$4$?AddLog@CHostStat@@QEAAXPEBDZZ 0000000140074314     HostStat.obj
 0004:00001320       $pdata$5$?AddLog@CHostStat@@QEAAXPEBDZZ 0000000140074320     HostStat.obj
 0004:0000132c       $pdata$?GatherFiles@CHostStat@@QEAAXPEAD@Z 000000014007432c     HostStat.obj
 0004:00001338       $pdata$?GetDataFolder@CHostStat@@QEAAXPEAD_K@Z 0000000140074338     HostStat.obj
 0004:00001344       $pdata$?AddUserPCSpec@CHostStat@@QEAAXGPEBD00I@Z 0000000140074344     HostStat.obj
 0004:00001350       $pdata$5$?AddUserPCSpec@CHostStat@@QEAAXGPEBD00I@Z 0000000140074350     HostStat.obj
 0004:0000135c       $pdata$6$?AddUserPCSpec@CHostStat@@QEAAXGPEBD00I@Z 000000014007435c     HostStat.obj
 0004:00001368       $pdata$??$sprintf_s@$0CAA@@cf@@YAHAEAY0CAA@DPEBDZZ 0000000140074368     HostStat.obj
 0004:00001374       $pdata$??$_Buynode@U?$pair@GUExtraStatsMemVerify@CHostStat@@@std@@@?$_Tree_comp_alloc@V?$_Tmap_traits@GUExtraStatsMemVerify@CHostStat@@U?$less@G@std@@V?$allocator@U?$pair@$$CBGUExtraStatsMemVerify@CHostStat@@@std@@@4@$0A@@std@@@std@@QEAAPEAU?$_Tree_node@U?$pair@$$CBGUExtraStatsMemVerify@CHostStat@@@std@@PEAX@1@$$QEAU?$pair@GUExtraStatsMemVerify@CHostStat@@@1@@Z 0000000140074374     HostStat.obj
 0004:00001374       $pdata$??$_Buynode@U?$pair@GUExtraStatsFPSVerify@CHostStat@@@std@@@?$_Tree_comp_alloc@V?$_Tmap_traits@GUExtraStatsFPSVerify@CHostStat@@U?$less@G@std@@V?$allocator@U?$pair@$$CBGUExtraStatsFPSVerify@CHostStat@@@std@@@4@$0A@@std@@@std@@QEAAPEAU?$_Tree_node@U?$pair@$$CBGUExtraStatsFPSVerify@CHostStat@@@std@@PEAX@1@$$QEAU?$pair@GUExtraStatsFPSVerify@CHostStat@@@1@@Z 0000000140074374     HostStat.obj
 0004:00001380       $pdata$??$_Insert_nohint@AEAU?$pair@$$CBGUExtraStatsMemVerify@CHostStat@@@std@@PEAU?$_Tree_node@U?$pair@$$CBGUExtraStatsMemVerify@CHostStat@@@std@@PEAX@2@@?$_Tree@V?$_Tmap_traits@GUExtraStatsMemVerify@CHostStat@@U?$less@G@std@@V?$allocator@U?$pair@$$CBGUExtraStatsMemVerify@CHostStat@@@std@@@4@$0A@@std@@@std@@IEAA?AU?$pair@V?$_Tree_iterator@V?$_Tree_val@U?$_Tree_simple_types@U?$pair@$$CBGUExtraStatsMemVerify@CHostStat@@@std@@@std@@@std@@@std@@_N@1@_NAEAU?$pair@$$CBGUExtraStatsMemVerify@CHostStat@@@1@PEAU?$_Tree_node@U?$pair@$$CBGUExtraStatsMemVerify@CHostStat@@@std@@PEAX@1@@Z 0000000140074380     HostStat.obj
 0004:00001380       $pdata$??$_Insert_nohint@AEAU?$pair@$$CBGUExtraStatsFPSVerify@CHostStat@@@std@@PEAU?$_Tree_node@U?$pair@$$CBGUExtraStatsFPSVerify@CHostStat@@@std@@PEAX@2@@?$_Tree@V?$_Tmap_traits@GUExtraStatsFPSVerify@CHostStat@@U?$less@G@std@@V?$allocator@U?$pair@$$CBGUExtraStatsFPSVerify@CHostStat@@@std@@@4@$0A@@std@@@std@@IEAA?AU?$pair@V?$_Tree_iterator@V?$_Tree_val@U?$_Tree_simple_types@U?$pair@$$CBGUExtraStatsFPSVerify@CHostStat@@@std@@@std@@@std@@@std@@_N@1@_NAEAU?$pair@$$CBGUExtraStatsFPSVerify@CHostStat@@@1@PEAU?$_Tree_node@U?$pair@$$CBGUExtraStatsFPSVerify@CHostStat@@@std@@PEAX@1@@Z 0000000140074380     HostStat.obj
 0004:0000138c       $pdata$?_Buynode0@?$_Tree_comp_alloc@V?$_Tmap_traits@GUExtraStatsFPSVerify@CHostStat@@U?$less@G@std@@V?$allocator@U?$pair@$$CBGUExtraStatsFPSVerify@CHostStat@@@std@@@4@$0A@@std@@@std@@QEAAPEAU?$_Tree_node@U?$pair@$$CBGUExtraStatsFPSVerify@CHostStat@@@std@@PEAX@2@XZ 000000014007438c     HostStat.obj
 0004:0000138c       $pdata$?_Buynode0@?$_Tree_comp_alloc@V?$_Tmap_traits@GUExtraStatsMemVerify@CHostStat@@U?$less@G@std@@V?$allocator@U?$pair@$$CBGUExtraStatsMemVerify@CHostStat@@@std@@@4@$0A@@std@@@std@@QEAAPEAU?$_Tree_node@U?$pair@$$CBGUExtraStatsMemVerify@CHostStat@@@std@@PEAX@2@XZ 000000014007438c     HostStat.obj
 0004:00001398       $pdata$??$_Insert_at@AEAU?$pair@$$CBGUExtraStatsFPSVerify@CHostStat@@@std@@PEAU?$_Tree_node@U?$pair@$$CBGUExtraStatsFPSVerify@CHostStat@@@std@@PEAX@2@@?$_Tree@V?$_Tmap_traits@GUExtraStatsFPSVerify@CHostStat@@U?$less@G@std@@V?$allocator@U?$pair@$$CBGUExtraStatsFPSVerify@CHostStat@@@std@@@4@$0A@@std@@@std@@IEAA?AV?$_Tree_iterator@V?$_Tree_val@U?$_Tree_simple_types@U?$pair@$$CBGUExtraStatsFPSVerify@CHostStat@@@std@@@std@@@std@@@1@_NPEAU?$_Tree_node@U?$pair@$$CBGUExtraStatsFPSVerify@CHostStat@@@std@@PEAX@1@AEAU?$pair@$$CBGUExtraStatsFPSVerify@CHostStat@@@1@1@Z 0000000140074398     HostStat.obj
 0004:00001398       $pdata$??$_Insert_at@AEAU?$pair@$$CBGUExtraStatsMemVerify@CHostStat@@@std@@PEAU?$_Tree_node@U?$pair@$$CBGUExtraStatsMemVerify@CHostStat@@@std@@PEAX@2@@?$_Tree@V?$_Tmap_traits@GUExtraStatsMemVerify@CHostStat@@U?$less@G@std@@V?$allocator@U?$pair@$$CBGUExtraStatsMemVerify@CHostStat@@@std@@@4@$0A@@std@@@std@@IEAA?AV?$_Tree_iterator@V?$_Tree_val@U?$_Tree_simple_types@U?$pair@$$CBGUExtraStatsMemVerify@CHostStat@@@std@@@std@@@std@@@1@_NPEAU?$_Tree_node@U?$pair@$$CBGUExtraStatsMemVerify@CHostStat@@@std@@PEAX@1@AEAU?$pair@$$CBGUExtraStatsMemVerify@CHostStat@@@1@1@Z 0000000140074398     HostStat.obj
 0004:000013a4       $pdata$?write@CIniSection@CIniReader@@QEAAKPEAX@Z 00000001400743a4     iniReader.obj
 0004:000013b0       $pdata$?setString@CIniSection@CIniReader@@QEAAXPEBD0@Z 00000001400743b0     iniReader.obj
 0004:000013bc       $pdata$?getString@CIniSection@CIniReader@@QEAA_KPEBDPEAD_K@Z 00000001400743bc     iniReader.obj
 0004:000013c8       $pdata$0$?getString@CIniSection@CIniReader@@QEAA_KPEBDPEAD_K@Z 00000001400743c8     iniReader.obj
 0004:000013d4       $pdata$1$?getString@CIniSection@CIniReader@@QEAA_KPEBDPEAD_K@Z 00000001400743d4     iniReader.obj
 0004:000013e0       $pdata$??1CIniReader@@QEAA@XZ 00000001400743e0     iniReader.obj
 0004:000013ec       $pdata$?clear@CIniReader@@QEAAXXZ 00000001400743ec     iniReader.obj
 0004:000013f8       $pdata$?read@CIniReader@@QEAAKPEBD@Z 00000001400743f8     iniReader.obj
 0004:00001404       $pdata$2$?read@CIniReader@@QEAAKPEBD@Z 0000000140074404     iniReader.obj
 0004:00001410       $pdata$3$?read@CIniReader@@QEAAKPEBD@Z 0000000140074410     iniReader.obj
 0004:0000141c       $pdata$4$?read@CIniReader@@QEAAKPEBD@Z 000000014007441c     iniReader.obj
 0004:00001428       $pdata$5$?read@CIniReader@@QEAAKPEBD@Z 0000000140074428     iniReader.obj
 0004:00001434       $pdata$?write@CIniReader@@QEAAKPEBD@Z 0000000140074434     iniReader.obj
 0004:00001440       $pdata$?parse@CIniReader@@QEAAKPEBD@Z 0000000140074440     iniReader.obj
 0004:0000144c       $pdata$?getInt@CIniReader@@QEAAHPEBD0H@Z 000000014007444c     iniReader.obj
 0004:00001458       $pdata$?getString@CIniReader@@QEAA_KPEBD0PEAD_K@Z 0000000140074458     iniReader.obj
 0004:00001464       $pdata$?getIntArray@CIniReader@@QEAA_KPEBD0PEAH_K@Z 0000000140074464     iniReader.obj
 0004:00001470       $pdata$1$?getIntArray@CIniReader@@QEAA_KPEBD0PEAH_K@Z 0000000140074470     iniReader.obj
 0004:0000147c       $pdata$2$?getIntArray@CIniReader@@QEAA_KPEBD0PEAH_K@Z 000000014007447c     iniReader.obj
 0004:00001488       $pdata$3$?getIntArray@CIniReader@@QEAA_KPEBD0PEAH_K@Z 0000000140074488     iniReader.obj
 0004:00001494       $pdata$?setString@CIniReader@@QEAAXPEBD00@Z 0000000140074494     iniReader.obj
 0004:000014a0       $pdata$?find@?$_Tree@V?$_Tmap_traits@V?$basic_string@DU?$char_traits@D@std@@V?$allocator@D@2@@std@@PEAVCIniSection@CIniReader@@U?$less@V?$basic_string@DU?$char_traits@D@std@@V?$allocator@D@2@@std@@@2@V?$allocator@U?$pair@$$CBV?$basic_string@DU?$char_traits@D@std@@V?$allocator@D@2@@std@@PEAVCIniSection@CIniReader@@@std@@@2@$0A@@std@@@std@@QEAA?AV?$_Tree_iterator@V?$_Tree_val@U?$_Tree_simple_types@U?$pair@$$CBV?$basic_string@DU?$char_traits@D@std@@V?$allocator@D@2@@std@@PEAVCIniSection@CIniReader@@@std@@@std@@@std@@@2@AEBV?$basic_string@DU?$char_traits@D@std@@V?$allocator@D@2@@2@@Z 00000001400744a0     iniReader.obj
 0004:000014ac       $pdata$1$?find@?$_Tree@V?$_Tmap_traits@V?$basic_string@DU?$char_traits@D@std@@V?$allocator@D@2@@std@@PEAVCIniSection@CIniReader@@U?$less@V?$basic_string@DU?$char_traits@D@std@@V?$allocator@D@2@@std@@@2@V?$allocator@U?$pair@$$CBV?$basic_string@DU?$char_traits@D@std@@V?$allocator@D@2@@std@@PEAVCIniSection@CIniReader@@@std@@@2@$0A@@std@@@std@@QEAA?AV?$_Tree_iterator@V?$_Tree_val@U?$_Tree_simple_types@U?$pair@$$CBV?$basic_string@DU?$char_traits@D@std@@V?$allocator@D@2@@std@@PEAVCIniSection@CIniReader@@@std@@@std@@@std@@@2@AEBV?$basic_string@DU?$char_traits@D@std@@V?$allocator@D@2@@2@@Z 00000001400744ac     iniReader.obj
 0004:000014b8       $pdata$2$?find@?$_Tree@V?$_Tmap_traits@V?$basic_string@DU?$char_traits@D@std@@V?$allocator@D@2@@std@@PEAVCIniSection@CIniReader@@U?$less@V?$basic_string@DU?$char_traits@D@std@@V?$allocator@D@2@@std@@@2@V?$allocator@U?$pair@$$CBV?$basic_string@DU?$char_traits@D@std@@V?$allocator@D@2@@std@@PEAVCIniSection@CIniReader@@@std@@@2@$0A@@std@@@std@@QEAA?AV?$_Tree_iterator@V?$_Tree_val@U?$_Tree_simple_types@U?$pair@$$CBV?$basic_string@DU?$char_traits@D@std@@V?$allocator@D@2@@std@@PEAVCIniSection@CIniReader@@@std@@@std@@@std@@@2@AEBV?$basic_string@DU?$char_traits@D@std@@V?$allocator@D@2@@2@@Z 00000001400744b8     iniReader.obj
 0004:000014c4       $pdata$3$?find@?$_Tree@V?$_Tmap_traits@V?$basic_string@DU?$char_traits@D@std@@V?$allocator@D@2@@std@@PEAVCIniSection@CIniReader@@U?$less@V?$basic_string@DU?$char_traits@D@std@@V?$allocator@D@2@@std@@@2@V?$allocator@U?$pair@$$CBV?$basic_string@DU?$char_traits@D@std@@V?$allocator@D@2@@std@@PEAVCIniSection@CIniReader@@@std@@@2@$0A@@std@@@std@@QEAA?AV?$_Tree_iterator@V?$_Tree_val@U?$_Tree_simple_types@U?$pair@$$CBV?$basic_string@DU?$char_traits@D@std@@V?$allocator@D@2@@std@@PEAVCIniSection@CIniReader@@@std@@@std@@@std@@@2@AEBV?$basic_string@DU?$char_traits@D@std@@V?$allocator@D@2@@2@@Z 00000001400744c4     iniReader.obj
 0004:000014d0       $pdata$4$?find@?$_Tree@V?$_Tmap_traits@V?$basic_string@DU?$char_traits@D@std@@V?$allocator@D@2@@std@@PEAVCIniSection@CIniReader@@U?$less@V?$basic_string@DU?$char_traits@D@std@@V?$allocator@D@2@@std@@@2@V?$allocator@U?$pair@$$CBV?$basic_string@DU?$char_traits@D@std@@V?$allocator@D@2@@std@@PEAVCIniSection@CIniReader@@@std@@@2@$0A@@std@@@std@@QEAA?AV?$_Tree_iterator@V?$_Tree_val@U?$_Tree_simple_types@U?$pair@$$CBV?$basic_string@DU?$char_traits@D@std@@V?$allocator@D@2@@std@@PEAVCIniSection@CIniReader@@@std@@@std@@@std@@@2@AEBV?$basic_string@DU?$char_traits@D@std@@V?$allocator@D@2@@2@@Z 00000001400744d0     iniReader.obj
 0004:000014dc       $pdata$?_Erase@?$_Tree@V?$_Tmap_traits@V?$basic_string@DU?$char_traits@D@std@@V?$allocator@D@2@@std@@PEAVCIniSection@CIniReader@@U?$less@V?$basic_string@DU?$char_traits@D@std@@V?$allocator@D@2@@std@@@2@V?$allocator@U?$pair@$$CBV?$basic_string@DU?$char_traits@D@std@@V?$allocator@D@2@@std@@PEAVCIniSection@CIniReader@@@std@@@2@$0A@@std@@@std@@IEAAXPEAU?$_Tree_node@U?$pair@$$CBV?$basic_string@DU?$char_traits@D@std@@V?$allocator@D@2@@std@@PEAVCIniSection@CIniReader@@@std@@PEAX@2@@Z 00000001400744dc     iniReader.obj
 0004:000014e8       $pdata$0$?_Erase@?$_Tree@V?$_Tmap_traits@V?$basic_string@DU?$char_traits@D@std@@V?$allocator@D@2@@std@@PEAVCIniSection@CIniReader@@U?$less@V?$basic_string@DU?$char_traits@D@std@@V?$allocator@D@2@@std@@@2@V?$allocator@U?$pair@$$CBV?$basic_string@DU?$char_traits@D@std@@V?$allocator@D@2@@std@@PEAVCIniSection@CIniReader@@@std@@@2@$0A@@std@@@std@@IEAAXPEAU?$_Tree_node@U?$pair@$$CBV?$basic_string@DU?$char_traits@D@std@@V?$allocator@D@2@@std@@PEAVCIniSection@CIniReader@@@std@@PEAX@2@@Z 00000001400744e8     iniReader.obj
 0004:000014f4       $pdata$1$?_Erase@?$_Tree@V?$_Tmap_traits@V?$basic_string@DU?$char_traits@D@std@@V?$allocator@D@2@@std@@PEAVCIniSection@CIniReader@@U?$less@V?$basic_string@DU?$char_traits@D@std@@V?$allocator@D@2@@std@@@2@V?$allocator@U?$pair@$$CBV?$basic_string@DU?$char_traits@D@std@@V?$allocator@D@2@@std@@PEAVCIniSection@CIniReader@@@std@@@2@$0A@@std@@@std@@IEAAXPEAU?$_Tree_node@U?$pair@$$CBV?$basic_string@DU?$char_traits@D@std@@V?$allocator@D@2@@std@@PEAVCIniSection@CIniReader@@@std@@PEAX@2@@Z 00000001400744f4     iniReader.obj
 0004:00001500       $pdata$2$?_Erase@?$_Tree@V?$_Tmap_traits@V?$basic_string@DU?$char_traits@D@std@@V?$allocator@D@2@@std@@PEAVCIniSection@CIniReader@@U?$less@V?$basic_string@DU?$char_traits@D@std@@V?$allocator@D@2@@std@@@2@V?$allocator@U?$pair@$$CBV?$basic_string@DU?$char_traits@D@std@@V?$allocator@D@2@@std@@PEAVCIniSection@CIniReader@@@std@@@2@$0A@@std@@@std@@IEAAXPEAU?$_Tree_node@U?$pair@$$CBV?$basic_string@DU?$char_traits@D@std@@V?$allocator@D@2@@std@@PEAVCIniSection@CIniReader@@@std@@PEAX@2@@Z 0000000140074500     iniReader.obj
 0004:0000150c       $pdata$?lower_bound@?$_Tree@V?$_Tmap_traits@V?$basic_string@DU?$char_traits@D@std@@V?$allocator@D@2@@std@@V12@U?$less@V?$basic_string@DU?$char_traits@D@std@@V?$allocator@D@2@@std@@@2@V?$allocator@U?$pair@$$CBV?$basic_string@DU?$char_traits@D@std@@V?$allocator@D@2@@std@@V12@@std@@@2@$0A@@std@@@std@@QEAA?AV?$_Tree_iterator@V?$_Tree_val@U?$_Tree_simple_types@U?$pair@$$CBV?$basic_string@DU?$char_traits@D@std@@V?$allocator@D@2@@std@@V12@@std@@@std@@@std@@@2@AEBV?$basic_string@DU?$char_traits@D@std@@V?$allocator@D@2@@2@@Z 000000014007450c     iniReader.obj
 0004:00001518       $pdata$2$?lower_bound@?$_Tree@V?$_Tmap_traits@V?$basic_string@DU?$char_traits@D@std@@V?$allocator@D@2@@std@@V12@U?$less@V?$basic_string@DU?$char_traits@D@std@@V?$allocator@D@2@@std@@@2@V?$allocator@U?$pair@$$CBV?$basic_string@DU?$char_traits@D@std@@V?$allocator@D@2@@std@@V12@@std@@@2@$0A@@std@@@std@@QEAA?AV?$_Tree_iterator@V?$_Tree_val@U?$_Tree_simple_types@U?$pair@$$CBV?$basic_string@DU?$char_traits@D@std@@V?$allocator@D@2@@std@@V12@@std@@@std@@@std@@@2@AEBV?$basic_string@DU?$char_traits@D@std@@V?$allocator@D@2@@2@@Z 0000000140074518     iniReader.obj
 0004:00001524       $pdata$4$?lower_bound@?$_Tree@V?$_Tmap_traits@V?$basic_string@DU?$char_traits@D@std@@V?$allocator@D@2@@std@@V12@U?$less@V?$basic_string@DU?$char_traits@D@std@@V?$allocator@D@2@@std@@@2@V?$allocator@U?$pair@$$CBV?$basic_string@DU?$char_traits@D@std@@V?$allocator@D@2@@std@@V12@@std@@@2@$0A@@std@@@std@@QEAA?AV?$_Tree_iterator@V?$_Tree_val@U?$_Tree_simple_types@U?$pair@$$CBV?$basic_string@DU?$char_traits@D@std@@V?$allocator@D@2@@std@@V12@@std@@@std@@@std@@@2@AEBV?$basic_string@DU?$char_traits@D@std@@V?$allocator@D@2@@2@@Z 0000000140074524     iniReader.obj
 0004:00001530       $pdata$5$?lower_bound@?$_Tree@V?$_Tmap_traits@V?$basic_string@DU?$char_traits@D@std@@V?$allocator@D@2@@std@@V12@U?$less@V?$basic_string@DU?$char_traits@D@std@@V?$allocator@D@2@@std@@@2@V?$allocator@U?$pair@$$CBV?$basic_string@DU?$char_traits@D@std@@V?$allocator@D@2@@std@@V12@@std@@@2@$0A@@std@@@std@@QEAA?AV?$_Tree_iterator@V?$_Tree_val@U?$_Tree_simple_types@U?$pair@$$CBV?$basic_string@DU?$char_traits@D@std@@V?$allocator@D@2@@std@@V12@@std@@@std@@@std@@@2@AEBV?$basic_string@DU?$char_traits@D@std@@V?$allocator@D@2@@2@@Z 0000000140074530     iniReader.obj
 0004:0000153c       $pdata$?erase@?$_Tree@V?$_Tmap_traits@V?$basic_string@DU?$char_traits@D@std@@V?$allocator@D@2@@std@@PEAVCIniSection@CIniReader@@U?$less@V?$basic_string@DU?$char_traits@D@std@@V?$allocator@D@2@@std@@@2@V?$allocator@U?$pair@$$CBV?$basic_string@DU?$char_traits@D@std@@V?$allocator@D@2@@std@@PEAVCIniSection@CIniReader@@@std@@@2@$0A@@std@@@std@@QEAA?AV?$_Tree_iterator@V?$_Tree_val@U?$_Tree_simple_types@U?$pair@$$CBV?$basic_string@DU?$char_traits@D@std@@V?$allocator@D@2@@std@@PEAVCIniSection@CIniReader@@@std@@@std@@@std@@@2@V?$_Tree_const_iterator@V?$_Tree_val@U?$_Tree_simple_types@U?$pair@$$CBV?$basic_string@DU?$char_traits@D@std@@V?$allocator@D@2@@std@@PEAVCIniSection@CIniReader@@@std@@@std@@@std@@@2@0@Z 000000014007453c     iniReader.obj
 0004:00001548       $pdata$?erase@?$_Tree@V?$_Tmap_traits@V?$basic_string@DU?$char_traits@D@std@@V?$allocator@D@2@@std@@V12@U?$less@V?$basic_string@DU?$char_traits@D@std@@V?$allocator@D@2@@std@@@2@V?$allocator@U?$pair@$$CBV?$basic_string@DU?$char_traits@D@std@@V?$allocator@D@2@@std@@V12@@std@@@2@$0A@@std@@@std@@QEAA?AV?$_Tree_iterator@V?$_Tree_val@U?$_Tree_simple_types@U?$pair@$$CBV?$basic_string@DU?$char_traits@D@std@@V?$allocator@D@2@@std@@V12@@std@@@std@@@std@@@2@V?$_Tree_const_iterator@V?$_Tree_val@U?$_Tree_simple_types@U?$pair@$$CBV?$basic_string@DU?$char_traits@D@std@@V?$allocator@D@2@@std@@V12@@std@@@std@@@std@@@2@0@Z 0000000140074548     iniReader.obj
 0004:00001554       $pdata$?_Extract@?$_Tree_val@U?$_Tree_simple_types@U?$pair@$$CBV?$basic_string@DU?$char_traits@D@std@@V?$allocator@D@2@@std@@V12@@std@@@std@@@std@@QEAAPEAU?$_Tree_node@U?$pair@$$CBV?$basic_string@DU?$char_traits@D@std@@V?$allocator@D@2@@std@@V12@@std@@PEAX@2@V?$_Tree_const_iterator@V?$_Tree_val@U?$_Tree_simple_types@U?$pair@$$CBV?$basic_string@DU?$char_traits@D@std@@V?$allocator@D@2@@std@@V12@@std@@@std@@@std@@@2@@Z 0000000140074554     iniReader.obj
 0004:00001554       $pdata$?_Extract@?$_Tree_val@U?$_Tree_simple_types@U?$pair@$$CBV?$basic_string@DU?$char_traits@D@std@@V?$allocator@D@2@@std@@PEAVCIniSection@CIniReader@@@std@@@std@@@std@@QEAAPEAU?$_Tree_node@U?$pair@$$CBV?$basic_string@DU?$char_traits@D@std@@V?$allocator@D@2@@std@@PEAVCIniSection@CIniReader@@@std@@PEAX@2@V?$_Tree_const_iterator@V?$_Tree_val@U?$_Tree_simple_types@U?$pair@$$CBV?$basic_string@DU?$char_traits@D@std@@V?$allocator@D@2@@std@@PEAVCIniSection@CIniReader@@@std@@@std@@@std@@@2@@Z 0000000140074554     iniReader.obj
 0004:00001554       $pdata$?_Extract@?$_Tree_val@U?$_Tree_simple_types@U?$pair@$$CB_JV?$basic_string@DU?$char_traits@D@std@@V?$allocator@D@2@@std@@@std@@@std@@@std@@QEAAPEAU?$_Tree_node@U?$pair@$$CB_JV?$basic_string@DU?$char_traits@D@std@@V?$allocator@D@2@@std@@@std@@PEAX@2@V?$_Tree_const_iterator@V?$_Tree_val@U?$_Tree_simple_types@U?$pair@$$CB_JV?$basic_string@DU?$char_traits@D@std@@V?$allocator@D@2@@std@@@std@@@std@@@std@@@2@@Z 0000000140074554     LoadXlsMsg.obj
 0004:00001560       $pdata$?_Buyheadnode@?$_Tree_comp_alloc@V?$_Tmap_traits@_JV?$basic_string@DU?$char_traits@D@std@@V?$allocator@D@2@@std@@U?$less@_J@2@V?$allocator@U?$pair@$$CB_JV?$basic_string@DU?$char_traits@D@std@@V?$allocator@D@2@@std@@@std@@@2@$0A@@std@@@std@@QEAAPEAU?$_Tree_node@U?$pair@$$CB_JV?$basic_string@DU?$char_traits@D@std@@V?$allocator@D@2@@std@@@std@@PEAX@2@XZ 0000000140074560     LoadXlsMsg.obj
 0004:00001560       $pdata$?_Buyheadnode@?$_Tree_comp_alloc@V?$_Tmap_traits@V?$basic_string@DU?$char_traits@D@std@@V?$allocator@D@2@@std@@PEAVCIniSection@CIniReader@@U?$less@V?$basic_string@DU?$char_traits@D@std@@V?$allocator@D@2@@std@@@2@V?$allocator@U?$pair@$$CBV?$basic_string@DU?$char_traits@D@std@@V?$allocator@D@2@@std@@PEAVCIniSection@CIniReader@@@std@@@2@$0A@@std@@@std@@QEAAPEAU?$_Tree_node@U?$pair@$$CBV?$basic_string@DU?$char_traits@D@std@@V?$allocator@D@2@@std@@PEAVCIniSection@CIniReader@@@std@@PEAX@2@XZ 0000000140074560     iniReader.obj
 0004:0000156c       $pdata$?_Buyheadnode@?$_Tree_comp_alloc@V?$_Tmap_traits@V?$basic_string@DU?$char_traits@D@std@@V?$allocator@D@2@@std@@V12@U?$less@V?$basic_string@DU?$char_traits@D@std@@V?$allocator@D@2@@std@@@2@V?$allocator@U?$pair@$$CBV?$basic_string@DU?$char_traits@D@std@@V?$allocator@D@2@@std@@V12@@std@@@2@$0A@@std@@@std@@QEAAPEAU?$_Tree_node@U?$pair@$$CBV?$basic_string@DU?$char_traits@D@std@@V?$allocator@D@2@@std@@V12@@std@@PEAX@2@XZ 000000014007456c     iniReader.obj
 0004:00001578       $pdata$?_Erase@?$_Tree@V?$_Tmap_traits@V?$basic_string@DU?$char_traits@D@std@@V?$allocator@D@2@@std@@V12@U?$less@V?$basic_string@DU?$char_traits@D@std@@V?$allocator@D@2@@std@@@2@V?$allocator@U?$pair@$$CBV?$basic_string@DU?$char_traits@D@std@@V?$allocator@D@2@@std@@V12@@std@@@2@$0A@@std@@@std@@IEAAXPEAU?$_Tree_node@U?$pair@$$CBV?$basic_string@DU?$char_traits@D@std@@V?$allocator@D@2@@std@@V12@@std@@PEAX@2@@Z 0000000140074578     iniReader.obj
 0004:00001584       $pdata$??$?HDU?$char_traits@D@std@@V?$allocator@D@1@@std@@YA?AV?$basic_string@DU?$char_traits@D@std@@V?$allocator@D@2@@0@$$QEAV10@QEBD@Z 0000000140074584     iniReader.obj
 0004:00001590       $pdata$??1?$pair@$$CBV?$basic_string@DU?$char_traits@D@std@@V?$allocator@D@2@@std@@V12@@std@@QEAA@XZ 0000000140074590     iniReader.obj
 0004:00001590       $pdata$??1Address@mailer@jwsmtp@@QEAA@XZ 0000000140074590     mailer.obj
 0004:0000159c       $pdata$??$_Buynode@U?$pair@PEADPEAVCIniSection@CIniReader@@@std@@@?$_Tree_comp_alloc@V?$_Tmap_traits@V?$basic_string@DU?$char_traits@D@std@@V?$allocator@D@2@@std@@PEAVCIniSection@CIniReader@@U?$less@V?$basic_string@DU?$char_traits@D@std@@V?$allocator@D@2@@std@@@2@V?$allocator@U?$pair@$$CBV?$basic_string@DU?$char_traits@D@std@@V?$allocator@D@2@@std@@PEAVCIniSection@CIniReader@@@std@@@2@$0A@@std@@@std@@QEAAPEAU?$_Tree_node@U?$pair@$$CBV?$basic_string@DU?$char_traits@D@std@@V?$allocator@D@2@@std@@PEAVCIniSection@CIniReader@@@std@@PEAX@1@$$QEAU?$pair@PEADPEAVCIniSection@CIniReader@@@1@@Z 000000014007459c     iniReader.obj
 0004:000015a8       $pdata$??$_Insert_nohint@AEAU?$pair@$$CBV?$basic_string@DU?$char_traits@D@std@@V?$allocator@D@2@@std@@PEAVCIniSection@CIniReader@@@std@@PEAU?$_Tree_node@U?$pair@$$CBV?$basic_string@DU?$char_traits@D@std@@V?$allocator@D@2@@std@@PEAVCIniSection@CIniReader@@@std@@PEAX@2@@?$_Tree@V?$_Tmap_traits@V?$basic_string@DU?$char_traits@D@std@@V?$allocator@D@2@@std@@PEAVCIniSection@CIniReader@@U?$less@V?$basic_string@DU?$char_traits@D@std@@V?$allocator@D@2@@std@@@2@V?$allocator@U?$pair@$$CBV?$basic_string@DU?$char_traits@D@std@@V?$allocator@D@2@@std@@PEAVCIniSection@CIniReader@@@std@@@2@$0A@@std@@@std@@IEAA?AU?$pair@V?$_Tree_iterator@V?$_Tree_val@U?$_Tree_simple_types@U?$pair@$$CBV?$basic_string@DU?$char_traits@D@std@@V?$allocator@D@2@@std@@PEAVCIniSection@CIniReader@@@std@@@std@@@std@@@std@@_N@1@_NAEAU?$pair@$$CBV?$basic_string@DU?$char_traits@D@std@@V?$allocator@D@2@@std@@PEAVCIniSection@CIniReader@@@1@PEAU?$_Tree_node@U?$pair@$$CBV?$basic_string@DU?$char_traits@D@std@@V?$allocator@D@2@@std@@PEAVCIniSection@CIniReader@@@std@@PEAX@1@@Z 00000001400745a8     iniReader.obj
 0004:000015b4       $pdata$?_Buynode0@?$_Tree_comp_alloc@V?$_Tmap_traits@_JV?$basic_string@DU?$char_traits@D@std@@V?$allocator@D@2@@std@@U?$less@_J@2@V?$allocator@U?$pair@$$CB_JV?$basic_string@DU?$char_traits@D@std@@V?$allocator@D@2@@std@@@std@@@2@$0A@@std@@@std@@QEAAPEAU?$_Tree_node@U?$pair@$$CB_JV?$basic_string@DU?$char_traits@D@std@@V?$allocator@D@2@@std@@@std@@PEAX@2@XZ 00000001400745b4     LoadXlsMsg.obj
 0004:000015b4       $pdata$?_Buynode0@?$_Tree_comp_alloc@V?$_Tmap_traits@V?$basic_string@DU?$char_traits@D@std@@V?$allocator@D@2@@std@@PEAVCIniSection@CIniReader@@U?$less@V?$basic_string@DU?$char_traits@D@std@@V?$allocator@D@2@@std@@@2@V?$allocator@U?$pair@$$CBV?$basic_string@DU?$char_traits@D@std@@V?$allocator@D@2@@std@@PEAVCIniSection@CIniReader@@@std@@@2@$0A@@std@@@std@@QEAAPEAU?$_Tree_node@U?$pair@$$CBV?$basic_string@DU?$char_traits@D@std@@V?$allocator@D@2@@std@@PEAVCIniSection@CIniReader@@@std@@PEAX@2@XZ 00000001400745b4     iniReader.obj
 0004:000015c0       $pdata$?_Destroy_if_node@?$_Tree@V?$_Tmap_traits@V?$basic_string@DU?$char_traits@D@std@@V?$allocator@D@2@@std@@PEAVCIniSection@CIniReader@@U?$less@V?$basic_string@DU?$char_traits@D@std@@V?$allocator@D@2@@std@@@2@V?$allocator@U?$pair@$$CBV?$basic_string@DU?$char_traits@D@std@@V?$allocator@D@2@@std@@PEAVCIniSection@CIniReader@@@std@@@2@$0A@@std@@@std@@IEAAXPEAU?$_Tree_node@U?$pair@$$CBV?$basic_string@DU?$char_traits@D@std@@V?$allocator@D@2@@std@@PEAVCIniSection@CIniReader@@@std@@PEAX@2@@Z 00000001400745c0     iniReader.obj
 0004:000015cc       $pdata$??$_Insert_at@AEAU?$pair@$$CBV?$basic_string@DU?$char_traits@D@std@@V?$allocator@D@2@@std@@PEAVCIniSection@CIniReader@@@std@@PEAU?$_Tree_node@U?$pair@$$CBV?$basic_string@DU?$char_traits@D@std@@V?$allocator@D@2@@std@@PEAVCIniSection@CIniReader@@@std@@PEAX@2@@?$_Tree@V?$_Tmap_traits@V?$basic_string@DU?$char_traits@D@std@@V?$allocator@D@2@@std@@PEAVCIniSection@CIniReader@@U?$less@V?$basic_string@DU?$char_traits@D@std@@V?$allocator@D@2@@std@@@2@V?$allocator@U?$pair@$$CBV?$basic_string@DU?$char_traits@D@std@@V?$allocator@D@2@@std@@PEAVCIniSection@CIniReader@@@std@@@2@$0A@@std@@@std@@IEAA?AV?$_Tree_iterator@V?$_Tree_val@U?$_Tree_simple_types@U?$pair@$$CBV?$basic_string@DU?$char_traits@D@std@@V?$allocator@D@2@@std@@PEAVCIniSection@CIniReader@@@std@@@std@@@std@@@1@_NPEAU?$_Tree_node@U?$pair@$$CBV?$basic_string@DU?$char_traits@D@std@@V?$allocator@D@2@@std@@PEAVCIniSection@CIniReader@@@std@@PEAX@1@AEAU?$pair@$$CBV?$basic_string@DU?$char_traits@D@std@@V?$allocator@D@2@@std@@PEAVCIniSection@CIniReader@@@1@1@Z 00000001400745cc     iniReader.obj
 0004:000015d8       $pdata$??$_Buynode@AEBUpiecewise_construct_t@std@@V?$tuple@$$QEAV?$basic_string@DU?$char_traits@D@std@@V?$allocator@D@2@@std@@@2@V?$tuple@$$V@2@@?$_Tree_comp_alloc@V?$_Tmap_traits@V?$basic_string@DU?$char_traits@D@std@@V?$allocator@D@2@@std@@V12@U?$less@V?$basic_string@DU?$char_traits@D@std@@V?$allocator@D@2@@std@@@2@V?$allocator@U?$pair@$$CBV?$basic_string@DU?$char_traits@D@std@@V?$allocator@D@2@@std@@V12@@std@@@2@$0A@@std@@@std@@QEAAPEAU?$_Tree_node@U?$pair@$$CBV?$basic_string@DU?$char_traits@D@std@@V?$allocator@D@2@@std@@V12@@std@@PEAX@1@AEBUpiecewise_construct_t@1@$$QEAV?$tuple@$$QEAV?$basic_string@DU?$char_traits@D@std@@V?$allocator@D@2@@std@@@1@$$QEAV?$tuple@$$V@1@@Z 00000001400745d8     iniReader.obj
 0004:000015e4       $pdata$??$_Insert_hint@AEAU?$pair@$$CBV?$basic_string@DU?$char_traits@D@std@@V?$allocator@D@2@@std@@V12@@std@@PEAU?$_Tree_node@U?$pair@$$CBV?$basic_string@DU?$char_traits@D@std@@V?$allocator@D@2@@std@@V12@@std@@PEAX@2@@?$_Tree@V?$_Tmap_traits@V?$basic_string@DU?$char_traits@D@std@@V?$allocator@D@2@@std@@V12@U?$less@V?$basic_string@DU?$char_traits@D@std@@V?$allocator@D@2@@std@@@2@V?$allocator@U?$pair@$$CBV?$basic_string@DU?$char_traits@D@std@@V?$allocator@D@2@@std@@V12@@std@@@2@$0A@@std@@@std@@IEAA?AV?$_Tree_iterator@V?$_Tree_val@U?$_Tree_simple_types@U?$pair@$$CBV?$basic_string@DU?$char_traits@D@std@@V?$allocator@D@2@@std@@V12@@std@@@std@@@std@@@1@V?$_Tree_const_iterator@V?$_Tree_val@U?$_Tree_simple_types@U?$pair@$$CBV?$basic_string@DU?$char_traits@D@std@@V?$allocator@D@2@@std@@V12@@std@@@std@@@std@@@1@AEAU?$pair@$$CBV?$basic_string@DU?$char_traits@D@std@@V?$allocator@D@2@@std@@V12@@1@PEAU?$_Tree_node@U?$pair@$$CBV?$basic_string@DU?$char_traits@D@std@@V?$allocator@D@2@@std@@V12@@std@@PEAX@1@@Z 00000001400745e4     iniReader.obj
 0004:000015f0       $pdata$?_Buynode0@?$_Tree_comp_alloc@V?$_Tmap_traits@V?$basic_string@DU?$char_traits@D@std@@V?$allocator@D@2@@std@@V12@U?$less@V?$basic_string@DU?$char_traits@D@std@@V?$allocator@D@2@@std@@@2@V?$allocator@U?$pair@$$CBV?$basic_string@DU?$char_traits@D@std@@V?$allocator@D@2@@std@@V12@@std@@@2@$0A@@std@@@std@@QEAAPEAU?$_Tree_node@U?$pair@$$CBV?$basic_string@DU?$char_traits@D@std@@V?$allocator@D@2@@std@@V12@@std@@PEAX@2@XZ 00000001400745f0     iniReader.obj
 0004:000015fc       $pdata$?_Destroy_if_node@?$_Tree@V?$_Tmap_traits@V?$basic_string@DU?$char_traits@D@std@@V?$allocator@D@2@@std@@V12@U?$less@V?$basic_string@DU?$char_traits@D@std@@V?$allocator@D@2@@std@@@2@V?$allocator@U?$pair@$$CBV?$basic_string@DU?$char_traits@D@std@@V?$allocator@D@2@@std@@V12@@std@@@2@$0A@@std@@@std@@IEAAXPEAU?$_Tree_node@U?$pair@$$CBV?$basic_string@DU?$char_traits@D@std@@V?$allocator@D@2@@std@@V12@@std@@PEAX@2@@Z 00000001400745fc     iniReader.obj
 0004:00001608       $pdata$??$_Insert_at@AEAU?$pair@$$CBV?$basic_string@DU?$char_traits@D@std@@V?$allocator@D@2@@std@@V12@@std@@PEAU?$_Tree_node@U?$pair@$$CBV?$basic_string@DU?$char_traits@D@std@@V?$allocator@D@2@@std@@V12@@std@@PEAX@2@@?$_Tree@V?$_Tmap_traits@V?$basic_string@DU?$char_traits@D@std@@V?$allocator@D@2@@std@@V12@U?$less@V?$basic_string@DU?$char_traits@D@std@@V?$allocator@D@2@@std@@@2@V?$allocator@U?$pair@$$CBV?$basic_string@DU?$char_traits@D@std@@V?$allocator@D@2@@std@@V12@@std@@@2@$0A@@std@@@std@@IEAA?AV?$_Tree_iterator@V?$_Tree_val@U?$_Tree_simple_types@U?$pair@$$CBV?$basic_string@DU?$char_traits@D@std@@V?$allocator@D@2@@std@@V12@@std@@@std@@@std@@@1@_NPEAU?$_Tree_node@U?$pair@$$CBV?$basic_string@DU?$char_traits@D@std@@V?$allocator@D@2@@std@@V12@@std@@PEAX@1@AEAU?$pair@$$CBV?$basic_string@DU?$char_traits@D@std@@V?$allocator@D@2@@std@@V12@@1@1@Z 0000000140074608     iniReader.obj
 0004:00001614       $pdata$??$_Insert_nohint@AEAU?$pair@$$CBV?$basic_string@DU?$char_traits@D@std@@V?$allocator@D@2@@std@@V12@@std@@PEAU?$_Tree_node@U?$pair@$$CBV?$basic_string@DU?$char_traits@D@std@@V?$allocator@D@2@@std@@V12@@std@@PEAX@2@@?$_Tree@V?$_Tmap_traits@V?$basic_string@DU?$char_traits@D@std@@V?$allocator@D@2@@std@@V12@U?$less@V?$basic_string@DU?$char_traits@D@std@@V?$allocator@D@2@@std@@@2@V?$allocator@U?$pair@$$CBV?$basic_string@DU?$char_traits@D@std@@V?$allocator@D@2@@std@@V12@@std@@@2@$0A@@std@@@std@@IEAA?AU?$pair@V?$_Tree_iterator@V?$_Tree_val@U?$_Tree_simple_types@U?$pair@$$CBV?$basic_string@DU?$char_traits@D@std@@V?$allocator@D@2@@std@@V12@@std@@@std@@@std@@@std@@_N@1@_NAEAU?$pair@$$CBV?$basic_string@DU?$char_traits@D@std@@V?$allocator@D@2@@std@@V12@@1@PEAU?$_Tree_node@U?$pair@$$CBV?$basic_string@DU?$char_traits@D@std@@V?$allocator@D@2@@std@@V12@@std@@PEAX@1@@Z 0000000140074614     iniReader.obj
 0004:00001620       $pdata$?auth_NTLM@mailer@jwsmtp@@AEAA_NAEBV?$basic_string@DU?$char_traits@D@std@@V?$allocator@D@2@@std@@AEB_K@Z 0000000140074620     auth.obj
 0004:0000162c       $pdata$?Send@jwsmtp@@YA_NAEAH_KPEBD1H@Z 000000014007462c     compat.obj
 0004:00001638       $pdata$?Recv@jwsmtp@@YA_NAEAH_KPEAD1H@Z 0000000140074638     compat.obj
 0004:00001644       $pdata$?initNetworking@jwsmtp@@YAXXZ 0000000140074644     compat.obj
 0004:00001650       $pdata$??0mailer@jwsmtp@@QEAA@PEBD0000G_N@Z 0000000140074650     mailer.obj
 0004:0000165c       $pdata$??1mailer@jwsmtp@@QEAA@XZ 000000014007465c     mailer.obj
 0004:00001668       $pdata$?checkRFCcompat@mailer@jwsmtp@@AEAAXXZ 0000000140074668     mailer.obj
 0004:00001674       $pdata$0$?checkRFCcompat@mailer@jwsmtp@@AEAAXXZ 0000000140074674     mailer.obj
 0004:00001680       $pdata$1$?checkRFCcompat@mailer@jwsmtp@@AEAAXXZ 0000000140074680     mailer.obj
 0004:0000168c       $pdata$?setsender@mailer@jwsmtp@@QEAA_NAEBV?$basic_string@DU?$char_traits@D@std@@V?$allocator@D@2@@std@@@Z 000000014007468c     mailer.obj
 0004:00001698       $pdata$?addrecipient@mailer@jwsmtp@@QEAA_NAEBV?$basic_string@DU?$char_traits@D@std@@V?$allocator@D@2@@std@@F@Z 0000000140074698     mailer.obj
 0004:000016a4       $pdata$??Rmailer@jwsmtp@@QEAAXXZ 00000001400746a4     mailer.obj
 0004:000016b0       $pdata$?makesmtpmessage@mailer@jwsmtp@@AEBA?AV?$vector@DV?$allocator@D@std@@@std@@XZ 00000001400746b0     mailer.obj
 0004:000016bc       $pdata$??1?$pair@V?$vector@DV?$allocator@D@std@@@std@@V?$basic_string@DU?$char_traits@D@std@@V?$allocator@D@2@@2@@std@@QEAA@XZ 00000001400746bc     mailer.obj
 0004:000016c8       $pdata$?gethostaddresses@mailer@jwsmtp@@AEAA_NAEAV?$vector@USOCKADDR_IN@jwsmtp@@V?$allocator@USOCKADDR_IN@jwsmtp@@@std@@@std@@@Z 00000001400746c8     mailer.obj
 0004:000016d4       $pdata$?parsename@mailer@jwsmtp@@AEAAXAEAHQEBEAEAV?$basic_string@DU?$char_traits@D@std@@V?$allocator@D@2@@std@@@Z 00000001400746d4     mailer.obj
 0004:000016e0       $pdata$?parseaddress@mailer@jwsmtp@@AEAA?AUAddress@12@AEBV?$basic_string@DU?$char_traits@D@std@@V?$allocator@D@2@@std@@@Z 00000001400746e0     mailer.obj
 0004:000016ec       $pdata$?authenticate@mailer@jwsmtp@@AEAA_NAEBV?$basic_string@DU?$char_traits@D@std@@V?$allocator@D@2@@std@@AEB_K@Z 00000001400746ec     mailer.obj
 0004:000016f8       $pdata$??1?$vector@U?$pair@UAddress@mailer@jwsmtp@@F@std@@V?$allocator@U?$pair@UAddress@mailer@jwsmtp@@F@std@@@2@@std@@QEAA@XZ 00000001400746f8     mailer.obj
 0004:00001704       $pdata$0$??1?$vector@U?$pair@UAddress@mailer@jwsmtp@@F@std@@V?$allocator@U?$pair@UAddress@mailer@jwsmtp@@F@std@@@2@@std@@QEAA@XZ 0000000140074704     mailer.obj
 0004:00001710       $pdata$1$??1?$vector@U?$pair@UAddress@mailer@jwsmtp@@F@std@@V?$allocator@U?$pair@UAddress@mailer@jwsmtp@@F@std@@@2@@std@@QEAA@XZ 0000000140074710     mailer.obj
 0004:0000171c       $pdata$??1?$vector@U?$pair@V?$vector@DV?$allocator@D@std@@@std@@V?$basic_string@DU?$char_traits@D@std@@V?$allocator@D@2@@2@@std@@V?$allocator@U?$pair@V?$vector@DV?$allocator@D@std@@@std@@V?$basic_string@DU?$char_traits@D@std@@V?$allocator@D@2@@2@@std@@@2@@std@@QEAA@XZ 000000014007471c     mailer.obj
 0004:00001728       $pdata$0$??1?$vector@U?$pair@V?$vector@DV?$allocator@D@std@@@std@@V?$basic_string@DU?$char_traits@D@std@@V?$allocator@D@2@@2@@std@@V?$allocator@U?$pair@V?$vector@DV?$allocator@D@std@@@std@@V?$basic_string@DU?$char_traits@D@std@@V?$allocator@D@2@@2@@std@@@2@@std@@QEAA@XZ 0000000140074728     mailer.obj
 0004:00001734       $pdata$1$??1?$vector@U?$pair@V?$vector@DV?$allocator@D@std@@@std@@V?$basic_string@DU?$char_traits@D@std@@V?$allocator@D@2@@2@@std@@V?$allocator@U?$pair@V?$vector@DV?$allocator@D@std@@@std@@V?$basic_string@DU?$char_traits@D@std@@V?$allocator@D@2@@2@@std@@@2@@std@@QEAA@XZ 0000000140074734     mailer.obj
 0004:00001740       $pdata$??1?$vector@USOCKADDR_IN@jwsmtp@@V?$allocator@USOCKADDR_IN@jwsmtp@@@std@@@std@@QEAA@XZ 0000000140074740     mailer.obj
 0004:00001740       $pdata$?_Tidy@?$vector@USOCKADDR_IN@jwsmtp@@V?$allocator@USOCKADDR_IN@jwsmtp@@@std@@@std@@AEAAXXZ 0000000140074740     mailer.obj
 0004:0000174c       $pdata$??1?$vector@DV?$allocator@D@std@@@std@@QEAA@XZ 000000014007474c     mailer.obj
 0004:0000174c       $pdata$?_Tidy@?$vector@DV?$allocator@D@std@@@std@@AEAAXXZ 000000014007474c     mailer.obj
 0004:00001758       $pdata$??$?HDU?$char_traits@D@std@@V?$allocator@D@1@@std@@YA?AV?$basic_string@DU?$char_traits@D@std@@V?$allocator@D@2@@0@$$QEAV10@0@Z 0000000140074758     mailer.obj
 0004:00001764       $pdata$1$??$?HDU?$char_traits@D@std@@V?$allocator@D@1@@std@@YA?AV?$basic_string@DU?$char_traits@D@std@@V?$allocator@D@2@@0@$$QEAV10@0@Z 0000000140074764     mailer.obj
 0004:00001770       $pdata$2$??$?HDU?$char_traits@D@std@@V?$allocator@D@1@@std@@YA?AV?$basic_string@DU?$char_traits@D@std@@V?$allocator@D@2@@0@$$QEAV10@0@Z 0000000140074770     mailer.obj
 0004:0000177c       $pdata$??$?9DU?$char_traits@D@std@@V?$allocator@D@1@@std@@YA_NAEBV?$basic_string@DU?$char_traits@D@std@@V?$allocator@D@2@@0@0@Z 000000014007477c     mailer.obj
 0004:00001788       $pdata$??$?9DU?$char_traits@D@std@@V?$allocator@D@1@@std@@YA_NAEBV?$basic_string@DU?$char_traits@D@std@@V?$allocator@D@2@@0@QEBD@Z 0000000140074788     mailer.obj
 0004:00001794       $pdata$??$insert@V?$_Vector_const_iterator@V?$_Vector_val@U?$_Simple_types@D@std@@@std@@@std@@X@?$vector@DV?$allocator@D@std@@@std@@QEAA?AV?$_Vector_iterator@V?$_Vector_val@U?$_Simple_types@D@std@@@std@@@1@V?$_Vector_const_iterator@V?$_Vector_val@U?$_Simple_types@D@std@@@std@@@1@00@Z 0000000140074794     mailer.obj
 0004:00001794       $pdata$??$insert@V?$_String_iterator@V?$_String_val@U?$_Simple_types@D@std@@@std@@@std@@X@?$vector@DV?$allocator@D@std@@@std@@QEAA?AV?$_Vector_iterator@V?$_Vector_val@U?$_Simple_types@D@std@@@std@@@1@V?$_Vector_const_iterator@V?$_Vector_val@U?$_Simple_types@D@std@@@std@@@1@V?$_String_iterator@V?$_String_val@U?$_Simple_types@D@std@@@std@@@1@1@Z 0000000140074794     mailer.obj
 0004:000017a0       $pdata$??$_Emplace_reallocate@AEBV?$basic_string@DU?$char_traits@D@std@@V?$allocator@D@2@@std@@@?$vector@V?$basic_string@DU?$char_traits@D@std@@V?$allocator@D@2@@std@@V?$allocator@V?$basic_string@DU?$char_traits@D@std@@V?$allocator@D@2@@std@@@2@@std@@QEAAPEAV?$basic_string@DU?$char_traits@D@std@@V?$allocator@D@2@@1@QEAV21@AEBV21@@Z 00000001400747a0     mailer.obj
 0004:000017ac       $pdata$??$_Emplace_reallocate@U?$pair@UAddress@mailer@jwsmtp@@F@std@@@?$vector@U?$pair@UAddress@mailer@jwsmtp@@F@std@@V?$allocator@U?$pair@UAddress@mailer@jwsmtp@@F@std@@@2@@std@@QEAAPEAU?$pair@UAddress@mailer@jwsmtp@@F@1@QEAU21@$$QEAU21@@Z 00000001400747ac     mailer.obj
 0004:000017b8       $pdata$3$??$_Emplace_reallocate@U?$pair@UAddress@mailer@jwsmtp@@F@std@@@?$vector@U?$pair@UAddress@mailer@jwsmtp@@F@std@@V?$allocator@U?$pair@UAddress@mailer@jwsmtp@@F@std@@@2@@std@@QEAAPEAU?$pair@UAddress@mailer@jwsmtp@@F@1@QEAU21@$$QEAU21@@Z 00000001400747b8     mailer.obj
 0004:000017c4       $pdata$5$??$_Emplace_reallocate@U?$pair@UAddress@mailer@jwsmtp@@F@std@@@?$vector@U?$pair@UAddress@mailer@jwsmtp@@F@std@@V?$allocator@U?$pair@UAddress@mailer@jwsmtp@@F@std@@@2@@std@@QEAAPEAU?$pair@UAddress@mailer@jwsmtp@@F@1@QEAU21@$$QEAU21@@Z 00000001400747c4     mailer.obj
 0004:000017d0       $pdata$6$??$_Emplace_reallocate@U?$pair@UAddress@mailer@jwsmtp@@F@std@@@?$vector@U?$pair@UAddress@mailer@jwsmtp@@F@std@@V?$allocator@U?$pair@UAddress@mailer@jwsmtp@@F@std@@@2@@std@@QEAAPEAU?$pair@UAddress@mailer@jwsmtp@@F@1@QEAU21@$$QEAU21@@Z 00000001400747d0     mailer.obj
 0004:000017dc       $pdata$??$_Emplace_reallocate@AEBUSOCKADDR_IN@jwsmtp@@@?$vector@USOCKADDR_IN@jwsmtp@@V?$allocator@USOCKADDR_IN@jwsmtp@@@std@@@std@@QEAAPEAUSOCKADDR_IN@jwsmtp@@QEAU23@AEBU23@@Z 00000001400747dc     mailer.obj
 0004:000017e8       $pdata$2$??$_Emplace_reallocate@AEBUSOCKADDR_IN@jwsmtp@@@?$vector@USOCKADDR_IN@jwsmtp@@V?$allocator@USOCKADDR_IN@jwsmtp@@@std@@@std@@QEAAPEAUSOCKADDR_IN@jwsmtp@@QEAU23@AEBU23@@Z 00000001400747e8     mailer.obj
 0004:000017f4       $pdata$4$??$_Emplace_reallocate@AEBUSOCKADDR_IN@jwsmtp@@@?$vector@USOCKADDR_IN@jwsmtp@@V?$allocator@USOCKADDR_IN@jwsmtp@@@std@@@std@@QEAAPEAUSOCKADDR_IN@jwsmtp@@QEAU23@AEBU23@@Z 00000001400747f4     mailer.obj
 0004:00001800       $pdata$5$??$_Emplace_reallocate@AEBUSOCKADDR_IN@jwsmtp@@@?$vector@USOCKADDR_IN@jwsmtp@@V?$allocator@USOCKADDR_IN@jwsmtp@@@std@@@std@@QEAAPEAUSOCKADDR_IN@jwsmtp@@QEAU23@AEBU23@@Z 0000000140074800     mailer.obj
 0004:0000180c       $pdata$??$_Emplace_reallocate@D@?$vector@DV?$allocator@D@std@@@std@@QEAAPEADQEAD$$QEAD@Z 000000014007480c     mailer.obj
 0004:0000180c       $pdata$??$_Emplace_reallocate@AEBD@?$vector@DV?$allocator@D@std@@@std@@QEAAPEADQEADAEBD@Z 000000014007480c     mailer.obj
 0004:00001818       $pdata$1$??$_Emplace_reallocate@AEBD@?$vector@DV?$allocator@D@std@@@std@@QEAAPEADQEADAEBD@Z 0000000140074818     mailer.obj
 0004:00001818       $pdata$1$??$_Emplace_reallocate@D@?$vector@DV?$allocator@D@std@@@std@@QEAAPEADQEAD$$QEAD@Z 0000000140074818     mailer.obj
 0004:00001824       $pdata$2$??$_Emplace_reallocate@D@?$vector@DV?$allocator@D@std@@@std@@QEAAPEADQEAD$$QEAD@Z 0000000140074824     mailer.obj
 0004:00001824       $pdata$2$??$_Emplace_reallocate@AEBD@?$vector@DV?$allocator@D@std@@@std@@QEAAPEADQEADAEBD@Z 0000000140074824     mailer.obj
 0004:00001830       $pdata$?_Change_array@?$vector@DV?$allocator@D@std@@@std@@AEAAXQEAD_K1@Z 0000000140074830     mailer.obj
 0004:0000183c       $pdata$?_Equal@?$basic_string@DU?$char_traits@D@std@@V?$allocator@D@2@@std@@QEBA_NQEBD@Z 000000014007483c     mailer.obj
 0004:00001848       $pdata$??$_Insert_range@PEBD@?$vector@DV?$allocator@D@std@@@std@@AEAAXV?$_Vector_const_iterator@V?$_Vector_val@U?$_Simple_types@D@std@@@std@@@1@PEBD1Uforward_iterator_tag@1@@Z 0000000140074848     mailer.obj
 0004:00001848       $pdata$??$_Insert_range@PEAD@?$vector@DV?$allocator@D@std@@@std@@AEAAXV?$_Vector_const_iterator@V?$_Vector_val@U?$_Simple_types@D@std@@@std@@@1@PEAD1Uforward_iterator_tag@1@@Z 0000000140074848     mailer.obj
 0004:00001854       $pdata$1$??$_Insert_range@PEAD@?$vector@DV?$allocator@D@std@@@std@@AEAAXV?$_Vector_const_iterator@V?$_Vector_val@U?$_Simple_types@D@std@@@std@@@1@PEAD1Uforward_iterator_tag@1@@Z 0000000140074854     mailer.obj
 0004:00001854       $pdata$1$??$_Insert_range@PEBD@?$vector@DV?$allocator@D@std@@@std@@AEAAXV?$_Vector_const_iterator@V?$_Vector_val@U?$_Simple_types@D@std@@@std@@@1@PEBD1Uforward_iterator_tag@1@@Z 0000000140074854     mailer.obj
 0004:00001860       $pdata$2$??$_Insert_range@PEAD@?$vector@DV?$allocator@D@std@@@std@@AEAAXV?$_Vector_const_iterator@V?$_Vector_val@U?$_Simple_types@D@std@@@std@@@1@PEAD1Uforward_iterator_tag@1@@Z 0000000140074860     mailer.obj
 0004:00001860       $pdata$2$??$_Insert_range@PEBD@?$vector@DV?$allocator@D@std@@@std@@AEAAXV?$_Vector_const_iterator@V?$_Vector_val@U?$_Simple_types@D@std@@@std@@@1@PEBD1Uforward_iterator_tag@1@@Z 0000000140074860     mailer.obj
 0004:0000186c       $pdata$3$??$_Insert_range@PEBD@?$vector@DV?$allocator@D@std@@@std@@AEAAXV?$_Vector_const_iterator@V?$_Vector_val@U?$_Simple_types@D@std@@@std@@@1@PEBD1Uforward_iterator_tag@1@@Z 000000014007486c     mailer.obj
 0004:0000186c       $pdata$3$??$_Insert_range@PEAD@?$vector@DV?$allocator@D@std@@@std@@AEAAXV?$_Vector_const_iterator@V?$_Vector_val@U?$_Simple_types@D@std@@@std@@@1@PEAD1Uforward_iterator_tag@1@@Z 000000014007486c     mailer.obj
 0004:00001878       $pdata$??$_Reallocate_grow_by@V<lambda_f3a66ab6a0570788f31503db83886f49>@@_KPEBD_K@?$basic_string@DU?$char_traits@D@std@@V?$allocator@D@2@@std@@QEAAAEAV01@_KV<lambda_f3a66ab6a0570788f31503db83886f49>@@_KPEBD2@Z 0000000140074878     mailer.obj
 0004:00001884       $pdata$2$??$_Reallocate_grow_by@V<lambda_f3a66ab6a0570788f31503db83886f49>@@_KPEBD_K@?$basic_string@DU?$char_traits@D@std@@V?$allocator@D@2@@std@@QEAAAEAV01@_KV<lambda_f3a66ab6a0570788f31503db83886f49>@@_KPEBD2@Z 0000000140074884     mailer.obj
 0004:00001890       $pdata$3$??$_Reallocate_grow_by@V<lambda_f3a66ab6a0570788f31503db83886f49>@@_KPEBD_K@?$basic_string@DU?$char_traits@D@std@@V?$allocator@D@2@@std@@QEAAAEAV01@_KV<lambda_f3a66ab6a0570788f31503db83886f49>@@_KPEBD2@Z 0000000140074890     mailer.obj
 0004:0000189c       $pdata$des_key_schedule    000000014007489c     des.obj
 0004:000018a8       $pdata$gl_des_ecb_crypt    00000001400748a8     des.obj
 0004:000018b4       $pdata$md4_finish_ctx      00000001400748b4     md4.obj
 0004:000018c0       $pdata$md4_process_bytes   00000001400748c0     md4.obj
 0004:000018cc       $pdata$0$md4_process_bytes 00000001400748cc     md4.obj
 0004:000018d8       $pdata$1$md4_process_bytes 00000001400748d8     md4.obj
 0004:000018e4       $pdata$2$md4_process_bytes 00000001400748e4     md4.obj
 0004:000018f0       $pdata$3$md4_process_bytes 00000001400748f0     md4.obj
 0004:000018fc       $pdata$md4_process_block   00000001400748fc     md4.obj
 0004:00001908       $pdata$7$md4_process_block 0000000140074908     md4.obj
 0004:00001914       $pdata$8$md4_process_block 0000000140074914     md4.obj
 0004:00001920       $pdata$ntlm_convert_key    0000000140074920     ntlmencrypt.obj
 0004:0000192c       $pdata$buildSmbNtlmAuthResponse 000000014007492c     smbutil.obj
 0004:00001938       $pdata$0$buildSmbNtlmAuthResponse 0000000140074938     smbutil.obj
 0004:00001944       $pdata$1$buildSmbNtlmAuthResponse 0000000140074944     smbutil.obj
 0004:00001950       $pdata$2$buildSmbNtlmAuthResponse 0000000140074950     smbutil.obj
 0004:0000195c       $pdata$3$buildSmbNtlmAuthResponse 000000014007495c     smbutil.obj
 0004:00001968       $pdata$4$buildSmbNtlmAuthResponse 0000000140074968     smbutil.obj
 0004:00001974       $pdata$?getHashFromFile@md5wrapper@@QEAA?AV?$basic_string@DU?$char_traits@D@std@@V?$allocator@D@2@@std@@V23@@Z 0000000140074974     md5wrapper.obj
 0004:00001980       $pdata$?_InitPathNameInfo@CHLogger@@CAXPEBD000@Z 0000000140074980     HostLogger.obj
 0004:0000198c       $pdata$?Log@CHLogger@@SAXW4ELOG_LEVEL@1@PEBDZZ 000000014007498c     HostLogger.obj
 0004:00001998       $pdata$?LogTimeOut@CHLogger@@SAXPEBDZZ 0000000140074998     HostLogger.obj
 0004:000019a4       $pdata$0$?LogTimeOut@CHLogger@@SAXPEBDZZ 00000001400749a4     HostLogger.obj
 0004:000019b0       $pdata$3$?LogTimeOut@CHLogger@@SAXPEBDZZ 00000001400749b0     HostLogger.obj
 0004:000019bc       $pdata$4$?LogTimeOut@CHLogger@@SAXPEBDZZ 00000001400749bc     HostLogger.obj
 0004:000019c8       $pdata$5$?LogTimeOut@CHLogger@@SAXPEBDZZ 00000001400749c8     HostLogger.obj
 0004:000019d4       $pdata$?LogPacket@CHLogger@@SAXPEBDZZ 00000001400749d4     HostLogger.obj
 0004:000019e0       $pdata$?LogModeUserCount@CHLogger@@SAXPEBDZZ 00000001400749e0     HostLogger.obj
 0004:000019ec       $pdata$0$?LogModeUserCount@CHLogger@@SAXPEBDZZ 00000001400749ec     HostLogger.obj
 0004:000019f8       $pdata$1$?LogModeUserCount@CHLogger@@SAXPEBDZZ 00000001400749f8     HostLogger.obj
 0004:00001a04       $pdata$2$?LogModeUserCount@CHLogger@@SAXPEBDZZ 0000000140074a04     HostLogger.obj
 0004:00001a10       $pdata$3$?LogModeUserCount@CHLogger@@SAXPEBDZZ 0000000140074a10     HostLogger.obj
 0004:00001a1c       $pdata$?LogServerAppUseCount@CHLogger@@SAXPEBDZZ 0000000140074a1c     HostLogger.obj
 0004:00001a28       $pdata$0$?LogServerAppUseCount@CHLogger@@SAXPEBDZZ 0000000140074a28     HostLogger.obj
 0004:00001a34       $pdata$1$?LogServerAppUseCount@CHLogger@@SAXPEBDZZ 0000000140074a34     HostLogger.obj
 0004:00001a40       $pdata$?LogRWProcessMemory@CHLogger@@SAXPEBDZZ 0000000140074a40     HostLogger.obj
 0004:00001a4c       $pdata$0$?LogRWProcessMemory@CHLogger@@SAXPEBDZZ 0000000140074a4c     HostLogger.obj
 0004:00001a58       $pdata$1$?LogRWProcessMemory@CHLogger@@SAXPEBDZZ 0000000140074a58     HostLogger.obj
 0004:00001a64       $pdata$2$?LogRWProcessMemory@CHLogger@@SAXPEBDZZ 0000000140074a64     HostLogger.obj
 0004:00001a70       $pdata$3$?LogRWProcessMemory@CHLogger@@SAXPEBDZZ 0000000140074a70     HostLogger.obj
 0004:00001a7c       $pdata$?LogIPCMessage@CHLogger@@SAXPEBDZZ 0000000140074a7c     HostLogger.obj
 0004:00001a88       $pdata$0$?LogIPCMessage@CHLogger@@SAXPEBDZZ 0000000140074a88     HostLogger.obj
 0004:00001a94       $pdata$1$?LogIPCMessage@CHLogger@@SAXPEBDZZ 0000000140074a94     HostLogger.obj
 0004:00001aa0       $pdata$2$?LogIPCMessage@CHLogger@@SAXPEBDZZ 0000000140074aa0     HostLogger.obj
 0004:00001aac       $pdata$3$?LogIPCMessage@CHLogger@@SAXPEBDZZ 0000000140074aac     HostLogger.obj
 0004:00001ab8       $pdata$?_BuildDirectory@CHLogger@@CAXAEBU_SYSTEMTIME@@@Z 0000000140074ab8     HostLogger.obj
 0004:00001ac4       $pdata$?_DoLogWithLevel@CHLogger@@CAXPEBDW4ELOG_LEVEL@1@0PEAD@Z 0000000140074ac4     HostLogger.obj
 0004:00001ad0       $pdata$??_GCMustSyncObjectLog@@UEAAPEAXI@Z 0000000140074ad0     HostLogger.obj
 0004:00001adc       $pdata$?Init@CLogMsgManager@@SA_NW4ESHARED_MEM_USAGE_TYPE@1@@Z 0000000140074adc     LogMsgManager.obj
 0004:00001ae8       $pdata$?GetString@CLogMsgManager@@SA?BV?$basic_string@DU?$char_traits@D@std@@V?$allocator@D@2@@std@@I@Z 0000000140074ae8     LogMsgManager.obj
 0004:00001af4       $pdata$0$?GetString@CLogMsgManager@@SA?BV?$basic_string@DU?$char_traits@D@std@@V?$allocator@D@2@@std@@I@Z 0000000140074af4     LogMsgManager.obj
 0004:00001b00       $pdata$1$?GetString@CLogMsgManager@@SA?BV?$basic_string@DU?$char_traits@D@std@@V?$allocator@D@2@@std@@I@Z 0000000140074b00     LogMsgManager.obj
 0004:00001b0c       $pdata$2$?GetString@CLogMsgManager@@SA?BV?$basic_string@DU?$char_traits@D@std@@V?$allocator@D@2@@std@@I@Z 0000000140074b0c     LogMsgManager.obj
 0004:00001b18       $pdata$3$?GetString@CLogMsgManager@@SA?BV?$basic_string@DU?$char_traits@D@std@@V?$allocator@D@2@@std@@I@Z 0000000140074b18     LogMsgManager.obj
 0004:00001b24       $pdata$?_WriteXlsDataToSharedMemory@CLogMsgManager@@CA_NXZ 0000000140074b24     LogMsgManager.obj
 0004:00001b30       $pdata$??$sprintf_s@$0CA@@cf@@YAHAEAY0CA@DPEBDZZ 0000000140074b30     LogMsgManager.obj
 0004:00001b3c       $pdata$??$_Emplace_reallocate@AEBQEAX@?$vector@PEAXV?$allocator@PEAX@std@@@std@@QEAAPEAPEAXQEAPEAXAEBQEAX@Z 0000000140074b3c     LogMsgManager.obj
 0004:00001b48       $pdata$2$??$_Emplace_reallocate@AEBQEAX@?$vector@PEAXV?$allocator@PEAX@std@@@std@@QEAAPEAPEAXQEAPEAXAEBQEAX@Z 0000000140074b48     LogMsgManager.obj
 0004:00001b54       $pdata$4$??$_Emplace_reallocate@AEBQEAX@?$vector@PEAXV?$allocator@PEAX@std@@@std@@QEAAPEAPEAXQEAPEAXAEBQEAX@Z 0000000140074b54     LogMsgManager.obj
 0004:00001b60       $pdata$5$??$_Emplace_reallocate@AEBQEAX@?$vector@PEAXV?$allocator@PEAX@std@@@std@@QEAAPEAPEAXQEAPEAXAEBQEAX@Z 0000000140074b60     LogMsgManager.obj
 0004:00001b6c       $pdata$??0FindXlsMsg@@QEAA@XZ 0000000140074b6c     LoadXlsMsg.obj
 0004:00001b78       $pdata$??_GFindXlsMsg@@UEAAPEAXI@Z 0000000140074b78     LoadXlsMsg.obj
 0004:00001b84       $pdata$?LoadWMszFile@FindXlsMsg@@QEAA_NPEAD@Z 0000000140074b84     LoadXlsMsg.obj
 0004:00001b90       $pdata$??A?$map@_JV?$basic_string@DU?$char_traits@D@std@@V?$allocator@D@2@@std@@U?$less@_J@2@V?$allocator@U?$pair@$$CB_JV?$basic_string@DU?$char_traits@D@std@@V?$allocator@D@2@@std@@@std@@@2@@std@@QEAAAEAV?$basic_string@DU?$char_traits@D@std@@V?$allocator@D@2@@1@AEB_J@Z 0000000140074b90     LoadXlsMsg.obj
 0004:00001b9c       $pdata$?_Erase@?$_Tree@V?$_Tmap_traits@_JV?$basic_string@DU?$char_traits@D@std@@V?$allocator@D@2@@std@@U?$less@_J@2@V?$allocator@U?$pair@$$CB_JV?$basic_string@DU?$char_traits@D@std@@V?$allocator@D@2@@std@@@std@@@2@$0A@@std@@@std@@IEAAXPEAU?$_Tree_node@U?$pair@$$CB_JV?$basic_string@DU?$char_traits@D@std@@V?$allocator@D@2@@std@@@std@@PEAX@2@@Z 0000000140074b9c     LoadXlsMsg.obj
 0004:00001ba8       $pdata$0$?_Erase@?$_Tree@V?$_Tmap_traits@_JV?$basic_string@DU?$char_traits@D@std@@V?$allocator@D@2@@std@@U?$less@_J@2@V?$allocator@U?$pair@$$CB_JV?$basic_string@DU?$char_traits@D@std@@V?$allocator@D@2@@std@@@std@@@2@$0A@@std@@@std@@IEAAXPEAU?$_Tree_node@U?$pair@$$CB_JV?$basic_string@DU?$char_traits@D@std@@V?$allocator@D@2@@std@@@std@@PEAX@2@@Z 0000000140074ba8     LoadXlsMsg.obj
 0004:00001bb4       $pdata$1$?_Erase@?$_Tree@V?$_Tmap_traits@_JV?$basic_string@DU?$char_traits@D@std@@V?$allocator@D@2@@std@@U?$less@_J@2@V?$allocator@U?$pair@$$CB_JV?$basic_string@DU?$char_traits@D@std@@V?$allocator@D@2@@std@@@std@@@2@$0A@@std@@@std@@IEAAXPEAU?$_Tree_node@U?$pair@$$CB_JV?$basic_string@DU?$char_traits@D@std@@V?$allocator@D@2@@std@@@std@@PEAX@2@@Z 0000000140074bb4     LoadXlsMsg.obj
 0004:00001bc0       $pdata$2$?_Erase@?$_Tree@V?$_Tmap_traits@_JV?$basic_string@DU?$char_traits@D@std@@V?$allocator@D@2@@std@@U?$less@_J@2@V?$allocator@U?$pair@$$CB_JV?$basic_string@DU?$char_traits@D@std@@V?$allocator@D@2@@std@@@std@@@2@$0A@@std@@@std@@IEAAXPEAU?$_Tree_node@U?$pair@$$CB_JV?$basic_string@DU?$char_traits@D@std@@V?$allocator@D@2@@std@@@std@@PEAX@2@@Z 0000000140074bc0     LoadXlsMsg.obj
 0004:00001bcc       $pdata$?erase@?$_Tree@V?$_Tmap_traits@_JV?$basic_string@DU?$char_traits@D@std@@V?$allocator@D@2@@std@@U?$less@_J@2@V?$allocator@U?$pair@$$CB_JV?$basic_string@DU?$char_traits@D@std@@V?$allocator@D@2@@std@@@std@@@2@$0A@@std@@@std@@QEAA?AV?$_Tree_iterator@V?$_Tree_val@U?$_Tree_simple_types@U?$pair@$$CB_JV?$basic_string@DU?$char_traits@D@std@@V?$allocator@D@2@@std@@@std@@@std@@@std@@@2@V?$_Tree_const_iterator@V?$_Tree_val@U?$_Tree_simple_types@U?$pair@$$CB_JV?$basic_string@DU?$char_traits@D@std@@V?$allocator@D@2@@std@@@std@@@std@@@std@@@2@0@Z 0000000140074bcc     LoadXlsMsg.obj
 0004:00001bd8       $pdata$??$_Buynode@AEBUpiecewise_construct_t@std@@V?$tuple@AEB_J@2@V?$tuple@$$V@2@@?$_Tree_comp_alloc@V?$_Tmap_traits@_JV?$basic_string@DU?$char_traits@D@std@@V?$allocator@D@2@@std@@U?$less@_J@2@V?$allocator@U?$pair@$$CB_JV?$basic_string@DU?$char_traits@D@std@@V?$allocator@D@2@@std@@@std@@@2@$0A@@std@@@std@@QEAAPEAU?$_Tree_node@U?$pair@$$CB_JV?$basic_string@DU?$char_traits@D@std@@V?$allocator@D@2@@std@@@std@@PEAX@1@AEBUpiecewise_construct_t@1@$$QEAV?$tuple@AEB_J@1@$$QEAV?$tuple@$$V@1@@Z 0000000140074bd8     LoadXlsMsg.obj
 0004:00001be4       $pdata$??$_Insert_hint@AEAU?$pair@$$CB_JV?$basic_string@DU?$char_traits@D@std@@V?$allocator@D@2@@std@@@std@@PEAU?$_Tree_node@U?$pair@$$CB_JV?$basic_string@DU?$char_traits@D@std@@V?$allocator@D@2@@std@@@std@@PEAX@2@@?$_Tree@V?$_Tmap_traits@_JV?$basic_string@DU?$char_traits@D@std@@V?$allocator@D@2@@std@@U?$less@_J@2@V?$allocator@U?$pair@$$CB_JV?$basic_string@DU?$char_traits@D@std@@V?$allocator@D@2@@std@@@std@@@2@$0A@@std@@@std@@IEAA?AV?$_Tree_iterator@V?$_Tree_val@U?$_Tree_simple_types@U?$pair@$$CB_JV?$basic_string@DU?$char_traits@D@std@@V?$allocator@D@2@@std@@@std@@@std@@@std@@@1@V?$_Tree_const_iterator@V?$_Tree_val@U?$_Tree_simple_types@U?$pair@$$CB_JV?$basic_string@DU?$char_traits@D@std@@V?$allocator@D@2@@std@@@std@@@std@@@std@@@1@AEAU?$pair@$$CB_JV?$basic_string@DU?$char_traits@D@std@@V?$allocator@D@2@@std@@@1@PEAU?$_Tree_node@U?$pair@$$CB_JV?$basic_string@DU?$char_traits@D@std@@V?$allocator@D@2@@std@@@std@@PEAX@1@@Z 0000000140074be4     LoadXlsMsg.obj
 0004:00001bf0       $pdata$?_Destroy_if_node@?$_Tree@V?$_Tmap_traits@_JV?$basic_string@DU?$char_traits@D@std@@V?$allocator@D@2@@std@@U?$less@_J@2@V?$allocator@U?$pair@$$CB_JV?$basic_string@DU?$char_traits@D@std@@V?$allocator@D@2@@std@@@std@@@2@$0A@@std@@@std@@IEAAXPEAU?$_Tree_node@U?$pair@$$CB_JV?$basic_string@DU?$char_traits@D@std@@V?$allocator@D@2@@std@@@std@@PEAX@2@@Z 0000000140074bf0     LoadXlsMsg.obj
 0004:00001bfc       $pdata$??$_Insert_at@AEAU?$pair@$$CB_JV?$basic_string@DU?$char_traits@D@std@@V?$allocator@D@2@@std@@@std@@PEAU?$_Tree_node@U?$pair@$$CB_JV?$basic_string@DU?$char_traits@D@std@@V?$allocator@D@2@@std@@@std@@PEAX@2@@?$_Tree@V?$_Tmap_traits@_JV?$basic_string@DU?$char_traits@D@std@@V?$allocator@D@2@@std@@U?$less@_J@2@V?$allocator@U?$pair@$$CB_JV?$basic_string@DU?$char_traits@D@std@@V?$allocator@D@2@@std@@@std@@@2@$0A@@std@@@std@@IEAA?AV?$_Tree_iterator@V?$_Tree_val@U?$_Tree_simple_types@U?$pair@$$CB_JV?$basic_string@DU?$char_traits@D@std@@V?$allocator@D@2@@std@@@std@@@std@@@std@@@1@_NPEAU?$_Tree_node@U?$pair@$$CB_JV?$basic_string@DU?$char_traits@D@std@@V?$allocator@D@2@@std@@@std@@PEAX@1@AEAU?$pair@$$CB_JV?$basic_string@DU?$char_traits@D@std@@V?$allocator@D@2@@std@@@1@1@Z 0000000140074bfc     LoadXlsMsg.obj
 0004:00001c08       $pdata$??$_Insert_nohint@AEAU?$pair@$$CB_JV?$basic_string@DU?$char_traits@D@std@@V?$allocator@D@2@@std@@@std@@PEAU?$_Tree_node@U?$pair@$$CB_JV?$basic_string@DU?$char_traits@D@std@@V?$allocator@D@2@@std@@@std@@PEAX@2@@?$_Tree@V?$_Tmap_traits@_JV?$basic_string@DU?$char_traits@D@std@@V?$allocator@D@2@@std@@U?$less@_J@2@V?$allocator@U?$pair@$$CB_JV?$basic_string@DU?$char_traits@D@std@@V?$allocator@D@2@@std@@@std@@@2@$0A@@std@@@std@@IEAA?AU?$pair@V?$_Tree_iterator@V?$_Tree_val@U?$_Tree_simple_types@U?$pair@$$CB_JV?$basic_string@DU?$char_traits@D@std@@V?$allocator@D@2@@std@@@std@@@std@@@std@@@std@@_N@1@_NAEAU?$pair@$$CB_JV?$basic_string@DU?$char_traits@D@std@@V?$allocator@D@2@@std@@@1@PEAU?$_Tree_node@U?$pair@$$CB_JV?$basic_string@DU?$char_traits@D@std@@V?$allocator@D@2@@std@@@std@@PEAX@1@@Z 0000000140074c08     LoadXlsMsg.obj
 0004:00001c14       $pdata$?base64encode@jwsmtp@@YA?AV?$vector@DV?$allocator@D@std@@@std@@AEBV23@_N@Z 0000000140074c14     base6409cee8549d9fd00dfa06fdadc87a8424.obj
 0004:00001c20       $pdata$?base64encode@jwsmtp@@YA?AV?$basic_string@DU?$char_traits@D@std@@V?$allocator@D@2@@std@@AEBV23@_N@Z 0000000140074c20     base6409cee8549d9fd00dfa06fdadc87a8424.obj
 0004:00001c2c       $pdata$?base64encode@jwsmtp@@YAXPEBDHPEAD_N@Z 0000000140074c2c     base6409cee8549d9fd00dfa06fdadc87a8424.obj
 0004:00001c38       $pdata$?base64decode@jwsmtp@@YAXAEBV?$vector@DV?$allocator@D@std@@@std@@AEAV23@@Z 0000000140074c38     base6409cee8549d9fd00dfa06fdadc87a8424.obj
 0004:00001c44       $pdata$?MD5Update@MD5@@QEAAXPEAUMD5_CTX@@PEAEI@Z 0000000140074c44     md55d7732e46e8b0b019ace15d3c50ded71.obj
 0004:00001c50       $pdata$?MD5Final@MD5@@QEAAXQEAEPEAUMD5_CTX@@@Z 0000000140074c50     md55d7732e46e8b0b019ace15d3c50ded71.obj
 0004:00001c5c       $pdata$?MD5Transform@MD5@@AEAAXQEAKQEAE@Z 0000000140074c5c     md55d7732e46e8b0b019ace15d3c50ded71.obj
 0004:00001c68       $pdata$?sprintf_s@internal@cf@@YAHPEAD_KPEBDAEAPEAD@Z 0000000140074c68     safe_string_x64:safe_string.obj
 0004:00001c74       $pdata$??_D?$basic_stringstream@DU?$char_traits@D@std@@V?$allocator@D@2@@std@@QEAAXXZ 0000000140074c74     safe_string_x64:safe_string.obj
 0004:00001c80       $pdata$?strcpy_s@cf@@YAHPEAD_KPEBD@Z 0000000140074c80     safe_string_x64:safe_string.obj
 0004:00001c8c       $pdata$?strncpy_s@cf@@YAHPEAD_KPEBD1@Z 0000000140074c8c     safe_string_x64:safe_string.obj
 0004:00001c98       $pdata$?sprintf_s@cf@@YAHPEAD_KPEBDZZ 0000000140074c98     safe_string_x64:safe_string.obj
 0004:00001ca4       $pdata$??0?$basic_stringstream@DU?$char_traits@D@std@@V?$allocator@D@2@@std@@QEAA@H@Z 0000000140074ca4     safe_string_x64:safe_string.obj
 0004:00001cb0       $pdata$?seekpos@?$basic_stringbuf@DU?$char_traits@D@std@@V?$allocator@D@2@@std@@MEAA?AV?$fpos@U_Mbstatet@@@2@V32@H@Z 0000000140074cb0     safe_string_x64:safe_string.obj
 0004:00001cbc       $pdata$?seekoff@?$basic_stringbuf@DU?$char_traits@D@std@@V?$allocator@D@2@@std@@MEAA?AV?$fpos@U_Mbstatet@@@2@_JHH@Z 0000000140074cbc     safe_string_x64:safe_string.obj
 0004:00001cc8       $pdata$?overflow@?$basic_stringbuf@DU?$char_traits@D@std@@V?$allocator@D@2@@std@@MEAAHH@Z 0000000140074cc8     safe_string_x64:safe_string.obj
 0004:00001cd4       $pdata$??1?$basic_stringbuf@DU?$char_traits@D@std@@V?$allocator@D@2@@std@@UEAA@XZ 0000000140074cd4     safe_string_x64:safe_string.obj
 0004:00001ce0       $pdata$??_G?$basic_stringstream@DU?$char_traits@D@std@@V?$allocator@D@2@@std@@UEAAPEAXI@Z 0000000140074ce0     safe_string_x64:safe_string.obj
 0004:00001cec       $pdata$??_G?$basic_stringbuf@DU?$char_traits@D@std@@V?$allocator@D@2@@std@@UEAAPEAXI@Z 0000000140074cec     safe_string_x64:safe_string.obj
 0004:00001d04       $pdata$?__scrt_initialize_thread_safe_statics@@YAHXZ 0000000140074d04     msvcrt:thread_safe_statics.obj
 0004:00001d10       $pdata$?__scrt_uninitialize_thread_safe_statics@@YAXXZ 0000000140074d10     msvcrt:thread_safe_statics.obj
 0004:00001d1c       $pdata$_Init_thread_abort  0000000140074d1c     msvcrt:thread_safe_statics.obj
 0004:00001d28       $pdata$_Init_thread_footer 0000000140074d28     msvcrt:thread_safe_statics.obj
 0004:00001d34       $pdata$_Init_thread_header 0000000140074d34     msvcrt:thread_safe_statics.obj
 0004:00001d40       $pdata$_Init_thread_notify 0000000140074d40     msvcrt:thread_safe_statics.obj
 0004:00001d4c       $pdata$_Init_thread_wait   0000000140074d4c     msvcrt:thread_safe_statics.obj
 0004:00001d58       $pdata$__scrt_acquire_startup_lock 0000000140074d58     msvcrt:utility.obj
 0004:00001d64       $pdata$__scrt_initialize_crt 0000000140074d64     msvcrt:utility.obj
 0004:00001d70       $pdata$__scrt_initialize_onexit_tables 0000000140074d70     msvcrt:utility.obj
 0004:00001d7c       $pdata$__scrt_is_nonwritable_in_current_image 0000000140074d7c     msvcrt:utility.obj
 0004:00001d88       $pdata$__scrt_release_startup_lock 0000000140074d88     msvcrt:utility.obj
 0004:00001d94       $pdata$__scrt_uninitialize_crt 0000000140074d94     msvcrt:utility.obj
 0004:00001da0       $pdata$_onexit             0000000140074da0     msvcrt:utility.obj
 0004:00001dac       $pdata$atexit              0000000140074dac     msvcrt:utility.obj
 0004:00001db8       $pdata$??_Gtype_info@@UEAAPEAXI@Z 0000000140074db8     msvcrt:std_type_info_static.obj
 0004:00001dc4       $pdata$??_L@YAXPEAX_K1P6AX0@Z2@Z 0000000140074dc4     msvcrt:ehvecctr.obj
 0004:00001dd0       $pdata$??_M@YAXPEAX_K1P6AX0@Z@Z 0000000140074dd0     msvcrt:ehvecdtr.obj
 0004:00001ddc       $pdata$?__ArrayUnwind@@YAXPEAX_K1P6AX0@Z@Z 0000000140074ddc     msvcrt:ehvecdtr.obj
 0004:00001de8       $pdata$__raise_securityfailure 0000000140074de8     msvcrt:gs_report.obj
 0004:00001df4       $pdata$__report_gsfailure  0000000140074df4     msvcrt:gs_report.obj
 0004:00001e00       $pdata$__report_rangecheckfailure 0000000140074e00     msvcrt:gs_report.obj
 0004:00001e0c       $pdata$__report_securityfailure 0000000140074e0c     msvcrt:gs_report.obj
 0004:00001e18       $pdata$capture_current_context 0000000140074e18     msvcrt:gs_report.obj
 0004:00001e24       $pdata$capture_previous_context 0000000140074e24     msvcrt:gs_report.obj
 0004:00001e30       $pdata$?pre_c_initialization@@YAHXZ 0000000140074e30     msvcrt:exe_winmain.obj
 0004:00001e3c       $pdata$?post_pgo_initialization@@YAHXZ 0000000140074e3c     msvcrt:exe_winmain.obj
 0004:00001e48       $pdata$?pre_cpp_initialization@@YAXXZ 0000000140074e48     msvcrt:exe_winmain.obj
 0004:00001e54       $pdata$?__scrt_common_main_seh@@YAHXZ 0000000140074e54     msvcrt:exe_winmain.obj
 0004:00001e60       $pdata$WinMainCRTStartup   0000000140074e60     msvcrt:exe_winmain.obj
 0004:00001e6c       $pdata$__scrt_fastfail     0000000140074e6c     msvcrt:utility_desktop.obj
 0004:00001e78       $pdata$__scrt_get_show_window_mode 0000000140074e78     msvcrt:utility_desktop.obj
 0004:00001e84       $pdata$__scrt_is_managed_app 0000000140074e84     msvcrt:utility_desktop.obj
 0004:00001e90       $pdata$__scrt_unhandled_exception_filter 0000000140074e90     msvcrt:utility_desktop.obj
 0004:00001e9c       $pdata$__isa_available_init 0000000140074e9c     msvcrt:cpu_disp.obj
 0004:00001ea8       $pdata$__security_init_cookie 0000000140074ea8     msvcrt:gs_support.obj
 0004:00001eb4       $pdata$__scrt_initialize_default_local_stdio_options 0000000140074eb4     msvcrt:default_local_stdio_options.obj
 0004:00001ec0       $pdata$_RTC_Initialize     0000000140074ec0     msvcrt:initsect.obj
 0004:00001ecc       $pdata$_RTC_Terminate      0000000140074ecc     msvcrt:initsect.obj
 0004:00001ed8       $pdata$__GSHandlerCheck    0000000140074ed8     msvcrt:gshandler.obj
 0004:00001ee4       $pdata$__GSHandlerCheckCommon 0000000140074ee4     msvcrt:gshandler.obj
 0004:00001ef0       $pdata$??0CAtlBaseModule@ATL@@QEAA@XZ 0000000140074ef0     atls:atlbase.obj
 0004:00001efc       $pdata$??1CAtlBaseModule@ATL@@QEAA@XZ 0000000140074efc     atls:atlbase.obj
 0004:00001f08       $pdata$??1_Fac_tidy_reg_t@std@@QEAA@XZ 0000000140074f08     msvcprt:locale0_implib.obj
 0004:00001f14       $pdata$?AfxInitialize@@YAHHK@Z 0000000140074f14     mfcs140:appmodul.obj
 0004:00001f20       $pdata$__GSHandlerCheck_EH 0000000140074f20     msvcrt:gshandlereh.obj
 0004:00001f44       $pdata$?catch$2@?0???$_Buynode@U?$pair@_JVDivisionPacket@@@std@@@?$_Tree_comp_alloc@V?$_Tmap_traits@_JVDivisionPacket@@U?$less@_J@std@@V?$allocator@U?$pair@$$CB_JVDivisionPacket@@@std@@@3@$0A@@std@@@std@@QEAAPEAU?$_Tree_node@U?$pair@$$CB_JVDivisionPacket@@@std@@PEAX@1@$$QEAU?$pair@_JVDivisionPacket@@@1@@Z@4HA 0000000140074f44     DivisionPacketReceiver.obj
 0004:00001f50       $pdata$?catch$2@?0???$_Insert_nohint@AEAU?$pair@$$CB_JVDivisionPacket@@@std@@PEAU?$_Tree_node@U?$pair@$$CB_JVDivisionPacket@@@std@@PEAX@2@@?$_Tree@V?$_Tmap_traits@_JVDivisionPacket@@U?$less@_J@std@@V?$allocator@U?$pair@$$CB_JVDivisionPacket@@@std@@@3@$0A@@std@@@std@@IEAA?AU?$pair@V?$_Tree_iterator@V?$_Tree_val@U?$_Tree_simple_types@U?$pair@$$CB_JVDivisionPacket@@@std@@@std@@@std@@@std@@_N@1@_NAEAU?$pair@$$CB_JVDivisionPacket@@@1@PEAU?$_Tree_node@U?$pair@$$CB_JVDivisionPacket@@@std@@PEAX@1@@Z@4HA 0000000140074f50     DivisionPacketReceiver.obj
 0004:00001f5c       $pdata$?dtor$1@?0??CRSUploader@@YAAEAVUploader@crs@@XZ@4HA 0000000140074f5c     BugReporter.obj
 0004:00001f68       $pdata$?dtor$13@?0???0CGameServerManagerDlg@@QEAA@PEAVCWnd@@@Z@4HA 0000000140074f68     GameServerManagerDlg.obj
 0004:00001f74       $pdata$?dtor$5@?0??InitializeManager@CGameServerManagerDlg@@QEAAHPEADKPEAPEAD@Z@4HA 0000000140074f74     GameServerManagerDlg.obj
 0004:00001f80       $pdata$?dtor$1@?0??InitializeManager@CGameServerManagerDlg@@QEAAHPEADKPEAPEAD@Z@4HA 0000000140074f80     GameServerManagerDlg.obj
 0004:00001f8c       $pdata$?dtor$2@?0??StringSplitToNumArray@CGameServerManagerDlg@@AEAAXV?$basic_string@DU?$char_traits@D@std@@V?$allocator@D@2@@std@@0PEAHAEAH@Z@4HA 0000000140074f8c     GameServerManagerDlg.obj
 0004:00001f98       $pdata$?dtor$8@?0???0CSharedMemoryLoader@@QEAA@XZ@4HA 0000000140074f98     GameServerManagerDlg.obj
 0004:00001fa4       $pdata$?dtor$14@?0???0CSharedMemoryLoader@@QEAA@XZ@4HA 0000000140074fa4     GameServerManagerDlg.obj
 0004:00001fb0       $pdata$?dtor$1@?0??OnReceiveFromGms@CGameServerManagerDlg@@AEAAXAEBUPROTO_STARTING_GAME_tag@@@Z@4HA 0000000140074fb0     GameServerManagerDlg.obj
 0004:00001fb0       $pdata$?dtor$1@?0??OnReceiveFromGms@CGameServerManagerDlg@@AEAAXAEBUPROTO_AUTOMATCH_GAME_START_REQ@@@Z@4HA 0000000140074fb0     GameServerManagerDlg.obj
 0004:00001fbc       $pdata$?dtor$1@?0??OnReceiveFromGms@CGameServerManagerDlg@@AEAAXAEBUPROTO_AUTOMATCH_GAME_ENTER_REQ@@@Z@4HA 0000000140074fbc     GameServerManagerDlg.obj
 0004:00001fc8       $pdata$?catch$1@?0???$_Setp@UGAMESERVERINFO@@@?$shared_ptr@UGAMESERVERINFO@@@std@@AEAAXPEAUGAMESERVERINFO@@U?$integral_constant@_N$0A@@1@@Z@4HA 0000000140074fc8     GameServerManagerDlg.obj
 0004:00001fd4       $pdata$?catch$0@?0???$_Insert_nohint@AEAU?$pair@$$CBIUPORTINFO@@@std@@PEAU?$_Tree_node@U?$pair@$$CBIUPORTINFO@@@std@@PEAX@2@@?$_Tree@V?$_Tmap_traits@IUPORTINFO@@U?$less@I@std@@V?$allocator@U?$pair@$$CBIUPORTINFO@@@std@@@3@$0A@@std@@@std@@IEAA?AU?$pair@V?$_Tree_iterator@V?$_Tree_val@U?$_Tree_simple_types@U?$pair@$$CBIUPORTINFO@@@std@@@std@@@std@@@std@@_N@1@_NAEAU?$pair@$$CBIUPORTINFO@@@1@PEAU?$_Tree_node@U?$pair@$$CBIUPORTINFO@@@std@@PEAX@1@@Z@4HA 0000000140074fd4     GameServerManagerDlg.obj
 0004:00001fe0       $pdata$?catch$0@?0???$_Insert_hint@AEAU?$pair@$$CBIUPORTINFO@@@std@@PEAU?$_Tree_node@U?$pair@$$CBIUPORTINFO@@@std@@PEAX@2@@?$_Tree@V?$_Tmap_traits@IUPORTINFO@@U?$less@I@std@@V?$allocator@U?$pair@$$CBIUPORTINFO@@@std@@@3@$0A@@std@@@std@@IEAA?AV?$_Tree_iterator@V?$_Tree_val@U?$_Tree_simple_types@U?$pair@$$CBIUPORTINFO@@@std@@@std@@@std@@@1@V?$_Tree_const_iterator@V?$_Tree_val@U?$_Tree_simple_types@U?$pair@$$CBIUPORTINFO@@@std@@@std@@@std@@@1@AEAU?$pair@$$CBIUPORTINFO@@@1@PEAU?$_Tree_node@U?$pair@$$CBIUPORTINFO@@@std@@PEAX@1@@Z@4HA 0000000140074fe0     GameServerManagerDlg.obj
 0004:00001fec       $pdata$?dtor$1@?0??init@SGGMProxyLoader@sggm_proxy@@QEAA_NPEAVMultiReceiver@2@@Z@4HA 0000000140074fec     GameServerManagerDlg.obj
 0004:00001ff8       $pdata$?dtor$0@?0???$?HDU?$char_traits@D@std@@V?$allocator@D@1@@std@@YA?AV?$basic_string@DU?$char_traits@D@std@@V?$allocator@D@2@@0@QEBDAEBV10@@Z@4HA 0000000140074ff8     CSmtp.obj
 0004:00002004       $pdata$?catch$4@?0???$?6U?$char_traits@D@std@@@std@@YAAEAV?$basic_ostream@DU?$char_traits@D@std@@@0@AEAV10@PEBD@Z@4HA 0000000140075004     md5_csmtp.obj
 0004:00002010       $pdata$?catch$0@?0???$_Insert_nohint@AEAU?$pair@$$CBGUExtraStatsFPSVerify@CHostStat@@@std@@PEAU?$_Tree_node@U?$pair@$$CBGUExtraStatsFPSVerify@CHostStat@@@std@@PEAX@2@@?$_Tree@V?$_Tmap_traits@GUExtraStatsFPSVerify@CHostStat@@U?$less@G@std@@V?$allocator@U?$pair@$$CBGUExtraStatsFPSVerify@CHostStat@@@std@@@4@$0A@@std@@@std@@IEAA?AU?$pair@V?$_Tree_iterator@V?$_Tree_val@U?$_Tree_simple_types@U?$pair@$$CBGUExtraStatsFPSVerify@CHostStat@@@std@@@std@@@std@@@std@@_N@1@_NAEAU?$pair@$$CBGUExtraStatsFPSVerify@CHostStat@@@1@PEAU?$_Tree_node@U?$pair@$$CBGUExtraStatsFPSVerify@CHostStat@@@std@@PEAX@1@@Z@4HA 0000000140075010     HostStat.obj
 0004:00002010       $pdata$?catch$0@?0???$_Insert_nohint@AEAU?$pair@$$CBGUExtraStatsMemVerify@CHostStat@@@std@@PEAU?$_Tree_node@U?$pair@$$CBGUExtraStatsMemVerify@CHostStat@@@std@@PEAX@2@@?$_Tree@V?$_Tmap_traits@GUExtraStatsMemVerify@CHostStat@@U?$less@G@std@@V?$allocator@U?$pair@$$CBGUExtraStatsMemVerify@CHostStat@@@std@@@4@$0A@@std@@@std@@IEAA?AU?$pair@V?$_Tree_iterator@V?$_Tree_val@U?$_Tree_simple_types@U?$pair@$$CBGUExtraStatsMemVerify@CHostStat@@@std@@@std@@@std@@@std@@_N@1@_NAEAU?$pair@$$CBGUExtraStatsMemVerify@CHostStat@@@1@PEAU?$_Tree_node@U?$pair@$$CBGUExtraStatsMemVerify@CHostStat@@@std@@PEAX@1@@Z@4HA 0000000140075010     HostStat.obj
 0004:0000201c       $pdata$?dtor$3@?0??write@CIniSection@CIniReader@@QEAAKPEAX@Z@4HA 000000014007501c     iniReader.obj
 0004:00002028       $pdata$?dtor$3@?0??write@CIniReader@@QEAAKPEBD@Z@4HA 0000000140075028     iniReader.obj
 0004:00002034       $pdata$?dtor$1@?0??setString@CIniReader@@QEAAXPEBD00@Z@4HA 0000000140075034     iniReader.obj
 0004:00002040       $pdata$?catch$1@?0???$_Buynode@U?$pair@PEADPEAVCIniSection@CIniReader@@@std@@@?$_Tree_comp_alloc@V?$_Tmap_traits@V?$basic_string@DU?$char_traits@D@std@@V?$allocator@D@2@@std@@PEAVCIniSection@CIniReader@@U?$less@V?$basic_string@DU?$char_traits@D@std@@V?$allocator@D@2@@std@@@2@V?$allocator@U?$pair@$$CBV?$basic_string@DU?$char_traits@D@std@@V?$allocator@D@2@@std@@PEAVCIniSection@CIniReader@@@std@@@2@$0A@@std@@@std@@QEAAPEAU?$_Tree_node@U?$pair@$$CBV?$basic_string@DU?$char_traits@D@std@@V?$allocator@D@2@@std@@PEAVCIniSection@CIniReader@@@std@@PEAX@1@$$QEAU?$pair@PEADPEAVCIniSection@CIniReader@@@1@@Z@4HA 0000000140075040     iniReader.obj
 0004:0000204c       $pdata$?catch$0@?0???$_Insert_nohint@AEAU?$pair@$$CBV?$basic_string@DU?$char_traits@D@std@@V?$allocator@D@2@@std@@PEAVCIniSection@CIniReader@@@std@@PEAU?$_Tree_node@U?$pair@$$CBV?$basic_string@DU?$char_traits@D@std@@V?$allocator@D@2@@std@@PEAVCIniSection@CIniReader@@@std@@PEAX@2@@?$_Tree@V?$_Tmap_traits@V?$basic_string@DU?$char_traits@D@std@@V?$allocator@D@2@@std@@PEAVCIniSection@CIniReader@@U?$less@V?$basic_string@DU?$char_traits@D@std@@V?$allocator@D@2@@std@@@2@V?$allocator@U?$pair@$$CBV?$basic_string@DU?$char_traits@D@std@@V?$allocator@D@2@@std@@PEAVCIniSection@CIniReader@@@std@@@2@$0A@@std@@@std@@IEAA?AU?$pair@V?$_Tree_iterator@V?$_Tree_val@U?$_Tree_simple_types@U?$pair@$$CBV?$basic_string@DU?$char_traits@D@std@@V?$allocator@D@2@@std@@PEAVCIniSection@CIniReader@@@std@@@std@@@std@@@std@@_N@1@_NAEAU?$pair@$$CBV?$basic_string@DU?$char_traits@D@std@@V?$allocator@D@2@@std@@PEAVCIniSection@CIniReader@@@1@PEAU?$_Tree_node@U?$pair@$$CBV?$basic_string@DU?$char_traits@D@std@@V?$allocator@D@2@@std@@PEAVCIniSection@CIniReader@@@std@@PEAX@1@@Z@4HA 000000014007504c     iniReader.obj
 0004:00002058       $pdata$?catch$0@?0???$_Insert_hint@AEAU?$pair@$$CBV?$basic_string@DU?$char_traits@D@std@@V?$allocator@D@2@@std@@V12@@std@@PEAU?$_Tree_node@U?$pair@$$CBV?$basic_string@DU?$char_traits@D@std@@V?$allocator@D@2@@std@@V12@@std@@PEAX@2@@?$_Tree@V?$_Tmap_traits@V?$basic_string@DU?$char_traits@D@std@@V?$allocator@D@2@@std@@V12@U?$less@V?$basic_string@DU?$char_traits@D@std@@V?$allocator@D@2@@std@@@2@V?$allocator@U?$pair@$$CBV?$basic_string@DU?$char_traits@D@std@@V?$allocator@D@2@@std@@V12@@std@@@2@$0A@@std@@@std@@IEAA?AV?$_Tree_iterator@V?$_Tree_val@U?$_Tree_simple_types@U?$pair@$$CBV?$basic_string@DU?$char_traits@D@std@@V?$allocator@D@2@@std@@V12@@std@@@std@@@std@@@1@V?$_Tree_const_iterator@V?$_Tree_val@U?$_Tree_simple_types@U?$pair@$$CBV?$basic_string@DU?$char_traits@D@std@@V?$allocator@D@2@@std@@V12@@std@@@std@@@std@@@1@AEAU?$pair@$$CBV?$basic_string@DU?$char_traits@D@std@@V?$allocator@D@2@@std@@V12@@1@PEAU?$_Tree_node@U?$pair@$$CBV?$basic_string@DU?$char_traits@D@std@@V?$allocator@D@2@@std@@V12@@std@@PEAX@1@@Z@4HA 0000000140075058     iniReader.obj
 0004:00002064       $pdata$?catch$0@?0???$_Insert_nohint@AEAU?$pair@$$CBV?$basic_string@DU?$char_traits@D@std@@V?$allocator@D@2@@std@@V12@@std@@PEAU?$_Tree_node@U?$pair@$$CBV?$basic_string@DU?$char_traits@D@std@@V?$allocator@D@2@@std@@V12@@std@@PEAX@2@@?$_Tree@V?$_Tmap_traits@V?$basic_string@DU?$char_traits@D@std@@V?$allocator@D@2@@std@@V12@U?$less@V?$basic_string@DU?$char_traits@D@std@@V?$allocator@D@2@@std@@@2@V?$allocator@U?$pair@$$CBV?$basic_string@DU?$char_traits@D@std@@V?$allocator@D@2@@std@@V12@@std@@@2@$0A@@std@@@std@@IEAA?AU?$pair@V?$_Tree_iterator@V?$_Tree_val@U?$_Tree_simple_types@U?$pair@$$CBV?$basic_string@DU?$char_traits@D@std@@V?$allocator@D@2@@std@@V12@@std@@@std@@@std@@@std@@_N@1@_NAEAU?$pair@$$CBV?$basic_string@DU?$char_traits@D@std@@V?$allocator@D@2@@std@@V12@@1@PEAU?$_Tree_node@U?$pair@$$CBV?$basic_string@DU?$char_traits@D@std@@V?$allocator@D@2@@std@@V12@@std@@PEAX@1@@Z@4HA 0000000140075064     iniReader.obj
 0004:00002070       $pdata$?dtor$137@?0???Rmailer@jwsmtp@@QEAAXXZ@4HA 0000000140075070     mailer.obj
 0004:0000207c       $pdata$?dtor$178@?0???Rmailer@jwsmtp@@QEAAXXZ@4HA 000000014007507c     mailer.obj
 0004:00002088       $pdata$?dtor$2@?0??makesmtpmessage@mailer@jwsmtp@@AEBA?AV?$vector@DV?$allocator@D@std@@@std@@XZ@4HA 0000000140075088     mailer.obj
 0004:00002094       $pdata$?dtor$54@?0??makesmtpmessage@mailer@jwsmtp@@AEBA?AV?$vector@DV?$allocator@D@std@@@std@@XZ@4HA 0000000140075094     mailer.obj
 0004:000020a0       $pdata$?dtor$90@?0??makesmtpmessage@mailer@jwsmtp@@AEBA?AV?$vector@DV?$allocator@D@std@@@std@@XZ@4HA 00000001400750a0     mailer.obj
 0004:000020ac       $pdata$?dtor$114@?0??makesmtpmessage@mailer@jwsmtp@@AEBA?AV?$vector@DV?$allocator@D@std@@@std@@XZ@4HA 00000001400750ac     mailer.obj
 0004:000020b8       $pdata$?dtor$126@?0??makesmtpmessage@mailer@jwsmtp@@AEBA?AV?$vector@DV?$allocator@D@std@@@std@@XZ@4HA 00000001400750b8     mailer.obj
 0004:000020c4       $pdata$?dtor$138@?0??makesmtpmessage@mailer@jwsmtp@@AEBA?AV?$vector@DV?$allocator@D@std@@@std@@XZ@4HA 00000001400750c4     mailer.obj
 0004:000020d0       $pdata$?dtor$150@?0??makesmtpmessage@mailer@jwsmtp@@AEBA?AV?$vector@DV?$allocator@D@std@@@std@@XZ@4HA 00000001400750d0     mailer.obj
 0004:000020dc       $pdata$?dtor$29@?0??authenticate@mailer@jwsmtp@@AEAA_NAEBV?$basic_string@DU?$char_traits@D@std@@V?$allocator@D@2@@std@@AEB_K@Z@4HA 00000001400750dc     mailer.obj
 0004:000020e8       $pdata$?dtor$41@?0??authenticate@mailer@jwsmtp@@AEAA_NAEBV?$basic_string@DU?$char_traits@D@std@@V?$allocator@D@2@@std@@AEB_K@Z@4HA 00000001400750e8     mailer.obj
 0004:000020f4       $pdata$?catch$3@?0???$_Emplace_reallocate@AEBV?$basic_string@DU?$char_traits@D@std@@V?$allocator@D@2@@std@@@?$vector@V?$basic_string@DU?$char_traits@D@std@@V?$allocator@D@2@@std@@V?$allocator@V?$basic_string@DU?$char_traits@D@std@@V?$allocator@D@2@@std@@@2@@std@@QEAAPEAV?$basic_string@DU?$char_traits@D@std@@V?$allocator@D@2@@1@QEAV21@AEBV21@@Z@4HA 00000001400750f4     mailer.obj
 0004:00002100       $pdata$?dtor$0@?0??Init@CLogMsgManager@@SA_NW4ESHARED_MEM_USAGE_TYPE@1@@Z@4HA 0000000140075100     LogMsgManager.obj
 0004:0000210c       $pdata$?dtor$1@?0??Init@CLogMsgManager@@SA_NW4ESHARED_MEM_USAGE_TYPE@1@@Z@4HA 000000014007510c     LogMsgManager.obj
 0004:00002118       $pdata$?catch$0@?0???$_Insert_hint@AEAU?$pair@$$CB_JV?$basic_string@DU?$char_traits@D@std@@V?$allocator@D@2@@std@@@std@@PEAU?$_Tree_node@U?$pair@$$CB_JV?$basic_string@DU?$char_traits@D@std@@V?$allocator@D@2@@std@@@std@@PEAX@2@@?$_Tree@V?$_Tmap_traits@_JV?$basic_string@DU?$char_traits@D@std@@V?$allocator@D@2@@std@@U?$less@_J@2@V?$allocator@U?$pair@$$CB_JV?$basic_string@DU?$char_traits@D@std@@V?$allocator@D@2@@std@@@std@@@2@$0A@@std@@@std@@IEAA?AV?$_Tree_iterator@V?$_Tree_val@U?$_Tree_simple_types@U?$pair@$$CB_JV?$basic_string@DU?$char_traits@D@std@@V?$allocator@D@2@@std@@@std@@@std@@@std@@@1@V?$_Tree_const_iterator@V?$_Tree_val@U?$_Tree_simple_types@U?$pair@$$CB_JV?$basic_string@DU?$char_traits@D@std@@V?$allocator@D@2@@std@@@std@@@std@@@std@@@1@AEAU?$pair@$$CB_JV?$basic_string@DU?$char_traits@D@std@@V?$allocator@D@2@@std@@@1@PEAU?$_Tree_node@U?$pair@$$CB_JV?$basic_string@DU?$char_traits@D@std@@V?$allocator@D@2@@std@@@std@@PEAX@1@@Z@4HA 0000000140075118     LoadXlsMsg.obj
 0004:00002124       $pdata$?catch$0@?0???$_Insert_nohint@AEAU?$pair@$$CB_JV?$basic_string@DU?$char_traits@D@std@@V?$allocator@D@2@@std@@@std@@PEAU?$_Tree_node@U?$pair@$$CB_JV?$basic_string@DU?$char_traits@D@std@@V?$allocator@D@2@@std@@@std@@PEAX@2@@?$_Tree@V?$_Tmap_traits@_JV?$basic_string@DU?$char_traits@D@std@@V?$allocator@D@2@@std@@U?$less@_J@2@V?$allocator@U?$pair@$$CB_JV?$basic_string@DU?$char_traits@D@std@@V?$allocator@D@2@@std@@@std@@@2@$0A@@std@@@std@@IEAA?AU?$pair@V?$_Tree_iterator@V?$_Tree_val@U?$_Tree_simple_types@U?$pair@$$CB_JV?$basic_string@DU?$char_traits@D@std@@V?$allocator@D@2@@std@@@std@@@std@@@std@@@std@@_N@1@_NAEAU?$pair@$$CB_JV?$basic_string@DU?$char_traits@D@std@@V?$allocator@D@2@@std@@@1@PEAU?$_Tree_node@U?$pair@$$CB_JV?$basic_string@DU?$char_traits@D@std@@V?$allocator@D@2@@std@@@std@@PEAX@1@@Z@4HA 0000000140075124     LoadXlsMsg.obj
 0004:00002130       $pdata$?dtor$0@?0??base64encode@jwsmtp@@YA?AV?$vector@DV?$allocator@D@std@@@std@@AEBV23@_N@Z@4HA 0000000140075130     base6409cee8549d9fd00dfa06fdadc87a8424.obj
 0004:0000213c       $pdata$?dtor$3@?0??base64encode@jwsmtp@@YA?AV?$basic_string@DU?$char_traits@D@std@@V?$allocator@D@2@@std@@AEBV23@_N@Z@4HA 000000014007513c     base6409cee8549d9fd00dfa06fdadc87a8424.obj
 0004:00002148       $pdata$?dtor$4@?0??sprintf_s@internal@cf@@YAHPEAD_KPEBDAEAPEAD@Z@4HA 0000000140075148     safe_string_x64:safe_string.obj
 0004:00002154       $pdata$?dtor$4@?0??strcpy_s@cf@@YAHPEAD_KPEBD@Z@4HA 0000000140075154     safe_string_x64:safe_string.obj
 0004:00002154       $pdata$?dtor$4@?0??strncpy_s@cf@@YAHPEAD_KPEBD1@Z@4HA 0000000140075154     safe_string_x64:safe_string.obj
 0004:00002160       $pdata$?dtor$0@?0???0?$basic_stringstream@DU?$char_traits@D@std@@V?$allocator@D@2@@std@@QEAA@H@Z@4HA 0000000140075160     safe_string_x64:safe_string.obj
 0004:0000216c       $pdata$__scrt_is_nonwritable_in_current_image$filt$0 000000014007516c     msvcrt:utility.obj
 0004:00002178       $pdata$?fin$0@?0???_L@YAXPEAX_K1P6AX0@Z2@Z@4HA 0000000140075178     msvcrt:ehvecctr.obj
 0004:00002184       $pdata$?fin$0@?0???_M@YAXPEAX_K1P6AX0@Z@Z@4HA 0000000140075184     msvcrt:ehvecdtr.obj
 0004:00002190       $pdata$?filt$0@?0??__ArrayUnwind@@YAXPEAX_K1P6AX0@Z@Z@4HA 0000000140075190     msvcrt:ehvecdtr.obj
 0004:0000219c       $pdata$?filt$0@?0??__scrt_common_main_seh@@YAHXZ@4HA 000000014007519c     msvcrt:exe_winmain.obj
 0004:000021a8       $pdata$??__Fthis_instance_@?1??Instance@DivisionPacketReceiver@@SAPEAV1@XZ@YAXXZ 00000001400751a8     DivisionPacketReceiver.obj
 0004:000021b4       $pdata$??__Fbase64_chars@@YAXXZ 00000001400751b4     base64.obj
 0004:000021c0       $pdata$??__F?m_strEtcFileFormat@CHLogger@@0V?$basic_string@DU?$char_traits@D@std@@V?$allocator@D@2@@std@@A@@YAXXZ 00000001400751c0     HostLogger.obj
 0004:000021cc       $pdata$??__F?m_strKernelFileFormat@CHLogger@@0V?$basic_string@DU?$char_traits@D@std@@V?$allocator@D@2@@std@@A@@YAXXZ 00000001400751cc     HostLogger.obj
 0004:000021d8       $pdata$??__F?m_strBRFileFormat@CHLogger@@0V?$basic_string@DU?$char_traits@D@std@@V?$allocator@D@2@@std@@A@@YAXXZ 00000001400751d8     HostLogger.obj
 0004:000021e4       $pdata$??__F?m_strFileFormat@CHLogger@@0V?$basic_string@DU?$char_traits@D@std@@V?$allocator@D@2@@std@@A@@YAXXZ 00000001400751e4     HostLogger.obj
 0004:000021f0       $pdata$??__F?m_strRWProcessMemoryFileFormat@CHLogger@@0V?$basic_string@DU?$char_traits@D@std@@V?$allocator@D@2@@std@@A@@YAXXZ 00000001400751f0     HostLogger.obj
 0004:000021fc       $pdata$??__F?m_strIPCMessageFileFormat@CHLogger@@0V?$basic_string@DU?$char_traits@D@std@@V?$allocator@D@2@@std@@A@@YAXXZ 00000001400751fc     HostLogger.obj
 0004:00002208       $pdata$??__F?m_strPacketFileFormat@CHLogger@@0V?$basic_string@DU?$char_traits@D@std@@V?$allocator@D@2@@std@@A@@YAXXZ 0000000140075208     HostLogger.obj
 0004:00002214       $pdata$??__F?m_strTimeOutFileFormat@CHLogger@@0V?$basic_string@DU?$char_traits@D@std@@V?$allocator@D@2@@std@@A@@YAXXZ 0000000140075214     HostLogger.obj
 0004:00002220       $pdata$??__F?m_strHostName@CHLogger@@0V?$basic_string@DU?$char_traits@D@std@@V?$allocator@D@2@@std@@A@@YAXXZ 0000000140075220     HostLogger.obj
 0004:0000222c       $pdata$??__F?m_strServerName@CHLogger@@0V?$basic_string@DU?$char_traits@D@std@@V?$allocator@D@2@@std@@A@@YAXXZ 000000014007522c     HostLogger.obj
 0004:00002238       $pdata$??__F?m_strLogFolder@CHLogger@@0V?$basic_string@DU?$char_traits@D@std@@V?$allocator@D@2@@std@@A@@YAXXZ 0000000140075238     HostLogger.obj
 0004:00002244       $pdata$??__F?m_strModeUserCountFormat@CHLogger@@0V?$basic_string@DU?$char_traits@D@std@@V?$allocator@D@2@@std@@A@@YAXXZ 0000000140075244     HostLogger.obj
 0004:00002250       $pdata$??__F?m_strServerAppUseCountFormat@CHLogger@@0V?$basic_string@DU?$char_traits@D@std@@V?$allocator@D@2@@std@@A@@YAXXZ 0000000140075250     HostLogger.obj
 0004:0000225c       $pdata$??__F?m_vectSharedMapHandles@CLogMsgManager@@0V?$vector@PEAXV?$allocator@PEAX@std@@@std@@A@@YAXXZ 000000014007525c     LogMsgManager.obj
 0005:000001e0       $R000000                   00000001400761e0     GameServerManager.res
 0005:000004c8       $R0002E8                   00000001400764c8     GameServerManager.res
 0005:000005f0       $R000410                   00000001400765f0     GameServerManager.res
 0005:00000618       $R000438                   0000000140076618     GameServerManager.res
 0005:000006f0       $R000510                   00000001400766f0     GameServerManager.res
 0005:00000948       $R000768                   0000000140076948     GameServerManager.res
 0005:00000c38       $R000A58                   0000000140076c38     GameServerManager.res

 Exports

  ordinal    name

